
gdi32.nostrip.dll:     file format pei-i386

Disassembly of section .text:

77ed1000 <_DllMain@12>:
	HANDLE	hDll,
	DWORD	dwReason,
	LPVOID	lpReserved
	)
{
77ed1000:	55                   	push   %ebp
	return TRUE;
}
77ed1001:	b8 01 00 00 00       	mov    $0x1,%eax
77ed1006:	89 e5                	mov    %esp,%ebp
77ed1008:	5d                   	pop    %ebp
77ed1009:	c2 0c 00             	ret    $0xc
77ed100c:	8d 74 26 00          	lea    0x0(%esi),%esi

77ed1010 <_GdiProcessSetup@0>:


VOID
WINAPI
GdiProcessSetup (VOID)
{
77ed1010:	55                   	push   %ebp
77ed1011:	89 e5                	mov    %esp,%ebp
77ed1013:	50                   	push   %eax
77ed1014:	50                   	push   %eax
	hProcessHeap = GetProcessHeap();
77ed1015:	e8 d6 88 00 00       	call   77ed98f0 <_GetProcessHeap@0>
77ed101a:	a3 00 c0 ed 77       	mov    %eax,0x77edc000
static __inline__ struct _TEB * NtCurrentTeb(void)
{
    struct _TEB *ret;

    __asm__ __volatile__ (
77ed101f:	64 a1 18 00 00 00    	mov    %fs:0x18,%eax
77ed1025:	8b 40 30             	mov    0x30(%eax),%eax
77ed1028:	8b 80 94 00 00 00    	mov    0x94(%eax),%eax
77ed102e:	a3 14 c0 ed 77       	mov    %eax,0x77edc014
77ed1033:	64 a1 18 00 00 00    	mov    %fs:0x18,%eax
77ed1039:	8b 40 20             	mov    0x20(%eax),%eax
77ed103c:	a3 10 c0 ed 77       	mov    %eax,0x77edc010
77ed1041:	c9                   	leave  
77ed1042:	c3                   	ret    
77ed1043:	8d b6 00 00 00 00    	lea    0x0(%esi),%esi
77ed1049:	8d bc 27 00 00 00 00 	lea    0x0(%edi),%edi

77ed1050 <_GdiDllInitialize@12>:

        /* map the gdi handle table to user space */
	GdiHandleTable = NtCurrentTeb()->Peb->GdiSharedHandleTable;
	CurrentProcessId = NtCurrentTeb()->Cid.UniqueProcess;
}


/*
 * @implemented
 */
BOOL
WINAPI
GdiDllInitialize (
	HANDLE	hDll,
	DWORD	dwReason,
	LPVOID	lpReserved
	)
{
77ed1050:	55                   	push   %ebp
77ed1051:	89 e5                	mov    %esp,%ebp
77ed1053:	52                   	push   %edx
77ed1054:	52                   	push   %edx
77ed1055:	8b 45 0c             	mov    0xc(%ebp),%eax
	switch (dwReason)
77ed1058:	83 f8 01             	cmp    $0x1,%eax
77ed105b:	74 0b                	je     77ed1068 <_GdiDllInitialize@12+0x18>
77ed105d:	83 f8 02             	cmp    $0x2,%eax
77ed1060:	74 0b                	je     77ed106d <_GdiDllInitialize@12+0x1d>
	{
		case DLL_PROCESS_ATTACH:
			GdiProcessSetup ();
			break;

		case DLL_THREAD_ATTACH:
			break;

		default:
			return FALSE;
77ed1062:	31 c0                	xor    %eax,%eax
	}

#if 0
	/* FIXME: working teb handling needed */
	NtCurrentTeb()->GdiTebBatch.Offset = 0;
	NtCurrentTeb()->GdiBatchCount = 0;
#endif

	return TRUE;
}
77ed1064:	c9                   	leave  
77ed1065:	c2 0c 00             	ret    $0xc
77ed1068:	e8 a3 ff ff ff       	call   77ed1010 <_GdiProcessSetup@0>
77ed106d:	b8 01 00 00 00       	mov    $0x1,%eax
77ed1072:	c9                   	leave  
77ed1073:	c2 0c 00             	ret    $0xc
77ed1076:	90                   	nop    
77ed1077:	90                   	nop    
77ed1078:	90                   	nop    
77ed1079:	90                   	nop    
77ed107a:	90                   	nop    
77ed107b:	90                   	nop    
77ed107c:	90                   	nop    
77ed107d:	90                   	nop    
77ed107e:	90                   	nop    
77ed107f:	90                   	nop    

77ed1080 <_HEAP_alloc>:
77ed1080:	55                   	push   %ebp
77ed1081:	89 e5                	mov    %esp,%ebp
77ed1083:	50                   	push   %eax
77ed1084:	50                   	push   %eax
77ed1085:	a1 00 c0 ed 77       	mov    0x77edc000,%eax
77ed108a:	85 c0                	test   %eax,%eax
77ed108c:	74 14                	je     77ed10a2 <_HEAP_alloc+0x22>
77ed108e:	51                   	push   %ecx
77ed108f:	8b 55 08             	mov    0x8(%ebp),%edx
77ed1092:	52                   	push   %edx
77ed1093:	6a 00                	push   $0x0
77ed1095:	a1 00 c0 ed 77       	mov    0x77edc000,%eax
77ed109a:	50                   	push   %eax
77ed109b:	e8 50 87 00 00       	call   77ed97f0 <_RtlAllocateHeap@12>
77ed10a0:	c9                   	leave  
77ed10a1:	c3                   	ret    
77ed10a2:	68 00 a0 ed 77       	push   $0x77eda000
77ed10a7:	6a 0c                	push   $0xc
77ed10a9:	68 01 a0 ed 77       	push   $0x77eda001
77ed10ae:	68 0d a0 ed 77       	push   $0x77eda00d
77ed10b3:	e8 48 87 00 00       	call   77ed9800 <_RtlAssert@16>
77ed10b8:	51                   	push   %ecx
77ed10b9:	8b 55 08             	mov    0x8(%ebp),%edx
77ed10bc:	52                   	push   %edx
77ed10bd:	6a 00                	push   $0x0
77ed10bf:	a1 00 c0 ed 77       	mov    0x77edc000,%eax
77ed10c4:	50                   	push   %eax
77ed10c5:	e8 26 87 00 00       	call   77ed97f0 <_RtlAllocateHeap@12>
77ed10ca:	c9                   	leave  
77ed10cb:	c3                   	ret    
77ed10cc:	8d 74 26 00          	lea    0x0(%esi),%esi

77ed10d0 <_HEAP_strdupA2W>:
77ed10d0:	55                   	push   %ebp
77ed10d1:	31 d2                	xor    %edx,%edx
77ed10d3:	89 e5                	mov    %esp,%ebp
77ed10d5:	57                   	push   %edi
77ed10d6:	56                   	push   %esi
77ed10d7:	53                   	push   %ebx
77ed10d8:	83 ec 0c             	sub    $0xc,%esp
77ed10db:	8b 45 08             	mov    0x8(%ebp),%eax
77ed10de:	8b 75 0c             	mov    0xc(%ebp),%esi
77ed10e1:	85 f6                	test   %esi,%esi
77ed10e3:	c7 00 00 00 00 00    	movl   $0x0,(%eax)
77ed10e9:	74 43                	je     77ed112e <_HEAP_strdupA2W+0x5e>
77ed10eb:	83 ec 0c             	sub    $0xc,%esp
77ed10ee:	56                   	push   %esi
77ed10ef:	e8 0c 88 00 00       	call   77ed9900 <_lstrlenA@4>
77ed10f4:	89 c3                	mov    %eax,%ebx
77ed10f6:	8d 3c 00             	lea    (%eax,%eax,1),%edi
77ed10f9:	8d 47 02             	lea    0x2(%edi),%eax
77ed10fc:	50                   	push   %eax
77ed10fd:	e8 7e ff ff ff       	call   77ed1080 <_HEAP_alloc>
77ed1102:	8b 55 08             	mov    0x8(%ebp),%edx
77ed1105:	83 c4 10             	add    $0x10,%esp
77ed1108:	85 c0                	test   %eax,%eax
77ed110a:	89 02                	mov    %eax,(%edx)
77ed110c:	ba 17 00 00 c0       	mov    $0xc0000017,%edx
77ed1111:	74 1b                	je     77ed112e <_HEAP_strdupA2W+0x5e>
77ed1113:	83 ec 0c             	sub    $0xc,%esp
77ed1116:	53                   	push   %ebx
77ed1117:	56                   	push   %esi
77ed1118:	6a 00                	push   $0x0
77ed111a:	57                   	push   %edi
77ed111b:	50                   	push   %eax
77ed111c:	e8 ef 86 00 00       	call   77ed9810 <_RtlMultiByteToUnicodeN@20>
77ed1121:	8b 4d 08             	mov    0x8(%ebp),%ecx
77ed1124:	8b 11                	mov    (%ecx),%edx
77ed1126:	66 c7 04 5a 00 00    	movw   $0x0,(%edx,%ebx,2)
77ed112c:	89 c2                	mov    %eax,%edx
77ed112e:	8d 65 f4             	lea    0xfffffff4(%ebp),%esp
77ed1131:	89 d0                	mov    %edx,%eax
77ed1133:	5b                   	pop    %ebx
77ed1134:	5e                   	pop    %esi
77ed1135:	5f                   	pop    %edi
77ed1136:	5d                   	pop    %ebp
77ed1137:	c3                   	ret    
77ed1138:	90                   	nop    
77ed1139:	8d b4 26 00 00 00 00 	lea    0x0(%esi),%esi

77ed1140 <_HEAP_free>:
77ed1140:	55                   	push   %ebp
77ed1141:	89 e5                	mov    %esp,%ebp
77ed1143:	52                   	push   %edx
77ed1144:	52                   	push   %edx
77ed1145:	a1 00 c0 ed 77       	mov    0x77edc000,%eax
77ed114a:	85 c0                	test   %eax,%eax
77ed114c:	74 14                	je     77ed1162 <_HEAP_free+0x22>
77ed114e:	50                   	push   %eax
77ed114f:	8b 45 08             	mov    0x8(%ebp),%eax
77ed1152:	50                   	push   %eax
77ed1153:	6a 00                	push   $0x0
77ed1155:	a1 00 c0 ed 77       	mov    0x77edc000,%eax
77ed115a:	50                   	push   %eax
77ed115b:	e8 c0 86 00 00       	call   77ed9820 <_RtlFreeHeap@12>
77ed1160:	c9                   	leave  
77ed1161:	c3                   	ret    
77ed1162:	68 00 a0 ed 77       	push   $0x77eda000
77ed1167:	6a 28                	push   $0x28
77ed1169:	68 01 a0 ed 77       	push   $0x77eda001
77ed116e:	68 0d a0 ed 77       	push   $0x77eda00d
77ed1173:	e8 88 86 00 00       	call   77ed9800 <_RtlAssert@16>
77ed1178:	50                   	push   %eax
77ed1179:	8b 45 08             	mov    0x8(%ebp),%eax
77ed117c:	50                   	push   %eax
77ed117d:	6a 00                	push   $0x0
77ed117f:	a1 00 c0 ed 77       	mov    0x77edc000,%eax
77ed1184:	50                   	push   %eax
77ed1185:	e8 96 86 00 00       	call   77ed9820 <_RtlFreeHeap@12>
77ed118a:	c9                   	leave  
77ed118b:	c3                   	ret    
77ed118c:	90                   	nop    
77ed118d:	90                   	nop    
77ed118e:	90                   	nop    
77ed118f:	90                   	nop    

77ed1190 <_GdiQueryTable@0>:
77ed1190:	55                   	push   %ebp
77ed1191:	a1 14 c0 ed 77       	mov    0x77edc014,%eax
77ed1196:	89 e5                	mov    %esp,%ebp
77ed1198:	5d                   	pop    %ebp
77ed1199:	c3                   	ret    
77ed119a:	8d b6 00 00 00 00    	lea    0x0(%esi),%esi

77ed11a0 <_GdiIsHandleValid>:
77ed11a0:	55                   	push   %ebp
77ed11a1:	a1 14 c0 ed 77       	mov    0x77edc014,%eax
77ed11a6:	89 e5                	mov    %esp,%ebp
77ed11a8:	8b 4d 08             	mov    0x8(%ebp),%ecx
77ed11ab:	89 ca                	mov    %ecx,%edx
77ed11ad:	81 e2 ff 3f 00 00    	and    $0x3fff,%edx
77ed11b3:	c1 e2 04             	shl    $0x4,%edx
77ed11b6:	01 c2                	add    %eax,%edx
77ed11b8:	8b 02                	mov    (%edx),%eax
77ed11ba:	85 c0                	test   %eax,%eax
77ed11bc:	74 12                	je     77ed11d0 <_GdiIsHandleValid+0x30>
77ed11be:	8b 42 08             	mov    0x8(%edx),%eax
77ed11c1:	81 e1 00 00 7f 00    	and    $0x7f0000,%ecx
77ed11c7:	25 00 00 7f 00       	and    $0x7f0000,%eax
77ed11cc:	39 c8                	cmp    %ecx,%eax
77ed11ce:	74 04                	je     77ed11d4 <_GdiIsHandleValid+0x34>
77ed11d0:	31 c0                	xor    %eax,%eax
77ed11d2:	5d                   	pop    %ebp
77ed11d3:	c3                   	ret    
77ed11d4:	8b 42 04             	mov    0x4(%edx),%eax
77ed11d7:	83 e0 fe             	and    $0xfffffffe,%eax
77ed11da:	74 08                	je     77ed11e4 <_GdiIsHandleValid+0x44>
77ed11dc:	3b 05 10 c0 ed 77    	cmp    0x77edc010,%eax
77ed11e2:	75 ec                	jne    77ed11d0 <_GdiIsHandleValid+0x30>
77ed11e4:	b8 01 00 00 00       	mov    $0x1,%eax
77ed11e9:	5d                   	pop    %ebp
77ed11ea:	c3                   	ret    
77ed11eb:	90                   	nop    
77ed11ec:	8d 74 26 00          	lea    0x0(%esi),%esi

77ed11f0 <_GdiGetHandleUserData>:
77ed11f0:	55                   	push   %ebp
77ed11f1:	a1 14 c0 ed 77       	mov    0x77edc014,%eax
77ed11f6:	89 e5                	mov    %esp,%ebp
77ed11f8:	8b 4d 08             	mov    0x8(%ebp),%ecx
77ed11fb:	89 ca                	mov    %ecx,%edx
77ed11fd:	81 e2 ff 3f 00 00    	and    $0x3fff,%edx
77ed1203:	c1 e2 04             	shl    $0x4,%edx
77ed1206:	01 c2                	add    %eax,%edx
77ed1208:	8b 02                	mov    (%edx),%eax
77ed120a:	85 c0                	test   %eax,%eax
77ed120c:	74 12                	je     77ed1220 <_GdiGetHandleUserData+0x30>
77ed120e:	8b 42 08             	mov    0x8(%edx),%eax
77ed1211:	81 e1 00 00 7f 00    	and    $0x7f0000,%ecx
77ed1217:	25 00 00 7f 00       	and    $0x7f0000,%eax
77ed121c:	39 c8                	cmp    %ecx,%eax
77ed121e:	74 04                	je     77ed1224 <_GdiGetHandleUserData+0x34>
77ed1220:	31 c0                	xor    %eax,%eax
77ed1222:	5d                   	pop    %ebp
77ed1223:	c3                   	ret    
77ed1224:	8b 42 04             	mov    0x4(%edx),%eax
77ed1227:	83 e0 fe             	and    $0xfffffffe,%eax
77ed122a:	74 08                	je     77ed1234 <_GdiGetHandleUserData+0x44>
77ed122c:	3b 05 10 c0 ed 77    	cmp    0x77edc010,%eax
77ed1232:	75 ec                	jne    77ed1220 <_GdiGetHandleUserData+0x30>
77ed1234:	8b 45 0c             	mov    0xc(%ebp),%eax
77ed1237:	8b 52 0c             	mov    0xc(%edx),%edx
77ed123a:	89 10                	mov    %edx,(%eax)
77ed123c:	b8 01 00 00 00       	mov    $0x1,%eax
77ed1241:	5d                   	pop    %ebp
77ed1242:	c3                   	ret    
77ed1243:	90                   	nop    
77ed1244:	90                   	nop    
77ed1245:	90                   	nop    
77ed1246:	90                   	nop    
77ed1247:	90                   	nop    
77ed1248:	90                   	nop    
77ed1249:	90                   	nop    
77ed124a:	90                   	nop    
77ed124b:	90                   	nop    
77ed124c:	90                   	nop    
77ed124d:	90                   	nop    
77ed124e:	90                   	nop    
77ed124f:	90                   	nop    

77ed1250 <_AnimatePalette@16>:
77ed1250:	55                   	push   %ebp
77ed1251:	89 e5                	mov    %esp,%ebp
77ed1253:	83 ec 10             	sub    $0x10,%esp
77ed1256:	68 10 a0 ed 77       	push   $0x77eda010
77ed125b:	68 20 a0 ed 77       	push   $0x77eda020
77ed1260:	ff 15 e8 10 ee 77    	call   *0x77ee10e8
77ed1266:	c7 04 24 78 00 00 00 	movl   $0x78,(%esp)
77ed126d:	e8 9e 86 00 00       	call   77ed9910 <_SetLastError@4>
77ed1272:	31 c0                	xor    %eax,%eax
77ed1274:	c9                   	leave  
77ed1275:	c2 10 00             	ret    $0x10
77ed1278:	90                   	nop    
77ed1279:	8d b4 26 00 00 00 00 	lea    0x0(%esi),%esi

77ed1280 <_CancelDC@4>:
77ed1280:	55                   	push   %ebp
77ed1281:	89 e5                	mov    %esp,%ebp
77ed1283:	83 ec 10             	sub    $0x10,%esp
77ed1286:	68 55 a0 ed 77       	push   $0x77eda055
77ed128b:	68 20 a0 ed 77       	push   $0x77eda020
77ed1290:	ff 15 e8 10 ee 77    	call   *0x77ee10e8
77ed1296:	c7 04 24 78 00 00 00 	movl   $0x78,(%esp)
77ed129d:	e8 6e 86 00 00       	call   77ed9910 <_SetLastError@4>
77ed12a2:	31 c0                	xor    %eax,%eax
77ed12a4:	c9                   	leave  
77ed12a5:	c2 04 00             	ret    $0x4
77ed12a8:	90                   	nop    
77ed12a9:	8d b4 26 00 00 00 00 	lea    0x0(%esi),%esi

77ed12b0 <_Chord@36>:
77ed12b0:	55                   	push   %ebp
77ed12b1:	89 e5                	mov    %esp,%ebp
77ed12b3:	83 ec 10             	sub    $0x10,%esp
77ed12b6:	68 5e a0 ed 77       	push   $0x77eda05e
77ed12bb:	68 20 a0 ed 77       	push   $0x77eda020
77ed12c0:	ff 15 e8 10 ee 77    	call   *0x77ee10e8
77ed12c6:	c7 04 24 78 00 00 00 	movl   $0x78,(%esp)
77ed12cd:	e8 3e 86 00 00       	call   77ed9910 <_SetLastError@4>
77ed12d2:	31 c0                	xor    %eax,%eax
77ed12d4:	c9                   	leave  
77ed12d5:	c2 24 00             	ret    $0x24
77ed12d8:	90                   	nop    
77ed12d9:	8d b4 26 00 00 00 00 	lea    0x0(%esi),%esi

77ed12e0 <_CloseMetaFile@4>:

/* EOF */
77ed12e0:	55                   	push   %ebp
77ed12e1:	89 e5                	mov    %esp,%ebp
77ed12e3:	83 ec 10             	sub    $0x10,%esp
77ed12e6:	68 64 a0 ed 77       	push   $0x77eda064
77ed12eb:	68 20 a0 ed 77       	push   $0x77eda020
77ed12f0:	ff 15 e8 10 ee 77    	call   *0x77ee10e8
77ed12f6:	c7 04 24 78 00 00 00 	movl   $0x78,(%esp)
77ed12fd:	e8 0e 86 00 00       	call   77ed9910 <_SetLastError@4>
77ed1302:	31 c0                	xor    %eax,%eax
77ed1304:	c9                   	leave  
77ed1305:	c2 04 00             	ret    $0x4
77ed1308:	90                   	nop    
77ed1309:	8d b4 26 00 00 00 00 	lea    0x0(%esi),%esi

77ed1310 <_CreateDIBPatternBrush@8>:
77ed1310:	55                   	push   %ebp
77ed1311:	89 e5                	mov    %esp,%ebp
77ed1313:	83 ec 10             	sub    $0x10,%esp
77ed1316:	68 72 a0 ed 77       	push   $0x77eda072
77ed131b:	68 20 a0 ed 77       	push   $0x77eda020
77ed1320:	ff 15 e8 10 ee 77    	call   *0x77ee10e8
77ed1326:	c7 04 24 78 00 00 00 	movl   $0x78,(%esp)
77ed132d:	e8 de 85 00 00       	call   77ed9910 <_SetLastError@4>
77ed1332:	31 c0                	xor    %eax,%eax
77ed1334:	c9                   	leave  
77ed1335:	c2 08 00             	ret    $0x8
77ed1338:	90                   	nop    
77ed1339:	8d b4 26 00 00 00 00 	lea    0x0(%esi),%esi

77ed1340 <_DeleteMetaFile@4>:
77ed1340:	55                   	push   %ebp
77ed1341:	89 e5                	mov    %esp,%ebp
77ed1343:	83 ec 10             	sub    $0x10,%esp
77ed1346:	68 88 a0 ed 77       	push   $0x77eda088
77ed134b:	68 20 a0 ed 77       	push   $0x77eda020
77ed1350:	ff 15 e8 10 ee 77    	call   *0x77ee10e8
77ed1356:	c7 04 24 78 00 00 00 	movl   $0x78,(%esp)
77ed135d:	e8 ae 85 00 00       	call   77ed9910 <_SetLastError@4>
77ed1362:	31 c0                	xor    %eax,%eax
77ed1364:	c9                   	leave  
77ed1365:	c2 04 00             	ret    $0x4
77ed1368:	90                   	nop    
77ed1369:	8d b4 26 00 00 00 00 	lea    0x0(%esi),%esi

77ed1370 <_DrawEscape@16>:
77ed1370:	55                   	push   %ebp
77ed1371:	89 e5                	mov    %esp,%ebp
77ed1373:	83 ec 10             	sub    $0x10,%esp
77ed1376:	68 97 a0 ed 77       	push   $0x77eda097
77ed137b:	68 20 a0 ed 77       	push   $0x77eda020
77ed1380:	ff 15 e8 10 ee 77    	call   *0x77ee10e8
77ed1386:	c7 04 24 78 00 00 00 	movl   $0x78,(%esp)
77ed138d:	e8 7e 85 00 00       	call   77ed9910 <_SetLastError@4>
77ed1392:	31 c0                	xor    %eax,%eax
77ed1394:	c9                   	leave  
77ed1395:	c2 10 00             	ret    $0x10
77ed1398:	90                   	nop    
77ed1399:	8d b4 26 00 00 00 00 	lea    0x0(%esi),%esi

77ed13a0 <_EnumObjects@16>:
77ed13a0:	55                   	push   %ebp
77ed13a1:	89 e5                	mov    %esp,%ebp
77ed13a3:	83 ec 10             	sub    $0x10,%esp
77ed13a6:	68 a2 a0 ed 77       	push   $0x77eda0a2
77ed13ab:	68 20 a0 ed 77       	push   $0x77eda020
77ed13b0:	ff 15 e8 10 ee 77    	call   *0x77ee10e8
77ed13b6:	c7 04 24 78 00 00 00 	movl   $0x78,(%esp)
77ed13bd:	e8 4e 85 00 00       	call   77ed9910 <_SetLastError@4>
77ed13c2:	31 c0                	xor    %eax,%eax
77ed13c4:	c9                   	leave  
77ed13c5:	c2 10 00             	ret    $0x10
77ed13c8:	90                   	nop    
77ed13c9:	8d b4 26 00 00 00 00 	lea    0x0(%esi),%esi

77ed13d0 <_Escape@20>:
77ed13d0:	55                   	push   %ebp
77ed13d1:	89 e5                	mov    %esp,%ebp
77ed13d3:	c9                   	leave  
77ed13d4:	e9 81 44 00 00       	jmp    77ed585a <_NtGdiEscape@20>
77ed13d9:	8d b4 26 00 00 00 00 	lea    0x0(%esi),%esi

77ed13e0 <_ExtCreateRegion@12>:
77ed13e0:	55                   	push   %ebp
77ed13e1:	89 e5                	mov    %esp,%ebp
77ed13e3:	83 ec 10             	sub    $0x10,%esp
77ed13e6:	68 ae a0 ed 77       	push   $0x77eda0ae
77ed13eb:	68 20 a0 ed 77       	push   $0x77eda020
77ed13f0:	ff 15 e8 10 ee 77    	call   *0x77ee10e8
77ed13f6:	c7 04 24 78 00 00 00 	movl   $0x78,(%esp)
77ed13fd:	e8 0e 85 00 00       	call   77ed9910 <_SetLastError@4>
77ed1402:	31 c0                	xor    %eax,%eax
77ed1404:	c9                   	leave  
77ed1405:	c2 0c 00             	ret    $0xc
77ed1408:	90                   	nop    
77ed1409:	8d b4 26 00 00 00 00 	lea    0x0(%esi),%esi

77ed1410 <_GetAspectRatioFilterEx@8>:
77ed1410:	55                   	push   %ebp
77ed1411:	89 e5                	mov    %esp,%ebp
77ed1413:	83 ec 10             	sub    $0x10,%esp
77ed1416:	68 be a0 ed 77       	push   $0x77eda0be
77ed141b:	68 20 a0 ed 77       	push   $0x77eda020
77ed1420:	ff 15 e8 10 ee 77    	call   *0x77ee10e8
77ed1426:	c7 04 24 78 00 00 00 	movl   $0x78,(%esp)
77ed142d:	e8 de 84 00 00       	call   77ed9910 <_SetLastError@4>
77ed1432:	31 c0                	xor    %eax,%eax
77ed1434:	c9                   	leave  
77ed1435:	c2 08 00             	ret    $0x8
77ed1438:	90                   	nop    
77ed1439:	8d b4 26 00 00 00 00 	lea    0x0(%esi),%esi

77ed1440 <_GetBoundsRect@12>:
77ed1440:	55                   	push   %ebp
77ed1441:	89 e5                	mov    %esp,%ebp
77ed1443:	83 ec 10             	sub    $0x10,%esp
77ed1446:	68 d5 a0 ed 77       	push   $0x77eda0d5
77ed144b:	68 20 a0 ed 77       	push   $0x77eda020
77ed1450:	ff 15 e8 10 ee 77    	call   *0x77ee10e8
77ed1456:	c7 04 24 78 00 00 00 	movl   $0x78,(%esp)
77ed145d:	e8 ae 84 00 00       	call   77ed9910 <_SetLastError@4>
77ed1462:	31 c0                	xor    %eax,%eax
77ed1464:	c9                   	leave  
77ed1465:	c2 0c 00             	ret    $0xc
77ed1468:	90                   	nop    
77ed1469:	8d b4 26 00 00 00 00 	lea    0x0(%esi),%esi

77ed1470 <_GetMetaRgn@8>:
77ed1470:	55                   	push   %ebp
77ed1471:	89 e5                	mov    %esp,%ebp
77ed1473:	83 ec 10             	sub    $0x10,%esp
77ed1476:	68 e3 a0 ed 77       	push   $0x77eda0e3
77ed147b:	68 20 a0 ed 77       	push   $0x77eda020
77ed1480:	ff 15 e8 10 ee 77    	call   *0x77ee10e8
77ed1486:	c7 04 24 78 00 00 00 	movl   $0x78,(%esp)
77ed148d:	e8 7e 84 00 00       	call   77ed9910 <_SetLastError@4>
77ed1492:	31 c0                	xor    %eax,%eax
77ed1494:	c9                   	leave  
77ed1495:	c2 08 00             	ret    $0x8
77ed1498:	90                   	nop    
77ed1499:	8d b4 26 00 00 00 00 	lea    0x0(%esi),%esi

77ed14a0 <_GetMetaFileBitsEx@12>:
77ed14a0:	55                   	push   %ebp
77ed14a1:	89 e5                	mov    %esp,%ebp
77ed14a3:	83 ec 10             	sub    $0x10,%esp
77ed14a6:	68 ee a0 ed 77       	push   $0x77eda0ee
77ed14ab:	68 20 a0 ed 77       	push   $0x77eda020
77ed14b0:	ff 15 e8 10 ee 77    	call   *0x77ee10e8
77ed14b6:	c7 04 24 78 00 00 00 	movl   $0x78,(%esp)
77ed14bd:	e8 4e 84 00 00       	call   77ed9910 <_SetLastError@4>
77ed14c2:	31 c0                	xor    %eax,%eax
77ed14c4:	c9                   	leave  
77ed14c5:	c2 0c 00             	ret    $0xc
77ed14c8:	90                   	nop    
77ed14c9:	8d b4 26 00 00 00 00 	lea    0x0(%esi),%esi

77ed14d0 <_GetRasterizerCaps@8>:
77ed14d0:	55                   	push   %ebp
77ed14d1:	89 e5                	mov    %esp,%ebp
77ed14d3:	83 ec 10             	sub    $0x10,%esp
77ed14d6:	68 00 a1 ed 77       	push   $0x77eda100
77ed14db:	68 20 a0 ed 77       	push   $0x77eda020
77ed14e0:	ff 15 e8 10 ee 77    	call   *0x77ee10e8
77ed14e6:	c7 04 24 78 00 00 00 	movl   $0x78,(%esp)
77ed14ed:	e8 1e 84 00 00       	call   77ed9910 <_SetLastError@4>
77ed14f2:	31 c0                	xor    %eax,%eax
77ed14f4:	c9                   	leave  
77ed14f5:	c2 08 00             	ret    $0x8
77ed14f8:	90                   	nop    
77ed14f9:	8d b4 26 00 00 00 00 	lea    0x0(%esi),%esi

77ed1500 <_GetSystemPaletteUse@4>:
77ed1500:	55                   	push   %ebp
77ed1501:	89 e5                	mov    %esp,%ebp
77ed1503:	c9                   	leave  
77ed1504:	e9 f2 47 00 00       	jmp    77ed5cfb <_NtGdiGetSystemPaletteUse@4>
77ed1509:	8d b4 26 00 00 00 00 	lea    0x0(%esi),%esi

77ed1510 <_GetTextCharacterExtra@4>:
77ed1510:	55                   	push   %ebp
77ed1511:	89 e5                	mov    %esp,%ebp
77ed1513:	83 ec 10             	sub    $0x10,%esp
77ed1516:	68 12 a1 ed 77       	push   $0x77eda112
77ed151b:	68 20 a0 ed 77       	push   $0x77eda020
77ed1520:	ff 15 e8 10 ee 77    	call   *0x77ee10e8
77ed1526:	c7 04 24 78 00 00 00 	movl   $0x78,(%esp)
77ed152d:	e8 de 83 00 00       	call   77ed9910 <_SetLastError@4>
77ed1532:	31 c0                	xor    %eax,%eax
77ed1534:	c9                   	leave  
77ed1535:	c2 04 00             	ret    $0x4
77ed1538:	90                   	nop    
77ed1539:	8d b4 26 00 00 00 00 	lea    0x0(%esi),%esi

77ed1540 <_GetTextCharset@4>:
77ed1540:	55                   	push   %ebp
77ed1541:	89 e5                	mov    %esp,%ebp
77ed1543:	83 ec 10             	sub    $0x10,%esp
77ed1546:	68 28 a1 ed 77       	push   $0x77eda128
77ed154b:	68 20 a0 ed 77       	push   $0x77eda020
77ed1550:	ff 15 e8 10 ee 77    	call   *0x77ee10e8
77ed1556:	c7 04 24 78 00 00 00 	movl   $0x78,(%esp)
77ed155d:	e8 ae 83 00 00       	call   77ed9910 <_SetLastError@4>
77ed1562:	31 c0                	xor    %eax,%eax
77ed1564:	c9                   	leave  
77ed1565:	c2 04 00             	ret    $0x4
77ed1568:	90                   	nop    
77ed1569:	8d b4 26 00 00 00 00 	lea    0x0(%esi),%esi

77ed1570 <_GetTextCharsetInfo@12>:
77ed1570:	55                   	push   %ebp
77ed1571:	89 e5                	mov    %esp,%ebp
77ed1573:	83 ec 10             	sub    $0x10,%esp
77ed1576:	68 37 a1 ed 77       	push   $0x77eda137
77ed157b:	68 20 a0 ed 77       	push   $0x77eda020
77ed1580:	ff 15 e8 10 ee 77    	call   *0x77ee10e8
77ed1586:	c7 04 24 78 00 00 00 	movl   $0x78,(%esp)
77ed158d:	e8 7e 83 00 00       	call   77ed9910 <_SetLastError@4>
77ed1592:	31 c0                	xor    %eax,%eax
77ed1594:	c9                   	leave  
77ed1595:	c2 0c 00             	ret    $0xc
77ed1598:	90                   	nop    
77ed1599:	8d b4 26 00 00 00 00 	lea    0x0(%esi),%esi

77ed15a0 <_GetFontLanguageInfo@4>:
77ed15a0:	55                   	push   %ebp
77ed15a1:	89 e5                	mov    %esp,%ebp
77ed15a3:	83 ec 10             	sub    $0x10,%esp
77ed15a6:	68 4a a1 ed 77       	push   $0x77eda14a
77ed15ab:	68 20 a0 ed 77       	push   $0x77eda020
77ed15b0:	ff 15 e8 10 ee 77    	call   *0x77ee10e8
77ed15b6:	c7 04 24 78 00 00 00 	movl   $0x78,(%esp)
77ed15bd:	e8 4e 83 00 00       	call   77ed9910 <_SetLastError@4>
77ed15c2:	31 c0                	xor    %eax,%eax
77ed15c4:	c9                   	leave  
77ed15c5:	c2 04 00             	ret    $0x4
77ed15c8:	90                   	nop    
77ed15c9:	8d b4 26 00 00 00 00 	lea    0x0(%esi),%esi

77ed15d0 <_PlayMetaFile@8>:
77ed15d0:	55                   	push   %ebp
77ed15d1:	89 e5                	mov    %esp,%ebp
77ed15d3:	83 ec 10             	sub    $0x10,%esp
77ed15d6:	68 5e a1 ed 77       	push   $0x77eda15e
77ed15db:	68 20 a0 ed 77       	push   $0x77eda020
77ed15e0:	ff 15 e8 10 ee 77    	call   *0x77ee10e8
77ed15e6:	c7 04 24 78 00 00 00 	movl   $0x78,(%esp)
77ed15ed:	e8 1e 83 00 00       	call   77ed9910 <_SetLastError@4>
77ed15f2:	31 c0                	xor    %eax,%eax
77ed15f4:	c9                   	leave  
77ed15f5:	c2 08 00             	ret    $0x8
77ed15f8:	90                   	nop    
77ed15f9:	8d b4 26 00 00 00 00 	lea    0x0(%esi),%esi

77ed1600 <_ResizePalette@8>:
77ed1600:	55                   	push   %ebp
77ed1601:	89 e5                	mov    %esp,%ebp
77ed1603:	83 ec 10             	sub    $0x10,%esp
77ed1606:	68 6b a1 ed 77       	push   $0x77eda16b
77ed160b:	68 20 a0 ed 77       	push   $0x77eda020
77ed1610:	ff 15 e8 10 ee 77    	call   *0x77ee10e8
77ed1616:	c7 04 24 78 00 00 00 	movl   $0x78,(%esp)
77ed161d:	e8 ee 82 00 00       	call   77ed9910 <_SetLastError@4>
77ed1622:	31 c0                	xor    %eax,%eax
77ed1624:	c9                   	leave  
77ed1625:	c2 08 00             	ret    $0x8
77ed1628:	90                   	nop    
77ed1629:	8d b4 26 00 00 00 00 	lea    0x0(%esi),%esi

77ed1630 <_SetMetaRgn@4>:
77ed1630:	55                   	push   %ebp
77ed1631:	89 e5                	mov    %esp,%ebp
77ed1633:	83 ec 10             	sub    $0x10,%esp
77ed1636:	68 79 a1 ed 77       	push   $0x77eda179
77ed163b:	68 20 a0 ed 77       	push   $0x77eda020
77ed1640:	ff 15 e8 10 ee 77    	call   *0x77ee10e8
77ed1646:	c7 04 24 78 00 00 00 	movl   $0x78,(%esp)
77ed164d:	e8 be 82 00 00       	call   77ed9910 <_SetLastError@4>
77ed1652:	31 c0                	xor    %eax,%eax
77ed1654:	c9                   	leave  
77ed1655:	c2 04 00             	ret    $0x4
77ed1658:	90                   	nop    
77ed1659:	8d b4 26 00 00 00 00 	lea    0x0(%esi),%esi

77ed1660 <_SetBoundsRect@12>:
77ed1660:	55                   	push   %ebp
77ed1661:	89 e5                	mov    %esp,%ebp
77ed1663:	83 ec 10             	sub    $0x10,%esp
77ed1666:	68 84 a1 ed 77       	push   $0x77eda184
77ed166b:	68 20 a0 ed 77       	push   $0x77eda020
77ed1670:	ff 15 e8 10 ee 77    	call   *0x77ee10e8
77ed1676:	c7 04 24 78 00 00 00 	movl   $0x78,(%esp)
77ed167d:	e8 8e 82 00 00       	call   77ed9910 <_SetLastError@4>
77ed1682:	31 c0                	xor    %eax,%eax
77ed1684:	c9                   	leave  
77ed1685:	c2 0c 00             	ret    $0xc
77ed1688:	90                   	nop    
77ed1689:	8d b4 26 00 00 00 00 	lea    0x0(%esi),%esi

77ed1690 <_SetMapperFlags@8>:
77ed1690:	55                   	push   %ebp
77ed1691:	89 e5                	mov    %esp,%ebp
77ed1693:	83 ec 10             	sub    $0x10,%esp
77ed1696:	68 92 a1 ed 77       	push   $0x77eda192
77ed169b:	68 20 a0 ed 77       	push   $0x77eda020
77ed16a0:	ff 15 e8 10 ee 77    	call   *0x77ee10e8
77ed16a6:	c7 04 24 78 00 00 00 	movl   $0x78,(%esp)
77ed16ad:	e8 5e 82 00 00       	call   77ed9910 <_SetLastError@4>
77ed16b2:	31 c0                	xor    %eax,%eax
77ed16b4:	c9                   	leave  
77ed16b5:	c2 08 00             	ret    $0x8
77ed16b8:	90                   	nop    
77ed16b9:	8d b4 26 00 00 00 00 	lea    0x0(%esi),%esi

77ed16c0 <_SetMetaFileBitsEx@8>:
77ed16c0:	55                   	push   %ebp
77ed16c1:	89 e5                	mov    %esp,%ebp
77ed16c3:	83 ec 10             	sub    $0x10,%esp
77ed16c6:	68 a1 a1 ed 77       	push   $0x77eda1a1
77ed16cb:	68 20 a0 ed 77       	push   $0x77eda020
77ed16d0:	ff 15 e8 10 ee 77    	call   *0x77ee10e8
77ed16d6:	c7 04 24 78 00 00 00 	movl   $0x78,(%esp)
77ed16dd:	e8 2e 82 00 00       	call   77ed9910 <_SetLastError@4>
77ed16e2:	31 c0                	xor    %eax,%eax
77ed16e4:	c9                   	leave  
77ed16e5:	c2 08 00             	ret    $0x8
77ed16e8:	90                   	nop    
77ed16e9:	8d b4 26 00 00 00 00 	lea    0x0(%esi),%esi

77ed16f0 <_SetSystemPaletteUse@8>:
77ed16f0:	55                   	push   %ebp
77ed16f1:	89 e5                	mov    %esp,%ebp
77ed16f3:	83 ec 10             	sub    $0x10,%esp
77ed16f6:	68 b3 a1 ed 77       	push   $0x77eda1b3
77ed16fb:	68 20 a0 ed 77       	push   $0x77eda020
77ed1700:	ff 15 e8 10 ee 77    	call   *0x77ee10e8
77ed1706:	c7 04 24 78 00 00 00 	movl   $0x78,(%esp)
77ed170d:	e8 fe 81 00 00       	call   77ed9910 <_SetLastError@4>
77ed1712:	31 c0                	xor    %eax,%eax
77ed1714:	c9                   	leave  
77ed1715:	c2 08 00             	ret    $0x8
77ed1718:	90                   	nop    
77ed1719:	8d b4 26 00 00 00 00 	lea    0x0(%esi),%esi

77ed1720 <_SetTextCharacterExtra@8>:
77ed1720:	55                   	push   %ebp
77ed1721:	89 e5                	mov    %esp,%ebp
77ed1723:	83 ec 10             	sub    $0x10,%esp
77ed1726:	68 c7 a1 ed 77       	push   $0x77eda1c7
77ed172b:	68 20 a0 ed 77       	push   $0x77eda020
77ed1730:	ff 15 e8 10 ee 77    	call   *0x77ee10e8
77ed1736:	c7 04 24 78 00 00 00 	movl   $0x78,(%esp)
77ed173d:	e8 ce 81 00 00       	call   77ed9910 <_SetLastError@4>
77ed1742:	31 c0                	xor    %eax,%eax
77ed1744:	c9                   	leave  
77ed1745:	c2 08 00             	ret    $0x8
77ed1748:	90                   	nop    
77ed1749:	8d b4 26 00 00 00 00 	lea    0x0(%esi),%esi

77ed1750 <_SetTextJustification@12>:
77ed1750:	55                   	push   %ebp
77ed1751:	89 e5                	mov    %esp,%ebp
77ed1753:	83 ec 10             	sub    $0x10,%esp
77ed1756:	68 dd a1 ed 77       	push   $0x77eda1dd
77ed175b:	68 20 a0 ed 77       	push   $0x77eda020
77ed1760:	ff 15 e8 10 ee 77    	call   *0x77ee10e8
77ed1766:	c7 04 24 78 00 00 00 	movl   $0x78,(%esp)
77ed176d:	e8 9e 81 00 00       	call   77ed9910 <_SetLastError@4>
77ed1772:	31 c0                	xor    %eax,%eax
77ed1774:	c9                   	leave  
77ed1775:	c2 0c 00             	ret    $0xc
77ed1778:	90                   	nop    
77ed1779:	8d b4 26 00 00 00 00 	lea    0x0(%esi),%esi

77ed1780 <_UpdateColors@4>:
77ed1780:	55                   	push   %ebp
77ed1781:	89 e5                	mov    %esp,%ebp
77ed1783:	83 ec 10             	sub    $0x10,%esp
77ed1786:	68 f2 a1 ed 77       	push   $0x77eda1f2
77ed178b:	68 20 a0 ed 77       	push   $0x77eda020
77ed1790:	ff 15 e8 10 ee 77    	call   *0x77ee10e8
77ed1796:	c7 04 24 78 00 00 00 	movl   $0x78,(%esp)
77ed179d:	e8 6e 81 00 00       	call   77ed9910 <_SetLastError@4>
77ed17a2:	31 c0                	xor    %eax,%eax
77ed17a4:	c9                   	leave  
77ed17a5:	c2 04 00             	ret    $0x4
77ed17a8:	90                   	nop    
77ed17a9:	8d b4 26 00 00 00 00 	lea    0x0(%esi),%esi

77ed17b0 <_PlayMetaFileRecord@16>:
77ed17b0:	55                   	push   %ebp
77ed17b1:	89 e5                	mov    %esp,%ebp
77ed17b3:	83 ec 10             	sub    $0x10,%esp
77ed17b6:	68 ff a1 ed 77       	push   $0x77eda1ff
77ed17bb:	68 20 a0 ed 77       	push   $0x77eda020
77ed17c0:	ff 15 e8 10 ee 77    	call   *0x77ee10e8
77ed17c6:	c7 04 24 78 00 00 00 	movl   $0x78,(%esp)
77ed17cd:	e8 3e 81 00 00       	call   77ed9910 <_SetLastError@4>
77ed17d2:	31 c0                	xor    %eax,%eax
77ed17d4:	c9                   	leave  
77ed17d5:	c2 10 00             	ret    $0x10
77ed17d8:	90                   	nop    
77ed17d9:	8d b4 26 00 00 00 00 	lea    0x0(%esi),%esi

77ed17e0 <_EnumMetaFile@16>:
77ed17e0:	55                   	push   %ebp
77ed17e1:	89 e5                	mov    %esp,%ebp
77ed17e3:	83 ec 10             	sub    $0x10,%esp
77ed17e6:	68 12 a2 ed 77       	push   $0x77eda212
77ed17eb:	68 20 a0 ed 77       	push   $0x77eda020
77ed17f0:	ff 15 e8 10 ee 77    	call   *0x77ee10e8
77ed17f6:	c7 04 24 78 00 00 00 	movl   $0x78,(%esp)
77ed17fd:	e8 0e 81 00 00       	call   77ed9910 <_SetLastError@4>
77ed1802:	31 c0                	xor    %eax,%eax
77ed1804:	c9                   	leave  
77ed1805:	c2 10 00             	ret    $0x10
77ed1808:	90                   	nop    
77ed1809:	8d b4 26 00 00 00 00 	lea    0x0(%esi),%esi

77ed1810 <_CloseEnhMetaFile@4>:
77ed1810:	55                   	push   %ebp
77ed1811:	89 e5                	mov    %esp,%ebp
77ed1813:	83 ec 10             	sub    $0x10,%esp
77ed1816:	68 1f a2 ed 77       	push   $0x77eda21f
77ed181b:	68 20 a0 ed 77       	push   $0x77eda020
77ed1820:	ff 15 e8 10 ee 77    	call   *0x77ee10e8
77ed1826:	c7 04 24 78 00 00 00 	movl   $0x78,(%esp)
77ed182d:	e8 de 80 00 00       	call   77ed9910 <_SetLastError@4>
77ed1832:	31 c0                	xor    %eax,%eax
77ed1834:	c9                   	leave  
77ed1835:	c2 04 00             	ret    $0x4
77ed1838:	90                   	nop    
77ed1839:	8d b4 26 00 00 00 00 	lea    0x0(%esi),%esi

77ed1840 <_DeleteEnhMetaFile@4>:
77ed1840:	55                   	push   %ebp
77ed1841:	89 e5                	mov    %esp,%ebp
77ed1843:	83 ec 10             	sub    $0x10,%esp
77ed1846:	68 30 a2 ed 77       	push   $0x77eda230
77ed184b:	68 20 a0 ed 77       	push   $0x77eda020
77ed1850:	ff 15 e8 10 ee 77    	call   *0x77ee10e8
77ed1856:	c7 04 24 78 00 00 00 	movl   $0x78,(%esp)
77ed185d:	e8 ae 80 00 00       	call   77ed9910 <_SetLastError@4>
77ed1862:	31 c0                	xor    %eax,%eax
77ed1864:	c9                   	leave  
77ed1865:	c2 04 00             	ret    $0x4
77ed1868:	90                   	nop    
77ed1869:	8d b4 26 00 00 00 00 	lea    0x0(%esi),%esi

77ed1870 <_EnumEnhMetaFile@20>:
77ed1870:	55                   	push   %ebp
77ed1871:	89 e5                	mov    %esp,%ebp
77ed1873:	83 ec 10             	sub    $0x10,%esp
77ed1876:	68 42 a2 ed 77       	push   $0x77eda242
77ed187b:	68 20 a0 ed 77       	push   $0x77eda020
77ed1880:	ff 15 e8 10 ee 77    	call   *0x77ee10e8
77ed1886:	c7 04 24 78 00 00 00 	movl   $0x78,(%esp)
77ed188d:	e8 7e 80 00 00       	call   77ed9910 <_SetLastError@4>
77ed1892:	31 c0                	xor    %eax,%eax
77ed1894:	c9                   	leave  
77ed1895:	c2 14 00             	ret    $0x14
77ed1898:	90                   	nop    
77ed1899:	8d b4 26 00 00 00 00 	lea    0x0(%esi),%esi

77ed18a0 <_GetEnhMetaFileBits@12>:
77ed18a0:	55                   	push   %ebp
77ed18a1:	89 e5                	mov    %esp,%ebp
77ed18a3:	83 ec 10             	sub    $0x10,%esp
77ed18a6:	68 52 a2 ed 77       	push   $0x77eda252
77ed18ab:	68 20 a0 ed 77       	push   $0x77eda020
77ed18b0:	ff 15 e8 10 ee 77    	call   *0x77ee10e8
77ed18b6:	c7 04 24 78 00 00 00 	movl   $0x78,(%esp)
77ed18bd:	e8 4e 80 00 00       	call   77ed9910 <_SetLastError@4>
77ed18c2:	31 c0                	xor    %eax,%eax
77ed18c4:	c9                   	leave  
77ed18c5:	c2 0c 00             	ret    $0xc
77ed18c8:	90                   	nop    
77ed18c9:	8d b4 26 00 00 00 00 	lea    0x0(%esi),%esi

77ed18d0 <_GetEnhMetaFileHeader@12>:
77ed18d0:	55                   	push   %ebp
77ed18d1:	89 e5                	mov    %esp,%ebp
77ed18d3:	83 ec 10             	sub    $0x10,%esp
77ed18d6:	68 65 a2 ed 77       	push   $0x77eda265
77ed18db:	68 20 a0 ed 77       	push   $0x77eda020
77ed18e0:	ff 15 e8 10 ee 77    	call   *0x77ee10e8
77ed18e6:	c7 04 24 78 00 00 00 	movl   $0x78,(%esp)
77ed18ed:	e8 1e 80 00 00       	call   77ed9910 <_SetLastError@4>
77ed18f2:	31 c0                	xor    %eax,%eax
77ed18f4:	c9                   	leave  
77ed18f5:	c2 0c 00             	ret    $0xc
77ed18f8:	90                   	nop    
77ed18f9:	8d b4 26 00 00 00 00 	lea    0x0(%esi),%esi

77ed1900 <_GetEnhMetaFilePaletteEntries@12>:
77ed1900:	55                   	push   %ebp
77ed1901:	89 e5                	mov    %esp,%ebp
77ed1903:	83 ec 10             	sub    $0x10,%esp
77ed1906:	68 7a a2 ed 77       	push   $0x77eda27a
77ed190b:	68 20 a0 ed 77       	push   $0x77eda020
77ed1910:	ff 15 e8 10 ee 77    	call   *0x77ee10e8
77ed1916:	c7 04 24 78 00 00 00 	movl   $0x78,(%esp)
77ed191d:	e8 ee 7f 00 00       	call   77ed9910 <_SetLastError@4>
77ed1922:	31 c0                	xor    %eax,%eax
77ed1924:	c9                   	leave  
77ed1925:	c2 0c 00             	ret    $0xc
77ed1928:	90                   	nop    
77ed1929:	8d b4 26 00 00 00 00 	lea    0x0(%esi),%esi

77ed1930 <_GetWinMetaFileBits@20>:
77ed1930:	55                   	push   %ebp
77ed1931:	89 e5                	mov    %esp,%ebp
77ed1933:	83 ec 10             	sub    $0x10,%esp
77ed1936:	68 97 a2 ed 77       	push   $0x77eda297
77ed193b:	68 20 a0 ed 77       	push   $0x77eda020
77ed1940:	ff 15 e8 10 ee 77    	call   *0x77ee10e8
77ed1946:	c7 04 24 78 00 00 00 	movl   $0x78,(%esp)
77ed194d:	e8 be 7f 00 00       	call   77ed9910 <_SetLastError@4>
77ed1952:	31 c0                	xor    %eax,%eax
77ed1954:	c9                   	leave  
77ed1955:	c2 14 00             	ret    $0x14
77ed1958:	90                   	nop    
77ed1959:	8d b4 26 00 00 00 00 	lea    0x0(%esi),%esi

77ed1960 <_PlayEnhMetaFile@12>:
77ed1960:	55                   	push   %ebp
77ed1961:	89 e5                	mov    %esp,%ebp
77ed1963:	83 ec 10             	sub    $0x10,%esp
77ed1966:	68 aa a2 ed 77       	push   $0x77eda2aa
77ed196b:	68 20 a0 ed 77       	push   $0x77eda020
77ed1970:	ff 15 e8 10 ee 77    	call   *0x77ee10e8
77ed1976:	c7 04 24 78 00 00 00 	movl   $0x78,(%esp)
77ed197d:	e8 8e 7f 00 00       	call   77ed9910 <_SetLastError@4>
77ed1982:	31 c0                	xor    %eax,%eax
77ed1984:	c9                   	leave  
77ed1985:	c2 0c 00             	ret    $0xc
77ed1988:	90                   	nop    
77ed1989:	8d b4 26 00 00 00 00 	lea    0x0(%esi),%esi

77ed1990 <_PlayEnhMetaFileRecord@16>:
77ed1990:	55                   	push   %ebp
77ed1991:	89 e5                	mov    %esp,%ebp
77ed1993:	83 ec 10             	sub    $0x10,%esp
77ed1996:	68 ba a2 ed 77       	push   $0x77eda2ba
77ed199b:	68 20 a0 ed 77       	push   $0x77eda020
77ed19a0:	ff 15 e8 10 ee 77    	call   *0x77ee10e8
77ed19a6:	c7 04 24 78 00 00 00 	movl   $0x78,(%esp)
77ed19ad:	e8 5e 7f 00 00       	call   77ed9910 <_SetLastError@4>
77ed19b2:	31 c0                	xor    %eax,%eax
77ed19b4:	c9                   	leave  
77ed19b5:	c2 10 00             	ret    $0x10
77ed19b8:	90                   	nop    
77ed19b9:	8d b4 26 00 00 00 00 	lea    0x0(%esi),%esi

77ed19c0 <_SetEnhMetaFileBits@8>:
77ed19c0:	55                   	push   %ebp
77ed19c1:	89 e5                	mov    %esp,%ebp
77ed19c3:	83 ec 10             	sub    $0x10,%esp
77ed19c6:	68 d0 a2 ed 77       	push   $0x77eda2d0
77ed19cb:	68 20 a0 ed 77       	push   $0x77eda020
77ed19d0:	ff 15 e8 10 ee 77    	call   *0x77ee10e8
77ed19d6:	c7 04 24 78 00 00 00 	movl   $0x78,(%esp)
77ed19dd:	e8 2e 7f 00 00       	call   77ed9910 <_SetLastError@4>
77ed19e2:	31 c0                	xor    %eax,%eax
77ed19e4:	c9                   	leave  
77ed19e5:	c2 08 00             	ret    $0x8
77ed19e8:	90                   	nop    
77ed19e9:	8d b4 26 00 00 00 00 	lea    0x0(%esi),%esi

77ed19f0 <_SetWinMetaFileBits@16>:
77ed19f0:	55                   	push   %ebp
77ed19f1:	89 e5                	mov    %esp,%ebp
77ed19f3:	83 ec 10             	sub    $0x10,%esp
77ed19f6:	68 e3 a2 ed 77       	push   $0x77eda2e3
77ed19fb:	68 20 a0 ed 77       	push   $0x77eda020
77ed1a00:	ff 15 e8 10 ee 77    	call   *0x77ee10e8
77ed1a06:	c7 04 24 78 00 00 00 	movl   $0x78,(%esp)
77ed1a0d:	e8 fe 7e 00 00       	call   77ed9910 <_SetLastError@4>
77ed1a12:	31 c0                	xor    %eax,%eax
77ed1a14:	c9                   	leave  
77ed1a15:	c2 10 00             	ret    $0x10
77ed1a18:	90                   	nop    
77ed1a19:	8d b4 26 00 00 00 00 	lea    0x0(%esi),%esi

77ed1a20 <_GdiComment@12>:
77ed1a20:	55                   	push   %ebp
77ed1a21:	89 e5                	mov    %esp,%ebp
77ed1a23:	83 ec 10             	sub    $0x10,%esp
77ed1a26:	68 f6 a2 ed 77       	push   $0x77eda2f6
77ed1a2b:	68 20 a0 ed 77       	push   $0x77eda020
77ed1a30:	ff 15 e8 10 ee 77    	call   *0x77ee10e8
77ed1a36:	c7 04 24 78 00 00 00 	movl   $0x78,(%esp)
77ed1a3d:	e8 ce 7e 00 00       	call   77ed9910 <_SetLastError@4>
77ed1a42:	31 c0                	xor    %eax,%eax
77ed1a44:	c9                   	leave  
77ed1a45:	c2 0c 00             	ret    $0xc
77ed1a48:	90                   	nop    
77ed1a49:	8d b4 26 00 00 00 00 	lea    0x0(%esi),%esi

77ed1a50 <_AngleArc@24>:
77ed1a50:	55                   	push   %ebp
77ed1a51:	89 e5                	mov    %esp,%ebp
77ed1a53:	83 ec 10             	sub    $0x10,%esp
77ed1a56:	68 01 a3 ed 77       	push   $0x77eda301
77ed1a5b:	68 20 a0 ed 77       	push   $0x77eda020
77ed1a60:	ff 15 e8 10 ee 77    	call   *0x77ee10e8
77ed1a66:	c7 04 24 78 00 00 00 	movl   $0x78,(%esp)
77ed1a6d:	e8 9e 7e 00 00       	call   77ed9910 <_SetLastError@4>
77ed1a72:	31 c0                	xor    %eax,%eax
77ed1a74:	c9                   	leave  
77ed1a75:	c2 18 00             	ret    $0x18
77ed1a78:	90                   	nop    
77ed1a79:	8d b4 26 00 00 00 00 	lea    0x0(%esi),%esi

77ed1a80 <_SetColorAdjustment@8>:
77ed1a80:	55                   	push   %ebp
77ed1a81:	89 e5                	mov    %esp,%ebp
77ed1a83:	83 ec 10             	sub    $0x10,%esp
77ed1a86:	68 0a a3 ed 77       	push   $0x77eda30a
77ed1a8b:	68 20 a0 ed 77       	push   $0x77eda020
77ed1a90:	ff 15 e8 10 ee 77    	call   *0x77ee10e8
77ed1a96:	c7 04 24 78 00 00 00 	movl   $0x78,(%esp)
77ed1a9d:	e8 6e 7e 00 00       	call   77ed9910 <_SetLastError@4>
77ed1aa2:	31 c0                	xor    %eax,%eax
77ed1aa4:	c9                   	leave  
77ed1aa5:	c2 08 00             	ret    $0x8
77ed1aa8:	90                   	nop    
77ed1aa9:	8d b4 26 00 00 00 00 	lea    0x0(%esi),%esi

77ed1ab0 <_GetColorAdjustment@8>:
77ed1ab0:	55                   	push   %ebp
77ed1ab1:	89 e5                	mov    %esp,%ebp
77ed1ab3:	83 ec 10             	sub    $0x10,%esp
77ed1ab6:	68 1d a3 ed 77       	push   $0x77eda31d
77ed1abb:	68 20 a0 ed 77       	push   $0x77eda020
77ed1ac0:	ff 15 e8 10 ee 77    	call   *0x77ee10e8
77ed1ac6:	c7 04 24 78 00 00 00 	movl   $0x78,(%esp)
77ed1acd:	e8 3e 7e 00 00       	call   77ed9910 <_SetLastError@4>
77ed1ad2:	31 c0                	xor    %eax,%eax
77ed1ad4:	c9                   	leave  
77ed1ad5:	c2 08 00             	ret    $0x8
77ed1ad8:	90                   	nop    
77ed1ad9:	8d b4 26 00 00 00 00 	lea    0x0(%esi),%esi

77ed1ae0 <_EndDoc@4>:
77ed1ae0:	55                   	push   %ebp
77ed1ae1:	89 e5                	mov    %esp,%ebp
77ed1ae3:	83 ec 10             	sub    $0x10,%esp
77ed1ae6:	68 30 a3 ed 77       	push   $0x77eda330
77ed1aeb:	68 20 a0 ed 77       	push   $0x77eda020
77ed1af0:	ff 15 e8 10 ee 77    	call   *0x77ee10e8
77ed1af6:	c7 04 24 78 00 00 00 	movl   $0x78,(%esp)
77ed1afd:	e8 0e 7e 00 00       	call   77ed9910 <_SetLastError@4>
77ed1b02:	31 c0                	xor    %eax,%eax
77ed1b04:	c9                   	leave  
77ed1b05:	c2 04 00             	ret    $0x4
77ed1b08:	90                   	nop    
77ed1b09:	8d b4 26 00 00 00 00 	lea    0x0(%esi),%esi

77ed1b10 <_StartPage@4>:
77ed1b10:	55                   	push   %ebp
77ed1b11:	89 e5                	mov    %esp,%ebp
77ed1b13:	83 ec 10             	sub    $0x10,%esp
77ed1b16:	68 37 a3 ed 77       	push   $0x77eda337
77ed1b1b:	68 20 a0 ed 77       	push   $0x77eda020
77ed1b20:	ff 15 e8 10 ee 77    	call   *0x77ee10e8
77ed1b26:	c7 04 24 78 00 00 00 	movl   $0x78,(%esp)
77ed1b2d:	e8 de 7d 00 00       	call   77ed9910 <_SetLastError@4>
77ed1b32:	31 c0                	xor    %eax,%eax
77ed1b34:	c9                   	leave  
77ed1b35:	c2 04 00             	ret    $0x4
77ed1b38:	90                   	nop    
77ed1b39:	8d b4 26 00 00 00 00 	lea    0x0(%esi),%esi

77ed1b40 <_EndPage@4>:
77ed1b40:	55                   	push   %ebp
77ed1b41:	89 e5                	mov    %esp,%ebp
77ed1b43:	83 ec 10             	sub    $0x10,%esp
77ed1b46:	68 41 a3 ed 77       	push   $0x77eda341
77ed1b4b:	68 20 a0 ed 77       	push   $0x77eda020
77ed1b50:	ff 15 e8 10 ee 77    	call   *0x77ee10e8
77ed1b56:	c7 04 24 78 00 00 00 	movl   $0x78,(%esp)
77ed1b5d:	e8 ae 7d 00 00       	call   77ed9910 <_SetLastError@4>
77ed1b62:	31 c0                	xor    %eax,%eax
77ed1b64:	c9                   	leave  
77ed1b65:	c2 04 00             	ret    $0x4
77ed1b68:	90                   	nop    
77ed1b69:	8d b4 26 00 00 00 00 	lea    0x0(%esi),%esi

77ed1b70 <_AbortDoc@4>:
77ed1b70:	55                   	push   %ebp
77ed1b71:	89 e5                	mov    %esp,%ebp
77ed1b73:	83 ec 10             	sub    $0x10,%esp
77ed1b76:	68 49 a3 ed 77       	push   $0x77eda349
77ed1b7b:	68 20 a0 ed 77       	push   $0x77eda020
77ed1b80:	ff 15 e8 10 ee 77    	call   *0x77ee10e8
77ed1b86:	c7 04 24 78 00 00 00 	movl   $0x78,(%esp)
77ed1b8d:	e8 7e 7d 00 00       	call   77ed9910 <_SetLastError@4>
77ed1b92:	31 c0                	xor    %eax,%eax
77ed1b94:	c9                   	leave  
77ed1b95:	c2 04 00             	ret    $0x4
77ed1b98:	90                   	nop    
77ed1b99:	8d b4 26 00 00 00 00 	lea    0x0(%esi),%esi

77ed1ba0 <_SetAbortProc@8>:
77ed1ba0:	55                   	push   %ebp
77ed1ba1:	89 e5                	mov    %esp,%ebp
77ed1ba3:	83 ec 10             	sub    $0x10,%esp
77ed1ba6:	68 52 a3 ed 77       	push   $0x77eda352
77ed1bab:	68 20 a0 ed 77       	push   $0x77eda020
77ed1bb0:	ff 15 e8 10 ee 77    	call   *0x77ee10e8
77ed1bb6:	c7 04 24 78 00 00 00 	movl   $0x78,(%esp)
77ed1bbd:	e8 4e 7d 00 00       	call   77ed9910 <_SetLastError@4>
77ed1bc2:	31 c0                	xor    %eax,%eax
77ed1bc4:	c9                   	leave  
77ed1bc5:	c2 08 00             	ret    $0x8
77ed1bc8:	90                   	nop    
77ed1bc9:	8d b4 26 00 00 00 00 	lea    0x0(%esi),%esi

77ed1bd0 <_AbortPath@4>:
77ed1bd0:	55                   	push   %ebp
77ed1bd1:	89 e5                	mov    %esp,%ebp
77ed1bd3:	83 ec 10             	sub    $0x10,%esp
77ed1bd6:	68 5f a3 ed 77       	push   $0x77eda35f
77ed1bdb:	68 20 a0 ed 77       	push   $0x77eda020
77ed1be0:	ff 15 e8 10 ee 77    	call   *0x77ee10e8
77ed1be6:	c7 04 24 78 00 00 00 	movl   $0x78,(%esp)
77ed1bed:	e8 1e 7d 00 00       	call   77ed9910 <_SetLastError@4>
77ed1bf2:	31 c0                	xor    %eax,%eax
77ed1bf4:	c9                   	leave  
77ed1bf5:	c2 04 00             	ret    $0x4
77ed1bf8:	90                   	nop    
77ed1bf9:	8d b4 26 00 00 00 00 	lea    0x0(%esi),%esi

77ed1c00 <_BeginPath@4>:
77ed1c00:	55                   	push   %ebp
77ed1c01:	89 e5                	mov    %esp,%ebp
77ed1c03:	83 ec 10             	sub    $0x10,%esp
77ed1c06:	68 69 a3 ed 77       	push   $0x77eda369
77ed1c0b:	68 20 a0 ed 77       	push   $0x77eda020
77ed1c10:	ff 15 e8 10 ee 77    	call   *0x77ee10e8
77ed1c16:	c7 04 24 78 00 00 00 	movl   $0x78,(%esp)
77ed1c1d:	e8 ee 7c 00 00       	call   77ed9910 <_SetLastError@4>
77ed1c22:	31 c0                	xor    %eax,%eax
77ed1c24:	c9                   	leave  
77ed1c25:	c2 04 00             	ret    $0x4
77ed1c28:	90                   	nop    
77ed1c29:	8d b4 26 00 00 00 00 	lea    0x0(%esi),%esi

77ed1c30 <_CloseFigure@4>:
77ed1c30:	55                   	push   %ebp
77ed1c31:	89 e5                	mov    %esp,%ebp
77ed1c33:	83 ec 10             	sub    $0x10,%esp
77ed1c36:	68 73 a3 ed 77       	push   $0x77eda373
77ed1c3b:	68 20 a0 ed 77       	push   $0x77eda020
77ed1c40:	ff 15 e8 10 ee 77    	call   *0x77ee10e8
77ed1c46:	c7 04 24 78 00 00 00 	movl   $0x78,(%esp)
77ed1c4d:	e8 be 7c 00 00       	call   77ed9910 <_SetLastError@4>
77ed1c52:	31 c0                	xor    %eax,%eax
77ed1c54:	c9                   	leave  
77ed1c55:	c2 04 00             	ret    $0x4
77ed1c58:	90                   	nop    
77ed1c59:	8d b4 26 00 00 00 00 	lea    0x0(%esi),%esi

77ed1c60 <_EndPath@4>:
77ed1c60:	55                   	push   %ebp
77ed1c61:	89 e5                	mov    %esp,%ebp
77ed1c63:	83 ec 10             	sub    $0x10,%esp
77ed1c66:	68 7f a3 ed 77       	push   $0x77eda37f
77ed1c6b:	68 20 a0 ed 77       	push   $0x77eda020
77ed1c70:	ff 15 e8 10 ee 77    	call   *0x77ee10e8
77ed1c76:	c7 04 24 78 00 00 00 	movl   $0x78,(%esp)
77ed1c7d:	e8 8e 7c 00 00       	call   77ed9910 <_SetLastError@4>
77ed1c82:	31 c0                	xor    %eax,%eax
77ed1c84:	c9                   	leave  
77ed1c85:	c2 04 00             	ret    $0x4
77ed1c88:	90                   	nop    
77ed1c89:	8d b4 26 00 00 00 00 	lea    0x0(%esi),%esi

77ed1c90 <_FillPath@4>:
77ed1c90:	55                   	push   %ebp
77ed1c91:	89 e5                	mov    %esp,%ebp
77ed1c93:	83 ec 10             	sub    $0x10,%esp
77ed1c96:	68 87 a3 ed 77       	push   $0x77eda387
77ed1c9b:	68 20 a0 ed 77       	push   $0x77eda020
77ed1ca0:	ff 15 e8 10 ee 77    	call   *0x77ee10e8
77ed1ca6:	c7 04 24 78 00 00 00 	movl   $0x78,(%esp)
77ed1cad:	e8 5e 7c 00 00       	call   77ed9910 <_SetLastError@4>
77ed1cb2:	31 c0                	xor    %eax,%eax
77ed1cb4:	c9                   	leave  
77ed1cb5:	c2 04 00             	ret    $0x4
77ed1cb8:	90                   	nop    
77ed1cb9:	8d b4 26 00 00 00 00 	lea    0x0(%esi),%esi

77ed1cc0 <_FlattenPath@4>:
77ed1cc0:	55                   	push   %ebp
77ed1cc1:	89 e5                	mov    %esp,%ebp
77ed1cc3:	83 ec 10             	sub    $0x10,%esp
77ed1cc6:	68 90 a3 ed 77       	push   $0x77eda390
77ed1ccb:	68 20 a0 ed 77       	push   $0x77eda020
77ed1cd0:	ff 15 e8 10 ee 77    	call   *0x77ee10e8
77ed1cd6:	c7 04 24 78 00 00 00 	movl   $0x78,(%esp)
77ed1cdd:	e8 2e 7c 00 00       	call   77ed9910 <_SetLastError@4>
77ed1ce2:	31 c0                	xor    %eax,%eax
77ed1ce4:	c9                   	leave  
77ed1ce5:	c2 04 00             	ret    $0x4
77ed1ce8:	90                   	nop    
77ed1ce9:	8d b4 26 00 00 00 00 	lea    0x0(%esi),%esi

77ed1cf0 <_GetPath@16>:
77ed1cf0:	55                   	push   %ebp
77ed1cf1:	89 e5                	mov    %esp,%ebp
77ed1cf3:	83 ec 10             	sub    $0x10,%esp
77ed1cf6:	68 9c a3 ed 77       	push   $0x77eda39c
77ed1cfb:	68 20 a0 ed 77       	push   $0x77eda020
77ed1d00:	ff 15 e8 10 ee 77    	call   *0x77ee10e8
77ed1d06:	c7 04 24 78 00 00 00 	movl   $0x78,(%esp)
77ed1d0d:	e8 fe 7b 00 00       	call   77ed9910 <_SetLastError@4>
77ed1d12:	31 c0                	xor    %eax,%eax
77ed1d14:	c9                   	leave  
77ed1d15:	c2 10 00             	ret    $0x10
77ed1d18:	90                   	nop    
77ed1d19:	8d b4 26 00 00 00 00 	lea    0x0(%esi),%esi

77ed1d20 <_PathToRegion@4>:
77ed1d20:	55                   	push   %ebp
77ed1d21:	89 e5                	mov    %esp,%ebp
77ed1d23:	83 ec 10             	sub    $0x10,%esp
77ed1d26:	68 a4 a3 ed 77       	push   $0x77eda3a4
77ed1d2b:	68 20 a0 ed 77       	push   $0x77eda020
77ed1d30:	ff 15 e8 10 ee 77    	call   *0x77ee10e8
77ed1d36:	c7 04 24 78 00 00 00 	movl   $0x78,(%esp)
77ed1d3d:	e8 ce 7b 00 00       	call   77ed9910 <_SetLastError@4>
77ed1d42:	31 c0                	xor    %eax,%eax
77ed1d44:	c9                   	leave  
77ed1d45:	c2 04 00             	ret    $0x4
77ed1d48:	90                   	nop    
77ed1d49:	8d b4 26 00 00 00 00 	lea    0x0(%esi),%esi

77ed1d50 <_PolyDraw@16>:
77ed1d50:	55                   	push   %ebp
77ed1d51:	89 e5                	mov    %esp,%ebp
77ed1d53:	83 ec 10             	sub    $0x10,%esp
77ed1d56:	68 b1 a3 ed 77       	push   $0x77eda3b1
77ed1d5b:	68 20 a0 ed 77       	push   $0x77eda020
77ed1d60:	ff 15 e8 10 ee 77    	call   *0x77ee10e8
77ed1d66:	c7 04 24 78 00 00 00 	movl   $0x78,(%esp)
77ed1d6d:	e8 9e 7b 00 00       	call   77ed9910 <_SetLastError@4>
77ed1d72:	31 c0                	xor    %eax,%eax
77ed1d74:	c9                   	leave  
77ed1d75:	c2 10 00             	ret    $0x10
77ed1d78:	90                   	nop    
77ed1d79:	8d b4 26 00 00 00 00 	lea    0x0(%esi),%esi

77ed1d80 <_SelectClipPath@8>:
77ed1d80:	55                   	push   %ebp
77ed1d81:	89 e5                	mov    %esp,%ebp
77ed1d83:	83 ec 10             	sub    $0x10,%esp
77ed1d86:	68 ba a3 ed 77       	push   $0x77eda3ba
77ed1d8b:	68 20 a0 ed 77       	push   $0x77eda020
77ed1d90:	ff 15 e8 10 ee 77    	call   *0x77ee10e8
77ed1d96:	c7 04 24 78 00 00 00 	movl   $0x78,(%esp)
77ed1d9d:	e8 6e 7b 00 00       	call   77ed9910 <_SetLastError@4>
77ed1da2:	31 c0                	xor    %eax,%eax
77ed1da4:	c9                   	leave  
77ed1da5:	c2 08 00             	ret    $0x8
77ed1da8:	90                   	nop    
77ed1da9:	8d b4 26 00 00 00 00 	lea    0x0(%esi),%esi

77ed1db0 <_SetMiterLimit@12>:
77ed1db0:	55                   	push   %ebp
77ed1db1:	89 e5                	mov    %esp,%ebp
77ed1db3:	83 ec 10             	sub    $0x10,%esp
77ed1db6:	68 c9 a3 ed 77       	push   $0x77eda3c9
77ed1dbb:	68 20 a0 ed 77       	push   $0x77eda020
77ed1dc0:	ff 15 e8 10 ee 77    	call   *0x77ee10e8
77ed1dc6:	c7 04 24 78 00 00 00 	movl   $0x78,(%esp)
77ed1dcd:	e8 3e 7b 00 00       	call   77ed9910 <_SetLastError@4>
77ed1dd2:	31 c0                	xor    %eax,%eax
77ed1dd4:	c9                   	leave  
77ed1dd5:	c2 0c 00             	ret    $0xc
77ed1dd8:	90                   	nop    
77ed1dd9:	8d b4 26 00 00 00 00 	lea    0x0(%esi),%esi

77ed1de0 <_StrokeAndFillPath@4>:
77ed1de0:	55                   	push   %ebp
77ed1de1:	89 e5                	mov    %esp,%ebp
77ed1de3:	83 ec 10             	sub    $0x10,%esp
77ed1de6:	68 d7 a3 ed 77       	push   $0x77eda3d7
77ed1deb:	68 20 a0 ed 77       	push   $0x77eda020
77ed1df0:	ff 15 e8 10 ee 77    	call   *0x77ee10e8
77ed1df6:	c7 04 24 78 00 00 00 	movl   $0x78,(%esp)
77ed1dfd:	e8 0e 7b 00 00       	call   77ed9910 <_SetLastError@4>
77ed1e02:	31 c0                	xor    %eax,%eax
77ed1e04:	c9                   	leave  
77ed1e05:	c2 04 00             	ret    $0x4
77ed1e08:	90                   	nop    
77ed1e09:	8d b4 26 00 00 00 00 	lea    0x0(%esi),%esi

77ed1e10 <_StrokePath@4>:
77ed1e10:	55                   	push   %ebp
77ed1e11:	89 e5                	mov    %esp,%ebp
77ed1e13:	83 ec 10             	sub    $0x10,%esp
77ed1e16:	68 e9 a3 ed 77       	push   $0x77eda3e9
77ed1e1b:	68 20 a0 ed 77       	push   $0x77eda020
77ed1e20:	ff 15 e8 10 ee 77    	call   *0x77ee10e8
77ed1e26:	c7 04 24 78 00 00 00 	movl   $0x78,(%esp)
77ed1e2d:	e8 de 7a 00 00       	call   77ed9910 <_SetLastError@4>
77ed1e32:	31 c0                	xor    %eax,%eax
77ed1e34:	c9                   	leave  
77ed1e35:	c2 04 00             	ret    $0x4
77ed1e38:	90                   	nop    
77ed1e39:	8d b4 26 00 00 00 00 	lea    0x0(%esi),%esi

77ed1e40 <_WidenPath@4>:
77ed1e40:	55                   	push   %ebp
77ed1e41:	89 e5                	mov    %esp,%ebp
77ed1e43:	83 ec 10             	sub    $0x10,%esp
77ed1e46:	68 f4 a3 ed 77       	push   $0x77eda3f4
77ed1e4b:	68 20 a0 ed 77       	push   $0x77eda020
77ed1e50:	ff 15 e8 10 ee 77    	call   *0x77ee10e8
77ed1e56:	c7 04 24 78 00 00 00 	movl   $0x78,(%esp)
77ed1e5d:	e8 ae 7a 00 00       	call   77ed9910 <_SetLastError@4>
77ed1e62:	31 c0                	xor    %eax,%eax
77ed1e64:	c9                   	leave  
77ed1e65:	c2 04 00             	ret    $0x4
77ed1e68:	90                   	nop    
77ed1e69:	8d b4 26 00 00 00 00 	lea    0x0(%esi),%esi

77ed1e70 <_GetMiterLimit@8>:
77ed1e70:	55                   	push   %ebp
77ed1e71:	89 e5                	mov    %esp,%ebp
77ed1e73:	83 ec 10             	sub    $0x10,%esp
77ed1e76:	68 fe a3 ed 77       	push   $0x77eda3fe
77ed1e7b:	68 20 a0 ed 77       	push   $0x77eda020
77ed1e80:	ff 15 e8 10 ee 77    	call   *0x77ee10e8
77ed1e86:	c7 04 24 78 00 00 00 	movl   $0x78,(%esp)
77ed1e8d:	e8 7e 7a 00 00       	call   77ed9910 <_SetLastError@4>
77ed1e92:	31 c0                	xor    %eax,%eax
77ed1e94:	c9                   	leave  
77ed1e95:	c2 08 00             	ret    $0x8
77ed1e98:	90                   	nop    
77ed1e99:	8d b4 26 00 00 00 00 	lea    0x0(%esi),%esi

77ed1ea0 <_ScaleViewportExtEx@24>:
77ed1ea0:	55                   	push   %ebp
77ed1ea1:	89 e5                	mov    %esp,%ebp
77ed1ea3:	83 ec 10             	sub    $0x10,%esp
77ed1ea6:	68 0c a4 ed 77       	push   $0x77eda40c
77ed1eab:	68 20 a0 ed 77       	push   $0x77eda020
77ed1eb0:	ff 15 e8 10 ee 77    	call   *0x77ee10e8
77ed1eb6:	c7 04 24 78 00 00 00 	movl   $0x78,(%esp)
77ed1ebd:	e8 4e 7a 00 00       	call   77ed9910 <_SetLastError@4>
77ed1ec2:	31 c0                	xor    %eax,%eax
77ed1ec4:	c9                   	leave  
77ed1ec5:	c2 18 00             	ret    $0x18
77ed1ec8:	90                   	nop    
77ed1ec9:	8d b4 26 00 00 00 00 	lea    0x0(%esi),%esi

77ed1ed0 <_ScaleWindowExtEx@24>:
77ed1ed0:	55                   	push   %ebp
77ed1ed1:	89 e5                	mov    %esp,%ebp
77ed1ed3:	83 ec 10             	sub    $0x10,%esp
77ed1ed6:	68 1f a4 ed 77       	push   $0x77eda41f
77ed1edb:	68 20 a0 ed 77       	push   $0x77eda020
77ed1ee0:	ff 15 e8 10 ee 77    	call   *0x77ee10e8
77ed1ee6:	c7 04 24 78 00 00 00 	movl   $0x78,(%esp)
77ed1eed:	e8 1e 7a 00 00       	call   77ed9910 <_SetLastError@4>
77ed1ef2:	31 c0                	xor    %eax,%eax
77ed1ef4:	c9                   	leave  
77ed1ef5:	c2 18 00             	ret    $0x18
77ed1ef8:	90                   	nop    
77ed1ef9:	8d b4 26 00 00 00 00 	lea    0x0(%esi),%esi

77ed1f00 <_UnrealizeObject@4>:
77ed1f00:	55                   	push   %ebp
77ed1f01:	89 e5                	mov    %esp,%ebp
77ed1f03:	83 ec 10             	sub    $0x10,%esp
77ed1f06:	68 30 a4 ed 77       	push   $0x77eda430
77ed1f0b:	68 20 a0 ed 77       	push   $0x77eda020
77ed1f10:	ff 15 e8 10 ee 77    	call   *0x77ee10e8
77ed1f16:	c7 04 24 78 00 00 00 	movl   $0x78,(%esp)
77ed1f1d:	e8 ee 79 00 00       	call   77ed9910 <_SetLastError@4>
77ed1f22:	31 c0                	xor    %eax,%eax
77ed1f24:	c9                   	leave  
77ed1f25:	c2 04 00             	ret    $0x4
77ed1f28:	90                   	nop    
77ed1f29:	8d b4 26 00 00 00 00 	lea    0x0(%esi),%esi

77ed1f30 <_GdiFlush@0>:
77ed1f30:	55                   	push   %ebp
77ed1f31:	b8 01 00 00 00       	mov    $0x1,%eax
77ed1f36:	89 e5                	mov    %esp,%ebp
77ed1f38:	5d                   	pop    %ebp
77ed1f39:	c3                   	ret    
77ed1f3a:	8d b6 00 00 00 00    	lea    0x0(%esi),%esi

77ed1f40 <_GdiSetBatchLimit@4>:
77ed1f40:	55                   	push   %ebp
77ed1f41:	89 e5                	mov    %esp,%ebp
77ed1f43:	83 ec 10             	sub    $0x10,%esp
77ed1f46:	68 40 a4 ed 77       	push   $0x77eda440
77ed1f4b:	68 20 a0 ed 77       	push   $0x77eda020
77ed1f50:	ff 15 e8 10 ee 77    	call   *0x77ee10e8
77ed1f56:	c7 04 24 78 00 00 00 	movl   $0x78,(%esp)
77ed1f5d:	e8 ae 79 00 00       	call   77ed9910 <_SetLastError@4>
77ed1f62:	31 c0                	xor    %eax,%eax
77ed1f64:	c9                   	leave  
77ed1f65:	c2 04 00             	ret    $0x4
77ed1f68:	90                   	nop    
77ed1f69:	8d b4 26 00 00 00 00 	lea    0x0(%esi),%esi

77ed1f70 <_GdiGetBatchLimit@0>:
77ed1f70:	55                   	push   %ebp
77ed1f71:	89 e5                	mov    %esp,%ebp
77ed1f73:	83 ec 10             	sub    $0x10,%esp
77ed1f76:	68 51 a4 ed 77       	push   $0x77eda451
77ed1f7b:	68 20 a0 ed 77       	push   $0x77eda020
77ed1f80:	ff 15 e8 10 ee 77    	call   *0x77ee10e8
77ed1f86:	c7 04 24 78 00 00 00 	movl   $0x78,(%esp)
77ed1f8d:	e8 7e 79 00 00       	call   77ed9910 <_SetLastError@4>
77ed1f92:	31 c0                	xor    %eax,%eax
77ed1f94:	c9                   	leave  
77ed1f95:	c3                   	ret    
77ed1f96:	8d 76 00             	lea    0x0(%esi),%esi
77ed1f99:	8d bc 27 00 00 00 00 	lea    0x0(%edi),%edi

77ed1fa0 <_SetICMMode@8>:
77ed1fa0:	55                   	push   %ebp
77ed1fa1:	89 e5                	mov    %esp,%ebp
77ed1fa3:	83 ec 10             	sub    $0x10,%esp
77ed1fa6:	68 62 a4 ed 77       	push   $0x77eda462
77ed1fab:	68 20 a0 ed 77       	push   $0x77eda020
77ed1fb0:	ff 15 e8 10 ee 77    	call   *0x77ee10e8
77ed1fb6:	c7 04 24 78 00 00 00 	movl   $0x78,(%esp)
77ed1fbd:	e8 4e 79 00 00       	call   77ed9910 <_SetLastError@4>
77ed1fc2:	31 c0                	xor    %eax,%eax
77ed1fc4:	c9                   	leave  
77ed1fc5:	c2 08 00             	ret    $0x8
77ed1fc8:	90                   	nop    
77ed1fc9:	8d b4 26 00 00 00 00 	lea    0x0(%esi),%esi

77ed1fd0 <_CheckColorsInGamut@16>:
77ed1fd0:	55                   	push   %ebp
77ed1fd1:	89 e5                	mov    %esp,%ebp
77ed1fd3:	83 ec 10             	sub    $0x10,%esp
77ed1fd6:	68 6d a4 ed 77       	push   $0x77eda46d
77ed1fdb:	68 20 a0 ed 77       	push   $0x77eda020
77ed1fe0:	ff 15 e8 10 ee 77    	call   *0x77ee10e8
77ed1fe6:	c7 04 24 78 00 00 00 	movl   $0x78,(%esp)
77ed1fed:	e8 1e 79 00 00       	call   77ed9910 <_SetLastError@4>
77ed1ff2:	31 c0                	xor    %eax,%eax
77ed1ff4:	c9                   	leave  
77ed1ff5:	c2 10 00             	ret    $0x10
77ed1ff8:	90                   	nop    
77ed1ff9:	8d b4 26 00 00 00 00 	lea    0x0(%esi),%esi

77ed2000 <_GetColorSpace@4>:
77ed2000:	55                   	push   %ebp
77ed2001:	89 e5                	mov    %esp,%ebp
77ed2003:	83 ec 10             	sub    $0x10,%esp
77ed2006:	68 80 a4 ed 77       	push   $0x77eda480
77ed200b:	68 20 a0 ed 77       	push   $0x77eda020
77ed2010:	ff 15 e8 10 ee 77    	call   *0x77ee10e8
77ed2016:	c7 04 24 78 00 00 00 	movl   $0x78,(%esp)
77ed201d:	e8 ee 78 00 00       	call   77ed9910 <_SetLastError@4>
77ed2022:	31 c0                	xor    %eax,%eax
77ed2024:	c9                   	leave  
77ed2025:	c2 04 00             	ret    $0x4
77ed2028:	90                   	nop    
77ed2029:	8d b4 26 00 00 00 00 	lea    0x0(%esi),%esi

77ed2030 <_SetColorSpace@8>:
77ed2030:	55                   	push   %ebp
77ed2031:	89 e5                	mov    %esp,%ebp
77ed2033:	83 ec 10             	sub    $0x10,%esp
77ed2036:	68 8e a4 ed 77       	push   $0x77eda48e
77ed203b:	68 20 a0 ed 77       	push   $0x77eda020
77ed2040:	ff 15 e8 10 ee 77    	call   *0x77ee10e8
77ed2046:	c7 04 24 78 00 00 00 	movl   $0x78,(%esp)
77ed204d:	e8 be 78 00 00       	call   77ed9910 <_SetLastError@4>
77ed2052:	31 c0                	xor    %eax,%eax
77ed2054:	c9                   	leave  
77ed2055:	c2 08 00             	ret    $0x8
77ed2058:	90                   	nop    
77ed2059:	8d b4 26 00 00 00 00 	lea    0x0(%esi),%esi

77ed2060 <_DeleteColorSpace@4>:
77ed2060:	55                   	push   %ebp
77ed2061:	89 e5                	mov    %esp,%ebp
77ed2063:	83 ec 10             	sub    $0x10,%esp
77ed2066:	68 9c a4 ed 77       	push   $0x77eda49c
77ed206b:	68 20 a0 ed 77       	push   $0x77eda020
77ed2070:	ff 15 e8 10 ee 77    	call   *0x77ee10e8
77ed2076:	c7 04 24 78 00 00 00 	movl   $0x78,(%esp)
77ed207d:	e8 8e 78 00 00       	call   77ed9910 <_SetLastError@4>
77ed2082:	31 c0                	xor    %eax,%eax
77ed2084:	c9                   	leave  
77ed2085:	c2 04 00             	ret    $0x4
77ed2088:	90                   	nop    
77ed2089:	8d b4 26 00 00 00 00 	lea    0x0(%esi),%esi

77ed2090 <_GetDeviceGammaRamp@8>:
77ed2090:	55                   	push   %ebp
77ed2091:	89 e5                	mov    %esp,%ebp
77ed2093:	83 ec 10             	sub    $0x10,%esp
77ed2096:	68 ad a4 ed 77       	push   $0x77eda4ad
77ed209b:	68 20 a0 ed 77       	push   $0x77eda020
77ed20a0:	ff 15 e8 10 ee 77    	call   *0x77ee10e8
77ed20a6:	c7 04 24 78 00 00 00 	movl   $0x78,(%esp)
77ed20ad:	e8 5e 78 00 00       	call   77ed9910 <_SetLastError@4>
77ed20b2:	31 c0                	xor    %eax,%eax
77ed20b4:	c9                   	leave  
77ed20b5:	c2 08 00             	ret    $0x8
77ed20b8:	90                   	nop    
77ed20b9:	8d b4 26 00 00 00 00 	lea    0x0(%esi),%esi

77ed20c0 <_SetDeviceGammaRamp@8>:
77ed20c0:	55                   	push   %ebp
77ed20c1:	89 e5                	mov    %esp,%ebp
77ed20c3:	83 ec 10             	sub    $0x10,%esp
77ed20c6:	68 c0 a4 ed 77       	push   $0x77eda4c0
77ed20cb:	68 20 a0 ed 77       	push   $0x77eda020
77ed20d0:	ff 15 e8 10 ee 77    	call   *0x77ee10e8
77ed20d6:	c7 04 24 78 00 00 00 	movl   $0x78,(%esp)
77ed20dd:	e8 2e 78 00 00       	call   77ed9910 <_SetLastError@4>
77ed20e2:	31 c0                	xor    %eax,%eax
77ed20e4:	c9                   	leave  
77ed20e5:	c2 08 00             	ret    $0x8
77ed20e8:	90                   	nop    
77ed20e9:	8d b4 26 00 00 00 00 	lea    0x0(%esi),%esi

77ed20f0 <_ColorMatchToTarget@12>:
77ed20f0:	55                   	push   %ebp
77ed20f1:	89 e5                	mov    %esp,%ebp
77ed20f3:	83 ec 10             	sub    $0x10,%esp
77ed20f6:	68 d3 a4 ed 77       	push   $0x77eda4d3
77ed20fb:	68 20 a0 ed 77       	push   $0x77eda020
77ed2100:	ff 15 e8 10 ee 77    	call   *0x77ee10e8
77ed2106:	c7 04 24 78 00 00 00 	movl   $0x78,(%esp)
77ed210d:	e8 fe 77 00 00       	call   77ed9910 <_SetLastError@4>
77ed2112:	31 c0                	xor    %eax,%eax
77ed2114:	c9                   	leave  
77ed2115:	c2 0c 00             	ret    $0xc
77ed2118:	90                   	nop    
77ed2119:	8d b4 26 00 00 00 00 	lea    0x0(%esi),%esi

77ed2120 <_wglCopyContext@12>:
77ed2120:	55                   	push   %ebp
77ed2121:	89 e5                	mov    %esp,%ebp
77ed2123:	83 ec 10             	sub    $0x10,%esp
77ed2126:	68 e6 a4 ed 77       	push   $0x77eda4e6
77ed212b:	68 20 a0 ed 77       	push   $0x77eda020
77ed2130:	ff 15 e8 10 ee 77    	call   *0x77ee10e8
77ed2136:	c7 04 24 78 00 00 00 	movl   $0x78,(%esp)
77ed213d:	e8 ce 77 00 00       	call   77ed9910 <_SetLastError@4>
77ed2142:	31 c0                	xor    %eax,%eax
77ed2144:	c9                   	leave  
77ed2145:	c2 0c 00             	ret    $0xc
77ed2148:	90                   	nop    
77ed2149:	8d b4 26 00 00 00 00 	lea    0x0(%esi),%esi

77ed2150 <_wglCreateContext@4>:
77ed2150:	55                   	push   %ebp
77ed2151:	89 e5                	mov    %esp,%ebp
77ed2153:	83 ec 10             	sub    $0x10,%esp
77ed2156:	68 f5 a4 ed 77       	push   $0x77eda4f5
77ed215b:	68 20 a0 ed 77       	push   $0x77eda020
77ed2160:	ff 15 e8 10 ee 77    	call   *0x77ee10e8
77ed2166:	c7 04 24 78 00 00 00 	movl   $0x78,(%esp)
77ed216d:	e8 9e 77 00 00       	call   77ed9910 <_SetLastError@4>
77ed2172:	31 c0                	xor    %eax,%eax
77ed2174:	c9                   	leave  
77ed2175:	c2 04 00             	ret    $0x4
77ed2178:	90                   	nop    
77ed2179:	8d b4 26 00 00 00 00 	lea    0x0(%esi),%esi

77ed2180 <_wglCreateLayerContext@8>:
77ed2180:	55                   	push   %ebp
77ed2181:	89 e5                	mov    %esp,%ebp
77ed2183:	83 ec 10             	sub    $0x10,%esp
77ed2186:	68 06 a5 ed 77       	push   $0x77eda506
77ed218b:	68 20 a0 ed 77       	push   $0x77eda020
77ed2190:	ff 15 e8 10 ee 77    	call   *0x77ee10e8
77ed2196:	c7 04 24 78 00 00 00 	movl   $0x78,(%esp)
77ed219d:	e8 6e 77 00 00       	call   77ed9910 <_SetLastError@4>
77ed21a2:	31 c0                	xor    %eax,%eax
77ed21a4:	c9                   	leave  
77ed21a5:	c2 08 00             	ret    $0x8
77ed21a8:	90                   	nop    
77ed21a9:	8d b4 26 00 00 00 00 	lea    0x0(%esi),%esi

77ed21b0 <_wglDeleteContext@4>:
77ed21b0:	55                   	push   %ebp
77ed21b1:	89 e5                	mov    %esp,%ebp
77ed21b3:	83 ec 10             	sub    $0x10,%esp
77ed21b6:	68 1c a5 ed 77       	push   $0x77eda51c
77ed21bb:	68 20 a0 ed 77       	push   $0x77eda020
77ed21c0:	ff 15 e8 10 ee 77    	call   *0x77ee10e8
77ed21c6:	c7 04 24 78 00 00 00 	movl   $0x78,(%esp)
77ed21cd:	e8 3e 77 00 00       	call   77ed9910 <_SetLastError@4>
77ed21d2:	31 c0                	xor    %eax,%eax
77ed21d4:	c9                   	leave  
77ed21d5:	c2 04 00             	ret    $0x4
77ed21d8:	90                   	nop    
77ed21d9:	8d b4 26 00 00 00 00 	lea    0x0(%esi),%esi

77ed21e0 <_wglGetCurrentContext@0>:
77ed21e0:	55                   	push   %ebp
77ed21e1:	89 e5                	mov    %esp,%ebp
77ed21e3:	83 ec 10             	sub    $0x10,%esp
77ed21e6:	68 2d a5 ed 77       	push   $0x77eda52d
77ed21eb:	68 20 a0 ed 77       	push   $0x77eda020
77ed21f0:	ff 15 e8 10 ee 77    	call   *0x77ee10e8
77ed21f6:	c7 04 24 78 00 00 00 	movl   $0x78,(%esp)
77ed21fd:	e8 0e 77 00 00       	call   77ed9910 <_SetLastError@4>
77ed2202:	31 c0                	xor    %eax,%eax
77ed2204:	c9                   	leave  
77ed2205:	c3                   	ret    
77ed2206:	8d 76 00             	lea    0x0(%esi),%esi
77ed2209:	8d bc 27 00 00 00 00 	lea    0x0(%edi),%edi

77ed2210 <_wglGetCurrentDC@0>:
77ed2210:	55                   	push   %ebp
77ed2211:	89 e5                	mov    %esp,%ebp
77ed2213:	83 ec 10             	sub    $0x10,%esp
77ed2216:	68 42 a5 ed 77       	push   $0x77eda542
77ed221b:	68 20 a0 ed 77       	push   $0x77eda020
77ed2220:	ff 15 e8 10 ee 77    	call   *0x77ee10e8
77ed2226:	c7 04 24 78 00 00 00 	movl   $0x78,(%esp)
77ed222d:	e8 de 76 00 00       	call   77ed9910 <_SetLastError@4>
77ed2232:	31 c0                	xor    %eax,%eax
77ed2234:	c9                   	leave  
77ed2235:	c3                   	ret    
77ed2236:	8d 76 00             	lea    0x0(%esi),%esi
77ed2239:	8d bc 27 00 00 00 00 	lea    0x0(%edi),%edi

77ed2240 <_wglGetProcAddress@4>:
77ed2240:	55                   	push   %ebp
77ed2241:	89 e5                	mov    %esp,%ebp
77ed2243:	83 ec 10             	sub    $0x10,%esp
77ed2246:	68 52 a5 ed 77       	push   $0x77eda552
77ed224b:	68 20 a0 ed 77       	push   $0x77eda020
77ed2250:	ff 15 e8 10 ee 77    	call   *0x77ee10e8
77ed2256:	c7 04 24 78 00 00 00 	movl   $0x78,(%esp)
77ed225d:	e8 ae 76 00 00       	call   77ed9910 <_SetLastError@4>
77ed2262:	31 c0                	xor    %eax,%eax
77ed2264:	c9                   	leave  
77ed2265:	c2 04 00             	ret    $0x4
77ed2268:	90                   	nop    
77ed2269:	8d b4 26 00 00 00 00 	lea    0x0(%esi),%esi

77ed2270 <_wglMakeCurrent@8>:
77ed2270:	55                   	push   %ebp
77ed2271:	89 e5                	mov    %esp,%ebp
77ed2273:	83 ec 10             	sub    $0x10,%esp
77ed2276:	68 64 a5 ed 77       	push   $0x77eda564
77ed227b:	68 20 a0 ed 77       	push   $0x77eda020
77ed2280:	ff 15 e8 10 ee 77    	call   *0x77ee10e8
77ed2286:	c7 04 24 78 00 00 00 	movl   $0x78,(%esp)
77ed228d:	e8 7e 76 00 00       	call   77ed9910 <_SetLastError@4>
77ed2292:	31 c0                	xor    %eax,%eax
77ed2294:	c9                   	leave  
77ed2295:	c2 08 00             	ret    $0x8
77ed2298:	90                   	nop    
77ed2299:	8d b4 26 00 00 00 00 	lea    0x0(%esi),%esi

77ed22a0 <_wglShareLists@8>:
77ed22a0:	55                   	push   %ebp
77ed22a1:	89 e5                	mov    %esp,%ebp
77ed22a3:	83 ec 10             	sub    $0x10,%esp
77ed22a6:	68 73 a5 ed 77       	push   $0x77eda573
77ed22ab:	68 20 a0 ed 77       	push   $0x77eda020
77ed22b0:	ff 15 e8 10 ee 77    	call   *0x77ee10e8
77ed22b6:	c7 04 24 78 00 00 00 	movl   $0x78,(%esp)
77ed22bd:	e8 4e 76 00 00       	call   77ed9910 <_SetLastError@4>
77ed22c2:	31 c0                	xor    %eax,%eax
77ed22c4:	c9                   	leave  
77ed22c5:	c2 08 00             	ret    $0x8
77ed22c8:	90                   	nop    
77ed22c9:	8d b4 26 00 00 00 00 	lea    0x0(%esi),%esi

77ed22d0 <_wglDescribeLayerPlane@20>:
77ed22d0:	55                   	push   %ebp
77ed22d1:	89 e5                	mov    %esp,%ebp
77ed22d3:	83 ec 10             	sub    $0x10,%esp
77ed22d6:	68 81 a5 ed 77       	push   $0x77eda581
77ed22db:	68 20 a0 ed 77       	push   $0x77eda020
77ed22e0:	ff 15 e8 10 ee 77    	call   *0x77ee10e8
77ed22e6:	c7 04 24 78 00 00 00 	movl   $0x78,(%esp)
77ed22ed:	e8 1e 76 00 00       	call   77ed9910 <_SetLastError@4>
77ed22f2:	31 c0                	xor    %eax,%eax
77ed22f4:	c9                   	leave  
77ed22f5:	c2 14 00             	ret    $0x14
77ed22f8:	90                   	nop    
77ed22f9:	8d b4 26 00 00 00 00 	lea    0x0(%esi),%esi

77ed2300 <_wglSetLayerPaletteEntries@20>:
77ed2300:	55                   	push   %ebp
77ed2301:	89 e5                	mov    %esp,%ebp
77ed2303:	83 ec 10             	sub    $0x10,%esp
77ed2306:	68 97 a5 ed 77       	push   $0x77eda597
77ed230b:	68 20 a0 ed 77       	push   $0x77eda020
77ed2310:	ff 15 e8 10 ee 77    	call   *0x77ee10e8
77ed2316:	c7 04 24 78 00 00 00 	movl   $0x78,(%esp)
77ed231d:	e8 ee 75 00 00       	call   77ed9910 <_SetLastError@4>
77ed2322:	31 c0                	xor    %eax,%eax
77ed2324:	c9                   	leave  
77ed2325:	c2 14 00             	ret    $0x14
77ed2328:	90                   	nop    
77ed2329:	8d b4 26 00 00 00 00 	lea    0x0(%esi),%esi

77ed2330 <_wglGetLayerPaletteEntries@20>:
77ed2330:	55                   	push   %ebp
77ed2331:	89 e5                	mov    %esp,%ebp
77ed2333:	83 ec 10             	sub    $0x10,%esp
77ed2336:	68 b1 a5 ed 77       	push   $0x77eda5b1
77ed233b:	68 20 a0 ed 77       	push   $0x77eda020
77ed2340:	ff 15 e8 10 ee 77    	call   *0x77ee10e8
77ed2346:	c7 04 24 78 00 00 00 	movl   $0x78,(%esp)
77ed234d:	e8 be 75 00 00       	call   77ed9910 <_SetLastError@4>
77ed2352:	31 c0                	xor    %eax,%eax
77ed2354:	c9                   	leave  
77ed2355:	c2 14 00             	ret    $0x14
77ed2358:	90                   	nop    
77ed2359:	8d b4 26 00 00 00 00 	lea    0x0(%esi),%esi

77ed2360 <_wglRealizeLayerPalette@12>:
77ed2360:	55                   	push   %ebp
77ed2361:	89 e5                	mov    %esp,%ebp
77ed2363:	83 ec 10             	sub    $0x10,%esp
77ed2366:	68 cb a5 ed 77       	push   $0x77eda5cb
77ed236b:	68 20 a0 ed 77       	push   $0x77eda020
77ed2370:	ff 15 e8 10 ee 77    	call   *0x77ee10e8
77ed2376:	c7 04 24 78 00 00 00 	movl   $0x78,(%esp)
77ed237d:	e8 8e 75 00 00       	call   77ed9910 <_SetLastError@4>
77ed2382:	31 c0                	xor    %eax,%eax
77ed2384:	c9                   	leave  
77ed2385:	c2 0c 00             	ret    $0xc
77ed2388:	90                   	nop    
77ed2389:	8d b4 26 00 00 00 00 	lea    0x0(%esi),%esi

77ed2390 <_wglSwapLayerBuffers@8>:
77ed2390:	55                   	push   %ebp
77ed2391:	89 e5                	mov    %esp,%ebp
77ed2393:	83 ec 10             	sub    $0x10,%esp
77ed2396:	68 e2 a5 ed 77       	push   $0x77eda5e2
77ed239b:	68 20 a0 ed 77       	push   $0x77eda020
77ed23a0:	ff 15 e8 10 ee 77    	call   *0x77ee10e8
77ed23a6:	c7 04 24 78 00 00 00 	movl   $0x78,(%esp)
77ed23ad:	e8 5e 75 00 00       	call   77ed9910 <_SetLastError@4>
77ed23b2:	31 c0                	xor    %eax,%eax
77ed23b4:	c9                   	leave  
77ed23b5:	c2 08 00             	ret    $0x8
77ed23b8:	90                   	nop    
77ed23b9:	8d b4 26 00 00 00 00 	lea    0x0(%esi),%esi

77ed23c0 <_GdiPlayDCScript@24>:
77ed23c0:	55                   	push   %ebp
77ed23c1:	89 e5                	mov    %esp,%ebp
77ed23c3:	83 ec 10             	sub    $0x10,%esp
77ed23c6:	68 f6 a5 ed 77       	push   $0x77eda5f6
77ed23cb:	68 20 a0 ed 77       	push   $0x77eda020
77ed23d0:	ff 15 e8 10 ee 77    	call   *0x77ee10e8
77ed23d6:	c7 04 24 78 00 00 00 	movl   $0x78,(%esp)
77ed23dd:	e8 2e 75 00 00       	call   77ed9910 <_SetLastError@4>
77ed23e2:	31 c0                	xor    %eax,%eax
77ed23e4:	c9                   	leave  
77ed23e5:	c2 18 00             	ret    $0x18
77ed23e8:	90                   	nop    
77ed23e9:	8d b4 26 00 00 00 00 	lea    0x0(%esi),%esi

77ed23f0 <_GdiPlayJournal@20>:
77ed23f0:	55                   	push   %ebp
77ed23f1:	89 e5                	mov    %esp,%ebp
77ed23f3:	83 ec 10             	sub    $0x10,%esp
77ed23f6:	68 06 a6 ed 77       	push   $0x77eda606
77ed23fb:	68 20 a0 ed 77       	push   $0x77eda020
77ed2400:	ff 15 e8 10 ee 77    	call   *0x77ee10e8
77ed2406:	c7 04 24 78 00 00 00 	movl   $0x78,(%esp)
77ed240d:	e8 fe 74 00 00       	call   77ed9910 <_SetLastError@4>
77ed2412:	31 c0                	xor    %eax,%eax
77ed2414:	c9                   	leave  
77ed2415:	c2 14 00             	ret    $0x14
77ed2418:	90                   	nop    
77ed2419:	8d b4 26 00 00 00 00 	lea    0x0(%esi),%esi

77ed2420 <_GdiPlayScript@28>:
77ed2420:	55                   	push   %ebp
77ed2421:	89 e5                	mov    %esp,%ebp
77ed2423:	83 ec 10             	sub    $0x10,%esp
77ed2426:	68 15 a6 ed 77       	push   $0x77eda615
77ed242b:	68 20 a0 ed 77       	push   $0x77eda020
77ed2430:	ff 15 e8 10 ee 77    	call   *0x77ee10e8
77ed2436:	c7 04 24 78 00 00 00 	movl   $0x78,(%esp)
77ed243d:	e8 ce 74 00 00       	call   77ed9910 <_SetLastError@4>
77ed2442:	31 c0                	xor    %eax,%eax
77ed2444:	c9                   	leave  
77ed2445:	c2 1c 00             	ret    $0x1c
77ed2448:	90                   	nop    
77ed2449:	8d b4 26 00 00 00 00 	lea    0x0(%esi),%esi

77ed2450 <_GetGlyphOutlineWow@28>:
77ed2450:	55                   	push   %ebp
77ed2451:	89 e5                	mov    %esp,%ebp
77ed2453:	83 ec 10             	sub    $0x10,%esp
77ed2456:	68 23 a6 ed 77       	push   $0x77eda623
77ed245b:	68 20 a0 ed 77       	push   $0x77eda020
77ed2460:	ff 15 e8 10 ee 77    	call   *0x77ee10e8
77ed2466:	c7 04 24 78 00 00 00 	movl   $0x78,(%esp)
77ed246d:	e8 9e 74 00 00       	call   77ed9910 <_SetLastError@4>
77ed2472:	31 c0                	xor    %eax,%eax
77ed2474:	c9                   	leave  
77ed2475:	c2 1c 00             	ret    $0x1c
77ed2478:	90                   	nop    
77ed2479:	8d b4 26 00 00 00 00 	lea    0x0(%esi),%esi

77ed2480 <_GetRandomRgn@12>:
77ed2480:	55                   	push   %ebp
77ed2481:	89 e5                	mov    %esp,%ebp
77ed2483:	83 ec 10             	sub    $0x10,%esp
77ed2486:	68 36 a6 ed 77       	push   $0x77eda636
77ed248b:	68 20 a0 ed 77       	push   $0x77eda020
77ed2490:	ff 15 e8 10 ee 77    	call   *0x77ee10e8
77ed2496:	c7 04 24 78 00 00 00 	movl   $0x78,(%esp)
77ed249d:	e8 6e 74 00 00       	call   77ed9910 <_SetLastError@4>
77ed24a2:	31 c0                	xor    %eax,%eax
77ed24a4:	c9                   	leave  
77ed24a5:	c2 0c 00             	ret    $0xc
77ed24a8:	90                   	nop    
77ed24a9:	8d b4 26 00 00 00 00 	lea    0x0(%esi),%esi

77ed24b0 <_SelectBrushLocal@8>:
77ed24b0:	55                   	push   %ebp
77ed24b1:	89 e5                	mov    %esp,%ebp
77ed24b3:	83 ec 10             	sub    $0x10,%esp
77ed24b6:	68 43 a6 ed 77       	push   $0x77eda643
77ed24bb:	68 20 a0 ed 77       	push   $0x77eda020
77ed24c0:	ff 15 e8 10 ee 77    	call   *0x77ee10e8
77ed24c6:	c7 04 24 78 00 00 00 	movl   $0x78,(%esp)
77ed24cd:	e8 3e 74 00 00       	call   77ed9910 <_SetLastError@4>
77ed24d2:	31 c0                	xor    %eax,%eax
77ed24d4:	c9                   	leave  
77ed24d5:	c2 08 00             	ret    $0x8
77ed24d8:	90                   	nop    
77ed24d9:	8d b4 26 00 00 00 00 	lea    0x0(%esi),%esi

77ed24e0 <_SelectFontLocal@8>:
77ed24e0:	55                   	push   %ebp
77ed24e1:	89 e5                	mov    %esp,%ebp
77ed24e3:	83 ec 10             	sub    $0x10,%esp
77ed24e6:	68 54 a6 ed 77       	push   $0x77eda654
77ed24eb:	68 20 a0 ed 77       	push   $0x77eda020
77ed24f0:	ff 15 e8 10 ee 77    	call   *0x77ee10e8
77ed24f6:	c7 04 24 78 00 00 00 	movl   $0x78,(%esp)
77ed24fd:	e8 0e 74 00 00       	call   77ed9910 <_SetLastError@4>
77ed2502:	31 c0                	xor    %eax,%eax
77ed2504:	c9                   	leave  
77ed2505:	c2 08 00             	ret    $0x8
77ed2508:	90                   	nop    
77ed2509:	8d b4 26 00 00 00 00 	lea    0x0(%esi),%esi

77ed2510 <_SetFontEnumeration@4>:
77ed2510:	55                   	push   %ebp
77ed2511:	89 e5                	mov    %esp,%ebp
77ed2513:	83 ec 10             	sub    $0x10,%esp
77ed2516:	68 64 a6 ed 77       	push   $0x77eda664
77ed251b:	68 20 a0 ed 77       	push   $0x77eda020
77ed2520:	ff 15 e8 10 ee 77    	call   *0x77ee10e8
77ed2526:	c7 04 24 78 00 00 00 	movl   $0x78,(%esp)
77ed252d:	e8 de 73 00 00       	call   77ed9910 <_SetLastError@4>
77ed2532:	31 c0                	xor    %eax,%eax
77ed2534:	c9                   	leave  
77ed2535:	c2 04 00             	ret    $0x4
77ed2538:	90                   	nop    
77ed2539:	8d b4 26 00 00 00 00 	lea    0x0(%esi),%esi

77ed2540 <_SetRelAbs@8>:
77ed2540:	55                   	push   %ebp
77ed2541:	89 e5                	mov    %esp,%ebp
77ed2543:	83 ec 10             	sub    $0x10,%esp
77ed2546:	68 77 a6 ed 77       	push   $0x77eda677
77ed254b:	68 20 a0 ed 77       	push   $0x77eda020
77ed2550:	ff 15 e8 10 ee 77    	call   *0x77ee10e8
77ed2556:	c7 04 24 78 00 00 00 	movl   $0x78,(%esp)
77ed255d:	e8 ae 73 00 00       	call   77ed9910 <_SetLastError@4>
77ed2562:	31 c0                	xor    %eax,%eax
77ed2564:	c9                   	leave  
77ed2565:	c2 08 00             	ret    $0x8
77ed2568:	90                   	nop    
77ed2569:	8d b4 26 00 00 00 00 	lea    0x0(%esi),%esi

77ed2570 <_gdiPlaySpoolStream@24>:
77ed2570:	55                   	push   %ebp
77ed2571:	89 e5                	mov    %esp,%ebp
77ed2573:	83 ec 10             	sub    $0x10,%esp
77ed2576:	68 81 a6 ed 77       	push   $0x77eda681
77ed257b:	68 20 a0 ed 77       	push   $0x77eda020
77ed2580:	ff 15 e8 10 ee 77    	call   *0x77ee10e8
77ed2586:	c7 04 24 78 00 00 00 	movl   $0x78,(%esp)
77ed258d:	e8 7e 73 00 00       	call   77ed9910 <_SetLastError@4>
77ed2592:	31 c0                	xor    %eax,%eax
77ed2594:	c9                   	leave  
77ed2595:	c2 18 00             	ret    $0x18
77ed2598:	90                   	nop    
77ed2599:	8d b4 26 00 00 00 00 	lea    0x0(%esi),%esi

77ed25a0 <_GetFontResourceInfo@16>:
77ed25a0:	55                   	push   %ebp
77ed25a1:	89 e5                	mov    %esp,%ebp
77ed25a3:	83 ec 10             	sub    $0x10,%esp
77ed25a6:	68 94 a6 ed 77       	push   $0x77eda694
77ed25ab:	68 20 a0 ed 77       	push   $0x77eda020
77ed25b0:	ff 15 e8 10 ee 77    	call   *0x77ee10e8
77ed25b6:	c7 04 24 78 00 00 00 	movl   $0x78,(%esp)
77ed25bd:	e8 4e 73 00 00       	call   77ed9910 <_SetLastError@4>
77ed25c2:	31 c0                	xor    %eax,%eax
77ed25c4:	c9                   	leave  
77ed25c5:	c2 10 00             	ret    $0x10
77ed25c8:	90                   	nop    
77ed25c9:	8d b4 26 00 00 00 00 	lea    0x0(%esi),%esi

77ed25d0 <_AddFontMemResourceEx@16>:
77ed25d0:	55                   	push   %ebp
77ed25d1:	89 e5                	mov    %esp,%ebp
77ed25d3:	83 ec 10             	sub    $0x10,%esp
77ed25d6:	68 a8 a6 ed 77       	push   $0x77eda6a8
77ed25db:	68 20 a0 ed 77       	push   $0x77eda020
77ed25e0:	ff 15 e8 10 ee 77    	call   *0x77ee10e8
77ed25e6:	c7 04 24 78 00 00 00 	movl   $0x78,(%esp)
77ed25ed:	e8 1e 73 00 00       	call   77ed9910 <_SetLastError@4>
77ed25f2:	31 c0                	xor    %eax,%eax
77ed25f4:	c9                   	leave  
77ed25f5:	c2 10 00             	ret    $0x10
77ed25f8:	90                   	nop    
77ed25f9:	8d b4 26 00 00 00 00 	lea    0x0(%esi),%esi

77ed2600 <_AddFontResourceTracking@8>:
77ed2600:	55                   	push   %ebp
77ed2601:	89 e5                	mov    %esp,%ebp
77ed2603:	83 ec 10             	sub    $0x10,%esp
77ed2606:	68 bd a6 ed 77       	push   $0x77eda6bd
77ed260b:	68 20 a0 ed 77       	push   $0x77eda020
77ed2610:	ff 15 e8 10 ee 77    	call   *0x77ee10e8
77ed2616:	c7 04 24 78 00 00 00 	movl   $0x78,(%esp)
77ed261d:	e8 ee 72 00 00       	call   77ed9910 <_SetLastError@4>
77ed2622:	31 c0                	xor    %eax,%eax
77ed2624:	c9                   	leave  
77ed2625:	c2 08 00             	ret    $0x8
77ed2628:	90                   	nop    
77ed2629:	8d b4 26 00 00 00 00 	lea    0x0(%esi),%esi

77ed2630 <_AnyLinkedFonts@0>:
77ed2630:	55                   	push   %ebp
77ed2631:	89 e5                	mov    %esp,%ebp
77ed2633:	83 ec 10             	sub    $0x10,%esp
77ed2636:	68 d5 a6 ed 77       	push   $0x77eda6d5
77ed263b:	68 20 a0 ed 77       	push   $0x77eda020
77ed2640:	ff 15 e8 10 ee 77    	call   *0x77ee10e8
77ed2646:	c7 04 24 78 00 00 00 	movl   $0x78,(%esp)
77ed264d:	e8 be 72 00 00       	call   77ed9910 <_SetLastError@4>
77ed2652:	31 c0                	xor    %eax,%eax
77ed2654:	c9                   	leave  
77ed2655:	c3                   	ret    
77ed2656:	8d 76 00             	lea    0x0(%esi),%esi
77ed2659:	8d bc 27 00 00 00 00 	lea    0x0(%edi),%edi

77ed2660 <_ClearBitmapAttributes@8>:
77ed2660:	55                   	push   %ebp
77ed2661:	89 e5                	mov    %esp,%ebp
77ed2663:	83 ec 10             	sub    $0x10,%esp
77ed2666:	68 e4 a6 ed 77       	push   $0x77eda6e4
77ed266b:	68 20 a0 ed 77       	push   $0x77eda020
77ed2670:	ff 15 e8 10 ee 77    	call   *0x77ee10e8
77ed2676:	c7 04 24 78 00 00 00 	movl   $0x78,(%esp)
77ed267d:	e8 8e 72 00 00       	call   77ed9910 <_SetLastError@4>
77ed2682:	31 c0                	xor    %eax,%eax
77ed2684:	c9                   	leave  
77ed2685:	c2 08 00             	ret    $0x8
77ed2688:	90                   	nop    
77ed2689:	8d b4 26 00 00 00 00 	lea    0x0(%esi),%esi

77ed2690 <_ClearBrushAttributes@8>:
77ed2690:	55                   	push   %ebp
77ed2691:	89 e5                	mov    %esp,%ebp
77ed2693:	83 ec 10             	sub    $0x10,%esp
77ed2696:	68 fa a6 ed 77       	push   $0x77eda6fa
77ed269b:	68 20 a0 ed 77       	push   $0x77eda020
77ed26a0:	ff 15 e8 10 ee 77    	call   *0x77ee10e8
77ed26a6:	c7 04 24 78 00 00 00 	movl   $0x78,(%esp)
77ed26ad:	e8 5e 72 00 00       	call   77ed9910 <_SetLastError@4>
77ed26b2:	31 c0                	xor    %eax,%eax
77ed26b4:	c9                   	leave  
77ed26b5:	c2 08 00             	ret    $0x8
77ed26b8:	90                   	nop    
77ed26b9:	8d b4 26 00 00 00 00 	lea    0x0(%esi),%esi

77ed26c0 <_ColorCorrectPalette@16>:
77ed26c0:	55                   	push   %ebp
77ed26c1:	89 e5                	mov    %esp,%ebp
77ed26c3:	83 ec 10             	sub    $0x10,%esp
77ed26c6:	68 0f a7 ed 77       	push   $0x77eda70f
77ed26cb:	68 20 a0 ed 77       	push   $0x77eda020
77ed26d0:	ff 15 e8 10 ee 77    	call   *0x77ee10e8
77ed26d6:	c7 04 24 78 00 00 00 	movl   $0x78,(%esp)
77ed26dd:	e8 2e 72 00 00       	call   77ed9910 <_SetLastError@4>
77ed26e2:	31 c0                	xor    %eax,%eax
77ed26e4:	c9                   	leave  
77ed26e5:	c2 10 00             	ret    $0x10
77ed26e8:	90                   	nop    
77ed26e9:	8d b4 26 00 00 00 00 	lea    0x0(%esi),%esi

77ed26f0 <_EnableEUDC@4>:
77ed26f0:	55                   	push   %ebp
77ed26f1:	89 e5                	mov    %esp,%ebp
77ed26f3:	83 ec 10             	sub    $0x10,%esp
77ed26f6:	68 23 a7 ed 77       	push   $0x77eda723
77ed26fb:	68 20 a0 ed 77       	push   $0x77eda020
77ed2700:	ff 15 e8 10 ee 77    	call   *0x77ee10e8
77ed2706:	c7 04 24 78 00 00 00 	movl   $0x78,(%esp)
77ed270d:	e8 fe 71 00 00       	call   77ed9910 <_SetLastError@4>
77ed2712:	31 c0                	xor    %eax,%eax
77ed2714:	c9                   	leave  
77ed2715:	c2 04 00             	ret    $0x4
77ed2718:	90                   	nop    
77ed2719:	8d b4 26 00 00 00 00 	lea    0x0(%esi),%esi

77ed2720 <_EndFormPage@4>:
77ed2720:	55                   	push   %ebp
77ed2721:	89 e5                	mov    %esp,%ebp
77ed2723:	83 ec 10             	sub    $0x10,%esp
77ed2726:	68 2e a7 ed 77       	push   $0x77eda72e
77ed272b:	68 20 a0 ed 77       	push   $0x77eda020
77ed2730:	ff 15 e8 10 ee 77    	call   *0x77ee10e8
77ed2736:	c7 04 24 78 00 00 00 	movl   $0x78,(%esp)
77ed273d:	e8 ce 71 00 00       	call   77ed9910 <_SetLastError@4>
77ed2742:	31 c0                	xor    %eax,%eax
77ed2744:	c9                   	leave  
77ed2745:	c2 04 00             	ret    $0x4
77ed2748:	90                   	nop    
77ed2749:	8d b4 26 00 00 00 00 	lea    0x0(%esi),%esi

77ed2750 <_FontIsLinked@4>:
77ed2750:	55                   	push   %ebp
77ed2751:	89 e5                	mov    %esp,%ebp
77ed2753:	83 ec 10             	sub    $0x10,%esp
77ed2756:	68 3a a7 ed 77       	push   $0x77eda73a
77ed275b:	68 20 a0 ed 77       	push   $0x77eda020
77ed2760:	ff 15 e8 10 ee 77    	call   *0x77ee10e8
77ed2766:	c7 04 24 78 00 00 00 	movl   $0x78,(%esp)
77ed276d:	e8 9e 71 00 00       	call   77ed9910 <_SetLastError@4>
77ed2772:	31 c0                	xor    %eax,%eax
77ed2774:	c9                   	leave  
77ed2775:	c2 04 00             	ret    $0x4
77ed2778:	90                   	nop    
77ed2779:	8d b4 26 00 00 00 00 	lea    0x0(%esi),%esi

77ed2780 <_GdiAddGlsBounds@8>:
77ed2780:	55                   	push   %ebp
77ed2781:	89 e5                	mov    %esp,%ebp
77ed2783:	83 ec 10             	sub    $0x10,%esp
77ed2786:	68 47 a7 ed 77       	push   $0x77eda747
77ed278b:	68 20 a0 ed 77       	push   $0x77eda020
77ed2790:	ff 15 e8 10 ee 77    	call   *0x77ee10e8
77ed2796:	c7 04 24 78 00 00 00 	movl   $0x78,(%esp)
77ed279d:	e8 6e 71 00 00       	call   77ed9910 <_SetLastError@4>
77ed27a2:	31 c0                	xor    %eax,%eax
77ed27a4:	c9                   	leave  
77ed27a5:	c2 08 00             	ret    $0x8
77ed27a8:	90                   	nop    
77ed27a9:	8d b4 26 00 00 00 00 	lea    0x0(%esi),%esi

77ed27b0 <_GdiAlphaBlend@44>:
77ed27b0:	55                   	push   %ebp
77ed27b1:	89 e5                	mov    %esp,%ebp
77ed27b3:	83 ec 10             	sub    $0x10,%esp
77ed27b6:	68 57 a7 ed 77       	push   $0x77eda757
77ed27bb:	68 20 a0 ed 77       	push   $0x77eda020
77ed27c0:	ff 15 e8 10 ee 77    	call   *0x77ee10e8
77ed27c6:	c7 04 24 78 00 00 00 	movl   $0x78,(%esp)
77ed27cd:	e8 3e 71 00 00       	call   77ed9910 <_SetLastError@4>
77ed27d2:	31 c0                	xor    %eax,%eax
77ed27d4:	c9                   	leave  
77ed27d5:	c2 2c 00             	ret    $0x2c
77ed27d8:	90                   	nop    
77ed27d9:	8d b4 26 00 00 00 00 	lea    0x0(%esi),%esi

77ed27e0 <_GdiArtificialDecrementDriver@8>:
77ed27e0:	55                   	push   %ebp
77ed27e1:	89 e5                	mov    %esp,%ebp
77ed27e3:	83 ec 10             	sub    $0x10,%esp
77ed27e6:	68 65 a7 ed 77       	push   $0x77eda765
77ed27eb:	68 20 a0 ed 77       	push   $0x77eda020
77ed27f0:	ff 15 e8 10 ee 77    	call   *0x77ee10e8
77ed27f6:	c7 04 24 78 00 00 00 	movl   $0x78,(%esp)
77ed27fd:	e8 0e 71 00 00       	call   77ed9910 <_SetLastError@4>
77ed2802:	31 c0                	xor    %eax,%eax
77ed2804:	c9                   	leave  
77ed2805:	c2 08 00             	ret    $0x8
77ed2808:	90                   	nop    
77ed2809:	8d b4 26 00 00 00 00 	lea    0x0(%esi),%esi

77ed2810 <_GdiCleanCacheDC@4>:
77ed2810:	55                   	push   %ebp
77ed2811:	89 e5                	mov    %esp,%ebp
77ed2813:	83 ec 10             	sub    $0x10,%esp
77ed2816:	68 82 a7 ed 77       	push   $0x77eda782
77ed281b:	68 20 a0 ed 77       	push   $0x77eda020
77ed2820:	ff 15 e8 10 ee 77    	call   *0x77ee10e8
77ed2826:	c7 04 24 78 00 00 00 	movl   $0x78,(%esp)
77ed282d:	e8 de 70 00 00       	call   77ed9910 <_SetLastError@4>
77ed2832:	31 c0                	xor    %eax,%eax
77ed2834:	c9                   	leave  
77ed2835:	c2 04 00             	ret    $0x4
77ed2838:	90                   	nop    
77ed2839:	8d b4 26 00 00 00 00 	lea    0x0(%esi),%esi

77ed2840 <_GdiConvertAndCheckDC@4>:
77ed2840:	55                   	push   %ebp
77ed2841:	89 e5                	mov    %esp,%ebp
77ed2843:	83 ec 10             	sub    $0x10,%esp
77ed2846:	68 92 a7 ed 77       	push   $0x77eda792
77ed284b:	68 20 a0 ed 77       	push   $0x77eda020
77ed2850:	ff 15 e8 10 ee 77    	call   *0x77ee10e8
77ed2856:	c7 04 24 78 00 00 00 	movl   $0x78,(%esp)
77ed285d:	e8 ae 70 00 00       	call   77ed9910 <_SetLastError@4>
77ed2862:	31 c0                	xor    %eax,%eax
77ed2864:	c9                   	leave  
77ed2865:	c2 04 00             	ret    $0x4
77ed2868:	90                   	nop    
77ed2869:	8d b4 26 00 00 00 00 	lea    0x0(%esi),%esi

77ed2870 <_GdiConvertBitmap@4>:
77ed2870:	55                   	push   %ebp
77ed2871:	89 e5                	mov    %esp,%ebp
77ed2873:	83 ec 10             	sub    $0x10,%esp
77ed2876:	68 a7 a7 ed 77       	push   $0x77eda7a7
77ed287b:	68 20 a0 ed 77       	push   $0x77eda020
77ed2880:	ff 15 e8 10 ee 77    	call   *0x77ee10e8
77ed2886:	c7 04 24 78 00 00 00 	movl   $0x78,(%esp)
77ed288d:	e8 7e 70 00 00       	call   77ed9910 <_SetLastError@4>
77ed2892:	31 c0                	xor    %eax,%eax
77ed2894:	c9                   	leave  
77ed2895:	c2 04 00             	ret    $0x4
77ed2898:	90                   	nop    
77ed2899:	8d b4 26 00 00 00 00 	lea    0x0(%esi),%esi

77ed28a0 <_GdiConvertBrush@4>:
77ed28a0:	55                   	push   %ebp
77ed28a1:	89 e5                	mov    %esp,%ebp
77ed28a3:	83 ec 10             	sub    $0x10,%esp
77ed28a6:	68 b8 a7 ed 77       	push   $0x77eda7b8
77ed28ab:	68 20 a0 ed 77       	push   $0x77eda020
77ed28b0:	ff 15 e8 10 ee 77    	call   *0x77ee10e8
77ed28b6:	c7 04 24 78 00 00 00 	movl   $0x78,(%esp)
77ed28bd:	e8 4e 70 00 00       	call   77ed9910 <_SetLastError@4>
77ed28c2:	31 c0                	xor    %eax,%eax
77ed28c4:	c9                   	leave  
77ed28c5:	c2 04 00             	ret    $0x4
77ed28c8:	90                   	nop    
77ed28c9:	8d b4 26 00 00 00 00 	lea    0x0(%esi),%esi

77ed28d0 <_GdiConvertDC@4>:
77ed28d0:	55                   	push   %ebp
77ed28d1:	89 e5                	mov    %esp,%ebp
77ed28d3:	83 ec 10             	sub    $0x10,%esp
77ed28d6:	68 c8 a7 ed 77       	push   $0x77eda7c8
77ed28db:	68 20 a0 ed 77       	push   $0x77eda020
77ed28e0:	ff 15 e8 10 ee 77    	call   *0x77ee10e8
77ed28e6:	c7 04 24 78 00 00 00 	movl   $0x78,(%esp)
77ed28ed:	e8 1e 70 00 00       	call   77ed9910 <_SetLastError@4>
77ed28f2:	31 c0                	xor    %eax,%eax
77ed28f4:	c9                   	leave  
77ed28f5:	c2 04 00             	ret    $0x4
77ed28f8:	90                   	nop    
77ed28f9:	8d b4 26 00 00 00 00 	lea    0x0(%esi),%esi

77ed2900 <_GdiConvertFont@4>:
77ed2900:	55                   	push   %ebp
77ed2901:	89 e5                	mov    %esp,%ebp
77ed2903:	83 ec 10             	sub    $0x10,%esp
77ed2906:	68 d5 a7 ed 77       	push   $0x77eda7d5
77ed290b:	68 20 a0 ed 77       	push   $0x77eda020
77ed2910:	ff 15 e8 10 ee 77    	call   *0x77ee10e8
77ed2916:	c7 04 24 78 00 00 00 	movl   $0x78,(%esp)
77ed291d:	e8 ee 6f 00 00       	call   77ed9910 <_SetLastError@4>
77ed2922:	31 c0                	xor    %eax,%eax
77ed2924:	c9                   	leave  
77ed2925:	c2 04 00             	ret    $0x4
77ed2928:	90                   	nop    
77ed2929:	8d b4 26 00 00 00 00 	lea    0x0(%esi),%esi

77ed2930 <_GdiConvertPalette@4>:
77ed2930:	55                   	push   %ebp
77ed2931:	89 e5                	mov    %esp,%ebp
77ed2933:	83 ec 10             	sub    $0x10,%esp
77ed2936:	68 e4 a7 ed 77       	push   $0x77eda7e4
77ed293b:	68 20 a0 ed 77       	push   $0x77eda020
77ed2940:	ff 15 e8 10 ee 77    	call   *0x77ee10e8
77ed2946:	c7 04 24 78 00 00 00 	movl   $0x78,(%esp)
77ed294d:	e8 be 6f 00 00       	call   77ed9910 <_SetLastError@4>
77ed2952:	31 c0                	xor    %eax,%eax
77ed2954:	c9                   	leave  
77ed2955:	c2 04 00             	ret    $0x4
77ed2958:	90                   	nop    
77ed2959:	8d b4 26 00 00 00 00 	lea    0x0(%esi),%esi

77ed2960 <_GdiConvertRegion@4>:
77ed2960:	55                   	push   %ebp
77ed2961:	89 e5                	mov    %esp,%ebp
77ed2963:	83 ec 10             	sub    $0x10,%esp
77ed2966:	68 f6 a7 ed 77       	push   $0x77eda7f6
77ed296b:	68 20 a0 ed 77       	push   $0x77eda020
77ed2970:	ff 15 e8 10 ee 77    	call   *0x77ee10e8
77ed2976:	c7 04 24 78 00 00 00 	movl   $0x78,(%esp)
77ed297d:	e8 8e 6f 00 00       	call   77ed9910 <_SetLastError@4>
77ed2982:	31 c0                	xor    %eax,%eax
77ed2984:	c9                   	leave  
77ed2985:	c2 04 00             	ret    $0x4
77ed2988:	90                   	nop    
77ed2989:	8d b4 26 00 00 00 00 	lea    0x0(%esi),%esi

77ed2990 <_GdiConvertEnhMetaFile@4>:
77ed2990:	55                   	push   %ebp
77ed2991:	89 e5                	mov    %esp,%ebp
77ed2993:	83 ec 10             	sub    $0x10,%esp
77ed2996:	68 07 a8 ed 77       	push   $0x77eda807
77ed299b:	68 20 a0 ed 77       	push   $0x77eda020
77ed29a0:	ff 15 e8 10 ee 77    	call   *0x77ee10e8
77ed29a6:	c7 04 24 78 00 00 00 	movl   $0x78,(%esp)
77ed29ad:	e8 5e 6f 00 00       	call   77ed9910 <_SetLastError@4>
77ed29b2:	31 c0                	xor    %eax,%eax
77ed29b4:	c9                   	leave  
77ed29b5:	c2 04 00             	ret    $0x4
77ed29b8:	90                   	nop    
77ed29b9:	8d b4 26 00 00 00 00 	lea    0x0(%esi),%esi

77ed29c0 <_GdiDeleteLocalDC@4>:
77ed29c0:	55                   	push   %ebp
77ed29c1:	89 e5                	mov    %esp,%ebp
77ed29c3:	83 ec 10             	sub    $0x10,%esp
77ed29c6:	68 1d a8 ed 77       	push   $0x77eda81d
77ed29cb:	68 20 a0 ed 77       	push   $0x77eda020
77ed29d0:	ff 15 e8 10 ee 77    	call   *0x77ee10e8
77ed29d6:	c7 04 24 78 00 00 00 	movl   $0x78,(%esp)
77ed29dd:	e8 2e 6f 00 00       	call   77ed9910 <_SetLastError@4>
77ed29e2:	31 c0                	xor    %eax,%eax
77ed29e4:	c9                   	leave  
77ed29e5:	c2 04 00             	ret    $0x4
77ed29e8:	90                   	nop    
77ed29e9:	8d b4 26 00 00 00 00 	lea    0x0(%esi),%esi

77ed29f0 <_GdiDescribePixelFormat@16>:
77ed29f0:	55                   	push   %ebp
77ed29f1:	89 e5                	mov    %esp,%ebp
77ed29f3:	83 ec 10             	sub    $0x10,%esp
77ed29f6:	68 2e a8 ed 77       	push   $0x77eda82e
77ed29fb:	68 20 a0 ed 77       	push   $0x77eda020
77ed2a00:	ff 15 e8 10 ee 77    	call   *0x77ee10e8
77ed2a06:	c7 04 24 78 00 00 00 	movl   $0x78,(%esp)
77ed2a0d:	e8 fe 6e 00 00       	call   77ed9910 <_SetLastError@4>
77ed2a12:	31 c0                	xor    %eax,%eax
77ed2a14:	c9                   	leave  
77ed2a15:	c2 10 00             	ret    $0x10
77ed2a18:	90                   	nop    
77ed2a19:	8d b4 26 00 00 00 00 	lea    0x0(%esi),%esi

77ed2a20 <_GdiDrawStream@12>:
77ed2a20:	55                   	push   %ebp
77ed2a21:	89 e5                	mov    %esp,%ebp
77ed2a23:	83 ec 10             	sub    $0x10,%esp
77ed2a26:	68 45 a8 ed 77       	push   $0x77eda845
77ed2a2b:	68 20 a0 ed 77       	push   $0x77eda020
77ed2a30:	ff 15 e8 10 ee 77    	call   *0x77ee10e8
77ed2a36:	c7 04 24 78 00 00 00 	movl   $0x78,(%esp)
77ed2a3d:	e8 ce 6e 00 00       	call   77ed9910 <_SetLastError@4>
77ed2a42:	31 c0                	xor    %eax,%eax
77ed2a44:	c9                   	leave  
77ed2a45:	c2 0c 00             	ret    $0xc
77ed2a48:	90                   	nop    
77ed2a49:	8d b4 26 00 00 00 00 	lea    0x0(%esi),%esi

77ed2a50 <_GdiFixUpHandle@4>:
77ed2a50:	55                   	push   %ebp
77ed2a51:	89 e5                	mov    %esp,%ebp
77ed2a53:	83 ec 10             	sub    $0x10,%esp
77ed2a56:	68 53 a8 ed 77       	push   $0x77eda853
77ed2a5b:	68 20 a0 ed 77       	push   $0x77eda020
77ed2a60:	ff 15 e8 10 ee 77    	call   *0x77ee10e8
77ed2a66:	c7 04 24 78 00 00 00 	movl   $0x78,(%esp)
77ed2a6d:	e8 9e 6e 00 00       	call   77ed9910 <_SetLastError@4>
77ed2a72:	31 c0                	xor    %eax,%eax
77ed2a74:	c9                   	leave  
77ed2a75:	c2 04 00             	ret    $0x4
77ed2a78:	90                   	nop    
77ed2a79:	8d b4 26 00 00 00 00 	lea    0x0(%esi),%esi

77ed2a80 <_GdiGetCodePage@4>:
77ed2a80:	55                   	push   %ebp
77ed2a81:	89 e5                	mov    %esp,%ebp
77ed2a83:	83 ec 10             	sub    $0x10,%esp
77ed2a86:	68 62 a8 ed 77       	push   $0x77eda862
77ed2a8b:	68 20 a0 ed 77       	push   $0x77eda020
77ed2a90:	ff 15 e8 10 ee 77    	call   *0x77ee10e8
77ed2a96:	c7 04 24 78 00 00 00 	movl   $0x78,(%esp)
77ed2a9d:	e8 6e 6e 00 00       	call   77ed9910 <_SetLastError@4>
77ed2aa2:	31 c0                	xor    %eax,%eax
77ed2aa4:	c9                   	leave  
77ed2aa5:	c2 04 00             	ret    $0x4
77ed2aa8:	90                   	nop    
77ed2aa9:	8d b4 26 00 00 00 00 	lea    0x0(%esi),%esi

77ed2ab0 <_GdiGetLocalBrush@4>:
77ed2ab0:	55                   	push   %ebp
77ed2ab1:	89 e5                	mov    %esp,%ebp
77ed2ab3:	83 ec 10             	sub    $0x10,%esp
77ed2ab6:	68 71 a8 ed 77       	push   $0x77eda871
77ed2abb:	68 20 a0 ed 77       	push   $0x77eda020
77ed2ac0:	ff 15 e8 10 ee 77    	call   *0x77ee10e8
77ed2ac6:	c7 04 24 78 00 00 00 	movl   $0x78,(%esp)
77ed2acd:	e8 3e 6e 00 00       	call   77ed9910 <_SetLastError@4>
77ed2ad2:	31 c0                	xor    %eax,%eax
77ed2ad4:	c9                   	leave  
77ed2ad5:	c2 04 00             	ret    $0x4
77ed2ad8:	90                   	nop    
77ed2ad9:	8d b4 26 00 00 00 00 	lea    0x0(%esi),%esi

77ed2ae0 <_GdiGetLocalDC@4>:
77ed2ae0:	55                   	push   %ebp
77ed2ae1:	89 e5                	mov    %esp,%ebp
77ed2ae3:	83 ec 10             	sub    $0x10,%esp
77ed2ae6:	68 82 a8 ed 77       	push   $0x77eda882
77ed2aeb:	68 20 a0 ed 77       	push   $0x77eda020
77ed2af0:	ff 15 e8 10 ee 77    	call   *0x77ee10e8
77ed2af6:	c7 04 24 78 00 00 00 	movl   $0x78,(%esp)
77ed2afd:	e8 0e 6e 00 00       	call   77ed9910 <_SetLastError@4>
77ed2b02:	31 c0                	xor    %eax,%eax
77ed2b04:	c9                   	leave  
77ed2b05:	c2 04 00             	ret    $0x4
77ed2b08:	90                   	nop    
77ed2b09:	8d b4 26 00 00 00 00 	lea    0x0(%esi),%esi

77ed2b10 <_GdiGetLocalFont@4>:
77ed2b10:	55                   	push   %ebp
77ed2b11:	89 e5                	mov    %esp,%ebp
77ed2b13:	83 ec 10             	sub    $0x10,%esp
77ed2b16:	68 90 a8 ed 77       	push   $0x77eda890
77ed2b1b:	68 20 a0 ed 77       	push   $0x77eda020
77ed2b20:	ff 15 e8 10 ee 77    	call   *0x77ee10e8
77ed2b26:	c7 04 24 78 00 00 00 	movl   $0x78,(%esp)
77ed2b2d:	e8 de 6d 00 00       	call   77ed9910 <_SetLastError@4>
77ed2b32:	31 c0                	xor    %eax,%eax
77ed2b34:	c9                   	leave  
77ed2b35:	c2 04 00             	ret    $0x4
77ed2b38:	90                   	nop    
77ed2b39:	8d b4 26 00 00 00 00 	lea    0x0(%esi),%esi

77ed2b40 <_GdiIsMetaFileDC@4>:
77ed2b40:	55                   	push   %ebp
77ed2b41:	89 e5                	mov    %esp,%ebp
77ed2b43:	83 ec 10             	sub    $0x10,%esp
77ed2b46:	68 a0 a8 ed 77       	push   $0x77eda8a0
77ed2b4b:	68 20 a0 ed 77       	push   $0x77eda020
77ed2b50:	ff 15 e8 10 ee 77    	call   *0x77ee10e8
77ed2b56:	c7 04 24 78 00 00 00 	movl   $0x78,(%esp)
77ed2b5d:	e8 ae 6d 00 00       	call   77ed9910 <_SetLastError@4>
77ed2b62:	31 c0                	xor    %eax,%eax
77ed2b64:	c9                   	leave  
77ed2b65:	c2 04 00             	ret    $0x4
77ed2b68:	90                   	nop    
77ed2b69:	8d b4 26 00 00 00 00 	lea    0x0(%esi),%esi

77ed2b70 <_GdiIsMetaPrintDC@4>:
77ed2b70:	55                   	push   %ebp
77ed2b71:	89 e5                	mov    %esp,%ebp
77ed2b73:	83 ec 10             	sub    $0x10,%esp
77ed2b76:	68 b0 a8 ed 77       	push   $0x77eda8b0
77ed2b7b:	68 20 a0 ed 77       	push   $0x77eda020
77ed2b80:	ff 15 e8 10 ee 77    	call   *0x77ee10e8
77ed2b86:	c7 04 24 78 00 00 00 	movl   $0x78,(%esp)
77ed2b8d:	e8 7e 6d 00 00       	call   77ed9910 <_SetLastError@4>
77ed2b92:	31 c0                	xor    %eax,%eax
77ed2b94:	c9                   	leave  
77ed2b95:	c2 04 00             	ret    $0x4
77ed2b98:	90                   	nop    
77ed2b99:	8d b4 26 00 00 00 00 	lea    0x0(%esi),%esi

77ed2ba0 <_GdiIsPlayMetafileDC@4>:
77ed2ba0:	55                   	push   %ebp
77ed2ba1:	89 e5                	mov    %esp,%ebp
77ed2ba3:	83 ec 10             	sub    $0x10,%esp
77ed2ba6:	68 c1 a8 ed 77       	push   $0x77eda8c1
77ed2bab:	68 20 a0 ed 77       	push   $0x77eda020
77ed2bb0:	ff 15 e8 10 ee 77    	call   *0x77ee10e8
77ed2bb6:	c7 04 24 78 00 00 00 	movl   $0x78,(%esp)
77ed2bbd:	e8 4e 6d 00 00       	call   77ed9910 <_SetLastError@4>
77ed2bc2:	31 c0                	xor    %eax,%eax
77ed2bc4:	c9                   	leave  
77ed2bc5:	c2 04 00             	ret    $0x4
77ed2bc8:	90                   	nop    
77ed2bc9:	8d b4 26 00 00 00 00 	lea    0x0(%esi),%esi

77ed2bd0 <_GdiReleaseDC@4>:
77ed2bd0:	55                   	push   %ebp
77ed2bd1:	89 e5                	mov    %esp,%ebp
77ed2bd3:	83 ec 10             	sub    $0x10,%esp
77ed2bd6:	68 d5 a8 ed 77       	push   $0x77eda8d5
77ed2bdb:	68 20 a0 ed 77       	push   $0x77eda020
77ed2be0:	ff 15 e8 10 ee 77    	call   *0x77ee10e8
77ed2be6:	c7 04 24 78 00 00 00 	movl   $0x78,(%esp)
77ed2bed:	e8 1e 6d 00 00       	call   77ed9910 <_SetLastError@4>
77ed2bf2:	31 c0                	xor    %eax,%eax
77ed2bf4:	c9                   	leave  
77ed2bf5:	c2 04 00             	ret    $0x4
77ed2bf8:	90                   	nop    
77ed2bf9:	8d b4 26 00 00 00 00 	lea    0x0(%esi),%esi

77ed2c00 <_GdiReleaseLocalDC@4>:
77ed2c00:	55                   	push   %ebp
77ed2c01:	89 e5                	mov    %esp,%ebp
77ed2c03:	83 ec 10             	sub    $0x10,%esp
77ed2c06:	68 e2 a8 ed 77       	push   $0x77eda8e2
77ed2c0b:	68 20 a0 ed 77       	push   $0x77eda020
77ed2c10:	ff 15 e8 10 ee 77    	call   *0x77ee10e8
77ed2c16:	c7 04 24 78 00 00 00 	movl   $0x78,(%esp)
77ed2c1d:	e8 ee 6c 00 00       	call   77ed9910 <_SetLastError@4>
77ed2c22:	31 c0                	xor    %eax,%eax
77ed2c24:	c9                   	leave  
77ed2c25:	c2 04 00             	ret    $0x4
77ed2c28:	90                   	nop    
77ed2c29:	8d b4 26 00 00 00 00 	lea    0x0(%esi),%esi

77ed2c30 <_GdiSetAttrs@4>:
77ed2c30:	55                   	push   %ebp
77ed2c31:	89 e5                	mov    %esp,%ebp
77ed2c33:	83 ec 10             	sub    $0x10,%esp
77ed2c36:	68 f4 a8 ed 77       	push   $0x77eda8f4
77ed2c3b:	68 20 a0 ed 77       	push   $0x77eda020
77ed2c40:	ff 15 e8 10 ee 77    	call   *0x77ee10e8
77ed2c46:	c7 04 24 78 00 00 00 	movl   $0x78,(%esp)
77ed2c4d:	e8 be 6c 00 00       	call   77ed9910 <_SetLastError@4>
77ed2c52:	31 c0                	xor    %eax,%eax
77ed2c54:	c9                   	leave  
77ed2c55:	c2 04 00             	ret    $0x4
77ed2c58:	90                   	nop    
77ed2c59:	8d b4 26 00 00 00 00 	lea    0x0(%esi),%esi

77ed2c60 <_GdiSetLastError@4>:
77ed2c60:	55                   	push   %ebp
77ed2c61:	89 e5                	mov    %esp,%ebp
77ed2c63:	83 ec 10             	sub    $0x10,%esp
77ed2c66:	68 00 a9 ed 77       	push   $0x77eda900
77ed2c6b:	68 20 a0 ed 77       	push   $0x77eda020
77ed2c70:	ff 15 e8 10 ee 77    	call   *0x77ee10e8
77ed2c76:	c7 45 08 78 00 00 00 	movl   $0x78,0x8(%ebp)
77ed2c7d:	83 c4 10             	add    $0x10,%esp
77ed2c80:	c9                   	leave  
77ed2c81:	e9 8a 6c 00 00       	jmp    77ed9910 <_SetLastError@4>
77ed2c86:	8d 76 00             	lea    0x0(%esi),%esi
77ed2c89:	8d bc 27 00 00 00 00 	lea    0x0(%edi),%edi

77ed2c90 <_GdiSetPixelFormat@8>:
77ed2c90:	55                   	push   %ebp
77ed2c91:	89 e5                	mov    %esp,%ebp
77ed2c93:	83 ec 10             	sub    $0x10,%esp
77ed2c96:	68 10 a9 ed 77       	push   $0x77eda910
77ed2c9b:	68 20 a0 ed 77       	push   $0x77eda020
77ed2ca0:	ff 15 e8 10 ee 77    	call   *0x77ee10e8
77ed2ca6:	c7 04 24 78 00 00 00 	movl   $0x78,(%esp)
77ed2cad:	e8 5e 6c 00 00       	call   77ed9910 <_SetLastError@4>
77ed2cb2:	31 c0                	xor    %eax,%eax
77ed2cb4:	c9                   	leave  
77ed2cb5:	c2 08 00             	ret    $0x8
77ed2cb8:	90                   	nop    
77ed2cb9:	8d b4 26 00 00 00 00 	lea    0x0(%esi),%esi

77ed2cc0 <_GdiValidateHandle@4>:
77ed2cc0:	55                   	push   %ebp
77ed2cc1:	89 e5                	mov    %esp,%ebp
77ed2cc3:	83 ec 10             	sub    $0x10,%esp
77ed2cc6:	68 22 a9 ed 77       	push   $0x77eda922
77ed2ccb:	68 20 a0 ed 77       	push   $0x77eda020
77ed2cd0:	ff 15 e8 10 ee 77    	call   *0x77ee10e8
77ed2cd6:	c7 04 24 78 00 00 00 	movl   $0x78,(%esp)
77ed2cdd:	e8 2e 6c 00 00       	call   77ed9910 <_SetLastError@4>
77ed2ce2:	31 c0                	xor    %eax,%eax
77ed2ce4:	c9                   	leave  
77ed2ce5:	c2 04 00             	ret    $0x4
77ed2ce8:	90                   	nop    
77ed2ce9:	8d b4 26 00 00 00 00 	lea    0x0(%esi),%esi

77ed2cf0 <_GdiSwapBuffers@4>:
77ed2cf0:	55                   	push   %ebp
77ed2cf1:	89 e5                	mov    %esp,%ebp
77ed2cf3:	83 ec 10             	sub    $0x10,%esp
77ed2cf6:	68 34 a9 ed 77       	push   $0x77eda934
77ed2cfb:	68 20 a0 ed 77       	push   $0x77eda020
77ed2d00:	ff 15 e8 10 ee 77    	call   *0x77ee10e8
77ed2d06:	c7 04 24 78 00 00 00 	movl   $0x78,(%esp)
77ed2d0d:	e8 fe 6b 00 00       	call   77ed9910 <_SetLastError@4>
77ed2d12:	31 c0                	xor    %eax,%eax
77ed2d14:	c9                   	leave  
77ed2d15:	c2 04 00             	ret    $0x4
77ed2d18:	90                   	nop    
77ed2d19:	8d b4 26 00 00 00 00 	lea    0x0(%esi),%esi

77ed2d20 <_GdiSetServerAttr@8>:
77ed2d20:	55                   	push   %ebp
77ed2d21:	89 e5                	mov    %esp,%ebp
77ed2d23:	83 ec 10             	sub    $0x10,%esp
77ed2d26:	68 43 a9 ed 77       	push   $0x77eda943
77ed2d2b:	68 20 a0 ed 77       	push   $0x77eda020
77ed2d30:	ff 15 e8 10 ee 77    	call   *0x77ee10e8
77ed2d36:	c7 04 24 78 00 00 00 	movl   $0x78,(%esp)
77ed2d3d:	e8 ce 6b 00 00       	call   77ed9910 <_SetLastError@4>
77ed2d42:	c9                   	leave  
77ed2d43:	c2 08 00             	ret    $0x8
77ed2d46:	8d 76 00             	lea    0x0(%esi),%esi
77ed2d49:	8d bc 27 00 00 00 00 	lea    0x0(%edi),%edi

77ed2d50 <_GetBitmapAttributes@4>:
77ed2d50:	55                   	push   %ebp
77ed2d51:	89 e5                	mov    %esp,%ebp
77ed2d53:	83 ec 10             	sub    $0x10,%esp
77ed2d56:	68 54 a9 ed 77       	push   $0x77eda954
77ed2d5b:	68 20 a0 ed 77       	push   $0x77eda020
77ed2d60:	ff 15 e8 10 ee 77    	call   *0x77ee10e8
77ed2d66:	c7 04 24 78 00 00 00 	movl   $0x78,(%esp)
77ed2d6d:	e8 9e 6b 00 00       	call   77ed9910 <_SetLastError@4>
77ed2d72:	31 c0                	xor    %eax,%eax
77ed2d74:	c9                   	leave  
77ed2d75:	c2 04 00             	ret    $0x4
77ed2d78:	90                   	nop    
77ed2d79:	8d b4 26 00 00 00 00 	lea    0x0(%esi),%esi

77ed2d80 <_GetBrushAttributes@4>:
77ed2d80:	55                   	push   %ebp
77ed2d81:	89 e5                	mov    %esp,%ebp
77ed2d83:	83 ec 10             	sub    $0x10,%esp
77ed2d86:	68 68 a9 ed 77       	push   $0x77eda968
77ed2d8b:	68 20 a0 ed 77       	push   $0x77eda020
77ed2d90:	ff 15 e8 10 ee 77    	call   *0x77ee10e8
77ed2d96:	c7 04 24 78 00 00 00 	movl   $0x78,(%esp)
77ed2d9d:	e8 6e 6b 00 00       	call   77ed9910 <_SetLastError@4>
77ed2da2:	31 c0                	xor    %eax,%eax
77ed2da4:	c9                   	leave  
77ed2da5:	c2 04 00             	ret    $0x4
77ed2da8:	90                   	nop    
77ed2da9:	8d b4 26 00 00 00 00 	lea    0x0(%esi),%esi

77ed2db0 <_GetCharABCWidthsI@20>:
77ed2db0:	55                   	push   %ebp
77ed2db1:	89 e5                	mov    %esp,%ebp
77ed2db3:	83 ec 10             	sub    $0x10,%esp
77ed2db6:	68 7b a9 ed 77       	push   $0x77eda97b
77ed2dbb:	68 20 a0 ed 77       	push   $0x77eda020
77ed2dc0:	ff 15 e8 10 ee 77    	call   *0x77ee10e8
77ed2dc6:	c7 04 24 78 00 00 00 	movl   $0x78,(%esp)
77ed2dcd:	e8 3e 6b 00 00       	call   77ed9910 <_SetLastError@4>
77ed2dd2:	31 c0                	xor    %eax,%eax
77ed2dd4:	c9                   	leave  
77ed2dd5:	c2 14 00             	ret    $0x14
77ed2dd8:	90                   	nop    
77ed2dd9:	8d b4 26 00 00 00 00 	lea    0x0(%esi),%esi

77ed2de0 <_GetCharWidthI@20>:
77ed2de0:	55                   	push   %ebp
77ed2de1:	89 e5                	mov    %esp,%ebp
77ed2de3:	83 ec 10             	sub    $0x10,%esp
77ed2de6:	68 8d a9 ed 77       	push   $0x77eda98d
77ed2deb:	68 20 a0 ed 77       	push   $0x77eda020
77ed2df0:	ff 15 e8 10 ee 77    	call   *0x77ee10e8
77ed2df6:	c7 04 24 78 00 00 00 	movl   $0x78,(%esp)
77ed2dfd:	e8 0e 6b 00 00       	call   77ed9910 <_SetLastError@4>
77ed2e02:	31 c0                	xor    %eax,%eax
77ed2e04:	c9                   	leave  
77ed2e05:	c2 14 00             	ret    $0x14
77ed2e08:	90                   	nop    
77ed2e09:	8d b4 26 00 00 00 00 	lea    0x0(%esi),%esi

77ed2e10 <_GetFontUnicodeRanges@8>:
77ed2e10:	55                   	push   %ebp
77ed2e11:	89 e5                	mov    %esp,%ebp
77ed2e13:	83 ec 10             	sub    $0x10,%esp
77ed2e16:	68 9b a9 ed 77       	push   $0x77eda99b
77ed2e1b:	68 20 a0 ed 77       	push   $0x77eda020
77ed2e20:	ff 15 e8 10 ee 77    	call   *0x77ee10e8
77ed2e26:	c7 04 24 78 00 00 00 	movl   $0x78,(%esp)
77ed2e2d:	e8 de 6a 00 00       	call   77ed9910 <_SetLastError@4>
77ed2e32:	31 c0                	xor    %eax,%eax
77ed2e34:	c9                   	leave  
77ed2e35:	c2 08 00             	ret    $0x8
77ed2e38:	90                   	nop    
77ed2e39:	8d b4 26 00 00 00 00 	lea    0x0(%esi),%esi

77ed2e40 <_GetEUDCTimeStamp@0>:
77ed2e40:	55                   	push   %ebp
77ed2e41:	89 e5                	mov    %esp,%ebp
77ed2e43:	83 ec 10             	sub    $0x10,%esp
77ed2e46:	68 b0 a9 ed 77       	push   $0x77eda9b0
77ed2e4b:	68 20 a0 ed 77       	push   $0x77eda020
77ed2e50:	ff 15 e8 10 ee 77    	call   *0x77ee10e8
77ed2e56:	c7 04 24 78 00 00 00 	movl   $0x78,(%esp)
77ed2e5d:	e8 ae 6a 00 00       	call   77ed9910 <_SetLastError@4>
77ed2e62:	31 c0                	xor    %eax,%eax
77ed2e64:	c9                   	leave  
77ed2e65:	c3                   	ret    
77ed2e66:	8d 76 00             	lea    0x0(%esi),%esi
77ed2e69:	8d bc 27 00 00 00 00 	lea    0x0(%edi),%edi

77ed2e70 <_GetFontAssocStatus@4>:
77ed2e70:	55                   	push   %ebp
77ed2e71:	89 e5                	mov    %esp,%ebp
77ed2e73:	83 ec 10             	sub    $0x10,%esp
77ed2e76:	68 c1 a9 ed 77       	push   $0x77eda9c1
77ed2e7b:	68 20 a0 ed 77       	push   $0x77eda020
77ed2e80:	ff 15 e8 10 ee 77    	call   *0x77ee10e8
77ed2e86:	c7 04 24 78 00 00 00 	movl   $0x78,(%esp)
77ed2e8d:	e8 7e 6a 00 00       	call   77ed9910 <_SetLastError@4>
77ed2e92:	31 c0                	xor    %eax,%eax
77ed2e94:	c9                   	leave  
77ed2e95:	c2 04 00             	ret    $0x4
77ed2e98:	90                   	nop    
77ed2e99:	8d b4 26 00 00 00 00 	lea    0x0(%esi),%esi

77ed2ea0 <_GetHFONT@4>:
77ed2ea0:	55                   	push   %ebp
77ed2ea1:	89 e5                	mov    %esp,%ebp
77ed2ea3:	83 ec 10             	sub    $0x10,%esp
77ed2ea6:	68 d4 a9 ed 77       	push   $0x77eda9d4
77ed2eab:	68 20 a0 ed 77       	push   $0x77eda020
77ed2eb0:	ff 15 e8 10 ee 77    	call   *0x77ee10e8
77ed2eb6:	c7 04 24 78 00 00 00 	movl   $0x78,(%esp)
77ed2ebd:	e8 4e 6a 00 00       	call   77ed9910 <_SetLastError@4>
77ed2ec2:	31 c0                	xor    %eax,%eax
77ed2ec4:	c9                   	leave  
77ed2ec5:	c2 04 00             	ret    $0x4
77ed2ec8:	90                   	nop    
77ed2ec9:	8d b4 26 00 00 00 00 	lea    0x0(%esi),%esi

77ed2ed0 <_GetLayout@4>:
77ed2ed0:	55                   	push   %ebp
77ed2ed1:	89 e5                	mov    %esp,%ebp
77ed2ed3:	83 ec 10             	sub    $0x10,%esp
77ed2ed6:	68 dd a9 ed 77       	push   $0x77eda9dd
77ed2edb:	68 20 a0 ed 77       	push   $0x77eda020
77ed2ee0:	ff 15 e8 10 ee 77    	call   *0x77ee10e8
77ed2ee6:	c7 04 24 78 00 00 00 	movl   $0x78,(%esp)
77ed2eed:	e8 1e 6a 00 00       	call   77ed9910 <_SetLastError@4>
77ed2ef2:	31 c0                	xor    %eax,%eax
77ed2ef4:	c9                   	leave  
77ed2ef5:	c2 04 00             	ret    $0x4
77ed2ef8:	90                   	nop    
77ed2ef9:	8d b4 26 00 00 00 00 	lea    0x0(%esi),%esi

77ed2f00 <_GetTextExtentExPointWPri@28>:
77ed2f00:	55                   	push   %ebp
77ed2f01:	89 e5                	mov    %esp,%ebp
77ed2f03:	83 ec 10             	sub    $0x10,%esp
77ed2f06:	68 e7 a9 ed 77       	push   $0x77eda9e7
77ed2f0b:	68 20 a0 ed 77       	push   $0x77eda020
77ed2f10:	ff 15 e8 10 ee 77    	call   *0x77ee10e8
77ed2f16:	c7 04 24 78 00 00 00 	movl   $0x78,(%esp)
77ed2f1d:	e8 ee 69 00 00       	call   77ed9910 <_SetLastError@4>
77ed2f22:	31 c0                	xor    %eax,%eax
77ed2f24:	c9                   	leave  
77ed2f25:	c2 1c 00             	ret    $0x1c
77ed2f28:	90                   	nop    
77ed2f29:	8d b4 26 00 00 00 00 	lea    0x0(%esi),%esi

77ed2f30 <_GetTextFaceAliasW@12>:
77ed2f30:	55                   	push   %ebp
77ed2f31:	89 e5                	mov    %esp,%ebp
77ed2f33:	83 ec 10             	sub    $0x10,%esp
77ed2f36:	68 00 aa ed 77       	push   $0x77edaa00
77ed2f3b:	68 20 a0 ed 77       	push   $0x77eda020
77ed2f40:	ff 15 e8 10 ee 77    	call   *0x77ee10e8
77ed2f46:	c7 04 24 78 00 00 00 	movl   $0x78,(%esp)
77ed2f4d:	e8 be 69 00 00       	call   77ed9910 <_SetLastError@4>
77ed2f52:	31 c0                	xor    %eax,%eax
77ed2f54:	c9                   	leave  
77ed2f55:	c2 0c 00             	ret    $0xc
77ed2f58:	90                   	nop    
77ed2f59:	8d b4 26 00 00 00 00 	lea    0x0(%esi),%esi

77ed2f60 <_GetTransform@12>:
77ed2f60:	55                   	push   %ebp
77ed2f61:	89 e5                	mov    %esp,%ebp
77ed2f63:	83 ec 10             	sub    $0x10,%esp
77ed2f66:	68 12 aa ed 77       	push   $0x77edaa12
77ed2f6b:	68 20 a0 ed 77       	push   $0x77eda020
77ed2f70:	ff 15 e8 10 ee 77    	call   *0x77ee10e8
77ed2f76:	c7 04 24 78 00 00 00 	movl   $0x78,(%esp)
77ed2f7d:	e8 8e 69 00 00       	call   77ed9910 <_SetLastError@4>
77ed2f82:	31 c0                	xor    %eax,%eax
77ed2f84:	c9                   	leave  
77ed2f85:	c2 0c 00             	ret    $0xc
77ed2f88:	90                   	nop    
77ed2f89:	8d b4 26 00 00 00 00 	lea    0x0(%esi),%esi

77ed2f90 <_HT_Get8BPPFormatPalette@16>:
77ed2f90:	55                   	push   %ebp
77ed2f91:	89 e5                	mov    %esp,%ebp
77ed2f93:	83 ec 10             	sub    $0x10,%esp
77ed2f96:	68 1f aa ed 77       	push   $0x77edaa1f
77ed2f9b:	68 20 a0 ed 77       	push   $0x77eda020
77ed2fa0:	ff 15 e8 10 ee 77    	call   *0x77ee10e8
77ed2fa6:	c7 04 24 78 00 00 00 	movl   $0x78,(%esp)
77ed2fad:	e8 5e 69 00 00       	call   77ed9910 <_SetLastError@4>
77ed2fb2:	31 c0                	xor    %eax,%eax
77ed2fb4:	c9                   	leave  
77ed2fb5:	c2 10 00             	ret    $0x10
77ed2fb8:	90                   	nop    
77ed2fb9:	8d b4 26 00 00 00 00 	lea    0x0(%esi),%esi

77ed2fc0 <_HT_Get8BPPMaskPalette@24>:
77ed2fc0:	55                   	push   %ebp
77ed2fc1:	89 e5                	mov    %esp,%ebp
77ed2fc3:	83 ec 10             	sub    $0x10,%esp
77ed2fc6:	68 37 aa ed 77       	push   $0x77edaa37
77ed2fcb:	68 20 a0 ed 77       	push   $0x77eda020
77ed2fd0:	ff 15 e8 10 ee 77    	call   *0x77ee10e8
77ed2fd6:	c7 04 24 78 00 00 00 	movl   $0x78,(%esp)
77ed2fdd:	e8 2e 69 00 00       	call   77ed9910 <_SetLastError@4>
77ed2fe2:	31 c0                	xor    %eax,%eax
77ed2fe4:	c9                   	leave  
77ed2fe5:	c2 18 00             	ret    $0x18
77ed2fe8:	90                   	nop    
77ed2fe9:	8d b4 26 00 00 00 00 	lea    0x0(%esi),%esi

77ed2ff0 <_MirrorRgn@8>:
77ed2ff0:	55                   	push   %ebp
77ed2ff1:	89 e5                	mov    %esp,%ebp
77ed2ff3:	83 ec 10             	sub    $0x10,%esp
77ed2ff6:	68 4d aa ed 77       	push   $0x77edaa4d
77ed2ffb:	68 20 a0 ed 77       	push   $0x77eda020
77ed3000:	ff 15 e8 10 ee 77    	call   *0x77ee10e8
77ed3006:	c7 04 24 78 00 00 00 	movl   $0x78,(%esp)
77ed300d:	e8 fe 68 00 00       	call   77ed9910 <_SetLastError@4>
77ed3012:	31 c0                	xor    %eax,%eax
77ed3014:	c9                   	leave  
77ed3015:	c2 08 00             	ret    $0x8
77ed3018:	90                   	nop    
77ed3019:	8d b4 26 00 00 00 00 	lea    0x0(%esi),%esi

77ed3020 <_NamedEscape@32>:
77ed3020:	55                   	push   %ebp
77ed3021:	89 e5                	mov    %esp,%ebp
77ed3023:	83 ec 10             	sub    $0x10,%esp
77ed3026:	68 57 aa ed 77       	push   $0x77edaa57
77ed302b:	68 20 a0 ed 77       	push   $0x77eda020
77ed3030:	ff 15 e8 10 ee 77    	call   *0x77ee10e8
77ed3036:	c7 04 24 78 00 00 00 	movl   $0x78,(%esp)
77ed303d:	e8 ce 68 00 00       	call   77ed9910 <_SetLastError@4>
77ed3042:	31 c0                	xor    %eax,%eax
77ed3044:	c9                   	leave  
77ed3045:	c2 20 00             	ret    $0x20
77ed3048:	90                   	nop    
77ed3049:	8d b4 26 00 00 00 00 	lea    0x0(%esi),%esi

77ed3050 <_QueryFontAssocStatus@0>:
77ed3050:	55                   	push   %ebp
77ed3051:	89 e5                	mov    %esp,%ebp
77ed3053:	83 ec 10             	sub    $0x10,%esp
77ed3056:	68 63 aa ed 77       	push   $0x77edaa63
77ed305b:	68 20 a0 ed 77       	push   $0x77eda020
77ed3060:	ff 15 e8 10 ee 77    	call   *0x77ee10e8
77ed3066:	c7 04 24 78 00 00 00 	movl   $0x78,(%esp)
77ed306d:	e8 9e 68 00 00       	call   77ed9910 <_SetLastError@4>
77ed3072:	31 c0                	xor    %eax,%eax
77ed3074:	c9                   	leave  
77ed3075:	c3                   	ret    
77ed3076:	8d 76 00             	lea    0x0(%esi),%esi
77ed3079:	8d bc 27 00 00 00 00 	lea    0x0(%edi),%edi

77ed3080 <_RemoveFontMemResourceEx@4>:
77ed3080:	55                   	push   %ebp
77ed3081:	89 e5                	mov    %esp,%ebp
77ed3083:	83 ec 10             	sub    $0x10,%esp
77ed3086:	68 78 aa ed 77       	push   $0x77edaa78
77ed308b:	68 20 a0 ed 77       	push   $0x77eda020
77ed3090:	ff 15 e8 10 ee 77    	call   *0x77ee10e8
77ed3096:	c7 04 24 78 00 00 00 	movl   $0x78,(%esp)
77ed309d:	e8 6e 68 00 00       	call   77ed9910 <_SetLastError@4>
77ed30a2:	31 c0                	xor    %eax,%eax
77ed30a4:	c9                   	leave  
77ed30a5:	c2 04 00             	ret    $0x4
77ed30a8:	90                   	nop    
77ed30a9:	8d b4 26 00 00 00 00 	lea    0x0(%esi),%esi

77ed30b0 <_RemoveFontResourceTracking@8>:
77ed30b0:	55                   	push   %ebp
77ed30b1:	89 e5                	mov    %esp,%ebp
77ed30b3:	83 ec 10             	sub    $0x10,%esp
77ed30b6:	68 90 aa ed 77       	push   $0x77edaa90
77ed30bb:	68 20 a0 ed 77       	push   $0x77eda020
77ed30c0:	ff 15 e8 10 ee 77    	call   *0x77ee10e8
77ed30c6:	c7 04 24 78 00 00 00 	movl   $0x78,(%esp)
77ed30cd:	e8 3e 68 00 00       	call   77ed9910 <_SetLastError@4>
77ed30d2:	31 c0                	xor    %eax,%eax
77ed30d4:	c9                   	leave  
77ed30d5:	c2 08 00             	ret    $0x8
77ed30d8:	90                   	nop    
77ed30d9:	8d b4 26 00 00 00 00 	lea    0x0(%esi),%esi

77ed30e0 <_SetBitmapAttributes@8>:
77ed30e0:	55                   	push   %ebp
77ed30e1:	89 e5                	mov    %esp,%ebp
77ed30e3:	83 ec 10             	sub    $0x10,%esp
77ed30e6:	68 ab aa ed 77       	push   $0x77edaaab
77ed30eb:	68 20 a0 ed 77       	push   $0x77eda020
77ed30f0:	ff 15 e8 10 ee 77    	call   *0x77ee10e8
77ed30f6:	c7 04 24 78 00 00 00 	movl   $0x78,(%esp)
77ed30fd:	e8 0e 68 00 00       	call   77ed9910 <_SetLastError@4>
77ed3102:	31 c0                	xor    %eax,%eax
77ed3104:	c9                   	leave  
77ed3105:	c2 08 00             	ret    $0x8
77ed3108:	90                   	nop    
77ed3109:	8d b4 26 00 00 00 00 	lea    0x0(%esi),%esi

77ed3110 <_SetBrushAttributes@8>:
77ed3110:	55                   	push   %ebp
77ed3111:	89 e5                	mov    %esp,%ebp
77ed3113:	83 ec 10             	sub    $0x10,%esp
77ed3116:	68 bf aa ed 77       	push   $0x77edaabf
77ed311b:	68 20 a0 ed 77       	push   $0x77eda020
77ed3120:	ff 15 e8 10 ee 77    	call   *0x77ee10e8
77ed3126:	c7 04 24 78 00 00 00 	movl   $0x78,(%esp)
77ed312d:	e8 de 67 00 00       	call   77ed9910 <_SetLastError@4>
77ed3132:	31 c0                	xor    %eax,%eax
77ed3134:	c9                   	leave  
77ed3135:	c2 08 00             	ret    $0x8
77ed3138:	90                   	nop    
77ed3139:	8d b4 26 00 00 00 00 	lea    0x0(%esi),%esi

77ed3140 <_SetLayout@8>:
77ed3140:	55                   	push   %ebp
77ed3141:	89 e5                	mov    %esp,%ebp
77ed3143:	83 ec 10             	sub    $0x10,%esp
77ed3146:	68 d2 aa ed 77       	push   $0x77edaad2
77ed314b:	68 20 a0 ed 77       	push   $0x77eda020
77ed3150:	ff 15 e8 10 ee 77    	call   *0x77ee10e8
77ed3156:	c7 04 24 78 00 00 00 	movl   $0x78,(%esp)
77ed315d:	e8 ae 67 00 00       	call   77ed9910 <_SetLastError@4>
77ed3162:	31 c0                	xor    %eax,%eax
77ed3164:	c9                   	leave  
77ed3165:	c2 08 00             	ret    $0x8
77ed3168:	90                   	nop    
77ed3169:	8d b4 26 00 00 00 00 	lea    0x0(%esi),%esi

77ed3170 <_SetLayoutWidth@12>:
77ed3170:	55                   	push   %ebp
77ed3171:	89 e5                	mov    %esp,%ebp
77ed3173:	83 ec 10             	sub    $0x10,%esp
77ed3176:	68 dc aa ed 77       	push   $0x77edaadc
77ed317b:	68 20 a0 ed 77       	push   $0x77eda020
77ed3180:	ff 15 e8 10 ee 77    	call   *0x77ee10e8
77ed3186:	c7 04 24 78 00 00 00 	movl   $0x78,(%esp)
77ed318d:	e8 7e 67 00 00       	call   77ed9910 <_SetLastError@4>
77ed3192:	31 c0                	xor    %eax,%eax
77ed3194:	c9                   	leave  
77ed3195:	c2 0c 00             	ret    $0xc
77ed3198:	90                   	nop    
77ed3199:	8d b4 26 00 00 00 00 	lea    0x0(%esi),%esi

77ed31a0 <_SetMagicColors@12>:
77ed31a0:	55                   	push   %ebp
77ed31a1:	89 e5                	mov    %esp,%ebp
77ed31a3:	83 ec 10             	sub    $0x10,%esp
77ed31a6:	68 eb aa ed 77       	push   $0x77edaaeb
77ed31ab:	68 20 a0 ed 77       	push   $0x77eda020
77ed31b0:	ff 15 e8 10 ee 77    	call   *0x77ee10e8
77ed31b6:	c7 04 24 78 00 00 00 	movl   $0x78,(%esp)
77ed31bd:	e8 4e 67 00 00       	call   77ed9910 <_SetLastError@4>
77ed31c2:	31 c0                	xor    %eax,%eax
77ed31c4:	c9                   	leave  
77ed31c5:	c2 0c 00             	ret    $0xc
77ed31c8:	90                   	nop    
77ed31c9:	8d b4 26 00 00 00 00 	lea    0x0(%esi),%esi

77ed31d0 <_SetVirtualResolution@20>:
77ed31d0:	55                   	push   %ebp
77ed31d1:	89 e5                	mov    %esp,%ebp
77ed31d3:	83 ec 10             	sub    $0x10,%esp
77ed31d6:	68 fa aa ed 77       	push   $0x77edaafa
77ed31db:	68 20 a0 ed 77       	push   $0x77eda020
77ed31e0:	ff 15 e8 10 ee 77    	call   *0x77ee10e8
77ed31e6:	c7 04 24 78 00 00 00 	movl   $0x78,(%esp)
77ed31ed:	e8 1e 67 00 00       	call   77ed9910 <_SetLastError@4>
77ed31f2:	31 c0                	xor    %eax,%eax
77ed31f4:	c9                   	leave  
77ed31f5:	c2 14 00             	ret    $0x14
77ed31f8:	90                   	nop    
77ed31f9:	8d b4 26 00 00 00 00 	lea    0x0(%esi),%esi

77ed3200 <_StartFormPage@4>:
77ed3200:	55                   	push   %ebp
77ed3201:	89 e5                	mov    %esp,%ebp
77ed3203:	83 ec 10             	sub    $0x10,%esp
77ed3206:	68 0f ab ed 77       	push   $0x77edab0f
77ed320b:	68 20 a0 ed 77       	push   $0x77eda020
77ed3210:	ff 15 e8 10 ee 77    	call   *0x77ee10e8
77ed3216:	c7 04 24 78 00 00 00 	movl   $0x78,(%esp)
77ed321d:	e8 ee 66 00 00       	call   77ed9910 <_SetLastError@4>
77ed3222:	31 c0                	xor    %eax,%eax
77ed3224:	c9                   	leave  
77ed3225:	c2 04 00             	ret    $0x4
77ed3228:	90                   	nop    
77ed3229:	8d b4 26 00 00 00 00 	lea    0x0(%esi),%esi

77ed3230 <_UnloadNetworkFonts@4>:
77ed3230:	55                   	push   %ebp
77ed3231:	89 e5                	mov    %esp,%ebp
77ed3233:	83 ec 10             	sub    $0x10,%esp
77ed3236:	68 1d ab ed 77       	push   $0x77edab1d
77ed323b:	68 20 a0 ed 77       	push   $0x77eda020
77ed3240:	ff 15 e8 10 ee 77    	call   *0x77ee10e8
77ed3246:	c7 45 08 78 00 00 00 	movl   $0x78,0x8(%ebp)
77ed324d:	83 c4 10             	add    $0x10,%esp
77ed3250:	c9                   	leave  
77ed3251:	e9 ba 66 00 00       	jmp    77ed9910 <_SetLastError@4>
77ed3256:	8d 76 00             	lea    0x0(%esi),%esi
77ed3259:	8d bc 27 00 00 00 00 	lea    0x0(%edi),%edi

77ed3260 <_GetTextExtentExPointI@28>:
77ed3260:	55                   	push   %ebp
77ed3261:	89 e5                	mov    %esp,%ebp
77ed3263:	83 ec 10             	sub    $0x10,%esp
77ed3266:	68 30 ab ed 77       	push   $0x77edab30
77ed326b:	68 20 a0 ed 77       	push   $0x77eda020
77ed3270:	ff 15 e8 10 ee 77    	call   *0x77ee10e8
77ed3276:	c7 04 24 78 00 00 00 	movl   $0x78,(%esp)
77ed327d:	e8 8e 66 00 00       	call   77ed9910 <_SetLastError@4>
77ed3282:	31 c0                	xor    %eax,%eax
77ed3284:	c9                   	leave  
77ed3285:	c2 1c 00             	ret    $0x1c
77ed3288:	90                   	nop    
77ed3289:	8d b4 26 00 00 00 00 	lea    0x0(%esi),%esi

77ed3290 <_GetTextExtentPointI@16>:
77ed3290:	55                   	push   %ebp
77ed3291:	89 e5                	mov    %esp,%ebp
77ed3293:	83 ec 10             	sub    $0x10,%esp
77ed3296:	68 46 ab ed 77       	push   $0x77edab46
77ed329b:	68 20 a0 ed 77       	push   $0x77eda020
77ed32a0:	ff 15 e8 10 ee 77    	call   *0x77ee10e8
77ed32a6:	c7 04 24 78 00 00 00 	movl   $0x78,(%esp)
77ed32ad:	e8 5e 66 00 00       	call   77ed9910 <_SetLastError@4>
77ed32b2:	31 c0                	xor    %eax,%eax
77ed32b4:	c9                   	leave  
77ed32b5:	c2 10 00             	ret    $0x10
77ed32b8:	90                   	nop    
77ed32b9:	8d b4 26 00 00 00 00 	lea    0x0(%esi),%esi

77ed32c0 <_GdiFullscreenControl@20>:
77ed32c0:	55                   	push   %ebp
77ed32c1:	89 e5                	mov    %esp,%ebp
77ed32c3:	83 ec 10             	sub    $0x10,%esp
77ed32c6:	68 5a ab ed 77       	push   $0x77edab5a
77ed32cb:	68 20 a0 ed 77       	push   $0x77eda020
77ed32d0:	ff 15 e8 10 ee 77    	call   *0x77ee10e8
77ed32d6:	c7 04 24 78 00 00 00 	movl   $0x78,(%esp)
77ed32dd:	e8 2e 66 00 00       	call   77ed9910 <_SetLastError@4>
77ed32e2:	31 c0                	xor    %eax,%eax
77ed32e4:	c9                   	leave  
77ed32e5:	c2 14 00             	ret    $0x14
77ed32e8:	90                   	nop    
77ed32e9:	8d b4 26 00 00 00 00 	lea    0x0(%esi),%esi

77ed32f0 <_GdiQueryFonts@12>:
77ed32f0:	55                   	push   %ebp
77ed32f1:	89 e5                	mov    %esp,%ebp
77ed32f3:	83 ec 10             	sub    $0x10,%esp
77ed32f6:	68 6f ab ed 77       	push   $0x77edab6f
77ed32fb:	68 20 a0 ed 77       	push   $0x77eda020
77ed3300:	ff 15 e8 10 ee 77    	call   *0x77ee10e8
77ed3306:	c7 04 24 78 00 00 00 	movl   $0x78,(%esp)
77ed330d:	e8 fe 65 00 00       	call   77ed9910 <_SetLastError@4>
77ed3312:	31 c0                	xor    %eax,%eax
77ed3314:	c9                   	leave  
77ed3315:	c2 0c 00             	ret    $0xc
77ed3318:	90                   	nop    
77ed3319:	8d b4 26 00 00 00 00 	lea    0x0(%esi),%esi

77ed3320 <_GdiRealizationInfo@8>:
77ed3320:	55                   	push   %ebp
77ed3321:	89 e5                	mov    %esp,%ebp
77ed3323:	83 ec 10             	sub    $0x10,%esp
77ed3326:	68 7d ab ed 77       	push   $0x77edab7d
77ed332b:	68 20 a0 ed 77       	push   $0x77eda020
77ed3330:	ff 15 e8 10 ee 77    	call   *0x77ee10e8
77ed3336:	c7 04 24 78 00 00 00 	movl   $0x78,(%esp)
77ed333d:	e8 ce 65 00 00       	call   77ed9910 <_SetLastError@4>
77ed3342:	31 c0                	xor    %eax,%eax
77ed3344:	c9                   	leave  
77ed3345:	c2 08 00             	ret    $0x8
77ed3348:	90                   	nop    
77ed3349:	8d b4 26 00 00 00 00 	lea    0x0(%esi),%esi

77ed3350 <_GetCharWidthInfo@8>:
77ed3350:	55                   	push   %ebp
77ed3351:	89 e5                	mov    %esp,%ebp
77ed3353:	83 ec 10             	sub    $0x10,%esp
77ed3356:	68 90 ab ed 77       	push   $0x77edab90
77ed335b:	68 20 a0 ed 77       	push   $0x77eda020
77ed3360:	ff 15 e8 10 ee 77    	call   *0x77ee10e8
77ed3366:	c7 04 24 78 00 00 00 	movl   $0x78,(%esp)
77ed336d:	e8 9e 65 00 00       	call   77ed9910 <_SetLastError@4>
77ed3372:	31 c0                	xor    %eax,%eax
77ed3374:	c9                   	leave  
77ed3375:	c2 08 00             	ret    $0x8
77ed3378:	90                   	nop    
77ed3379:	8d b4 26 00 00 00 00 	lea    0x0(%esi),%esi

77ed3380 <_GetETM@8>:
77ed3380:	55                   	push   %ebp
77ed3381:	89 e5                	mov    %esp,%ebp
77ed3383:	83 ec 10             	sub    $0x10,%esp
77ed3386:	68 a1 ab ed 77       	push   $0x77edaba1
77ed338b:	68 20 a0 ed 77       	push   $0x77eda020
77ed3390:	ff 15 e8 10 ee 77    	call   *0x77ee10e8
77ed3396:	c7 04 24 78 00 00 00 	movl   $0x78,(%esp)
77ed339d:	e8 6e 65 00 00       	call   77ed9910 <_SetLastError@4>
77ed33a2:	31 c0                	xor    %eax,%eax
77ed33a4:	c9                   	leave  
77ed33a5:	c2 08 00             	ret    $0x8
77ed33a8:	90                   	nop    
77ed33a9:	8d b4 26 00 00 00 00 	lea    0x0(%esi),%esi

77ed33b0 <_GdiAddGlsRecord@16>:
77ed33b0:	55                   	push   %ebp
77ed33b1:	89 e5                	mov    %esp,%ebp
77ed33b3:	83 ec 10             	sub    $0x10,%esp
77ed33b6:	68 a8 ab ed 77       	push   $0x77edaba8
77ed33bb:	68 20 a0 ed 77       	push   $0x77eda020
77ed33c0:	ff 15 e8 10 ee 77    	call   *0x77ee10e8
77ed33c6:	c7 04 24 78 00 00 00 	movl   $0x78,(%esp)
77ed33cd:	e8 3e 65 00 00       	call   77ed9910 <_SetLastError@4>
77ed33d2:	31 c0                	xor    %eax,%eax
77ed33d4:	c9                   	leave  
77ed33d5:	c2 10 00             	ret    $0x10
77ed33d8:	90                   	nop    
77ed33d9:	8d b4 26 00 00 00 00 	lea    0x0(%esi),%esi

77ed33e0 <_GdiConvertMetaFilePict@4>:
77ed33e0:	55                   	push   %ebp
77ed33e1:	89 e5                	mov    %esp,%ebp
77ed33e3:	83 ec 10             	sub    $0x10,%esp
77ed33e6:	68 b8 ab ed 77       	push   $0x77edabb8
77ed33eb:	68 20 a0 ed 77       	push   $0x77eda020
77ed33f0:	ff 15 e8 10 ee 77    	call   *0x77ee10e8
77ed33f6:	c7 04 24 78 00 00 00 	movl   $0x78,(%esp)
77ed33fd:	e8 0e 65 00 00       	call   77ed9910 <_SetLastError@4>
77ed3402:	31 c0                	xor    %eax,%eax
77ed3404:	c9                   	leave  
77ed3405:	c2 04 00             	ret    $0x4
77ed3408:	90                   	nop    
77ed3409:	8d b4 26 00 00 00 00 	lea    0x0(%esi),%esi

77ed3410 <_GdiConvertToDevmodeW@4>:
77ed3410:	55                   	push   %ebp
77ed3411:	89 e5                	mov    %esp,%ebp
77ed3413:	83 ec 10             	sub    $0x10,%esp
77ed3416:	68 cf ab ed 77       	push   $0x77edabcf
77ed341b:	68 20 a0 ed 77       	push   $0x77eda020
77ed3420:	ff 15 e8 10 ee 77    	call   *0x77ee10e8
77ed3426:	c7 04 24 78 00 00 00 	movl   $0x78,(%esp)
77ed342d:	e8 de 64 00 00       	call   77ed9910 <_SetLastError@4>
77ed3432:	31 c0                	xor    %eax,%eax
77ed3434:	c9                   	leave  
77ed3435:	c2 04 00             	ret    $0x4
77ed3438:	90                   	nop    
77ed3439:	8d b4 26 00 00 00 00 	lea    0x0(%esi),%esi

77ed3440 <_GdiCreateLocalEnhMetaFile@4>:
77ed3440:	55                   	push   %ebp
77ed3441:	89 e5                	mov    %esp,%ebp
77ed3443:	83 ec 10             	sub    $0x10,%esp
77ed3446:	68 e4 ab ed 77       	push   $0x77edabe4
77ed344b:	68 20 a0 ed 77       	push   $0x77eda020
77ed3450:	ff 15 e8 10 ee 77    	call   *0x77ee10e8
77ed3456:	c7 04 24 78 00 00 00 	movl   $0x78,(%esp)
77ed345d:	e8 ae 64 00 00       	call   77ed9910 <_SetLastError@4>
77ed3462:	31 c0                	xor    %eax,%eax
77ed3464:	c9                   	leave  
77ed3465:	c2 04 00             	ret    $0x4
77ed3468:	90                   	nop    
77ed3469:	8d b4 26 00 00 00 00 	lea    0x0(%esi),%esi

77ed3470 <_GdiCreateLocalMetaFilePict@4>:
77ed3470:	55                   	push   %ebp
77ed3471:	89 e5                	mov    %esp,%ebp
77ed3473:	83 ec 10             	sub    $0x10,%esp
77ed3476:	68 fe ab ed 77       	push   $0x77edabfe
77ed347b:	68 20 a0 ed 77       	push   $0x77eda020
77ed3480:	ff 15 e8 10 ee 77    	call   *0x77ee10e8
77ed3486:	c7 04 24 78 00 00 00 	movl   $0x78,(%esp)
77ed348d:	e8 7e 64 00 00       	call   77ed9910 <_SetLastError@4>
77ed3492:	31 c0                	xor    %eax,%eax
77ed3494:	c9                   	leave  
77ed3495:	c2 04 00             	ret    $0x4
77ed3498:	90                   	nop    
77ed3499:	8d b4 26 00 00 00 00 	lea    0x0(%esi),%esi

77ed34a0 <_GdiGetCharDimensions@12>:
77ed34a0:	55                   	push   %ebp
77ed34a1:	89 e5                	mov    %esp,%ebp
77ed34a3:	83 ec 10             	sub    $0x10,%esp
77ed34a6:	68 19 ac ed 77       	push   $0x77edac19
77ed34ab:	68 20 a0 ed 77       	push   $0x77eda020
77ed34b0:	ff 15 e8 10 ee 77    	call   *0x77ee10e8
77ed34b6:	c7 04 24 78 00 00 00 	movl   $0x78,(%esp)
77ed34bd:	e8 4e 64 00 00       	call   77ed9910 <_SetLastError@4>
77ed34c2:	31 c0                	xor    %eax,%eax
77ed34c4:	c9                   	leave  
77ed34c5:	c2 0c 00             	ret    $0xc
77ed34c8:	90                   	nop    
77ed34c9:	8d b4 26 00 00 00 00 	lea    0x0(%esi),%esi

77ed34d0 <_GdiGetSpoolFileHandle@12>:
77ed34d0:	55                   	push   %ebp
77ed34d1:	89 e5                	mov    %esp,%ebp
77ed34d3:	83 ec 10             	sub    $0x10,%esp
77ed34d6:	68 2e ac ed 77       	push   $0x77edac2e
77ed34db:	68 20 a0 ed 77       	push   $0x77eda020
77ed34e0:	ff 15 e8 10 ee 77    	call   *0x77ee10e8
77ed34e6:	c7 04 24 78 00 00 00 	movl   $0x78,(%esp)
77ed34ed:	e8 1e 64 00 00       	call   77ed9910 <_SetLastError@4>
77ed34f2:	31 c0                	xor    %eax,%eax
77ed34f4:	c9                   	leave  
77ed34f5:	c2 0c 00             	ret    $0xc
77ed34f8:	90                   	nop    
77ed34f9:	8d b4 26 00 00 00 00 	lea    0x0(%esi),%esi

77ed3500 <_GdiDeleteSpoolFileHandle@4>:
77ed3500:	55                   	push   %ebp
77ed3501:	89 e5                	mov    %esp,%ebp
77ed3503:	83 ec 10             	sub    $0x10,%esp
77ed3506:	68 44 ac ed 77       	push   $0x77edac44
77ed350b:	68 20 a0 ed 77       	push   $0x77eda020
77ed3510:	ff 15 e8 10 ee 77    	call   *0x77ee10e8
77ed3516:	c7 04 24 78 00 00 00 	movl   $0x78,(%esp)
77ed351d:	e8 ee 63 00 00       	call   77ed9910 <_SetLastError@4>
77ed3522:	31 c0                	xor    %eax,%eax
77ed3524:	c9                   	leave  
77ed3525:	c2 04 00             	ret    $0x4
77ed3528:	90                   	nop    
77ed3529:	8d b4 26 00 00 00 00 	lea    0x0(%esi),%esi

77ed3530 <_GdiGetPageCount@4>:
77ed3530:	55                   	push   %ebp
77ed3531:	89 e5                	mov    %esp,%ebp
77ed3533:	83 ec 10             	sub    $0x10,%esp
77ed3536:	68 5d ac ed 77       	push   $0x77edac5d
77ed353b:	68 20 a0 ed 77       	push   $0x77eda020
77ed3540:	ff 15 e8 10 ee 77    	call   *0x77ee10e8
77ed3546:	c7 04 24 78 00 00 00 	movl   $0x78,(%esp)
77ed354d:	e8 be 63 00 00       	call   77ed9910 <_SetLastError@4>
77ed3552:	31 c0                	xor    %eax,%eax
77ed3554:	c9                   	leave  
77ed3555:	c2 04 00             	ret    $0x4
77ed3558:	90                   	nop    
77ed3559:	8d b4 26 00 00 00 00 	lea    0x0(%esi),%esi

77ed3560 <_GdiGetDC@4>:
77ed3560:	55                   	push   %ebp
77ed3561:	89 e5                	mov    %esp,%ebp
77ed3563:	83 ec 10             	sub    $0x10,%esp
77ed3566:	68 6d ac ed 77       	push   $0x77edac6d
77ed356b:	68 20 a0 ed 77       	push   $0x77eda020
77ed3570:	ff 15 e8 10 ee 77    	call   *0x77ee10e8
77ed3576:	c7 04 24 78 00 00 00 	movl   $0x78,(%esp)
77ed357d:	e8 8e 63 00 00       	call   77ed9910 <_SetLastError@4>
77ed3582:	31 c0                	xor    %eax,%eax
77ed3584:	c9                   	leave  
77ed3585:	c2 04 00             	ret    $0x4
77ed3588:	90                   	nop    
77ed3589:	8d b4 26 00 00 00 00 	lea    0x0(%esi),%esi

77ed3590 <_GdiGetPageHandle@12>:
77ed3590:	55                   	push   %ebp
77ed3591:	89 e5                	mov    %esp,%ebp
77ed3593:	83 ec 10             	sub    $0x10,%esp
77ed3596:	68 76 ac ed 77       	push   $0x77edac76
77ed359b:	68 20 a0 ed 77       	push   $0x77eda020
77ed35a0:	ff 15 e8 10 ee 77    	call   *0x77ee10e8
77ed35a6:	c7 04 24 78 00 00 00 	movl   $0x78,(%esp)
77ed35ad:	e8 5e 63 00 00       	call   77ed9910 <_SetLastError@4>
77ed35b2:	31 c0                	xor    %eax,%eax
77ed35b4:	c9                   	leave  
77ed35b5:	c2 0c 00             	ret    $0xc
77ed35b8:	90                   	nop    
77ed35b9:	8d b4 26 00 00 00 00 	lea    0x0(%esi),%esi

77ed35c0 <_GdiStartDocEMF@8>:
77ed35c0:	55                   	push   %ebp
77ed35c1:	89 e5                	mov    %esp,%ebp
77ed35c3:	83 ec 10             	sub    $0x10,%esp
77ed35c6:	68 87 ac ed 77       	push   $0x77edac87
77ed35cb:	68 20 a0 ed 77       	push   $0x77eda020
77ed35d0:	ff 15 e8 10 ee 77    	call   *0x77ee10e8
77ed35d6:	c7 04 24 78 00 00 00 	movl   $0x78,(%esp)
77ed35dd:	e8 2e 63 00 00       	call   77ed9910 <_SetLastError@4>
77ed35e2:	31 c0                	xor    %eax,%eax
77ed35e4:	c9                   	leave  
77ed35e5:	c2 08 00             	ret    $0x8
77ed35e8:	90                   	nop    
77ed35e9:	8d b4 26 00 00 00 00 	lea    0x0(%esi),%esi

77ed35f0 <_GdiStartPageEMF@4>:
77ed35f0:	55                   	push   %ebp
77ed35f1:	89 e5                	mov    %esp,%ebp
77ed35f3:	83 ec 10             	sub    $0x10,%esp
77ed35f6:	68 96 ac ed 77       	push   $0x77edac96
77ed35fb:	68 20 a0 ed 77       	push   $0x77eda020
77ed3600:	ff 15 e8 10 ee 77    	call   *0x77ee10e8
77ed3606:	c7 04 24 78 00 00 00 	movl   $0x78,(%esp)
77ed360d:	e8 fe 62 00 00       	call   77ed9910 <_SetLastError@4>
77ed3612:	31 c0                	xor    %eax,%eax
77ed3614:	c9                   	leave  
77ed3615:	c2 04 00             	ret    $0x4
77ed3618:	90                   	nop    
77ed3619:	8d b4 26 00 00 00 00 	lea    0x0(%esi),%esi

77ed3620 <_GdiPlayPageEMF@20>:
77ed3620:	55                   	push   %ebp
77ed3621:	89 e5                	mov    %esp,%ebp
77ed3623:	83 ec 10             	sub    $0x10,%esp
77ed3626:	68 a6 ac ed 77       	push   $0x77edaca6
77ed362b:	68 20 a0 ed 77       	push   $0x77eda020
77ed3630:	ff 15 e8 10 ee 77    	call   *0x77ee10e8
77ed3636:	c7 04 24 78 00 00 00 	movl   $0x78,(%esp)
77ed363d:	e8 ce 62 00 00       	call   77ed9910 <_SetLastError@4>
77ed3642:	31 c0                	xor    %eax,%eax
77ed3644:	c9                   	leave  
77ed3645:	c2 14 00             	ret    $0x14
77ed3648:	90                   	nop    
77ed3649:	8d b4 26 00 00 00 00 	lea    0x0(%esi),%esi

77ed3650 <_GdiEndPageEMF@8>:
77ed3650:	55                   	push   %ebp
77ed3651:	89 e5                	mov    %esp,%ebp
77ed3653:	83 ec 10             	sub    $0x10,%esp
77ed3656:	68 b5 ac ed 77       	push   $0x77edacb5
77ed365b:	68 20 a0 ed 77       	push   $0x77eda020
77ed3660:	ff 15 e8 10 ee 77    	call   *0x77ee10e8
77ed3666:	c7 04 24 78 00 00 00 	movl   $0x78,(%esp)
77ed366d:	e8 9e 62 00 00       	call   77ed9910 <_SetLastError@4>
77ed3672:	31 c0                	xor    %eax,%eax
77ed3674:	c9                   	leave  
77ed3675:	c2 08 00             	ret    $0x8
77ed3678:	90                   	nop    
77ed3679:	8d b4 26 00 00 00 00 	lea    0x0(%esi),%esi

77ed3680 <_GdiEndDocEMF@4>:
77ed3680:	55                   	push   %ebp
77ed3681:	89 e5                	mov    %esp,%ebp
77ed3683:	83 ec 10             	sub    $0x10,%esp
77ed3686:	68 c3 ac ed 77       	push   $0x77edacc3
77ed368b:	68 20 a0 ed 77       	push   $0x77eda020
77ed3690:	ff 15 e8 10 ee 77    	call   *0x77ee10e8
77ed3696:	c7 04 24 78 00 00 00 	movl   $0x78,(%esp)
77ed369d:	e8 6e 62 00 00       	call   77ed9910 <_SetLastError@4>
77ed36a2:	31 c0                	xor    %eax,%eax
77ed36a4:	c9                   	leave  
77ed36a5:	c2 04 00             	ret    $0x4
77ed36a8:	90                   	nop    
77ed36a9:	8d b4 26 00 00 00 00 	lea    0x0(%esi),%esi

77ed36b0 <_GdiGetDevmodeForPage@16>:
77ed36b0:	55                   	push   %ebp
77ed36b1:	89 e5                	mov    %esp,%ebp
77ed36b3:	83 ec 10             	sub    $0x10,%esp
77ed36b6:	68 d0 ac ed 77       	push   $0x77edacd0
77ed36bb:	68 20 a0 ed 77       	push   $0x77eda020
77ed36c0:	ff 15 e8 10 ee 77    	call   *0x77ee10e8
77ed36c6:	c7 04 24 78 00 00 00 	movl   $0x78,(%esp)
77ed36cd:	e8 3e 62 00 00       	call   77ed9910 <_SetLastError@4>
77ed36d2:	31 c0                	xor    %eax,%eax
77ed36d4:	c9                   	leave  
77ed36d5:	c2 10 00             	ret    $0x10
77ed36d8:	90                   	nop    
77ed36d9:	8d b4 26 00 00 00 00 	lea    0x0(%esi),%esi

77ed36e0 <_GdiResetDCEMF@8>:
77ed36e0:	55                   	push   %ebp
77ed36e1:	89 e5                	mov    %esp,%ebp
77ed36e3:	83 ec 10             	sub    $0x10,%esp
77ed36e6:	68 e5 ac ed 77       	push   $0x77edace5
77ed36eb:	68 20 a0 ed 77       	push   $0x77eda020
77ed36f0:	ff 15 e8 10 ee 77    	call   *0x77ee10e8
77ed36f6:	c7 04 24 78 00 00 00 	movl   $0x78,(%esp)
77ed36fd:	e8 0e 62 00 00       	call   77ed9910 <_SetLastError@4>
77ed3702:	31 c0                	xor    %eax,%eax
77ed3704:	c9                   	leave  
77ed3705:	c2 08 00             	ret    $0x8
77ed3708:	90                   	nop    
77ed3709:	8d b4 26 00 00 00 00 	lea    0x0(%esi),%esi

77ed3710 <_BRUSHOBJ_hGetColorTransform@4>:
77ed3710:	55                   	push   %ebp
77ed3711:	89 e5                	mov    %esp,%ebp
77ed3713:	83 ec 10             	sub    $0x10,%esp
77ed3716:	68 f3 ac ed 77       	push   $0x77edacf3
77ed371b:	68 20 a0 ed 77       	push   $0x77eda020
77ed3720:	ff 15 e8 10 ee 77    	call   *0x77ee10e8
77ed3726:	c7 04 24 78 00 00 00 	movl   $0x78,(%esp)
77ed372d:	e8 de 61 00 00       	call   77ed9910 <_SetLastError@4>
77ed3732:	31 c0                	xor    %eax,%eax
77ed3734:	c9                   	leave  
77ed3735:	c2 04 00             	ret    $0x4
77ed3738:	90                   	nop    
77ed3739:	8d b4 26 00 00 00 00 	lea    0x0(%esi),%esi

77ed3740 <_BRUSHOBJ_pvAllocRbrush@8>:
77ed3740:	55                   	push   %ebp
77ed3741:	89 e5                	mov    %esp,%ebp
77ed3743:	83 ec 10             	sub    $0x10,%esp
77ed3746:	68 0f ad ed 77       	push   $0x77edad0f
77ed374b:	68 20 a0 ed 77       	push   $0x77eda020
77ed3750:	ff 15 e8 10 ee 77    	call   *0x77ee10e8
77ed3756:	c7 04 24 78 00 00 00 	movl   $0x78,(%esp)
77ed375d:	e8 ae 61 00 00       	call   77ed9910 <_SetLastError@4>
77ed3762:	31 c0                	xor    %eax,%eax
77ed3764:	c9                   	leave  
77ed3765:	c2 08 00             	ret    $0x8
77ed3768:	90                   	nop    
77ed3769:	8d b4 26 00 00 00 00 	lea    0x0(%esi),%esi

77ed3770 <_BRUSHOBJ_pvGetRbrush@4>:
77ed3770:	55                   	push   %ebp
77ed3771:	89 e5                	mov    %esp,%ebp
77ed3773:	83 ec 10             	sub    $0x10,%esp
77ed3776:	68 26 ad ed 77       	push   $0x77edad26
77ed377b:	68 20 a0 ed 77       	push   $0x77eda020
77ed3780:	ff 15 e8 10 ee 77    	call   *0x77ee10e8
77ed3786:	c7 04 24 78 00 00 00 	movl   $0x78,(%esp)
77ed378d:	e8 7e 61 00 00       	call   77ed9910 <_SetLastError@4>
77ed3792:	31 c0                	xor    %eax,%eax
77ed3794:	c9                   	leave  
77ed3795:	c2 04 00             	ret    $0x4
77ed3798:	90                   	nop    
77ed3799:	8d b4 26 00 00 00 00 	lea    0x0(%esi),%esi

77ed37a0 <_BRUSHOBJ_ulGetBrushColor@4>:
77ed37a0:	55                   	push   %ebp
77ed37a1:	89 e5                	mov    %esp,%ebp
77ed37a3:	83 ec 10             	sub    $0x10,%esp
77ed37a6:	68 3b ad ed 77       	push   $0x77edad3b
77ed37ab:	68 20 a0 ed 77       	push   $0x77eda020
77ed37b0:	ff 15 e8 10 ee 77    	call   *0x77ee10e8
77ed37b6:	c7 04 24 78 00 00 00 	movl   $0x78,(%esp)
77ed37bd:	e8 4e 61 00 00       	call   77ed9910 <_SetLastError@4>
77ed37c2:	31 c0                	xor    %eax,%eax
77ed37c4:	c9                   	leave  
77ed37c5:	c2 04 00             	ret    $0x4
77ed37c8:	90                   	nop    
77ed37c9:	8d b4 26 00 00 00 00 	lea    0x0(%esi),%esi

77ed37d0 <_CLIPOBJ_bEnum@12>:
77ed37d0:	55                   	push   %ebp
77ed37d1:	89 e5                	mov    %esp,%ebp
77ed37d3:	83 ec 10             	sub    $0x10,%esp
77ed37d6:	68 54 ad ed 77       	push   $0x77edad54
77ed37db:	68 20 a0 ed 77       	push   $0x77eda020
77ed37e0:	ff 15 e8 10 ee 77    	call   *0x77ee10e8
77ed37e6:	c7 04 24 78 00 00 00 	movl   $0x78,(%esp)
77ed37ed:	e8 1e 61 00 00       	call   77ed9910 <_SetLastError@4>
77ed37f2:	31 c0                	xor    %eax,%eax
77ed37f4:	c9                   	leave  
77ed37f5:	c2 0c 00             	ret    $0xc
77ed37f8:	90                   	nop    
77ed37f9:	8d b4 26 00 00 00 00 	lea    0x0(%esi),%esi

77ed3800 <_CLIPOBJ_cEnumStart@20>:
77ed3800:	55                   	push   %ebp
77ed3801:	89 e5                	mov    %esp,%ebp
77ed3803:	83 ec 10             	sub    $0x10,%esp
77ed3806:	68 62 ad ed 77       	push   $0x77edad62
77ed380b:	68 20 a0 ed 77       	push   $0x77eda020
77ed3810:	ff 15 e8 10 ee 77    	call   *0x77ee10e8
77ed3816:	c7 04 24 78 00 00 00 	movl   $0x78,(%esp)
77ed381d:	e8 ee 60 00 00       	call   77ed9910 <_SetLastError@4>
77ed3822:	31 c0                	xor    %eax,%eax
77ed3824:	c9                   	leave  
77ed3825:	c2 14 00             	ret    $0x14
77ed3828:	90                   	nop    
77ed3829:	8d b4 26 00 00 00 00 	lea    0x0(%esi),%esi

77ed3830 <_CLIPOBJ_ppoGetPath@4>:
77ed3830:	55                   	push   %ebp
77ed3831:	89 e5                	mov    %esp,%ebp
77ed3833:	83 ec 10             	sub    $0x10,%esp
77ed3836:	68 75 ad ed 77       	push   $0x77edad75
77ed383b:	68 20 a0 ed 77       	push   $0x77eda020
77ed3840:	ff 15 e8 10 ee 77    	call   *0x77ee10e8
77ed3846:	c7 04 24 78 00 00 00 	movl   $0x78,(%esp)
77ed384d:	e8 be 60 00 00       	call   77ed9910 <_SetLastError@4>
77ed3852:	31 c0                	xor    %eax,%eax
77ed3854:	c9                   	leave  
77ed3855:	c2 04 00             	ret    $0x4
77ed3858:	90                   	nop    
77ed3859:	8d b4 26 00 00 00 00 	lea    0x0(%esi),%esi

77ed3860 <_EngAcquireSemaphore@4>:
77ed3860:	55                   	push   %ebp
77ed3861:	89 e5                	mov    %esp,%ebp
77ed3863:	83 ec 10             	sub    $0x10,%esp
77ed3866:	68 88 ad ed 77       	push   $0x77edad88
77ed386b:	68 20 a0 ed 77       	push   $0x77eda020
77ed3870:	ff 15 e8 10 ee 77    	call   *0x77ee10e8
77ed3876:	c7 45 08 78 00 00 00 	movl   $0x78,0x8(%ebp)
77ed387d:	83 c4 10             	add    $0x10,%esp
77ed3880:	c9                   	leave  
77ed3881:	e9 8a 60 00 00       	jmp    77ed9910 <_SetLastError@4>
77ed3886:	8d 76 00             	lea    0x0(%esi),%esi
77ed3889:	8d bc 27 00 00 00 00 	lea    0x0(%edi),%edi

77ed3890 <_EngAlphaBlend@28>:
77ed3890:	55                   	push   %ebp
77ed3891:	89 e5                	mov    %esp,%ebp
77ed3893:	83 ec 10             	sub    $0x10,%esp
77ed3896:	68 9c ad ed 77       	push   $0x77edad9c
77ed389b:	68 20 a0 ed 77       	push   $0x77eda020
77ed38a0:	ff 15 e8 10 ee 77    	call   *0x77ee10e8
77ed38a6:	c7 04 24 78 00 00 00 	movl   $0x78,(%esp)
77ed38ad:	e8 5e 60 00 00       	call   77ed9910 <_SetLastError@4>
77ed38b2:	31 c0                	xor    %eax,%eax
77ed38b4:	c9                   	leave  
77ed38b5:	c2 1c 00             	ret    $0x1c
77ed38b8:	90                   	nop    
77ed38b9:	8d b4 26 00 00 00 00 	lea    0x0(%esi),%esi

77ed38c0 <_EngAssociateSurface@12>:
77ed38c0:	55                   	push   %ebp
77ed38c1:	89 e5                	mov    %esp,%ebp
77ed38c3:	83 ec 10             	sub    $0x10,%esp
77ed38c6:	68 aa ad ed 77       	push   $0x77edadaa
77ed38cb:	68 20 a0 ed 77       	push   $0x77eda020
77ed38d0:	ff 15 e8 10 ee 77    	call   *0x77ee10e8
77ed38d6:	c7 04 24 78 00 00 00 	movl   $0x78,(%esp)
77ed38dd:	e8 2e 60 00 00       	call   77ed9910 <_SetLastError@4>
77ed38e2:	31 c0                	xor    %eax,%eax
77ed38e4:	c9                   	leave  
77ed38e5:	c2 0c 00             	ret    $0xc
77ed38e8:	90                   	nop    
77ed38e9:	8d b4 26 00 00 00 00 	lea    0x0(%esi),%esi

77ed38f0 <_EngBitBlt@44>:
77ed38f0:	55                   	push   %ebp
77ed38f1:	89 e5                	mov    %esp,%ebp
77ed38f3:	83 ec 10             	sub    $0x10,%esp
77ed38f6:	68 be ad ed 77       	push   $0x77edadbe
77ed38fb:	68 20 a0 ed 77       	push   $0x77eda020
77ed3900:	ff 15 e8 10 ee 77    	call   *0x77ee10e8
77ed3906:	c7 04 24 78 00 00 00 	movl   $0x78,(%esp)
77ed390d:	e8 fe 5f 00 00       	call   77ed9910 <_SetLastError@4>
77ed3912:	31 c0                	xor    %eax,%eax
77ed3914:	c9                   	leave  
77ed3915:	c2 2c 00             	ret    $0x2c
77ed3918:	90                   	nop    
77ed3919:	8d b4 26 00 00 00 00 	lea    0x0(%esi),%esi

77ed3920 <_EngCheckAbort@4>:
77ed3920:	55                   	push   %ebp
77ed3921:	89 e5                	mov    %esp,%ebp
77ed3923:	83 ec 10             	sub    $0x10,%esp
77ed3926:	68 c8 ad ed 77       	push   $0x77edadc8
77ed392b:	68 20 a0 ed 77       	push   $0x77eda020
77ed3930:	ff 15 e8 10 ee 77    	call   *0x77ee10e8
77ed3936:	c7 04 24 78 00 00 00 	movl   $0x78,(%esp)
77ed393d:	e8 ce 5f 00 00       	call   77ed9910 <_SetLastError@4>
77ed3942:	31 c0                	xor    %eax,%eax
77ed3944:	c9                   	leave  
77ed3945:	c2 04 00             	ret    $0x4
77ed3948:	90                   	nop    
77ed3949:	8d b4 26 00 00 00 00 	lea    0x0(%esi),%esi

77ed3950 <_EngComputeGlyphSet@12>:
77ed3950:	55                   	push   %ebp
77ed3951:	89 e5                	mov    %esp,%ebp
77ed3953:	83 ec 10             	sub    $0x10,%esp
77ed3956:	68 d6 ad ed 77       	push   $0x77edadd6
77ed395b:	68 20 a0 ed 77       	push   $0x77eda020
77ed3960:	ff 15 e8 10 ee 77    	call   *0x77ee10e8
77ed3966:	c7 04 24 78 00 00 00 	movl   $0x78,(%esp)
77ed396d:	e8 9e 5f 00 00       	call   77ed9910 <_SetLastError@4>
77ed3972:	31 c0                	xor    %eax,%eax
77ed3974:	c9                   	leave  
77ed3975:	c2 0c 00             	ret    $0xc
77ed3978:	90                   	nop    
77ed3979:	8d b4 26 00 00 00 00 	lea    0x0(%esi),%esi

77ed3980 <_EngCopyBits@24>:
77ed3980:	55                   	push   %ebp
77ed3981:	89 e5                	mov    %esp,%ebp
77ed3983:	83 ec 10             	sub    $0x10,%esp
77ed3986:	68 e9 ad ed 77       	push   $0x77edade9
77ed398b:	68 20 a0 ed 77       	push   $0x77eda020
77ed3990:	ff 15 e8 10 ee 77    	call   *0x77ee10e8
77ed3996:	c7 04 24 78 00 00 00 	movl   $0x78,(%esp)
77ed399d:	e8 6e 5f 00 00       	call   77ed9910 <_SetLastError@4>
77ed39a2:	31 c0                	xor    %eax,%eax
77ed39a4:	c9                   	leave  
77ed39a5:	c2 18 00             	ret    $0x18
77ed39a8:	90                   	nop    
77ed39a9:	8d b4 26 00 00 00 00 	lea    0x0(%esi),%esi

77ed39b0 <_EngCreateBitmap@24>:
77ed39b0:	55                   	push   %ebp
77ed39b1:	89 e5                	mov    %esp,%ebp
77ed39b3:	83 ec 10             	sub    $0x10,%esp
77ed39b6:	68 f5 ad ed 77       	push   $0x77edadf5
77ed39bb:	68 20 a0 ed 77       	push   $0x77eda020
77ed39c0:	ff 15 e8 10 ee 77    	call   *0x77ee10e8
77ed39c6:	c7 04 24 78 00 00 00 	movl   $0x78,(%esp)
77ed39cd:	e8 3e 5f 00 00       	call   77ed9910 <_SetLastError@4>
77ed39d2:	31 c0                	xor    %eax,%eax
77ed39d4:	c9                   	leave  
77ed39d5:	c2 18 00             	ret    $0x18
77ed39d8:	90                   	nop    
77ed39d9:	8d b4 26 00 00 00 00 	lea    0x0(%esi),%esi

77ed39e0 <_EngCreateClip@0>:
77ed39e0:	55                   	push   %ebp
77ed39e1:	89 e5                	mov    %esp,%ebp
77ed39e3:	83 ec 10             	sub    $0x10,%esp
77ed39e6:	68 05 ae ed 77       	push   $0x77edae05
77ed39eb:	68 20 a0 ed 77       	push   $0x77eda020
77ed39f0:	ff 15 e8 10 ee 77    	call   *0x77ee10e8
77ed39f6:	c7 04 24 78 00 00 00 	movl   $0x78,(%esp)
77ed39fd:	e8 0e 5f 00 00       	call   77ed9910 <_SetLastError@4>
77ed3a02:	31 c0                	xor    %eax,%eax
77ed3a04:	c9                   	leave  
77ed3a05:	c3                   	ret    
77ed3a06:	8d 76 00             	lea    0x0(%esi),%esi
77ed3a09:	8d bc 27 00 00 00 00 	lea    0x0(%edi),%edi

77ed3a10 <_EngCreateDeviceBitmap@16>:
77ed3a10:	55                   	push   %ebp
77ed3a11:	89 e5                	mov    %esp,%ebp
77ed3a13:	83 ec 10             	sub    $0x10,%esp
77ed3a16:	68 13 ae ed 77       	push   $0x77edae13
77ed3a1b:	68 20 a0 ed 77       	push   $0x77eda020
77ed3a20:	ff 15 e8 10 ee 77    	call   *0x77ee10e8
77ed3a26:	c7 04 24 78 00 00 00 	movl   $0x78,(%esp)
77ed3a2d:	e8 de 5e 00 00       	call   77ed9910 <_SetLastError@4>
77ed3a32:	31 c0                	xor    %eax,%eax
77ed3a34:	c9                   	leave  
77ed3a35:	c2 10 00             	ret    $0x10
77ed3a38:	90                   	nop    
77ed3a39:	8d b4 26 00 00 00 00 	lea    0x0(%esi),%esi

77ed3a40 <_EngCreateDeviceSurface@16>:
77ed3a40:	55                   	push   %ebp
77ed3a41:	89 e5                	mov    %esp,%ebp
77ed3a43:	83 ec 10             	sub    $0x10,%esp
77ed3a46:	68 29 ae ed 77       	push   $0x77edae29
77ed3a4b:	68 20 a0 ed 77       	push   $0x77eda020
77ed3a50:	ff 15 e8 10 ee 77    	call   *0x77ee10e8
77ed3a56:	c7 04 24 78 00 00 00 	movl   $0x78,(%esp)
77ed3a5d:	e8 ae 5e 00 00       	call   77ed9910 <_SetLastError@4>
77ed3a62:	31 c0                	xor    %eax,%eax
77ed3a64:	c9                   	leave  
77ed3a65:	c2 10 00             	ret    $0x10
77ed3a68:	90                   	nop    
77ed3a69:	8d b4 26 00 00 00 00 	lea    0x0(%esi),%esi

77ed3a70 <_EngCreatePalette@24>:
77ed3a70:	55                   	push   %ebp
77ed3a71:	89 e5                	mov    %esp,%ebp
77ed3a73:	83 ec 10             	sub    $0x10,%esp
77ed3a76:	68 40 ae ed 77       	push   $0x77edae40
77ed3a7b:	68 20 a0 ed 77       	push   $0x77eda020
77ed3a80:	ff 15 e8 10 ee 77    	call   *0x77ee10e8
77ed3a86:	c7 04 24 78 00 00 00 	movl   $0x78,(%esp)
77ed3a8d:	e8 7e 5e 00 00       	call   77ed9910 <_SetLastError@4>
77ed3a92:	31 c0                	xor    %eax,%eax
77ed3a94:	c9                   	leave  
77ed3a95:	c2 18 00             	ret    $0x18
77ed3a98:	90                   	nop    
77ed3a99:	8d b4 26 00 00 00 00 	lea    0x0(%esi),%esi

77ed3aa0 <_EngCreateSemaphore@0>:
77ed3aa0:	55                   	push   %ebp
77ed3aa1:	89 e5                	mov    %esp,%ebp
77ed3aa3:	83 ec 10             	sub    $0x10,%esp
77ed3aa6:	68 51 ae ed 77       	push   $0x77edae51
77ed3aab:	68 20 a0 ed 77       	push   $0x77eda020
77ed3ab0:	ff 15 e8 10 ee 77    	call   *0x77ee10e8
77ed3ab6:	c7 04 24 78 00 00 00 	movl   $0x78,(%esp)
77ed3abd:	e8 4e 5e 00 00       	call   77ed9910 <_SetLastError@4>
77ed3ac2:	31 c0                	xor    %eax,%eax
77ed3ac4:	c9                   	leave  
77ed3ac5:	c3                   	ret    
77ed3ac6:	8d 76 00             	lea    0x0(%esi),%esi
77ed3ac9:	8d bc 27 00 00 00 00 	lea    0x0(%edi),%edi

77ed3ad0 <_EngDeleteClip@4>:
77ed3ad0:	55                   	push   %ebp
77ed3ad1:	89 e5                	mov    %esp,%ebp
77ed3ad3:	83 ec 10             	sub    $0x10,%esp
77ed3ad6:	68 64 ae ed 77       	push   $0x77edae64
77ed3adb:	68 20 a0 ed 77       	push   $0x77eda020
77ed3ae0:	ff 15 e8 10 ee 77    	call   *0x77ee10e8
77ed3ae6:	c7 45 08 78 00 00 00 	movl   $0x78,0x8(%ebp)
77ed3aed:	83 c4 10             	add    $0x10,%esp
77ed3af0:	c9                   	leave  
77ed3af1:	e9 1a 5e 00 00       	jmp    77ed9910 <_SetLastError@4>
77ed3af6:	8d 76 00             	lea    0x0(%esi),%esi
77ed3af9:	8d bc 27 00 00 00 00 	lea    0x0(%edi),%edi

77ed3b00 <_EngDeletePalette@4>:
77ed3b00:	55                   	push   %ebp
77ed3b01:	89 e5                	mov    %esp,%ebp
77ed3b03:	83 ec 10             	sub    $0x10,%esp
77ed3b06:	68 72 ae ed 77       	push   $0x77edae72
77ed3b0b:	68 20 a0 ed 77       	push   $0x77eda020
77ed3b10:	ff 15 e8 10 ee 77    	call   *0x77ee10e8
77ed3b16:	c7 04 24 78 00 00 00 	movl   $0x78,(%esp)
77ed3b1d:	e8 ee 5d 00 00       	call   77ed9910 <_SetLastError@4>
77ed3b22:	31 c0                	xor    %eax,%eax
77ed3b24:	c9                   	leave  
77ed3b25:	c2 04 00             	ret    $0x4
77ed3b28:	90                   	nop    
77ed3b29:	8d b4 26 00 00 00 00 	lea    0x0(%esi),%esi

77ed3b30 <_EngDeletePath@4>:
77ed3b30:	55                   	push   %ebp
77ed3b31:	89 e5                	mov    %esp,%ebp
77ed3b33:	83 ec 10             	sub    $0x10,%esp
77ed3b36:	68 83 ae ed 77       	push   $0x77edae83
77ed3b3b:	68 20 a0 ed 77       	push   $0x77eda020
77ed3b40:	ff 15 e8 10 ee 77    	call   *0x77ee10e8
77ed3b46:	c7 45 08 78 00 00 00 	movl   $0x78,0x8(%ebp)
77ed3b4d:	83 c4 10             	add    $0x10,%esp
77ed3b50:	c9                   	leave  
77ed3b51:	e9 ba 5d 00 00       	jmp    77ed9910 <_SetLastError@4>
77ed3b56:	8d 76 00             	lea    0x0(%esi),%esi
77ed3b59:	8d bc 27 00 00 00 00 	lea    0x0(%edi),%edi

77ed3b60 <_EngDeleteSemaphore@4>:
77ed3b60:	55                   	push   %ebp
77ed3b61:	89 e5                	mov    %esp,%ebp
77ed3b63:	83 ec 10             	sub    $0x10,%esp
77ed3b66:	68 91 ae ed 77       	push   $0x77edae91
77ed3b6b:	68 20 a0 ed 77       	push   $0x77eda020
77ed3b70:	ff 15 e8 10 ee 77    	call   *0x77ee10e8
77ed3b76:	c7 45 08 78 00 00 00 	movl   $0x78,0x8(%ebp)
77ed3b7d:	83 c4 10             	add    $0x10,%esp
77ed3b80:	c9                   	leave  
77ed3b81:	e9 8a 5d 00 00       	jmp    77ed9910 <_SetLastError@4>
77ed3b86:	8d 76 00             	lea    0x0(%esi),%esi
77ed3b89:	8d bc 27 00 00 00 00 	lea    0x0(%edi),%edi

77ed3b90 <_EngDeleteSurface@4>:
77ed3b90:	55                   	push   %ebp
77ed3b91:	89 e5                	mov    %esp,%ebp
77ed3b93:	83 ec 10             	sub    $0x10,%esp
77ed3b96:	68 a4 ae ed 77       	push   $0x77edaea4
77ed3b9b:	68 20 a0 ed 77       	push   $0x77eda020
77ed3ba0:	ff 15 e8 10 ee 77    	call   *0x77ee10e8
77ed3ba6:	c7 04 24 78 00 00 00 	movl   $0x78,(%esp)
77ed3bad:	e8 5e 5d 00 00       	call   77ed9910 <_SetLastError@4>
77ed3bb2:	31 c0                	xor    %eax,%eax
77ed3bb4:	c9                   	leave  
77ed3bb5:	c2 04 00             	ret    $0x4
77ed3bb8:	90                   	nop    
77ed3bb9:	8d b4 26 00 00 00 00 	lea    0x0(%esi),%esi

77ed3bc0 <_EngEraseSurface@12>:
77ed3bc0:	55                   	push   %ebp
77ed3bc1:	89 e5                	mov    %esp,%ebp
77ed3bc3:	83 ec 10             	sub    $0x10,%esp
77ed3bc6:	68 b5 ae ed 77       	push   $0x77edaeb5
77ed3bcb:	68 20 a0 ed 77       	push   $0x77eda020
77ed3bd0:	ff 15 e8 10 ee 77    	call   *0x77ee10e8
77ed3bd6:	c7 04 24 78 00 00 00 	movl   $0x78,(%esp)
77ed3bdd:	e8 2e 5d 00 00       	call   77ed9910 <_SetLastError@4>
77ed3be2:	31 c0                	xor    %eax,%eax
77ed3be4:	c9                   	leave  
77ed3be5:	c2 0c 00             	ret    $0xc
77ed3be8:	90                   	nop    
77ed3be9:	8d b4 26 00 00 00 00 	lea    0x0(%esi),%esi

77ed3bf0 <_EngFillPath@28>:
77ed3bf0:	55                   	push   %ebp
77ed3bf1:	89 e5                	mov    %esp,%ebp
77ed3bf3:	83 ec 10             	sub    $0x10,%esp
77ed3bf6:	68 c5 ae ed 77       	push   $0x77edaec5
77ed3bfb:	68 20 a0 ed 77       	push   $0x77eda020
77ed3c00:	ff 15 e8 10 ee 77    	call   *0x77ee10e8
77ed3c06:	c7 04 24 78 00 00 00 	movl   $0x78,(%esp)
77ed3c0d:	e8 fe 5c 00 00       	call   77ed9910 <_SetLastError@4>
77ed3c12:	31 c0                	xor    %eax,%eax
77ed3c14:	c9                   	leave  
77ed3c15:	c2 1c 00             	ret    $0x1c
77ed3c18:	90                   	nop    
77ed3c19:	8d b4 26 00 00 00 00 	lea    0x0(%esi),%esi

77ed3c20 <_EngFindResource@16>:
77ed3c20:	55                   	push   %ebp
77ed3c21:	89 e5                	mov    %esp,%ebp
77ed3c23:	83 ec 10             	sub    $0x10,%esp
77ed3c26:	68 d1 ae ed 77       	push   $0x77edaed1
77ed3c2b:	68 20 a0 ed 77       	push   $0x77eda020
77ed3c30:	ff 15 e8 10 ee 77    	call   *0x77ee10e8
77ed3c36:	c7 04 24 78 00 00 00 	movl   $0x78,(%esp)
77ed3c3d:	e8 ce 5c 00 00       	call   77ed9910 <_SetLastError@4>
77ed3c42:	31 c0                	xor    %eax,%eax
77ed3c44:	c9                   	leave  
77ed3c45:	c2 10 00             	ret    $0x10
77ed3c48:	90                   	nop    
77ed3c49:	8d b4 26 00 00 00 00 	lea    0x0(%esi),%esi

77ed3c50 <_EngFreeModule@4>:
77ed3c50:	55                   	push   %ebp
77ed3c51:	89 e5                	mov    %esp,%ebp
77ed3c53:	83 ec 10             	sub    $0x10,%esp
77ed3c56:	68 e1 ae ed 77       	push   $0x77edaee1
77ed3c5b:	68 20 a0 ed 77       	push   $0x77eda020
77ed3c60:	ff 15 e8 10 ee 77    	call   *0x77ee10e8
77ed3c66:	c7 45 08 78 00 00 00 	movl   $0x78,0x8(%ebp)
77ed3c6d:	83 c4 10             	add    $0x10,%esp
77ed3c70:	c9                   	leave  
77ed3c71:	e9 9a 5c 00 00       	jmp    77ed9910 <_SetLastError@4>
77ed3c76:	8d 76 00             	lea    0x0(%esi),%esi
77ed3c79:	8d bc 27 00 00 00 00 	lea    0x0(%edi),%edi

77ed3c80 <_EngGetCurrentCodePage@8>:
77ed3c80:	55                   	push   %ebp
77ed3c81:	89 e5                	mov    %esp,%ebp
77ed3c83:	83 ec 10             	sub    $0x10,%esp
77ed3c86:	68 ef ae ed 77       	push   $0x77edaeef
77ed3c8b:	68 20 a0 ed 77       	push   $0x77eda020
77ed3c90:	ff 15 e8 10 ee 77    	call   *0x77ee10e8
77ed3c96:	c7 04 24 78 00 00 00 	movl   $0x78,(%esp)
77ed3c9d:	e8 6e 5c 00 00       	call   77ed9910 <_SetLastError@4>
77ed3ca2:	c9                   	leave  
77ed3ca3:	c2 08 00             	ret    $0x8
77ed3ca6:	8d 76 00             	lea    0x0(%esi),%esi
77ed3ca9:	8d bc 27 00 00 00 00 	lea    0x0(%edi),%edi

77ed3cb0 <_EngGetDriverName@4>:
77ed3cb0:	55                   	push   %ebp
77ed3cb1:	89 e5                	mov    %esp,%ebp
77ed3cb3:	83 ec 10             	sub    $0x10,%esp
77ed3cb6:	68 05 af ed 77       	push   $0x77edaf05
77ed3cbb:	68 20 a0 ed 77       	push   $0x77eda020
77ed3cc0:	ff 15 e8 10 ee 77    	call   *0x77ee10e8
77ed3cc6:	c7 04 24 78 00 00 00 	movl   $0x78,(%esp)
77ed3ccd:	e8 3e 5c 00 00       	call   77ed9910 <_SetLastError@4>
77ed3cd2:	31 c0                	xor    %eax,%eax
77ed3cd4:	c9                   	leave  
77ed3cd5:	c2 04 00             	ret    $0x4
77ed3cd8:	90                   	nop    
77ed3cd9:	8d b4 26 00 00 00 00 	lea    0x0(%esi),%esi

77ed3ce0 <_EngGetPrinterDataFileName@4>:
77ed3ce0:	55                   	push   %ebp
77ed3ce1:	89 e5                	mov    %esp,%ebp
77ed3ce3:	83 ec 10             	sub    $0x10,%esp
77ed3ce6:	68 16 af ed 77       	push   $0x77edaf16
77ed3ceb:	68 20 a0 ed 77       	push   $0x77eda020
77ed3cf0:	ff 15 e8 10 ee 77    	call   *0x77ee10e8
77ed3cf6:	c7 04 24 78 00 00 00 	movl   $0x78,(%esp)
77ed3cfd:	e8 0e 5c 00 00       	call   77ed9910 <_SetLastError@4>
77ed3d02:	31 c0                	xor    %eax,%eax
77ed3d04:	c9                   	leave  
77ed3d05:	c2 04 00             	ret    $0x4
77ed3d08:	90                   	nop    
77ed3d09:	8d b4 26 00 00 00 00 	lea    0x0(%esi),%esi

77ed3d10 <_EngGradientFill@40>:
77ed3d10:	55                   	push   %ebp
77ed3d11:	89 e5                	mov    %esp,%ebp
77ed3d13:	83 ec 10             	sub    $0x10,%esp
77ed3d16:	68 30 af ed 77       	push   $0x77edaf30
77ed3d1b:	68 20 a0 ed 77       	push   $0x77eda020
77ed3d20:	ff 15 e8 10 ee 77    	call   *0x77ee10e8
77ed3d26:	c7 04 24 78 00 00 00 	movl   $0x78,(%esp)
77ed3d2d:	e8 de 5b 00 00       	call   77ed9910 <_SetLastError@4>
77ed3d32:	31 c0                	xor    %eax,%eax
77ed3d34:	c9                   	leave  
77ed3d35:	c2 28 00             	ret    $0x28
77ed3d38:	90                   	nop    
77ed3d39:	8d b4 26 00 00 00 00 	lea    0x0(%esi),%esi

77ed3d40 <_EngLineTo@36>:
77ed3d40:	55                   	push   %ebp
77ed3d41:	89 e5                	mov    %esp,%ebp
77ed3d43:	83 ec 10             	sub    $0x10,%esp
77ed3d46:	68 40 af ed 77       	push   $0x77edaf40
77ed3d4b:	68 20 a0 ed 77       	push   $0x77eda020
77ed3d50:	ff 15 e8 10 ee 77    	call   *0x77ee10e8
77ed3d56:	c7 04 24 78 00 00 00 	movl   $0x78,(%esp)
77ed3d5d:	e8 ae 5b 00 00       	call   77ed9910 <_SetLastError@4>
77ed3d62:	31 c0                	xor    %eax,%eax
77ed3d64:	c9                   	leave  
77ed3d65:	c2 24 00             	ret    $0x24
77ed3d68:	90                   	nop    
77ed3d69:	8d b4 26 00 00 00 00 	lea    0x0(%esi),%esi

77ed3d70 <_EngLoadModule@4>:
77ed3d70:	55                   	push   %ebp
77ed3d71:	89 e5                	mov    %esp,%ebp
77ed3d73:	83 ec 10             	sub    $0x10,%esp
77ed3d76:	68 4a af ed 77       	push   $0x77edaf4a
77ed3d7b:	68 20 a0 ed 77       	push   $0x77eda020
77ed3d80:	ff 15 e8 10 ee 77    	call   *0x77ee10e8
77ed3d86:	c7 04 24 78 00 00 00 	movl   $0x78,(%esp)
77ed3d8d:	e8 7e 5b 00 00       	call   77ed9910 <_SetLastError@4>
77ed3d92:	31 c0                	xor    %eax,%eax
77ed3d94:	c9                   	leave  
77ed3d95:	c2 04 00             	ret    $0x4
77ed3d98:	90                   	nop    
77ed3d99:	8d b4 26 00 00 00 00 	lea    0x0(%esi),%esi

77ed3da0 <_EngLockSurface@4>:
77ed3da0:	55                   	push   %ebp
77ed3da1:	89 e5                	mov    %esp,%ebp
77ed3da3:	83 ec 10             	sub    $0x10,%esp
77ed3da6:	68 58 af ed 77       	push   $0x77edaf58
77ed3dab:	68 20 a0 ed 77       	push   $0x77eda020
77ed3db0:	ff 15 e8 10 ee 77    	call   *0x77ee10e8
77ed3db6:	c7 04 24 78 00 00 00 	movl   $0x78,(%esp)
77ed3dbd:	e8 4e 5b 00 00       	call   77ed9910 <_SetLastError@4>
77ed3dc2:	31 c0                	xor    %eax,%eax
77ed3dc4:	c9                   	leave  
77ed3dc5:	c2 04 00             	ret    $0x4
77ed3dc8:	90                   	nop    
77ed3dc9:	8d b4 26 00 00 00 00 	lea    0x0(%esi),%esi

77ed3dd0 <_EngMarkBandingSurface@4>:
77ed3dd0:	55                   	push   %ebp
77ed3dd1:	89 e5                	mov    %esp,%ebp
77ed3dd3:	83 ec 10             	sub    $0x10,%esp
77ed3dd6:	68 67 af ed 77       	push   $0x77edaf67
77ed3ddb:	68 20 a0 ed 77       	push   $0x77eda020
77ed3de0:	ff 15 e8 10 ee 77    	call   *0x77ee10e8
77ed3de6:	c7 04 24 78 00 00 00 	movl   $0x78,(%esp)
77ed3ded:	e8 1e 5b 00 00       	call   77ed9910 <_SetLastError@4>
77ed3df2:	31 c0                	xor    %eax,%eax
77ed3df4:	c9                   	leave  
77ed3df5:	c2 04 00             	ret    $0x4
77ed3df8:	90                   	nop    
77ed3df9:	8d b4 26 00 00 00 00 	lea    0x0(%esi),%esi

77ed3e00 <_EngMultiByteToUnicodeN@20>:
77ed3e00:	55                   	push   %ebp
77ed3e01:	89 e5                	mov    %esp,%ebp
77ed3e03:	83 ec 10             	sub    $0x10,%esp
77ed3e06:	68 7d af ed 77       	push   $0x77edaf7d
77ed3e0b:	68 20 a0 ed 77       	push   $0x77eda020
77ed3e10:	ff 15 e8 10 ee 77    	call   *0x77ee10e8
77ed3e16:	c7 04 24 78 00 00 00 	movl   $0x78,(%esp)
77ed3e1d:	e8 ee 5a 00 00       	call   77ed9910 <_SetLastError@4>
77ed3e22:	c9                   	leave  
77ed3e23:	c2 14 00             	ret    $0x14
77ed3e26:	8d 76 00             	lea    0x0(%esi),%esi
77ed3e29:	8d bc 27 00 00 00 00 	lea    0x0(%edi),%edi

77ed3e30 <_EngMultiByteToWideChar@20>:
77ed3e30:	55                   	push   %ebp
77ed3e31:	89 e5                	mov    %esp,%ebp
77ed3e33:	83 ec 10             	sub    $0x10,%esp
77ed3e36:	68 94 af ed 77       	push   $0x77edaf94
77ed3e3b:	68 20 a0 ed 77       	push   $0x77eda020
77ed3e40:	ff 15 e8 10 ee 77    	call   *0x77ee10e8
77ed3e46:	c7 04 24 78 00 00 00 	movl   $0x78,(%esp)
77ed3e4d:	e8 be 5a 00 00       	call   77ed9910 <_SetLastError@4>
77ed3e52:	31 c0                	xor    %eax,%eax
77ed3e54:	c9                   	leave  
77ed3e55:	c2 14 00             	ret    $0x14
77ed3e58:	90                   	nop    
77ed3e59:	8d b4 26 00 00 00 00 	lea    0x0(%esi),%esi

77ed3e60 <_EngPaint@20>:
77ed3e60:	55                   	push   %ebp
77ed3e61:	89 e5                	mov    %esp,%ebp
77ed3e63:	83 ec 10             	sub    $0x10,%esp
77ed3e66:	68 ab af ed 77       	push   $0x77edafab
77ed3e6b:	68 20 a0 ed 77       	push   $0x77eda020
77ed3e70:	ff 15 e8 10 ee 77    	call   *0x77ee10e8
77ed3e76:	c7 04 24 78 00 00 00 	movl   $0x78,(%esp)
77ed3e7d:	e8 8e 5a 00 00       	call   77ed9910 <_SetLastError@4>
77ed3e82:	31 c0                	xor    %eax,%eax
77ed3e84:	c9                   	leave  
77ed3e85:	c2 14 00             	ret    $0x14
77ed3e88:	90                   	nop    
77ed3e89:	8d b4 26 00 00 00 00 	lea    0x0(%esi),%esi

77ed3e90 <_EngPlgBlt@44>:
77ed3e90:	55                   	push   %ebp
77ed3e91:	89 e5                	mov    %esp,%ebp
77ed3e93:	83 ec 10             	sub    $0x10,%esp
77ed3e96:	68 b4 af ed 77       	push   $0x77edafb4
77ed3e9b:	68 20 a0 ed 77       	push   $0x77eda020
77ed3ea0:	ff 15 e8 10 ee 77    	call   *0x77ee10e8
77ed3ea6:	c7 04 24 78 00 00 00 	movl   $0x78,(%esp)
77ed3ead:	e8 5e 5a 00 00       	call   77ed9910 <_SetLastError@4>
77ed3eb2:	31 c0                	xor    %eax,%eax
77ed3eb4:	c9                   	leave  
77ed3eb5:	c2 2c 00             	ret    $0x2c
77ed3eb8:	90                   	nop    
77ed3eb9:	8d b4 26 00 00 00 00 	lea    0x0(%esi),%esi

77ed3ec0 <_EngQueryEMFInfo@8>:
77ed3ec0:	55                   	push   %ebp
77ed3ec1:	89 e5                	mov    %esp,%ebp
77ed3ec3:	83 ec 10             	sub    $0x10,%esp
77ed3ec6:	68 be af ed 77       	push   $0x77edafbe
77ed3ecb:	68 20 a0 ed 77       	push   $0x77eda020
77ed3ed0:	ff 15 e8 10 ee 77    	call   *0x77ee10e8
77ed3ed6:	c7 04 24 78 00 00 00 	movl   $0x78,(%esp)
77ed3edd:	e8 2e 5a 00 00       	call   77ed9910 <_SetLastError@4>
77ed3ee2:	31 c0                	xor    %eax,%eax
77ed3ee4:	c9                   	leave  
77ed3ee5:	c2 08 00             	ret    $0x8
77ed3ee8:	90                   	nop    
77ed3ee9:	8d b4 26 00 00 00 00 	lea    0x0(%esi),%esi

77ed3ef0 <_EngQueryLocalTime@4>:
77ed3ef0:	55                   	push   %ebp
77ed3ef1:	89 e5                	mov    %esp,%ebp
77ed3ef3:	83 ec 10             	sub    $0x10,%esp
77ed3ef6:	68 ce af ed 77       	push   $0x77edafce
77ed3efb:	68 20 a0 ed 77       	push   $0x77eda020
77ed3f00:	ff 15 e8 10 ee 77    	call   *0x77ee10e8
77ed3f06:	c7 45 08 78 00 00 00 	movl   $0x78,0x8(%ebp)
77ed3f0d:	83 c4 10             	add    $0x10,%esp
77ed3f10:	c9                   	leave  
77ed3f11:	e9 fa 59 00 00       	jmp    77ed9910 <_SetLastError@4>
77ed3f16:	8d 76 00             	lea    0x0(%esi),%esi
77ed3f19:	8d bc 27 00 00 00 00 	lea    0x0(%edi),%edi

77ed3f20 <_EngReleaseSemaphore@4>:
77ed3f20:	55                   	push   %ebp
77ed3f21:	89 e5                	mov    %esp,%ebp
77ed3f23:	83 ec 10             	sub    $0x10,%esp
77ed3f26:	68 e0 af ed 77       	push   $0x77edafe0
77ed3f2b:	68 20 a0 ed 77       	push   $0x77eda020
77ed3f30:	ff 15 e8 10 ee 77    	call   *0x77ee10e8
77ed3f36:	c7 45 08 78 00 00 00 	movl   $0x78,0x8(%ebp)
77ed3f3d:	83 c4 10             	add    $0x10,%esp
77ed3f40:	c9                   	leave  
77ed3f41:	e9 ca 59 00 00       	jmp    77ed9910 <_SetLastError@4>
77ed3f46:	8d 76 00             	lea    0x0(%esi),%esi
77ed3f49:	8d bc 27 00 00 00 00 	lea    0x0(%edi),%edi

77ed3f50 <_EngStretchBlt@44>:
77ed3f50:	55                   	push   %ebp
77ed3f51:	89 e5                	mov    %esp,%ebp
77ed3f53:	83 ec 10             	sub    $0x10,%esp
77ed3f56:	68 f4 af ed 77       	push   $0x77edaff4
77ed3f5b:	68 20 a0 ed 77       	push   $0x77eda020
77ed3f60:	ff 15 e8 10 ee 77    	call   *0x77ee10e8
77ed3f66:	c7 04 24 78 00 00 00 	movl   $0x78,(%esp)
77ed3f6d:	e8 9e 59 00 00       	call   77ed9910 <_SetLastError@4>
77ed3f72:	31 c0                	xor    %eax,%eax
77ed3f74:	c9                   	leave  
77ed3f75:	c2 2c 00             	ret    $0x2c
77ed3f78:	90                   	nop    
77ed3f79:	8d b4 26 00 00 00 00 	lea    0x0(%esi),%esi

77ed3f80 <_EngStretchBltROP@52>:
77ed3f80:	55                   	push   %ebp
77ed3f81:	89 e5                	mov    %esp,%ebp
77ed3f83:	83 ec 10             	sub    $0x10,%esp
77ed3f86:	68 02 b0 ed 77       	push   $0x77edb002
77ed3f8b:	68 20 a0 ed 77       	push   $0x77eda020
77ed3f90:	ff 15 e8 10 ee 77    	call   *0x77ee10e8
77ed3f96:	c7 04 24 78 00 00 00 	movl   $0x78,(%esp)
77ed3f9d:	e8 6e 59 00 00       	call   77ed9910 <_SetLastError@4>
77ed3fa2:	31 c0                	xor    %eax,%eax
77ed3fa4:	c9                   	leave  
77ed3fa5:	c2 34 00             	ret    $0x34
77ed3fa8:	90                   	nop    
77ed3fa9:	8d b4 26 00 00 00 00 	lea    0x0(%esi),%esi

77ed3fb0 <_EngStrokeAndFillPath@40>:
77ed3fb0:	55                   	push   %ebp
77ed3fb1:	89 e5                	mov    %esp,%ebp
77ed3fb3:	83 ec 10             	sub    $0x10,%esp
77ed3fb6:	68 13 b0 ed 77       	push   $0x77edb013
77ed3fbb:	68 20 a0 ed 77       	push   $0x77eda020
77ed3fc0:	ff 15 e8 10 ee 77    	call   *0x77ee10e8
77ed3fc6:	c7 04 24 78 00 00 00 	movl   $0x78,(%esp)
77ed3fcd:	e8 3e 59 00 00       	call   77ed9910 <_SetLastError@4>
77ed3fd2:	31 c0                	xor    %eax,%eax
77ed3fd4:	c9                   	leave  
77ed3fd5:	c2 28 00             	ret    $0x28
77ed3fd8:	90                   	nop    
77ed3fd9:	8d b4 26 00 00 00 00 	lea    0x0(%esi),%esi

77ed3fe0 <_EngStrokePath@32>:
77ed3fe0:	55                   	push   %ebp
77ed3fe1:	89 e5                	mov    %esp,%ebp
77ed3fe3:	83 ec 10             	sub    $0x10,%esp
77ed3fe6:	68 28 b0 ed 77       	push   $0x77edb028
77ed3feb:	68 20 a0 ed 77       	push   $0x77eda020
77ed3ff0:	ff 15 e8 10 ee 77    	call   *0x77ee10e8
77ed3ff6:	c7 04 24 78 00 00 00 	movl   $0x78,(%esp)
77ed3ffd:	e8 0e 59 00 00       	call   77ed9910 <_SetLastError@4>
77ed4002:	31 c0                	xor    %eax,%eax
77ed4004:	c9                   	leave  
77ed4005:	c2 20 00             	ret    $0x20
77ed4008:	90                   	nop    
77ed4009:	8d b4 26 00 00 00 00 	lea    0x0(%esi),%esi

77ed4010 <_EngTextOut@40>:
77ed4010:	55                   	push   %ebp
77ed4011:	89 e5                	mov    %esp,%ebp
77ed4013:	83 ec 10             	sub    $0x10,%esp
77ed4016:	68 36 b0 ed 77       	push   $0x77edb036
77ed401b:	68 20 a0 ed 77       	push   $0x77eda020
77ed4020:	ff 15 e8 10 ee 77    	call   *0x77ee10e8
77ed4026:	c7 04 24 78 00 00 00 	movl   $0x78,(%esp)
77ed402d:	e8 de 58 00 00       	call   77ed9910 <_SetLastError@4>
77ed4032:	31 c0                	xor    %eax,%eax
77ed4034:	c9                   	leave  
77ed4035:	c2 28 00             	ret    $0x28
77ed4038:	90                   	nop    
77ed4039:	8d b4 26 00 00 00 00 	lea    0x0(%esi),%esi

77ed4040 <_EngTransparentBlt@32>:
77ed4040:	55                   	push   %ebp
77ed4041:	89 e5                	mov    %esp,%ebp
77ed4043:	83 ec 10             	sub    $0x10,%esp
77ed4046:	68 41 b0 ed 77       	push   $0x77edb041
77ed404b:	68 20 a0 ed 77       	push   $0x77eda020
77ed4050:	ff 15 e8 10 ee 77    	call   *0x77ee10e8
77ed4056:	c7 04 24 78 00 00 00 	movl   $0x78,(%esp)
77ed405d:	e8 ae 58 00 00       	call   77ed9910 <_SetLastError@4>
77ed4062:	31 c0                	xor    %eax,%eax
77ed4064:	c9                   	leave  
77ed4065:	c2 20 00             	ret    $0x20
77ed4068:	90                   	nop    
77ed4069:	8d b4 26 00 00 00 00 	lea    0x0(%esi),%esi

77ed4070 <_EngUnicodeToMultiByteN@20>:
77ed4070:	55                   	push   %ebp
77ed4071:	89 e5                	mov    %esp,%ebp
77ed4073:	83 ec 10             	sub    $0x10,%esp
77ed4076:	68 53 b0 ed 77       	push   $0x77edb053
77ed407b:	68 20 a0 ed 77       	push   $0x77eda020
77ed4080:	ff 15 e8 10 ee 77    	call   *0x77ee10e8
77ed4086:	c7 04 24 78 00 00 00 	movl   $0x78,(%esp)
77ed408d:	e8 7e 58 00 00       	call   77ed9910 <_SetLastError@4>
77ed4092:	c9                   	leave  
77ed4093:	c2 14 00             	ret    $0x14
77ed4096:	8d 76 00             	lea    0x0(%esi),%esi
77ed4099:	8d bc 27 00 00 00 00 	lea    0x0(%edi),%edi

77ed40a0 <_EngUnlockSurface@4>:
77ed40a0:	55                   	push   %ebp
77ed40a1:	89 e5                	mov    %esp,%ebp
77ed40a3:	83 ec 10             	sub    $0x10,%esp
77ed40a6:	68 6a b0 ed 77       	push   $0x77edb06a
77ed40ab:	68 20 a0 ed 77       	push   $0x77eda020
77ed40b0:	ff 15 e8 10 ee 77    	call   *0x77ee10e8
77ed40b6:	c7 45 08 78 00 00 00 	movl   $0x78,0x8(%ebp)
77ed40bd:	83 c4 10             	add    $0x10,%esp
77ed40c0:	c9                   	leave  
77ed40c1:	e9 4a 58 00 00       	jmp    77ed9910 <_SetLastError@4>
77ed40c6:	8d 76 00             	lea    0x0(%esi),%esi
77ed40c9:	8d bc 27 00 00 00 00 	lea    0x0(%edi),%edi

77ed40d0 <_EngWideCharToMultiByte@20>:
77ed40d0:	55                   	push   %ebp
77ed40d1:	89 e5                	mov    %esp,%ebp
77ed40d3:	83 ec 10             	sub    $0x10,%esp
77ed40d6:	68 7b b0 ed 77       	push   $0x77edb07b
77ed40db:	68 20 a0 ed 77       	push   $0x77eda020
77ed40e0:	ff 15 e8 10 ee 77    	call   *0x77ee10e8
77ed40e6:	c7 04 24 78 00 00 00 	movl   $0x78,(%esp)
77ed40ed:	e8 1e 58 00 00       	call   77ed9910 <_SetLastError@4>
77ed40f2:	31 c0                	xor    %eax,%eax
77ed40f4:	c9                   	leave  
77ed40f5:	c2 14 00             	ret    $0x14
77ed40f8:	90                   	nop    
77ed40f9:	8d b4 26 00 00 00 00 	lea    0x0(%esi),%esi

77ed4100 <_FONTOBJ_cGetAllGlyphHandles@8>:
77ed4100:	55                   	push   %ebp
77ed4101:	89 e5                	mov    %esp,%ebp
77ed4103:	83 ec 10             	sub    $0x10,%esp
77ed4106:	68 92 b0 ed 77       	push   $0x77edb092
77ed410b:	68 20 a0 ed 77       	push   $0x77eda020
77ed4110:	ff 15 e8 10 ee 77    	call   *0x77ee10e8
77ed4116:	c7 04 24 78 00 00 00 	movl   $0x78,(%esp)
77ed411d:	e8 ee 57 00 00       	call   77ed9910 <_SetLastError@4>
77ed4122:	31 c0                	xor    %eax,%eax
77ed4124:	c9                   	leave  
77ed4125:	c2 08 00             	ret    $0x8
77ed4128:	90                   	nop    
77ed4129:	8d b4 26 00 00 00 00 	lea    0x0(%esi),%esi

77ed4130 <_FONTOBJ_cGetGlyphs@20>:
77ed4130:	55                   	push   %ebp
77ed4131:	89 e5                	mov    %esp,%ebp
77ed4133:	83 ec 10             	sub    $0x10,%esp
77ed4136:	68 ae b0 ed 77       	push   $0x77edb0ae
77ed413b:	68 20 a0 ed 77       	push   $0x77eda020
77ed4140:	ff 15 e8 10 ee 77    	call   *0x77ee10e8
77ed4146:	c7 04 24 78 00 00 00 	movl   $0x78,(%esp)
77ed414d:	e8 be 57 00 00       	call   77ed9910 <_SetLastError@4>
77ed4152:	31 c0                	xor    %eax,%eax
77ed4154:	c9                   	leave  
77ed4155:	c2 14 00             	ret    $0x14
77ed4158:	90                   	nop    
77ed4159:	8d b4 26 00 00 00 00 	lea    0x0(%esi),%esi

77ed4160 <_FONTOBJ_pQueryGlyphAttrs@8>:
77ed4160:	55                   	push   %ebp
77ed4161:	89 e5                	mov    %esp,%ebp
77ed4163:	83 ec 10             	sub    $0x10,%esp
77ed4166:	68 c1 b0 ed 77       	push   $0x77edb0c1
77ed416b:	68 20 a0 ed 77       	push   $0x77eda020
77ed4170:	ff 15 e8 10 ee 77    	call   *0x77ee10e8
77ed4176:	c7 04 24 78 00 00 00 	movl   $0x78,(%esp)
77ed417d:	e8 8e 57 00 00       	call   77ed9910 <_SetLastError@4>
77ed4182:	31 c0                	xor    %eax,%eax
77ed4184:	c9                   	leave  
77ed4185:	c2 08 00             	ret    $0x8
77ed4188:	90                   	nop    
77ed4189:	8d b4 26 00 00 00 00 	lea    0x0(%esi),%esi

77ed4190 <_FONTOBJ_pfdg@4>:
77ed4190:	55                   	push   %ebp
77ed4191:	89 e5                	mov    %esp,%ebp
77ed4193:	83 ec 10             	sub    $0x10,%esp
77ed4196:	68 da b0 ed 77       	push   $0x77edb0da
77ed419b:	68 20 a0 ed 77       	push   $0x77eda020
77ed41a0:	ff 15 e8 10 ee 77    	call   *0x77ee10e8
77ed41a6:	c7 04 24 78 00 00 00 	movl   $0x78,(%esp)
77ed41ad:	e8 5e 57 00 00       	call   77ed9910 <_SetLastError@4>
77ed41b2:	31 c0                	xor    %eax,%eax
77ed41b4:	c9                   	leave  
77ed41b5:	c2 04 00             	ret    $0x4
77ed41b8:	90                   	nop    
77ed41b9:	8d b4 26 00 00 00 00 	lea    0x0(%esi),%esi

77ed41c0 <_FONTOBJ_pifi@4>:
77ed41c0:	55                   	push   %ebp
77ed41c1:	89 e5                	mov    %esp,%ebp
77ed41c3:	83 ec 10             	sub    $0x10,%esp
77ed41c6:	68 e7 b0 ed 77       	push   $0x77edb0e7
77ed41cb:	68 20 a0 ed 77       	push   $0x77eda020
77ed41d0:	ff 15 e8 10 ee 77    	call   *0x77ee10e8
77ed41d6:	c7 04 24 78 00 00 00 	movl   $0x78,(%esp)
77ed41dd:	e8 2e 57 00 00       	call   77ed9910 <_SetLastError@4>
77ed41e2:	31 c0                	xor    %eax,%eax
77ed41e4:	c9                   	leave  
77ed41e5:	c2 04 00             	ret    $0x4
77ed41e8:	90                   	nop    
77ed41e9:	8d b4 26 00 00 00 00 	lea    0x0(%esi),%esi

77ed41f0 <_FONTOBJ_pvTrueTypeFontFile@8>:
77ed41f0:	55                   	push   %ebp
77ed41f1:	89 e5                	mov    %esp,%ebp
77ed41f3:	83 ec 10             	sub    $0x10,%esp
77ed41f6:	68 f4 b0 ed 77       	push   $0x77edb0f4
77ed41fb:	68 20 a0 ed 77       	push   $0x77eda020
77ed4200:	ff 15 e8 10 ee 77    	call   *0x77ee10e8
77ed4206:	c7 04 24 78 00 00 00 	movl   $0x78,(%esp)
77ed420d:	e8 fe 56 00 00       	call   77ed9910 <_SetLastError@4>
77ed4212:	31 c0                	xor    %eax,%eax
77ed4214:	c9                   	leave  
77ed4215:	c2 08 00             	ret    $0x8
77ed4218:	90                   	nop    
77ed4219:	8d b4 26 00 00 00 00 	lea    0x0(%esi),%esi

77ed4220 <_FONTOBJ_pxoGetXform@4>:
77ed4220:	55                   	push   %ebp
77ed4221:	89 e5                	mov    %esp,%ebp
77ed4223:	83 ec 10             	sub    $0x10,%esp
77ed4226:	68 0f b1 ed 77       	push   $0x77edb10f
77ed422b:	68 20 a0 ed 77       	push   $0x77eda020
77ed4230:	ff 15 e8 10 ee 77    	call   *0x77ee10e8
77ed4236:	c7 04 24 78 00 00 00 	movl   $0x78,(%esp)
77ed423d:	e8 ce 56 00 00       	call   77ed9910 <_SetLastError@4>
77ed4242:	31 c0                	xor    %eax,%eax
77ed4244:	c9                   	leave  
77ed4245:	c2 04 00             	ret    $0x4
77ed4248:	90                   	nop    
77ed4249:	8d b4 26 00 00 00 00 	lea    0x0(%esi),%esi

77ed4250 <_FONTOBJ_vGetInfo@12>:
77ed4250:	55                   	push   %ebp
77ed4251:	89 e5                	mov    %esp,%ebp
77ed4253:	83 ec 10             	sub    $0x10,%esp
77ed4256:	68 23 b1 ed 77       	push   $0x77edb123
77ed425b:	68 20 a0 ed 77       	push   $0x77eda020
77ed4260:	ff 15 e8 10 ee 77    	call   *0x77ee10e8
77ed4266:	c7 04 24 78 00 00 00 	movl   $0x78,(%esp)
77ed426d:	e8 9e 56 00 00       	call   77ed9910 <_SetLastError@4>
77ed4272:	c9                   	leave  
77ed4273:	c2 0c 00             	ret    $0xc
77ed4276:	8d 76 00             	lea    0x0(%esi),%esi
77ed4279:	8d bc 27 00 00 00 00 	lea    0x0(%edi),%edi

77ed4280 <_PATHOBJ_bEnum@8>:
77ed4280:	55                   	push   %ebp
77ed4281:	89 e5                	mov    %esp,%ebp
77ed4283:	83 ec 10             	sub    $0x10,%esp
77ed4286:	68 34 b1 ed 77       	push   $0x77edb134
77ed428b:	68 20 a0 ed 77       	push   $0x77eda020
77ed4290:	ff 15 e8 10 ee 77    	call   *0x77ee10e8
77ed4296:	c7 04 24 78 00 00 00 	movl   $0x78,(%esp)
77ed429d:	e8 6e 56 00 00       	call   77ed9910 <_SetLastError@4>
77ed42a2:	31 c0                	xor    %eax,%eax
77ed42a4:	c9                   	leave  
77ed42a5:	c2 08 00             	ret    $0x8
77ed42a8:	90                   	nop    
77ed42a9:	8d b4 26 00 00 00 00 	lea    0x0(%esi),%esi

77ed42b0 <_PATHOBJ_bEnumClipLines@12>:
77ed42b0:	55                   	push   %ebp
77ed42b1:	89 e5                	mov    %esp,%ebp
77ed42b3:	83 ec 10             	sub    $0x10,%esp
77ed42b6:	68 42 b1 ed 77       	push   $0x77edb142
77ed42bb:	68 20 a0 ed 77       	push   $0x77eda020
77ed42c0:	ff 15 e8 10 ee 77    	call   *0x77ee10e8
77ed42c6:	c7 04 24 78 00 00 00 	movl   $0x78,(%esp)
77ed42cd:	e8 3e 56 00 00       	call   77ed9910 <_SetLastError@4>
77ed42d2:	31 c0                	xor    %eax,%eax
77ed42d4:	c9                   	leave  
77ed42d5:	c2 0c 00             	ret    $0xc
77ed42d8:	90                   	nop    
77ed42d9:	8d b4 26 00 00 00 00 	lea    0x0(%esi),%esi

77ed42e0 <_PATHOBJ_vEnumStart@4>:
77ed42e0:	55                   	push   %ebp
77ed42e1:	89 e5                	mov    %esp,%ebp
77ed42e3:	83 ec 10             	sub    $0x10,%esp
77ed42e6:	68 59 b1 ed 77       	push   $0x77edb159
77ed42eb:	68 20 a0 ed 77       	push   $0x77eda020
77ed42f0:	ff 15 e8 10 ee 77    	call   *0x77ee10e8
77ed42f6:	c7 45 08 78 00 00 00 	movl   $0x78,0x8(%ebp)
77ed42fd:	83 c4 10             	add    $0x10,%esp
77ed4300:	c9                   	leave  
77ed4301:	e9 0a 56 00 00       	jmp    77ed9910 <_SetLastError@4>
77ed4306:	8d 76 00             	lea    0x0(%esi),%esi
77ed4309:	8d bc 27 00 00 00 00 	lea    0x0(%edi),%edi

77ed4310 <_PATHOBJ_vEnumStartClipLines@16>:
77ed4310:	55                   	push   %ebp
77ed4311:	89 e5                	mov    %esp,%ebp
77ed4313:	83 ec 10             	sub    $0x10,%esp
77ed4316:	68 6c b1 ed 77       	push   $0x77edb16c
77ed431b:	68 20 a0 ed 77       	push   $0x77eda020
77ed4320:	ff 15 e8 10 ee 77    	call   *0x77ee10e8
77ed4326:	c7 04 24 78 00 00 00 	movl   $0x78,(%esp)
77ed432d:	e8 de 55 00 00       	call   77ed9910 <_SetLastError@4>
77ed4332:	c9                   	leave  
77ed4333:	c2 10 00             	ret    $0x10
77ed4336:	8d 76 00             	lea    0x0(%esi),%esi
77ed4339:	8d bc 27 00 00 00 00 	lea    0x0(%edi),%edi

77ed4340 <_PATHOBJ_vGetBounds@8>:
77ed4340:	55                   	push   %ebp
77ed4341:	89 e5                	mov    %esp,%ebp
77ed4343:	83 ec 10             	sub    $0x10,%esp
77ed4346:	68 88 b1 ed 77       	push   $0x77edb188
77ed434b:	68 20 a0 ed 77       	push   $0x77eda020
77ed4350:	ff 15 e8 10 ee 77    	call   *0x77ee10e8
77ed4356:	c7 04 24 78 00 00 00 	movl   $0x78,(%esp)
77ed435d:	e8 ae 55 00 00       	call   77ed9910 <_SetLastError@4>
77ed4362:	c9                   	leave  
77ed4363:	c2 08 00             	ret    $0x8
77ed4366:	8d 76 00             	lea    0x0(%esi),%esi
77ed4369:	8d bc 27 00 00 00 00 	lea    0x0(%edi),%edi

77ed4370 <_STROBJ_bEnum@12>:
77ed4370:	55                   	push   %ebp
77ed4371:	89 e5                	mov    %esp,%ebp
77ed4373:	83 ec 10             	sub    $0x10,%esp
77ed4376:	68 9b b1 ed 77       	push   $0x77edb19b
77ed437b:	68 20 a0 ed 77       	push   $0x77eda020
77ed4380:	ff 15 e8 10 ee 77    	call   *0x77ee10e8
77ed4386:	c7 04 24 78 00 00 00 	movl   $0x78,(%esp)
77ed438d:	e8 7e 55 00 00       	call   77ed9910 <_SetLastError@4>
77ed4392:	31 c0                	xor    %eax,%eax
77ed4394:	c9                   	leave  
77ed4395:	c2 0c 00             	ret    $0xc
77ed4398:	90                   	nop    
77ed4399:	8d b4 26 00 00 00 00 	lea    0x0(%esi),%esi

77ed43a0 <_STROBJ_bEnumPositionsOnly@12>:
77ed43a0:	55                   	push   %ebp
77ed43a1:	89 e5                	mov    %esp,%ebp
77ed43a3:	83 ec 10             	sub    $0x10,%esp
77ed43a6:	68 a8 b1 ed 77       	push   $0x77edb1a8
77ed43ab:	68 20 a0 ed 77       	push   $0x77eda020
77ed43b0:	ff 15 e8 10 ee 77    	call   *0x77ee10e8
77ed43b6:	c7 04 24 78 00 00 00 	movl   $0x78,(%esp)
77ed43bd:	e8 4e 55 00 00       	call   77ed9910 <_SetLastError@4>
77ed43c2:	31 c0                	xor    %eax,%eax
77ed43c4:	c9                   	leave  
77ed43c5:	c2 0c 00             	ret    $0xc
77ed43c8:	90                   	nop    
77ed43c9:	8d b4 26 00 00 00 00 	lea    0x0(%esi),%esi

77ed43d0 <_STROBJ_bGetAdvanceWidths@16>:
77ed43d0:	55                   	push   %ebp
77ed43d1:	89 e5                	mov    %esp,%ebp
77ed43d3:	83 ec 10             	sub    $0x10,%esp
77ed43d6:	68 c2 b1 ed 77       	push   $0x77edb1c2
77ed43db:	68 20 a0 ed 77       	push   $0x77eda020
77ed43e0:	ff 15 e8 10 ee 77    	call   *0x77ee10e8
77ed43e6:	c7 04 24 78 00 00 00 	movl   $0x78,(%esp)
77ed43ed:	e8 1e 55 00 00       	call   77ed9910 <_SetLastError@4>
77ed43f2:	31 c0                	xor    %eax,%eax
77ed43f4:	c9                   	leave  
77ed43f5:	c2 10 00             	ret    $0x10
77ed43f8:	90                   	nop    
77ed43f9:	8d b4 26 00 00 00 00 	lea    0x0(%esi),%esi

77ed4400 <_STROBJ_dwGetCodePage@4>:
77ed4400:	55                   	push   %ebp
77ed4401:	89 e5                	mov    %esp,%ebp
77ed4403:	83 ec 10             	sub    $0x10,%esp
77ed4406:	68 db b1 ed 77       	push   $0x77edb1db
77ed440b:	68 20 a0 ed 77       	push   $0x77eda020
77ed4410:	ff 15 e8 10 ee 77    	call   *0x77ee10e8
77ed4416:	c7 04 24 78 00 00 00 	movl   $0x78,(%esp)
77ed441d:	e8 ee 54 00 00       	call   77ed9910 <_SetLastError@4>
77ed4422:	31 c0                	xor    %eax,%eax
77ed4424:	c9                   	leave  
77ed4425:	c2 04 00             	ret    $0x4
77ed4428:	90                   	nop    
77ed4429:	8d b4 26 00 00 00 00 	lea    0x0(%esi),%esi

77ed4430 <_STROBJ_vEnumStart@4>:
77ed4430:	55                   	push   %ebp
77ed4431:	89 e5                	mov    %esp,%ebp
77ed4433:	83 ec 10             	sub    $0x10,%esp
77ed4436:	68 f0 b1 ed 77       	push   $0x77edb1f0
77ed443b:	68 20 a0 ed 77       	push   $0x77eda020
77ed4440:	ff 15 e8 10 ee 77    	call   *0x77ee10e8
77ed4446:	c7 45 08 78 00 00 00 	movl   $0x78,0x8(%ebp)
77ed444d:	83 c4 10             	add    $0x10,%esp
77ed4450:	c9                   	leave  
77ed4451:	e9 ba 54 00 00       	jmp    77ed9910 <_SetLastError@4>
77ed4456:	8d 76 00             	lea    0x0(%esi),%esi
77ed4459:	8d bc 27 00 00 00 00 	lea    0x0(%edi),%edi

77ed4460 <_XFORMOBJ_bApplyXform@20>:
77ed4460:	55                   	push   %ebp
77ed4461:	89 e5                	mov    %esp,%ebp
77ed4463:	83 ec 10             	sub    $0x10,%esp
77ed4466:	68 02 b2 ed 77       	push   $0x77edb202
77ed446b:	68 20 a0 ed 77       	push   $0x77eda020
77ed4470:	ff 15 e8 10 ee 77    	call   *0x77ee10e8
77ed4476:	c7 04 24 78 00 00 00 	movl   $0x78,(%esp)
77ed447d:	e8 8e 54 00 00       	call   77ed9910 <_SetLastError@4>
77ed4482:	31 c0                	xor    %eax,%eax
77ed4484:	c9                   	leave  
77ed4485:	c2 14 00             	ret    $0x14
77ed4488:	90                   	nop    
77ed4489:	8d b4 26 00 00 00 00 	lea    0x0(%esi),%esi

77ed4490 <_XFORMOBJ_iGetXform@8>:
77ed4490:	55                   	push   %ebp
77ed4491:	89 e5                	mov    %esp,%ebp
77ed4493:	83 ec 10             	sub    $0x10,%esp
77ed4496:	68 17 b2 ed 77       	push   $0x77edb217
77ed449b:	68 20 a0 ed 77       	push   $0x77eda020
77ed44a0:	ff 15 e8 10 ee 77    	call   *0x77ee10e8
77ed44a6:	c7 04 24 78 00 00 00 	movl   $0x78,(%esp)
77ed44ad:	e8 5e 54 00 00       	call   77ed9910 <_SetLastError@4>
77ed44b2:	31 c0                	xor    %eax,%eax
77ed44b4:	c9                   	leave  
77ed44b5:	c2 08 00             	ret    $0x8
77ed44b8:	90                   	nop    
77ed44b9:	8d b4 26 00 00 00 00 	lea    0x0(%esi),%esi

77ed44c0 <_XLATEOBJ_cGetPalette@16>:
77ed44c0:	55                   	push   %ebp
77ed44c1:	89 e5                	mov    %esp,%ebp
77ed44c3:	83 ec 10             	sub    $0x10,%esp
77ed44c6:	68 2a b2 ed 77       	push   $0x77edb22a
77ed44cb:	68 20 a0 ed 77       	push   $0x77eda020
77ed44d0:	ff 15 e8 10 ee 77    	call   *0x77ee10e8
77ed44d6:	c7 04 24 78 00 00 00 	movl   $0x78,(%esp)
77ed44dd:	e8 2e 54 00 00       	call   77ed9910 <_SetLastError@4>
77ed44e2:	31 c0                	xor    %eax,%eax
77ed44e4:	c9                   	leave  
77ed44e5:	c2 10 00             	ret    $0x10
77ed44e8:	90                   	nop    
77ed44e9:	8d b4 26 00 00 00 00 	lea    0x0(%esi),%esi

77ed44f0 <_XLATEOBJ_hGetColorTransform@4>:
77ed44f0:	55                   	push   %ebp
77ed44f1:	89 e5                	mov    %esp,%ebp
77ed44f3:	83 ec 10             	sub    $0x10,%esp
77ed44f6:	68 3f b2 ed 77       	push   $0x77edb23f
77ed44fb:	68 20 a0 ed 77       	push   $0x77eda020
77ed4500:	ff 15 e8 10 ee 77    	call   *0x77ee10e8
77ed4506:	c7 04 24 78 00 00 00 	movl   $0x78,(%esp)
77ed450d:	e8 fe 53 00 00       	call   77ed9910 <_SetLastError@4>
77ed4512:	31 c0                	xor    %eax,%eax
77ed4514:	c9                   	leave  
77ed4515:	c2 04 00             	ret    $0x4
77ed4518:	90                   	nop    
77ed4519:	8d b4 26 00 00 00 00 	lea    0x0(%esi),%esi

77ed4520 <_XLATEOBJ_iXlate@8>:
77ed4520:	55                   	push   %ebp
77ed4521:	89 e5                	mov    %esp,%ebp
77ed4523:	83 ec 10             	sub    $0x10,%esp
77ed4526:	68 5b b2 ed 77       	push   $0x77edb25b
77ed452b:	68 20 a0 ed 77       	push   $0x77eda020
77ed4530:	ff 15 e8 10 ee 77    	call   *0x77ee10e8
77ed4536:	c7 04 24 78 00 00 00 	movl   $0x78,(%esp)
77ed453d:	e8 ce 53 00 00       	call   77ed9910 <_SetLastError@4>
77ed4542:	31 c0                	xor    %eax,%eax
77ed4544:	c9                   	leave  
77ed4545:	c2 08 00             	ret    $0x8
77ed4548:	90                   	nop    
77ed4549:	8d b4 26 00 00 00 00 	lea    0x0(%esi),%esi

77ed4550 <_XLATEOBJ_piVector@4>:
77ed4550:	55                   	push   %ebp
77ed4551:	89 e5                	mov    %esp,%ebp
77ed4553:	83 ec 10             	sub    $0x10,%esp
77ed4556:	68 6b b2 ed 77       	push   $0x77edb26b
77ed455b:	68 20 a0 ed 77       	push   $0x77eda020
77ed4560:	ff 15 e8 10 ee 77    	call   *0x77ee10e8
77ed4566:	c7 04 24 78 00 00 00 	movl   $0x78,(%esp)
77ed456d:	e8 9e 53 00 00       	call   77ed9910 <_SetLastError@4>
77ed4572:	31 c0                	xor    %eax,%eax
77ed4574:	c9                   	leave  
77ed4575:	c2 04 00             	ret    $0x4
77ed4578:	90                   	nop    
77ed4579:	8d b4 26 00 00 00 00 	lea    0x0(%esi),%esi

77ed4580 <_DdCreateDirectDrawObject@8>:
77ed4580:	55                   	push   %ebp
77ed4581:	89 e5                	mov    %esp,%ebp
77ed4583:	83 ec 10             	sub    $0x10,%esp
77ed4586:	68 7d b2 ed 77       	push   $0x77edb27d
77ed458b:	68 20 a0 ed 77       	push   $0x77eda020
77ed4590:	ff 15 e8 10 ee 77    	call   *0x77ee10e8
77ed4596:	c7 04 24 78 00 00 00 	movl   $0x78,(%esp)
77ed459d:	e8 6e 53 00 00       	call   77ed9910 <_SetLastError@4>
77ed45a2:	31 c0                	xor    %eax,%eax
77ed45a4:	c9                   	leave  
77ed45a5:	c2 08 00             	ret    $0x8
77ed45a8:	90                   	nop    
77ed45a9:	8d b4 26 00 00 00 00 	lea    0x0(%esi),%esi

77ed45b0 <_DdQueryDirectDrawObject@44>:
77ed45b0:	55                   	push   %ebp
77ed45b1:	89 e5                	mov    %esp,%ebp
77ed45b3:	83 ec 10             	sub    $0x10,%esp
77ed45b6:	68 96 b2 ed 77       	push   $0x77edb296
77ed45bb:	68 20 a0 ed 77       	push   $0x77eda020
77ed45c0:	ff 15 e8 10 ee 77    	call   *0x77ee10e8
77ed45c6:	c7 04 24 78 00 00 00 	movl   $0x78,(%esp)
77ed45cd:	e8 3e 53 00 00       	call   77ed9910 <_SetLastError@4>
77ed45d2:	31 c0                	xor    %eax,%eax
77ed45d4:	c9                   	leave  
77ed45d5:	c2 2c 00             	ret    $0x2c
77ed45d8:	90                   	nop    
77ed45d9:	8d b4 26 00 00 00 00 	lea    0x0(%esi),%esi

77ed45e0 <_DdDeleteDirectDrawObject@4>:
77ed45e0:	55                   	push   %ebp
77ed45e1:	89 e5                	mov    %esp,%ebp
77ed45e3:	83 ec 10             	sub    $0x10,%esp
77ed45e6:	68 ae b2 ed 77       	push   $0x77edb2ae
77ed45eb:	68 20 a0 ed 77       	push   $0x77eda020
77ed45f0:	ff 15 e8 10 ee 77    	call   *0x77ee10e8
77ed45f6:	c7 04 24 78 00 00 00 	movl   $0x78,(%esp)
77ed45fd:	e8 0e 53 00 00       	call   77ed9910 <_SetLastError@4>
77ed4602:	31 c0                	xor    %eax,%eax
77ed4604:	c9                   	leave  
77ed4605:	c2 04 00             	ret    $0x4
77ed4608:	90                   	nop    
77ed4609:	8d b4 26 00 00 00 00 	lea    0x0(%esi),%esi

77ed4610 <_DdCreateSurfaceObject@8>:
77ed4610:	55                   	push   %ebp
77ed4611:	89 e5                	mov    %esp,%ebp
77ed4613:	83 ec 10             	sub    $0x10,%esp
77ed4616:	68 c7 b2 ed 77       	push   $0x77edb2c7
77ed461b:	68 20 a0 ed 77       	push   $0x77eda020
77ed4620:	ff 15 e8 10 ee 77    	call   *0x77ee10e8
77ed4626:	c7 04 24 78 00 00 00 	movl   $0x78,(%esp)
77ed462d:	e8 de 52 00 00       	call   77ed9910 <_SetLastError@4>
77ed4632:	31 c0                	xor    %eax,%eax
77ed4634:	c9                   	leave  
77ed4635:	c2 08 00             	ret    $0x8
77ed4638:	90                   	nop    
77ed4639:	8d b4 26 00 00 00 00 	lea    0x0(%esi),%esi

77ed4640 <_DdDeleteSurfaceObject@4>:
77ed4640:	55                   	push   %ebp
77ed4641:	89 e5                	mov    %esp,%ebp
77ed4643:	83 ec 10             	sub    $0x10,%esp
77ed4646:	68 dd b2 ed 77       	push   $0x77edb2dd
77ed464b:	68 20 a0 ed 77       	push   $0x77eda020
77ed4650:	ff 15 e8 10 ee 77    	call   *0x77ee10e8
77ed4656:	c7 04 24 78 00 00 00 	movl   $0x78,(%esp)
77ed465d:	e8 ae 52 00 00       	call   77ed9910 <_SetLastError@4>
77ed4662:	31 c0                	xor    %eax,%eax
77ed4664:	c9                   	leave  
77ed4665:	c2 04 00             	ret    $0x4
77ed4668:	90                   	nop    
77ed4669:	8d b4 26 00 00 00 00 	lea    0x0(%esi),%esi

77ed4670 <_DdResetVisrgn@8>:
77ed4670:	55                   	push   %ebp
77ed4671:	89 e5                	mov    %esp,%ebp
77ed4673:	83 ec 10             	sub    $0x10,%esp
77ed4676:	68 f3 b2 ed 77       	push   $0x77edb2f3
77ed467b:	68 20 a0 ed 77       	push   $0x77eda020
77ed4680:	ff 15 e8 10 ee 77    	call   *0x77ee10e8
77ed4686:	c7 04 24 78 00 00 00 	movl   $0x78,(%esp)
77ed468d:	e8 7e 52 00 00       	call   77ed9910 <_SetLastError@4>
77ed4692:	31 c0                	xor    %eax,%eax
77ed4694:	c9                   	leave  
77ed4695:	c2 08 00             	ret    $0x8
77ed4698:	90                   	nop    
77ed4699:	8d b4 26 00 00 00 00 	lea    0x0(%esi),%esi

77ed46a0 <_DdGetDC@8>:
77ed46a0:	55                   	push   %ebp
77ed46a1:	89 e5                	mov    %esp,%ebp
77ed46a3:	83 ec 10             	sub    $0x10,%esp
77ed46a6:	68 01 b3 ed 77       	push   $0x77edb301
77ed46ab:	68 20 a0 ed 77       	push   $0x77eda020
77ed46b0:	ff 15 e8 10 ee 77    	call   *0x77ee10e8
77ed46b6:	c7 04 24 78 00 00 00 	movl   $0x78,(%esp)
77ed46bd:	e8 4e 52 00 00       	call   77ed9910 <_SetLastError@4>
77ed46c2:	31 c0                	xor    %eax,%eax
77ed46c4:	c9                   	leave  
77ed46c5:	c2 08 00             	ret    $0x8
77ed46c8:	90                   	nop    
77ed46c9:	8d b4 26 00 00 00 00 	lea    0x0(%esi),%esi

77ed46d0 <_DdReleaseDC@4>:
77ed46d0:	55                   	push   %ebp
77ed46d1:	89 e5                	mov    %esp,%ebp
77ed46d3:	83 ec 10             	sub    $0x10,%esp
77ed46d6:	68 09 b3 ed 77       	push   $0x77edb309
77ed46db:	68 20 a0 ed 77       	push   $0x77eda020
77ed46e0:	ff 15 e8 10 ee 77    	call   *0x77ee10e8
77ed46e6:	c7 04 24 78 00 00 00 	movl   $0x78,(%esp)
77ed46ed:	e8 1e 52 00 00       	call   77ed9910 <_SetLastError@4>
77ed46f2:	31 c0                	xor    %eax,%eax
77ed46f4:	c9                   	leave  
77ed46f5:	c2 04 00             	ret    $0x4
77ed46f8:	90                   	nop    
77ed46f9:	8d b4 26 00 00 00 00 	lea    0x0(%esi),%esi

77ed4700 <_DdCreateDIBSection@24>:
77ed4700:	55                   	push   %ebp
77ed4701:	89 e5                	mov    %esp,%ebp
77ed4703:	83 ec 10             	sub    $0x10,%esp
77ed4706:	68 15 b3 ed 77       	push   $0x77edb315
77ed470b:	68 20 a0 ed 77       	push   $0x77eda020
77ed4710:	ff 15 e8 10 ee 77    	call   *0x77ee10e8
77ed4716:	c7 04 24 78 00 00 00 	movl   $0x78,(%esp)
77ed471d:	e8 ee 51 00 00       	call   77ed9910 <_SetLastError@4>
77ed4722:	31 c0                	xor    %eax,%eax
77ed4724:	c9                   	leave  
77ed4725:	c2 18 00             	ret    $0x18
77ed4728:	90                   	nop    
77ed4729:	8d b4 26 00 00 00 00 	lea    0x0(%esi),%esi

77ed4730 <_DdReenableDirectDrawObject@8>:
77ed4730:	55                   	push   %ebp
77ed4731:	89 e5                	mov    %esp,%ebp
77ed4733:	83 ec 10             	sub    $0x10,%esp
77ed4736:	68 28 b3 ed 77       	push   $0x77edb328
77ed473b:	68 20 a0 ed 77       	push   $0x77eda020
77ed4740:	ff 15 e8 10 ee 77    	call   *0x77ee10e8
77ed4746:	c7 04 24 78 00 00 00 	movl   $0x78,(%esp)
77ed474d:	e8 be 51 00 00       	call   77ed9910 <_SetLastError@4>
77ed4752:	31 c0                	xor    %eax,%eax
77ed4754:	c9                   	leave  
77ed4755:	c2 08 00             	ret    $0x8
77ed4758:	90                   	nop    
77ed4759:	8d b4 26 00 00 00 00 	lea    0x0(%esi),%esi

77ed4760 <_DdAttachSurface@8>:
77ed4760:	55                   	push   %ebp
77ed4761:	89 e5                	mov    %esp,%ebp
77ed4763:	83 ec 10             	sub    $0x10,%esp
77ed4766:	68 43 b3 ed 77       	push   $0x77edb343
77ed476b:	68 20 a0 ed 77       	push   $0x77eda020
77ed4770:	ff 15 e8 10 ee 77    	call   *0x77ee10e8
77ed4776:	c7 04 24 78 00 00 00 	movl   $0x78,(%esp)
77ed477d:	e8 8e 51 00 00       	call   77ed9910 <_SetLastError@4>
77ed4782:	31 c0                	xor    %eax,%eax
77ed4784:	c9                   	leave  
77ed4785:	c2 08 00             	ret    $0x8
77ed4788:	90                   	nop    
77ed4789:	8d b4 26 00 00 00 00 	lea    0x0(%esi),%esi

77ed4790 <_DdUnattachSurface@8>:
77ed4790:	55                   	push   %ebp
77ed4791:	89 e5                	mov    %esp,%ebp
77ed4793:	83 ec 10             	sub    $0x10,%esp
77ed4796:	68 53 b3 ed 77       	push   $0x77edb353
77ed479b:	68 20 a0 ed 77       	push   $0x77eda020
77ed47a0:	ff 15 e8 10 ee 77    	call   *0x77ee10e8
77ed47a6:	c7 04 24 78 00 00 00 	movl   $0x78,(%esp)
77ed47ad:	e8 5e 51 00 00       	call   77ed9910 <_SetLastError@4>
77ed47b2:	c9                   	leave  
77ed47b3:	c2 08 00             	ret    $0x8
77ed47b6:	8d 76 00             	lea    0x0(%esi),%esi
77ed47b9:	8d bc 27 00 00 00 00 	lea    0x0(%edi),%edi

77ed47c0 <_DdQueryDisplaySettingsUniqueness@0>:
77ed47c0:	55                   	push   %ebp
77ed47c1:	89 e5                	mov    %esp,%ebp
77ed47c3:	83 ec 10             	sub    $0x10,%esp
77ed47c6:	68 70 b3 ed 77       	push   $0x77edb370
77ed47cb:	68 20 a0 ed 77       	push   $0x77eda020
77ed47d0:	ff 15 e8 10 ee 77    	call   *0x77ee10e8
77ed47d6:	c7 04 24 78 00 00 00 	movl   $0x78,(%esp)
77ed47dd:	e8 2e 51 00 00       	call   77ed9910 <_SetLastError@4>
77ed47e2:	31 c0                	xor    %eax,%eax
77ed47e4:	c9                   	leave  
77ed47e5:	c3                   	ret    
77ed47e6:	8d 76 00             	lea    0x0(%esi),%esi
77ed47e9:	8d bc 27 00 00 00 00 	lea    0x0(%edi),%edi

77ed47f0 <_DdGetDxHandle@12>:
77ed47f0:	55                   	push   %ebp
77ed47f1:	89 e5                	mov    %esp,%ebp
77ed47f3:	83 ec 10             	sub    $0x10,%esp
77ed47f6:	68 91 b3 ed 77       	push   $0x77edb391
77ed47fb:	68 20 a0 ed 77       	push   $0x77eda020
77ed4800:	ff 15 e8 10 ee 77    	call   *0x77ee10e8
77ed4806:	c7 04 24 78 00 00 00 	movl   $0x78,(%esp)
77ed480d:	e8 fe 50 00 00       	call   77ed9910 <_SetLastError@4>
77ed4812:	31 c0                	xor    %eax,%eax
77ed4814:	c9                   	leave  
77ed4815:	c2 0c 00             	ret    $0xc
77ed4818:	90                   	nop    
77ed4819:	8d b4 26 00 00 00 00 	lea    0x0(%esi),%esi

77ed4820 <_DdSetGammaRamp@12>:
77ed4820:	55                   	push   %ebp
77ed4821:	89 e5                	mov    %esp,%ebp
77ed4823:	83 ec 10             	sub    $0x10,%esp
77ed4826:	68 9f b3 ed 77       	push   $0x77edb39f
77ed482b:	68 20 a0 ed 77       	push   $0x77eda020
77ed4830:	ff 15 e8 10 ee 77    	call   *0x77ee10e8
77ed4836:	c7 04 24 78 00 00 00 	movl   $0x78,(%esp)
77ed483d:	e8 ce 50 00 00       	call   77ed9910 <_SetLastError@4>
77ed4842:	31 c0                	xor    %eax,%eax
77ed4844:	c9                   	leave  
77ed4845:	c2 0c 00             	ret    $0xc
77ed4848:	90                   	nop    
77ed4849:	8d b4 26 00 00 00 00 	lea    0x0(%esi),%esi

77ed4850 <_DdSwapTextureHandles@12>:
77ed4850:	55                   	push   %ebp
77ed4851:	89 e5                	mov    %esp,%ebp
77ed4853:	83 ec 10             	sub    $0x10,%esp
77ed4856:	68 ae b3 ed 77       	push   $0x77edb3ae
77ed485b:	68 20 a0 ed 77       	push   $0x77eda020
77ed4860:	ff 15 e8 10 ee 77    	call   *0x77ee10e8
77ed4866:	c7 04 24 78 00 00 00 	movl   $0x78,(%esp)
77ed486d:	e8 9e 50 00 00       	call   77ed9910 <_SetLastError@4>
77ed4872:	31 c0                	xor    %eax,%eax
77ed4874:	c9                   	leave  
77ed4875:	c2 0c 00             	ret    $0xc
77ed4878:	90                   	nop    
77ed4879:	8d b4 26 00 00 00 00 	lea    0x0(%esi),%esi

77ed4880 <_GdiPlayEMF@20>:
77ed4880:	55                   	push   %ebp
77ed4881:	89 e5                	mov    %esp,%ebp
77ed4883:	83 ec 10             	sub    $0x10,%esp
77ed4886:	68 c3 b3 ed 77       	push   $0x77edb3c3
77ed488b:	68 20 a0 ed 77       	push   $0x77eda020
77ed4890:	ff 15 e8 10 ee 77    	call   *0x77ee10e8
77ed4896:	c7 04 24 78 00 00 00 	movl   $0x78,(%esp)
77ed489d:	e8 6e 50 00 00       	call   77ed9910 <_SetLastError@4>
77ed48a2:	31 c0                	xor    %eax,%eax
77ed48a4:	c9                   	leave  
77ed48a5:	c2 14 00             	ret    $0x14
77ed48a8:	90                   	nop    
77ed48a9:	8d b4 26 00 00 00 00 	lea    0x0(%esi),%esi

77ed48b0 <_GdiInitSpool@0>:
77ed48b0:	55                   	push   %ebp
77ed48b1:	89 e5                	mov    %esp,%ebp
77ed48b3:	83 ec 10             	sub    $0x10,%esp
77ed48b6:	68 ce b3 ed 77       	push   $0x77edb3ce
77ed48bb:	68 20 a0 ed 77       	push   $0x77eda020
77ed48c0:	ff 15 e8 10 ee 77    	call   *0x77ee10e8
77ed48c6:	c7 04 24 78 00 00 00 	movl   $0x78,(%esp)
77ed48cd:	e8 3e 50 00 00       	call   77ed9910 <_SetLastError@4>
77ed48d2:	31 c0                	xor    %eax,%eax
77ed48d4:	c9                   	leave  
77ed48d5:	c3                   	ret    
77ed48d6:	8d 76 00             	lea    0x0(%esi),%esi
77ed48d9:	8d bc 27 00 00 00 00 	lea    0x0(%edi),%edi

77ed48e0 <_GdiPlayPrivatePageEMF@12>:
77ed48e0:	55                   	push   %ebp
77ed48e1:	89 e5                	mov    %esp,%ebp
77ed48e3:	83 ec 10             	sub    $0x10,%esp
77ed48e6:	68 db b3 ed 77       	push   $0x77edb3db
77ed48eb:	68 20 a0 ed 77       	push   $0x77eda020
77ed48f0:	ff 15 e8 10 ee 77    	call   *0x77ee10e8
77ed48f6:	c7 04 24 78 00 00 00 	movl   $0x78,(%esp)
77ed48fd:	e8 0e 50 00 00       	call   77ed9910 <_SetLastError@4>
77ed4902:	31 c0                	xor    %eax,%eax
77ed4904:	c9                   	leave  
77ed4905:	c2 0c 00             	ret    $0xc
77ed4908:	90                   	nop    
77ed4909:	8d b4 26 00 00 00 00 	lea    0x0(%esi),%esi

77ed4910 <_GdiInitializeLanguagePack@4>:
77ed4910:	55                   	push   %ebp
77ed4911:	89 e5                	mov    %esp,%ebp
77ed4913:	83 ec 10             	sub    $0x10,%esp
77ed4916:	68 f1 b3 ed 77       	push   $0x77edb3f1
77ed491b:	68 20 a0 ed 77       	push   $0x77eda020
77ed4920:	ff 15 e8 10 ee 77    	call   *0x77ee10e8
77ed4926:	c7 45 08 78 00 00 00 	movl   $0x78,0x8(%ebp)
77ed492d:	83 c4 10             	add    $0x10,%esp
77ed4930:	c9                   	leave  
77ed4931:	e9 da 4f 00 00       	jmp    77ed9910 <_SetLastError@4>
77ed4936:	90                   	nop    
77ed4937:	90                   	nop    
77ed4938:	90                   	nop    
77ed4939:	90                   	nop    
77ed493a:	90                   	nop    
77ed493b:	90                   	nop    
77ed493c:	90                   	nop    
77ed493d:	90                   	nop    
77ed493e:	90                   	nop    
77ed493f:	90                   	nop    

77ed4940 <_DeviceCapabilitiesExA@20>:
77ed4940:	55                   	push   %ebp
77ed4941:	89 e5                	mov    %esp,%ebp
77ed4943:	83 ec 10             	sub    $0x10,%esp
77ed4946:	68 10 b4 ed 77       	push   $0x77edb410
77ed494b:	68 28 b4 ed 77       	push   $0x77edb428
77ed4950:	ff 15 e8 10 ee 77    	call   *0x77ee10e8
77ed4956:	c7 04 24 78 00 00 00 	movl   $0x78,(%esp)
77ed495d:	e8 ae 4f 00 00       	call   77ed9910 <_SetLastError@4>
77ed4962:	31 c0                	xor    %eax,%eax
77ed4964:	c9                   	leave  
77ed4965:	c2 14 00             	ret    $0x14
77ed4968:	90                   	nop    
77ed4969:	8d b4 26 00 00 00 00 	lea    0x0(%esi),%esi

77ed4970 <_EnumFontsA@16>:
77ed4970:	55                   	push   %ebp
77ed4971:	89 e5                	mov    %esp,%ebp
77ed4973:	83 ec 10             	sub    $0x10,%esp
77ed4976:	68 5d b4 ed 77       	push   $0x77edb45d
77ed497b:	68 28 b4 ed 77       	push   $0x77edb428
77ed4980:	ff 15 e8 10 ee 77    	call   *0x77ee10e8
77ed4986:	c7 04 24 78 00 00 00 	movl   $0x78,(%esp)
77ed498d:	e8 7e 4f 00 00       	call   77ed9910 <_SetLastError@4>
77ed4992:	31 c0                	xor    %eax,%eax
77ed4994:	c9                   	leave  
77ed4995:	c2 10 00             	ret    $0x10
77ed4998:	90                   	nop    
77ed4999:	8d b4 26 00 00 00 00 	lea    0x0(%esi),%esi

77ed49a0 <_GetOutlineTextMetricsA@12>:
77ed49a0:	55                   	push   %ebp
77ed49a1:	89 e5                	mov    %esp,%ebp
77ed49a3:	83 ec 10             	sub    $0x10,%esp
77ed49a6:	68 68 b4 ed 77       	push   $0x77edb468
77ed49ab:	68 28 b4 ed 77       	push   $0x77edb428
77ed49b0:	ff 15 e8 10 ee 77    	call   *0x77ee10e8
77ed49b6:	c7 04 24 78 00 00 00 	movl   $0x78,(%esp)
77ed49bd:	e8 4e 4f 00 00       	call   77ed9910 <_SetLastError@4>
77ed49c2:	31 c0                	xor    %eax,%eax
77ed49c4:	c9                   	leave  
77ed49c5:	c2 0c 00             	ret    $0xc
77ed49c8:	90                   	nop    
77ed49c9:	8d b4 26 00 00 00 00 	lea    0x0(%esi),%esi

77ed49d0 <_GetCharacterPlacementA@24>:
77ed49d0:	55                   	push   %ebp
77ed49d1:	89 e5                	mov    %esp,%ebp
77ed49d3:	83 ec 10             	sub    $0x10,%esp
77ed49d6:	68 7f b4 ed 77       	push   $0x77edb47f
77ed49db:	68 28 b4 ed 77       	push   $0x77edb428
77ed49e0:	ff 15 e8 10 ee 77    	call   *0x77ee10e8
77ed49e6:	c7 04 24 78 00 00 00 	movl   $0x78,(%esp)
77ed49ed:	e8 1e 4f 00 00       	call   77ed9910 <_SetLastError@4>
77ed49f2:	31 c0                	xor    %eax,%eax
77ed49f4:	c9                   	leave  
77ed49f5:	c2 18 00             	ret    $0x18
77ed49f8:	90                   	nop    
77ed49f9:	8d b4 26 00 00 00 00 	lea    0x0(%esi),%esi

77ed4a00 <_StartDocA@8>:
77ed4a00:	55                   	push   %ebp
77ed4a01:	89 e5                	mov    %esp,%ebp
77ed4a03:	83 ec 10             	sub    $0x10,%esp
77ed4a06:	68 96 b4 ed 77       	push   $0x77edb496
77ed4a0b:	68 28 b4 ed 77       	push   $0x77edb428
77ed4a10:	ff 15 e8 10 ee 77    	call   *0x77ee10e8
77ed4a16:	c7 04 24 78 00 00 00 	movl   $0x78,(%esp)
77ed4a1d:	e8 ee 4e 00 00       	call   77ed9910 <_SetLastError@4>
77ed4a22:	31 c0                	xor    %eax,%eax
77ed4a24:	c9                   	leave  
77ed4a25:	c2 08 00             	ret    $0x8
77ed4a28:	90                   	nop    
77ed4a29:	8d b4 26 00 00 00 00 	lea    0x0(%esi),%esi

77ed4a30 <_PolyTextOutA@12>:
77ed4a30:	55                   	push   %ebp
77ed4a31:	89 e5                	mov    %esp,%ebp
77ed4a33:	83 ec 10             	sub    $0x10,%esp
77ed4a36:	68 a0 b4 ed 77       	push   $0x77edb4a0
77ed4a3b:	68 28 b4 ed 77       	push   $0x77edb428
77ed4a40:	ff 15 e8 10 ee 77    	call   *0x77ee10e8
77ed4a46:	c7 04 24 78 00 00 00 	movl   $0x78,(%esp)
77ed4a4d:	e8 be 4e 00 00       	call   77ed9910 <_SetLastError@4>
77ed4a52:	31 c0                	xor    %eax,%eax
77ed4a54:	c9                   	leave  
77ed4a55:	c2 0c 00             	ret    $0xc
77ed4a58:	90                   	nop    
77ed4a59:	8d b4 26 00 00 00 00 	lea    0x0(%esi),%esi

77ed4a60 <_GetKerningPairsA@12>:
77ed4a60:	55                   	push   %ebp
77ed4a61:	89 e5                	mov    %esp,%ebp
77ed4a63:	83 ec 10             	sub    $0x10,%esp
77ed4a66:	68 ad b4 ed 77       	push   $0x77edb4ad
77ed4a6b:	68 28 b4 ed 77       	push   $0x77edb428
77ed4a70:	ff 15 e8 10 ee 77    	call   *0x77ee10e8
77ed4a76:	c7 04 24 78 00 00 00 	movl   $0x78,(%esp)
77ed4a7d:	e8 8e 4e 00 00       	call   77ed9910 <_SetLastError@4>
77ed4a82:	31 c0                	xor    %eax,%eax
77ed4a84:	c9                   	leave  
77ed4a85:	c2 0c 00             	ret    $0xc
77ed4a88:	90                   	nop    
77ed4a89:	8d b4 26 00 00 00 00 	lea    0x0(%esi),%esi

77ed4a90 <_GetLogColorSpaceA@12>:
77ed4a90:	55                   	push   %ebp
77ed4a91:	89 e5                	mov    %esp,%ebp
77ed4a93:	83 ec 10             	sub    $0x10,%esp
77ed4a96:	68 be b4 ed 77       	push   $0x77edb4be
77ed4a9b:	68 28 b4 ed 77       	push   $0x77edb428
77ed4aa0:	ff 15 e8 10 ee 77    	call   *0x77ee10e8
77ed4aa6:	c7 04 24 78 00 00 00 	movl   $0x78,(%esp)
77ed4aad:	e8 5e 4e 00 00       	call   77ed9910 <_SetLastError@4>
77ed4ab2:	31 c0                	xor    %eax,%eax
77ed4ab4:	c9                   	leave  
77ed4ab5:	c2 0c 00             	ret    $0xc
77ed4ab8:	90                   	nop    
77ed4ab9:	8d b4 26 00 00 00 00 	lea    0x0(%esi),%esi

77ed4ac0 <_CreateColorSpaceA@4>:
77ed4ac0:	55                   	push   %ebp
77ed4ac1:	89 e5                	mov    %esp,%ebp
77ed4ac3:	83 ec 10             	sub    $0x10,%esp
77ed4ac6:	68 d0 b4 ed 77       	push   $0x77edb4d0
77ed4acb:	68 28 b4 ed 77       	push   $0x77edb428
77ed4ad0:	ff 15 e8 10 ee 77    	call   *0x77ee10e8
77ed4ad6:	c7 04 24 78 00 00 00 	movl   $0x78,(%esp)
77ed4add:	e8 2e 4e 00 00       	call   77ed9910 <_SetLastError@4>
77ed4ae2:	31 c0                	xor    %eax,%eax
77ed4ae4:	c9                   	leave  
77ed4ae5:	c2 04 00             	ret    $0x4
77ed4ae8:	90                   	nop    
77ed4ae9:	8d b4 26 00 00 00 00 	lea    0x0(%esi),%esi

77ed4af0 <_GetICMProfileA@12>:
77ed4af0:	55                   	push   %ebp
77ed4af1:	89 e5                	mov    %esp,%ebp
77ed4af3:	83 ec 10             	sub    $0x10,%esp
77ed4af6:	68 e2 b4 ed 77       	push   $0x77edb4e2
77ed4afb:	68 28 b4 ed 77       	push   $0x77edb428
77ed4b00:	ff 15 e8 10 ee 77    	call   *0x77ee10e8
77ed4b06:	c7 04 24 78 00 00 00 	movl   $0x78,(%esp)
77ed4b0d:	e8 fe 4d 00 00       	call   77ed9910 <_SetLastError@4>
77ed4b12:	31 c0                	xor    %eax,%eax
77ed4b14:	c9                   	leave  
77ed4b15:	c2 0c 00             	ret    $0xc
77ed4b18:	90                   	nop    
77ed4b19:	8d b4 26 00 00 00 00 	lea    0x0(%esi),%esi

77ed4b20 <_SetICMProfileA@8>:
77ed4b20:	55                   	push   %ebp
77ed4b21:	89 e5                	mov    %esp,%ebp
77ed4b23:	83 ec 10             	sub    $0x10,%esp
77ed4b26:	68 f1 b4 ed 77       	push   $0x77edb4f1
77ed4b2b:	68 28 b4 ed 77       	push   $0x77edb428
77ed4b30:	ff 15 e8 10 ee 77    	call   *0x77ee10e8
77ed4b36:	c7 04 24 78 00 00 00 	movl   $0x78,(%esp)
77ed4b3d:	e8 ce 4d 00 00       	call   77ed9910 <_SetLastError@4>
77ed4b42:	31 c0                	xor    %eax,%eax
77ed4b44:	c9                   	leave  
77ed4b45:	c2 08 00             	ret    $0x8
77ed4b48:	90                   	nop    
77ed4b49:	8d b4 26 00 00 00 00 	lea    0x0(%esi),%esi

77ed4b50 <_EnumICMProfilesA@12>:
77ed4b50:	55                   	push   %ebp
77ed4b51:	89 e5                	mov    %esp,%ebp
77ed4b53:	83 ec 10             	sub    $0x10,%esp
77ed4b56:	68 00 b5 ed 77       	push   $0x77edb500
77ed4b5b:	68 28 b4 ed 77       	push   $0x77edb428
77ed4b60:	ff 15 e8 10 ee 77    	call   *0x77ee10e8
77ed4b66:	c7 04 24 78 00 00 00 	movl   $0x78,(%esp)
77ed4b6d:	e8 9e 4d 00 00       	call   77ed9910 <_SetLastError@4>
77ed4b72:	31 c0                	xor    %eax,%eax
77ed4b74:	c9                   	leave  
77ed4b75:	c2 0c 00             	ret    $0xc
77ed4b78:	90                   	nop    
77ed4b79:	8d b4 26 00 00 00 00 	lea    0x0(%esi),%esi

77ed4b80 <_wglUseFontBitmapsA@16>:
77ed4b80:	55                   	push   %ebp
77ed4b81:	89 e5                	mov    %esp,%ebp
77ed4b83:	83 ec 10             	sub    $0x10,%esp
77ed4b86:	68 11 b5 ed 77       	push   $0x77edb511
77ed4b8b:	68 28 b4 ed 77       	push   $0x77edb428
77ed4b90:	ff 15 e8 10 ee 77    	call   *0x77ee10e8
77ed4b96:	c7 04 24 78 00 00 00 	movl   $0x78,(%esp)
77ed4b9d:	e8 6e 4d 00 00       	call   77ed9910 <_SetLastError@4>
77ed4ba2:	31 c0                	xor    %eax,%eax
77ed4ba4:	c9                   	leave  
77ed4ba5:	c2 10 00             	ret    $0x10
77ed4ba8:	90                   	nop    
77ed4ba9:	8d b4 26 00 00 00 00 	lea    0x0(%esi),%esi

77ed4bb0 <_wglUseFontOutlinesA@32>:
77ed4bb0:	55                   	push   %ebp
77ed4bb1:	89 e5                	mov    %esp,%ebp
77ed4bb3:	83 ec 10             	sub    $0x10,%esp
77ed4bb6:	68 24 b5 ed 77       	push   $0x77edb524
77ed4bbb:	68 28 b4 ed 77       	push   $0x77edb428
77ed4bc0:	ff 15 e8 10 ee 77    	call   *0x77ee10e8
77ed4bc6:	c7 04 24 78 00 00 00 	movl   $0x78,(%esp)
77ed4bcd:	e8 3e 4d 00 00       	call   77ed9910 <_SetLastError@4>
77ed4bd2:	31 c0                	xor    %eax,%eax
77ed4bd4:	c9                   	leave  
77ed4bd5:	c2 20 00             	ret    $0x20
77ed4bd8:	90                   	nop    
77ed4bd9:	8d b4 26 00 00 00 00 	lea    0x0(%esi),%esi

77ed4be0 <_UpdateICMRegKeyA@16>:
77ed4be0:	55                   	push   %ebp
77ed4be1:	89 e5                	mov    %esp,%ebp
77ed4be3:	83 ec 10             	sub    $0x10,%esp
77ed4be6:	68 38 b5 ed 77       	push   $0x77edb538
77ed4beb:	68 28 b4 ed 77       	push   $0x77edb428
77ed4bf0:	ff 15 e8 10 ee 77    	call   *0x77ee10e8
77ed4bf6:	c7 04 24 78 00 00 00 	movl   $0x78,(%esp)
77ed4bfd:	e8 0e 4d 00 00       	call   77ed9910 <_SetLastError@4>
77ed4c02:	31 c0                	xor    %eax,%eax
77ed4c04:	c9                   	leave  
77ed4c05:	c2 10 00             	ret    $0x10
77ed4c08:	90                   	nop    
77ed4c09:	8d b4 26 00 00 00 00 	lea    0x0(%esi),%esi

77ed4c10 <_RemoveFontResourceExA@12>:
77ed4c10:	55                   	push   %ebp
77ed4c11:	89 e5                	mov    %esp,%ebp
77ed4c13:	83 ec 10             	sub    $0x10,%esp
77ed4c16:	68 49 b5 ed 77       	push   $0x77edb549
77ed4c1b:	68 28 b4 ed 77       	push   $0x77edb428
77ed4c20:	ff 15 e8 10 ee 77    	call   *0x77ee10e8
77ed4c26:	c7 04 24 78 00 00 00 	movl   $0x78,(%esp)
77ed4c2d:	e8 de 4c 00 00       	call   77ed9910 <_SetLastError@4>
77ed4c32:	31 c0                	xor    %eax,%eax
77ed4c34:	c9                   	leave  
77ed4c35:	c2 0c 00             	ret    $0xc
77ed4c38:	90                   	nop    
77ed4c39:	8d b4 26 00 00 00 00 	lea    0x0(%esi),%esi

77ed4c40 <_CreateFontIndirectExA@4>:
77ed4c40:	55                   	push   %ebp
77ed4c41:	89 e5                	mov    %esp,%ebp
77ed4c43:	83 ec 10             	sub    $0x10,%esp
77ed4c46:	68 5f b5 ed 77       	push   $0x77edb55f
77ed4c4b:	68 28 b4 ed 77       	push   $0x77edb428
77ed4c50:	ff 15 e8 10 ee 77    	call   *0x77ee10e8
77ed4c56:	c7 04 24 78 00 00 00 	movl   $0x78,(%esp)
77ed4c5d:	e8 ae 4c 00 00       	call   77ed9910 <_SetLastError@4>
77ed4c62:	31 c0                	xor    %eax,%eax
77ed4c64:	c9                   	leave  
77ed4c65:	c2 04 00             	ret    $0x4
77ed4c68:	90                   	nop    
77ed4c69:	8d b4 26 00 00 00 00 	lea    0x0(%esi),%esi

77ed4c70 <_GetGlyphIndicesA@20>:
77ed4c70:	55                   	push   %ebp
77ed4c71:	89 e5                	mov    %esp,%ebp
77ed4c73:	83 ec 10             	sub    $0x10,%esp
77ed4c76:	68 75 b5 ed 77       	push   $0x77edb575
77ed4c7b:	68 28 b4 ed 77       	push   $0x77edb428
77ed4c80:	ff 15 e8 10 ee 77    	call   *0x77ee10e8
77ed4c86:	c7 04 24 78 00 00 00 	movl   $0x78,(%esp)
77ed4c8d:	e8 7e 4c 00 00       	call   77ed9910 <_SetLastError@4>
77ed4c92:	31 c0                	xor    %eax,%eax
77ed4c94:	c9                   	leave  
77ed4c95:	c2 14 00             	ret    $0x14
77ed4c98:	90                   	nop    
77ed4c99:	8d b4 26 00 00 00 00 	lea    0x0(%esi),%esi

77ed4ca0 <_GetStringBitmapA@20>:
77ed4ca0:	55                   	push   %ebp
77ed4ca1:	89 e5                	mov    %esp,%ebp
77ed4ca3:	83 ec 10             	sub    $0x10,%esp
77ed4ca6:	68 86 b5 ed 77       	push   $0x77edb586
77ed4cab:	68 28 b4 ed 77       	push   $0x77edb428
77ed4cb0:	ff 15 e8 10 ee 77    	call   *0x77ee10e8
77ed4cb6:	c7 04 24 78 00 00 00 	movl   $0x78,(%esp)
77ed4cbd:	e8 4e 4c 00 00       	call   77ed9910 <_SetLastError@4>
77ed4cc2:	31 c0                	xor    %eax,%eax
77ed4cc4:	c9                   	leave  
77ed4cc5:	c2 14 00             	ret    $0x14
77ed4cc8:	90                   	nop    
77ed4cc9:	90                   	nop    
77ed4cca:	90                   	nop    
77ed4ccb:	90                   	nop    
77ed4ccc:	90                   	nop    
77ed4ccd:	90                   	nop    
77ed4cce:	90                   	nop    
77ed4ccf:	90                   	nop    

77ed4cd0 <_DeviceCapabilitiesExW@20>:
77ed4cd0:	55                   	push   %ebp
77ed4cd1:	89 e5                	mov    %esp,%ebp
77ed4cd3:	83 ec 10             	sub    $0x10,%esp
77ed4cd6:	68 a0 b5 ed 77       	push   $0x77edb5a0
77ed4cdb:	68 b8 b5 ed 77       	push   $0x77edb5b8
77ed4ce0:	ff 15 e8 10 ee 77    	call   *0x77ee10e8
77ed4ce6:	c7 04 24 78 00 00 00 	movl   $0x78,(%esp)
77ed4ced:	e8 1e 4c 00 00       	call   77ed9910 <_SetLastError@4>
77ed4cf2:	31 c0                	xor    %eax,%eax
77ed4cf4:	c9                   	leave  
77ed4cf5:	c2 14 00             	ret    $0x14
77ed4cf8:	90                   	nop    
77ed4cf9:	8d b4 26 00 00 00 00 	lea    0x0(%esi),%esi

77ed4d00 <_EnumFontsW@16>:
77ed4d00:	55                   	push   %ebp
77ed4d01:	89 e5                	mov    %esp,%ebp
77ed4d03:	83 ec 10             	sub    $0x10,%esp
77ed4d06:	68 ed b5 ed 77       	push   $0x77edb5ed
77ed4d0b:	68 b8 b5 ed 77       	push   $0x77edb5b8
77ed4d10:	ff 15 e8 10 ee 77    	call   *0x77ee10e8
77ed4d16:	c7 04 24 78 00 00 00 	movl   $0x78,(%esp)
77ed4d1d:	e8 ee 4b 00 00       	call   77ed9910 <_SetLastError@4>
77ed4d22:	31 c0                	xor    %eax,%eax
77ed4d24:	c9                   	leave  
77ed4d25:	c2 10 00             	ret    $0x10
77ed4d28:	90                   	nop    
77ed4d29:	8d b4 26 00 00 00 00 	lea    0x0(%esi),%esi

77ed4d30 <_GetOutlineTextMetricsW@12>:
77ed4d30:	55                   	push   %ebp
77ed4d31:	89 e5                	mov    %esp,%ebp
77ed4d33:	83 ec 10             	sub    $0x10,%esp
77ed4d36:	68 f8 b5 ed 77       	push   $0x77edb5f8
77ed4d3b:	68 b8 b5 ed 77       	push   $0x77edb5b8
77ed4d40:	ff 15 e8 10 ee 77    	call   *0x77ee10e8
77ed4d46:	c7 04 24 78 00 00 00 	movl   $0x78,(%esp)
77ed4d4d:	e8 be 4b 00 00       	call   77ed9910 <_SetLastError@4>
77ed4d52:	31 c0                	xor    %eax,%eax
77ed4d54:	c9                   	leave  
77ed4d55:	c2 0c 00             	ret    $0xc
77ed4d58:	90                   	nop    
77ed4d59:	8d b4 26 00 00 00 00 	lea    0x0(%esi),%esi

77ed4d60 <_PolyTextOutW@12>:
77ed4d60:	55                   	push   %ebp
77ed4d61:	89 e5                	mov    %esp,%ebp
77ed4d63:	83 ec 10             	sub    $0x10,%esp
77ed4d66:	68 0f b6 ed 77       	push   $0x77edb60f
77ed4d6b:	68 b8 b5 ed 77       	push   $0x77edb5b8
77ed4d70:	ff 15 e8 10 ee 77    	call   *0x77ee10e8
77ed4d76:	c7 04 24 78 00 00 00 	movl   $0x78,(%esp)
77ed4d7d:	e8 8e 4b 00 00       	call   77ed9910 <_SetLastError@4>
77ed4d82:	31 c0                	xor    %eax,%eax
77ed4d84:	c9                   	leave  
77ed4d85:	c2 0c 00             	ret    $0xc
77ed4d88:	90                   	nop    
77ed4d89:	8d b4 26 00 00 00 00 	lea    0x0(%esi),%esi

77ed4d90 <_GetKerningPairsW@12>:
77ed4d90:	55                   	push   %ebp
77ed4d91:	89 e5                	mov    %esp,%ebp
77ed4d93:	83 ec 10             	sub    $0x10,%esp
77ed4d96:	68 1c b6 ed 77       	push   $0x77edb61c
77ed4d9b:	68 b8 b5 ed 77       	push   $0x77edb5b8
77ed4da0:	ff 15 e8 10 ee 77    	call   *0x77ee10e8
77ed4da6:	c7 04 24 78 00 00 00 	movl   $0x78,(%esp)
77ed4dad:	e8 5e 4b 00 00       	call   77ed9910 <_SetLastError@4>
77ed4db2:	31 c0                	xor    %eax,%eax
77ed4db4:	c9                   	leave  
77ed4db5:	c2 0c 00             	ret    $0xc
77ed4db8:	90                   	nop    
77ed4db9:	8d b4 26 00 00 00 00 	lea    0x0(%esi),%esi

77ed4dc0 <_GetLogColorSpaceW@12>:
77ed4dc0:	55                   	push   %ebp
77ed4dc1:	89 e5                	mov    %esp,%ebp
77ed4dc3:	83 ec 10             	sub    $0x10,%esp
77ed4dc6:	68 2d b6 ed 77       	push   $0x77edb62d
77ed4dcb:	68 b8 b5 ed 77       	push   $0x77edb5b8
77ed4dd0:	ff 15 e8 10 ee 77    	call   *0x77ee10e8
77ed4dd6:	c7 04 24 78 00 00 00 	movl   $0x78,(%esp)
77ed4ddd:	e8 2e 4b 00 00       	call   77ed9910 <_SetLastError@4>
77ed4de2:	31 c0                	xor    %eax,%eax
77ed4de4:	c9                   	leave  
77ed4de5:	c2 0c 00             	ret    $0xc
77ed4de8:	90                   	nop    
77ed4de9:	8d b4 26 00 00 00 00 	lea    0x0(%esi),%esi

77ed4df0 <_CreateColorSpaceW@4>:
77ed4df0:	55                   	push   %ebp
77ed4df1:	89 e5                	mov    %esp,%ebp
77ed4df3:	83 ec 10             	sub    $0x10,%esp
77ed4df6:	68 3f b6 ed 77       	push   $0x77edb63f
77ed4dfb:	68 b8 b5 ed 77       	push   $0x77edb5b8
77ed4e00:	ff 15 e8 10 ee 77    	call   *0x77ee10e8
77ed4e06:	c7 04 24 78 00 00 00 	movl   $0x78,(%esp)
77ed4e0d:	e8 fe 4a 00 00       	call   77ed9910 <_SetLastError@4>
77ed4e12:	31 c0                	xor    %eax,%eax
77ed4e14:	c9                   	leave  
77ed4e15:	c2 04 00             	ret    $0x4
77ed4e18:	90                   	nop    
77ed4e19:	8d b4 26 00 00 00 00 	lea    0x0(%esi),%esi

77ed4e20 <_GetICMProfileW@12>:
77ed4e20:	55                   	push   %ebp
77ed4e21:	89 e5                	mov    %esp,%ebp
77ed4e23:	83 ec 10             	sub    $0x10,%esp
77ed4e26:	68 51 b6 ed 77       	push   $0x77edb651
77ed4e2b:	68 b8 b5 ed 77       	push   $0x77edb5b8
77ed4e30:	ff 15 e8 10 ee 77    	call   *0x77ee10e8
77ed4e36:	c7 04 24 78 00 00 00 	movl   $0x78,(%esp)
77ed4e3d:	e8 ce 4a 00 00       	call   77ed9910 <_SetLastError@4>
77ed4e42:	31 c0                	xor    %eax,%eax
77ed4e44:	c9                   	leave  
77ed4e45:	c2 0c 00             	ret    $0xc
77ed4e48:	90                   	nop    
77ed4e49:	8d b4 26 00 00 00 00 	lea    0x0(%esi),%esi

77ed4e50 <_SetICMProfileW@8>:
77ed4e50:	55                   	push   %ebp
77ed4e51:	89 e5                	mov    %esp,%ebp
77ed4e53:	83 ec 10             	sub    $0x10,%esp
77ed4e56:	68 60 b6 ed 77       	push   $0x77edb660
77ed4e5b:	68 b8 b5 ed 77       	push   $0x77edb5b8
77ed4e60:	ff 15 e8 10 ee 77    	call   *0x77ee10e8
77ed4e66:	c7 04 24 78 00 00 00 	movl   $0x78,(%esp)
77ed4e6d:	e8 9e 4a 00 00       	call   77ed9910 <_SetLastError@4>
77ed4e72:	31 c0                	xor    %eax,%eax
77ed4e74:	c9                   	leave  
77ed4e75:	c2 08 00             	ret    $0x8
77ed4e78:	90                   	nop    
77ed4e79:	8d b4 26 00 00 00 00 	lea    0x0(%esi),%esi

77ed4e80 <_EnumICMProfilesW@12>:
77ed4e80:	55                   	push   %ebp
77ed4e81:	89 e5                	mov    %esp,%ebp
77ed4e83:	83 ec 10             	sub    $0x10,%esp
77ed4e86:	68 6f b6 ed 77       	push   $0x77edb66f
77ed4e8b:	68 b8 b5 ed 77       	push   $0x77edb5b8
77ed4e90:	ff 15 e8 10 ee 77    	call   *0x77ee10e8
77ed4e96:	c7 04 24 78 00 00 00 	movl   $0x78,(%esp)
77ed4e9d:	e8 6e 4a 00 00       	call   77ed9910 <_SetLastError@4>
77ed4ea2:	31 c0                	xor    %eax,%eax
77ed4ea4:	c9                   	leave  
77ed4ea5:	c2 0c 00             	ret    $0xc
77ed4ea8:	90                   	nop    
77ed4ea9:	8d b4 26 00 00 00 00 	lea    0x0(%esi),%esi

77ed4eb0 <_wglUseFontBitmapsW@16>:
77ed4eb0:	55                   	push   %ebp
77ed4eb1:	89 e5                	mov    %esp,%ebp
77ed4eb3:	83 ec 10             	sub    $0x10,%esp
77ed4eb6:	68 80 b6 ed 77       	push   $0x77edb680
77ed4ebb:	68 b8 b5 ed 77       	push   $0x77edb5b8
77ed4ec0:	ff 15 e8 10 ee 77    	call   *0x77ee10e8
77ed4ec6:	c7 04 24 78 00 00 00 	movl   $0x78,(%esp)
77ed4ecd:	e8 3e 4a 00 00       	call   77ed9910 <_SetLastError@4>
77ed4ed2:	31 c0                	xor    %eax,%eax
77ed4ed4:	c9                   	leave  
77ed4ed5:	c2 10 00             	ret    $0x10
77ed4ed8:	90                   	nop    
77ed4ed9:	8d b4 26 00 00 00 00 	lea    0x0(%esi),%esi

77ed4ee0 <_wglUseFontOutlinesW@32>:
77ed4ee0:	55                   	push   %ebp
77ed4ee1:	89 e5                	mov    %esp,%ebp
77ed4ee3:	83 ec 10             	sub    $0x10,%esp
77ed4ee6:	68 93 b6 ed 77       	push   $0x77edb693
77ed4eeb:	68 b8 b5 ed 77       	push   $0x77edb5b8
77ed4ef0:	ff 15 e8 10 ee 77    	call   *0x77ee10e8
77ed4ef6:	c7 04 24 78 00 00 00 	movl   $0x78,(%esp)
77ed4efd:	e8 0e 4a 00 00       	call   77ed9910 <_SetLastError@4>
77ed4f02:	31 c0                	xor    %eax,%eax
77ed4f04:	c9                   	leave  
77ed4f05:	c2 20 00             	ret    $0x20
77ed4f08:	90                   	nop    
77ed4f09:	8d b4 26 00 00 00 00 	lea    0x0(%esi),%esi

77ed4f10 <_UpdateICMRegKeyW@16>:
77ed4f10:	55                   	push   %ebp
77ed4f11:	89 e5                	mov    %esp,%ebp
77ed4f13:	83 ec 10             	sub    $0x10,%esp
77ed4f16:	68 a7 b6 ed 77       	push   $0x77edb6a7
77ed4f1b:	68 b8 b5 ed 77       	push   $0x77edb5b8
77ed4f20:	ff 15 e8 10 ee 77    	call   *0x77ee10e8
77ed4f26:	c7 04 24 78 00 00 00 	movl   $0x78,(%esp)
77ed4f2d:	e8 de 49 00 00       	call   77ed9910 <_SetLastError@4>
77ed4f32:	31 c0                	xor    %eax,%eax
77ed4f34:	c9                   	leave  
77ed4f35:	c2 10 00             	ret    $0x10
77ed4f38:	90                   	nop    
77ed4f39:	8d b4 26 00 00 00 00 	lea    0x0(%esi),%esi

77ed4f40 <_GetFontResourceInfoW@16>:
77ed4f40:	55                   	push   %ebp
77ed4f41:	89 e5                	mov    %esp,%ebp
77ed4f43:	83 ec 10             	sub    $0x10,%esp
77ed4f46:	68 b8 b6 ed 77       	push   $0x77edb6b8
77ed4f4b:	68 b8 b5 ed 77       	push   $0x77edb5b8
77ed4f50:	ff 15 e8 10 ee 77    	call   *0x77ee10e8
77ed4f56:	c7 04 24 78 00 00 00 	movl   $0x78,(%esp)
77ed4f5d:	e8 ae 49 00 00       	call   77ed9910 <_SetLastError@4>
77ed4f62:	31 c0                	xor    %eax,%eax
77ed4f64:	c9                   	leave  
77ed4f65:	c2 10 00             	ret    $0x10
77ed4f68:	90                   	nop    
77ed4f69:	8d b4 26 00 00 00 00 	lea    0x0(%esi),%esi

77ed4f70 <_EudcLoadLinkW@16>:
77ed4f70:	55                   	push   %ebp
77ed4f71:	89 e5                	mov    %esp,%ebp
77ed4f73:	83 ec 10             	sub    $0x10,%esp
77ed4f76:	68 cd b6 ed 77       	push   $0x77edb6cd
77ed4f7b:	68 b8 b5 ed 77       	push   $0x77edb5b8
77ed4f80:	ff 15 e8 10 ee 77    	call   *0x77ee10e8
77ed4f86:	c7 04 24 78 00 00 00 	movl   $0x78,(%esp)
77ed4f8d:	e8 7e 49 00 00       	call   77ed9910 <_SetLastError@4>
77ed4f92:	31 c0                	xor    %eax,%eax
77ed4f94:	c9                   	leave  
77ed4f95:	c2 10 00             	ret    $0x10
77ed4f98:	90                   	nop    
77ed4f99:	8d b4 26 00 00 00 00 	lea    0x0(%esi),%esi

77ed4fa0 <_EudcUnloadLinkW@8>:
77ed4fa0:	55                   	push   %ebp
77ed4fa1:	89 e5                	mov    %esp,%ebp
77ed4fa3:	83 ec 10             	sub    $0x10,%esp
77ed4fa6:	68 db b6 ed 77       	push   $0x77edb6db
77ed4fab:	68 b8 b5 ed 77       	push   $0x77edb5b8
77ed4fb0:	ff 15 e8 10 ee 77    	call   *0x77ee10e8
77ed4fb6:	c7 04 24 78 00 00 00 	movl   $0x78,(%esp)
77ed4fbd:	e8 4e 49 00 00       	call   77ed9910 <_SetLastError@4>
77ed4fc2:	31 c0                	xor    %eax,%eax
77ed4fc4:	c9                   	leave  
77ed4fc5:	c2 08 00             	ret    $0x8
77ed4fc8:	90                   	nop    
77ed4fc9:	8d b4 26 00 00 00 00 	lea    0x0(%esi),%esi

77ed4fd0 <_GdiAddFontResourceW@12>:
77ed4fd0:	55                   	push   %ebp
77ed4fd1:	89 e5                	mov    %esp,%ebp
77ed4fd3:	83 ec 10             	sub    $0x10,%esp
77ed4fd6:	68 eb b6 ed 77       	push   $0x77edb6eb
77ed4fdb:	68 b8 b5 ed 77       	push   $0x77edb5b8
77ed4fe0:	ff 15 e8 10 ee 77    	call   *0x77ee10e8
77ed4fe6:	c7 04 24 78 00 00 00 	movl   $0x78,(%esp)
77ed4fed:	e8 1e 49 00 00       	call   77ed9910 <_SetLastError@4>
77ed4ff2:	31 c0                	xor    %eax,%eax
77ed4ff4:	c9                   	leave  
77ed4ff5:	c2 0c 00             	ret    $0xc
77ed4ff8:	90                   	nop    
77ed4ff9:	8d b4 26 00 00 00 00 	lea    0x0(%esi),%esi

77ed5000 <_GdiConsoleTextOut@16>:
77ed5000:	55                   	push   %ebp
77ed5001:	89 e5                	mov    %esp,%ebp
77ed5003:	83 ec 10             	sub    $0x10,%esp
77ed5006:	68 ff b6 ed 77       	push   $0x77edb6ff
77ed500b:	68 b8 b5 ed 77       	push   $0x77edb5b8
77ed5010:	ff 15 e8 10 ee 77    	call   *0x77ee10e8
77ed5016:	c7 04 24 78 00 00 00 	movl   $0x78,(%esp)
77ed501d:	e8 ee 48 00 00       	call   77ed9910 <_SetLastError@4>
77ed5022:	31 c0                	xor    %eax,%eax
77ed5024:	c9                   	leave  
77ed5025:	c2 10 00             	ret    $0x10
77ed5028:	90                   	nop    
77ed5029:	8d b4 26 00 00 00 00 	lea    0x0(%esi),%esi

77ed5030 <_GetEUDCTimeStampExW@4>:
77ed5030:	55                   	push   %ebp
77ed5031:	89 e5                	mov    %esp,%ebp
77ed5033:	83 ec 10             	sub    $0x10,%esp
77ed5036:	68 11 b7 ed 77       	push   $0x77edb711
77ed503b:	68 b8 b5 ed 77       	push   $0x77edb5b8
77ed5040:	ff 15 e8 10 ee 77    	call   *0x77ee10e8
77ed5046:	c7 04 24 78 00 00 00 	movl   $0x78,(%esp)
77ed504d:	e8 be 48 00 00       	call   77ed9910 <_SetLastError@4>
77ed5052:	31 c0                	xor    %eax,%eax
77ed5054:	c9                   	leave  
77ed5055:	c2 04 00             	ret    $0x4
77ed5058:	90                   	nop    
77ed5059:	8d b4 26 00 00 00 00 	lea    0x0(%esi),%esi

77ed5060 <_RemoveFontResourceExW@12>:
77ed5060:	55                   	push   %ebp
77ed5061:	89 e5                	mov    %esp,%ebp
77ed5063:	83 ec 10             	sub    $0x10,%esp
77ed5066:	68 25 b7 ed 77       	push   $0x77edb725
77ed506b:	68 b8 b5 ed 77       	push   $0x77edb5b8
77ed5070:	ff 15 e8 10 ee 77    	call   *0x77ee10e8
77ed5076:	c7 04 24 78 00 00 00 	movl   $0x78,(%esp)
77ed507d:	e8 8e 48 00 00       	call   77ed9910 <_SetLastError@4>
77ed5082:	31 c0                	xor    %eax,%eax
77ed5084:	c9                   	leave  
77ed5085:	c2 0c 00             	ret    $0xc
77ed5088:	90                   	nop    
77ed5089:	8d b4 26 00 00 00 00 	lea    0x0(%esi),%esi

77ed5090 <_bInitSystemAndFontsDirectoriesW@8>:
77ed5090:	55                   	push   %ebp
77ed5091:	89 e5                	mov    %esp,%ebp
77ed5093:	83 ec 10             	sub    $0x10,%esp
77ed5096:	68 40 b7 ed 77       	push   $0x77edb740
77ed509b:	68 b8 b5 ed 77       	push   $0x77edb5b8
77ed50a0:	ff 15 e8 10 ee 77    	call   *0x77ee10e8
77ed50a6:	c7 04 24 78 00 00 00 	movl   $0x78,(%esp)
77ed50ad:	e8 5e 48 00 00       	call   77ed9910 <_SetLastError@4>
77ed50b2:	31 c0                	xor    %eax,%eax
77ed50b4:	c9                   	leave  
77ed50b5:	c2 08 00             	ret    $0x8
77ed50b8:	90                   	nop    
77ed50b9:	8d b4 26 00 00 00 00 	lea    0x0(%esi),%esi

77ed50c0 <_bMakePathNameW@16>:
77ed50c0:	55                   	push   %ebp
77ed50c1:	89 e5                	mov    %esp,%ebp
77ed50c3:	83 ec 10             	sub    $0x10,%esp
77ed50c6:	68 60 b7 ed 77       	push   $0x77edb760
77ed50cb:	68 b8 b5 ed 77       	push   $0x77edb5b8
77ed50d0:	ff 15 e8 10 ee 77    	call   *0x77ee10e8
77ed50d6:	c7 04 24 78 00 00 00 	movl   $0x78,(%esp)
77ed50dd:	e8 2e 48 00 00       	call   77ed9910 <_SetLastError@4>
77ed50e2:	31 c0                	xor    %eax,%eax
77ed50e4:	c9                   	leave  
77ed50e5:	c2 10 00             	ret    $0x10
77ed50e8:	90                   	nop    
77ed50e9:	8d b4 26 00 00 00 00 	lea    0x0(%esi),%esi

77ed50f0 <_CreateFontIndirectExW@4>:
77ed50f0:	55                   	push   %ebp
77ed50f1:	89 e5                	mov    %esp,%ebp
77ed50f3:	83 ec 10             	sub    $0x10,%esp
77ed50f6:	68 6f b7 ed 77       	push   $0x77edb76f
77ed50fb:	68 b8 b5 ed 77       	push   $0x77edb5b8
77ed5100:	ff 15 e8 10 ee 77    	call   *0x77ee10e8
77ed5106:	c7 04 24 78 00 00 00 	movl   $0x78,(%esp)
77ed510d:	e8 fe 47 00 00       	call   77ed9910 <_SetLastError@4>
77ed5112:	31 c0                	xor    %eax,%eax
77ed5114:	c9                   	leave  
77ed5115:	c2 04 00             	ret    $0x4
77ed5118:	90                   	nop    
77ed5119:	8d b4 26 00 00 00 00 	lea    0x0(%esi),%esi

77ed5120 <_GetGlyphIndicesW@20>:
77ed5120:	55                   	push   %ebp
77ed5121:	89 e5                	mov    %esp,%ebp
77ed5123:	83 ec 10             	sub    $0x10,%esp
77ed5126:	68 85 b7 ed 77       	push   $0x77edb785
77ed512b:	68 b8 b5 ed 77       	push   $0x77edb5b8
77ed5130:	ff 15 e8 10 ee 77    	call   *0x77ee10e8
77ed5136:	c7 04 24 78 00 00 00 	movl   $0x78,(%esp)
77ed513d:	e8 ce 47 00 00       	call   77ed9910 <_SetLastError@4>
77ed5142:	31 c0                	xor    %eax,%eax
77ed5144:	c9                   	leave  
77ed5145:	c2 14 00             	ret    $0x14
77ed5148:	90                   	nop    
77ed5149:	8d b4 26 00 00 00 00 	lea    0x0(%esi),%esi

77ed5150 <_GetStringBitmapW@20>:
77ed5150:	55                   	push   %ebp
77ed5151:	89 e5                	mov    %esp,%ebp
77ed5153:	83 ec 10             	sub    $0x10,%esp
77ed5156:	68 96 b7 ed 77       	push   $0x77edb796
77ed515b:	68 b8 b5 ed 77       	push   $0x77edb5b8
77ed5160:	ff 15 e8 10 ee 77    	call   *0x77ee10e8
77ed5166:	c7 04 24 78 00 00 00 	movl   $0x78,(%esp)
77ed516d:	e8 9e 47 00 00       	call   77ed9910 <_SetLastError@4>
77ed5172:	31 c0                	xor    %eax,%eax
77ed5174:	c9                   	leave  
77ed5175:	c2 14 00             	ret    $0x14
77ed5178:	90                   	nop    
77ed5179:	90                   	nop    
77ed517a:	90                   	nop    
77ed517b:	90                   	nop    
77ed517c:	90                   	nop    
77ed517d:	90                   	nop    
77ed517e:	90                   	nop    
77ed517f:	90                   	nop    

77ed5180 <_OpenGLEnable>:
77ed5180:	55                   	push   %ebp
77ed5181:	89 e5                	mov    %esp,%ebp
77ed5183:	50                   	push   %eax
77ed5184:	50                   	push   %eax
77ed5185:	a1 20 c0 ed 77       	mov    0x77edc020,%eax
77ed518a:	85 c0                	test   %eax,%eax
77ed518c:	74 46                	je     77ed51d4 <_OpenGLEnable+0x54>
77ed518e:	a1 68 c0 ed 77       	mov    0x77edc068,%eax
77ed5193:	85 c0                	test   %eax,%eax
77ed5195:	74 61                	je     77ed51f8 <_OpenGLEnable+0x78>
77ed5197:	a1 58 c0 ed 77       	mov    0x77edc058,%eax
77ed519c:	85 c0                	test   %eax,%eax
77ed519e:	0f 84 7c 00 00 00    	je     77ed5220 <_OpenGLEnable+0xa0>
77ed51a4:	a1 28 c0 ed 77       	mov    0x77edc028,%eax
77ed51a9:	85 c0                	test   %eax,%eax
77ed51ab:	0f 84 9f 00 00 00    	je     77ed5250 <_OpenGLEnable+0xd0>
77ed51b1:	a1 48 c0 ed 77       	mov    0x77edc048,%eax
77ed51b6:	85 c0                	test   %eax,%eax
77ed51b8:	0f 84 e7 00 00 00    	je     77ed52a5 <_OpenGLEnable+0x125>
77ed51be:	a1 38 c0 ed 77       	mov    0x77edc038,%eax
77ed51c3:	85 c0                	test   %eax,%eax
77ed51c5:	0f 84 ad 00 00 00    	je     77ed5278 <_OpenGLEnable+0xf8>
77ed51cb:	ba 01 00 00 00       	mov    $0x1,%edx
77ed51d0:	89 d0                	mov    %edx,%eax
77ed51d2:	c9                   	leave  
77ed51d3:	c3                   	ret    
77ed51d4:	83 ec 0c             	sub    $0xc,%esp
77ed51d7:	68 c0 b7 ed 77       	push   $0x77edb7c0
77ed51dc:	e8 3f 47 00 00       	call   77ed9920 <_LoadLibraryA@4>
77ed51e1:	31 d2                	xor    %edx,%edx
77ed51e3:	83 c4 0c             	add    $0xc,%esp
77ed51e6:	a3 20 c0 ed 77       	mov    %eax,0x77edc020
77ed51eb:	85 c0                	test   %eax,%eax
77ed51ed:	74 e1                	je     77ed51d0 <_OpenGLEnable+0x50>
77ed51ef:	a1 68 c0 ed 77       	mov    0x77edc068,%eax
77ed51f4:	85 c0                	test   %eax,%eax
77ed51f6:	75 9f                	jne    77ed5197 <_OpenGLEnable+0x17>
77ed51f8:	50                   	push   %eax
77ed51f9:	50                   	push   %eax
77ed51fa:	68 cd b7 ed 77       	push   $0x77edb7cd
77ed51ff:	a1 20 c0 ed 77       	mov    0x77edc020,%eax
77ed5204:	50                   	push   %eax
77ed5205:	e8 26 47 00 00       	call   77ed9930 <_GetProcAddress@8>
77ed520a:	a3 68 c0 ed 77       	mov    %eax,0x77edc068
77ed520f:	5a                   	pop    %edx
77ed5210:	31 d2                	xor    %edx,%edx
77ed5212:	59                   	pop    %ecx
77ed5213:	85 c0                	test   %eax,%eax
77ed5215:	74 b9                	je     77ed51d0 <_OpenGLEnable+0x50>
77ed5217:	a1 58 c0 ed 77       	mov    0x77edc058,%eax
77ed521c:	85 c0                	test   %eax,%eax
77ed521e:	75 84                	jne    77ed51a4 <_OpenGLEnable+0x24>
77ed5220:	50                   	push   %eax
77ed5221:	50                   	push   %eax
77ed5222:	68 e2 b7 ed 77       	push   $0x77edb7e2
77ed5227:	a1 20 c0 ed 77       	mov    0x77edc020,%eax
77ed522c:	50                   	push   %eax
77ed522d:	e8 fe 46 00 00       	call   77ed9930 <_GetProcAddress@8>
77ed5232:	a3 58 c0 ed 77       	mov    %eax,0x77edc058
77ed5237:	5a                   	pop    %edx
77ed5238:	31 d2                	xor    %edx,%edx
77ed523a:	59                   	pop    %ecx
77ed523b:	85 c0                	test   %eax,%eax
77ed523d:	74 91                	je     77ed51d0 <_OpenGLEnable+0x50>
77ed523f:	a1 28 c0 ed 77       	mov    0x77edc028,%eax
77ed5244:	85 c0                	test   %eax,%eax
77ed5246:	0f 85 65 ff ff ff    	jne    77ed51b1 <_OpenGLEnable+0x31>
77ed524c:	8d 74 26 00          	lea    0x0(%esi),%esi
77ed5250:	50                   	push   %eax
77ed5251:	50                   	push   %eax
77ed5252:	68 f4 b7 ed 77       	push   $0x77edb7f4
77ed5257:	a1 20 c0 ed 77       	mov    0x77edc020,%eax
77ed525c:	50                   	push   %eax
77ed525d:	e8 ce 46 00 00       	call   77ed9930 <_GetProcAddress@8>
77ed5262:	a3 28 c0 ed 77       	mov    %eax,0x77edc028
77ed5267:	5a                   	pop    %edx
77ed5268:	31 d2                	xor    %edx,%edx
77ed526a:	59                   	pop    %ecx
77ed526b:	85 c0                	test   %eax,%eax
77ed526d:	0f 84 5d ff ff ff    	je     77ed51d0 <_OpenGLEnable+0x50>
77ed5273:	e9 39 ff ff ff       	jmp    77ed51b1 <_OpenGLEnable+0x31>
77ed5278:	50                   	push   %eax
77ed5279:	50                   	push   %eax
77ed527a:	68 03 b8 ed 77       	push   $0x77edb803
77ed527f:	a1 20 c0 ed 77       	mov    0x77edc020,%eax
77ed5284:	50                   	push   %eax
77ed5285:	e8 a6 46 00 00       	call   77ed9930 <_GetProcAddress@8>
77ed528a:	a3 38 c0 ed 77       	mov    %eax,0x77edc038
77ed528f:	5a                   	pop    %edx
77ed5290:	31 d2                	xor    %edx,%edx
77ed5292:	59                   	pop    %ecx
77ed5293:	85 c0                	test   %eax,%eax
77ed5295:	0f 84 35 ff ff ff    	je     77ed51d0 <_OpenGLEnable+0x50>
77ed529b:	ba 01 00 00 00       	mov    $0x1,%edx
77ed52a0:	e9 2b ff ff ff       	jmp    77ed51d0 <_OpenGLEnable+0x50>
77ed52a5:	50                   	push   %eax
77ed52a6:	50                   	push   %eax
77ed52a7:	68 15 b8 ed 77       	push   $0x77edb815
77ed52ac:	a1 20 c0 ed 77       	mov    0x77edc020,%eax
77ed52b1:	50                   	push   %eax
77ed52b2:	e8 79 46 00 00       	call   77ed9930 <_GetProcAddress@8>
77ed52b7:	a3 48 c0 ed 77       	mov    %eax,0x77edc048
77ed52bc:	5a                   	pop    %edx
77ed52bd:	31 d2                	xor    %edx,%edx
77ed52bf:	59                   	pop    %ecx
77ed52c0:	85 c0                	test   %eax,%eax
77ed52c2:	0f 85 f6 fe ff ff    	jne    77ed51be <_OpenGLEnable+0x3e>
77ed52c8:	89 d0                	mov    %edx,%eax
77ed52ca:	c9                   	leave  
77ed52cb:	c3                   	ret    
77ed52cc:	8d 74 26 00          	lea    0x0(%esi),%esi

77ed52d0 <_ChoosePixelFormat@8>:
77ed52d0:	55                   	push   %ebp
77ed52d1:	89 e5                	mov    %esp,%ebp
77ed52d3:	51                   	push   %ecx
77ed52d4:	51                   	push   %ecx
77ed52d5:	a1 68 c0 ed 77       	mov    0x77edc068,%eax
77ed52da:	85 c0                	test   %eax,%eax
77ed52dc:	75 10                	jne    77ed52ee <_ChoosePixelFormat@8+0x1e>
77ed52de:	e8 9d fe ff ff       	call   77ed5180 <_OpenGLEnable>
77ed52e3:	31 d2                	xor    %edx,%edx
77ed52e5:	85 c0                	test   %eax,%eax
77ed52e7:	74 13                	je     77ed52fc <_ChoosePixelFormat@8+0x2c>
77ed52e9:	a1 68 c0 ed 77       	mov    0x77edc068,%eax
77ed52ee:	8b 4d 0c             	mov    0xc(%ebp),%ecx
77ed52f1:	52                   	push   %edx
77ed52f2:	52                   	push   %edx
77ed52f3:	8b 55 08             	mov    0x8(%ebp),%edx
77ed52f6:	51                   	push   %ecx
77ed52f7:	52                   	push   %edx
77ed52f8:	ff d0                	call   *%eax
77ed52fa:	89 c2                	mov    %eax,%edx
77ed52fc:	89 d0                	mov    %edx,%eax
77ed52fe:	c9                   	leave  
77ed52ff:	c2 08 00             	ret    $0x8
77ed5302:	8d b4 26 00 00 00 00 	lea    0x0(%esi),%esi
77ed5309:	8d bc 27 00 00 00 00 	lea    0x0(%edi),%edi

77ed5310 <_DescribePixelFormat@16>:
77ed5310:	55                   	push   %ebp
77ed5311:	89 e5                	mov    %esp,%ebp
77ed5313:	50                   	push   %eax
77ed5314:	50                   	push   %eax
77ed5315:	a1 48 c0 ed 77       	mov    0x77edc048,%eax
77ed531a:	85 c0                	test   %eax,%eax
77ed531c:	75 10                	jne    77ed532e <_DescribePixelFormat@16+0x1e>
77ed531e:	e8 5d fe ff ff       	call   77ed5180 <_OpenGLEnable>
77ed5323:	31 d2                	xor    %edx,%edx
77ed5325:	85 c0                	test   %eax,%eax
77ed5327:	74 19                	je     77ed5342 <_DescribePixelFormat@16+0x32>
77ed5329:	a1 48 c0 ed 77       	mov    0x77edc048,%eax
77ed532e:	8b 4d 14             	mov    0x14(%ebp),%ecx
77ed5331:	8b 55 10             	mov    0x10(%ebp),%edx
77ed5334:	51                   	push   %ecx
77ed5335:	8b 4d 0c             	mov    0xc(%ebp),%ecx
77ed5338:	52                   	push   %edx
77ed5339:	8b 55 08             	mov    0x8(%ebp),%edx
77ed533c:	51                   	push   %ecx
77ed533d:	52                   	push   %edx
77ed533e:	ff d0                	call   *%eax
77ed5340:	89 c2                	mov    %eax,%edx
77ed5342:	89 d0                	mov    %edx,%eax
77ed5344:	c9                   	leave  
77ed5345:	c2 10 00             	ret    $0x10
77ed5348:	90                   	nop    
77ed5349:	8d b4 26 00 00 00 00 	lea    0x0(%esi),%esi

77ed5350 <_GetPixelFormat@4>:
77ed5350:	55                   	push   %ebp
77ed5351:	89 e5                	mov    %esp,%ebp
77ed5353:	51                   	push   %ecx
77ed5354:	51                   	push   %ecx
77ed5355:	a1 38 c0 ed 77       	mov    0x77edc038,%eax
77ed535a:	85 c0                	test   %eax,%eax
77ed535c:	75 10                	jne    77ed536e <_GetPixelFormat@4+0x1e>
77ed535e:	e8 1d fe ff ff       	call   77ed5180 <_OpenGLEnable>
77ed5363:	31 d2                	xor    %edx,%edx
77ed5365:	85 c0                	test   %eax,%eax
77ed5367:	74 10                	je     77ed5379 <_GetPixelFormat@4+0x29>
77ed5369:	a1 38 c0 ed 77       	mov    0x77edc038,%eax
77ed536e:	83 ec 0c             	sub    $0xc,%esp
77ed5371:	8b 55 08             	mov    0x8(%ebp),%edx
77ed5374:	52                   	push   %edx
77ed5375:	ff d0                	call   *%eax
77ed5377:	89 c2                	mov    %eax,%edx
77ed5379:	89 d0                	mov    %edx,%eax
77ed537b:	c9                   	leave  
77ed537c:	c2 04 00             	ret    $0x4
77ed537f:	90                   	nop    

77ed5380 <_SetPixelFormat@12>:
77ed5380:	55                   	push   %ebp
77ed5381:	89 e5                	mov    %esp,%ebp
77ed5383:	50                   	push   %eax
77ed5384:	50                   	push   %eax
77ed5385:	a1 58 c0 ed 77       	mov    0x77edc058,%eax
77ed538a:	85 c0                	test   %eax,%eax
77ed538c:	75 10                	jne    77ed539e <_SetPixelFormat@12+0x1e>
77ed538e:	e8 ed fd ff ff       	call   77ed5180 <_OpenGLEnable>
77ed5393:	31 d2                	xor    %edx,%edx
77ed5395:	85 c0                	test   %eax,%eax
77ed5397:	74 16                	je     77ed53af <_SetPixelFormat@12+0x2f>
77ed5399:	a1 58 c0 ed 77       	mov    0x77edc058,%eax
77ed539e:	8b 55 10             	mov    0x10(%ebp),%edx
77ed53a1:	51                   	push   %ecx
77ed53a2:	8b 4d 0c             	mov    0xc(%ebp),%ecx
77ed53a5:	52                   	push   %edx
77ed53a6:	8b 55 08             	mov    0x8(%ebp),%edx
77ed53a9:	51                   	push   %ecx
77ed53aa:	52                   	push   %edx
77ed53ab:	ff d0                	call   *%eax
77ed53ad:	89 c2                	mov    %eax,%edx
77ed53af:	89 d0                	mov    %edx,%eax
77ed53b1:	c9                   	leave  
77ed53b2:	c2 0c 00             	ret    $0xc
77ed53b5:	8d 74 26 00          	lea    0x0(%esi),%esi
77ed53b9:	8d bc 27 00 00 00 00 	lea    0x0(%edi),%edi

77ed53c0 <_SwapBuffers@4>:
77ed53c0:	55                   	push   %ebp
77ed53c1:	89 e5                	mov    %esp,%ebp
77ed53c3:	51                   	push   %ecx
77ed53c4:	51                   	push   %ecx
77ed53c5:	a1 28 c0 ed 77       	mov    0x77edc028,%eax
77ed53ca:	85 c0                	test   %eax,%eax
77ed53cc:	75 10                	jne    77ed53de <_SwapBuffers@4+0x1e>
77ed53ce:	e8 ad fd ff ff       	call   77ed5180 <_OpenGLEnable>
77ed53d3:	31 d2                	xor    %edx,%edx
77ed53d5:	85 c0                	test   %eax,%eax
77ed53d7:	74 10                	je     77ed53e9 <_SwapBuffers@4+0x29>
77ed53d9:	a1 28 c0 ed 77       	mov    0x77edc028,%eax
77ed53de:	83 ec 0c             	sub    $0xc,%esp
77ed53e1:	8b 55 08             	mov    0x8(%ebp),%edx
77ed53e4:	52                   	push   %edx
77ed53e5:	ff d0                	call   *%eax
77ed53e7:	89 c2                	mov    %eax,%edx
77ed53e9:	89 d0                	mov    %edx,%eax
77ed53eb:	c9                   	leave  
77ed53ec:	c2 04 00             	ret    $0x4
77ed53ef:	90                   	nop    

77ed53f0 <_GetEnhMetaFilePixelFormat@12>:
77ed53f0:	55                   	push   %ebp
77ed53f1:	89 e5                	mov    %esp,%ebp
77ed53f3:	83 ec 7c             	sub    $0x7c,%esp
77ed53f6:	8d 45 88             	lea    0xffffff88(%ebp),%eax
77ed53f9:	50                   	push   %eax
77ed53fa:	6a 6c                	push   $0x6c
77ed53fc:	8b 4d 08             	mov    0x8(%ebp),%ecx
77ed53ff:	51                   	push   %ecx
77ed5400:	e8 cb c4 ff ff       	call   77ed18d0 <_GetEnhMetaFileHeader@12>
77ed5405:	5a                   	pop    %edx
77ed5406:	85 c0                	test   %eax,%eax
77ed5408:	74 0e                	je     77ed5418 <_GetEnhMetaFilePixelFormat@12+0x28>
77ed540a:	8b 45 e8             	mov    0xffffffe8(%ebp),%eax
77ed540d:	85 c0                	test   %eax,%eax
77ed540f:	74 07                	je     77ed5418 <_GetEnhMetaFilePixelFormat@12+0x28>
77ed5411:	8b 45 e0             	mov    0xffffffe0(%ebp),%eax
77ed5414:	85 c0                	test   %eax,%eax
77ed5416:	75 06                	jne    77ed541e <_GetEnhMetaFilePixelFormat@12+0x2e>
77ed5418:	31 c0                	xor    %eax,%eax
77ed541a:	c9                   	leave  
77ed541b:	c2 0c 00             	ret    $0xc
77ed541e:	50                   	push   %eax
77ed541f:	8b 45 0c             	mov    0xc(%ebp),%eax
77ed5422:	50                   	push   %eax
77ed5423:	8b 45 e4             	mov    0xffffffe4(%ebp),%eax
77ed5426:	50                   	push   %eax
77ed5427:	8b 45 10             	mov    0x10(%ebp),%eax
77ed542a:	50                   	push   %eax
77ed542b:	e8 10 44 00 00       	call   77ed9840 <_memcpy>
77ed5430:	8b 45 e0             	mov    0xffffffe0(%ebp),%eax
77ed5433:	c9                   	leave  
77ed5434:	c2 0c 00             	ret    $0xc
77ed5437:	90                   	nop    
77ed5438:	90                   	nop    
77ed5439:	90                   	nop    
77ed543a:	90                   	nop    
77ed543b:	90                   	nop    
77ed543c:	90                   	nop    
77ed543d:	90                   	nop    
77ed543e:	90                   	nop    
77ed543f:	90                   	nop    

77ed5440 <_NtGdiAbortDoc@4>:

.global _NtGdiAbortDoc@4
_NtGdiAbortDoc@4:

    movl $0x1000, %eax
77ed5440:	b8 00 10 00 00       	mov    $0x1000,%eax
    movl $KUSER_SHARED_SYSCALL, %ecx
77ed5445:	b9 00 03 fe 7f       	mov    $0x7ffe0300,%ecx
    call *%ecx
77ed544a:	ff d1                	call   *%ecx
    ret $0x4
77ed544c:	c2 04 00             	ret    $0x4

77ed544f <_NtGdiAbortPath@4>:

.global _NtGdiAbortPath@4
_NtGdiAbortPath@4:

    movl $0x1001, %eax
77ed544f:	b8 01 10 00 00       	mov    $0x1001,%eax
    movl $KUSER_SHARED_SYSCALL, %ecx
77ed5454:	b9 00 03 fe 7f       	mov    $0x7ffe0300,%ecx
    call *%ecx
77ed5459:	ff d1                	call   *%ecx
    ret $0x4
77ed545b:	c2 04 00             	ret    $0x4

77ed545e <_NtGdiAddFontResource@8>:

.global _NtGdiAddFontResource@8
_NtGdiAddFontResource@8:

    movl $0x1002, %eax
77ed545e:	b8 02 10 00 00       	mov    $0x1002,%eax
    movl $KUSER_SHARED_SYSCALL, %ecx
77ed5463:	b9 00 03 fe 7f       	mov    $0x7ffe0300,%ecx
    call *%ecx
77ed5468:	ff d1                	call   *%ecx
    ret $0x8
77ed546a:	c2 08 00             	ret    $0x8

77ed546d <_NtGdiAngleArc@24>:

.global _NtGdiAngleArc@24
_NtGdiAngleArc@24:

    movl $0x1003, %eax
77ed546d:	b8 03 10 00 00       	mov    $0x1003,%eax
    movl $KUSER_SHARED_SYSCALL, %ecx
77ed5472:	b9 00 03 fe 7f       	mov    $0x7ffe0300,%ecx
    call *%ecx
77ed5477:	ff d1                	call   *%ecx
    ret $0x18
77ed5479:	c2 18 00             	ret    $0x18

77ed547c <_NtGdiAnimatePalette@16>:

.global _NtGdiAnimatePalette@16
_NtGdiAnimatePalette@16:

    movl $0x1004, %eax
77ed547c:	b8 04 10 00 00       	mov    $0x1004,%eax
    movl $KUSER_SHARED_SYSCALL, %ecx
77ed5481:	b9 00 03 fe 7f       	mov    $0x7ffe0300,%ecx
    call *%ecx
77ed5486:	ff d1                	call   *%ecx
    ret $0x10
77ed5488:	c2 10 00             	ret    $0x10

77ed548b <_NtGdiArc@36>:

.global _NtGdiArc@36
_NtGdiArc@36:

    movl $0x1005, %eax
77ed548b:	b8 05 10 00 00       	mov    $0x1005,%eax
    movl $KUSER_SHARED_SYSCALL, %ecx
77ed5490:	b9 00 03 fe 7f       	mov    $0x7ffe0300,%ecx
    call *%ecx
77ed5495:	ff d1                	call   *%ecx
    ret $0x24
77ed5497:	c2 24 00             	ret    $0x24

77ed549a <_NtGdiArcTo@36>:

.global _NtGdiArcTo@36
_NtGdiArcTo@36:

    movl $0x1006, %eax
77ed549a:	b8 06 10 00 00       	mov    $0x1006,%eax
    movl $KUSER_SHARED_SYSCALL, %ecx
77ed549f:	b9 00 03 fe 7f       	mov    $0x7ffe0300,%ecx
    call *%ecx
77ed54a4:	ff d1                	call   *%ecx
    ret $0x24
77ed54a6:	c2 24 00             	ret    $0x24

77ed54a9 <_NtGdiBeginPath@4>:

.global _NtGdiBeginPath@4
_NtGdiBeginPath@4:

    movl $0x1007, %eax
77ed54a9:	b8 07 10 00 00       	mov    $0x1007,%eax
    movl $KUSER_SHARED_SYSCALL, %ecx
77ed54ae:	b9 00 03 fe 7f       	mov    $0x7ffe0300,%ecx
    call *%ecx
77ed54b3:	ff d1                	call   *%ecx
    ret $0x4
77ed54b5:	c2 04 00             	ret    $0x4

77ed54b8 <_NtGdiBitBlt@36>:

.global _NtGdiBitBlt@36
_NtGdiBitBlt@36:

    movl $0x1008, %eax
77ed54b8:	b8 08 10 00 00       	mov    $0x1008,%eax
    movl $KUSER_SHARED_SYSCALL, %ecx
77ed54bd:	b9 00 03 fe 7f       	mov    $0x7ffe0300,%ecx
    call *%ecx
77ed54c2:	ff d1                	call   *%ecx
    ret $0x24
77ed54c4:	c2 24 00             	ret    $0x24

77ed54c7 <_NtGdiCancelDC@4>:

.global _NtGdiCancelDC@4
_NtGdiCancelDC@4:

    movl $0x1009, %eax
77ed54c7:	b8 09 10 00 00       	mov    $0x1009,%eax
    movl $KUSER_SHARED_SYSCALL, %ecx
77ed54cc:	b9 00 03 fe 7f       	mov    $0x7ffe0300,%ecx
    call *%ecx
77ed54d1:	ff d1                	call   *%ecx
    ret $0x4
77ed54d3:	c2 04 00             	ret    $0x4

77ed54d6 <_NtGdiCheckColorsInGamut@16>:

.global _NtGdiCheckColorsInGamut@16
_NtGdiCheckColorsInGamut@16:

    movl $0x100a, %eax
77ed54d6:	b8 0a 10 00 00       	mov    $0x100a,%eax
    movl $KUSER_SHARED_SYSCALL, %ecx
77ed54db:	b9 00 03 fe 7f       	mov    $0x7ffe0300,%ecx
    call *%ecx
77ed54e0:	ff d1                	call   *%ecx
    ret $0x10
77ed54e2:	c2 10 00             	ret    $0x10

77ed54e5 <_NtGdiChord@36>:

.global _NtGdiChord@36
_NtGdiChord@36:

    movl $0x100b, %eax
77ed54e5:	b8 0b 10 00 00       	mov    $0x100b,%eax
    movl $KUSER_SHARED_SYSCALL, %ecx
77ed54ea:	b9 00 03 fe 7f       	mov    $0x7ffe0300,%ecx
    call *%ecx
77ed54ef:	ff d1                	call   *%ecx
    ret $0x24
77ed54f1:	c2 24 00             	ret    $0x24

77ed54f4 <_NtGdiCloseEnhMetaFile@4>:

.global _NtGdiCloseEnhMetaFile@4
_NtGdiCloseEnhMetaFile@4:

    movl $0x100c, %eax
77ed54f4:	b8 0c 10 00 00       	mov    $0x100c,%eax
    movl $KUSER_SHARED_SYSCALL, %ecx
77ed54f9:	b9 00 03 fe 7f       	mov    $0x7ffe0300,%ecx
    call *%ecx
77ed54fe:	ff d1                	call   *%ecx
    ret $0x4
77ed5500:	c2 04 00             	ret    $0x4

77ed5503 <_NtGdiCloseFigure@4>:

.global _NtGdiCloseFigure@4
_NtGdiCloseFigure@4:

    movl $0x100d, %eax
77ed5503:	b8 0d 10 00 00       	mov    $0x100d,%eax
    movl $KUSER_SHARED_SYSCALL, %ecx
77ed5508:	b9 00 03 fe 7f       	mov    $0x7ffe0300,%ecx
    call *%ecx
77ed550d:	ff d1                	call   *%ecx
    ret $0x4
77ed550f:	c2 04 00             	ret    $0x4

77ed5512 <_NtGdiCloseMetaFile@4>:

.global _NtGdiCloseMetaFile@4
_NtGdiCloseMetaFile@4:

    movl $0x100e, %eax
77ed5512:	b8 0e 10 00 00       	mov    $0x100e,%eax
    movl $KUSER_SHARED_SYSCALL, %ecx
77ed5517:	b9 00 03 fe 7f       	mov    $0x7ffe0300,%ecx
    call *%ecx
77ed551c:	ff d1                	call   *%ecx
    ret $0x4
77ed551e:	c2 04 00             	ret    $0x4

77ed5521 <_NtGdiColorMatchToTarget@12>:

.global _NtGdiColorMatchToTarget@12
_NtGdiColorMatchToTarget@12:

    movl $0x100f, %eax
77ed5521:	b8 0f 10 00 00       	mov    $0x100f,%eax
    movl $KUSER_SHARED_SYSCALL, %ecx
77ed5526:	b9 00 03 fe 7f       	mov    $0x7ffe0300,%ecx
    call *%ecx
77ed552b:	ff d1                	call   *%ecx
    ret $0xc
77ed552d:	c2 0c 00             	ret    $0xc

77ed5530 <_NtGdiCombineRgn@16>:

.global _NtGdiCombineRgn@16
_NtGdiCombineRgn@16:

    movl $0x1010, %eax
77ed5530:	b8 10 10 00 00       	mov    $0x1010,%eax
    movl $KUSER_SHARED_SYSCALL, %ecx
77ed5535:	b9 00 03 fe 7f       	mov    $0x7ffe0300,%ecx
    call *%ecx
77ed553a:	ff d1                	call   *%ecx
    ret $0x10
77ed553c:	c2 10 00             	ret    $0x10

77ed553f <_NtGdiCombineTransform@12>:

.global _NtGdiCombineTransform@12
_NtGdiCombineTransform@12:

    movl $0x1011, %eax
77ed553f:	b8 11 10 00 00       	mov    $0x1011,%eax
    movl $KUSER_SHARED_SYSCALL, %ecx
77ed5544:	b9 00 03 fe 7f       	mov    $0x7ffe0300,%ecx
    call *%ecx
77ed5549:	ff d1                	call   *%ecx
    ret $0xc
77ed554b:	c2 0c 00             	ret    $0xc

77ed554e <_NtGdiCopyEnhMetaFile@8>:

.global _NtGdiCopyEnhMetaFile@8
_NtGdiCopyEnhMetaFile@8:

    movl $0x1012, %eax
77ed554e:	b8 12 10 00 00       	mov    $0x1012,%eax
    movl $KUSER_SHARED_SYSCALL, %ecx
77ed5553:	b9 00 03 fe 7f       	mov    $0x7ffe0300,%ecx
    call *%ecx
77ed5558:	ff d1                	call   *%ecx
    ret $0x8
77ed555a:	c2 08 00             	ret    $0x8

77ed555d <_NtGdiCopyMetaFile@8>:

.global _NtGdiCopyMetaFile@8
_NtGdiCopyMetaFile@8:

    movl $0x1013, %eax
77ed555d:	b8 13 10 00 00       	mov    $0x1013,%eax
    movl $KUSER_SHARED_SYSCALL, %ecx
77ed5562:	b9 00 03 fe 7f       	mov    $0x7ffe0300,%ecx
    call *%ecx
77ed5567:	ff d1                	call   *%ecx
    ret $0x8
77ed5569:	c2 08 00             	ret    $0x8

77ed556c <_NtGdiCreateBitmap@20>:

.global _NtGdiCreateBitmap@20
_NtGdiCreateBitmap@20:

    movl $0x1014, %eax
77ed556c:	b8 14 10 00 00       	mov    $0x1014,%eax
    movl $KUSER_SHARED_SYSCALL, %ecx
77ed5571:	b9 00 03 fe 7f       	mov    $0x7ffe0300,%ecx
    call *%ecx
77ed5576:	ff d1                	call   *%ecx
    ret $0x14
77ed5578:	c2 14 00             	ret    $0x14

77ed557b <_NtGdiCreateBitmapIndirect@4>:

.global _NtGdiCreateBitmapIndirect@4
_NtGdiCreateBitmapIndirect@4:

    movl $0x1015, %eax
77ed557b:	b8 15 10 00 00       	mov    $0x1015,%eax
    movl $KUSER_SHARED_SYSCALL, %ecx
77ed5580:	b9 00 03 fe 7f       	mov    $0x7ffe0300,%ecx
    call *%ecx
77ed5585:	ff d1                	call   *%ecx
    ret $0x4
77ed5587:	c2 04 00             	ret    $0x4

77ed558a <_NtGdiCreateBrushIndirect@4>:

.global _NtGdiCreateBrushIndirect@4
_NtGdiCreateBrushIndirect@4:

    movl $0x1016, %eax
77ed558a:	b8 16 10 00 00       	mov    $0x1016,%eax
    movl $KUSER_SHARED_SYSCALL, %ecx
77ed558f:	b9 00 03 fe 7f       	mov    $0x7ffe0300,%ecx
    call *%ecx
77ed5594:	ff d1                	call   *%ecx
    ret $0x4
77ed5596:	c2 04 00             	ret    $0x4

77ed5599 <_NtGdiCreateColorSpace@4>:

.global _NtGdiCreateColorSpace@4
_NtGdiCreateColorSpace@4:

    movl $0x1017, %eax
77ed5599:	b8 17 10 00 00       	mov    $0x1017,%eax
    movl $KUSER_SHARED_SYSCALL, %ecx
77ed559e:	b9 00 03 fe 7f       	mov    $0x7ffe0300,%ecx
    call *%ecx
77ed55a3:	ff d1                	call   *%ecx
    ret $0x4
77ed55a5:	c2 04 00             	ret    $0x4

77ed55a8 <_NtGdiCreateCompatibleBitmap@12>:

.global _NtGdiCreateCompatibleBitmap@12
_NtGdiCreateCompatibleBitmap@12:

    movl $0x1018, %eax
77ed55a8:	b8 18 10 00 00       	mov    $0x1018,%eax
    movl $KUSER_SHARED_SYSCALL, %ecx
77ed55ad:	b9 00 03 fe 7f       	mov    $0x7ffe0300,%ecx
    call *%ecx
77ed55b2:	ff d1                	call   *%ecx
    ret $0xc
77ed55b4:	c2 0c 00             	ret    $0xc

77ed55b7 <_NtGdiCreateCompatableDC@4>:

.global _NtGdiCreateCompatableDC@4
_NtGdiCreateCompatableDC@4:

    movl $0x1019, %eax
77ed55b7:	b8 19 10 00 00       	mov    $0x1019,%eax
    movl $KUSER_SHARED_SYSCALL, %ecx
77ed55bc:	b9 00 03 fe 7f       	mov    $0x7ffe0300,%ecx
    call *%ecx
77ed55c1:	ff d1                	call   *%ecx
    ret $0x4
77ed55c3:	c2 04 00             	ret    $0x4

77ed55c6 <_NtGdiCreateDC@16>:

.global _NtGdiCreateDC@16
_NtGdiCreateDC@16:

    movl $0x101a, %eax
77ed55c6:	b8 1a 10 00 00       	mov    $0x101a,%eax
    movl $KUSER_SHARED_SYSCALL, %ecx
77ed55cb:	b9 00 03 fe 7f       	mov    $0x7ffe0300,%ecx
    call *%ecx
77ed55d0:	ff d1                	call   *%ecx
    ret $0x10
77ed55d2:	c2 10 00             	ret    $0x10

77ed55d5 <_NtGdiCreateDIBitmap@24>:

.global _NtGdiCreateDIBitmap@24
_NtGdiCreateDIBitmap@24:

    movl $0x101b, %eax
77ed55d5:	b8 1b 10 00 00       	mov    $0x101b,%eax
    movl $KUSER_SHARED_SYSCALL, %ecx
77ed55da:	b9 00 03 fe 7f       	mov    $0x7ffe0300,%ecx
    call *%ecx
77ed55df:	ff d1                	call   *%ecx
    ret $0x18
77ed55e1:	c2 18 00             	ret    $0x18

77ed55e4 <_NtGdiCreateDIBPatternBrush@8>:

.global _NtGdiCreateDIBPatternBrush@8
_NtGdiCreateDIBPatternBrush@8:

    movl $0x101c, %eax
77ed55e4:	b8 1c 10 00 00       	mov    $0x101c,%eax
    movl $KUSER_SHARED_SYSCALL, %ecx
77ed55e9:	b9 00 03 fe 7f       	mov    $0x7ffe0300,%ecx
    call *%ecx
77ed55ee:	ff d1                	call   *%ecx
    ret $0x8
77ed55f0:	c2 08 00             	ret    $0x8

77ed55f3 <_NtGdiCreateDIBPatternBrushPt@8>:

.global _NtGdiCreateDIBPatternBrushPt@8
_NtGdiCreateDIBPatternBrushPt@8:

    movl $0x101d, %eax
77ed55f3:	b8 1d 10 00 00       	mov    $0x101d,%eax
    movl $KUSER_SHARED_SYSCALL, %ecx
77ed55f8:	b9 00 03 fe 7f       	mov    $0x7ffe0300,%ecx
    call *%ecx
77ed55fd:	ff d1                	call   *%ecx
    ret $0x8
77ed55ff:	c2 08 00             	ret    $0x8

77ed5602 <_NtGdiCreateDIBSection@24>:

.global _NtGdiCreateDIBSection@24
_NtGdiCreateDIBSection@24:

    movl $0x101e, %eax
77ed5602:	b8 1e 10 00 00       	mov    $0x101e,%eax
    movl $KUSER_SHARED_SYSCALL, %ecx
77ed5607:	b9 00 03 fe 7f       	mov    $0x7ffe0300,%ecx
    call *%ecx
77ed560c:	ff d1                	call   *%ecx
    ret $0x18
77ed560e:	c2 18 00             	ret    $0x18

77ed5611 <_NtGdiCreateDiscardableBitmap@12>:

.global _NtGdiCreateDiscardableBitmap@12
_NtGdiCreateDiscardableBitmap@12:

    movl $0x101f, %eax
77ed5611:	b8 1f 10 00 00       	mov    $0x101f,%eax
    movl $KUSER_SHARED_SYSCALL, %ecx
77ed5616:	b9 00 03 fe 7f       	mov    $0x7ffe0300,%ecx
    call *%ecx
77ed561b:	ff d1                	call   *%ecx
    ret $0xc
77ed561d:	c2 0c 00             	ret    $0xc

77ed5620 <_NtGdiCreateEllipticRgn@16>:

.global _NtGdiCreateEllipticRgn@16
_NtGdiCreateEllipticRgn@16:

    movl $0x1020, %eax
77ed5620:	b8 20 10 00 00       	mov    $0x1020,%eax
    movl $KUSER_SHARED_SYSCALL, %ecx
77ed5625:	b9 00 03 fe 7f       	mov    $0x7ffe0300,%ecx
    call *%ecx
77ed562a:	ff d1                	call   *%ecx
    ret $0x10
77ed562c:	c2 10 00             	ret    $0x10

77ed562f <_NtGdiCreateEllipticRgnIndirect@4>:

.global _NtGdiCreateEllipticRgnIndirect@4
_NtGdiCreateEllipticRgnIndirect@4:

    movl $0x1021, %eax
77ed562f:	b8 21 10 00 00       	mov    $0x1021,%eax
    movl $KUSER_SHARED_SYSCALL, %ecx
77ed5634:	b9 00 03 fe 7f       	mov    $0x7ffe0300,%ecx
    call *%ecx
77ed5639:	ff d1                	call   *%ecx
    ret $0x4
77ed563b:	c2 04 00             	ret    $0x4

77ed563e <_NtGdiCreateEnhMetaFile@16>:

.global _NtGdiCreateEnhMetaFile@16
_NtGdiCreateEnhMetaFile@16:

    movl $0x1022, %eax
77ed563e:	b8 22 10 00 00       	mov    $0x1022,%eax
    movl $KUSER_SHARED_SYSCALL, %ecx
77ed5643:	b9 00 03 fe 7f       	mov    $0x7ffe0300,%ecx
    call *%ecx
77ed5648:	ff d1                	call   *%ecx
    ret $0x10
77ed564a:	c2 10 00             	ret    $0x10

77ed564d <_NtGdiCreateFont@56>:

.global _NtGdiCreateFont@56
_NtGdiCreateFont@56:

    movl $0x1023, %eax
77ed564d:	b8 23 10 00 00       	mov    $0x1023,%eax
    movl $KUSER_SHARED_SYSCALL, %ecx
77ed5652:	b9 00 03 fe 7f       	mov    $0x7ffe0300,%ecx
    call *%ecx
77ed5657:	ff d1                	call   *%ecx
    ret $0x38
77ed5659:	c2 38 00             	ret    $0x38

77ed565c <_NtGdiCreateFontIndirect@4>:

.global _NtGdiCreateFontIndirect@4
_NtGdiCreateFontIndirect@4:

    movl $0x1024, %eax
77ed565c:	b8 24 10 00 00       	mov    $0x1024,%eax
    movl $KUSER_SHARED_SYSCALL, %ecx
77ed5661:	b9 00 03 fe 7f       	mov    $0x7ffe0300,%ecx
    call *%ecx
77ed5666:	ff d1                	call   *%ecx
    ret $0x4
77ed5668:	c2 04 00             	ret    $0x4

77ed566b <_NtGdiCreateHalftonePalette@4>:

.global _NtGdiCreateHalftonePalette@4
_NtGdiCreateHalftonePalette@4:

    movl $0x1025, %eax
77ed566b:	b8 25 10 00 00       	mov    $0x1025,%eax
    movl $KUSER_SHARED_SYSCALL, %ecx
77ed5670:	b9 00 03 fe 7f       	mov    $0x7ffe0300,%ecx
    call *%ecx
77ed5675:	ff d1                	call   *%ecx
    ret $0x4
77ed5677:	c2 04 00             	ret    $0x4

77ed567a <_NtGdiCreateHatchBrush@8>:

.global _NtGdiCreateHatchBrush@8
_NtGdiCreateHatchBrush@8:

    movl $0x1026, %eax
77ed567a:	b8 26 10 00 00       	mov    $0x1026,%eax
    movl $KUSER_SHARED_SYSCALL, %ecx
77ed567f:	b9 00 03 fe 7f       	mov    $0x7ffe0300,%ecx
    call *%ecx
77ed5684:	ff d1                	call   *%ecx
    ret $0x8
77ed5686:	c2 08 00             	ret    $0x8

77ed5689 <_NtGdiCreateIC@16>:

.global _NtGdiCreateIC@16
_NtGdiCreateIC@16:

    movl $0x1027, %eax
77ed5689:	b8 27 10 00 00       	mov    $0x1027,%eax
    movl $KUSER_SHARED_SYSCALL, %ecx
77ed568e:	b9 00 03 fe 7f       	mov    $0x7ffe0300,%ecx
    call *%ecx
77ed5693:	ff d1                	call   *%ecx
    ret $0x10
77ed5695:	c2 10 00             	ret    $0x10

77ed5698 <_NtGdiCreateMetaFile@4>:

.global _NtGdiCreateMetaFile@4
_NtGdiCreateMetaFile@4:

    movl $0x1028, %eax
77ed5698:	b8 28 10 00 00       	mov    $0x1028,%eax
    movl $KUSER_SHARED_SYSCALL, %ecx
77ed569d:	b9 00 03 fe 7f       	mov    $0x7ffe0300,%ecx
    call *%ecx
77ed56a2:	ff d1                	call   *%ecx
    ret $0x4
77ed56a4:	c2 04 00             	ret    $0x4

77ed56a7 <_NtGdiCreatePalette@4>:

.global _NtGdiCreatePalette@4
_NtGdiCreatePalette@4:

    movl $0x1029, %eax
77ed56a7:	b8 29 10 00 00       	mov    $0x1029,%eax
    movl $KUSER_SHARED_SYSCALL, %ecx
77ed56ac:	b9 00 03 fe 7f       	mov    $0x7ffe0300,%ecx
    call *%ecx
77ed56b1:	ff d1                	call   *%ecx
    ret $0x4
77ed56b3:	c2 04 00             	ret    $0x4

77ed56b6 <_NtGdiCreatePatternBrush@4>:

.global _NtGdiCreatePatternBrush@4
_NtGdiCreatePatternBrush@4:

    movl $0x102a, %eax
77ed56b6:	b8 2a 10 00 00       	mov    $0x102a,%eax
    movl $KUSER_SHARED_SYSCALL, %ecx
77ed56bb:	b9 00 03 fe 7f       	mov    $0x7ffe0300,%ecx
    call *%ecx
77ed56c0:	ff d1                	call   *%ecx
    ret $0x4
77ed56c2:	c2 04 00             	ret    $0x4

77ed56c5 <_NtGdiCreatePen@12>:

.global _NtGdiCreatePen@12
_NtGdiCreatePen@12:

    movl $0x102b, %eax
77ed56c5:	b8 2b 10 00 00       	mov    $0x102b,%eax
    movl $KUSER_SHARED_SYSCALL, %ecx
77ed56ca:	b9 00 03 fe 7f       	mov    $0x7ffe0300,%ecx
    call *%ecx
77ed56cf:	ff d1                	call   *%ecx
    ret $0xc
77ed56d1:	c2 0c 00             	ret    $0xc

77ed56d4 <_NtGdiCreatePenIndirect@4>:

.global _NtGdiCreatePenIndirect@4
_NtGdiCreatePenIndirect@4:

    movl $0x102c, %eax
77ed56d4:	b8 2c 10 00 00       	mov    $0x102c,%eax
    movl $KUSER_SHARED_SYSCALL, %ecx
77ed56d9:	b9 00 03 fe 7f       	mov    $0x7ffe0300,%ecx
    call *%ecx
77ed56de:	ff d1                	call   *%ecx
    ret $0x4
77ed56e0:	c2 04 00             	ret    $0x4

77ed56e3 <_NtGdiCreatePolygonRgn@12>:

.global _NtGdiCreatePolygonRgn@12
_NtGdiCreatePolygonRgn@12:

    movl $0x102d, %eax
77ed56e3:	b8 2d 10 00 00       	mov    $0x102d,%eax
    movl $KUSER_SHARED_SYSCALL, %ecx
77ed56e8:	b9 00 03 fe 7f       	mov    $0x7ffe0300,%ecx
    call *%ecx
77ed56ed:	ff d1                	call   *%ecx
    ret $0xc
77ed56ef:	c2 0c 00             	ret    $0xc

77ed56f2 <_NtGdiCreatePolyPolygonRgn@16>:

.global _NtGdiCreatePolyPolygonRgn@16
_NtGdiCreatePolyPolygonRgn@16:

    movl $0x102e, %eax
77ed56f2:	b8 2e 10 00 00       	mov    $0x102e,%eax
    movl $KUSER_SHARED_SYSCALL, %ecx
77ed56f7:	b9 00 03 fe 7f       	mov    $0x7ffe0300,%ecx
    call *%ecx
77ed56fc:	ff d1                	call   *%ecx
    ret $0x10
77ed56fe:	c2 10 00             	ret    $0x10

77ed5701 <_NtGdiCreateRectRgn@16>:

.global _NtGdiCreateRectRgn@16
_NtGdiCreateRectRgn@16:

    movl $0x102f, %eax
77ed5701:	b8 2f 10 00 00       	mov    $0x102f,%eax
    movl $KUSER_SHARED_SYSCALL, %ecx
77ed5706:	b9 00 03 fe 7f       	mov    $0x7ffe0300,%ecx
    call *%ecx
77ed570b:	ff d1                	call   *%ecx
    ret $0x10
77ed570d:	c2 10 00             	ret    $0x10

77ed5710 <_NtGdiCreateRectRgnIndirect@4>:

.global _NtGdiCreateRectRgnIndirect@4
_NtGdiCreateRectRgnIndirect@4:

    movl $0x1030, %eax
77ed5710:	b8 30 10 00 00       	mov    $0x1030,%eax
    movl $KUSER_SHARED_SYSCALL, %ecx
77ed5715:	b9 00 03 fe 7f       	mov    $0x7ffe0300,%ecx
    call *%ecx
77ed571a:	ff d1                	call   *%ecx
    ret $0x4
77ed571c:	c2 04 00             	ret    $0x4

77ed571f <_NtGdiCreateRoundRectRgn@24>:

.global _NtGdiCreateRoundRectRgn@24
_NtGdiCreateRoundRectRgn@24:

    movl $0x1031, %eax
77ed571f:	b8 31 10 00 00       	mov    $0x1031,%eax
    movl $KUSER_SHARED_SYSCALL, %ecx
77ed5724:	b9 00 03 fe 7f       	mov    $0x7ffe0300,%ecx
    call *%ecx
77ed5729:	ff d1                	call   *%ecx
    ret $0x18
77ed572b:	c2 18 00             	ret    $0x18

77ed572e <_NtGdiCreateScalableFontResource@16>:

.global _NtGdiCreateScalableFontResource@16
_NtGdiCreateScalableFontResource@16:

    movl $0x1032, %eax
77ed572e:	b8 32 10 00 00       	mov    $0x1032,%eax
    movl $KUSER_SHARED_SYSCALL, %ecx
77ed5733:	b9 00 03 fe 7f       	mov    $0x7ffe0300,%ecx
    call *%ecx
77ed5738:	ff d1                	call   *%ecx
    ret $0x10
77ed573a:	c2 10 00             	ret    $0x10

77ed573d <_NtGdiCreateSolidBrush@4>:

.global _NtGdiCreateSolidBrush@4
_NtGdiCreateSolidBrush@4:

    movl $0x1033, %eax
77ed573d:	b8 33 10 00 00       	mov    $0x1033,%eax
    movl $KUSER_SHARED_SYSCALL, %ecx
77ed5742:	b9 00 03 fe 7f       	mov    $0x7ffe0300,%ecx
    call *%ecx
77ed5747:	ff d1                	call   *%ecx
    ret $0x4
77ed5749:	c2 04 00             	ret    $0x4

77ed574c <_NtGdiDPtoLP@12>:

.global _NtGdiDPtoLP@12
_NtGdiDPtoLP@12:

    movl $0x1034, %eax
77ed574c:	b8 34 10 00 00       	mov    $0x1034,%eax
    movl $KUSER_SHARED_SYSCALL, %ecx
77ed5751:	b9 00 03 fe 7f       	mov    $0x7ffe0300,%ecx
    call *%ecx
77ed5756:	ff d1                	call   *%ecx
    ret $0xc
77ed5758:	c2 0c 00             	ret    $0xc

77ed575b <_NtGdiDeleteColorSpace@4>:

.global _NtGdiDeleteColorSpace@4
_NtGdiDeleteColorSpace@4:

    movl $0x1035, %eax
77ed575b:	b8 35 10 00 00       	mov    $0x1035,%eax
    movl $KUSER_SHARED_SYSCALL, %ecx
77ed5760:	b9 00 03 fe 7f       	mov    $0x7ffe0300,%ecx
    call *%ecx
77ed5765:	ff d1                	call   *%ecx
    ret $0x4
77ed5767:	c2 04 00             	ret    $0x4

77ed576a <_NtGdiDeleteDC@4>:

.global _NtGdiDeleteDC@4
_NtGdiDeleteDC@4:

    movl $0x1036, %eax
77ed576a:	b8 36 10 00 00       	mov    $0x1036,%eax
    movl $KUSER_SHARED_SYSCALL, %ecx
77ed576f:	b9 00 03 fe 7f       	mov    $0x7ffe0300,%ecx
    call *%ecx
77ed5774:	ff d1                	call   *%ecx
    ret $0x4
77ed5776:	c2 04 00             	ret    $0x4

77ed5779 <_NtGdiDeleteEnhMetaFile@4>:

.global _NtGdiDeleteEnhMetaFile@4
_NtGdiDeleteEnhMetaFile@4:

    movl $0x1037, %eax
77ed5779:	b8 37 10 00 00       	mov    $0x1037,%eax
    movl $KUSER_SHARED_SYSCALL, %ecx
77ed577e:	b9 00 03 fe 7f       	mov    $0x7ffe0300,%ecx
    call *%ecx
77ed5783:	ff d1                	call   *%ecx
    ret $0x4
77ed5785:	c2 04 00             	ret    $0x4

77ed5788 <_NtGdiDeleteMetaFile@4>:

.global _NtGdiDeleteMetaFile@4
_NtGdiDeleteMetaFile@4:

    movl $0x1038, %eax
77ed5788:	b8 38 10 00 00       	mov    $0x1038,%eax
    movl $KUSER_SHARED_SYSCALL, %ecx
77ed578d:	b9 00 03 fe 7f       	mov    $0x7ffe0300,%ecx
    call *%ecx
77ed5792:	ff d1                	call   *%ecx
    ret $0x4
77ed5794:	c2 04 00             	ret    $0x4

77ed5797 <_NtGdiDeleteObject@4>:

.global _NtGdiDeleteObject@4
_NtGdiDeleteObject@4:

    movl $0x1039, %eax
77ed5797:	b8 39 10 00 00       	mov    $0x1039,%eax
    movl $KUSER_SHARED_SYSCALL, %ecx
77ed579c:	b9 00 03 fe 7f       	mov    $0x7ffe0300,%ecx
    call *%ecx
77ed57a1:	ff d1                	call   *%ecx
    ret $0x4
77ed57a3:	c2 04 00             	ret    $0x4

77ed57a6 <_NtGdiDescribePixelFormat@16>:

.global _NtGdiDescribePixelFormat@16
_NtGdiDescribePixelFormat@16:

    movl $0x103a, %eax
77ed57a6:	b8 3a 10 00 00       	mov    $0x103a,%eax
    movl $KUSER_SHARED_SYSCALL, %ecx
77ed57ab:	b9 00 03 fe 7f       	mov    $0x7ffe0300,%ecx
    call *%ecx
77ed57b0:	ff d1                	call   *%ecx
    ret $0x10
77ed57b2:	c2 10 00             	ret    $0x10

77ed57b5 <_NtGdiDrawEscape@16>:

.global _NtGdiDrawEscape@16
_NtGdiDrawEscape@16:

    movl $0x103b, %eax
77ed57b5:	b8 3b 10 00 00       	mov    $0x103b,%eax
    movl $KUSER_SHARED_SYSCALL, %ecx
77ed57ba:	b9 00 03 fe 7f       	mov    $0x7ffe0300,%ecx
    call *%ecx
77ed57bf:	ff d1                	call   *%ecx
    ret $0x10
77ed57c1:	c2 10 00             	ret    $0x10

77ed57c4 <_NtGdiEllipse@20>:

.global _NtGdiEllipse@20
_NtGdiEllipse@20:

    movl $0x103c, %eax
77ed57c4:	b8 3c 10 00 00       	mov    $0x103c,%eax
    movl $KUSER_SHARED_SYSCALL, %ecx
77ed57c9:	b9 00 03 fe 7f       	mov    $0x7ffe0300,%ecx
    call *%ecx
77ed57ce:	ff d1                	call   *%ecx
    ret $0x14
77ed57d0:	c2 14 00             	ret    $0x14

77ed57d3 <_NtGdiEndDoc@4>:

.global _NtGdiEndDoc@4
_NtGdiEndDoc@4:

    movl $0x103d, %eax
77ed57d3:	b8 3d 10 00 00       	mov    $0x103d,%eax
    movl $KUSER_SHARED_SYSCALL, %ecx
77ed57d8:	b9 00 03 fe 7f       	mov    $0x7ffe0300,%ecx
    call *%ecx
77ed57dd:	ff d1                	call   *%ecx
    ret $0x4
77ed57df:	c2 04 00             	ret    $0x4

77ed57e2 <_NtGdiEndPage@4>:

.global _NtGdiEndPage@4
_NtGdiEndPage@4:

    movl $0x103e, %eax
77ed57e2:	b8 3e 10 00 00       	mov    $0x103e,%eax
    movl $KUSER_SHARED_SYSCALL, %ecx
77ed57e7:	b9 00 03 fe 7f       	mov    $0x7ffe0300,%ecx
    call *%ecx
77ed57ec:	ff d1                	call   *%ecx
    ret $0x4
77ed57ee:	c2 04 00             	ret    $0x4

77ed57f1 <_NtGdiEndPath@4>:

.global _NtGdiEndPath@4
_NtGdiEndPath@4:

    movl $0x103f, %eax
77ed57f1:	b8 3f 10 00 00       	mov    $0x103f,%eax
    movl $KUSER_SHARED_SYSCALL, %ecx
77ed57f6:	b9 00 03 fe 7f       	mov    $0x7ffe0300,%ecx
    call *%ecx
77ed57fb:	ff d1                	call   *%ecx
    ret $0x4
77ed57fd:	c2 04 00             	ret    $0x4

77ed5800 <_NtGdiEnumEnhMetaFile@20>:

.global _NtGdiEnumEnhMetaFile@20
_NtGdiEnumEnhMetaFile@20:

    movl $0x1040, %eax
77ed5800:	b8 40 10 00 00       	mov    $0x1040,%eax
    movl $KUSER_SHARED_SYSCALL, %ecx
77ed5805:	b9 00 03 fe 7f       	mov    $0x7ffe0300,%ecx
    call *%ecx
77ed580a:	ff d1                	call   *%ecx
    ret $0x14
77ed580c:	c2 14 00             	ret    $0x14

77ed580f <_NtGdiEnumFonts@16>:

.global _NtGdiEnumFonts@16
_NtGdiEnumFonts@16:

    movl $0x1041, %eax
77ed580f:	b8 41 10 00 00       	mov    $0x1041,%eax
    movl $KUSER_SHARED_SYSCALL, %ecx
77ed5814:	b9 00 03 fe 7f       	mov    $0x7ffe0300,%ecx
    call *%ecx
77ed5819:	ff d1                	call   *%ecx
    ret $0x10
77ed581b:	c2 10 00             	ret    $0x10

77ed581e <_NtGdiEnumICMProfiles@12>:

.global _NtGdiEnumICMProfiles@12
_NtGdiEnumICMProfiles@12:

    movl $0x1042, %eax
77ed581e:	b8 42 10 00 00       	mov    $0x1042,%eax
    movl $KUSER_SHARED_SYSCALL, %ecx
77ed5823:	b9 00 03 fe 7f       	mov    $0x7ffe0300,%ecx
    call *%ecx
77ed5828:	ff d1                	call   *%ecx
    ret $0xc
77ed582a:	c2 0c 00             	ret    $0xc

77ed582d <_NtGdiEnumMetaFile@16>:

.global _NtGdiEnumMetaFile@16
_NtGdiEnumMetaFile@16:

    movl $0x1043, %eax
77ed582d:	b8 43 10 00 00       	mov    $0x1043,%eax
    movl $KUSER_SHARED_SYSCALL, %ecx
77ed5832:	b9 00 03 fe 7f       	mov    $0x7ffe0300,%ecx
    call *%ecx
77ed5837:	ff d1                	call   *%ecx
    ret $0x10
77ed5839:	c2 10 00             	ret    $0x10

77ed583c <_NtGdiEnumObjects@16>:

.global _NtGdiEnumObjects@16
_NtGdiEnumObjects@16:

    movl $0x1044, %eax
77ed583c:	b8 44 10 00 00       	mov    $0x1044,%eax
    movl $KUSER_SHARED_SYSCALL, %ecx
77ed5841:	b9 00 03 fe 7f       	mov    $0x7ffe0300,%ecx
    call *%ecx
77ed5846:	ff d1                	call   *%ecx
    ret $0x10
77ed5848:	c2 10 00             	ret    $0x10

77ed584b <_NtGdiEqualRgn@8>:

.global _NtGdiEqualRgn@8
_NtGdiEqualRgn@8:

    movl $0x1045, %eax
77ed584b:	b8 45 10 00 00       	mov    $0x1045,%eax
    movl $KUSER_SHARED_SYSCALL, %ecx
77ed5850:	b9 00 03 fe 7f       	mov    $0x7ffe0300,%ecx
    call *%ecx
77ed5855:	ff d1                	call   *%ecx
    ret $0x8
77ed5857:	c2 08 00             	ret    $0x8

77ed585a <_NtGdiEscape@20>:

.global _NtGdiEscape@20
_NtGdiEscape@20:

    movl $0x1046, %eax
77ed585a:	b8 46 10 00 00       	mov    $0x1046,%eax
    movl $KUSER_SHARED_SYSCALL, %ecx
77ed585f:	b9 00 03 fe 7f       	mov    $0x7ffe0300,%ecx
    call *%ecx
77ed5864:	ff d1                	call   *%ecx
    ret $0x14
77ed5866:	c2 14 00             	ret    $0x14

77ed5869 <_NtGdiExcludeClipRect@20>:

.global _NtGdiExcludeClipRect@20
_NtGdiExcludeClipRect@20:

    movl $0x1047, %eax
77ed5869:	b8 47 10 00 00       	mov    $0x1047,%eax
    movl $KUSER_SHARED_SYSCALL, %ecx
77ed586e:	b9 00 03 fe 7f       	mov    $0x7ffe0300,%ecx
    call *%ecx
77ed5873:	ff d1                	call   *%ecx
    ret $0x14
77ed5875:	c2 14 00             	ret    $0x14

77ed5878 <_NtGdiExtCreatePen@20>:

.global _NtGdiExtCreatePen@20
_NtGdiExtCreatePen@20:

    movl $0x1048, %eax
77ed5878:	b8 48 10 00 00       	mov    $0x1048,%eax
    movl $KUSER_SHARED_SYSCALL, %ecx
77ed587d:	b9 00 03 fe 7f       	mov    $0x7ffe0300,%ecx
    call *%ecx
77ed5882:	ff d1                	call   *%ecx
    ret $0x14
77ed5884:	c2 14 00             	ret    $0x14

77ed5887 <_NtGdiExtCreateRegion@12>:

.global _NtGdiExtCreateRegion@12
_NtGdiExtCreateRegion@12:

    movl $0x1049, %eax
77ed5887:	b8 49 10 00 00       	mov    $0x1049,%eax
    movl $KUSER_SHARED_SYSCALL, %ecx
77ed588c:	b9 00 03 fe 7f       	mov    $0x7ffe0300,%ecx
    call *%ecx
77ed5891:	ff d1                	call   *%ecx
    ret $0xc
77ed5893:	c2 0c 00             	ret    $0xc

77ed5896 <_NtGdiExtEscape@24>:

.global _NtGdiExtEscape@24
_NtGdiExtEscape@24:

    movl $0x104a, %eax
77ed5896:	b8 4a 10 00 00       	mov    $0x104a,%eax
    movl $KUSER_SHARED_SYSCALL, %ecx
77ed589b:	b9 00 03 fe 7f       	mov    $0x7ffe0300,%ecx
    call *%ecx
77ed58a0:	ff d1                	call   *%ecx
    ret $0x18
77ed58a2:	c2 18 00             	ret    $0x18

77ed58a5 <_NtGdiExtFloodFill@20>:

.global _NtGdiExtFloodFill@20
_NtGdiExtFloodFill@20:

    movl $0x104b, %eax
77ed58a5:	b8 4b 10 00 00       	mov    $0x104b,%eax
    movl $KUSER_SHARED_SYSCALL, %ecx
77ed58aa:	b9 00 03 fe 7f       	mov    $0x7ffe0300,%ecx
    call *%ecx
77ed58af:	ff d1                	call   *%ecx
    ret $0x14
77ed58b1:	c2 14 00             	ret    $0x14

77ed58b4 <_NtGdiExtSelectClipRgn@12>:

.global _NtGdiExtSelectClipRgn@12
_NtGdiExtSelectClipRgn@12:

    movl $0x104c, %eax
77ed58b4:	b8 4c 10 00 00       	mov    $0x104c,%eax
    movl $KUSER_SHARED_SYSCALL, %ecx
77ed58b9:	b9 00 03 fe 7f       	mov    $0x7ffe0300,%ecx
    call *%ecx
77ed58be:	ff d1                	call   *%ecx
    ret $0xc
77ed58c0:	c2 0c 00             	ret    $0xc

77ed58c3 <_NtGdiExtTextOut@32>:

.global _NtGdiExtTextOut@32
_NtGdiExtTextOut@32:

    movl $0x104d, %eax
77ed58c3:	b8 4d 10 00 00       	mov    $0x104d,%eax
    movl $KUSER_SHARED_SYSCALL, %ecx
77ed58c8:	b9 00 03 fe 7f       	mov    $0x7ffe0300,%ecx
    call *%ecx
77ed58cd:	ff d1                	call   *%ecx
    ret $0x20
77ed58cf:	c2 20 00             	ret    $0x20

77ed58d2 <_NtGdiFillPath@4>:

.global _NtGdiFillPath@4
_NtGdiFillPath@4:

    movl $0x104e, %eax
77ed58d2:	b8 4e 10 00 00       	mov    $0x104e,%eax
    movl $KUSER_SHARED_SYSCALL, %ecx
77ed58d7:	b9 00 03 fe 7f       	mov    $0x7ffe0300,%ecx
    call *%ecx
77ed58dc:	ff d1                	call   *%ecx
    ret $0x4
77ed58de:	c2 04 00             	ret    $0x4

77ed58e1 <_NtGdiFillRgn@12>:

.global _NtGdiFillRgn@12
_NtGdiFillRgn@12:

    movl $0x104f, %eax
77ed58e1:	b8 4f 10 00 00       	mov    $0x104f,%eax
    movl $KUSER_SHARED_SYSCALL, %ecx
77ed58e6:	b9 00 03 fe 7f       	mov    $0x7ffe0300,%ecx
    call *%ecx
77ed58eb:	ff d1                	call   *%ecx
    ret $0xc
77ed58ed:	c2 0c 00             	ret    $0xc

77ed58f0 <_NtGdiFixBrushOrgEx@0>:

.global _NtGdiFixBrushOrgEx@0
_NtGdiFixBrushOrgEx@0:

    movl $0x1050, %eax
77ed58f0:	b8 50 10 00 00       	mov    $0x1050,%eax
    movl $KUSER_SHARED_SYSCALL, %ecx
77ed58f5:	b9 00 03 fe 7f       	mov    $0x7ffe0300,%ecx
    call *%ecx
77ed58fa:	ff d1                	call   *%ecx
    ret $0x0
77ed58fc:	c2 00 00             	ret    $0x0

77ed58ff <_NtGdiFlattenPath@4>:

.global _NtGdiFlattenPath@4
_NtGdiFlattenPath@4:

    movl $0x1051, %eax
77ed58ff:	b8 51 10 00 00       	mov    $0x1051,%eax
    movl $KUSER_SHARED_SYSCALL, %ecx
77ed5904:	b9 00 03 fe 7f       	mov    $0x7ffe0300,%ecx
    call *%ecx
77ed5909:	ff d1                	call   *%ecx
    ret $0x4
77ed590b:	c2 04 00             	ret    $0x4

77ed590e <_NtGdiFloodFill@16>:

.global _NtGdiFloodFill@16
_NtGdiFloodFill@16:

    movl $0x1052, %eax
77ed590e:	b8 52 10 00 00       	mov    $0x1052,%eax
    movl $KUSER_SHARED_SYSCALL, %ecx
77ed5913:	b9 00 03 fe 7f       	mov    $0x7ffe0300,%ecx
    call *%ecx
77ed5918:	ff d1                	call   *%ecx
    ret $0x10
77ed591a:	c2 10 00             	ret    $0x10

77ed591d <_NtGdiFrameRgn@20>:

.global _NtGdiFrameRgn@20
_NtGdiFrameRgn@20:

    movl $0x1053, %eax
77ed591d:	b8 53 10 00 00       	mov    $0x1053,%eax
    movl $KUSER_SHARED_SYSCALL, %ecx
77ed5922:	b9 00 03 fe 7f       	mov    $0x7ffe0300,%ecx
    call *%ecx
77ed5927:	ff d1                	call   *%ecx
    ret $0x14
77ed5929:	c2 14 00             	ret    $0x14

77ed592c <_NtGdiGdiComment@12>:

.global _NtGdiGdiComment@12
_NtGdiGdiComment@12:

    movl $0x1054, %eax
77ed592c:	b8 54 10 00 00       	mov    $0x1054,%eax
    movl $KUSER_SHARED_SYSCALL, %ecx
77ed5931:	b9 00 03 fe 7f       	mov    $0x7ffe0300,%ecx
    call *%ecx
77ed5936:	ff d1                	call   *%ecx
    ret $0xc
77ed5938:	c2 0c 00             	ret    $0xc

77ed593b <_NtGdiGdiFlush@0>:

.global _NtGdiGdiFlush@0
_NtGdiGdiFlush@0:

    movl $0x1055, %eax
77ed593b:	b8 55 10 00 00       	mov    $0x1055,%eax
    movl $KUSER_SHARED_SYSCALL, %ecx
77ed5940:	b9 00 03 fe 7f       	mov    $0x7ffe0300,%ecx
    call *%ecx
77ed5945:	ff d1                	call   *%ecx
    ret $0x0
77ed5947:	c2 00 00             	ret    $0x0

77ed594a <_NtGdiGdiGetBatchLimit@0>:

.global _NtGdiGdiGetBatchLimit@0
_NtGdiGdiGetBatchLimit@0:

    movl $0x1056, %eax
77ed594a:	b8 56 10 00 00       	mov    $0x1056,%eax
    movl $KUSER_SHARED_SYSCALL, %ecx
77ed594f:	b9 00 03 fe 7f       	mov    $0x7ffe0300,%ecx
    call *%ecx
77ed5954:	ff d1                	call   *%ecx
    ret $0x0
77ed5956:	c2 00 00             	ret    $0x0

77ed5959 <_NtGdiGdiSetBatchLimit@4>:

.global _NtGdiGdiSetBatchLimit@4
_NtGdiGdiSetBatchLimit@4:

    movl $0x1057, %eax
77ed5959:	b8 57 10 00 00       	mov    $0x1057,%eax
    movl $KUSER_SHARED_SYSCALL, %ecx
77ed595e:	b9 00 03 fe 7f       	mov    $0x7ffe0300,%ecx
    call *%ecx
77ed5963:	ff d1                	call   *%ecx
    ret $0x4
77ed5965:	c2 04 00             	ret    $0x4

77ed5968 <_NtGdiGetArcDirection@4>:

.global _NtGdiGetArcDirection@4
_NtGdiGetArcDirection@4:

    movl $0x1058, %eax
77ed5968:	b8 58 10 00 00       	mov    $0x1058,%eax
    movl $KUSER_SHARED_SYSCALL, %ecx
77ed596d:	b9 00 03 fe 7f       	mov    $0x7ffe0300,%ecx
    call *%ecx
77ed5972:	ff d1                	call   *%ecx
    ret $0x4
77ed5974:	c2 04 00             	ret    $0x4

77ed5977 <_NtGdiGetAspectRatioFilterEx@8>:

.global _NtGdiGetAspectRatioFilterEx@8
_NtGdiGetAspectRatioFilterEx@8:

    movl $0x1059, %eax
77ed5977:	b8 59 10 00 00       	mov    $0x1059,%eax
    movl $KUSER_SHARED_SYSCALL, %ecx
77ed597c:	b9 00 03 fe 7f       	mov    $0x7ffe0300,%ecx
    call *%ecx
77ed5981:	ff d1                	call   *%ecx
    ret $0x8
77ed5983:	c2 08 00             	ret    $0x8

77ed5986 <_NtGdiGetBitmapBits@12>:

.global _NtGdiGetBitmapBits@12
_NtGdiGetBitmapBits@12:

    movl $0x105a, %eax
77ed5986:	b8 5a 10 00 00       	mov    $0x105a,%eax
    movl $KUSER_SHARED_SYSCALL, %ecx
77ed598b:	b9 00 03 fe 7f       	mov    $0x7ffe0300,%ecx
    call *%ecx
77ed5990:	ff d1                	call   *%ecx
    ret $0xc
77ed5992:	c2 0c 00             	ret    $0xc

77ed5995 <_NtGdiGetBitmapDimensionEx@8>:

.global _NtGdiGetBitmapDimensionEx@8
_NtGdiGetBitmapDimensionEx@8:

    movl $0x105b, %eax
77ed5995:	b8 5b 10 00 00       	mov    $0x105b,%eax
    movl $KUSER_SHARED_SYSCALL, %ecx
77ed599a:	b9 00 03 fe 7f       	mov    $0x7ffe0300,%ecx
    call *%ecx
77ed599f:	ff d1                	call   *%ecx
    ret $0x8
77ed59a1:	c2 08 00             	ret    $0x8

77ed59a4 <_NtGdiGetBkColor@4>:

.global _NtGdiGetBkColor@4
_NtGdiGetBkColor@4:

    movl $0x105c, %eax
77ed59a4:	b8 5c 10 00 00       	mov    $0x105c,%eax
    movl $KUSER_SHARED_SYSCALL, %ecx
77ed59a9:	b9 00 03 fe 7f       	mov    $0x7ffe0300,%ecx
    call *%ecx
77ed59ae:	ff d1                	call   *%ecx
    ret $0x4
77ed59b0:	c2 04 00             	ret    $0x4

77ed59b3 <_NtGdiGetBkMode@4>:

.global _NtGdiGetBkMode@4
_NtGdiGetBkMode@4:

    movl $0x105d, %eax
77ed59b3:	b8 5d 10 00 00       	mov    $0x105d,%eax
    movl $KUSER_SHARED_SYSCALL, %ecx
77ed59b8:	b9 00 03 fe 7f       	mov    $0x7ffe0300,%ecx
    call *%ecx
77ed59bd:	ff d1                	call   *%ecx
    ret $0x4
77ed59bf:	c2 04 00             	ret    $0x4

77ed59c2 <_NtGdiGetBoundsRect@12>:

.global _NtGdiGetBoundsRect@12
_NtGdiGetBoundsRect@12:

    movl $0x105e, %eax
77ed59c2:	b8 5e 10 00 00       	mov    $0x105e,%eax
    movl $KUSER_SHARED_SYSCALL, %ecx
77ed59c7:	b9 00 03 fe 7f       	mov    $0x7ffe0300,%ecx
    call *%ecx
77ed59cc:	ff d1                	call   *%ecx
    ret $0xc
77ed59ce:	c2 0c 00             	ret    $0xc

77ed59d1 <_NtGdiGetBrushOrgEx@8>:

.global _NtGdiGetBrushOrgEx@8
_NtGdiGetBrushOrgEx@8:

    movl $0x105f, %eax
77ed59d1:	b8 5f 10 00 00       	mov    $0x105f,%eax
    movl $KUSER_SHARED_SYSCALL, %ecx
77ed59d6:	b9 00 03 fe 7f       	mov    $0x7ffe0300,%ecx
    call *%ecx
77ed59db:	ff d1                	call   *%ecx
    ret $0x8
77ed59dd:	c2 08 00             	ret    $0x8

77ed59e0 <_NtGdiGetCharABCWidths@16>:

.global _NtGdiGetCharABCWidths@16
_NtGdiGetCharABCWidths@16:

    movl $0x1060, %eax
77ed59e0:	b8 60 10 00 00       	mov    $0x1060,%eax
    movl $KUSER_SHARED_SYSCALL, %ecx
77ed59e5:	b9 00 03 fe 7f       	mov    $0x7ffe0300,%ecx
    call *%ecx
77ed59ea:	ff d1                	call   *%ecx
    ret $0x10
77ed59ec:	c2 10 00             	ret    $0x10

77ed59ef <_NtGdiGetCharABCWidthsFloat@16>:

.global _NtGdiGetCharABCWidthsFloat@16
_NtGdiGetCharABCWidthsFloat@16:

    movl $0x1061, %eax
77ed59ef:	b8 61 10 00 00       	mov    $0x1061,%eax
    movl $KUSER_SHARED_SYSCALL, %ecx
77ed59f4:	b9 00 03 fe 7f       	mov    $0x7ffe0300,%ecx
    call *%ecx
77ed59f9:	ff d1                	call   *%ecx
    ret $0x10
77ed59fb:	c2 10 00             	ret    $0x10

77ed59fe <_NtGdiGetCharacterPlacement@24>:

.global _NtGdiGetCharacterPlacement@24
_NtGdiGetCharacterPlacement@24:

    movl $0x1062, %eax
77ed59fe:	b8 62 10 00 00       	mov    $0x1062,%eax
    movl $KUSER_SHARED_SYSCALL, %ecx
77ed5a03:	b9 00 03 fe 7f       	mov    $0x7ffe0300,%ecx
    call *%ecx
77ed5a08:	ff d1                	call   *%ecx
    ret $0x18
77ed5a0a:	c2 18 00             	ret    $0x18

77ed5a0d <_NtGdiGetCharWidth32@16>:

.global _NtGdiGetCharWidth32@16
_NtGdiGetCharWidth32@16:

    movl $0x1063, %eax
77ed5a0d:	b8 63 10 00 00       	mov    $0x1063,%eax
    movl $KUSER_SHARED_SYSCALL, %ecx
77ed5a12:	b9 00 03 fe 7f       	mov    $0x7ffe0300,%ecx
    call *%ecx
77ed5a17:	ff d1                	call   *%ecx
    ret $0x10
77ed5a19:	c2 10 00             	ret    $0x10

77ed5a1c <_NtGdiGetCharWidthFloat@16>:

.global _NtGdiGetCharWidthFloat@16
_NtGdiGetCharWidthFloat@16:

    movl $0x1064, %eax
77ed5a1c:	b8 64 10 00 00       	mov    $0x1064,%eax
    movl $KUSER_SHARED_SYSCALL, %ecx
77ed5a21:	b9 00 03 fe 7f       	mov    $0x7ffe0300,%ecx
    call *%ecx
77ed5a26:	ff d1                	call   *%ecx
    ret $0x10
77ed5a28:	c2 10 00             	ret    $0x10

77ed5a2b <_NtGdiGetClipBox@8>:

.global _NtGdiGetClipBox@8
_NtGdiGetClipBox@8:

    movl $0x1065, %eax
77ed5a2b:	b8 65 10 00 00       	mov    $0x1065,%eax
    movl $KUSER_SHARED_SYSCALL, %ecx
77ed5a30:	b9 00 03 fe 7f       	mov    $0x7ffe0300,%ecx
    call *%ecx
77ed5a35:	ff d1                	call   *%ecx
    ret $0x8
77ed5a37:	c2 08 00             	ret    $0x8

77ed5a3a <_NtGdiGetClipRgn@4>:

.global _NtGdiGetClipRgn@4
_NtGdiGetClipRgn@4:

    movl $0x1066, %eax
77ed5a3a:	b8 66 10 00 00       	mov    $0x1066,%eax
    movl $KUSER_SHARED_SYSCALL, %ecx
77ed5a3f:	b9 00 03 fe 7f       	mov    $0x7ffe0300,%ecx
    call *%ecx
77ed5a44:	ff d1                	call   *%ecx
    ret $0x4
77ed5a46:	c2 04 00             	ret    $0x4

77ed5a49 <_NtGdiGetColorAdjustment@8>:

.global _NtGdiGetColorAdjustment@8
_NtGdiGetColorAdjustment@8:

    movl $0x1067, %eax
77ed5a49:	b8 67 10 00 00       	mov    $0x1067,%eax
    movl $KUSER_SHARED_SYSCALL, %ecx
77ed5a4e:	b9 00 03 fe 7f       	mov    $0x7ffe0300,%ecx
    call *%ecx
77ed5a53:	ff d1                	call   *%ecx
    ret $0x8
77ed5a55:	c2 08 00             	ret    $0x8

77ed5a58 <_NtGdiGetColorSpace@4>:

.global _NtGdiGetColorSpace@4
_NtGdiGetColorSpace@4:

    movl $0x1068, %eax
77ed5a58:	b8 68 10 00 00       	mov    $0x1068,%eax
    movl $KUSER_SHARED_SYSCALL, %ecx
77ed5a5d:	b9 00 03 fe 7f       	mov    $0x7ffe0300,%ecx
    call *%ecx
77ed5a62:	ff d1                	call   *%ecx
    ret $0x4
77ed5a64:	c2 04 00             	ret    $0x4

77ed5a67 <_NtGdiGetCurrentObject@8>:

.global _NtGdiGetCurrentObject@8
_NtGdiGetCurrentObject@8:

    movl $0x1069, %eax
77ed5a67:	b8 69 10 00 00       	mov    $0x1069,%eax
    movl $KUSER_SHARED_SYSCALL, %ecx
77ed5a6c:	b9 00 03 fe 7f       	mov    $0x7ffe0300,%ecx
    call *%ecx
77ed5a71:	ff d1                	call   *%ecx
    ret $0x8
77ed5a73:	c2 08 00             	ret    $0x8

77ed5a76 <_NtGdiGetCurrentPositionEx@8>:

.global _NtGdiGetCurrentPositionEx@8
_NtGdiGetCurrentPositionEx@8:

    movl $0x106a, %eax
77ed5a76:	b8 6a 10 00 00       	mov    $0x106a,%eax
    movl $KUSER_SHARED_SYSCALL, %ecx
77ed5a7b:	b9 00 03 fe 7f       	mov    $0x7ffe0300,%ecx
    call *%ecx
77ed5a80:	ff d1                	call   *%ecx
    ret $0x8
77ed5a82:	c2 08 00             	ret    $0x8

77ed5a85 <_NtGdiGetDCOrgEx@8>:

.global _NtGdiGetDCOrgEx@8
_NtGdiGetDCOrgEx@8:

    movl $0x106b, %eax
77ed5a85:	b8 6b 10 00 00       	mov    $0x106b,%eax
    movl $KUSER_SHARED_SYSCALL, %ecx
77ed5a8a:	b9 00 03 fe 7f       	mov    $0x7ffe0300,%ecx
    call *%ecx
77ed5a8f:	ff d1                	call   *%ecx
    ret $0x8
77ed5a91:	c2 08 00             	ret    $0x8

77ed5a94 <_NtGdiGetDIBColorTable@16>:

.global _NtGdiGetDIBColorTable@16
_NtGdiGetDIBColorTable@16:

    movl $0x106c, %eax
77ed5a94:	b8 6c 10 00 00       	mov    $0x106c,%eax
    movl $KUSER_SHARED_SYSCALL, %ecx
77ed5a99:	b9 00 03 fe 7f       	mov    $0x7ffe0300,%ecx
    call *%ecx
77ed5a9e:	ff d1                	call   *%ecx
    ret $0x10
77ed5aa0:	c2 10 00             	ret    $0x10

77ed5aa3 <_NtGdiGetDIBits@28>:

.global _NtGdiGetDIBits@28
_NtGdiGetDIBits@28:

    movl $0x106d, %eax
77ed5aa3:	b8 6d 10 00 00       	mov    $0x106d,%eax
    movl $KUSER_SHARED_SYSCALL, %ecx
77ed5aa8:	b9 00 03 fe 7f       	mov    $0x7ffe0300,%ecx
    call *%ecx
77ed5aad:	ff d1                	call   *%ecx
    ret $0x1c
77ed5aaf:	c2 1c 00             	ret    $0x1c

77ed5ab2 <_NtGdiGetDeviceCaps@8>:

.global _NtGdiGetDeviceCaps@8
_NtGdiGetDeviceCaps@8:

    movl $0x106e, %eax
77ed5ab2:	b8 6e 10 00 00       	mov    $0x106e,%eax
    movl $KUSER_SHARED_SYSCALL, %ecx
77ed5ab7:	b9 00 03 fe 7f       	mov    $0x7ffe0300,%ecx
    call *%ecx
77ed5abc:	ff d1                	call   *%ecx
    ret $0x8
77ed5abe:	c2 08 00             	ret    $0x8

77ed5ac1 <_NtGdiGetDeviceGammaRamp@8>:

.global _NtGdiGetDeviceGammaRamp@8
_NtGdiGetDeviceGammaRamp@8:

    movl $0x106f, %eax
77ed5ac1:	b8 6f 10 00 00       	mov    $0x106f,%eax
    movl $KUSER_SHARED_SYSCALL, %ecx
77ed5ac6:	b9 00 03 fe 7f       	mov    $0x7ffe0300,%ecx
    call *%ecx
77ed5acb:	ff d1                	call   *%ecx
    ret $0x8
77ed5acd:	c2 08 00             	ret    $0x8

77ed5ad0 <_NtGdiGetEnhMetaFile@4>:

.global _NtGdiGetEnhMetaFile@4
_NtGdiGetEnhMetaFile@4:

    movl $0x1070, %eax
77ed5ad0:	b8 70 10 00 00       	mov    $0x1070,%eax
    movl $KUSER_SHARED_SYSCALL, %ecx
77ed5ad5:	b9 00 03 fe 7f       	mov    $0x7ffe0300,%ecx
    call *%ecx
77ed5ada:	ff d1                	call   *%ecx
    ret $0x4
77ed5adc:	c2 04 00             	ret    $0x4

77ed5adf <_NtGdiGetEnhMetaFileBits@12>:

.global _NtGdiGetEnhMetaFileBits@12
_NtGdiGetEnhMetaFileBits@12:

    movl $0x1071, %eax
77ed5adf:	b8 71 10 00 00       	mov    $0x1071,%eax
    movl $KUSER_SHARED_SYSCALL, %ecx
77ed5ae4:	b9 00 03 fe 7f       	mov    $0x7ffe0300,%ecx
    call *%ecx
77ed5ae9:	ff d1                	call   *%ecx
    ret $0xc
77ed5aeb:	c2 0c 00             	ret    $0xc

77ed5aee <_NtGdiGetEnhMetaFileDescription@12>:

.global _NtGdiGetEnhMetaFileDescription@12
_NtGdiGetEnhMetaFileDescription@12:

    movl $0x1072, %eax
77ed5aee:	b8 72 10 00 00       	mov    $0x1072,%eax
    movl $KUSER_SHARED_SYSCALL, %ecx
77ed5af3:	b9 00 03 fe 7f       	mov    $0x7ffe0300,%ecx
    call *%ecx
77ed5af8:	ff d1                	call   *%ecx
    ret $0xc
77ed5afa:	c2 0c 00             	ret    $0xc

77ed5afd <_NtGdiGetEnhMetaFileHeader@12>:

.global _NtGdiGetEnhMetaFileHeader@12
_NtGdiGetEnhMetaFileHeader@12:

    movl $0x1073, %eax
77ed5afd:	b8 73 10 00 00       	mov    $0x1073,%eax
    movl $KUSER_SHARED_SYSCALL, %ecx
77ed5b02:	b9 00 03 fe 7f       	mov    $0x7ffe0300,%ecx
    call *%ecx
77ed5b07:	ff d1                	call   *%ecx
    ret $0xc
77ed5b09:	c2 0c 00             	ret    $0xc

77ed5b0c <_NtGdiGetEnhMetaFilePaletteEntries@12>:

.global _NtGdiGetEnhMetaFilePaletteEntries@12
_NtGdiGetEnhMetaFilePaletteEntries@12:

    movl $0x1074, %eax
77ed5b0c:	b8 74 10 00 00       	mov    $0x1074,%eax
    movl $KUSER_SHARED_SYSCALL, %ecx
77ed5b11:	b9 00 03 fe 7f       	mov    $0x7ffe0300,%ecx
    call *%ecx
77ed5b16:	ff d1                	call   *%ecx
    ret $0xc
77ed5b18:	c2 0c 00             	ret    $0xc

77ed5b1b <_NtGdiGetEnhMetaFilePixelFormat@12>:

.global _NtGdiGetEnhMetaFilePixelFormat@12
_NtGdiGetEnhMetaFilePixelFormat@12:

    movl $0x1075, %eax
77ed5b1b:	b8 75 10 00 00       	mov    $0x1075,%eax
    movl $KUSER_SHARED_SYSCALL, %ecx
77ed5b20:	b9 00 03 fe 7f       	mov    $0x7ffe0300,%ecx
    call *%ecx
77ed5b25:	ff d1                	call   *%ecx
    ret $0xc
77ed5b27:	c2 0c 00             	ret    $0xc

77ed5b2a <_NtGdiGetFontData@20>:

.global _NtGdiGetFontData@20
_NtGdiGetFontData@20:

    movl $0x1076, %eax
77ed5b2a:	b8 76 10 00 00       	mov    $0x1076,%eax
    movl $KUSER_SHARED_SYSCALL, %ecx
77ed5b2f:	b9 00 03 fe 7f       	mov    $0x7ffe0300,%ecx
    call *%ecx
77ed5b34:	ff d1                	call   *%ecx
    ret $0x14
77ed5b36:	c2 14 00             	ret    $0x14

77ed5b39 <_NtGdiGetFontFamilyInfo@16>:

.global _NtGdiGetFontFamilyInfo@16
_NtGdiGetFontFamilyInfo@16:

    movl $0x1077, %eax
77ed5b39:	b8 77 10 00 00       	mov    $0x1077,%eax
    movl $KUSER_SHARED_SYSCALL, %ecx
77ed5b3e:	b9 00 03 fe 7f       	mov    $0x7ffe0300,%ecx
    call *%ecx
77ed5b43:	ff d1                	call   *%ecx
    ret $0x10
77ed5b45:	c2 10 00             	ret    $0x10

77ed5b48 <_NtGdiGetFontLanguageInfo@4>:

.global _NtGdiGetFontLanguageInfo@4
_NtGdiGetFontLanguageInfo@4:

    movl $0x1078, %eax
77ed5b48:	b8 78 10 00 00       	mov    $0x1078,%eax
    movl $KUSER_SHARED_SYSCALL, %ecx
77ed5b4d:	b9 00 03 fe 7f       	mov    $0x7ffe0300,%ecx
    call *%ecx
77ed5b52:	ff d1                	call   *%ecx
    ret $0x4
77ed5b54:	c2 04 00             	ret    $0x4

77ed5b57 <_NtGdiGetGlyphOutline@28>:

.global _NtGdiGetGlyphOutline@28
_NtGdiGetGlyphOutline@28:

    movl $0x1079, %eax
77ed5b57:	b8 79 10 00 00       	mov    $0x1079,%eax
    movl $KUSER_SHARED_SYSCALL, %ecx
77ed5b5c:	b9 00 03 fe 7f       	mov    $0x7ffe0300,%ecx
    call *%ecx
77ed5b61:	ff d1                	call   *%ecx
    ret $0x1c
77ed5b63:	c2 1c 00             	ret    $0x1c

77ed5b66 <_NtGdiGetGraphicsMode@4>:

.global _NtGdiGetGraphicsMode@4
_NtGdiGetGraphicsMode@4:

    movl $0x107a, %eax
77ed5b66:	b8 7a 10 00 00       	mov    $0x107a,%eax
    movl $KUSER_SHARED_SYSCALL, %ecx
77ed5b6b:	b9 00 03 fe 7f       	mov    $0x7ffe0300,%ecx
    call *%ecx
77ed5b70:	ff d1                	call   *%ecx
    ret $0x4
77ed5b72:	c2 04 00             	ret    $0x4

77ed5b75 <_NtGdiGetICMProfile@12>:

.global _NtGdiGetICMProfile@12
_NtGdiGetICMProfile@12:

    movl $0x107b, %eax
77ed5b75:	b8 7b 10 00 00       	mov    $0x107b,%eax
    movl $KUSER_SHARED_SYSCALL, %ecx
77ed5b7a:	b9 00 03 fe 7f       	mov    $0x7ffe0300,%ecx
    call *%ecx
77ed5b7f:	ff d1                	call   *%ecx
    ret $0xc
77ed5b81:	c2 0c 00             	ret    $0xc

77ed5b84 <_NtGdiGetKerningPairs@12>:

.global _NtGdiGetKerningPairs@12
_NtGdiGetKerningPairs@12:

    movl $0x107c, %eax
77ed5b84:	b8 7c 10 00 00       	mov    $0x107c,%eax
    movl $KUSER_SHARED_SYSCALL, %ecx
77ed5b89:	b9 00 03 fe 7f       	mov    $0x7ffe0300,%ecx
    call *%ecx
77ed5b8e:	ff d1                	call   *%ecx
    ret $0xc
77ed5b90:	c2 0c 00             	ret    $0xc

77ed5b93 <_NtGdiGetLogColorSpace@12>:

.global _NtGdiGetLogColorSpace@12
_NtGdiGetLogColorSpace@12:

    movl $0x107d, %eax
77ed5b93:	b8 7d 10 00 00       	mov    $0x107d,%eax
    movl $KUSER_SHARED_SYSCALL, %ecx
77ed5b98:	b9 00 03 fe 7f       	mov    $0x7ffe0300,%ecx
    call *%ecx
77ed5b9d:	ff d1                	call   *%ecx
    ret $0xc
77ed5b9f:	c2 0c 00             	ret    $0xc

77ed5ba2 <_NtGdiGetMapMode@4>:

.global _NtGdiGetMapMode@4
_NtGdiGetMapMode@4:

    movl $0x107e, %eax
77ed5ba2:	b8 7e 10 00 00       	mov    $0x107e,%eax
    movl $KUSER_SHARED_SYSCALL, %ecx
77ed5ba7:	b9 00 03 fe 7f       	mov    $0x7ffe0300,%ecx
    call *%ecx
77ed5bac:	ff d1                	call   *%ecx
    ret $0x4
77ed5bae:	c2 04 00             	ret    $0x4

77ed5bb1 <_NtGdiGetMetaFile@4>:

.global _NtGdiGetMetaFile@4
_NtGdiGetMetaFile@4:

    movl $0x107f, %eax
77ed5bb1:	b8 7f 10 00 00       	mov    $0x107f,%eax
    movl $KUSER_SHARED_SYSCALL, %ecx
77ed5bb6:	b9 00 03 fe 7f       	mov    $0x7ffe0300,%ecx
    call *%ecx
77ed5bbb:	ff d1                	call   *%ecx
    ret $0x4
77ed5bbd:	c2 04 00             	ret    $0x4

77ed5bc0 <_NtGdiGetMetaFileBitsEx@12>:

.global _NtGdiGetMetaFileBitsEx@12
_NtGdiGetMetaFileBitsEx@12:

    movl $0x1080, %eax
77ed5bc0:	b8 80 10 00 00       	mov    $0x1080,%eax
    movl $KUSER_SHARED_SYSCALL, %ecx
77ed5bc5:	b9 00 03 fe 7f       	mov    $0x7ffe0300,%ecx
    call *%ecx
77ed5bca:	ff d1                	call   *%ecx
    ret $0xc
77ed5bcc:	c2 0c 00             	ret    $0xc

77ed5bcf <_NtGdiGetMetaRgn@8>:

.global _NtGdiGetMetaRgn@8
_NtGdiGetMetaRgn@8:

    movl $0x1081, %eax
77ed5bcf:	b8 81 10 00 00       	mov    $0x1081,%eax
    movl $KUSER_SHARED_SYSCALL, %ecx
77ed5bd4:	b9 00 03 fe 7f       	mov    $0x7ffe0300,%ecx
    call *%ecx
77ed5bd9:	ff d1                	call   *%ecx
    ret $0x8
77ed5bdb:	c2 08 00             	ret    $0x8

77ed5bde <_NtGdiGetMiterLimit@8>:

.global _NtGdiGetMiterLimit@8
_NtGdiGetMiterLimit@8:

    movl $0x1082, %eax
77ed5bde:	b8 82 10 00 00       	mov    $0x1082,%eax
    movl $KUSER_SHARED_SYSCALL, %ecx
77ed5be3:	b9 00 03 fe 7f       	mov    $0x7ffe0300,%ecx
    call *%ecx
77ed5be8:	ff d1                	call   *%ecx
    ret $0x8
77ed5bea:	c2 08 00             	ret    $0x8

77ed5bed <_NtGdiGetNearestColor@8>:

.global _NtGdiGetNearestColor@8
_NtGdiGetNearestColor@8:

    movl $0x1083, %eax
77ed5bed:	b8 83 10 00 00       	mov    $0x1083,%eax
    movl $KUSER_SHARED_SYSCALL, %ecx
77ed5bf2:	b9 00 03 fe 7f       	mov    $0x7ffe0300,%ecx
    call *%ecx
77ed5bf7:	ff d1                	call   *%ecx
    ret $0x8
77ed5bf9:	c2 08 00             	ret    $0x8

77ed5bfc <_NtGdiGetNearestPaletteIndex@8>:

.global _NtGdiGetNearestPaletteIndex@8
_NtGdiGetNearestPaletteIndex@8:

    movl $0x1084, %eax
77ed5bfc:	b8 84 10 00 00       	mov    $0x1084,%eax
    movl $KUSER_SHARED_SYSCALL, %ecx
77ed5c01:	b9 00 03 fe 7f       	mov    $0x7ffe0300,%ecx
    call *%ecx
77ed5c06:	ff d1                	call   *%ecx
    ret $0x8
77ed5c08:	c2 08 00             	ret    $0x8

77ed5c0b <_NtGdiGetObject@12>:

.global _NtGdiGetObject@12
_NtGdiGetObject@12:

    movl $0x1085, %eax
77ed5c0b:	b8 85 10 00 00       	mov    $0x1085,%eax
    movl $KUSER_SHARED_SYSCALL, %ecx
77ed5c10:	b9 00 03 fe 7f       	mov    $0x7ffe0300,%ecx
    call *%ecx
77ed5c15:	ff d1                	call   *%ecx
    ret $0xc
77ed5c17:	c2 0c 00             	ret    $0xc

77ed5c1a <_NtGdiGetObjectType@4>:

.global _NtGdiGetObjectType@4
_NtGdiGetObjectType@4:

    movl $0x1086, %eax
77ed5c1a:	b8 86 10 00 00       	mov    $0x1086,%eax
    movl $KUSER_SHARED_SYSCALL, %ecx
77ed5c1f:	b9 00 03 fe 7f       	mov    $0x7ffe0300,%ecx
    call *%ecx
77ed5c24:	ff d1                	call   *%ecx
    ret $0x4
77ed5c26:	c2 04 00             	ret    $0x4

77ed5c29 <_NtGdiGetOutlineTextMetrics@12>:

.global _NtGdiGetOutlineTextMetrics@12
_NtGdiGetOutlineTextMetrics@12:

    movl $0x1087, %eax
77ed5c29:	b8 87 10 00 00       	mov    $0x1087,%eax
    movl $KUSER_SHARED_SYSCALL, %ecx
77ed5c2e:	b9 00 03 fe 7f       	mov    $0x7ffe0300,%ecx
    call *%ecx
77ed5c33:	ff d1                	call   *%ecx
    ret $0xc
77ed5c35:	c2 0c 00             	ret    $0xc

77ed5c38 <_NtGdiGetPaletteEntries@16>:

.global _NtGdiGetPaletteEntries@16
_NtGdiGetPaletteEntries@16:

    movl $0x1088, %eax
77ed5c38:	b8 88 10 00 00       	mov    $0x1088,%eax
    movl $KUSER_SHARED_SYSCALL, %ecx
77ed5c3d:	b9 00 03 fe 7f       	mov    $0x7ffe0300,%ecx
    call *%ecx
77ed5c42:	ff d1                	call   *%ecx
    ret $0x10
77ed5c44:	c2 10 00             	ret    $0x10

77ed5c47 <_NtGdiGetPath@16>:

.global _NtGdiGetPath@16
_NtGdiGetPath@16:

    movl $0x1089, %eax
77ed5c47:	b8 89 10 00 00       	mov    $0x1089,%eax
    movl $KUSER_SHARED_SYSCALL, %ecx
77ed5c4c:	b9 00 03 fe 7f       	mov    $0x7ffe0300,%ecx
    call *%ecx
77ed5c51:	ff d1                	call   *%ecx
    ret $0x10
77ed5c53:	c2 10 00             	ret    $0x10

77ed5c56 <_NtGdiGetPixel@12>:

.global _NtGdiGetPixel@12
_NtGdiGetPixel@12:

    movl $0x108a, %eax
77ed5c56:	b8 8a 10 00 00       	mov    $0x108a,%eax
    movl $KUSER_SHARED_SYSCALL, %ecx
77ed5c5b:	b9 00 03 fe 7f       	mov    $0x7ffe0300,%ecx
    call *%ecx
77ed5c60:	ff d1                	call   *%ecx
    ret $0xc
77ed5c62:	c2 0c 00             	ret    $0xc

77ed5c65 <_NtGdiGetPixelFormat@4>:

.global _NtGdiGetPixelFormat@4
_NtGdiGetPixelFormat@4:

    movl $0x108b, %eax
77ed5c65:	b8 8b 10 00 00       	mov    $0x108b,%eax
    movl $KUSER_SHARED_SYSCALL, %ecx
77ed5c6a:	b9 00 03 fe 7f       	mov    $0x7ffe0300,%ecx
    call *%ecx
77ed5c6f:	ff d1                	call   *%ecx
    ret $0x4
77ed5c71:	c2 04 00             	ret    $0x4

77ed5c74 <_NtGdiGetPolyFillMode@4>:

.global _NtGdiGetPolyFillMode@4
_NtGdiGetPolyFillMode@4:

    movl $0x108c, %eax
77ed5c74:	b8 8c 10 00 00       	mov    $0x108c,%eax
    movl $KUSER_SHARED_SYSCALL, %ecx
77ed5c79:	b9 00 03 fe 7f       	mov    $0x7ffe0300,%ecx
    call *%ecx
77ed5c7e:	ff d1                	call   *%ecx
    ret $0x4
77ed5c80:	c2 04 00             	ret    $0x4

77ed5c83 <_NtGdiGetROP2@4>:

.global _NtGdiGetROP2@4
_NtGdiGetROP2@4:

    movl $0x108d, %eax
77ed5c83:	b8 8d 10 00 00       	mov    $0x108d,%eax
    movl $KUSER_SHARED_SYSCALL, %ecx
77ed5c88:	b9 00 03 fe 7f       	mov    $0x7ffe0300,%ecx
    call *%ecx
77ed5c8d:	ff d1                	call   *%ecx
    ret $0x4
77ed5c8f:	c2 04 00             	ret    $0x4

77ed5c92 <_NtGdiGetRasterizerCaps@8>:

.global _NtGdiGetRasterizerCaps@8
_NtGdiGetRasterizerCaps@8:

    movl $0x108e, %eax
77ed5c92:	b8 8e 10 00 00       	mov    $0x108e,%eax
    movl $KUSER_SHARED_SYSCALL, %ecx
77ed5c97:	b9 00 03 fe 7f       	mov    $0x7ffe0300,%ecx
    call *%ecx
77ed5c9c:	ff d1                	call   *%ecx
    ret $0x8
77ed5c9e:	c2 08 00             	ret    $0x8

77ed5ca1 <_NtGdiGetRelAbs@4>:

.global _NtGdiGetRelAbs@4
_NtGdiGetRelAbs@4:

    movl $0x108f, %eax
77ed5ca1:	b8 8f 10 00 00       	mov    $0x108f,%eax
    movl $KUSER_SHARED_SYSCALL, %ecx
77ed5ca6:	b9 00 03 fe 7f       	mov    $0x7ffe0300,%ecx
    call *%ecx
77ed5cab:	ff d1                	call   *%ecx
    ret $0x4
77ed5cad:	c2 04 00             	ret    $0x4

77ed5cb0 <_NtGdiGetRegionData@12>:

.global _NtGdiGetRegionData@12
_NtGdiGetRegionData@12:

    movl $0x1090, %eax
77ed5cb0:	b8 90 10 00 00       	mov    $0x1090,%eax
    movl $KUSER_SHARED_SYSCALL, %ecx
77ed5cb5:	b9 00 03 fe 7f       	mov    $0x7ffe0300,%ecx
    call *%ecx
77ed5cba:	ff d1                	call   *%ecx
    ret $0xc
77ed5cbc:	c2 0c 00             	ret    $0xc

77ed5cbf <_NtGdiGetRgnBox@8>:

.global _NtGdiGetRgnBox@8
_NtGdiGetRgnBox@8:

    movl $0x1091, %eax
77ed5cbf:	b8 91 10 00 00       	mov    $0x1091,%eax
    movl $KUSER_SHARED_SYSCALL, %ecx
77ed5cc4:	b9 00 03 fe 7f       	mov    $0x7ffe0300,%ecx
    call *%ecx
77ed5cc9:	ff d1                	call   *%ecx
    ret $0x8
77ed5ccb:	c2 08 00             	ret    $0x8

77ed5cce <_NtGdiGetStockObject@4>:

.global _NtGdiGetStockObject@4
_NtGdiGetStockObject@4:

    movl $0x1092, %eax
77ed5cce:	b8 92 10 00 00       	mov    $0x1092,%eax
    movl $KUSER_SHARED_SYSCALL, %ecx
77ed5cd3:	b9 00 03 fe 7f       	mov    $0x7ffe0300,%ecx
    call *%ecx
77ed5cd8:	ff d1                	call   *%ecx
    ret $0x4
77ed5cda:	c2 04 00             	ret    $0x4

77ed5cdd <_NtGdiGetStretchBltMode@4>:

.global _NtGdiGetStretchBltMode@4
_NtGdiGetStretchBltMode@4:

    movl $0x1093, %eax
77ed5cdd:	b8 93 10 00 00       	mov    $0x1093,%eax
    movl $KUSER_SHARED_SYSCALL, %ecx
77ed5ce2:	b9 00 03 fe 7f       	mov    $0x7ffe0300,%ecx
    call *%ecx
77ed5ce7:	ff d1                	call   *%ecx
    ret $0x4
77ed5ce9:	c2 04 00             	ret    $0x4

77ed5cec <_NtGdiGetSystemPaletteEntries@16>:

.global _NtGdiGetSystemPaletteEntries@16
_NtGdiGetSystemPaletteEntries@16:

    movl $0x1094, %eax
77ed5cec:	b8 94 10 00 00       	mov    $0x1094,%eax
    movl $KUSER_SHARED_SYSCALL, %ecx
77ed5cf1:	b9 00 03 fe 7f       	mov    $0x7ffe0300,%ecx
    call *%ecx
77ed5cf6:	ff d1                	call   *%ecx
    ret $0x10
77ed5cf8:	c2 10 00             	ret    $0x10

77ed5cfb <_NtGdiGetSystemPaletteUse@4>:

.global _NtGdiGetSystemPaletteUse@4
_NtGdiGetSystemPaletteUse@4:

    movl $0x1095, %eax
77ed5cfb:	b8 95 10 00 00       	mov    $0x1095,%eax
    movl $KUSER_SHARED_SYSCALL, %ecx
77ed5d00:	b9 00 03 fe 7f       	mov    $0x7ffe0300,%ecx
    call *%ecx
77ed5d05:	ff d1                	call   *%ecx
    ret $0x4
77ed5d07:	c2 04 00             	ret    $0x4

77ed5d0a <_NtGdiGetTextAlign@4>:

.global _NtGdiGetTextAlign@4
_NtGdiGetTextAlign@4:

    movl $0x1096, %eax
77ed5d0a:	b8 96 10 00 00       	mov    $0x1096,%eax
    movl $KUSER_SHARED_SYSCALL, %ecx
77ed5d0f:	b9 00 03 fe 7f       	mov    $0x7ffe0300,%ecx
    call *%ecx
77ed5d14:	ff d1                	call   *%ecx
    ret $0x4
77ed5d16:	c2 04 00             	ret    $0x4

77ed5d19 <_NtGdiGetTextCharset@4>:

.global _NtGdiGetTextCharset@4
_NtGdiGetTextCharset@4:

    movl $0x1097, %eax
77ed5d19:	b8 97 10 00 00       	mov    $0x1097,%eax
    movl $KUSER_SHARED_SYSCALL, %ecx
77ed5d1e:	b9 00 03 fe 7f       	mov    $0x7ffe0300,%ecx
    call *%ecx
77ed5d23:	ff d1                	call   *%ecx
    ret $0x4
77ed5d25:	c2 04 00             	ret    $0x4

77ed5d28 <_NtGdiGetTextCharsetInfo@12>:

.global _NtGdiGetTextCharsetInfo@12
_NtGdiGetTextCharsetInfo@12:

    movl $0x1098, %eax
77ed5d28:	b8 98 10 00 00       	mov    $0x1098,%eax
    movl $KUSER_SHARED_SYSCALL, %ecx
77ed5d2d:	b9 00 03 fe 7f       	mov    $0x7ffe0300,%ecx
    call *%ecx
77ed5d32:	ff d1                	call   *%ecx
    ret $0xc
77ed5d34:	c2 0c 00             	ret    $0xc

77ed5d37 <_NtGdiGetTextColor@4>:

.global _NtGdiGetTextColor@4
_NtGdiGetTextColor@4:

    movl $0x1099, %eax
77ed5d37:	b8 99 10 00 00       	mov    $0x1099,%eax
    movl $KUSER_SHARED_SYSCALL, %ecx
77ed5d3c:	b9 00 03 fe 7f       	mov    $0x7ffe0300,%ecx
    call *%ecx
77ed5d41:	ff d1                	call   *%ecx
    ret $0x4
77ed5d43:	c2 04 00             	ret    $0x4

77ed5d46 <_NtGdiGetTextExtentExPoint@28>:

.global _NtGdiGetTextExtentExPoint@28
_NtGdiGetTextExtentExPoint@28:

    movl $0x109a, %eax
77ed5d46:	b8 9a 10 00 00       	mov    $0x109a,%eax
    movl $KUSER_SHARED_SYSCALL, %ecx
77ed5d4b:	b9 00 03 fe 7f       	mov    $0x7ffe0300,%ecx
    call *%ecx
77ed5d50:	ff d1                	call   *%ecx
    ret $0x1c
77ed5d52:	c2 1c 00             	ret    $0x1c

77ed5d55 <_NtGdiGetTextExtentPoint@16>:

.global _NtGdiGetTextExtentPoint@16
_NtGdiGetTextExtentPoint@16:

    movl $0x109b, %eax
77ed5d55:	b8 9b 10 00 00       	mov    $0x109b,%eax
    movl $KUSER_SHARED_SYSCALL, %ecx
77ed5d5a:	b9 00 03 fe 7f       	mov    $0x7ffe0300,%ecx
    call *%ecx
77ed5d5f:	ff d1                	call   *%ecx
    ret $0x10
77ed5d61:	c2 10 00             	ret    $0x10

77ed5d64 <_NtGdiGetTextExtentPoint32@16>:

.global _NtGdiGetTextExtentPoint32@16
_NtGdiGetTextExtentPoint32@16:

    movl $0x109c, %eax
77ed5d64:	b8 9c 10 00 00       	mov    $0x109c,%eax
    movl $KUSER_SHARED_SYSCALL, %ecx
77ed5d69:	b9 00 03 fe 7f       	mov    $0x7ffe0300,%ecx
    call *%ecx
77ed5d6e:	ff d1                	call   *%ecx
    ret $0x10
77ed5d70:	c2 10 00             	ret    $0x10

77ed5d73 <_NtGdiGetTextFace@12>:

.global _NtGdiGetTextFace@12
_NtGdiGetTextFace@12:

    movl $0x109d, %eax
77ed5d73:	b8 9d 10 00 00       	mov    $0x109d,%eax
    movl $KUSER_SHARED_SYSCALL, %ecx
77ed5d78:	b9 00 03 fe 7f       	mov    $0x7ffe0300,%ecx
    call *%ecx
77ed5d7d:	ff d1                	call   *%ecx
    ret $0xc
77ed5d7f:	c2 0c 00             	ret    $0xc

77ed5d82 <_NtGdiGetTextMetrics@8>:

.global _NtGdiGetTextMetrics@8
_NtGdiGetTextMetrics@8:

    movl $0x109e, %eax
77ed5d82:	b8 9e 10 00 00       	mov    $0x109e,%eax
    movl $KUSER_SHARED_SYSCALL, %ecx
77ed5d87:	b9 00 03 fe 7f       	mov    $0x7ffe0300,%ecx
    call *%ecx
77ed5d8c:	ff d1                	call   *%ecx
    ret $0x8
77ed5d8e:	c2 08 00             	ret    $0x8

77ed5d91 <_NtGdiGetViewportExtEx@8>:

.global _NtGdiGetViewportExtEx@8
_NtGdiGetViewportExtEx@8:

    movl $0x109f, %eax
77ed5d91:	b8 9f 10 00 00       	mov    $0x109f,%eax
    movl $KUSER_SHARED_SYSCALL, %ecx
77ed5d96:	b9 00 03 fe 7f       	mov    $0x7ffe0300,%ecx
    call *%ecx
77ed5d9b:	ff d1                	call   *%ecx
    ret $0x8
77ed5d9d:	c2 08 00             	ret    $0x8

77ed5da0 <_NtGdiGetViewportOrgEx@8>:

.global _NtGdiGetViewportOrgEx@8
_NtGdiGetViewportOrgEx@8:

    movl $0x10a0, %eax
77ed5da0:	b8 a0 10 00 00       	mov    $0x10a0,%eax
    movl $KUSER_SHARED_SYSCALL, %ecx
77ed5da5:	b9 00 03 fe 7f       	mov    $0x7ffe0300,%ecx
    call *%ecx
77ed5daa:	ff d1                	call   *%ecx
    ret $0x8
77ed5dac:	c2 08 00             	ret    $0x8

77ed5daf <_NtGdiGetWinMetaFileBits@20>:

.global _NtGdiGetWinMetaFileBits@20
_NtGdiGetWinMetaFileBits@20:

    movl $0x10a1, %eax
77ed5daf:	b8 a1 10 00 00       	mov    $0x10a1,%eax
    movl $KUSER_SHARED_SYSCALL, %ecx
77ed5db4:	b9 00 03 fe 7f       	mov    $0x7ffe0300,%ecx
    call *%ecx
77ed5db9:	ff d1                	call   *%ecx
    ret $0x14
77ed5dbb:	c2 14 00             	ret    $0x14

77ed5dbe <_NtGdiGetWindowExtEx@8>:

.global _NtGdiGetWindowExtEx@8
_NtGdiGetWindowExtEx@8:

    movl $0x10a2, %eax
77ed5dbe:	b8 a2 10 00 00       	mov    $0x10a2,%eax
    movl $KUSER_SHARED_SYSCALL, %ecx
77ed5dc3:	b9 00 03 fe 7f       	mov    $0x7ffe0300,%ecx
    call *%ecx
77ed5dc8:	ff d1                	call   *%ecx
    ret $0x8
77ed5dca:	c2 08 00             	ret    $0x8

77ed5dcd <_NtGdiGetWindowOrgEx@8>:

.global _NtGdiGetWindowOrgEx@8
_NtGdiGetWindowOrgEx@8:

    movl $0x10a3, %eax
77ed5dcd:	b8 a3 10 00 00       	mov    $0x10a3,%eax
    movl $KUSER_SHARED_SYSCALL, %ecx
77ed5dd2:	b9 00 03 fe 7f       	mov    $0x7ffe0300,%ecx
    call *%ecx
77ed5dd7:	ff d1                	call   *%ecx
    ret $0x8
77ed5dd9:	c2 08 00             	ret    $0x8

77ed5ddc <_NtGdiGetWorldTransform@8>:

.global _NtGdiGetWorldTransform@8
_NtGdiGetWorldTransform@8:

    movl $0x10a4, %eax
77ed5ddc:	b8 a4 10 00 00       	mov    $0x10a4,%eax
    movl $KUSER_SHARED_SYSCALL, %ecx
77ed5de1:	b9 00 03 fe 7f       	mov    $0x7ffe0300,%ecx
    call *%ecx
77ed5de6:	ff d1                	call   *%ecx
    ret $0x8
77ed5de8:	c2 08 00             	ret    $0x8

77ed5deb <_NtGdiGradientFill@24>:

.global _NtGdiGradientFill@24
_NtGdiGradientFill@24:

    movl $0x10a5, %eax
77ed5deb:	b8 a5 10 00 00       	mov    $0x10a5,%eax
    movl $KUSER_SHARED_SYSCALL, %ecx
77ed5df0:	b9 00 03 fe 7f       	mov    $0x7ffe0300,%ecx
    call *%ecx
77ed5df5:	ff d1                	call   *%ecx
    ret $0x18
77ed5df7:	c2 18 00             	ret    $0x18

77ed5dfa <_NtGdiIntersectClipRect@20>:

.global _NtGdiIntersectClipRect@20
_NtGdiIntersectClipRect@20:

    movl $0x10a6, %eax
77ed5dfa:	b8 a6 10 00 00       	mov    $0x10a6,%eax
    movl $KUSER_SHARED_SYSCALL, %ecx
77ed5dff:	b9 00 03 fe 7f       	mov    $0x7ffe0300,%ecx
    call *%ecx
77ed5e04:	ff d1                	call   *%ecx
    ret $0x14
77ed5e06:	c2 14 00             	ret    $0x14

77ed5e09 <_NtGdiInvertRgn@8>:

.global _NtGdiInvertRgn@8
_NtGdiInvertRgn@8:

    movl $0x10a7, %eax
77ed5e09:	b8 a7 10 00 00       	mov    $0x10a7,%eax
    movl $KUSER_SHARED_SYSCALL, %ecx
77ed5e0e:	b9 00 03 fe 7f       	mov    $0x7ffe0300,%ecx
    call *%ecx
77ed5e13:	ff d1                	call   *%ecx
    ret $0x8
77ed5e15:	c2 08 00             	ret    $0x8

77ed5e18 <_NtGdiLPtoDP@12>:

.global _NtGdiLPtoDP@12
_NtGdiLPtoDP@12:

    movl $0x10a8, %eax
77ed5e18:	b8 a8 10 00 00       	mov    $0x10a8,%eax
    movl $KUSER_SHARED_SYSCALL, %ecx
77ed5e1d:	b9 00 03 fe 7f       	mov    $0x7ffe0300,%ecx
    call *%ecx
77ed5e22:	ff d1                	call   *%ecx
    ret $0xc
77ed5e24:	c2 0c 00             	ret    $0xc

77ed5e27 <_NtGdiLineTo@12>:

.global _NtGdiLineTo@12
_NtGdiLineTo@12:

    movl $0x10a9, %eax
77ed5e27:	b8 a9 10 00 00       	mov    $0x10a9,%eax
    movl $KUSER_SHARED_SYSCALL, %ecx
77ed5e2c:	b9 00 03 fe 7f       	mov    $0x7ffe0300,%ecx
    call *%ecx
77ed5e31:	ff d1                	call   *%ecx
    ret $0xc
77ed5e33:	c2 0c 00             	ret    $0xc

77ed5e36 <_NtGdiMaskBlt@48>:

.global _NtGdiMaskBlt@48
_NtGdiMaskBlt@48:

    movl $0x10aa, %eax
77ed5e36:	b8 aa 10 00 00       	mov    $0x10aa,%eax
    movl $KUSER_SHARED_SYSCALL, %ecx
77ed5e3b:	b9 00 03 fe 7f       	mov    $0x7ffe0300,%ecx
    call *%ecx
77ed5e40:	ff d1                	call   *%ecx
    ret $0x30
77ed5e42:	c2 30 00             	ret    $0x30

77ed5e45 <_NtGdiModifyWorldTransform@12>:

.global _NtGdiModifyWorldTransform@12
_NtGdiModifyWorldTransform@12:

    movl $0x10ab, %eax
77ed5e45:	b8 ab 10 00 00       	mov    $0x10ab,%eax
    movl $KUSER_SHARED_SYSCALL, %ecx
77ed5e4a:	b9 00 03 fe 7f       	mov    $0x7ffe0300,%ecx
    call *%ecx
77ed5e4f:	ff d1                	call   *%ecx
    ret $0xc
77ed5e51:	c2 0c 00             	ret    $0xc

77ed5e54 <_NtGdiMoveToEx@16>:

.global _NtGdiMoveToEx@16
_NtGdiMoveToEx@16:

    movl $0x10ac, %eax
77ed5e54:	b8 ac 10 00 00       	mov    $0x10ac,%eax
    movl $KUSER_SHARED_SYSCALL, %ecx
77ed5e59:	b9 00 03 fe 7f       	mov    $0x7ffe0300,%ecx
    call *%ecx
77ed5e5e:	ff d1                	call   *%ecx
    ret $0x10
77ed5e60:	c2 10 00             	ret    $0x10

77ed5e63 <_NtGdiOffsetClipRgn@12>:

.global _NtGdiOffsetClipRgn@12
_NtGdiOffsetClipRgn@12:

    movl $0x10ad, %eax
77ed5e63:	b8 ad 10 00 00       	mov    $0x10ad,%eax
    movl $KUSER_SHARED_SYSCALL, %ecx
77ed5e68:	b9 00 03 fe 7f       	mov    $0x7ffe0300,%ecx
    call *%ecx
77ed5e6d:	ff d1                	call   *%ecx
    ret $0xc
77ed5e6f:	c2 0c 00             	ret    $0xc

77ed5e72 <_NtGdiOffsetRgn@12>:

.global _NtGdiOffsetRgn@12
_NtGdiOffsetRgn@12:

    movl $0x10ae, %eax
77ed5e72:	b8 ae 10 00 00       	mov    $0x10ae,%eax
    movl $KUSER_SHARED_SYSCALL, %ecx
77ed5e77:	b9 00 03 fe 7f       	mov    $0x7ffe0300,%ecx
    call *%ecx
77ed5e7c:	ff d1                	call   *%ecx
    ret $0xc
77ed5e7e:	c2 0c 00             	ret    $0xc

77ed5e81 <_NtGdiOffsetViewportOrgEx@16>:

.global _NtGdiOffsetViewportOrgEx@16
_NtGdiOffsetViewportOrgEx@16:

    movl $0x10af, %eax
77ed5e81:	b8 af 10 00 00       	mov    $0x10af,%eax
    movl $KUSER_SHARED_SYSCALL, %ecx
77ed5e86:	b9 00 03 fe 7f       	mov    $0x7ffe0300,%ecx
    call *%ecx
77ed5e8b:	ff d1                	call   *%ecx
    ret $0x10
77ed5e8d:	c2 10 00             	ret    $0x10

77ed5e90 <_NtGdiOffsetWindowOrgEx@16>:

.global _NtGdiOffsetWindowOrgEx@16
_NtGdiOffsetWindowOrgEx@16:

    movl $0x10b0, %eax
77ed5e90:	b8 b0 10 00 00       	mov    $0x10b0,%eax
    movl $KUSER_SHARED_SYSCALL, %ecx
77ed5e95:	b9 00 03 fe 7f       	mov    $0x7ffe0300,%ecx
    call *%ecx
77ed5e9a:	ff d1                	call   *%ecx
    ret $0x10
77ed5e9c:	c2 10 00             	ret    $0x10

77ed5e9f <_NtGdiPaintRgn@8>:

.global _NtGdiPaintRgn@8
_NtGdiPaintRgn@8:

    movl $0x10b1, %eax
77ed5e9f:	b8 b1 10 00 00       	mov    $0x10b1,%eax
    movl $KUSER_SHARED_SYSCALL, %ecx
77ed5ea4:	b9 00 03 fe 7f       	mov    $0x7ffe0300,%ecx
    call *%ecx
77ed5ea9:	ff d1                	call   *%ecx
    ret $0x8
77ed5eab:	c2 08 00             	ret    $0x8

77ed5eae <_NtGdiPatBlt@24>:

.global _NtGdiPatBlt@24
_NtGdiPatBlt@24:

    movl $0x10b2, %eax
77ed5eae:	b8 b2 10 00 00       	mov    $0x10b2,%eax
    movl $KUSER_SHARED_SYSCALL, %ecx
77ed5eb3:	b9 00 03 fe 7f       	mov    $0x7ffe0300,%ecx
    call *%ecx
77ed5eb8:	ff d1                	call   *%ecx
    ret $0x18
77ed5eba:	c2 18 00             	ret    $0x18

77ed5ebd <_NtGdiPathToRegion@4>:

.global _NtGdiPathToRegion@4
_NtGdiPathToRegion@4:

    movl $0x10b3, %eax
77ed5ebd:	b8 b3 10 00 00       	mov    $0x10b3,%eax
    movl $KUSER_SHARED_SYSCALL, %ecx
77ed5ec2:	b9 00 03 fe 7f       	mov    $0x7ffe0300,%ecx
    call *%ecx
77ed5ec7:	ff d1                	call   *%ecx
    ret $0x4
77ed5ec9:	c2 04 00             	ret    $0x4

77ed5ecc <_NtGdiPie@36>:

.global _NtGdiPie@36
_NtGdiPie@36:

    movl $0x10b4, %eax
77ed5ecc:	b8 b4 10 00 00       	mov    $0x10b4,%eax
    movl $KUSER_SHARED_SYSCALL, %ecx
77ed5ed1:	b9 00 03 fe 7f       	mov    $0x7ffe0300,%ecx
    call *%ecx
77ed5ed6:	ff d1                	call   *%ecx
    ret $0x24
77ed5ed8:	c2 24 00             	ret    $0x24

77ed5edb <_NtGdiPlayEnhMetaFile@12>:

.global _NtGdiPlayEnhMetaFile@12
_NtGdiPlayEnhMetaFile@12:

    movl $0x10b5, %eax
77ed5edb:	b8 b5 10 00 00       	mov    $0x10b5,%eax
    movl $KUSER_SHARED_SYSCALL, %ecx
77ed5ee0:	b9 00 03 fe 7f       	mov    $0x7ffe0300,%ecx
    call *%ecx
77ed5ee5:	ff d1                	call   *%ecx
    ret $0xc
77ed5ee7:	c2 0c 00             	ret    $0xc

77ed5eea <_NtGdiPlayEnhMetaFileRecord@16>:

.global _NtGdiPlayEnhMetaFileRecord@16
_NtGdiPlayEnhMetaFileRecord@16:

    movl $0x10b6, %eax
77ed5eea:	b8 b6 10 00 00       	mov    $0x10b6,%eax
    movl $KUSER_SHARED_SYSCALL, %ecx
77ed5eef:	b9 00 03 fe 7f       	mov    $0x7ffe0300,%ecx
    call *%ecx
77ed5ef4:	ff d1                	call   *%ecx
    ret $0x10
77ed5ef6:	c2 10 00             	ret    $0x10

77ed5ef9 <_NtGdiPlayMetaFile@8>:

.global _NtGdiPlayMetaFile@8
_NtGdiPlayMetaFile@8:

    movl $0x10b7, %eax
77ed5ef9:	b8 b7 10 00 00       	mov    $0x10b7,%eax
    movl $KUSER_SHARED_SYSCALL, %ecx
77ed5efe:	b9 00 03 fe 7f       	mov    $0x7ffe0300,%ecx
    call *%ecx
77ed5f03:	ff d1                	call   *%ecx
    ret $0x8
77ed5f05:	c2 08 00             	ret    $0x8

77ed5f08 <_NtGdiPlayMetaFileRecord@16>:

.global _NtGdiPlayMetaFileRecord@16
_NtGdiPlayMetaFileRecord@16:

    movl $0x10b8, %eax
77ed5f08:	b8 b8 10 00 00       	mov    $0x10b8,%eax
    movl $KUSER_SHARED_SYSCALL, %ecx
77ed5f0d:	b9 00 03 fe 7f       	mov    $0x7ffe0300,%ecx
    call *%ecx
77ed5f12:	ff d1                	call   *%ecx
    ret $0x10
77ed5f14:	c2 10 00             	ret    $0x10

77ed5f17 <_NtGdiPlgBlt@40>:

.global _NtGdiPlgBlt@40
_NtGdiPlgBlt@40:

    movl $0x10b9, %eax
77ed5f17:	b8 b9 10 00 00       	mov    $0x10b9,%eax
    movl $KUSER_SHARED_SYSCALL, %ecx
77ed5f1c:	b9 00 03 fe 7f       	mov    $0x7ffe0300,%ecx
    call *%ecx
77ed5f21:	ff d1                	call   *%ecx
    ret $0x28
77ed5f23:	c2 28 00             	ret    $0x28

77ed5f26 <_NtGdiPolyBezier@12>:

.global _NtGdiPolyBezier@12
_NtGdiPolyBezier@12:

    movl $0x10ba, %eax
77ed5f26:	b8 ba 10 00 00       	mov    $0x10ba,%eax
    movl $KUSER_SHARED_SYSCALL, %ecx
77ed5f2b:	b9 00 03 fe 7f       	mov    $0x7ffe0300,%ecx
    call *%ecx
77ed5f30:	ff d1                	call   *%ecx
    ret $0xc
77ed5f32:	c2 0c 00             	ret    $0xc

77ed5f35 <_NtGdiPolyBezierTo@12>:

.global _NtGdiPolyBezierTo@12
_NtGdiPolyBezierTo@12:

    movl $0x10bb, %eax
77ed5f35:	b8 bb 10 00 00       	mov    $0x10bb,%eax
    movl $KUSER_SHARED_SYSCALL, %ecx
77ed5f3a:	b9 00 03 fe 7f       	mov    $0x7ffe0300,%ecx
    call *%ecx
77ed5f3f:	ff d1                	call   *%ecx
    ret $0xc
77ed5f41:	c2 0c 00             	ret    $0xc

77ed5f44 <_NtGdiPolyDraw@16>:

.global _NtGdiPolyDraw@16
_NtGdiPolyDraw@16:

    movl $0x10bc, %eax
77ed5f44:	b8 bc 10 00 00       	mov    $0x10bc,%eax
    movl $KUSER_SHARED_SYSCALL, %ecx
77ed5f49:	b9 00 03 fe 7f       	mov    $0x7ffe0300,%ecx
    call *%ecx
77ed5f4e:	ff d1                	call   *%ecx
    ret $0x10
77ed5f50:	c2 10 00             	ret    $0x10

77ed5f53 <_NtGdiPolyline@12>:

.global _NtGdiPolyline@12
_NtGdiPolyline@12:

    movl $0x10bd, %eax
77ed5f53:	b8 bd 10 00 00       	mov    $0x10bd,%eax
    movl $KUSER_SHARED_SYSCALL, %ecx
77ed5f58:	b9 00 03 fe 7f       	mov    $0x7ffe0300,%ecx
    call *%ecx
77ed5f5d:	ff d1                	call   *%ecx
    ret $0xc
77ed5f5f:	c2 0c 00             	ret    $0xc

77ed5f62 <_NtGdiPolylineTo@12>:

.global _NtGdiPolylineTo@12
_NtGdiPolylineTo@12:

    movl $0x10be, %eax
77ed5f62:	b8 be 10 00 00       	mov    $0x10be,%eax
    movl $KUSER_SHARED_SYSCALL, %ecx
77ed5f67:	b9 00 03 fe 7f       	mov    $0x7ffe0300,%ecx
    call *%ecx
77ed5f6c:	ff d1                	call   *%ecx
    ret $0xc
77ed5f6e:	c2 0c 00             	ret    $0xc

77ed5f71 <_NtGdiPolyPatBlt@20>:

.global _NtGdiPolyPatBlt@20
_NtGdiPolyPatBlt@20:

    movl $0x10bf, %eax
77ed5f71:	b8 bf 10 00 00       	mov    $0x10bf,%eax
    movl $KUSER_SHARED_SYSCALL, %ecx
77ed5f76:	b9 00 03 fe 7f       	mov    $0x7ffe0300,%ecx
    call *%ecx
77ed5f7b:	ff d1                	call   *%ecx
    ret $0x14
77ed5f7d:	c2 14 00             	ret    $0x14

77ed5f80 <_NtGdiPolyPolyline@16>:

.global _NtGdiPolyPolyline@16
_NtGdiPolyPolyline@16:

    movl $0x10c0, %eax
77ed5f80:	b8 c0 10 00 00       	mov    $0x10c0,%eax
    movl $KUSER_SHARED_SYSCALL, %ecx
77ed5f85:	b9 00 03 fe 7f       	mov    $0x7ffe0300,%ecx
    call *%ecx
77ed5f8a:	ff d1                	call   *%ecx
    ret $0x10
77ed5f8c:	c2 10 00             	ret    $0x10

77ed5f8f <_NtGdiPolyTextOut@12>:

.global _NtGdiPolyTextOut@12
_NtGdiPolyTextOut@12:

    movl $0x10c1, %eax
77ed5f8f:	b8 c1 10 00 00       	mov    $0x10c1,%eax
    movl $KUSER_SHARED_SYSCALL, %ecx
77ed5f94:	b9 00 03 fe 7f       	mov    $0x7ffe0300,%ecx
    call *%ecx
77ed5f99:	ff d1                	call   *%ecx
    ret $0xc
77ed5f9b:	c2 0c 00             	ret    $0xc

77ed5f9e <_NtGdiPolygon@12>:

.global _NtGdiPolygon@12
_NtGdiPolygon@12:

    movl $0x10c2, %eax
77ed5f9e:	b8 c2 10 00 00       	mov    $0x10c2,%eax
    movl $KUSER_SHARED_SYSCALL, %ecx
77ed5fa3:	b9 00 03 fe 7f       	mov    $0x7ffe0300,%ecx
    call *%ecx
77ed5fa8:	ff d1                	call   *%ecx
    ret $0xc
77ed5faa:	c2 0c 00             	ret    $0xc

77ed5fad <_NtGdiPolyPolygon@16>:

.global _NtGdiPolyPolygon@16
_NtGdiPolyPolygon@16:

    movl $0x10c3, %eax
77ed5fad:	b8 c3 10 00 00       	mov    $0x10c3,%eax
    movl $KUSER_SHARED_SYSCALL, %ecx
77ed5fb2:	b9 00 03 fe 7f       	mov    $0x7ffe0300,%ecx
    call *%ecx
77ed5fb7:	ff d1                	call   *%ecx
    ret $0x10
77ed5fb9:	c2 10 00             	ret    $0x10

77ed5fbc <_NtGdiPtInRegion@12>:

.global _NtGdiPtInRegion@12
_NtGdiPtInRegion@12:

    movl $0x10c4, %eax
77ed5fbc:	b8 c4 10 00 00       	mov    $0x10c4,%eax
    movl $KUSER_SHARED_SYSCALL, %ecx
77ed5fc1:	b9 00 03 fe 7f       	mov    $0x7ffe0300,%ecx
    call *%ecx
77ed5fc6:	ff d1                	call   *%ecx
    ret $0xc
77ed5fc8:	c2 0c 00             	ret    $0xc

77ed5fcb <_NtGdiPtVisible@12>:

.global _NtGdiPtVisible@12
_NtGdiPtVisible@12:

    movl $0x10c5, %eax
77ed5fcb:	b8 c5 10 00 00       	mov    $0x10c5,%eax
    movl $KUSER_SHARED_SYSCALL, %ecx
77ed5fd0:	b9 00 03 fe 7f       	mov    $0x7ffe0300,%ecx
    call *%ecx
77ed5fd5:	ff d1                	call   *%ecx
    ret $0xc
77ed5fd7:	c2 0c 00             	ret    $0xc

77ed5fda <_NtGdiRealizePalette@4>:

.global _NtGdiRealizePalette@4
_NtGdiRealizePalette@4:

    movl $0x10c6, %eax
77ed5fda:	b8 c6 10 00 00       	mov    $0x10c6,%eax
    movl $KUSER_SHARED_SYSCALL, %ecx
77ed5fdf:	b9 00 03 fe 7f       	mov    $0x7ffe0300,%ecx
    call *%ecx
77ed5fe4:	ff d1                	call   *%ecx
    ret $0x4
77ed5fe6:	c2 04 00             	ret    $0x4

77ed5fe9 <_NtGdiRectInRegion@8>:

.global _NtGdiRectInRegion@8
_NtGdiRectInRegion@8:

    movl $0x10c7, %eax
77ed5fe9:	b8 c7 10 00 00       	mov    $0x10c7,%eax
    movl $KUSER_SHARED_SYSCALL, %ecx
77ed5fee:	b9 00 03 fe 7f       	mov    $0x7ffe0300,%ecx
    call *%ecx
77ed5ff3:	ff d1                	call   *%ecx
    ret $0x8
77ed5ff5:	c2 08 00             	ret    $0x8

77ed5ff8 <_NtGdiRectVisible@8>:

.global _NtGdiRectVisible@8
_NtGdiRectVisible@8:

    movl $0x10c8, %eax
77ed5ff8:	b8 c8 10 00 00       	mov    $0x10c8,%eax
    movl $KUSER_SHARED_SYSCALL, %ecx
77ed5ffd:	b9 00 03 fe 7f       	mov    $0x7ffe0300,%ecx
    call *%ecx
77ed6002:	ff d1                	call   *%ecx
    ret $0x8
77ed6004:	c2 08 00             	ret    $0x8

77ed6007 <_NtGdiRectangle@20>:

.global _NtGdiRectangle@20
_NtGdiRectangle@20:

    movl $0x10c9, %eax
77ed6007:	b8 c9 10 00 00       	mov    $0x10c9,%eax
    movl $KUSER_SHARED_SYSCALL, %ecx
77ed600c:	b9 00 03 fe 7f       	mov    $0x7ffe0300,%ecx
    call *%ecx
77ed6011:	ff d1                	call   *%ecx
    ret $0x14
77ed6013:	c2 14 00             	ret    $0x14

77ed6016 <_NtGdiRemoveFontResource@4>:

.global _NtGdiRemoveFontResource@4
_NtGdiRemoveFontResource@4:

    movl $0x10ca, %eax
77ed6016:	b8 ca 10 00 00       	mov    $0x10ca,%eax
    movl $KUSER_SHARED_SYSCALL, %ecx
77ed601b:	b9 00 03 fe 7f       	mov    $0x7ffe0300,%ecx
    call *%ecx
77ed6020:	ff d1                	call   *%ecx
    ret $0x4
77ed6022:	c2 04 00             	ret    $0x4

77ed6025 <_NtGdiResetDC@8>:

.global _NtGdiResetDC@8
_NtGdiResetDC@8:

    movl $0x10cb, %eax
77ed6025:	b8 cb 10 00 00       	mov    $0x10cb,%eax
    movl $KUSER_SHARED_SYSCALL, %ecx
77ed602a:	b9 00 03 fe 7f       	mov    $0x7ffe0300,%ecx
    call *%ecx
77ed602f:	ff d1                	call   *%ecx
    ret $0x8
77ed6031:	c2 08 00             	ret    $0x8

77ed6034 <_NtGdiResizePalette@8>:

.global _NtGdiResizePalette@8
_NtGdiResizePalette@8:

    movl $0x10cc, %eax
77ed6034:	b8 cc 10 00 00       	mov    $0x10cc,%eax
    movl $KUSER_SHARED_SYSCALL, %ecx
77ed6039:	b9 00 03 fe 7f       	mov    $0x7ffe0300,%ecx
    call *%ecx
77ed603e:	ff d1                	call   *%ecx
    ret $0x8
77ed6040:	c2 08 00             	ret    $0x8

77ed6043 <_NtGdiRestoreDC@8>:

.global _NtGdiRestoreDC@8
_NtGdiRestoreDC@8:

    movl $0x10cd, %eax
77ed6043:	b8 cd 10 00 00       	mov    $0x10cd,%eax
    movl $KUSER_SHARED_SYSCALL, %ecx
77ed6048:	b9 00 03 fe 7f       	mov    $0x7ffe0300,%ecx
    call *%ecx
77ed604d:	ff d1                	call   *%ecx
    ret $0x8
77ed604f:	c2 08 00             	ret    $0x8

77ed6052 <_NtGdiRoundRect@28>:

.global _NtGdiRoundRect@28
_NtGdiRoundRect@28:

    movl $0x10ce, %eax
77ed6052:	b8 ce 10 00 00       	mov    $0x10ce,%eax
    movl $KUSER_SHARED_SYSCALL, %ecx
77ed6057:	b9 00 03 fe 7f       	mov    $0x7ffe0300,%ecx
    call *%ecx
77ed605c:	ff d1                	call   *%ecx
    ret $0x1c
77ed605e:	c2 1c 00             	ret    $0x1c

77ed6061 <_NtGdiSaveDC@4>:

.global _NtGdiSaveDC@4
_NtGdiSaveDC@4:

    movl $0x10cf, %eax
77ed6061:	b8 cf 10 00 00       	mov    $0x10cf,%eax
    movl $KUSER_SHARED_SYSCALL, %ecx
77ed6066:	b9 00 03 fe 7f       	mov    $0x7ffe0300,%ecx
    call *%ecx
77ed606b:	ff d1                	call   *%ecx
    ret $0x4
77ed606d:	c2 04 00             	ret    $0x4

77ed6070 <_NtGdiScaleViewportExtEx@24>:

.global _NtGdiScaleViewportExtEx@24
_NtGdiScaleViewportExtEx@24:

    movl $0x10d0, %eax
77ed6070:	b8 d0 10 00 00       	mov    $0x10d0,%eax
    movl $KUSER_SHARED_SYSCALL, %ecx
77ed6075:	b9 00 03 fe 7f       	mov    $0x7ffe0300,%ecx
    call *%ecx
77ed607a:	ff d1                	call   *%ecx
    ret $0x18
77ed607c:	c2 18 00             	ret    $0x18

77ed607f <_NtGdiScaleWindowExtEx@24>:

.global _NtGdiScaleWindowExtEx@24
_NtGdiScaleWindowExtEx@24:

    movl $0x10d1, %eax
77ed607f:	b8 d1 10 00 00       	mov    $0x10d1,%eax
    movl $KUSER_SHARED_SYSCALL, %ecx
77ed6084:	b9 00 03 fe 7f       	mov    $0x7ffe0300,%ecx
    call *%ecx
77ed6089:	ff d1                	call   *%ecx
    ret $0x18
77ed608b:	c2 18 00             	ret    $0x18

77ed608e <_NtGdiSelectClipPath@8>:

.global _NtGdiSelectClipPath@8
_NtGdiSelectClipPath@8:

    movl $0x10d2, %eax
77ed608e:	b8 d2 10 00 00       	mov    $0x10d2,%eax
    movl $KUSER_SHARED_SYSCALL, %ecx
77ed6093:	b9 00 03 fe 7f       	mov    $0x7ffe0300,%ecx
    call *%ecx
77ed6098:	ff d1                	call   *%ecx
    ret $0x8
77ed609a:	c2 08 00             	ret    $0x8

77ed609d <_NtGdiSelectClipRgn@8>:

.global _NtGdiSelectClipRgn@8
_NtGdiSelectClipRgn@8:

    movl $0x10d3, %eax
77ed609d:	b8 d3 10 00 00       	mov    $0x10d3,%eax
    movl $KUSER_SHARED_SYSCALL, %ecx
77ed60a2:	b9 00 03 fe 7f       	mov    $0x7ffe0300,%ecx
    call *%ecx
77ed60a7:	ff d1                	call   *%ecx
    ret $0x8
77ed60a9:	c2 08 00             	ret    $0x8

77ed60ac <_NtGdiSelectObject@8>:

.global _NtGdiSelectObject@8
_NtGdiSelectObject@8:

    movl $0x10d4, %eax
77ed60ac:	b8 d4 10 00 00       	mov    $0x10d4,%eax
    movl $KUSER_SHARED_SYSCALL, %ecx
77ed60b1:	b9 00 03 fe 7f       	mov    $0x7ffe0300,%ecx
    call *%ecx
77ed60b6:	ff d1                	call   *%ecx
    ret $0x8
77ed60b8:	c2 08 00             	ret    $0x8

77ed60bb <_NtGdiSelectPalette@12>:

.global _NtGdiSelectPalette@12
_NtGdiSelectPalette@12:

    movl $0x10d5, %eax
77ed60bb:	b8 d5 10 00 00       	mov    $0x10d5,%eax
    movl $KUSER_SHARED_SYSCALL, %ecx
77ed60c0:	b9 00 03 fe 7f       	mov    $0x7ffe0300,%ecx
    call *%ecx
77ed60c5:	ff d1                	call   *%ecx
    ret $0xc
77ed60c7:	c2 0c 00             	ret    $0xc

77ed60ca <_NtGdiSetAbortProc@8>:

.global _NtGdiSetAbortProc@8
_NtGdiSetAbortProc@8:

    movl $0x10d6, %eax
77ed60ca:	b8 d6 10 00 00       	mov    $0x10d6,%eax
    movl $KUSER_SHARED_SYSCALL, %ecx
77ed60cf:	b9 00 03 fe 7f       	mov    $0x7ffe0300,%ecx
    call *%ecx
77ed60d4:	ff d1                	call   *%ecx
    ret $0x8
77ed60d6:	c2 08 00             	ret    $0x8

77ed60d9 <_NtGdiSetArcDirection@8>:

.global _NtGdiSetArcDirection@8
_NtGdiSetArcDirection@8:

    movl $0x10d7, %eax
77ed60d9:	b8 d7 10 00 00       	mov    $0x10d7,%eax
    movl $KUSER_SHARED_SYSCALL, %ecx
77ed60de:	b9 00 03 fe 7f       	mov    $0x7ffe0300,%ecx
    call *%ecx
77ed60e3:	ff d1                	call   *%ecx
    ret $0x8
77ed60e5:	c2 08 00             	ret    $0x8

77ed60e8 <_NtGdiSetBitmapBits@12>:

.global _NtGdiSetBitmapBits@12
_NtGdiSetBitmapBits@12:

    movl $0x10d8, %eax
77ed60e8:	b8 d8 10 00 00       	mov    $0x10d8,%eax
    movl $KUSER_SHARED_SYSCALL, %ecx
77ed60ed:	b9 00 03 fe 7f       	mov    $0x7ffe0300,%ecx
    call *%ecx
77ed60f2:	ff d1                	call   *%ecx
    ret $0xc
77ed60f4:	c2 0c 00             	ret    $0xc

77ed60f7 <_NtGdiSetBitmapDimensionEx@16>:

.global _NtGdiSetBitmapDimensionEx@16
_NtGdiSetBitmapDimensionEx@16:

    movl $0x10d9, %eax
77ed60f7:	b8 d9 10 00 00       	mov    $0x10d9,%eax
    movl $KUSER_SHARED_SYSCALL, %ecx
77ed60fc:	b9 00 03 fe 7f       	mov    $0x7ffe0300,%ecx
    call *%ecx
77ed6101:	ff d1                	call   *%ecx
    ret $0x10
77ed6103:	c2 10 00             	ret    $0x10

77ed6106 <_NtGdiSetBkColor@8>:

.global _NtGdiSetBkColor@8
_NtGdiSetBkColor@8:

    movl $0x10da, %eax
77ed6106:	b8 da 10 00 00       	mov    $0x10da,%eax
    movl $KUSER_SHARED_SYSCALL, %ecx
77ed610b:	b9 00 03 fe 7f       	mov    $0x7ffe0300,%ecx
    call *%ecx
77ed6110:	ff d1                	call   *%ecx
    ret $0x8
77ed6112:	c2 08 00             	ret    $0x8

77ed6115 <_NtGdiSetBkMode@8>:

.global _NtGdiSetBkMode@8
_NtGdiSetBkMode@8:

    movl $0x10db, %eax
77ed6115:	b8 db 10 00 00       	mov    $0x10db,%eax
    movl $KUSER_SHARED_SYSCALL, %ecx
77ed611a:	b9 00 03 fe 7f       	mov    $0x7ffe0300,%ecx
    call *%ecx
77ed611f:	ff d1                	call   *%ecx
    ret $0x8
77ed6121:	c2 08 00             	ret    $0x8

77ed6124 <_NtGdiSetBoundsRect@12>:

.global _NtGdiSetBoundsRect@12
_NtGdiSetBoundsRect@12:

    movl $0x10dc, %eax
77ed6124:	b8 dc 10 00 00       	mov    $0x10dc,%eax
    movl $KUSER_SHARED_SYSCALL, %ecx
77ed6129:	b9 00 03 fe 7f       	mov    $0x7ffe0300,%ecx
    call *%ecx
77ed612e:	ff d1                	call   *%ecx
    ret $0xc
77ed6130:	c2 0c 00             	ret    $0xc

77ed6133 <_NtGdiSetBrushOrgEx@16>:

.global _NtGdiSetBrushOrgEx@16
_NtGdiSetBrushOrgEx@16:

    movl $0x10dd, %eax
77ed6133:	b8 dd 10 00 00       	mov    $0x10dd,%eax
    movl $KUSER_SHARED_SYSCALL, %ecx
77ed6138:	b9 00 03 fe 7f       	mov    $0x7ffe0300,%ecx
    call *%ecx
77ed613d:	ff d1                	call   *%ecx
    ret $0x10
77ed613f:	c2 10 00             	ret    $0x10

77ed6142 <_NtGdiSetColorAdjustment@8>:

.global _NtGdiSetColorAdjustment@8
_NtGdiSetColorAdjustment@8:

    movl $0x10de, %eax
77ed6142:	b8 de 10 00 00       	mov    $0x10de,%eax
    movl $KUSER_SHARED_SYSCALL, %ecx
77ed6147:	b9 00 03 fe 7f       	mov    $0x7ffe0300,%ecx
    call *%ecx
77ed614c:	ff d1                	call   *%ecx
    ret $0x8
77ed614e:	c2 08 00             	ret    $0x8

77ed6151 <_NtGdiSetColorSpace@8>:

.global _NtGdiSetColorSpace@8
_NtGdiSetColorSpace@8:

    movl $0x10df, %eax
77ed6151:	b8 df 10 00 00       	mov    $0x10df,%eax
    movl $KUSER_SHARED_SYSCALL, %ecx
77ed6156:	b9 00 03 fe 7f       	mov    $0x7ffe0300,%ecx
    call *%ecx
77ed615b:	ff d1                	call   *%ecx
    ret $0x8
77ed615d:	c2 08 00             	ret    $0x8

77ed6160 <_NtGdiSetDIBColorTable@16>:

.global _NtGdiSetDIBColorTable@16
_NtGdiSetDIBColorTable@16:

    movl $0x10e0, %eax
77ed6160:	b8 e0 10 00 00       	mov    $0x10e0,%eax
    movl $KUSER_SHARED_SYSCALL, %ecx
77ed6165:	b9 00 03 fe 7f       	mov    $0x7ffe0300,%ecx
    call *%ecx
77ed616a:	ff d1                	call   *%ecx
    ret $0x10
77ed616c:	c2 10 00             	ret    $0x10

77ed616f <_NtGdiSetDIBits@28>:

.global _NtGdiSetDIBits@28
_NtGdiSetDIBits@28:

    movl $0x10e1, %eax
77ed616f:	b8 e1 10 00 00       	mov    $0x10e1,%eax
    movl $KUSER_SHARED_SYSCALL, %ecx
77ed6174:	b9 00 03 fe 7f       	mov    $0x7ffe0300,%ecx
    call *%ecx
77ed6179:	ff d1                	call   *%ecx
    ret $0x1c
77ed617b:	c2 1c 00             	ret    $0x1c

77ed617e <_NtGdiSetDIBitsToDevice@48>:

.global _NtGdiSetDIBitsToDevice@48
_NtGdiSetDIBitsToDevice@48:

    movl $0x10e2, %eax
77ed617e:	b8 e2 10 00 00       	mov    $0x10e2,%eax
    movl $KUSER_SHARED_SYSCALL, %ecx
77ed6183:	b9 00 03 fe 7f       	mov    $0x7ffe0300,%ecx
    call *%ecx
77ed6188:	ff d1                	call   *%ecx
    ret $0x30
77ed618a:	c2 30 00             	ret    $0x30

77ed618d <_NtGdiSetDeviceGammaRamp@8>:

.global _NtGdiSetDeviceGammaRamp@8
_NtGdiSetDeviceGammaRamp@8:

    movl $0x10e3, %eax
77ed618d:	b8 e3 10 00 00       	mov    $0x10e3,%eax
    movl $KUSER_SHARED_SYSCALL, %ecx
77ed6192:	b9 00 03 fe 7f       	mov    $0x7ffe0300,%ecx
    call *%ecx
77ed6197:	ff d1                	call   *%ecx
    ret $0x8
77ed6199:	c2 08 00             	ret    $0x8

77ed619c <_NtGdiSetEnhMetaFileBits@8>:

.global _NtGdiSetEnhMetaFileBits@8
_NtGdiSetEnhMetaFileBits@8:

    movl $0x10e4, %eax
77ed619c:	b8 e4 10 00 00       	mov    $0x10e4,%eax
    movl $KUSER_SHARED_SYSCALL, %ecx
77ed61a1:	b9 00 03 fe 7f       	mov    $0x7ffe0300,%ecx
    call *%ecx
77ed61a6:	ff d1                	call   *%ecx
    ret $0x8
77ed61a8:	c2 08 00             	ret    $0x8

77ed61ab <_NtGdiSetGraphicsMode@8>:

.global _NtGdiSetGraphicsMode@8
_NtGdiSetGraphicsMode@8:

    movl $0x10e5, %eax
77ed61ab:	b8 e5 10 00 00       	mov    $0x10e5,%eax
    movl $KUSER_SHARED_SYSCALL, %ecx
77ed61b0:	b9 00 03 fe 7f       	mov    $0x7ffe0300,%ecx
    call *%ecx
77ed61b5:	ff d1                	call   *%ecx
    ret $0x8
77ed61b7:	c2 08 00             	ret    $0x8

77ed61ba <_NtGdiSetICMMode@8>:

.global _NtGdiSetICMMode@8
_NtGdiSetICMMode@8:

    movl $0x10e6, %eax
77ed61ba:	b8 e6 10 00 00       	mov    $0x10e6,%eax
    movl $KUSER_SHARED_SYSCALL, %ecx
77ed61bf:	b9 00 03 fe 7f       	mov    $0x7ffe0300,%ecx
    call *%ecx
77ed61c4:	ff d1                	call   *%ecx
    ret $0x8
77ed61c6:	c2 08 00             	ret    $0x8

77ed61c9 <_NtGdiSetICMProfile@8>:

.global _NtGdiSetICMProfile@8
_NtGdiSetICMProfile@8:

    movl $0x10e7, %eax
77ed61c9:	b8 e7 10 00 00       	mov    $0x10e7,%eax
    movl $KUSER_SHARED_SYSCALL, %ecx
77ed61ce:	b9 00 03 fe 7f       	mov    $0x7ffe0300,%ecx
    call *%ecx
77ed61d3:	ff d1                	call   *%ecx
    ret $0x8
77ed61d5:	c2 08 00             	ret    $0x8

77ed61d8 <_NtGdiSetMapMode@8>:

.global _NtGdiSetMapMode@8
_NtGdiSetMapMode@8:

    movl $0x10e8, %eax
77ed61d8:	b8 e8 10 00 00       	mov    $0x10e8,%eax
    movl $KUSER_SHARED_SYSCALL, %ecx
77ed61dd:	b9 00 03 fe 7f       	mov    $0x7ffe0300,%ecx
    call *%ecx
77ed61e2:	ff d1                	call   *%ecx
    ret $0x8
77ed61e4:	c2 08 00             	ret    $0x8

77ed61e7 <_NtGdiSetMapperFlags@8>:

.global _NtGdiSetMapperFlags@8
_NtGdiSetMapperFlags@8:

    movl $0x10e9, %eax
77ed61e7:	b8 e9 10 00 00       	mov    $0x10e9,%eax
    movl $KUSER_SHARED_SYSCALL, %ecx
77ed61ec:	b9 00 03 fe 7f       	mov    $0x7ffe0300,%ecx
    call *%ecx
77ed61f1:	ff d1                	call   *%ecx
    ret $0x8
77ed61f3:	c2 08 00             	ret    $0x8

77ed61f6 <_NtGdiSetMetaFileBitsEx@8>:

.global _NtGdiSetMetaFileBitsEx@8
_NtGdiSetMetaFileBitsEx@8:

    movl $0x10ea, %eax
77ed61f6:	b8 ea 10 00 00       	mov    $0x10ea,%eax
    movl $KUSER_SHARED_SYSCALL, %ecx
77ed61fb:	b9 00 03 fe 7f       	mov    $0x7ffe0300,%ecx
    call *%ecx
77ed6200:	ff d1                	call   *%ecx
    ret $0x8
77ed6202:	c2 08 00             	ret    $0x8

77ed6205 <_NtGdiSetMetaRgn@4>:

.global _NtGdiSetMetaRgn@4
_NtGdiSetMetaRgn@4:

    movl $0x10eb, %eax
77ed6205:	b8 eb 10 00 00       	mov    $0x10eb,%eax
    movl $KUSER_SHARED_SYSCALL, %ecx
77ed620a:	b9 00 03 fe 7f       	mov    $0x7ffe0300,%ecx
    call *%ecx
77ed620f:	ff d1                	call   *%ecx
    ret $0x4
77ed6211:	c2 04 00             	ret    $0x4

77ed6214 <_NtGdiSetMiterLimit@12>:

.global _NtGdiSetMiterLimit@12
_NtGdiSetMiterLimit@12:

    movl $0x10ec, %eax
77ed6214:	b8 ec 10 00 00       	mov    $0x10ec,%eax
    movl $KUSER_SHARED_SYSCALL, %ecx
77ed6219:	b9 00 03 fe 7f       	mov    $0x7ffe0300,%ecx
    call *%ecx
77ed621e:	ff d1                	call   *%ecx
    ret $0xc
77ed6220:	c2 0c 00             	ret    $0xc

77ed6223 <_NtGdiSetPaletteEntries@16>:

.global _NtGdiSetPaletteEntries@16
_NtGdiSetPaletteEntries@16:

    movl $0x10ed, %eax
77ed6223:	b8 ed 10 00 00       	mov    $0x10ed,%eax
    movl $KUSER_SHARED_SYSCALL, %ecx
77ed6228:	b9 00 03 fe 7f       	mov    $0x7ffe0300,%ecx
    call *%ecx
77ed622d:	ff d1                	call   *%ecx
    ret $0x10
77ed622f:	c2 10 00             	ret    $0x10

77ed6232 <_NtGdiSetPixel@16>:

.global _NtGdiSetPixel@16
_NtGdiSetPixel@16:

    movl $0x10ee, %eax
77ed6232:	b8 ee 10 00 00       	mov    $0x10ee,%eax
    movl $KUSER_SHARED_SYSCALL, %ecx
77ed6237:	b9 00 03 fe 7f       	mov    $0x7ffe0300,%ecx
    call *%ecx
77ed623c:	ff d1                	call   *%ecx
    ret $0x10
77ed623e:	c2 10 00             	ret    $0x10

77ed6241 <_NtGdiSetPixelFormat@12>:

.global _NtGdiSetPixelFormat@12
_NtGdiSetPixelFormat@12:

    movl $0x10ef, %eax
77ed6241:	b8 ef 10 00 00       	mov    $0x10ef,%eax
    movl $KUSER_SHARED_SYSCALL, %ecx
77ed6246:	b9 00 03 fe 7f       	mov    $0x7ffe0300,%ecx
    call *%ecx
77ed624b:	ff d1                	call   *%ecx
    ret $0xc
77ed624d:	c2 0c 00             	ret    $0xc

77ed6250 <_NtGdiSetPixelV@16>:

.global _NtGdiSetPixelV@16
_NtGdiSetPixelV@16:

    movl $0x10f0, %eax
77ed6250:	b8 f0 10 00 00       	mov    $0x10f0,%eax
    movl $KUSER_SHARED_SYSCALL, %ecx
77ed6255:	b9 00 03 fe 7f       	mov    $0x7ffe0300,%ecx
    call *%ecx
77ed625a:	ff d1                	call   *%ecx
    ret $0x10
77ed625c:	c2 10 00             	ret    $0x10

77ed625f <_NtGdiSetPolyFillMode@8>:

.global _NtGdiSetPolyFillMode@8
_NtGdiSetPolyFillMode@8:

    movl $0x10f1, %eax
77ed625f:	b8 f1 10 00 00       	mov    $0x10f1,%eax
    movl $KUSER_SHARED_SYSCALL, %ecx
77ed6264:	b9 00 03 fe 7f       	mov    $0x7ffe0300,%ecx
    call *%ecx
77ed6269:	ff d1                	call   *%ecx
    ret $0x8
77ed626b:	c2 08 00             	ret    $0x8

77ed626e <_NtGdiSetROP2@8>:

.global _NtGdiSetROP2@8
_NtGdiSetROP2@8:

    movl $0x10f2, %eax
77ed626e:	b8 f2 10 00 00       	mov    $0x10f2,%eax
    movl $KUSER_SHARED_SYSCALL, %ecx
77ed6273:	b9 00 03 fe 7f       	mov    $0x7ffe0300,%ecx
    call *%ecx
77ed6278:	ff d1                	call   *%ecx
    ret $0x8
77ed627a:	c2 08 00             	ret    $0x8

77ed627d <_NtGdiSetRectRgn@20>:

.global _NtGdiSetRectRgn@20
_NtGdiSetRectRgn@20:

    movl $0x10f3, %eax
77ed627d:	b8 f3 10 00 00       	mov    $0x10f3,%eax
    movl $KUSER_SHARED_SYSCALL, %ecx
77ed6282:	b9 00 03 fe 7f       	mov    $0x7ffe0300,%ecx
    call *%ecx
77ed6287:	ff d1                	call   *%ecx
    ret $0x14
77ed6289:	c2 14 00             	ret    $0x14

77ed628c <_NtGdiSetStretchBltMode@8>:

.global _NtGdiSetStretchBltMode@8
_NtGdiSetStretchBltMode@8:

    movl $0x10f4, %eax
77ed628c:	b8 f4 10 00 00       	mov    $0x10f4,%eax
    movl $KUSER_SHARED_SYSCALL, %ecx
77ed6291:	b9 00 03 fe 7f       	mov    $0x7ffe0300,%ecx
    call *%ecx
77ed6296:	ff d1                	call   *%ecx
    ret $0x8
77ed6298:	c2 08 00             	ret    $0x8

77ed629b <_NtGdiSetSystemPaletteUse@8>:

.global _NtGdiSetSystemPaletteUse@8
_NtGdiSetSystemPaletteUse@8:

    movl $0x10f5, %eax
77ed629b:	b8 f5 10 00 00       	mov    $0x10f5,%eax
    movl $KUSER_SHARED_SYSCALL, %ecx
77ed62a0:	b9 00 03 fe 7f       	mov    $0x7ffe0300,%ecx
    call *%ecx
77ed62a5:	ff d1                	call   *%ecx
    ret $0x8
77ed62a7:	c2 08 00             	ret    $0x8

77ed62aa <_NtGdiSetTextAlign@8>:

.global _NtGdiSetTextAlign@8
_NtGdiSetTextAlign@8:

    movl $0x10f6, %eax
77ed62aa:	b8 f6 10 00 00       	mov    $0x10f6,%eax
    movl $KUSER_SHARED_SYSCALL, %ecx
77ed62af:	b9 00 03 fe 7f       	mov    $0x7ffe0300,%ecx
    call *%ecx
77ed62b4:	ff d1                	call   *%ecx
    ret $0x8
77ed62b6:	c2 08 00             	ret    $0x8

77ed62b9 <_NtGdiSetTextColor@8>:

.global _NtGdiSetTextColor@8
_NtGdiSetTextColor@8:

    movl $0x10f7, %eax
77ed62b9:	b8 f7 10 00 00       	mov    $0x10f7,%eax
    movl $KUSER_SHARED_SYSCALL, %ecx
77ed62be:	b9 00 03 fe 7f       	mov    $0x7ffe0300,%ecx
    call *%ecx
77ed62c3:	ff d1                	call   *%ecx
    ret $0x8
77ed62c5:	c2 08 00             	ret    $0x8

77ed62c8 <_NtGdiSetTextJustification@12>:

.global _NtGdiSetTextJustification@12
_NtGdiSetTextJustification@12:

    movl $0x10f8, %eax
77ed62c8:	b8 f8 10 00 00       	mov    $0x10f8,%eax
    movl $KUSER_SHARED_SYSCALL, %ecx
77ed62cd:	b9 00 03 fe 7f       	mov    $0x7ffe0300,%ecx
    call *%ecx
77ed62d2:	ff d1                	call   *%ecx
    ret $0xc
77ed62d4:	c2 0c 00             	ret    $0xc

77ed62d7 <_NtGdiSetViewportExtEx@16>:

.global _NtGdiSetViewportExtEx@16
_NtGdiSetViewportExtEx@16:

    movl $0x10f9, %eax
77ed62d7:	b8 f9 10 00 00       	mov    $0x10f9,%eax
    movl $KUSER_SHARED_SYSCALL, %ecx
77ed62dc:	b9 00 03 fe 7f       	mov    $0x7ffe0300,%ecx
    call *%ecx
77ed62e1:	ff d1                	call   *%ecx
    ret $0x10
77ed62e3:	c2 10 00             	ret    $0x10

77ed62e6 <_NtGdiSetViewportOrgEx@16>:

.global _NtGdiSetViewportOrgEx@16
_NtGdiSetViewportOrgEx@16:

    movl $0x10fa, %eax
77ed62e6:	b8 fa 10 00 00       	mov    $0x10fa,%eax
    movl $KUSER_SHARED_SYSCALL, %ecx
77ed62eb:	b9 00 03 fe 7f       	mov    $0x7ffe0300,%ecx
    call *%ecx
77ed62f0:	ff d1                	call   *%ecx
    ret $0x10
77ed62f2:	c2 10 00             	ret    $0x10

77ed62f5 <_NtGdiSetWindowExtEx@16>:

.global _NtGdiSetWindowExtEx@16
_NtGdiSetWindowExtEx@16:

    movl $0x10fb, %eax
77ed62f5:	b8 fb 10 00 00       	mov    $0x10fb,%eax
    movl $KUSER_SHARED_SYSCALL, %ecx
77ed62fa:	b9 00 03 fe 7f       	mov    $0x7ffe0300,%ecx
    call *%ecx
77ed62ff:	ff d1                	call   *%ecx
    ret $0x10
77ed6301:	c2 10 00             	ret    $0x10

77ed6304 <_NtGdiSetWindowOrgEx@16>:

.global _NtGdiSetWindowOrgEx@16
_NtGdiSetWindowOrgEx@16:

    movl $0x10fc, %eax
77ed6304:	b8 fc 10 00 00       	mov    $0x10fc,%eax
    movl $KUSER_SHARED_SYSCALL, %ecx
77ed6309:	b9 00 03 fe 7f       	mov    $0x7ffe0300,%ecx
    call *%ecx
77ed630e:	ff d1                	call   *%ecx
    ret $0x10
77ed6310:	c2 10 00             	ret    $0x10

77ed6313 <_NtGdiSetWorldTransform@8>:

.global _NtGdiSetWorldTransform@8
_NtGdiSetWorldTransform@8:

    movl $0x10fd, %eax
77ed6313:	b8 fd 10 00 00       	mov    $0x10fd,%eax
    movl $KUSER_SHARED_SYSCALL, %ecx
77ed6318:	b9 00 03 fe 7f       	mov    $0x7ffe0300,%ecx
    call *%ecx
77ed631d:	ff d1                	call   *%ecx
    ret $0x8
77ed631f:	c2 08 00             	ret    $0x8

77ed6322 <_NtGdiStartDoc@8>:

.global _NtGdiStartDoc@8
_NtGdiStartDoc@8:

    movl $0x10fe, %eax
77ed6322:	b8 fe 10 00 00       	mov    $0x10fe,%eax
    movl $KUSER_SHARED_SYSCALL, %ecx
77ed6327:	b9 00 03 fe 7f       	mov    $0x7ffe0300,%ecx
    call *%ecx
77ed632c:	ff d1                	call   *%ecx
    ret $0x8
77ed632e:	c2 08 00             	ret    $0x8

77ed6331 <_NtGdiStartPage@4>:

.global _NtGdiStartPage@4
_NtGdiStartPage@4:

    movl $0x10ff, %eax
77ed6331:	b8 ff 10 00 00       	mov    $0x10ff,%eax
    movl $KUSER_SHARED_SYSCALL, %ecx
77ed6336:	b9 00 03 fe 7f       	mov    $0x7ffe0300,%ecx
    call *%ecx
77ed633b:	ff d1                	call   *%ecx
    ret $0x4
77ed633d:	c2 04 00             	ret    $0x4

77ed6340 <_NtGdiStretchBlt@44>:

.global _NtGdiStretchBlt@44
_NtGdiStretchBlt@44:

    movl $0x1100, %eax
77ed6340:	b8 00 11 00 00       	mov    $0x1100,%eax
    movl $KUSER_SHARED_SYSCALL, %ecx
77ed6345:	b9 00 03 fe 7f       	mov    $0x7ffe0300,%ecx
    call *%ecx
77ed634a:	ff d1                	call   *%ecx
    ret $0x2c
77ed634c:	c2 2c 00             	ret    $0x2c

77ed634f <_NtGdiStretchDIBits@52>:

.global _NtGdiStretchDIBits@52
_NtGdiStretchDIBits@52:

    movl $0x1101, %eax
77ed634f:	b8 01 11 00 00       	mov    $0x1101,%eax
    movl $KUSER_SHARED_SYSCALL, %ecx
77ed6354:	b9 00 03 fe 7f       	mov    $0x7ffe0300,%ecx
    call *%ecx
77ed6359:	ff d1                	call   *%ecx
    ret $0x34
77ed635b:	c2 34 00             	ret    $0x34

77ed635e <_NtGdiStrokeAndFillPath@4>:

.global _NtGdiStrokeAndFillPath@4
_NtGdiStrokeAndFillPath@4:

    movl $0x1102, %eax
77ed635e:	b8 02 11 00 00       	mov    $0x1102,%eax
    movl $KUSER_SHARED_SYSCALL, %ecx
77ed6363:	b9 00 03 fe 7f       	mov    $0x7ffe0300,%ecx
    call *%ecx
77ed6368:	ff d1                	call   *%ecx
    ret $0x4
77ed636a:	c2 04 00             	ret    $0x4

77ed636d <_NtGdiStrokePath@4>:

.global _NtGdiStrokePath@4
_NtGdiStrokePath@4:

    movl $0x1103, %eax
77ed636d:	b8 03 11 00 00       	mov    $0x1103,%eax
    movl $KUSER_SHARED_SYSCALL, %ecx
77ed6372:	b9 00 03 fe 7f       	mov    $0x7ffe0300,%ecx
    call *%ecx
77ed6377:	ff d1                	call   *%ecx
    ret $0x4
77ed6379:	c2 04 00             	ret    $0x4

77ed637c <_NtGdiSwapBuffers@4>:

.global _NtGdiSwapBuffers@4
_NtGdiSwapBuffers@4:

    movl $0x1104, %eax
77ed637c:	b8 04 11 00 00       	mov    $0x1104,%eax
    movl $KUSER_SHARED_SYSCALL, %ecx
77ed6381:	b9 00 03 fe 7f       	mov    $0x7ffe0300,%ecx
    call *%ecx
77ed6386:	ff d1                	call   *%ecx
    ret $0x4
77ed6388:	c2 04 00             	ret    $0x4

77ed638b <_NtGdiTextOut@20>:

.global _NtGdiTextOut@20
_NtGdiTextOut@20:

    movl $0x1105, %eax
77ed638b:	b8 05 11 00 00       	mov    $0x1105,%eax
    movl $KUSER_SHARED_SYSCALL, %ecx
77ed6390:	b9 00 03 fe 7f       	mov    $0x7ffe0300,%ecx
    call *%ecx
77ed6395:	ff d1                	call   *%ecx
    ret $0x14
77ed6397:	c2 14 00             	ret    $0x14

77ed639a <_NtGdiTransparentBlt@44>:

.global _NtGdiTransparentBlt@44
_NtGdiTransparentBlt@44:

    movl $0x1106, %eax
77ed639a:	b8 06 11 00 00       	mov    $0x1106,%eax
    movl $KUSER_SHARED_SYSCALL, %ecx
77ed639f:	b9 00 03 fe 7f       	mov    $0x7ffe0300,%ecx
    call *%ecx
77ed63a4:	ff d1                	call   *%ecx
    ret $0x2c
77ed63a6:	c2 2c 00             	ret    $0x2c

77ed63a9 <_NtGdiTranslateCharsetInfo@12>:

.global _NtGdiTranslateCharsetInfo@12
_NtGdiTranslateCharsetInfo@12:

    movl $0x1107, %eax
77ed63a9:	b8 07 11 00 00       	mov    $0x1107,%eax
    movl $KUSER_SHARED_SYSCALL, %ecx
77ed63ae:	b9 00 03 fe 7f       	mov    $0x7ffe0300,%ecx
    call *%ecx
77ed63b3:	ff d1                	call   *%ecx
    ret $0xc
77ed63b5:	c2 0c 00             	ret    $0xc

77ed63b8 <_NtGdiUnrealizeObject@8>:

.global _NtGdiUnrealizeObject@8
_NtGdiUnrealizeObject@8:

    movl $0x1108, %eax
77ed63b8:	b8 08 11 00 00       	mov    $0x1108,%eax
    movl $KUSER_SHARED_SYSCALL, %ecx
77ed63bd:	b9 00 03 fe 7f       	mov    $0x7ffe0300,%ecx
    call *%ecx
77ed63c2:	ff d1                	call   *%ecx
    ret $0x8
77ed63c4:	c2 08 00             	ret    $0x8

77ed63c7 <_NtGdiUpdateColors@4>:

.global _NtGdiUpdateColors@4
_NtGdiUpdateColors@4:

    movl $0x1109, %eax
77ed63c7:	b8 09 11 00 00       	mov    $0x1109,%eax
    movl $KUSER_SHARED_SYSCALL, %ecx
77ed63cc:	b9 00 03 fe 7f       	mov    $0x7ffe0300,%ecx
    call *%ecx
77ed63d1:	ff d1                	call   *%ecx
    ret $0x4
77ed63d3:	c2 04 00             	ret    $0x4

77ed63d6 <_NtGdiUpdateICMRegKey@16>:

.global _NtGdiUpdateICMRegKey@16
_NtGdiUpdateICMRegKey@16:

    movl $0x110a, %eax
77ed63d6:	b8 0a 11 00 00       	mov    $0x110a,%eax
    movl $KUSER_SHARED_SYSCALL, %ecx
77ed63db:	b9 00 03 fe 7f       	mov    $0x7ffe0300,%ecx
    call *%ecx
77ed63e0:	ff d1                	call   *%ecx
    ret $0x10
77ed63e2:	c2 10 00             	ret    $0x10

77ed63e5 <_NtGdiWidenPath@4>:

.global _NtGdiWidenPath@4
_NtGdiWidenPath@4:

    movl $0x110b, %eax
77ed63e5:	b8 0b 11 00 00       	mov    $0x110b,%eax
    movl $KUSER_SHARED_SYSCALL, %ecx
77ed63ea:	b9 00 03 fe 7f       	mov    $0x7ffe0300,%ecx
    call *%ecx
77ed63ef:	ff d1                	call   *%ecx
    ret $0x4
77ed63f1:	c2 04 00             	ret    $0x4

77ed63f4 <_NtUserActivateKeyboardLayout@8>:

.global _NtUserActivateKeyboardLayout@8
_NtUserActivateKeyboardLayout@8:

    movl $0x110c, %eax
77ed63f4:	b8 0c 11 00 00       	mov    $0x110c,%eax
    movl $KUSER_SHARED_SYSCALL, %ecx
77ed63f9:	b9 00 03 fe 7f       	mov    $0x7ffe0300,%ecx
    call *%ecx
77ed63fe:	ff d1                	call   *%ecx
    ret $0x8
77ed6400:	c2 08 00             	ret    $0x8

77ed6403 <_NtUserAlterWindowStyle@12>:

.global _NtUserAlterWindowStyle@12
_NtUserAlterWindowStyle@12:

    movl $0x110d, %eax
77ed6403:	b8 0d 11 00 00       	mov    $0x110d,%eax
    movl $KUSER_SHARED_SYSCALL, %ecx
77ed6408:	b9 00 03 fe 7f       	mov    $0x7ffe0300,%ecx
    call *%ecx
77ed640d:	ff d1                	call   *%ecx
    ret $0xc
77ed640f:	c2 0c 00             	ret    $0xc

77ed6412 <_NtUserAttachThreadInput@12>:

.global _NtUserAttachThreadInput@12
_NtUserAttachThreadInput@12:

    movl $0x110e, %eax
77ed6412:	b8 0e 11 00 00       	mov    $0x110e,%eax
    movl $KUSER_SHARED_SYSCALL, %ecx
77ed6417:	b9 00 03 fe 7f       	mov    $0x7ffe0300,%ecx
    call *%ecx
77ed641c:	ff d1                	call   *%ecx
    ret $0xc
77ed641e:	c2 0c 00             	ret    $0xc

77ed6421 <_NtUserBeginPaint@8>:

.global _NtUserBeginPaint@8
_NtUserBeginPaint@8:

    movl $0x110f, %eax
77ed6421:	b8 0f 11 00 00       	mov    $0x110f,%eax
    movl $KUSER_SHARED_SYSCALL, %ecx
77ed6426:	b9 00 03 fe 7f       	mov    $0x7ffe0300,%ecx
    call *%ecx
77ed642b:	ff d1                	call   *%ecx
    ret $0x8
77ed642d:	c2 08 00             	ret    $0x8

77ed6430 <_NtUserBitBltSysBmp@32>:

.global _NtUserBitBltSysBmp@32
_NtUserBitBltSysBmp@32:

    movl $0x1110, %eax
77ed6430:	b8 10 11 00 00       	mov    $0x1110,%eax
    movl $KUSER_SHARED_SYSCALL, %ecx
77ed6435:	b9 00 03 fe 7f       	mov    $0x7ffe0300,%ecx
    call *%ecx
77ed643a:	ff d1                	call   *%ecx
    ret $0x20
77ed643c:	c2 20 00             	ret    $0x20

77ed643f <_NtUserBlockInput@4>:

.global _NtUserBlockInput@4
_NtUserBlockInput@4:

    movl $0x1111, %eax
77ed643f:	b8 11 11 00 00       	mov    $0x1111,%eax
    movl $KUSER_SHARED_SYSCALL, %ecx
77ed6444:	b9 00 03 fe 7f       	mov    $0x7ffe0300,%ecx
    call *%ecx
77ed6449:	ff d1                	call   *%ecx
    ret $0x4
77ed644b:	c2 04 00             	ret    $0x4

77ed644e <_NtUserBuildHwndList@28>:

.global _NtUserBuildHwndList@28
_NtUserBuildHwndList@28:

    movl $0x1112, %eax
77ed644e:	b8 12 11 00 00       	mov    $0x1112,%eax
    movl $KUSER_SHARED_SYSCALL, %ecx
77ed6453:	b9 00 03 fe 7f       	mov    $0x7ffe0300,%ecx
    call *%ecx
77ed6458:	ff d1                	call   *%ecx
    ret $0x1c
77ed645a:	c2 1c 00             	ret    $0x1c

77ed645d <_NtUserBuildMenuItemList@16>:

.global _NtUserBuildMenuItemList@16
_NtUserBuildMenuItemList@16:

    movl $0x1113, %eax
77ed645d:	b8 13 11 00 00       	mov    $0x1113,%eax
    movl $KUSER_SHARED_SYSCALL, %ecx
77ed6462:	b9 00 03 fe 7f       	mov    $0x7ffe0300,%ecx
    call *%ecx
77ed6467:	ff d1                	call   *%ecx
    ret $0x10
77ed6469:	c2 10 00             	ret    $0x10

77ed646c <_NtUserBuildNameList@16>:

.global _NtUserBuildNameList@16
_NtUserBuildNameList@16:

    movl $0x1114, %eax
77ed646c:	b8 14 11 00 00       	mov    $0x1114,%eax
    movl $KUSER_SHARED_SYSCALL, %ecx
77ed6471:	b9 00 03 fe 7f       	mov    $0x7ffe0300,%ecx
    call *%ecx
77ed6476:	ff d1                	call   *%ecx
    ret $0x10
77ed6478:	c2 10 00             	ret    $0x10

77ed647b <_NtUserBuildPropList@16>:

.global _NtUserBuildPropList@16
_NtUserBuildPropList@16:

    movl $0x1115, %eax
77ed647b:	b8 15 11 00 00       	mov    $0x1115,%eax
    movl $KUSER_SHARED_SYSCALL, %ecx
77ed6480:	b9 00 03 fe 7f       	mov    $0x7ffe0300,%ecx
    call *%ecx
77ed6485:	ff d1                	call   *%ecx
    ret $0x10
77ed6487:	c2 10 00             	ret    $0x10

77ed648a <_NtUserCallHwnd@8>:

.global _NtUserCallHwnd@8
_NtUserCallHwnd@8:

    movl $0x1116, %eax
77ed648a:	b8 16 11 00 00       	mov    $0x1116,%eax
    movl $KUSER_SHARED_SYSCALL, %ecx
77ed648f:	b9 00 03 fe 7f       	mov    $0x7ffe0300,%ecx
    call *%ecx
77ed6494:	ff d1                	call   *%ecx
    ret $0x8
77ed6496:	c2 08 00             	ret    $0x8

77ed6499 <_NtUserCallHwndLock@8>:

.global _NtUserCallHwndLock@8
_NtUserCallHwndLock@8:

    movl $0x1117, %eax
77ed6499:	b8 17 11 00 00       	mov    $0x1117,%eax
    movl $KUSER_SHARED_SYSCALL, %ecx
77ed649e:	b9 00 03 fe 7f       	mov    $0x7ffe0300,%ecx
    call *%ecx
77ed64a3:	ff d1                	call   *%ecx
    ret $0x8
77ed64a5:	c2 08 00             	ret    $0x8

77ed64a8 <_NtUserCallHwndOpt@8>:

.global _NtUserCallHwndOpt@8
_NtUserCallHwndOpt@8:

    movl $0x1118, %eax
77ed64a8:	b8 18 11 00 00       	mov    $0x1118,%eax
    movl $KUSER_SHARED_SYSCALL, %ecx
77ed64ad:	b9 00 03 fe 7f       	mov    $0x7ffe0300,%ecx
    call *%ecx
77ed64b2:	ff d1                	call   *%ecx
    ret $0x8
77ed64b4:	c2 08 00             	ret    $0x8

77ed64b7 <_NtUserCallHwndParam@12>:

.global _NtUserCallHwndParam@12
_NtUserCallHwndParam@12:

    movl $0x1119, %eax
77ed64b7:	b8 19 11 00 00       	mov    $0x1119,%eax
    movl $KUSER_SHARED_SYSCALL, %ecx
77ed64bc:	b9 00 03 fe 7f       	mov    $0x7ffe0300,%ecx
    call *%ecx
77ed64c1:	ff d1                	call   *%ecx
    ret $0xc
77ed64c3:	c2 0c 00             	ret    $0xc

77ed64c6 <_NtUserCallHwndParamLock@12>:

.global _NtUserCallHwndParamLock@12
_NtUserCallHwndParamLock@12:

    movl $0x111a, %eax
77ed64c6:	b8 1a 11 00 00       	mov    $0x111a,%eax
    movl $KUSER_SHARED_SYSCALL, %ecx
77ed64cb:	b9 00 03 fe 7f       	mov    $0x7ffe0300,%ecx
    call *%ecx
77ed64d0:	ff d1                	call   *%ecx
    ret $0xc
77ed64d2:	c2 0c 00             	ret    $0xc

77ed64d5 <_NtUserCallMsgFilter@8>:

.global _NtUserCallMsgFilter@8
_NtUserCallMsgFilter@8:

    movl $0x111b, %eax
77ed64d5:	b8 1b 11 00 00       	mov    $0x111b,%eax
    movl $KUSER_SHARED_SYSCALL, %ecx
77ed64da:	b9 00 03 fe 7f       	mov    $0x7ffe0300,%ecx
    call *%ecx
77ed64df:	ff d1                	call   *%ecx
    ret $0x8
77ed64e1:	c2 08 00             	ret    $0x8

77ed64e4 <_NtUserCallNextHookEx@16>:

.global _NtUserCallNextHookEx@16
_NtUserCallNextHookEx@16:

    movl $0x111c, %eax
77ed64e4:	b8 1c 11 00 00       	mov    $0x111c,%eax
    movl $KUSER_SHARED_SYSCALL, %ecx
77ed64e9:	b9 00 03 fe 7f       	mov    $0x7ffe0300,%ecx
    call *%ecx
77ed64ee:	ff d1                	call   *%ecx
    ret $0x10
77ed64f0:	c2 10 00             	ret    $0x10

77ed64f3 <_NtUserCallNoParam@4>:

.global _NtUserCallNoParam@4
_NtUserCallNoParam@4:

    movl $0x111d, %eax
77ed64f3:	b8 1d 11 00 00       	mov    $0x111d,%eax
    movl $KUSER_SHARED_SYSCALL, %ecx
77ed64f8:	b9 00 03 fe 7f       	mov    $0x7ffe0300,%ecx
    call *%ecx
77ed64fd:	ff d1                	call   *%ecx
    ret $0x4
77ed64ff:	c2 04 00             	ret    $0x4

77ed6502 <_NtUserCallOneParam@8>:

.global _NtUserCallOneParam@8
_NtUserCallOneParam@8:

    movl $0x111e, %eax
77ed6502:	b8 1e 11 00 00       	mov    $0x111e,%eax
    movl $KUSER_SHARED_SYSCALL, %ecx
77ed6507:	b9 00 03 fe 7f       	mov    $0x7ffe0300,%ecx
    call *%ecx
77ed650c:	ff d1                	call   *%ecx
    ret $0x8
77ed650e:	c2 08 00             	ret    $0x8

77ed6511 <_NtUserCallTwoParam@12>:

.global _NtUserCallTwoParam@12
_NtUserCallTwoParam@12:

    movl $0x111f, %eax
77ed6511:	b8 1f 11 00 00       	mov    $0x111f,%eax
    movl $KUSER_SHARED_SYSCALL, %ecx
77ed6516:	b9 00 03 fe 7f       	mov    $0x7ffe0300,%ecx
    call *%ecx
77ed651b:	ff d1                	call   *%ecx
    ret $0xc
77ed651d:	c2 0c 00             	ret    $0xc

77ed6520 <_NtUserChangeClipboardChain@8>:

.global _NtUserChangeClipboardChain@8
_NtUserChangeClipboardChain@8:

    movl $0x1120, %eax
77ed6520:	b8 20 11 00 00       	mov    $0x1120,%eax
    movl $KUSER_SHARED_SYSCALL, %ecx
77ed6525:	b9 00 03 fe 7f       	mov    $0x7ffe0300,%ecx
    call *%ecx
77ed652a:	ff d1                	call   *%ecx
    ret $0x8
77ed652c:	c2 08 00             	ret    $0x8

77ed652f <_NtUserChangeDisplaySettings@20>:

.global _NtUserChangeDisplaySettings@20
_NtUserChangeDisplaySettings@20:

    movl $0x1121, %eax
77ed652f:	b8 21 11 00 00       	mov    $0x1121,%eax
    movl $KUSER_SHARED_SYSCALL, %ecx
77ed6534:	b9 00 03 fe 7f       	mov    $0x7ffe0300,%ecx
    call *%ecx
77ed6539:	ff d1                	call   *%ecx
    ret $0x14
77ed653b:	c2 14 00             	ret    $0x14

77ed653e <_NtUserCheckMenuItem@12>:

.global _NtUserCheckMenuItem@12
_NtUserCheckMenuItem@12:

    movl $0x1122, %eax
77ed653e:	b8 22 11 00 00       	mov    $0x1122,%eax
    movl $KUSER_SHARED_SYSCALL, %ecx
77ed6543:	b9 00 03 fe 7f       	mov    $0x7ffe0300,%ecx
    call *%ecx
77ed6548:	ff d1                	call   *%ecx
    ret $0xc
77ed654a:	c2 0c 00             	ret    $0xc

77ed654d <_NtUserChildWindowFromPointEx@16>:

.global _NtUserChildWindowFromPointEx@16
_NtUserChildWindowFromPointEx@16:

    movl $0x1123, %eax
77ed654d:	b8 23 11 00 00       	mov    $0x1123,%eax
    movl $KUSER_SHARED_SYSCALL, %ecx
77ed6552:	b9 00 03 fe 7f       	mov    $0x7ffe0300,%ecx
    call *%ecx
77ed6557:	ff d1                	call   *%ecx
    ret $0x10
77ed6559:	c2 10 00             	ret    $0x10

77ed655c <_NtUserClipCursor@4>:

.global _NtUserClipCursor@4
_NtUserClipCursor@4:

    movl $0x1124, %eax
77ed655c:	b8 24 11 00 00       	mov    $0x1124,%eax
    movl $KUSER_SHARED_SYSCALL, %ecx
77ed6561:	b9 00 03 fe 7f       	mov    $0x7ffe0300,%ecx
    call *%ecx
77ed6566:	ff d1                	call   *%ecx
    ret $0x4
77ed6568:	c2 04 00             	ret    $0x4

77ed656b <_NtUserCloseClipboard@0>:

.global _NtUserCloseClipboard@0
_NtUserCloseClipboard@0:

    movl $0x1125, %eax
77ed656b:	b8 25 11 00 00       	mov    $0x1125,%eax
    movl $KUSER_SHARED_SYSCALL, %ecx
77ed6570:	b9 00 03 fe 7f       	mov    $0x7ffe0300,%ecx
    call *%ecx
77ed6575:	ff d1                	call   *%ecx
    ret $0x0
77ed6577:	c2 00 00             	ret    $0x0

77ed657a <_NtUserCloseDesktop@4>:

.global _NtUserCloseDesktop@4
_NtUserCloseDesktop@4:

    movl $0x1126, %eax
77ed657a:	b8 26 11 00 00       	mov    $0x1126,%eax
    movl $KUSER_SHARED_SYSCALL, %ecx
77ed657f:	b9 00 03 fe 7f       	mov    $0x7ffe0300,%ecx
    call *%ecx
77ed6584:	ff d1                	call   *%ecx
    ret $0x4
77ed6586:	c2 04 00             	ret    $0x4

77ed6589 <_NtUserCloseWindowStation@4>:

.global _NtUserCloseWindowStation@4
_NtUserCloseWindowStation@4:

    movl $0x1127, %eax
77ed6589:	b8 27 11 00 00       	mov    $0x1127,%eax
    movl $KUSER_SHARED_SYSCALL, %ecx
77ed658e:	b9 00 03 fe 7f       	mov    $0x7ffe0300,%ecx
    call *%ecx
77ed6593:	ff d1                	call   *%ecx
    ret $0x4
77ed6595:	c2 04 00             	ret    $0x4

77ed6598 <_NtUserConvertMemHandle@8>:

.global _NtUserConvertMemHandle@8
_NtUserConvertMemHandle@8:

    movl $0x1128, %eax
77ed6598:	b8 28 11 00 00       	mov    $0x1128,%eax
    movl $KUSER_SHARED_SYSCALL, %ecx
77ed659d:	b9 00 03 fe 7f       	mov    $0x7ffe0300,%ecx
    call *%ecx
77ed65a2:	ff d1                	call   *%ecx
    ret $0x8
77ed65a4:	c2 08 00             	ret    $0x8

77ed65a7 <_NtUserCopyAcceleratorTable@12>:

.global _NtUserCopyAcceleratorTable@12
_NtUserCopyAcceleratorTable@12:

    movl $0x1129, %eax
77ed65a7:	b8 29 11 00 00       	mov    $0x1129,%eax
    movl $KUSER_SHARED_SYSCALL, %ecx
77ed65ac:	b9 00 03 fe 7f       	mov    $0x7ffe0300,%ecx
    call *%ecx
77ed65b1:	ff d1                	call   *%ecx
    ret $0xc
77ed65b3:	c2 0c 00             	ret    $0xc

77ed65b6 <_NtUserCountClipboardFormats@0>:

.global _NtUserCountClipboardFormats@0
_NtUserCountClipboardFormats@0:

    movl $0x112a, %eax
77ed65b6:	b8 2a 11 00 00       	mov    $0x112a,%eax
    movl $KUSER_SHARED_SYSCALL, %ecx
77ed65bb:	b9 00 03 fe 7f       	mov    $0x7ffe0300,%ecx
    call *%ecx
77ed65c0:	ff d1                	call   *%ecx
    ret $0x0
77ed65c2:	c2 00 00             	ret    $0x0

77ed65c5 <_NtUserCreateAcceleratorTable@8>:

.global _NtUserCreateAcceleratorTable@8
_NtUserCreateAcceleratorTable@8:

    movl $0x112b, %eax
77ed65c5:	b8 2b 11 00 00       	mov    $0x112b,%eax
    movl $KUSER_SHARED_SYSCALL, %ecx
77ed65ca:	b9 00 03 fe 7f       	mov    $0x7ffe0300,%ecx
    call *%ecx
77ed65cf:	ff d1                	call   *%ecx
    ret $0x8
77ed65d1:	c2 08 00             	ret    $0x8

77ed65d4 <_NtUserCreateCaret@16>:

.global _NtUserCreateCaret@16
_NtUserCreateCaret@16:

    movl $0x112c, %eax
77ed65d4:	b8 2c 11 00 00       	mov    $0x112c,%eax
    movl $KUSER_SHARED_SYSCALL, %ecx
77ed65d9:	b9 00 03 fe 7f       	mov    $0x7ffe0300,%ecx
    call *%ecx
77ed65de:	ff d1                	call   *%ecx
    ret $0x10
77ed65e0:	c2 10 00             	ret    $0x10

77ed65e3 <_NtUserCreateCursorIconHandle@8>:

.global _NtUserCreateCursorIconHandle@8
_NtUserCreateCursorIconHandle@8:

    movl $0x112d, %eax
77ed65e3:	b8 2d 11 00 00       	mov    $0x112d,%eax
    movl $KUSER_SHARED_SYSCALL, %ecx
77ed65e8:	b9 00 03 fe 7f       	mov    $0x7ffe0300,%ecx
    call *%ecx
77ed65ed:	ff d1                	call   *%ecx
    ret $0x8
77ed65ef:	c2 08 00             	ret    $0x8

77ed65f2 <_NtUserCreateDesktop@20>:

.global _NtUserCreateDesktop@20
_NtUserCreateDesktop@20:

    movl $0x112e, %eax
77ed65f2:	b8 2e 11 00 00       	mov    $0x112e,%eax
    movl $KUSER_SHARED_SYSCALL, %ecx
77ed65f7:	b9 00 03 fe 7f       	mov    $0x7ffe0300,%ecx
    call *%ecx
77ed65fc:	ff d1                	call   *%ecx
    ret $0x14
77ed65fe:	c2 14 00             	ret    $0x14

77ed6601 <_NtUserCreateLocalMemHandle@16>:

.global _NtUserCreateLocalMemHandle@16
_NtUserCreateLocalMemHandle@16:

    movl $0x112f, %eax
77ed6601:	b8 2f 11 00 00       	mov    $0x112f,%eax
    movl $KUSER_SHARED_SYSCALL, %ecx
77ed6606:	b9 00 03 fe 7f       	mov    $0x7ffe0300,%ecx
    call *%ecx
77ed660b:	ff d1                	call   *%ecx
    ret $0x10
77ed660d:	c2 10 00             	ret    $0x10

77ed6610 <_NtUserCreateMenu@4>:

.global _NtUserCreateMenu@4
_NtUserCreateMenu@4:

    movl $0x1130, %eax
77ed6610:	b8 30 11 00 00       	mov    $0x1130,%eax
    movl $KUSER_SHARED_SYSCALL, %ecx
77ed6615:	b9 00 03 fe 7f       	mov    $0x7ffe0300,%ecx
    call *%ecx
77ed661a:	ff d1                	call   *%ecx
    ret $0x4
77ed661c:	c2 04 00             	ret    $0x4

77ed661f <_NtUserCreateWindowEx@56>:

.global _NtUserCreateWindowEx@56
_NtUserCreateWindowEx@56:

    movl $0x1131, %eax
77ed661f:	b8 31 11 00 00       	mov    $0x1131,%eax
    movl $KUSER_SHARED_SYSCALL, %ecx
77ed6624:	b9 00 03 fe 7f       	mov    $0x7ffe0300,%ecx
    call *%ecx
77ed6629:	ff d1                	call   *%ecx
    ret $0x38
77ed662b:	c2 38 00             	ret    $0x38

77ed662e <_NtUserCreateWindowStation@24>:

.global _NtUserCreateWindowStation@24
_NtUserCreateWindowStation@24:

    movl $0x1132, %eax
77ed662e:	b8 32 11 00 00       	mov    $0x1132,%eax
    movl $KUSER_SHARED_SYSCALL, %ecx
77ed6633:	b9 00 03 fe 7f       	mov    $0x7ffe0300,%ecx
    call *%ecx
77ed6638:	ff d1                	call   *%ecx
    ret $0x18
77ed663a:	c2 18 00             	ret    $0x18

77ed663d <_NtUserDdeGetQualityOfService@12>:

.global _NtUserDdeGetQualityOfService@12
_NtUserDdeGetQualityOfService@12:

    movl $0x1133, %eax
77ed663d:	b8 33 11 00 00       	mov    $0x1133,%eax
    movl $KUSER_SHARED_SYSCALL, %ecx
77ed6642:	b9 00 03 fe 7f       	mov    $0x7ffe0300,%ecx
    call *%ecx
77ed6647:	ff d1                	call   *%ecx
    ret $0xc
77ed6649:	c2 0c 00             	ret    $0xc

77ed664c <_NtUserDdeInitialize@20>:

.global _NtUserDdeInitialize@20
_NtUserDdeInitialize@20:

    movl $0x1134, %eax
77ed664c:	b8 34 11 00 00       	mov    $0x1134,%eax
    movl $KUSER_SHARED_SYSCALL, %ecx
77ed6651:	b9 00 03 fe 7f       	mov    $0x7ffe0300,%ecx
    call *%ecx
77ed6656:	ff d1                	call   *%ecx
    ret $0x14
77ed6658:	c2 14 00             	ret    $0x14

77ed665b <_NtUserDdeSetQualityOfService@12>:

.global _NtUserDdeSetQualityOfService@12
_NtUserDdeSetQualityOfService@12:

    movl $0x1135, %eax
77ed665b:	b8 35 11 00 00       	mov    $0x1135,%eax
    movl $KUSER_SHARED_SYSCALL, %ecx
77ed6660:	b9 00 03 fe 7f       	mov    $0x7ffe0300,%ecx
    call *%ecx
77ed6665:	ff d1                	call   *%ecx
    ret $0xc
77ed6667:	c2 0c 00             	ret    $0xc

77ed666a <_NtUserDeferWindowPos@32>:

.global _NtUserDeferWindowPos@32
_NtUserDeferWindowPos@32:

    movl $0x1136, %eax
77ed666a:	b8 36 11 00 00       	mov    $0x1136,%eax
    movl $KUSER_SHARED_SYSCALL, %ecx
77ed666f:	b9 00 03 fe 7f       	mov    $0x7ffe0300,%ecx
    call *%ecx
77ed6674:	ff d1                	call   *%ecx
    ret $0x20
77ed6676:	c2 20 00             	ret    $0x20

77ed6679 <_NtUserDefSetText@8>:

.global _NtUserDefSetText@8
_NtUserDefSetText@8:

    movl $0x1137, %eax
77ed6679:	b8 37 11 00 00       	mov    $0x1137,%eax
    movl $KUSER_SHARED_SYSCALL, %ecx
77ed667e:	b9 00 03 fe 7f       	mov    $0x7ffe0300,%ecx
    call *%ecx
77ed6683:	ff d1                	call   *%ecx
    ret $0x8
77ed6685:	c2 08 00             	ret    $0x8

77ed6688 <_NtUserDeleteMenu@12>:

.global _NtUserDeleteMenu@12
_NtUserDeleteMenu@12:

    movl $0x1138, %eax
77ed6688:	b8 38 11 00 00       	mov    $0x1138,%eax
    movl $KUSER_SHARED_SYSCALL, %ecx
77ed668d:	b9 00 03 fe 7f       	mov    $0x7ffe0300,%ecx
    call *%ecx
77ed6692:	ff d1                	call   *%ecx
    ret $0xc
77ed6694:	c2 0c 00             	ret    $0xc

77ed6697 <_NtUserDestroyAcceleratorTable@4>:

.global _NtUserDestroyAcceleratorTable@4
_NtUserDestroyAcceleratorTable@4:

    movl $0x1139, %eax
77ed6697:	b8 39 11 00 00       	mov    $0x1139,%eax
    movl $KUSER_SHARED_SYSCALL, %ecx
77ed669c:	b9 00 03 fe 7f       	mov    $0x7ffe0300,%ecx
    call *%ecx
77ed66a1:	ff d1                	call   *%ecx
    ret $0x4
77ed66a3:	c2 04 00             	ret    $0x4

77ed66a6 <_NtUserDestroyCursorIcon@8>:

.global _NtUserDestroyCursorIcon@8
_NtUserDestroyCursorIcon@8:

    movl $0x113a, %eax
77ed66a6:	b8 3a 11 00 00       	mov    $0x113a,%eax
    movl $KUSER_SHARED_SYSCALL, %ecx
77ed66ab:	b9 00 03 fe 7f       	mov    $0x7ffe0300,%ecx
    call *%ecx
77ed66b0:	ff d1                	call   *%ecx
    ret $0x8
77ed66b2:	c2 08 00             	ret    $0x8

77ed66b5 <_NtUserDestroyMenu@4>:

.global _NtUserDestroyMenu@4
_NtUserDestroyMenu@4:

    movl $0x113b, %eax
77ed66b5:	b8 3b 11 00 00       	mov    $0x113b,%eax
    movl $KUSER_SHARED_SYSCALL, %ecx
77ed66ba:	b9 00 03 fe 7f       	mov    $0x7ffe0300,%ecx
    call *%ecx
77ed66bf:	ff d1                	call   *%ecx
    ret $0x4
77ed66c1:	c2 04 00             	ret    $0x4

77ed66c4 <_NtUserDestroyWindow@4>:

.global _NtUserDestroyWindow@4
_NtUserDestroyWindow@4:

    movl $0x113c, %eax
77ed66c4:	b8 3c 11 00 00       	mov    $0x113c,%eax
    movl $KUSER_SHARED_SYSCALL, %ecx
77ed66c9:	b9 00 03 fe 7f       	mov    $0x7ffe0300,%ecx
    call *%ecx
77ed66ce:	ff d1                	call   *%ecx
    ret $0x4
77ed66d0:	c2 04 00             	ret    $0x4

77ed66d3 <_NtUserDispatchMessage@4>:

.global _NtUserDispatchMessage@4
_NtUserDispatchMessage@4:

    movl $0x113d, %eax
77ed66d3:	b8 3d 11 00 00       	mov    $0x113d,%eax
    movl $KUSER_SHARED_SYSCALL, %ecx
77ed66d8:	b9 00 03 fe 7f       	mov    $0x7ffe0300,%ecx
    call *%ecx
77ed66dd:	ff d1                	call   *%ecx
    ret $0x4
77ed66df:	c2 04 00             	ret    $0x4

77ed66e2 <_NtUserDragDetect@12>:

.global _NtUserDragDetect@12
_NtUserDragDetect@12:

    movl $0x113e, %eax
77ed66e2:	b8 3e 11 00 00       	mov    $0x113e,%eax
    movl $KUSER_SHARED_SYSCALL, %ecx
77ed66e7:	b9 00 03 fe 7f       	mov    $0x7ffe0300,%ecx
    call *%ecx
77ed66ec:	ff d1                	call   *%ecx
    ret $0xc
77ed66ee:	c2 0c 00             	ret    $0xc

77ed66f1 <_NtUserDragObject@20>:

.global _NtUserDragObject@20
_NtUserDragObject@20:

    movl $0x113f, %eax
77ed66f1:	b8 3f 11 00 00       	mov    $0x113f,%eax
    movl $KUSER_SHARED_SYSCALL, %ecx
77ed66f6:	b9 00 03 fe 7f       	mov    $0x7ffe0300,%ecx
    call *%ecx
77ed66fb:	ff d1                	call   *%ecx
    ret $0x14
77ed66fd:	c2 14 00             	ret    $0x14

77ed6700 <_NtUserDrawAnimatedRects@16>:

.global _NtUserDrawAnimatedRects@16
_NtUserDrawAnimatedRects@16:

    movl $0x1140, %eax
77ed6700:	b8 40 11 00 00       	mov    $0x1140,%eax
    movl $KUSER_SHARED_SYSCALL, %ecx
77ed6705:	b9 00 03 fe 7f       	mov    $0x7ffe0300,%ecx
    call *%ecx
77ed670a:	ff d1                	call   *%ecx
    ret $0x10
77ed670c:	c2 10 00             	ret    $0x10

77ed670f <_NtUserDrawCaption@16>:

.global _NtUserDrawCaption@16
_NtUserDrawCaption@16:

    movl $0x1141, %eax
77ed670f:	b8 41 11 00 00       	mov    $0x1141,%eax
    movl $KUSER_SHARED_SYSCALL, %ecx
77ed6714:	b9 00 03 fe 7f       	mov    $0x7ffe0300,%ecx
    call *%ecx
77ed6719:	ff d1                	call   *%ecx
    ret $0x10
77ed671b:	c2 10 00             	ret    $0x10

77ed671e <_NtUserDrawCaptionTemp@28>:

.global _NtUserDrawCaptionTemp@28
_NtUserDrawCaptionTemp@28:

    movl $0x1142, %eax
77ed671e:	b8 42 11 00 00       	mov    $0x1142,%eax
    movl $KUSER_SHARED_SYSCALL, %ecx
77ed6723:	b9 00 03 fe 7f       	mov    $0x7ffe0300,%ecx
    call *%ecx
77ed6728:	ff d1                	call   *%ecx
    ret $0x1c
77ed672a:	c2 1c 00             	ret    $0x1c

77ed672d <_NtUserDrawIconEx@44>:

.global _NtUserDrawIconEx@44
_NtUserDrawIconEx@44:

    movl $0x1143, %eax
77ed672d:	b8 43 11 00 00       	mov    $0x1143,%eax
    movl $KUSER_SHARED_SYSCALL, %ecx
77ed6732:	b9 00 03 fe 7f       	mov    $0x7ffe0300,%ecx
    call *%ecx
77ed6737:	ff d1                	call   *%ecx
    ret $0x2c
77ed6739:	c2 2c 00             	ret    $0x2c

77ed673c <_NtUserDrawMenuBarTemp@20>:

.global _NtUserDrawMenuBarTemp@20
_NtUserDrawMenuBarTemp@20:

    movl $0x1144, %eax
77ed673c:	b8 44 11 00 00       	mov    $0x1144,%eax
    movl $KUSER_SHARED_SYSCALL, %ecx
77ed6741:	b9 00 03 fe 7f       	mov    $0x7ffe0300,%ecx
    call *%ecx
77ed6746:	ff d1                	call   *%ecx
    ret $0x14
77ed6748:	c2 14 00             	ret    $0x14

77ed674b <_NtUserEmptyClipboard@0>:

.global _NtUserEmptyClipboard@0
_NtUserEmptyClipboard@0:

    movl $0x1145, %eax
77ed674b:	b8 45 11 00 00       	mov    $0x1145,%eax
    movl $KUSER_SHARED_SYSCALL, %ecx
77ed6750:	b9 00 03 fe 7f       	mov    $0x7ffe0300,%ecx
    call *%ecx
77ed6755:	ff d1                	call   *%ecx
    ret $0x0
77ed6757:	c2 00 00             	ret    $0x0

77ed675a <_NtUserEnableMenuItem@12>:

.global _NtUserEnableMenuItem@12
_NtUserEnableMenuItem@12:

    movl $0x1146, %eax
77ed675a:	b8 46 11 00 00       	mov    $0x1146,%eax
    movl $KUSER_SHARED_SYSCALL, %ecx
77ed675f:	b9 00 03 fe 7f       	mov    $0x7ffe0300,%ecx
    call *%ecx
77ed6764:	ff d1                	call   *%ecx
    ret $0xc
77ed6766:	c2 0c 00             	ret    $0xc

77ed6769 <_NtUserEnableScrollBar@12>:

.global _NtUserEnableScrollBar@12
_NtUserEnableScrollBar@12:

    movl $0x1147, %eax
77ed6769:	b8 47 11 00 00       	mov    $0x1147,%eax
    movl $KUSER_SHARED_SYSCALL, %ecx
77ed676e:	b9 00 03 fe 7f       	mov    $0x7ffe0300,%ecx
    call *%ecx
77ed6773:	ff d1                	call   *%ecx
    ret $0xc
77ed6775:	c2 0c 00             	ret    $0xc

77ed6778 <_NtUserEndDeferWindowPosEx@8>:

.global _NtUserEndDeferWindowPosEx@8
_NtUserEndDeferWindowPosEx@8:

    movl $0x1148, %eax
77ed6778:	b8 48 11 00 00       	mov    $0x1148,%eax
    movl $KUSER_SHARED_SYSCALL, %ecx
77ed677d:	b9 00 03 fe 7f       	mov    $0x7ffe0300,%ecx
    call *%ecx
77ed6782:	ff d1                	call   *%ecx
    ret $0x8
77ed6784:	c2 08 00             	ret    $0x8

77ed6787 <_NtUserEndMenu@0>:

.global _NtUserEndMenu@0
_NtUserEndMenu@0:

    movl $0x1149, %eax
77ed6787:	b8 49 11 00 00       	mov    $0x1149,%eax
    movl $KUSER_SHARED_SYSCALL, %ecx
77ed678c:	b9 00 03 fe 7f       	mov    $0x7ffe0300,%ecx
    call *%ecx
77ed6791:	ff d1                	call   *%ecx
    ret $0x0
77ed6793:	c2 00 00             	ret    $0x0

77ed6796 <_NtUserEndPaint@8>:

.global _NtUserEndPaint@8
_NtUserEndPaint@8:

    movl $0x114a, %eax
77ed6796:	b8 4a 11 00 00       	mov    $0x114a,%eax
    movl $KUSER_SHARED_SYSCALL, %ecx
77ed679b:	b9 00 03 fe 7f       	mov    $0x7ffe0300,%ecx
    call *%ecx
77ed67a0:	ff d1                	call   *%ecx
    ret $0x8
77ed67a2:	c2 08 00             	ret    $0x8

77ed67a5 <_NtUserEnumDisplayDevices@16>:

.global _NtUserEnumDisplayDevices@16
_NtUserEnumDisplayDevices@16:

    movl $0x114b, %eax
77ed67a5:	b8 4b 11 00 00       	mov    $0x114b,%eax
    movl $KUSER_SHARED_SYSCALL, %ecx
77ed67aa:	b9 00 03 fe 7f       	mov    $0x7ffe0300,%ecx
    call *%ecx
77ed67af:	ff d1                	call   *%ecx
    ret $0x10
77ed67b1:	c2 10 00             	ret    $0x10

77ed67b4 <_NtUserEnumDisplayMonitors@20>:

.global _NtUserEnumDisplayMonitors@20
_NtUserEnumDisplayMonitors@20:

    movl $0x114c, %eax
77ed67b4:	b8 4c 11 00 00       	mov    $0x114c,%eax
    movl $KUSER_SHARED_SYSCALL, %ecx
77ed67b9:	b9 00 03 fe 7f       	mov    $0x7ffe0300,%ecx
    call *%ecx
77ed67be:	ff d1                	call   *%ecx
    ret $0x14
77ed67c0:	c2 14 00             	ret    $0x14

77ed67c3 <_NtUserEnumDisplaySettings@16>:

.global _NtUserEnumDisplaySettings@16
_NtUserEnumDisplaySettings@16:

    movl $0x114d, %eax
77ed67c3:	b8 4d 11 00 00       	mov    $0x114d,%eax
    movl $KUSER_SHARED_SYSCALL, %ecx
77ed67c8:	b9 00 03 fe 7f       	mov    $0x7ffe0300,%ecx
    call *%ecx
77ed67cd:	ff d1                	call   *%ecx
    ret $0x10
77ed67cf:	c2 10 00             	ret    $0x10

77ed67d2 <_NtUserEvent@4>:

.global _NtUserEvent@4
_NtUserEvent@4:

    movl $0x114e, %eax
77ed67d2:	b8 4e 11 00 00       	mov    $0x114e,%eax
    movl $KUSER_SHARED_SYSCALL, %ecx
77ed67d7:	b9 00 03 fe 7f       	mov    $0x7ffe0300,%ecx
    call *%ecx
77ed67dc:	ff d1                	call   *%ecx
    ret $0x4
77ed67de:	c2 04 00             	ret    $0x4

77ed67e1 <_NtUserExcludeUpdateRgn@8>:

.global _NtUserExcludeUpdateRgn@8
_NtUserExcludeUpdateRgn@8:

    movl $0x114f, %eax
77ed67e1:	b8 4f 11 00 00       	mov    $0x114f,%eax
    movl $KUSER_SHARED_SYSCALL, %ecx
77ed67e6:	b9 00 03 fe 7f       	mov    $0x7ffe0300,%ecx
    call *%ecx
77ed67eb:	ff d1                	call   *%ecx
    ret $0x8
77ed67ed:	c2 08 00             	ret    $0x8

77ed67f0 <_NtUserFillWindow@16>:

.global _NtUserFillWindow@16
_NtUserFillWindow@16:

    movl $0x1150, %eax
77ed67f0:	b8 50 11 00 00       	mov    $0x1150,%eax
    movl $KUSER_SHARED_SYSCALL, %ecx
77ed67f5:	b9 00 03 fe 7f       	mov    $0x7ffe0300,%ecx
    call *%ecx
77ed67fa:	ff d1                	call   *%ecx
    ret $0x10
77ed67fc:	c2 10 00             	ret    $0x10

77ed67ff <_NtUserFindExistingCursorIcon@16>:

.global _NtUserFindExistingCursorIcon@16
_NtUserFindExistingCursorIcon@16:

    movl $0x1151, %eax
77ed67ff:	b8 51 11 00 00       	mov    $0x1151,%eax
    movl $KUSER_SHARED_SYSCALL, %ecx
77ed6804:	b9 00 03 fe 7f       	mov    $0x7ffe0300,%ecx
    call *%ecx
77ed6809:	ff d1                	call   *%ecx
    ret $0x10
77ed680b:	c2 10 00             	ret    $0x10

77ed680e <_NtUserFindWindowEx@16>:

.global _NtUserFindWindowEx@16
_NtUserFindWindowEx@16:

    movl $0x1152, %eax
77ed680e:	b8 52 11 00 00       	mov    $0x1152,%eax
    movl $KUSER_SHARED_SYSCALL, %ecx
77ed6813:	b9 00 03 fe 7f       	mov    $0x7ffe0300,%ecx
    call *%ecx
77ed6818:	ff d1                	call   *%ecx
    ret $0x10
77ed681a:	c2 10 00             	ret    $0x10

77ed681d <_NtUserFlashWindowEx@4>:

.global _NtUserFlashWindowEx@4
_NtUserFlashWindowEx@4:

    movl $0x1153, %eax
77ed681d:	b8 53 11 00 00       	mov    $0x1153,%eax
    movl $KUSER_SHARED_SYSCALL, %ecx
77ed6822:	b9 00 03 fe 7f       	mov    $0x7ffe0300,%ecx
    call *%ecx
77ed6827:	ff d1                	call   *%ecx
    ret $0x4
77ed6829:	c2 04 00             	ret    $0x4

77ed682c <_NtUserGetActiveWindow@0>:

.global _NtUserGetActiveWindow@0
_NtUserGetActiveWindow@0:

    movl $0x1154, %eax
77ed682c:	b8 54 11 00 00       	mov    $0x1154,%eax
    movl $KUSER_SHARED_SYSCALL, %ecx
77ed6831:	b9 00 03 fe 7f       	mov    $0x7ffe0300,%ecx
    call *%ecx
77ed6836:	ff d1                	call   *%ecx
    ret $0x0
77ed6838:	c2 00 00             	ret    $0x0

77ed683b <_NtUserGetAltTabInfo@24>:

.global _NtUserGetAltTabInfo@24
_NtUserGetAltTabInfo@24:

    movl $0x1155, %eax
77ed683b:	b8 55 11 00 00       	mov    $0x1155,%eax
    movl $KUSER_SHARED_SYSCALL, %ecx
77ed6840:	b9 00 03 fe 7f       	mov    $0x7ffe0300,%ecx
    call *%ecx
77ed6845:	ff d1                	call   *%ecx
    ret $0x18
77ed6847:	c2 18 00             	ret    $0x18

77ed684a <_NtUserGetAncestor@8>:

.global _NtUserGetAncestor@8
_NtUserGetAncestor@8:

    movl $0x1156, %eax
77ed684a:	b8 56 11 00 00       	mov    $0x1156,%eax
    movl $KUSER_SHARED_SYSCALL, %ecx
77ed684f:	b9 00 03 fe 7f       	mov    $0x7ffe0300,%ecx
    call *%ecx
77ed6854:	ff d1                	call   *%ecx
    ret $0x8
77ed6856:	c2 08 00             	ret    $0x8

77ed6859 <_NtUserGetAsyncKeyState@4>:

.global _NtUserGetAsyncKeyState@4
_NtUserGetAsyncKeyState@4:

    movl $0x1157, %eax
77ed6859:	b8 57 11 00 00       	mov    $0x1157,%eax
    movl $KUSER_SHARED_SYSCALL, %ecx
77ed685e:	b9 00 03 fe 7f       	mov    $0x7ffe0300,%ecx
    call *%ecx
77ed6863:	ff d1                	call   *%ecx
    ret $0x4
77ed6865:	c2 04 00             	ret    $0x4

77ed6868 <_NtUserGetCapture@0>:

.global _NtUserGetCapture@0
_NtUserGetCapture@0:

    movl $0x1158, %eax
77ed6868:	b8 58 11 00 00       	mov    $0x1158,%eax
    movl $KUSER_SHARED_SYSCALL, %ecx
77ed686d:	b9 00 03 fe 7f       	mov    $0x7ffe0300,%ecx
    call *%ecx
77ed6872:	ff d1                	call   *%ecx
    ret $0x0
77ed6874:	c2 00 00             	ret    $0x0

77ed6877 <_NtUserGetCaretBlinkTime@0>:

.global _NtUserGetCaretBlinkTime@0
_NtUserGetCaretBlinkTime@0:

    movl $0x1159, %eax
77ed6877:	b8 59 11 00 00       	mov    $0x1159,%eax
    movl $KUSER_SHARED_SYSCALL, %ecx
77ed687c:	b9 00 03 fe 7f       	mov    $0x7ffe0300,%ecx
    call *%ecx
77ed6881:	ff d1                	call   *%ecx
    ret $0x0
77ed6883:	c2 00 00             	ret    $0x0

77ed6886 <_NtUserGetCaretPos@4>:

.global _NtUserGetCaretPos@4
_NtUserGetCaretPos@4:

    movl $0x115a, %eax
77ed6886:	b8 5a 11 00 00       	mov    $0x115a,%eax
    movl $KUSER_SHARED_SYSCALL, %ecx
77ed688b:	b9 00 03 fe 7f       	mov    $0x7ffe0300,%ecx
    call *%ecx
77ed6890:	ff d1                	call   *%ecx
    ret $0x4
77ed6892:	c2 04 00             	ret    $0x4

77ed6895 <_NtUserGetClassInfo@20>:

.global _NtUserGetClassInfo@20
_NtUserGetClassInfo@20:

    movl $0x115b, %eax
77ed6895:	b8 5b 11 00 00       	mov    $0x115b,%eax
    movl $KUSER_SHARED_SYSCALL, %ecx
77ed689a:	b9 00 03 fe 7f       	mov    $0x7ffe0300,%ecx
    call *%ecx
77ed689f:	ff d1                	call   *%ecx
    ret $0x14
77ed68a1:	c2 14 00             	ret    $0x14

77ed68a4 <_NtUserGetClassLong@12>:

.global _NtUserGetClassLong@12
_NtUserGetClassLong@12:

    movl $0x115c, %eax
77ed68a4:	b8 5c 11 00 00       	mov    $0x115c,%eax
    movl $KUSER_SHARED_SYSCALL, %ecx
77ed68a9:	b9 00 03 fe 7f       	mov    $0x7ffe0300,%ecx
    call *%ecx
77ed68ae:	ff d1                	call   *%ecx
    ret $0xc
77ed68b0:	c2 0c 00             	ret    $0xc

77ed68b3 <_NtUserGetClassName@12>:

.global _NtUserGetClassName@12
_NtUserGetClassName@12:

    movl $0x115d, %eax
77ed68b3:	b8 5d 11 00 00       	mov    $0x115d,%eax
    movl $KUSER_SHARED_SYSCALL, %ecx
77ed68b8:	b9 00 03 fe 7f       	mov    $0x7ffe0300,%ecx
    call *%ecx
77ed68bd:	ff d1                	call   *%ecx
    ret $0xc
77ed68bf:	c2 0c 00             	ret    $0xc

77ed68c2 <_NtUserGetClientOrigin@8>:

.global _NtUserGetClientOrigin@8
_NtUserGetClientOrigin@8:

    movl $0x115e, %eax
77ed68c2:	b8 5e 11 00 00       	mov    $0x115e,%eax
    movl $KUSER_SHARED_SYSCALL, %ecx
77ed68c7:	b9 00 03 fe 7f       	mov    $0x7ffe0300,%ecx
    call *%ecx
77ed68cc:	ff d1                	call   *%ecx
    ret $0x8
77ed68ce:	c2 08 00             	ret    $0x8

77ed68d1 <_NtUserGetClientRect@8>:

.global _NtUserGetClientRect@8
_NtUserGetClientRect@8:

    movl $0x115f, %eax
77ed68d1:	b8 5f 11 00 00       	mov    $0x115f,%eax
    movl $KUSER_SHARED_SYSCALL, %ecx
77ed68d6:	b9 00 03 fe 7f       	mov    $0x7ffe0300,%ecx
    call *%ecx
77ed68db:	ff d1                	call   *%ecx
    ret $0x8
77ed68dd:	c2 08 00             	ret    $0x8

77ed68e0 <_NtUserGetClipboardData@8>:

.global _NtUserGetClipboardData@8
_NtUserGetClipboardData@8:

    movl $0x1160, %eax
77ed68e0:	b8 60 11 00 00       	mov    $0x1160,%eax
    movl $KUSER_SHARED_SYSCALL, %ecx
77ed68e5:	b9 00 03 fe 7f       	mov    $0x7ffe0300,%ecx
    call *%ecx
77ed68ea:	ff d1                	call   *%ecx
    ret $0x8
77ed68ec:	c2 08 00             	ret    $0x8

77ed68ef <_NtUserGetClipboardFormatName@12>:

.global _NtUserGetClipboardFormatName@12
_NtUserGetClipboardFormatName@12:

    movl $0x1161, %eax
77ed68ef:	b8 61 11 00 00       	mov    $0x1161,%eax
    movl $KUSER_SHARED_SYSCALL, %ecx
77ed68f4:	b9 00 03 fe 7f       	mov    $0x7ffe0300,%ecx
    call *%ecx
77ed68f9:	ff d1                	call   *%ecx
    ret $0xc
77ed68fb:	c2 0c 00             	ret    $0xc

77ed68fe <_NtUserGetClipboardOwner@0>:

.global _NtUserGetClipboardOwner@0
_NtUserGetClipboardOwner@0:

    movl $0x1162, %eax
77ed68fe:	b8 62 11 00 00       	mov    $0x1162,%eax
    movl $KUSER_SHARED_SYSCALL, %ecx
77ed6903:	b9 00 03 fe 7f       	mov    $0x7ffe0300,%ecx
    call *%ecx
77ed6908:	ff d1                	call   *%ecx
    ret $0x0
77ed690a:	c2 00 00             	ret    $0x0

77ed690d <_NtUserGetClipboardSequenceNumber@0>:

.global _NtUserGetClipboardSequenceNumber@0
_NtUserGetClipboardSequenceNumber@0:

    movl $0x1163, %eax
77ed690d:	b8 63 11 00 00       	mov    $0x1163,%eax
    movl $KUSER_SHARED_SYSCALL, %ecx
77ed6912:	b9 00 03 fe 7f       	mov    $0x7ffe0300,%ecx
    call *%ecx
77ed6917:	ff d1                	call   *%ecx
    ret $0x0
77ed6919:	c2 00 00             	ret    $0x0

77ed691c <_NtUserGetClipboardViewer@0>:

.global _NtUserGetClipboardViewer@0
_NtUserGetClipboardViewer@0:

    movl $0x1164, %eax
77ed691c:	b8 64 11 00 00       	mov    $0x1164,%eax
    movl $KUSER_SHARED_SYSCALL, %ecx
77ed6921:	b9 00 03 fe 7f       	mov    $0x7ffe0300,%ecx
    call *%ecx
77ed6926:	ff d1                	call   *%ecx
    ret $0x0
77ed6928:	c2 00 00             	ret    $0x0

77ed692b <_NtUserGetClipCursor@4>:

.global _NtUserGetClipCursor@4
_NtUserGetClipCursor@4:

    movl $0x1165, %eax
77ed692b:	b8 65 11 00 00       	mov    $0x1165,%eax
    movl $KUSER_SHARED_SYSCALL, %ecx
77ed6930:	b9 00 03 fe 7f       	mov    $0x7ffe0300,%ecx
    call *%ecx
77ed6935:	ff d1                	call   *%ecx
    ret $0x4
77ed6937:	c2 04 00             	ret    $0x4

77ed693a <_NtUserGetComboBoxInfo@8>:

.global _NtUserGetComboBoxInfo@8
_NtUserGetComboBoxInfo@8:

    movl $0x1166, %eax
77ed693a:	b8 66 11 00 00       	mov    $0x1166,%eax
    movl $KUSER_SHARED_SYSCALL, %ecx
77ed693f:	b9 00 03 fe 7f       	mov    $0x7ffe0300,%ecx
    call *%ecx
77ed6944:	ff d1                	call   *%ecx
    ret $0x8
77ed6946:	c2 08 00             	ret    $0x8

77ed6949 <_NtUserGetControlBrush@12>:

.global _NtUserGetControlBrush@12
_NtUserGetControlBrush@12:

    movl $0x1167, %eax
77ed6949:	b8 67 11 00 00       	mov    $0x1167,%eax
    movl $KUSER_SHARED_SYSCALL, %ecx
77ed694e:	b9 00 03 fe 7f       	mov    $0x7ffe0300,%ecx
    call *%ecx
77ed6953:	ff d1                	call   *%ecx
    ret $0xc
77ed6955:	c2 0c 00             	ret    $0xc

77ed6958 <_NtUserGetControlColor@16>:

.global _NtUserGetControlColor@16
_NtUserGetControlColor@16:

    movl $0x1168, %eax
77ed6958:	b8 68 11 00 00       	mov    $0x1168,%eax
    movl $KUSER_SHARED_SYSCALL, %ecx
77ed695d:	b9 00 03 fe 7f       	mov    $0x7ffe0300,%ecx
    call *%ecx
77ed6962:	ff d1                	call   *%ecx
    ret $0x10
77ed6964:	c2 10 00             	ret    $0x10

77ed6967 <_NtUserGetCPD@12>:

.global _NtUserGetCPD@12
_NtUserGetCPD@12:

    movl $0x1169, %eax
77ed6967:	b8 69 11 00 00       	mov    $0x1169,%eax
    movl $KUSER_SHARED_SYSCALL, %ecx
77ed696c:	b9 00 03 fe 7f       	mov    $0x7ffe0300,%ecx
    call *%ecx
77ed6971:	ff d1                	call   *%ecx
    ret $0xc
77ed6973:	c2 0c 00             	ret    $0xc

77ed6976 <_NtUserGetCursorFrameInfo@16>:

.global _NtUserGetCursorFrameInfo@16
_NtUserGetCursorFrameInfo@16:

    movl $0x116a, %eax
77ed6976:	b8 6a 11 00 00       	mov    $0x116a,%eax
    movl $KUSER_SHARED_SYSCALL, %ecx
77ed697b:	b9 00 03 fe 7f       	mov    $0x7ffe0300,%ecx
    call *%ecx
77ed6980:	ff d1                	call   *%ecx
    ret $0x10
77ed6982:	c2 10 00             	ret    $0x10

77ed6985 <_NtUserGetCursorInfo@4>:

.global _NtUserGetCursorInfo@4
_NtUserGetCursorInfo@4:

    movl $0x116b, %eax
77ed6985:	b8 6b 11 00 00       	mov    $0x116b,%eax
    movl $KUSER_SHARED_SYSCALL, %ecx
77ed698a:	b9 00 03 fe 7f       	mov    $0x7ffe0300,%ecx
    call *%ecx
77ed698f:	ff d1                	call   *%ecx
    ret $0x4
77ed6991:	c2 04 00             	ret    $0x4

77ed6994 <_NtUserGetDC@4>:

.global _NtUserGetDC@4
_NtUserGetDC@4:

    movl $0x116c, %eax
77ed6994:	b8 6c 11 00 00       	mov    $0x116c,%eax
    movl $KUSER_SHARED_SYSCALL, %ecx
77ed6999:	b9 00 03 fe 7f       	mov    $0x7ffe0300,%ecx
    call *%ecx
77ed699e:	ff d1                	call   *%ecx
    ret $0x4
77ed69a0:	c2 04 00             	ret    $0x4

77ed69a3 <_NtUserGetDCEx@12>:

.global _NtUserGetDCEx@12
_NtUserGetDCEx@12:

    movl $0x116d, %eax
77ed69a3:	b8 6d 11 00 00       	mov    $0x116d,%eax
    movl $KUSER_SHARED_SYSCALL, %ecx
77ed69a8:	b9 00 03 fe 7f       	mov    $0x7ffe0300,%ecx
    call *%ecx
77ed69ad:	ff d1                	call   *%ecx
    ret $0xc
77ed69af:	c2 0c 00             	ret    $0xc

77ed69b2 <_NtUserGetMenuDefaultItem@12>:

.global _NtUserGetMenuDefaultItem@12
_NtUserGetMenuDefaultItem@12:

    movl $0x116e, %eax
77ed69b2:	b8 6e 11 00 00       	mov    $0x116e,%eax
    movl $KUSER_SHARED_SYSCALL, %ecx
77ed69b7:	b9 00 03 fe 7f       	mov    $0x7ffe0300,%ecx
    call *%ecx
77ed69bc:	ff d1                	call   *%ecx
    ret $0xc
77ed69be:	c2 0c 00             	ret    $0xc

77ed69c1 <_NtUserGetDoubleClickTime@0>:

.global _NtUserGetDoubleClickTime@0
_NtUserGetDoubleClickTime@0:

    movl $0x116f, %eax
77ed69c1:	b8 6f 11 00 00       	mov    $0x116f,%eax
    movl $KUSER_SHARED_SYSCALL, %ecx
77ed69c6:	b9 00 03 fe 7f       	mov    $0x7ffe0300,%ecx
    call *%ecx
77ed69cb:	ff d1                	call   *%ecx
    ret $0x0
77ed69cd:	c2 00 00             	ret    $0x0

77ed69d0 <_NtUserGetForegroundWindow@0>:

.global _NtUserGetForegroundWindow@0
_NtUserGetForegroundWindow@0:

    movl $0x1170, %eax
77ed69d0:	b8 70 11 00 00       	mov    $0x1170,%eax
    movl $KUSER_SHARED_SYSCALL, %ecx
77ed69d5:	b9 00 03 fe 7f       	mov    $0x7ffe0300,%ecx
    call *%ecx
77ed69da:	ff d1                	call   *%ecx
    ret $0x0
77ed69dc:	c2 00 00             	ret    $0x0

77ed69df <_NtUserGetGuiResources@8>:

.global _NtUserGetGuiResources@8
_NtUserGetGuiResources@8:

    movl $0x1171, %eax
77ed69df:	b8 71 11 00 00       	mov    $0x1171,%eax
    movl $KUSER_SHARED_SYSCALL, %ecx
77ed69e4:	b9 00 03 fe 7f       	mov    $0x7ffe0300,%ecx
    call *%ecx
77ed69e9:	ff d1                	call   *%ecx
    ret $0x8
77ed69eb:	c2 08 00             	ret    $0x8

77ed69ee <_NtUserGetGUIThreadInfo@8>:

.global _NtUserGetGUIThreadInfo@8
_NtUserGetGUIThreadInfo@8:

    movl $0x1172, %eax
77ed69ee:	b8 72 11 00 00       	mov    $0x1172,%eax
    movl $KUSER_SHARED_SYSCALL, %ecx
77ed69f3:	b9 00 03 fe 7f       	mov    $0x7ffe0300,%ecx
    call *%ecx
77ed69f8:	ff d1                	call   *%ecx
    ret $0x8
77ed69fa:	c2 08 00             	ret    $0x8

77ed69fd <_NtUserGetCursorIconInfo@8>:

.global _NtUserGetCursorIconInfo@8
_NtUserGetCursorIconInfo@8:

    movl $0x1173, %eax
77ed69fd:	b8 73 11 00 00       	mov    $0x1173,%eax
    movl $KUSER_SHARED_SYSCALL, %ecx
77ed6a02:	b9 00 03 fe 7f       	mov    $0x7ffe0300,%ecx
    call *%ecx
77ed6a07:	ff d1                	call   *%ecx
    ret $0x8
77ed6a09:	c2 08 00             	ret    $0x8

77ed6a0c <_NtUserGetCursorIconSize@12>:

.global _NtUserGetCursorIconSize@12
_NtUserGetCursorIconSize@12:

    movl $0x1174, %eax
77ed6a0c:	b8 74 11 00 00       	mov    $0x1174,%eax
    movl $KUSER_SHARED_SYSCALL, %ecx
77ed6a11:	b9 00 03 fe 7f       	mov    $0x7ffe0300,%ecx
    call *%ecx
77ed6a16:	ff d1                	call   *%ecx
    ret $0xc
77ed6a18:	c2 0c 00             	ret    $0xc

77ed6a1b <_NtUserGetImeHotKey@16>:

.global _NtUserGetImeHotKey@16
_NtUserGetImeHotKey@16:

    movl $0x1175, %eax
77ed6a1b:	b8 75 11 00 00       	mov    $0x1175,%eax
    movl $KUSER_SHARED_SYSCALL, %ecx
77ed6a20:	b9 00 03 fe 7f       	mov    $0x7ffe0300,%ecx
    call *%ecx
77ed6a25:	ff d1                	call   *%ecx
    ret $0x10
77ed6a27:	c2 10 00             	ret    $0x10

77ed6a2a <_NtUserGetInternalWindowPos@12>:

.global _NtUserGetInternalWindowPos@12
_NtUserGetInternalWindowPos@12:

    movl $0x1176, %eax
77ed6a2a:	b8 76 11 00 00       	mov    $0x1176,%eax
    movl $KUSER_SHARED_SYSCALL, %ecx
77ed6a2f:	b9 00 03 fe 7f       	mov    $0x7ffe0300,%ecx
    call *%ecx
77ed6a34:	ff d1                	call   *%ecx
    ret $0xc
77ed6a36:	c2 0c 00             	ret    $0xc

77ed6a39 <_NtUserGetKeyboardLayoutList@8>:

.global _NtUserGetKeyboardLayoutList@8
_NtUserGetKeyboardLayoutList@8:

    movl $0x1177, %eax
77ed6a39:	b8 77 11 00 00       	mov    $0x1177,%eax
    movl $KUSER_SHARED_SYSCALL, %ecx
77ed6a3e:	b9 00 03 fe 7f       	mov    $0x7ffe0300,%ecx
    call *%ecx
77ed6a43:	ff d1                	call   *%ecx
    ret $0x8
77ed6a45:	c2 08 00             	ret    $0x8

77ed6a48 <_NtUserGetKeyboardLayoutName@4>:

.global _NtUserGetKeyboardLayoutName@4
_NtUserGetKeyboardLayoutName@4:

    movl $0x1178, %eax
77ed6a48:	b8 78 11 00 00       	mov    $0x1178,%eax
    movl $KUSER_SHARED_SYSCALL, %ecx
77ed6a4d:	b9 00 03 fe 7f       	mov    $0x7ffe0300,%ecx
    call *%ecx
77ed6a52:	ff d1                	call   *%ecx
    ret $0x4
77ed6a54:	c2 04 00             	ret    $0x4

77ed6a57 <_NtUserGetKeyboardState@4>:

.global _NtUserGetKeyboardState@4
_NtUserGetKeyboardState@4:

    movl $0x1179, %eax
77ed6a57:	b8 79 11 00 00       	mov    $0x1179,%eax
    movl $KUSER_SHARED_SYSCALL, %ecx
77ed6a5c:	b9 00 03 fe 7f       	mov    $0x7ffe0300,%ecx
    call *%ecx
77ed6a61:	ff d1                	call   *%ecx
    ret $0x4
77ed6a63:	c2 04 00             	ret    $0x4

77ed6a66 <_NtUserGetKeyNameText@12>:

.global _NtUserGetKeyNameText@12
_NtUserGetKeyNameText@12:

    movl $0x117a, %eax
77ed6a66:	b8 7a 11 00 00       	mov    $0x117a,%eax
    movl $KUSER_SHARED_SYSCALL, %ecx
77ed6a6b:	b9 00 03 fe 7f       	mov    $0x7ffe0300,%ecx
    call *%ecx
77ed6a70:	ff d1                	call   *%ecx
    ret $0xc
77ed6a72:	c2 0c 00             	ret    $0xc

77ed6a75 <_NtUserGetKeyState@4>:

.global _NtUserGetKeyState@4
_NtUserGetKeyState@4:

    movl $0x117b, %eax
77ed6a75:	b8 7b 11 00 00       	mov    $0x117b,%eax
    movl $KUSER_SHARED_SYSCALL, %ecx
77ed6a7a:	b9 00 03 fe 7f       	mov    $0x7ffe0300,%ecx
    call *%ecx
77ed6a7f:	ff d1                	call   *%ecx
    ret $0x4
77ed6a81:	c2 04 00             	ret    $0x4

77ed6a84 <_NtUserGetListBoxInfo@4>:

.global _NtUserGetListBoxInfo@4
_NtUserGetListBoxInfo@4:

    movl $0x117c, %eax
77ed6a84:	b8 7c 11 00 00       	mov    $0x117c,%eax
    movl $KUSER_SHARED_SYSCALL, %ecx
77ed6a89:	b9 00 03 fe 7f       	mov    $0x7ffe0300,%ecx
    call *%ecx
77ed6a8e:	ff d1                	call   *%ecx
    ret $0x4
77ed6a90:	c2 04 00             	ret    $0x4

77ed6a93 <_NtUserGetMenuBarInfo@16>:

.global _NtUserGetMenuBarInfo@16
_NtUserGetMenuBarInfo@16:

    movl $0x117d, %eax
77ed6a93:	b8 7d 11 00 00       	mov    $0x117d,%eax
    movl $KUSER_SHARED_SYSCALL, %ecx
77ed6a98:	b9 00 03 fe 7f       	mov    $0x7ffe0300,%ecx
    call *%ecx
77ed6a9d:	ff d1                	call   *%ecx
    ret $0x10
77ed6a9f:	c2 10 00             	ret    $0x10

77ed6aa2 <_NtUserGetMenuIndex@8>:

.global _NtUserGetMenuIndex@8
_NtUserGetMenuIndex@8:

    movl $0x117e, %eax
77ed6aa2:	b8 7e 11 00 00       	mov    $0x117e,%eax
    movl $KUSER_SHARED_SYSCALL, %ecx
77ed6aa7:	b9 00 03 fe 7f       	mov    $0x7ffe0300,%ecx
    call *%ecx
77ed6aac:	ff d1                	call   *%ecx
    ret $0x8
77ed6aae:	c2 08 00             	ret    $0x8

77ed6ab1 <_NtUserGetMenuItemRect@16>:

.global _NtUserGetMenuItemRect@16
_NtUserGetMenuItemRect@16:

    movl $0x117f, %eax
77ed6ab1:	b8 7f 11 00 00       	mov    $0x117f,%eax
    movl $KUSER_SHARED_SYSCALL, %ecx
77ed6ab6:	b9 00 03 fe 7f       	mov    $0x7ffe0300,%ecx
    call *%ecx
77ed6abb:	ff d1                	call   *%ecx
    ret $0x10
77ed6abd:	c2 10 00             	ret    $0x10

77ed6ac0 <_NtUserGetMessage@16>:

.global _NtUserGetMessage@16
_NtUserGetMessage@16:

    movl $0x1180, %eax
77ed6ac0:	b8 80 11 00 00       	mov    $0x1180,%eax
    movl $KUSER_SHARED_SYSCALL, %ecx
77ed6ac5:	b9 00 03 fe 7f       	mov    $0x7ffe0300,%ecx
    call *%ecx
77ed6aca:	ff d1                	call   *%ecx
    ret $0x10
77ed6acc:	c2 10 00             	ret    $0x10

77ed6acf <_NtUserGetMinMaxInfo@12>:

.global _NtUserGetMinMaxInfo@12
_NtUserGetMinMaxInfo@12:

    movl $0x1181, %eax
77ed6acf:	b8 81 11 00 00       	mov    $0x1181,%eax
    movl $KUSER_SHARED_SYSCALL, %ecx
77ed6ad4:	b9 00 03 fe 7f       	mov    $0x7ffe0300,%ecx
    call *%ecx
77ed6ad9:	ff d1                	call   *%ecx
    ret $0xc
77ed6adb:	c2 0c 00             	ret    $0xc

77ed6ade <_NtUserGetMonitorInfo@8>:

.global _NtUserGetMonitorInfo@8
_NtUserGetMonitorInfo@8:

    movl $0x1182, %eax
77ed6ade:	b8 82 11 00 00       	mov    $0x1182,%eax
    movl $KUSER_SHARED_SYSCALL, %ecx
77ed6ae3:	b9 00 03 fe 7f       	mov    $0x7ffe0300,%ecx
    call *%ecx
77ed6ae8:	ff d1                	call   *%ecx
    ret $0x8
77ed6aea:	c2 08 00             	ret    $0x8

77ed6aed <_NtUserGetMouseMovePointsEx@20>:

.global _NtUserGetMouseMovePointsEx@20
_NtUserGetMouseMovePointsEx@20:

    movl $0x1183, %eax
77ed6aed:	b8 83 11 00 00       	mov    $0x1183,%eax
    movl $KUSER_SHARED_SYSCALL, %ecx
77ed6af2:	b9 00 03 fe 7f       	mov    $0x7ffe0300,%ecx
    call *%ecx
77ed6af7:	ff d1                	call   *%ecx
    ret $0x14
77ed6af9:	c2 14 00             	ret    $0x14

77ed6afc <_NtUserGetObjectInformation@20>:

.global _NtUserGetObjectInformation@20
_NtUserGetObjectInformation@20:

    movl $0x1184, %eax
77ed6afc:	b8 84 11 00 00       	mov    $0x1184,%eax
    movl $KUSER_SHARED_SYSCALL, %ecx
77ed6b01:	b9 00 03 fe 7f       	mov    $0x7ffe0300,%ecx
    call *%ecx
77ed6b06:	ff d1                	call   *%ecx
    ret $0x14
77ed6b08:	c2 14 00             	ret    $0x14

77ed6b0b <_NtUserGetOpenClipboardWindow@0>:

.global _NtUserGetOpenClipboardWindow@0
_NtUserGetOpenClipboardWindow@0:

    movl $0x1185, %eax
77ed6b0b:	b8 85 11 00 00       	mov    $0x1185,%eax
    movl $KUSER_SHARED_SYSCALL, %ecx
77ed6b10:	b9 00 03 fe 7f       	mov    $0x7ffe0300,%ecx
    call *%ecx
77ed6b15:	ff d1                	call   *%ecx
    ret $0x0
77ed6b17:	c2 00 00             	ret    $0x0

77ed6b1a <_NtUserGetProp@8>:

.global _NtUserGetProp@8
_NtUserGetProp@8:

    movl $0x1186, %eax
77ed6b1a:	b8 86 11 00 00       	mov    $0x1186,%eax
    movl $KUSER_SHARED_SYSCALL, %ecx
77ed6b1f:	b9 00 03 fe 7f       	mov    $0x7ffe0300,%ecx
    call *%ecx
77ed6b24:	ff d1                	call   *%ecx
    ret $0x8
77ed6b26:	c2 08 00             	ret    $0x8

77ed6b29 <_NtUserGetPriorityClipboardFormat@8>:

.global _NtUserGetPriorityClipboardFormat@8
_NtUserGetPriorityClipboardFormat@8:

    movl $0x1187, %eax
77ed6b29:	b8 87 11 00 00       	mov    $0x1187,%eax
    movl $KUSER_SHARED_SYSCALL, %ecx
77ed6b2e:	b9 00 03 fe 7f       	mov    $0x7ffe0300,%ecx
    call *%ecx
77ed6b33:	ff d1                	call   *%ecx
    ret $0x8
77ed6b35:	c2 08 00             	ret    $0x8

77ed6b38 <_NtUserGetProcessWindowStation@0>:

.global _NtUserGetProcessWindowStation@0
_NtUserGetProcessWindowStation@0:

    movl $0x1188, %eax
77ed6b38:	b8 88 11 00 00       	mov    $0x1188,%eax
    movl $KUSER_SHARED_SYSCALL, %ecx
77ed6b3d:	b9 00 03 fe 7f       	mov    $0x7ffe0300,%ecx
    call *%ecx
77ed6b42:	ff d1                	call   *%ecx
    ret $0x0
77ed6b44:	c2 00 00             	ret    $0x0

77ed6b47 <_NtUserGetScrollBarInfo@12>:

.global _NtUserGetScrollBarInfo@12
_NtUserGetScrollBarInfo@12:

    movl $0x1189, %eax
77ed6b47:	b8 89 11 00 00       	mov    $0x1189,%eax
    movl $KUSER_SHARED_SYSCALL, %ecx
77ed6b4c:	b9 00 03 fe 7f       	mov    $0x7ffe0300,%ecx
    call *%ecx
77ed6b51:	ff d1                	call   *%ecx
    ret $0xc
77ed6b53:	c2 0c 00             	ret    $0xc

77ed6b56 <_NtUserGetScrollInfo@12>:

.global _NtUserGetScrollInfo@12
_NtUserGetScrollInfo@12:

    movl $0x118a, %eax
77ed6b56:	b8 8a 11 00 00       	mov    $0x118a,%eax
    movl $KUSER_SHARED_SYSCALL, %ecx
77ed6b5b:	b9 00 03 fe 7f       	mov    $0x7ffe0300,%ecx
    call *%ecx
77ed6b60:	ff d1                	call   *%ecx
    ret $0xc
77ed6b62:	c2 0c 00             	ret    $0xc

77ed6b65 <_NtUserGetSystemMenu@8>:

.global _NtUserGetSystemMenu@8
_NtUserGetSystemMenu@8:

    movl $0x118b, %eax
77ed6b65:	b8 8b 11 00 00       	mov    $0x118b,%eax
    movl $KUSER_SHARED_SYSCALL, %ecx
77ed6b6a:	b9 00 03 fe 7f       	mov    $0x7ffe0300,%ecx
    call *%ecx
77ed6b6f:	ff d1                	call   *%ecx
    ret $0x8
77ed6b71:	c2 08 00             	ret    $0x8

77ed6b74 <_NtUserGetSystemMetrics@4>:

.global _NtUserGetSystemMetrics@4
_NtUserGetSystemMetrics@4:

    movl $0x118c, %eax
77ed6b74:	b8 8c 11 00 00       	mov    $0x118c,%eax
    movl $KUSER_SHARED_SYSCALL, %ecx
77ed6b79:	b9 00 03 fe 7f       	mov    $0x7ffe0300,%ecx
    call *%ecx
77ed6b7e:	ff d1                	call   *%ecx
    ret $0x4
77ed6b80:	c2 04 00             	ret    $0x4

77ed6b83 <_NtUserGetThreadDesktop@8>:

.global _NtUserGetThreadDesktop@8
_NtUserGetThreadDesktop@8:

    movl $0x118d, %eax
77ed6b83:	b8 8d 11 00 00       	mov    $0x118d,%eax
    movl $KUSER_SHARED_SYSCALL, %ecx
77ed6b88:	b9 00 03 fe 7f       	mov    $0x7ffe0300,%ecx
    call *%ecx
77ed6b8d:	ff d1                	call   *%ecx
    ret $0x8
77ed6b8f:	c2 08 00             	ret    $0x8

77ed6b92 <_NtUserGetThreadState@4>:

.global _NtUserGetThreadState@4
_NtUserGetThreadState@4:

    movl $0x118e, %eax
77ed6b92:	b8 8e 11 00 00       	mov    $0x118e,%eax
    movl $KUSER_SHARED_SYSCALL, %ecx
77ed6b97:	b9 00 03 fe 7f       	mov    $0x7ffe0300,%ecx
    call *%ecx
77ed6b9c:	ff d1                	call   *%ecx
    ret $0x4
77ed6b9e:	c2 04 00             	ret    $0x4

77ed6ba1 <_NtUserGetTitleBarInfo@8>:

.global _NtUserGetTitleBarInfo@8
_NtUserGetTitleBarInfo@8:

    movl $0x118f, %eax
77ed6ba1:	b8 8f 11 00 00       	mov    $0x118f,%eax
    movl $KUSER_SHARED_SYSCALL, %ecx
77ed6ba6:	b9 00 03 fe 7f       	mov    $0x7ffe0300,%ecx
    call *%ecx
77ed6bab:	ff d1                	call   *%ecx
    ret $0x8
77ed6bad:	c2 08 00             	ret    $0x8

77ed6bb0 <_NtUserGetUpdateRect@12>:

.global _NtUserGetUpdateRect@12
_NtUserGetUpdateRect@12:

    movl $0x1190, %eax
77ed6bb0:	b8 90 11 00 00       	mov    $0x1190,%eax
    movl $KUSER_SHARED_SYSCALL, %ecx
77ed6bb5:	b9 00 03 fe 7f       	mov    $0x7ffe0300,%ecx
    call *%ecx
77ed6bba:	ff d1                	call   *%ecx
    ret $0xc
77ed6bbc:	c2 0c 00             	ret    $0xc

77ed6bbf <_NtUserGetUpdateRgn@12>:

.global _NtUserGetUpdateRgn@12
_NtUserGetUpdateRgn@12:

    movl $0x1191, %eax
77ed6bbf:	b8 91 11 00 00       	mov    $0x1191,%eax
    movl $KUSER_SHARED_SYSCALL, %ecx
77ed6bc4:	b9 00 03 fe 7f       	mov    $0x7ffe0300,%ecx
    call *%ecx
77ed6bc9:	ff d1                	call   *%ecx
    ret $0xc
77ed6bcb:	c2 0c 00             	ret    $0xc

77ed6bce <_NtUserGetWindowDC@4>:

.global _NtUserGetWindowDC@4
_NtUserGetWindowDC@4:

    movl $0x1192, %eax
77ed6bce:	b8 92 11 00 00       	mov    $0x1192,%eax
    movl $KUSER_SHARED_SYSCALL, %ecx
77ed6bd3:	b9 00 03 fe 7f       	mov    $0x7ffe0300,%ecx
    call *%ecx
77ed6bd8:	ff d1                	call   *%ecx
    ret $0x4
77ed6bda:	c2 04 00             	ret    $0x4

77ed6bdd <_NtUserGetWindowPlacement@8>:

.global _NtUserGetWindowPlacement@8
_NtUserGetWindowPlacement@8:

    movl $0x1193, %eax
77ed6bdd:	b8 93 11 00 00       	mov    $0x1193,%eax
    movl $KUSER_SHARED_SYSCALL, %ecx
77ed6be2:	b9 00 03 fe 7f       	mov    $0x7ffe0300,%ecx
    call *%ecx
77ed6be7:	ff d1                	call   *%ecx
    ret $0x8
77ed6be9:	c2 08 00             	ret    $0x8

77ed6bec <_NtUserGetWindowLong@12>:

.global _NtUserGetWindowLong@12
_NtUserGetWindowLong@12:

    movl $0x1194, %eax
77ed6bec:	b8 94 11 00 00       	mov    $0x1194,%eax
    movl $KUSER_SHARED_SYSCALL, %ecx
77ed6bf1:	b9 00 03 fe 7f       	mov    $0x7ffe0300,%ecx
    call *%ecx
77ed6bf6:	ff d1                	call   *%ecx
    ret $0xc
77ed6bf8:	c2 0c 00             	ret    $0xc

77ed6bfb <_NtUserGetWindowRect@8>:

.global _NtUserGetWindowRect@8
_NtUserGetWindowRect@8:

    movl $0x1195, %eax
77ed6bfb:	b8 95 11 00 00       	mov    $0x1195,%eax
    movl $KUSER_SHARED_SYSCALL, %ecx
77ed6c00:	b9 00 03 fe 7f       	mov    $0x7ffe0300,%ecx
    call *%ecx
77ed6c05:	ff d1                	call   *%ecx
    ret $0x8
77ed6c07:	c2 08 00             	ret    $0x8

77ed6c0a <_NtUserGetWOWClass@8>:

.global _NtUserGetWOWClass@8
_NtUserGetWOWClass@8:

    movl $0x1196, %eax
77ed6c0a:	b8 96 11 00 00       	mov    $0x1196,%eax
    movl $KUSER_SHARED_SYSCALL, %ecx
77ed6c0f:	b9 00 03 fe 7f       	mov    $0x7ffe0300,%ecx
    call *%ecx
77ed6c14:	ff d1                	call   *%ecx
    ret $0x8
77ed6c16:	c2 08 00             	ret    $0x8

77ed6c19 <_NtUserHideCaret@4>:

.global _NtUserHideCaret@4
_NtUserHideCaret@4:

    movl $0x1197, %eax
77ed6c19:	b8 97 11 00 00       	mov    $0x1197,%eax
    movl $KUSER_SHARED_SYSCALL, %ecx
77ed6c1e:	b9 00 03 fe 7f       	mov    $0x7ffe0300,%ecx
    call *%ecx
77ed6c23:	ff d1                	call   *%ecx
    ret $0x4
77ed6c25:	c2 04 00             	ret    $0x4

77ed6c28 <_NtUserHiliteMenuItem@16>:

.global _NtUserHiliteMenuItem@16
_NtUserHiliteMenuItem@16:

    movl $0x1198, %eax
77ed6c28:	b8 98 11 00 00       	mov    $0x1198,%eax
    movl $KUSER_SHARED_SYSCALL, %ecx
77ed6c2d:	b9 00 03 fe 7f       	mov    $0x7ffe0300,%ecx
    call *%ecx
77ed6c32:	ff d1                	call   *%ecx
    ret $0x10
77ed6c34:	c2 10 00             	ret    $0x10

77ed6c37 <_NtUserImpersonateDdeClientWindow@8>:

.global _NtUserImpersonateDdeClientWindow@8
_NtUserImpersonateDdeClientWindow@8:

    movl $0x1199, %eax
77ed6c37:	b8 99 11 00 00       	mov    $0x1199,%eax
    movl $KUSER_SHARED_SYSCALL, %ecx
77ed6c3c:	b9 00 03 fe 7f       	mov    $0x7ffe0300,%ecx
    call *%ecx
77ed6c41:	ff d1                	call   *%ecx
    ret $0x8
77ed6c43:	c2 08 00             	ret    $0x8

77ed6c46 <_NtUserInitializeClientPfnArrays@16>:

.global _NtUserInitializeClientPfnArrays@16
_NtUserInitializeClientPfnArrays@16:

    movl $0x119a, %eax
77ed6c46:	b8 9a 11 00 00       	mov    $0x119a,%eax
    movl $KUSER_SHARED_SYSCALL, %ecx
77ed6c4b:	b9 00 03 fe 7f       	mov    $0x7ffe0300,%ecx
    call *%ecx
77ed6c50:	ff d1                	call   *%ecx
    ret $0x10
77ed6c52:	c2 10 00             	ret    $0x10

77ed6c55 <_NtUserInitTask@44>:

.global _NtUserInitTask@44
_NtUserInitTask@44:

    movl $0x119b, %eax
77ed6c55:	b8 9b 11 00 00       	mov    $0x119b,%eax
    movl $KUSER_SHARED_SYSCALL, %ecx
77ed6c5a:	b9 00 03 fe 7f       	mov    $0x7ffe0300,%ecx
    call *%ecx
77ed6c5f:	ff d1                	call   *%ecx
    ret $0x2c
77ed6c61:	c2 2c 00             	ret    $0x2c

77ed6c64 <_NtUserInsertMenuItem@16>:

.global _NtUserInsertMenuItem@16
_NtUserInsertMenuItem@16:

    movl $0x119c, %eax
77ed6c64:	b8 9c 11 00 00       	mov    $0x119c,%eax
    movl $KUSER_SHARED_SYSCALL, %ecx
77ed6c69:	b9 00 03 fe 7f       	mov    $0x7ffe0300,%ecx
    call *%ecx
77ed6c6e:	ff d1                	call   *%ecx
    ret $0x10
77ed6c70:	c2 10 00             	ret    $0x10

77ed6c73 <_NtUserInternalGetWindowText@12>:

.global _NtUserInternalGetWindowText@12
_NtUserInternalGetWindowText@12:

    movl $0x119d, %eax
77ed6c73:	b8 9d 11 00 00       	mov    $0x119d,%eax
    movl $KUSER_SHARED_SYSCALL, %ecx
77ed6c78:	b9 00 03 fe 7f       	mov    $0x7ffe0300,%ecx
    call *%ecx
77ed6c7d:	ff d1                	call   *%ecx
    ret $0xc
77ed6c7f:	c2 0c 00             	ret    $0xc

77ed6c82 <_NtUserInvalidateRect@12>:

.global _NtUserInvalidateRect@12
_NtUserInvalidateRect@12:

    movl $0x119e, %eax
77ed6c82:	b8 9e 11 00 00       	mov    $0x119e,%eax
    movl $KUSER_SHARED_SYSCALL, %ecx
77ed6c87:	b9 00 03 fe 7f       	mov    $0x7ffe0300,%ecx
    call *%ecx
77ed6c8c:	ff d1                	call   *%ecx
    ret $0xc
77ed6c8e:	c2 0c 00             	ret    $0xc

77ed6c91 <_NtUserInvalidateRgn@12>:

.global _NtUserInvalidateRgn@12
_NtUserInvalidateRgn@12:

    movl $0x119f, %eax
77ed6c91:	b8 9f 11 00 00       	mov    $0x119f,%eax
    movl $KUSER_SHARED_SYSCALL, %ecx
77ed6c96:	b9 00 03 fe 7f       	mov    $0x7ffe0300,%ecx
    call *%ecx
77ed6c9b:	ff d1                	call   *%ecx
    ret $0xc
77ed6c9d:	c2 0c 00             	ret    $0xc

77ed6ca0 <_NtUserIsClipboardFormatAvailable@4>:

.global _NtUserIsClipboardFormatAvailable@4
_NtUserIsClipboardFormatAvailable@4:

    movl $0x11a0, %eax
77ed6ca0:	b8 a0 11 00 00       	mov    $0x11a0,%eax
    movl $KUSER_SHARED_SYSCALL, %ecx
77ed6ca5:	b9 00 03 fe 7f       	mov    $0x7ffe0300,%ecx
    call *%ecx
77ed6caa:	ff d1                	call   *%ecx
    ret $0x4
77ed6cac:	c2 04 00             	ret    $0x4

77ed6caf <_NtUserKillSystemTimer@8>:

.global _NtUserKillSystemTimer@8
_NtUserKillSystemTimer@8:

    movl $0x11a1, %eax
77ed6caf:	b8 a1 11 00 00       	mov    $0x11a1,%eax
    movl $KUSER_SHARED_SYSCALL, %ecx
77ed6cb4:	b9 00 03 fe 7f       	mov    $0x7ffe0300,%ecx
    call *%ecx
77ed6cb9:	ff d1                	call   *%ecx
    ret $0x8
77ed6cbb:	c2 08 00             	ret    $0x8

77ed6cbe <_NtUserKillTimer@8>:

.global _NtUserKillTimer@8
_NtUserKillTimer@8:

    movl $0x11a2, %eax
77ed6cbe:	b8 a2 11 00 00       	mov    $0x11a2,%eax
    movl $KUSER_SHARED_SYSCALL, %ecx
77ed6cc3:	b9 00 03 fe 7f       	mov    $0x7ffe0300,%ecx
    call *%ecx
77ed6cc8:	ff d1                	call   *%ecx
    ret $0x8
77ed6cca:	c2 08 00             	ret    $0x8

77ed6ccd <_NtUserLoadKeyboardLayoutEx@24>:

.global _NtUserLoadKeyboardLayoutEx@24
_NtUserLoadKeyboardLayoutEx@24:

    movl $0x11a3, %eax
77ed6ccd:	b8 a3 11 00 00       	mov    $0x11a3,%eax
    movl $KUSER_SHARED_SYSCALL, %ecx
77ed6cd2:	b9 00 03 fe 7f       	mov    $0x7ffe0300,%ecx
    call *%ecx
77ed6cd7:	ff d1                	call   *%ecx
    ret $0x18
77ed6cd9:	c2 18 00             	ret    $0x18

77ed6cdc <_NtUserLockWindowStation@4>:

.global _NtUserLockWindowStation@4
_NtUserLockWindowStation@4:

    movl $0x11a4, %eax
77ed6cdc:	b8 a4 11 00 00       	mov    $0x11a4,%eax
    movl $KUSER_SHARED_SYSCALL, %ecx
77ed6ce1:	b9 00 03 fe 7f       	mov    $0x7ffe0300,%ecx
    call *%ecx
77ed6ce6:	ff d1                	call   *%ecx
    ret $0x4
77ed6ce8:	c2 04 00             	ret    $0x4

77ed6ceb <_NtUserLockWindowUpdate@4>:

.global _NtUserLockWindowUpdate@4
_NtUserLockWindowUpdate@4:

    movl $0x11a5, %eax
77ed6ceb:	b8 a5 11 00 00       	mov    $0x11a5,%eax
    movl $KUSER_SHARED_SYSCALL, %ecx
77ed6cf0:	b9 00 03 fe 7f       	mov    $0x7ffe0300,%ecx
    call *%ecx
77ed6cf5:	ff d1                	call   *%ecx
    ret $0x4
77ed6cf7:	c2 04 00             	ret    $0x4

77ed6cfa <_NtUserLockWorkStation@0>:

.global _NtUserLockWorkStation@0
_NtUserLockWorkStation@0:

    movl $0x11a6, %eax
77ed6cfa:	b8 a6 11 00 00       	mov    $0x11a6,%eax
    movl $KUSER_SHARED_SYSCALL, %ecx
77ed6cff:	b9 00 03 fe 7f       	mov    $0x7ffe0300,%ecx
    call *%ecx
77ed6d04:	ff d1                	call   *%ecx
    ret $0x0
77ed6d06:	c2 00 00             	ret    $0x0

77ed6d09 <_NtUserMapVirtualKeyEx@16>:

.global _NtUserMapVirtualKeyEx@16
_NtUserMapVirtualKeyEx@16:

    movl $0x11a7, %eax
77ed6d09:	b8 a7 11 00 00       	mov    $0x11a7,%eax
    movl $KUSER_SHARED_SYSCALL, %ecx
77ed6d0e:	b9 00 03 fe 7f       	mov    $0x7ffe0300,%ecx
    call *%ecx
77ed6d13:	ff d1                	call   *%ecx
    ret $0x10
77ed6d15:	c2 10 00             	ret    $0x10

77ed6d18 <_NtUserMenuInfo@12>:

.global _NtUserMenuInfo@12
_NtUserMenuInfo@12:

    movl $0x11a8, %eax
77ed6d18:	b8 a8 11 00 00       	mov    $0x11a8,%eax
    movl $KUSER_SHARED_SYSCALL, %ecx
77ed6d1d:	b9 00 03 fe 7f       	mov    $0x7ffe0300,%ecx
    call *%ecx
77ed6d22:	ff d1                	call   *%ecx
    ret $0xc
77ed6d24:	c2 0c 00             	ret    $0xc

77ed6d27 <_NtUserMenuItemFromPoint@16>:

.global _NtUserMenuItemFromPoint@16
_NtUserMenuItemFromPoint@16:

    movl $0x11a9, %eax
77ed6d27:	b8 a9 11 00 00       	mov    $0x11a9,%eax
    movl $KUSER_SHARED_SYSCALL, %ecx
77ed6d2c:	b9 00 03 fe 7f       	mov    $0x7ffe0300,%ecx
    call *%ecx
77ed6d31:	ff d1                	call   *%ecx
    ret $0x10
77ed6d33:	c2 10 00             	ret    $0x10

77ed6d36 <_NtUserMenuItemInfo@20>:

.global _NtUserMenuItemInfo@20
_NtUserMenuItemInfo@20:

    movl $0x11aa, %eax
77ed6d36:	b8 aa 11 00 00       	mov    $0x11aa,%eax
    movl $KUSER_SHARED_SYSCALL, %ecx
77ed6d3b:	b9 00 03 fe 7f       	mov    $0x7ffe0300,%ecx
    call *%ecx
77ed6d40:	ff d1                	call   *%ecx
    ret $0x14
77ed6d42:	c2 14 00             	ret    $0x14

77ed6d45 <_NtUserMessageCall@28>:

.global _NtUserMessageCall@28
_NtUserMessageCall@28:

    movl $0x11ab, %eax
77ed6d45:	b8 ab 11 00 00       	mov    $0x11ab,%eax
    movl $KUSER_SHARED_SYSCALL, %ecx
77ed6d4a:	b9 00 03 fe 7f       	mov    $0x7ffe0300,%ecx
    call *%ecx
77ed6d4f:	ff d1                	call   *%ecx
    ret $0x1c
77ed6d51:	c2 1c 00             	ret    $0x1c

77ed6d54 <_NtUserMNDragLeave@0>:

.global _NtUserMNDragLeave@0
_NtUserMNDragLeave@0:

    movl $0x11ac, %eax
77ed6d54:	b8 ac 11 00 00       	mov    $0x11ac,%eax
    movl $KUSER_SHARED_SYSCALL, %ecx
77ed6d59:	b9 00 03 fe 7f       	mov    $0x7ffe0300,%ecx
    call *%ecx
77ed6d5e:	ff d1                	call   *%ecx
    ret $0x0
77ed6d60:	c2 00 00             	ret    $0x0

77ed6d63 <_NtUserMNDragOver@8>:

.global _NtUserMNDragOver@8
_NtUserMNDragOver@8:

    movl $0x11ad, %eax
77ed6d63:	b8 ad 11 00 00       	mov    $0x11ad,%eax
    movl $KUSER_SHARED_SYSCALL, %ecx
77ed6d68:	b9 00 03 fe 7f       	mov    $0x7ffe0300,%ecx
    call *%ecx
77ed6d6d:	ff d1                	call   *%ecx
    ret $0x8
77ed6d6f:	c2 08 00             	ret    $0x8

77ed6d72 <_NtUserModifyUserStartupInfoFlags@8>:

.global _NtUserModifyUserStartupInfoFlags@8
_NtUserModifyUserStartupInfoFlags@8:

    movl $0x11ae, %eax
77ed6d72:	b8 ae 11 00 00       	mov    $0x11ae,%eax
    movl $KUSER_SHARED_SYSCALL, %ecx
77ed6d77:	b9 00 03 fe 7f       	mov    $0x7ffe0300,%ecx
    call *%ecx
77ed6d7c:	ff d1                	call   *%ecx
    ret $0x8
77ed6d7e:	c2 08 00             	ret    $0x8

77ed6d81 <_NtUserMonitorFromPoint@12>:

.global _NtUserMonitorFromPoint@12
_NtUserMonitorFromPoint@12:

    movl $0x11af, %eax
77ed6d81:	b8 af 11 00 00       	mov    $0x11af,%eax
    movl $KUSER_SHARED_SYSCALL, %ecx
77ed6d86:	b9 00 03 fe 7f       	mov    $0x7ffe0300,%ecx
    call *%ecx
77ed6d8b:	ff d1                	call   *%ecx
    ret $0xc
77ed6d8d:	c2 0c 00             	ret    $0xc

77ed6d90 <_NtUserMonitorFromRect@8>:

.global _NtUserMonitorFromRect@8
_NtUserMonitorFromRect@8:

    movl $0x11b0, %eax
77ed6d90:	b8 b0 11 00 00       	mov    $0x11b0,%eax
    movl $KUSER_SHARED_SYSCALL, %ecx
77ed6d95:	b9 00 03 fe 7f       	mov    $0x7ffe0300,%ecx
    call *%ecx
77ed6d9a:	ff d1                	call   *%ecx
    ret $0x8
77ed6d9c:	c2 08 00             	ret    $0x8

77ed6d9f <_NtUserMonitorFromWindow@8>:

.global _NtUserMonitorFromWindow@8
_NtUserMonitorFromWindow@8:

    movl $0x11b1, %eax
77ed6d9f:	b8 b1 11 00 00       	mov    $0x11b1,%eax
    movl $KUSER_SHARED_SYSCALL, %ecx
77ed6da4:	b9 00 03 fe 7f       	mov    $0x7ffe0300,%ecx
    call *%ecx
77ed6da9:	ff d1                	call   *%ecx
    ret $0x8
77ed6dab:	c2 08 00             	ret    $0x8

77ed6dae <_NtUserMoveWindow@24>:

.global _NtUserMoveWindow@24
_NtUserMoveWindow@24:

    movl $0x11b2, %eax
77ed6dae:	b8 b2 11 00 00       	mov    $0x11b2,%eax
    movl $KUSER_SHARED_SYSCALL, %ecx
77ed6db3:	b9 00 03 fe 7f       	mov    $0x7ffe0300,%ecx
    call *%ecx
77ed6db8:	ff d1                	call   *%ecx
    ret $0x18
77ed6dba:	c2 18 00             	ret    $0x18

77ed6dbd <_NtUserNotifyIMEStatus@12>:

.global _NtUserNotifyIMEStatus@12
_NtUserNotifyIMEStatus@12:

    movl $0x11b3, %eax
77ed6dbd:	b8 b3 11 00 00       	mov    $0x11b3,%eax
    movl $KUSER_SHARED_SYSCALL, %ecx
77ed6dc2:	b9 00 03 fe 7f       	mov    $0x7ffe0300,%ecx
    call *%ecx
77ed6dc7:	ff d1                	call   *%ecx
    ret $0xc
77ed6dc9:	c2 0c 00             	ret    $0xc

77ed6dcc <_NtUserNotifyWinEvent@16>:

.global _NtUserNotifyWinEvent@16
_NtUserNotifyWinEvent@16:

    movl $0x11b4, %eax
77ed6dcc:	b8 b4 11 00 00       	mov    $0x11b4,%eax
    movl $KUSER_SHARED_SYSCALL, %ecx
77ed6dd1:	b9 00 03 fe 7f       	mov    $0x7ffe0300,%ecx
    call *%ecx
77ed6dd6:	ff d1                	call   *%ecx
    ret $0x10
77ed6dd8:	c2 10 00             	ret    $0x10

77ed6ddb <_NtUserOpenClipboard@8>:

.global _NtUserOpenClipboard@8
_NtUserOpenClipboard@8:

    movl $0x11b5, %eax
77ed6ddb:	b8 b5 11 00 00       	mov    $0x11b5,%eax
    movl $KUSER_SHARED_SYSCALL, %ecx
77ed6de0:	b9 00 03 fe 7f       	mov    $0x7ffe0300,%ecx
    call *%ecx
77ed6de5:	ff d1                	call   *%ecx
    ret $0x8
77ed6de7:	c2 08 00             	ret    $0x8

77ed6dea <_NtUserOpenDesktop@12>:

.global _NtUserOpenDesktop@12
_NtUserOpenDesktop@12:

    movl $0x11b6, %eax
77ed6dea:	b8 b6 11 00 00       	mov    $0x11b6,%eax
    movl $KUSER_SHARED_SYSCALL, %ecx
77ed6def:	b9 00 03 fe 7f       	mov    $0x7ffe0300,%ecx
    call *%ecx
77ed6df4:	ff d1                	call   *%ecx
    ret $0xc
77ed6df6:	c2 0c 00             	ret    $0xc

77ed6df9 <_NtUserOpenInputDesktop@12>:

.global _NtUserOpenInputDesktop@12
_NtUserOpenInputDesktop@12:

    movl $0x11b7, %eax
77ed6df9:	b8 b7 11 00 00       	mov    $0x11b7,%eax
    movl $KUSER_SHARED_SYSCALL, %ecx
77ed6dfe:	b9 00 03 fe 7f       	mov    $0x7ffe0300,%ecx
    call *%ecx
77ed6e03:	ff d1                	call   *%ecx
    ret $0xc
77ed6e05:	c2 0c 00             	ret    $0xc

77ed6e08 <_NtUserOpenWindowStation@8>:

.global _NtUserOpenWindowStation@8
_NtUserOpenWindowStation@8:

    movl $0x11b8, %eax
77ed6e08:	b8 b8 11 00 00       	mov    $0x11b8,%eax
    movl $KUSER_SHARED_SYSCALL, %ecx
77ed6e0d:	b9 00 03 fe 7f       	mov    $0x7ffe0300,%ecx
    call *%ecx
77ed6e12:	ff d1                	call   *%ecx
    ret $0x8
77ed6e14:	c2 08 00             	ret    $0x8

77ed6e17 <_NtUserPaintDesktop@4>:

.global _NtUserPaintDesktop@4
_NtUserPaintDesktop@4:

    movl $0x11b9, %eax
77ed6e17:	b8 b9 11 00 00       	mov    $0x11b9,%eax
    movl $KUSER_SHARED_SYSCALL, %ecx
77ed6e1c:	b9 00 03 fe 7f       	mov    $0x7ffe0300,%ecx
    call *%ecx
77ed6e21:	ff d1                	call   *%ecx
    ret $0x4
77ed6e23:	c2 04 00             	ret    $0x4

77ed6e26 <_NtUserPeekMessage@20>:

.global _NtUserPeekMessage@20
_NtUserPeekMessage@20:

    movl $0x11ba, %eax
77ed6e26:	b8 ba 11 00 00       	mov    $0x11ba,%eax
    movl $KUSER_SHARED_SYSCALL, %ecx
77ed6e2b:	b9 00 03 fe 7f       	mov    $0x7ffe0300,%ecx
    call *%ecx
77ed6e30:	ff d1                	call   *%ecx
    ret $0x14
77ed6e32:	c2 14 00             	ret    $0x14

77ed6e35 <_NtUserPostMessage@16>:

.global _NtUserPostMessage@16
_NtUserPostMessage@16:

    movl $0x11bb, %eax
77ed6e35:	b8 bb 11 00 00       	mov    $0x11bb,%eax
    movl $KUSER_SHARED_SYSCALL, %ecx
77ed6e3a:	b9 00 03 fe 7f       	mov    $0x7ffe0300,%ecx
    call *%ecx
77ed6e3f:	ff d1                	call   *%ecx
    ret $0x10
77ed6e41:	c2 10 00             	ret    $0x10

77ed6e44 <_NtUserPostThreadMessage@16>:

.global _NtUserPostThreadMessage@16
_NtUserPostThreadMessage@16:

    movl $0x11bc, %eax
77ed6e44:	b8 bc 11 00 00       	mov    $0x11bc,%eax
    movl $KUSER_SHARED_SYSCALL, %ecx
77ed6e49:	b9 00 03 fe 7f       	mov    $0x7ffe0300,%ecx
    call *%ecx
77ed6e4e:	ff d1                	call   *%ecx
    ret $0x10
77ed6e50:	c2 10 00             	ret    $0x10

77ed6e53 <_NtUserQuerySendMessage@4>:

.global _NtUserQuerySendMessage@4
_NtUserQuerySendMessage@4:

    movl $0x11bd, %eax
77ed6e53:	b8 bd 11 00 00       	mov    $0x11bd,%eax
    movl $KUSER_SHARED_SYSCALL, %ecx
77ed6e58:	b9 00 03 fe 7f       	mov    $0x7ffe0300,%ecx
    call *%ecx
77ed6e5d:	ff d1                	call   *%ecx
    ret $0x4
77ed6e5f:	c2 04 00             	ret    $0x4

77ed6e62 <_NtUserQueryUserCounters@20>:

.global _NtUserQueryUserCounters@20
_NtUserQueryUserCounters@20:

    movl $0x11be, %eax
77ed6e62:	b8 be 11 00 00       	mov    $0x11be,%eax
    movl $KUSER_SHARED_SYSCALL, %ecx
77ed6e67:	b9 00 03 fe 7f       	mov    $0x7ffe0300,%ecx
    call *%ecx
77ed6e6c:	ff d1                	call   *%ecx
    ret $0x14
77ed6e6e:	c2 14 00             	ret    $0x14

77ed6e71 <_NtUserQueryWindow@8>:

.global _NtUserQueryWindow@8
_NtUserQueryWindow@8:

    movl $0x11bf, %eax
77ed6e71:	b8 bf 11 00 00       	mov    $0x11bf,%eax
    movl $KUSER_SHARED_SYSCALL, %ecx
77ed6e76:	b9 00 03 fe 7f       	mov    $0x7ffe0300,%ecx
    call *%ecx
77ed6e7b:	ff d1                	call   *%ecx
    ret $0x8
77ed6e7d:	c2 08 00             	ret    $0x8

77ed6e80 <_NtUserReleaseDC@8>:

.global _NtUserReleaseDC@8
_NtUserReleaseDC@8:

    movl $0x11c0, %eax
77ed6e80:	b8 c0 11 00 00       	mov    $0x11c0,%eax
    movl $KUSER_SHARED_SYSCALL, %ecx
77ed6e85:	b9 00 03 fe 7f       	mov    $0x7ffe0300,%ecx
    call *%ecx
77ed6e8a:	ff d1                	call   *%ecx
    ret $0x8
77ed6e8c:	c2 08 00             	ret    $0x8

77ed6e8f <_NtUserRealChildWindowFromPoint@12>:

.global _NtUserRealChildWindowFromPoint@12
_NtUserRealChildWindowFromPoint@12:

    movl $0x11c1, %eax
77ed6e8f:	b8 c1 11 00 00       	mov    $0x11c1,%eax
    movl $KUSER_SHARED_SYSCALL, %ecx
77ed6e94:	b9 00 03 fe 7f       	mov    $0x7ffe0300,%ecx
    call *%ecx
77ed6e99:	ff d1                	call   *%ecx
    ret $0xc
77ed6e9b:	c2 0c 00             	ret    $0xc

77ed6e9e <_NtUserRedrawWindow@16>:

.global _NtUserRedrawWindow@16
_NtUserRedrawWindow@16:

    movl $0x11c2, %eax
77ed6e9e:	b8 c2 11 00 00       	mov    $0x11c2,%eax
    movl $KUSER_SHARED_SYSCALL, %ecx
77ed6ea3:	b9 00 03 fe 7f       	mov    $0x7ffe0300,%ecx
    call *%ecx
77ed6ea8:	ff d1                	call   *%ecx
    ret $0x10
77ed6eaa:	c2 10 00             	ret    $0x10

77ed6ead <_NtUserRegisterClassExWOW@28>:

.global _NtUserRegisterClassExWOW@28
_NtUserRegisterClassExWOW@28:

    movl $0x11c3, %eax
77ed6ead:	b8 c3 11 00 00       	mov    $0x11c3,%eax
    movl $KUSER_SHARED_SYSCALL, %ecx
77ed6eb2:	b9 00 03 fe 7f       	mov    $0x7ffe0300,%ecx
    call *%ecx
77ed6eb7:	ff d1                	call   *%ecx
    ret $0x1c
77ed6eb9:	c2 1c 00             	ret    $0x1c

77ed6ebc <_NtUserRegisterHotKey@16>:

.global _NtUserRegisterHotKey@16
_NtUserRegisterHotKey@16:

    movl $0x11c4, %eax
77ed6ebc:	b8 c4 11 00 00       	mov    $0x11c4,%eax
    movl $KUSER_SHARED_SYSCALL, %ecx
77ed6ec1:	b9 00 03 fe 7f       	mov    $0x7ffe0300,%ecx
    call *%ecx
77ed6ec6:	ff d1                	call   *%ecx
    ret $0x10
77ed6ec8:	c2 10 00             	ret    $0x10

77ed6ecb <_NtUserRegisterTasklist@4>:

.global _NtUserRegisterTasklist@4
_NtUserRegisterTasklist@4:

    movl $0x11c5, %eax
77ed6ecb:	b8 c5 11 00 00       	mov    $0x11c5,%eax
    movl $KUSER_SHARED_SYSCALL, %ecx
77ed6ed0:	b9 00 03 fe 7f       	mov    $0x7ffe0300,%ecx
    call *%ecx
77ed6ed5:	ff d1                	call   *%ecx
    ret $0x4
77ed6ed7:	c2 04 00             	ret    $0x4

77ed6eda <_NtUserRegisterWindowMessage@4>:

.global _NtUserRegisterWindowMessage@4
_NtUserRegisterWindowMessage@4:

    movl $0x11c6, %eax
77ed6eda:	b8 c6 11 00 00       	mov    $0x11c6,%eax
    movl $KUSER_SHARED_SYSCALL, %ecx
77ed6edf:	b9 00 03 fe 7f       	mov    $0x7ffe0300,%ecx
    call *%ecx
77ed6ee4:	ff d1                	call   *%ecx
    ret $0x4
77ed6ee6:	c2 04 00             	ret    $0x4

77ed6ee9 <_NtUserRemoveMenu@12>:

.global _NtUserRemoveMenu@12
_NtUserRemoveMenu@12:

    movl $0x11c7, %eax
77ed6ee9:	b8 c7 11 00 00       	mov    $0x11c7,%eax
    movl $KUSER_SHARED_SYSCALL, %ecx
77ed6eee:	b9 00 03 fe 7f       	mov    $0x7ffe0300,%ecx
    call *%ecx
77ed6ef3:	ff d1                	call   *%ecx
    ret $0xc
77ed6ef5:	c2 0c 00             	ret    $0xc

77ed6ef8 <_NtUserRemoveProp@8>:

.global _NtUserRemoveProp@8
_NtUserRemoveProp@8:

    movl $0x11c8, %eax
77ed6ef8:	b8 c8 11 00 00       	mov    $0x11c8,%eax
    movl $KUSER_SHARED_SYSCALL, %ecx
77ed6efd:	b9 00 03 fe 7f       	mov    $0x7ffe0300,%ecx
    call *%ecx
77ed6f02:	ff d1                	call   *%ecx
    ret $0x8
77ed6f04:	c2 08 00             	ret    $0x8

77ed6f07 <_NtUserResolveDesktopForWOW@4>:

.global _NtUserResolveDesktopForWOW@4
_NtUserResolveDesktopForWOW@4:

    movl $0x11c9, %eax
77ed6f07:	b8 c9 11 00 00       	mov    $0x11c9,%eax
    movl $KUSER_SHARED_SYSCALL, %ecx
77ed6f0c:	b9 00 03 fe 7f       	mov    $0x7ffe0300,%ecx
    call *%ecx
77ed6f11:	ff d1                	call   *%ecx
    ret $0x4
77ed6f13:	c2 04 00             	ret    $0x4

77ed6f16 <_NtUserSBGetParms@16>:

.global _NtUserSBGetParms@16
_NtUserSBGetParms@16:

    movl $0x11ca, %eax
77ed6f16:	b8 ca 11 00 00       	mov    $0x11ca,%eax
    movl $KUSER_SHARED_SYSCALL, %ecx
77ed6f1b:	b9 00 03 fe 7f       	mov    $0x7ffe0300,%ecx
    call *%ecx
77ed6f20:	ff d1                	call   *%ecx
    ret $0x10
77ed6f22:	c2 10 00             	ret    $0x10

77ed6f25 <_NtUserScrollDC@28>:

.global _NtUserScrollDC@28
_NtUserScrollDC@28:

    movl $0x11cb, %eax
77ed6f25:	b8 cb 11 00 00       	mov    $0x11cb,%eax
    movl $KUSER_SHARED_SYSCALL, %ecx
77ed6f2a:	b9 00 03 fe 7f       	mov    $0x7ffe0300,%ecx
    call *%ecx
77ed6f2f:	ff d1                	call   *%ecx
    ret $0x1c
77ed6f31:	c2 1c 00             	ret    $0x1c

77ed6f34 <_NtUserScrollWindowEx@32>:

.global _NtUserScrollWindowEx@32
_NtUserScrollWindowEx@32:

    movl $0x11cc, %eax
77ed6f34:	b8 cc 11 00 00       	mov    $0x11cc,%eax
    movl $KUSER_SHARED_SYSCALL, %ecx
77ed6f39:	b9 00 03 fe 7f       	mov    $0x7ffe0300,%ecx
    call *%ecx
77ed6f3e:	ff d1                	call   *%ecx
    ret $0x20
77ed6f40:	c2 20 00             	ret    $0x20

77ed6f43 <_NtUserSendInput@12>:

.global _NtUserSendInput@12
_NtUserSendInput@12:

    movl $0x11cd, %eax
77ed6f43:	b8 cd 11 00 00       	mov    $0x11cd,%eax
    movl $KUSER_SHARED_SYSCALL, %ecx
77ed6f48:	b9 00 03 fe 7f       	mov    $0x7ffe0300,%ecx
    call *%ecx
77ed6f4d:	ff d1                	call   *%ecx
    ret $0xc
77ed6f4f:	c2 0c 00             	ret    $0xc

77ed6f52 <_NtUserSendMessage@20>:

.global _NtUserSendMessage@20
_NtUserSendMessage@20:

    movl $0x11ce, %eax
77ed6f52:	b8 ce 11 00 00       	mov    $0x11ce,%eax
    movl $KUSER_SHARED_SYSCALL, %ecx
77ed6f57:	b9 00 03 fe 7f       	mov    $0x7ffe0300,%ecx
    call *%ecx
77ed6f5c:	ff d1                	call   *%ecx
    ret $0x14
77ed6f5e:	c2 14 00             	ret    $0x14

77ed6f61 <_NtUserSendMessageCallback@24>:

.global _NtUserSendMessageCallback@24
_NtUserSendMessageCallback@24:

    movl $0x11cf, %eax
77ed6f61:	b8 cf 11 00 00       	mov    $0x11cf,%eax
    movl $KUSER_SHARED_SYSCALL, %ecx
77ed6f66:	b9 00 03 fe 7f       	mov    $0x7ffe0300,%ecx
    call *%ecx
77ed6f6b:	ff d1                	call   *%ecx
    ret $0x18
77ed6f6d:	c2 18 00             	ret    $0x18

77ed6f70 <_NtUserSendMessageTimeout@32>:

.global _NtUserSendMessageTimeout@32
_NtUserSendMessageTimeout@32:

    movl $0x11d0, %eax
77ed6f70:	b8 d0 11 00 00       	mov    $0x11d0,%eax
    movl $KUSER_SHARED_SYSCALL, %ecx
77ed6f75:	b9 00 03 fe 7f       	mov    $0x7ffe0300,%ecx
    call *%ecx
77ed6f7a:	ff d1                	call   *%ecx
    ret $0x20
77ed6f7c:	c2 20 00             	ret    $0x20

77ed6f7f <_NtUserSendNotifyMessage@16>:

.global _NtUserSendNotifyMessage@16
_NtUserSendNotifyMessage@16:

    movl $0x11d1, %eax
77ed6f7f:	b8 d1 11 00 00       	mov    $0x11d1,%eax
    movl $KUSER_SHARED_SYSCALL, %ecx
77ed6f84:	b9 00 03 fe 7f       	mov    $0x7ffe0300,%ecx
    call *%ecx
77ed6f89:	ff d1                	call   *%ecx
    ret $0x10
77ed6f8b:	c2 10 00             	ret    $0x10

77ed6f8e <_NtUserSetActiveWindow@4>:

.global _NtUserSetActiveWindow@4
_NtUserSetActiveWindow@4:

    movl $0x11d2, %eax
77ed6f8e:	b8 d2 11 00 00       	mov    $0x11d2,%eax
    movl $KUSER_SHARED_SYSCALL, %ecx
77ed6f93:	b9 00 03 fe 7f       	mov    $0x7ffe0300,%ecx
    call *%ecx
77ed6f98:	ff d1                	call   *%ecx
    ret $0x4
77ed6f9a:	c2 04 00             	ret    $0x4

77ed6f9d <_NtUserSetCapture@4>:

.global _NtUserSetCapture@4
_NtUserSetCapture@4:

    movl $0x11d3, %eax
77ed6f9d:	b8 d3 11 00 00       	mov    $0x11d3,%eax
    movl $KUSER_SHARED_SYSCALL, %ecx
77ed6fa2:	b9 00 03 fe 7f       	mov    $0x7ffe0300,%ecx
    call *%ecx
77ed6fa7:	ff d1                	call   *%ecx
    ret $0x4
77ed6fa9:	c2 04 00             	ret    $0x4

77ed6fac <_NtUserSetClassLong@16>:

.global _NtUserSetClassLong@16
_NtUserSetClassLong@16:

    movl $0x11d4, %eax
77ed6fac:	b8 d4 11 00 00       	mov    $0x11d4,%eax
    movl $KUSER_SHARED_SYSCALL, %ecx
77ed6fb1:	b9 00 03 fe 7f       	mov    $0x7ffe0300,%ecx
    call *%ecx
77ed6fb6:	ff d1                	call   *%ecx
    ret $0x10
77ed6fb8:	c2 10 00             	ret    $0x10

77ed6fbb <_NtUserSetClassWord@12>:

.global _NtUserSetClassWord@12
_NtUserSetClassWord@12:

    movl $0x11d5, %eax
77ed6fbb:	b8 d5 11 00 00       	mov    $0x11d5,%eax
    movl $KUSER_SHARED_SYSCALL, %ecx
77ed6fc0:	b9 00 03 fe 7f       	mov    $0x7ffe0300,%ecx
    call *%ecx
77ed6fc5:	ff d1                	call   *%ecx
    ret $0xc
77ed6fc7:	c2 0c 00             	ret    $0xc

77ed6fca <_NtUserSetClipboardData@12>:

.global _NtUserSetClipboardData@12
_NtUserSetClipboardData@12:

    movl $0x11d6, %eax
77ed6fca:	b8 d6 11 00 00       	mov    $0x11d6,%eax
    movl $KUSER_SHARED_SYSCALL, %ecx
77ed6fcf:	b9 00 03 fe 7f       	mov    $0x7ffe0300,%ecx
    call *%ecx
77ed6fd4:	ff d1                	call   *%ecx
    ret $0xc
77ed6fd6:	c2 0c 00             	ret    $0xc

77ed6fd9 <_NtUserSetClipboardViewer@4>:

.global _NtUserSetClipboardViewer@4
_NtUserSetClipboardViewer@4:

    movl $0x11d7, %eax
77ed6fd9:	b8 d7 11 00 00       	mov    $0x11d7,%eax
    movl $KUSER_SHARED_SYSCALL, %ecx
77ed6fde:	b9 00 03 fe 7f       	mov    $0x7ffe0300,%ecx
    call *%ecx
77ed6fe3:	ff d1                	call   *%ecx
    ret $0x4
77ed6fe5:	c2 04 00             	ret    $0x4

77ed6fe8 <_NtUserSetConsoleReserveKeys@8>:

.global _NtUserSetConsoleReserveKeys@8
_NtUserSetConsoleReserveKeys@8:

    movl $0x11d8, %eax
77ed6fe8:	b8 d8 11 00 00       	mov    $0x11d8,%eax
    movl $KUSER_SHARED_SYSCALL, %ecx
77ed6fed:	b9 00 03 fe 7f       	mov    $0x7ffe0300,%ecx
    call *%ecx
77ed6ff2:	ff d1                	call   *%ecx
    ret $0x8
77ed6ff4:	c2 08 00             	ret    $0x8

77ed6ff7 <_NtUserSetCursor@4>:

.global _NtUserSetCursor@4
_NtUserSetCursor@4:

    movl $0x11d9, %eax
77ed6ff7:	b8 d9 11 00 00       	mov    $0x11d9,%eax
    movl $KUSER_SHARED_SYSCALL, %ecx
77ed6ffc:	b9 00 03 fe 7f       	mov    $0x7ffe0300,%ecx
    call *%ecx
77ed7001:	ff d1                	call   *%ecx
    ret $0x4
77ed7003:	c2 04 00             	ret    $0x4

77ed7006 <_NtUserSetCursorIconContents@8>:

.global _NtUserSetCursorIconContents@8
_NtUserSetCursorIconContents@8:

    movl $0x11da, %eax
77ed7006:	b8 da 11 00 00       	mov    $0x11da,%eax
    movl $KUSER_SHARED_SYSCALL, %ecx
77ed700b:	b9 00 03 fe 7f       	mov    $0x7ffe0300,%ecx
    call *%ecx
77ed7010:	ff d1                	call   *%ecx
    ret $0x8
77ed7012:	c2 08 00             	ret    $0x8

77ed7015 <_NtUserSetCursorIconData@24>:

.global _NtUserSetCursorIconData@24
_NtUserSetCursorIconData@24:

    movl $0x11db, %eax
77ed7015:	b8 db 11 00 00       	mov    $0x11db,%eax
    movl $KUSER_SHARED_SYSCALL, %ecx
77ed701a:	b9 00 03 fe 7f       	mov    $0x7ffe0300,%ecx
    call *%ecx
77ed701f:	ff d1                	call   *%ecx
    ret $0x18
77ed7021:	c2 18 00             	ret    $0x18

77ed7024 <_NtUserSetDbgTag@8>:

.global _NtUserSetDbgTag@8
_NtUserSetDbgTag@8:

    movl $0x11dc, %eax
77ed7024:	b8 dc 11 00 00       	mov    $0x11dc,%eax
    movl $KUSER_SHARED_SYSCALL, %ecx
77ed7029:	b9 00 03 fe 7f       	mov    $0x7ffe0300,%ecx
    call *%ecx
77ed702e:	ff d1                	call   *%ecx
    ret $0x8
77ed7030:	c2 08 00             	ret    $0x8

77ed7033 <_NtUserSetFocus@4>:

.global _NtUserSetFocus@4
_NtUserSetFocus@4:

    movl $0x11dd, %eax
77ed7033:	b8 dd 11 00 00       	mov    $0x11dd,%eax
    movl $KUSER_SHARED_SYSCALL, %ecx
77ed7038:	b9 00 03 fe 7f       	mov    $0x7ffe0300,%ecx
    call *%ecx
77ed703d:	ff d1                	call   *%ecx
    ret $0x4
77ed703f:	c2 04 00             	ret    $0x4

77ed7042 <_NtUserSetImeHotKey@20>:

.global _NtUserSetImeHotKey@20
_NtUserSetImeHotKey@20:

    movl $0x11de, %eax
77ed7042:	b8 de 11 00 00       	mov    $0x11de,%eax
    movl $KUSER_SHARED_SYSCALL, %ecx
77ed7047:	b9 00 03 fe 7f       	mov    $0x7ffe0300,%ecx
    call *%ecx
77ed704c:	ff d1                	call   *%ecx
    ret $0x14
77ed704e:	c2 14 00             	ret    $0x14

77ed7051 <_NtUserSetImeOwnerWindow@8>:

.global _NtUserSetImeOwnerWindow@8
_NtUserSetImeOwnerWindow@8:

    movl $0x11df, %eax
77ed7051:	b8 df 11 00 00       	mov    $0x11df,%eax
    movl $KUSER_SHARED_SYSCALL, %ecx
77ed7056:	b9 00 03 fe 7f       	mov    $0x7ffe0300,%ecx
    call *%ecx
77ed705b:	ff d1                	call   *%ecx
    ret $0x8
77ed705d:	c2 08 00             	ret    $0x8

77ed7060 <_NtUserSetInternalWindowPos@16>:

.global _NtUserSetInternalWindowPos@16
_NtUserSetInternalWindowPos@16:

    movl $0x11e0, %eax
77ed7060:	b8 e0 11 00 00       	mov    $0x11e0,%eax
    movl $KUSER_SHARED_SYSCALL, %ecx
77ed7065:	b9 00 03 fe 7f       	mov    $0x7ffe0300,%ecx
    call *%ecx
77ed706a:	ff d1                	call   *%ecx
    ret $0x10
77ed706c:	c2 10 00             	ret    $0x10

77ed706f <_NtUserSetKeyboardState@4>:

.global _NtUserSetKeyboardState@4
_NtUserSetKeyboardState@4:

    movl $0x11e1, %eax
77ed706f:	b8 e1 11 00 00       	mov    $0x11e1,%eax
    movl $KUSER_SHARED_SYSCALL, %ecx
77ed7074:	b9 00 03 fe 7f       	mov    $0x7ffe0300,%ecx
    call *%ecx
77ed7079:	ff d1                	call   *%ecx
    ret $0x4
77ed707b:	c2 04 00             	ret    $0x4

77ed707e <_NtUserSetLayeredWindowAttributes@16>:

.global _NtUserSetLayeredWindowAttributes@16
_NtUserSetLayeredWindowAttributes@16:

    movl $0x11e2, %eax
77ed707e:	b8 e2 11 00 00       	mov    $0x11e2,%eax
    movl $KUSER_SHARED_SYSCALL, %ecx
77ed7083:	b9 00 03 fe 7f       	mov    $0x7ffe0300,%ecx
    call *%ecx
77ed7088:	ff d1                	call   *%ecx
    ret $0x10
77ed708a:	c2 10 00             	ret    $0x10

77ed708d <_NtUserSetLogonNotifyWindow@4>:

.global _NtUserSetLogonNotifyWindow@4
_NtUserSetLogonNotifyWindow@4:

    movl $0x11e3, %eax
77ed708d:	b8 e3 11 00 00       	mov    $0x11e3,%eax
    movl $KUSER_SHARED_SYSCALL, %ecx
77ed7092:	b9 00 03 fe 7f       	mov    $0x7ffe0300,%ecx
    call *%ecx
77ed7097:	ff d1                	call   *%ecx
    ret $0x4
77ed7099:	c2 04 00             	ret    $0x4

77ed709c <_NtUserSetMenu@12>:

.global _NtUserSetMenu@12
_NtUserSetMenu@12:

    movl $0x11e4, %eax
77ed709c:	b8 e4 11 00 00       	mov    $0x11e4,%eax
    movl $KUSER_SHARED_SYSCALL, %ecx
77ed70a1:	b9 00 03 fe 7f       	mov    $0x7ffe0300,%ecx
    call *%ecx
77ed70a6:	ff d1                	call   *%ecx
    ret $0xc
77ed70a8:	c2 0c 00             	ret    $0xc

77ed70ab <_NtUserSetMenuContextHelpId@8>:

.global _NtUserSetMenuContextHelpId@8
_NtUserSetMenuContextHelpId@8:

    movl $0x11e5, %eax
77ed70ab:	b8 e5 11 00 00       	mov    $0x11e5,%eax
    movl $KUSER_SHARED_SYSCALL, %ecx
77ed70b0:	b9 00 03 fe 7f       	mov    $0x7ffe0300,%ecx
    call *%ecx
77ed70b5:	ff d1                	call   *%ecx
    ret $0x8
77ed70b7:	c2 08 00             	ret    $0x8

77ed70ba <_NtUserSetMenuDefaultItem@12>:

.global _NtUserSetMenuDefaultItem@12
_NtUserSetMenuDefaultItem@12:

    movl $0x11e6, %eax
77ed70ba:	b8 e6 11 00 00       	mov    $0x11e6,%eax
    movl $KUSER_SHARED_SYSCALL, %ecx
77ed70bf:	b9 00 03 fe 7f       	mov    $0x7ffe0300,%ecx
    call *%ecx
77ed70c4:	ff d1                	call   *%ecx
    ret $0xc
77ed70c6:	c2 0c 00             	ret    $0xc

77ed70c9 <_NtUserSetMenuFlagRtoL@4>:

.global _NtUserSetMenuFlagRtoL@4
_NtUserSetMenuFlagRtoL@4:

    movl $0x11e7, %eax
77ed70c9:	b8 e7 11 00 00       	mov    $0x11e7,%eax
    movl $KUSER_SHARED_SYSCALL, %ecx
77ed70ce:	b9 00 03 fe 7f       	mov    $0x7ffe0300,%ecx
    call *%ecx
77ed70d3:	ff d1                	call   *%ecx
    ret $0x4
77ed70d5:	c2 04 00             	ret    $0x4

77ed70d8 <_NtUserSetObjectInformation@16>:

.global _NtUserSetObjectInformation@16
_NtUserSetObjectInformation@16:

    movl $0x11e8, %eax
77ed70d8:	b8 e8 11 00 00       	mov    $0x11e8,%eax
    movl $KUSER_SHARED_SYSCALL, %ecx
77ed70dd:	b9 00 03 fe 7f       	mov    $0x7ffe0300,%ecx
    call *%ecx
77ed70e2:	ff d1                	call   *%ecx
    ret $0x10
77ed70e4:	c2 10 00             	ret    $0x10

77ed70e7 <_NtUserSetParent@8>:

.global _NtUserSetParent@8
_NtUserSetParent@8:

    movl $0x11e9, %eax
77ed70e7:	b8 e9 11 00 00       	mov    $0x11e9,%eax
    movl $KUSER_SHARED_SYSCALL, %ecx
77ed70ec:	b9 00 03 fe 7f       	mov    $0x7ffe0300,%ecx
    call *%ecx
77ed70f1:	ff d1                	call   *%ecx
    ret $0x8
77ed70f3:	c2 08 00             	ret    $0x8

77ed70f6 <_NtUserSetProcessWindowStation@4>:

.global _NtUserSetProcessWindowStation@4
_NtUserSetProcessWindowStation@4:

    movl $0x11ea, %eax
77ed70f6:	b8 ea 11 00 00       	mov    $0x11ea,%eax
    movl $KUSER_SHARED_SYSCALL, %ecx
77ed70fb:	b9 00 03 fe 7f       	mov    $0x7ffe0300,%ecx
    call *%ecx
77ed7100:	ff d1                	call   *%ecx
    ret $0x4
77ed7102:	c2 04 00             	ret    $0x4

77ed7105 <_NtUserSetProp@12>:

.global _NtUserSetProp@12
_NtUserSetProp@12:

    movl $0x11eb, %eax
77ed7105:	b8 eb 11 00 00       	mov    $0x11eb,%eax
    movl $KUSER_SHARED_SYSCALL, %ecx
77ed710a:	b9 00 03 fe 7f       	mov    $0x7ffe0300,%ecx
    call *%ecx
77ed710f:	ff d1                	call   *%ecx
    ret $0xc
77ed7111:	c2 0c 00             	ret    $0xc

77ed7114 <_NtUserSetRipFlags@8>:

.global _NtUserSetRipFlags@8
_NtUserSetRipFlags@8:

    movl $0x11ec, %eax
77ed7114:	b8 ec 11 00 00       	mov    $0x11ec,%eax
    movl $KUSER_SHARED_SYSCALL, %ecx
77ed7119:	b9 00 03 fe 7f       	mov    $0x7ffe0300,%ecx
    call *%ecx
77ed711e:	ff d1                	call   *%ecx
    ret $0x8
77ed7120:	c2 08 00             	ret    $0x8

77ed7123 <_NtUserSetScrollBarInfo@12>:

.global _NtUserSetScrollBarInfo@12
_NtUserSetScrollBarInfo@12:

    movl $0x11ed, %eax
77ed7123:	b8 ed 11 00 00       	mov    $0x11ed,%eax
    movl $KUSER_SHARED_SYSCALL, %ecx
77ed7128:	b9 00 03 fe 7f       	mov    $0x7ffe0300,%ecx
    call *%ecx
77ed712d:	ff d1                	call   *%ecx
    ret $0xc
77ed712f:	c2 0c 00             	ret    $0xc

77ed7132 <_NtUserSetScrollInfo@16>:

.global _NtUserSetScrollInfo@16
_NtUserSetScrollInfo@16:

    movl $0x11ee, %eax
77ed7132:	b8 ee 11 00 00       	mov    $0x11ee,%eax
    movl $KUSER_SHARED_SYSCALL, %ecx
77ed7137:	b9 00 03 fe 7f       	mov    $0x7ffe0300,%ecx
    call *%ecx
77ed713c:	ff d1                	call   *%ecx
    ret $0x10
77ed713e:	c2 10 00             	ret    $0x10

77ed7141 <_NtUserSetShellWindowEx@8>:

.global _NtUserSetShellWindowEx@8
_NtUserSetShellWindowEx@8:

    movl $0x11ef, %eax
77ed7141:	b8 ef 11 00 00       	mov    $0x11ef,%eax
    movl $KUSER_SHARED_SYSCALL, %ecx
77ed7146:	b9 00 03 fe 7f       	mov    $0x7ffe0300,%ecx
    call *%ecx
77ed714b:	ff d1                	call   *%ecx
    ret $0x8
77ed714d:	c2 08 00             	ret    $0x8

77ed7150 <_NtUserSetSysColors@16>:

.global _NtUserSetSysColors@16
_NtUserSetSysColors@16:

    movl $0x11f0, %eax
77ed7150:	b8 f0 11 00 00       	mov    $0x11f0,%eax
    movl $KUSER_SHARED_SYSCALL, %ecx
77ed7155:	b9 00 03 fe 7f       	mov    $0x7ffe0300,%ecx
    call *%ecx
77ed715a:	ff d1                	call   *%ecx
    ret $0x10
77ed715c:	c2 10 00             	ret    $0x10

77ed715f <_NtUserSetSystemCursor@8>:

.global _NtUserSetSystemCursor@8
_NtUserSetSystemCursor@8:

    movl $0x11f1, %eax
77ed715f:	b8 f1 11 00 00       	mov    $0x11f1,%eax
    movl $KUSER_SHARED_SYSCALL, %ecx
77ed7164:	b9 00 03 fe 7f       	mov    $0x7ffe0300,%ecx
    call *%ecx
77ed7169:	ff d1                	call   *%ecx
    ret $0x8
77ed716b:	c2 08 00             	ret    $0x8

77ed716e <_NtUserSetSystemMenu@8>:

.global _NtUserSetSystemMenu@8
_NtUserSetSystemMenu@8:

    movl $0x11f2, %eax
77ed716e:	b8 f2 11 00 00       	mov    $0x11f2,%eax
    movl $KUSER_SHARED_SYSCALL, %ecx
77ed7173:	b9 00 03 fe 7f       	mov    $0x7ffe0300,%ecx
    call *%ecx
77ed7178:	ff d1                	call   *%ecx
    ret $0x8
77ed717a:	c2 08 00             	ret    $0x8

77ed717d <_NtUserSetSystemTimer@16>:

.global _NtUserSetSystemTimer@16
_NtUserSetSystemTimer@16:

    movl $0x11f3, %eax
77ed717d:	b8 f3 11 00 00       	mov    $0x11f3,%eax
    movl $KUSER_SHARED_SYSCALL, %ecx
77ed7182:	b9 00 03 fe 7f       	mov    $0x7ffe0300,%ecx
    call *%ecx
77ed7187:	ff d1                	call   *%ecx
    ret $0x10
77ed7189:	c2 10 00             	ret    $0x10

77ed718c <_NtUserSetThreadDesktop@4>:

.global _NtUserSetThreadDesktop@4
_NtUserSetThreadDesktop@4:

    movl $0x11f4, %eax
77ed718c:	b8 f4 11 00 00       	mov    $0x11f4,%eax
    movl $KUSER_SHARED_SYSCALL, %ecx
77ed7191:	b9 00 03 fe 7f       	mov    $0x7ffe0300,%ecx
    call *%ecx
77ed7196:	ff d1                	call   *%ecx
    ret $0x4
77ed7198:	c2 04 00             	ret    $0x4

77ed719b <_NtUserSetThreadState@8>:

.global _NtUserSetThreadState@8
_NtUserSetThreadState@8:

    movl $0x11f5, %eax
77ed719b:	b8 f5 11 00 00       	mov    $0x11f5,%eax
    movl $KUSER_SHARED_SYSCALL, %ecx
77ed71a0:	b9 00 03 fe 7f       	mov    $0x7ffe0300,%ecx
    call *%ecx
77ed71a5:	ff d1                	call   *%ecx
    ret $0x8
77ed71a7:	c2 08 00             	ret    $0x8

77ed71aa <_NtUserSetTimer@16>:

.global _NtUserSetTimer@16
_NtUserSetTimer@16:

    movl $0x11f6, %eax
77ed71aa:	b8 f6 11 00 00       	mov    $0x11f6,%eax
    movl $KUSER_SHARED_SYSCALL, %ecx
77ed71af:	b9 00 03 fe 7f       	mov    $0x7ffe0300,%ecx
    call *%ecx
77ed71b4:	ff d1                	call   *%ecx
    ret $0x10
77ed71b6:	c2 10 00             	ret    $0x10

77ed71b9 <_NtUserSetWindowFNID@8>:

.global _NtUserSetWindowFNID@8
_NtUserSetWindowFNID@8:

    movl $0x11f7, %eax
77ed71b9:	b8 f7 11 00 00       	mov    $0x11f7,%eax
    movl $KUSER_SHARED_SYSCALL, %ecx
77ed71be:	b9 00 03 fe 7f       	mov    $0x7ffe0300,%ecx
    call *%ecx
77ed71c3:	ff d1                	call   *%ecx
    ret $0x8
77ed71c5:	c2 08 00             	ret    $0x8

77ed71c8 <_NtUserSetWindowLong@16>:

.global _NtUserSetWindowLong@16
_NtUserSetWindowLong@16:

    movl $0x11f8, %eax
77ed71c8:	b8 f8 11 00 00       	mov    $0x11f8,%eax
    movl $KUSER_SHARED_SYSCALL, %ecx
77ed71cd:	b9 00 03 fe 7f       	mov    $0x7ffe0300,%ecx
    call *%ecx
77ed71d2:	ff d1                	call   *%ecx
    ret $0x10
77ed71d4:	c2 10 00             	ret    $0x10

77ed71d7 <_NtUserSetWindowPlacement@8>:

.global _NtUserSetWindowPlacement@8
_NtUserSetWindowPlacement@8:

    movl $0x11f9, %eax
77ed71d7:	b8 f9 11 00 00       	mov    $0x11f9,%eax
    movl $KUSER_SHARED_SYSCALL, %ecx
77ed71dc:	b9 00 03 fe 7f       	mov    $0x7ffe0300,%ecx
    call *%ecx
77ed71e1:	ff d1                	call   *%ecx
    ret $0x8
77ed71e3:	c2 08 00             	ret    $0x8

77ed71e6 <_NtUserSetWindowPos@28>:

.global _NtUserSetWindowPos@28
_NtUserSetWindowPos@28:

    movl $0x11fa, %eax
77ed71e6:	b8 fa 11 00 00       	mov    $0x11fa,%eax
    movl $KUSER_SHARED_SYSCALL, %ecx
77ed71eb:	b9 00 03 fe 7f       	mov    $0x7ffe0300,%ecx
    call *%ecx
77ed71f0:	ff d1                	call   *%ecx
    ret $0x1c
77ed71f2:	c2 1c 00             	ret    $0x1c

77ed71f5 <_NtUserSetWindowRgn@12>:

.global _NtUserSetWindowRgn@12
_NtUserSetWindowRgn@12:

    movl $0x11fb, %eax
77ed71f5:	b8 fb 11 00 00       	mov    $0x11fb,%eax
    movl $KUSER_SHARED_SYSCALL, %ecx
77ed71fa:	b9 00 03 fe 7f       	mov    $0x7ffe0300,%ecx
    call *%ecx
77ed71ff:	ff d1                	call   *%ecx
    ret $0xc
77ed7201:	c2 0c 00             	ret    $0xc

77ed7204 <_NtUserSetWindowsHookAW@12>:

.global _NtUserSetWindowsHookAW@12
_NtUserSetWindowsHookAW@12:

    movl $0x11fc, %eax
77ed7204:	b8 fc 11 00 00       	mov    $0x11fc,%eax
    movl $KUSER_SHARED_SYSCALL, %ecx
77ed7209:	b9 00 03 fe 7f       	mov    $0x7ffe0300,%ecx
    call *%ecx
77ed720e:	ff d1                	call   *%ecx
    ret $0xc
77ed7210:	c2 0c 00             	ret    $0xc

77ed7213 <_NtUserSetWindowsHookEx@24>:

.global _NtUserSetWindowsHookEx@24
_NtUserSetWindowsHookEx@24:

    movl $0x11fd, %eax
77ed7213:	b8 fd 11 00 00       	mov    $0x11fd,%eax
    movl $KUSER_SHARED_SYSCALL, %ecx
77ed7218:	b9 00 03 fe 7f       	mov    $0x7ffe0300,%ecx
    call *%ecx
77ed721d:	ff d1                	call   *%ecx
    ret $0x18
77ed721f:	c2 18 00             	ret    $0x18

77ed7222 <_NtUserSetWindowStationUser@16>:

.global _NtUserSetWindowStationUser@16
_NtUserSetWindowStationUser@16:

    movl $0x11fe, %eax
77ed7222:	b8 fe 11 00 00       	mov    $0x11fe,%eax
    movl $KUSER_SHARED_SYSCALL, %ecx
77ed7227:	b9 00 03 fe 7f       	mov    $0x7ffe0300,%ecx
    call *%ecx
77ed722c:	ff d1                	call   *%ecx
    ret $0x10
77ed722e:	c2 10 00             	ret    $0x10

77ed7231 <_NtUserSetWindowWord@12>:

.global _NtUserSetWindowWord@12
_NtUserSetWindowWord@12:

    movl $0x11ff, %eax
77ed7231:	b8 ff 11 00 00       	mov    $0x11ff,%eax
    movl $KUSER_SHARED_SYSCALL, %ecx
77ed7236:	b9 00 03 fe 7f       	mov    $0x7ffe0300,%ecx
    call *%ecx
77ed723b:	ff d1                	call   *%ecx
    ret $0xc
77ed723d:	c2 0c 00             	ret    $0xc

77ed7240 <_NtUserSetWinEventHook@32>:

.global _NtUserSetWinEventHook@32
_NtUserSetWinEventHook@32:

    movl $0x1200, %eax
77ed7240:	b8 00 12 00 00       	mov    $0x1200,%eax
    movl $KUSER_SHARED_SYSCALL, %ecx
77ed7245:	b9 00 03 fe 7f       	mov    $0x7ffe0300,%ecx
    call *%ecx
77ed724a:	ff d1                	call   *%ecx
    ret $0x20
77ed724c:	c2 20 00             	ret    $0x20

77ed724f <_NtUserShowCaret@4>:

.global _NtUserShowCaret@4
_NtUserShowCaret@4:

    movl $0x1201, %eax
77ed724f:	b8 01 12 00 00       	mov    $0x1201,%eax
    movl $KUSER_SHARED_SYSCALL, %ecx
77ed7254:	b9 00 03 fe 7f       	mov    $0x7ffe0300,%ecx
    call *%ecx
77ed7259:	ff d1                	call   *%ecx
    ret $0x4
77ed725b:	c2 04 00             	ret    $0x4

77ed725e <_NtUserShowScrollBar@12>:

.global _NtUserShowScrollBar@12
_NtUserShowScrollBar@12:

    movl $0x1202, %eax
77ed725e:	b8 02 12 00 00       	mov    $0x1202,%eax
    movl $KUSER_SHARED_SYSCALL, %ecx
77ed7263:	b9 00 03 fe 7f       	mov    $0x7ffe0300,%ecx
    call *%ecx
77ed7268:	ff d1                	call   *%ecx
    ret $0xc
77ed726a:	c2 0c 00             	ret    $0xc

77ed726d <_NtUserShowWindow@8>:

.global _NtUserShowWindow@8
_NtUserShowWindow@8:

    movl $0x1203, %eax
77ed726d:	b8 03 12 00 00       	mov    $0x1203,%eax
    movl $KUSER_SHARED_SYSCALL, %ecx
77ed7272:	b9 00 03 fe 7f       	mov    $0x7ffe0300,%ecx
    call *%ecx
77ed7277:	ff d1                	call   *%ecx
    ret $0x8
77ed7279:	c2 08 00             	ret    $0x8

77ed727c <_NtUserShowWindowAsync@8>:

.global _NtUserShowWindowAsync@8
_NtUserShowWindowAsync@8:

    movl $0x1204, %eax
77ed727c:	b8 04 12 00 00       	mov    $0x1204,%eax
    movl $KUSER_SHARED_SYSCALL, %ecx
77ed7281:	b9 00 03 fe 7f       	mov    $0x7ffe0300,%ecx
    call *%ecx
77ed7286:	ff d1                	call   *%ecx
    ret $0x8
77ed7288:	c2 08 00             	ret    $0x8

77ed728b <_NtUserSwitchDesktop@4>:

.global _NtUserSwitchDesktop@4
_NtUserSwitchDesktop@4:

    movl $0x1205, %eax
77ed728b:	b8 05 12 00 00       	mov    $0x1205,%eax
    movl $KUSER_SHARED_SYSCALL, %ecx
77ed7290:	b9 00 03 fe 7f       	mov    $0x7ffe0300,%ecx
    call *%ecx
77ed7295:	ff d1                	call   *%ecx
    ret $0x4
77ed7297:	c2 04 00             	ret    $0x4

77ed729a <_NtUserSystemParametersInfo@16>:

.global _NtUserSystemParametersInfo@16
_NtUserSystemParametersInfo@16:

    movl $0x1206, %eax
77ed729a:	b8 06 12 00 00       	mov    $0x1206,%eax
    movl $KUSER_SHARED_SYSCALL, %ecx
77ed729f:	b9 00 03 fe 7f       	mov    $0x7ffe0300,%ecx
    call *%ecx
77ed72a4:	ff d1                	call   *%ecx
    ret $0x10
77ed72a6:	c2 10 00             	ret    $0x10

77ed72a9 <_NtUserThunkedMenuInfo@8>:

.global _NtUserThunkedMenuInfo@8
_NtUserThunkedMenuInfo@8:

    movl $0x1207, %eax
77ed72a9:	b8 07 12 00 00       	mov    $0x1207,%eax
    movl $KUSER_SHARED_SYSCALL, %ecx
77ed72ae:	b9 00 03 fe 7f       	mov    $0x7ffe0300,%ecx
    call *%ecx
77ed72b3:	ff d1                	call   *%ecx
    ret $0x8
77ed72b5:	c2 08 00             	ret    $0x8

77ed72b8 <_NtUserThunkedMenuItemInfo@24>:

.global _NtUserThunkedMenuItemInfo@24
_NtUserThunkedMenuItemInfo@24:

    movl $0x1208, %eax
77ed72b8:	b8 08 12 00 00       	mov    $0x1208,%eax
    movl $KUSER_SHARED_SYSCALL, %ecx
77ed72bd:	b9 00 03 fe 7f       	mov    $0x7ffe0300,%ecx
    call *%ecx
77ed72c2:	ff d1                	call   *%ecx
    ret $0x18
77ed72c4:	c2 18 00             	ret    $0x18

77ed72c7 <_NtUserToUnicodeEx@28>:

.global _NtUserToUnicodeEx@28
_NtUserToUnicodeEx@28:

    movl $0x1209, %eax
77ed72c7:	b8 09 12 00 00       	mov    $0x1209,%eax
    movl $KUSER_SHARED_SYSCALL, %ecx
77ed72cc:	b9 00 03 fe 7f       	mov    $0x7ffe0300,%ecx
    call *%ecx
77ed72d1:	ff d1                	call   *%ecx
    ret $0x1c
77ed72d3:	c2 1c 00             	ret    $0x1c

77ed72d6 <_NtUserTrackMouseEvent@4>:

.global _NtUserTrackMouseEvent@4
_NtUserTrackMouseEvent@4:

    movl $0x120a, %eax
77ed72d6:	b8 0a 12 00 00       	mov    $0x120a,%eax
    movl $KUSER_SHARED_SYSCALL, %ecx
77ed72db:	b9 00 03 fe 7f       	mov    $0x7ffe0300,%ecx
    call *%ecx
77ed72e0:	ff d1                	call   *%ecx
    ret $0x4
77ed72e2:	c2 04 00             	ret    $0x4

77ed72e5 <_NtUserTrackPopupMenuEx@24>:

.global _NtUserTrackPopupMenuEx@24
_NtUserTrackPopupMenuEx@24:

    movl $0x120b, %eax
77ed72e5:	b8 0b 12 00 00       	mov    $0x120b,%eax
    movl $KUSER_SHARED_SYSCALL, %ecx
77ed72ea:	b9 00 03 fe 7f       	mov    $0x7ffe0300,%ecx
    call *%ecx
77ed72ef:	ff d1                	call   *%ecx
    ret $0x18
77ed72f1:	c2 18 00             	ret    $0x18

77ed72f4 <_NtUserTranslateAccelerator@12>:

.global _NtUserTranslateAccelerator@12
_NtUserTranslateAccelerator@12:

    movl $0x120c, %eax
77ed72f4:	b8 0c 12 00 00       	mov    $0x120c,%eax
    movl $KUSER_SHARED_SYSCALL, %ecx
77ed72f9:	b9 00 03 fe 7f       	mov    $0x7ffe0300,%ecx
    call *%ecx
77ed72fe:	ff d1                	call   *%ecx
    ret $0xc
77ed7300:	c2 0c 00             	ret    $0xc

77ed7303 <_NtUserTranslateMessage@8>:

.global _NtUserTranslateMessage@8
_NtUserTranslateMessage@8:

    movl $0x120d, %eax
77ed7303:	b8 0d 12 00 00       	mov    $0x120d,%eax
    movl $KUSER_SHARED_SYSCALL, %ecx
77ed7308:	b9 00 03 fe 7f       	mov    $0x7ffe0300,%ecx
    call *%ecx
77ed730d:	ff d1                	call   *%ecx
    ret $0x8
77ed730f:	c2 08 00             	ret    $0x8

77ed7312 <_NtUserUnhookWindowsHookEx@4>:

.global _NtUserUnhookWindowsHookEx@4
_NtUserUnhookWindowsHookEx@4:

    movl $0x120e, %eax
77ed7312:	b8 0e 12 00 00       	mov    $0x120e,%eax
    movl $KUSER_SHARED_SYSCALL, %ecx
77ed7317:	b9 00 03 fe 7f       	mov    $0x7ffe0300,%ecx
    call *%ecx
77ed731c:	ff d1                	call   *%ecx
    ret $0x4
77ed731e:	c2 04 00             	ret    $0x4

77ed7321 <_NtUserUnhookWinEvent@4>:

.global _NtUserUnhookWinEvent@4
_NtUserUnhookWinEvent@4:

    movl $0x120f, %eax
77ed7321:	b8 0f 12 00 00       	mov    $0x120f,%eax
    movl $KUSER_SHARED_SYSCALL, %ecx
77ed7326:	b9 00 03 fe 7f       	mov    $0x7ffe0300,%ecx
    call *%ecx
77ed732b:	ff d1                	call   *%ecx
    ret $0x4
77ed732d:	c2 04 00             	ret    $0x4

77ed7330 <_NtUserUnloadKeyboardLayout@4>:

.global _NtUserUnloadKeyboardLayout@4
_NtUserUnloadKeyboardLayout@4:

    movl $0x1210, %eax
77ed7330:	b8 10 12 00 00       	mov    $0x1210,%eax
    movl $KUSER_SHARED_SYSCALL, %ecx
77ed7335:	b9 00 03 fe 7f       	mov    $0x7ffe0300,%ecx
    call *%ecx
77ed733a:	ff d1                	call   *%ecx
    ret $0x4
77ed733c:	c2 04 00             	ret    $0x4

77ed733f <_NtUserUnlockWindowStation@4>:

.global _NtUserUnlockWindowStation@4
_NtUserUnlockWindowStation@4:

    movl $0x1211, %eax
77ed733f:	b8 11 12 00 00       	mov    $0x1211,%eax
    movl $KUSER_SHARED_SYSCALL, %ecx
77ed7344:	b9 00 03 fe 7f       	mov    $0x7ffe0300,%ecx
    call *%ecx
77ed7349:	ff d1                	call   *%ecx
    ret $0x4
77ed734b:	c2 04 00             	ret    $0x4

77ed734e <_NtUserUnregisterClass@12>:

.global _NtUserUnregisterClass@12
_NtUserUnregisterClass@12:

    movl $0x1212, %eax
77ed734e:	b8 12 12 00 00       	mov    $0x1212,%eax
    movl $KUSER_SHARED_SYSCALL, %ecx
77ed7353:	b9 00 03 fe 7f       	mov    $0x7ffe0300,%ecx
    call *%ecx
77ed7358:	ff d1                	call   *%ecx
    ret $0xc
77ed735a:	c2 0c 00             	ret    $0xc

77ed735d <_NtUserUnregisterHotKey@8>:

.global _NtUserUnregisterHotKey@8
_NtUserUnregisterHotKey@8:

    movl $0x1213, %eax
77ed735d:	b8 13 12 00 00       	mov    $0x1213,%eax
    movl $KUSER_SHARED_SYSCALL, %ecx
77ed7362:	b9 00 03 fe 7f       	mov    $0x7ffe0300,%ecx
    call *%ecx
77ed7367:	ff d1                	call   *%ecx
    ret $0x8
77ed7369:	c2 08 00             	ret    $0x8

77ed736c <_NtUserUpdateInputContext@12>:

.global _NtUserUpdateInputContext@12
_NtUserUpdateInputContext@12:

    movl $0x1214, %eax
77ed736c:	b8 14 12 00 00       	mov    $0x1214,%eax
    movl $KUSER_SHARED_SYSCALL, %ecx
77ed7371:	b9 00 03 fe 7f       	mov    $0x7ffe0300,%ecx
    call *%ecx
77ed7376:	ff d1                	call   *%ecx
    ret $0xc
77ed7378:	c2 0c 00             	ret    $0xc

77ed737b <_NtUserUpdateInstance@12>:

.global _NtUserUpdateInstance@12
_NtUserUpdateInstance@12:

    movl $0x1215, %eax
77ed737b:	b8 15 12 00 00       	mov    $0x1215,%eax
    movl $KUSER_SHARED_SYSCALL, %ecx
77ed7380:	b9 00 03 fe 7f       	mov    $0x7ffe0300,%ecx
    call *%ecx
77ed7385:	ff d1                	call   *%ecx
    ret $0xc
77ed7387:	c2 0c 00             	ret    $0xc

77ed738a <_NtUserUpdateWindow@4>:

.global _NtUserUpdateWindow@4
_NtUserUpdateWindow@4:

    movl $0x1216, %eax
77ed738a:	b8 16 12 00 00       	mov    $0x1216,%eax
    movl $KUSER_SHARED_SYSCALL, %ecx
77ed738f:	b9 00 03 fe 7f       	mov    $0x7ffe0300,%ecx
    call *%ecx
77ed7394:	ff d1                	call   *%ecx
    ret $0x4
77ed7396:	c2 04 00             	ret    $0x4

77ed7399 <_NtUserUpdateLayeredWindow@36>:

.global _NtUserUpdateLayeredWindow@36
_NtUserUpdateLayeredWindow@36:

    movl $0x1217, %eax
77ed7399:	b8 17 12 00 00       	mov    $0x1217,%eax
    movl $KUSER_SHARED_SYSCALL, %ecx
77ed739e:	b9 00 03 fe 7f       	mov    $0x7ffe0300,%ecx
    call *%ecx
77ed73a3:	ff d1                	call   *%ecx
    ret $0x24
77ed73a5:	c2 24 00             	ret    $0x24

77ed73a8 <_NtUserUpdatePerUserSystemParameters@8>:

.global _NtUserUpdatePerUserSystemParameters@8
_NtUserUpdatePerUserSystemParameters@8:

    movl $0x1218, %eax
77ed73a8:	b8 18 12 00 00       	mov    $0x1218,%eax
    movl $KUSER_SHARED_SYSCALL, %ecx
77ed73ad:	b9 00 03 fe 7f       	mov    $0x7ffe0300,%ecx
    call *%ecx
77ed73b2:	ff d1                	call   *%ecx
    ret $0x8
77ed73b4:	c2 08 00             	ret    $0x8

77ed73b7 <_NtUserUserHandleGrantAccess@12>:

.global _NtUserUserHandleGrantAccess@12
_NtUserUserHandleGrantAccess@12:

    movl $0x1219, %eax
77ed73b7:	b8 19 12 00 00       	mov    $0x1219,%eax
    movl $KUSER_SHARED_SYSCALL, %ecx
77ed73bc:	b9 00 03 fe 7f       	mov    $0x7ffe0300,%ecx
    call *%ecx
77ed73c1:	ff d1                	call   *%ecx
    ret $0xc
77ed73c3:	c2 0c 00             	ret    $0xc

77ed73c6 <_NtUserValidateHandleSecure@4>:

.global _NtUserValidateHandleSecure@4
_NtUserValidateHandleSecure@4:

    movl $0x121a, %eax
77ed73c6:	b8 1a 12 00 00       	mov    $0x121a,%eax
    movl $KUSER_SHARED_SYSCALL, %ecx
77ed73cb:	b9 00 03 fe 7f       	mov    $0x7ffe0300,%ecx
    call *%ecx
77ed73d0:	ff d1                	call   *%ecx
    ret $0x4
77ed73d2:	c2 04 00             	ret    $0x4

77ed73d5 <_NtUserValidateRect@8>:

.global _NtUserValidateRect@8
_NtUserValidateRect@8:

    movl $0x121b, %eax
77ed73d5:	b8 1b 12 00 00       	mov    $0x121b,%eax
    movl $KUSER_SHARED_SYSCALL, %ecx
77ed73da:	b9 00 03 fe 7f       	mov    $0x7ffe0300,%ecx
    call *%ecx
77ed73df:	ff d1                	call   *%ecx
    ret $0x8
77ed73e1:	c2 08 00             	ret    $0x8

77ed73e4 <_NtUserVkKeyScanEx@12>:

.global _NtUserVkKeyScanEx@12
_NtUserVkKeyScanEx@12:

    movl $0x121c, %eax
77ed73e4:	b8 1c 12 00 00       	mov    $0x121c,%eax
    movl $KUSER_SHARED_SYSCALL, %ecx
77ed73e9:	b9 00 03 fe 7f       	mov    $0x7ffe0300,%ecx
    call *%ecx
77ed73ee:	ff d1                	call   *%ecx
    ret $0xc
77ed73f0:	c2 0c 00             	ret    $0xc

77ed73f3 <_NtUserWaitForInputIdle@12>:

.global _NtUserWaitForInputIdle@12
_NtUserWaitForInputIdle@12:

    movl $0x121d, %eax
77ed73f3:	b8 1d 12 00 00       	mov    $0x121d,%eax
    movl $KUSER_SHARED_SYSCALL, %ecx
77ed73f8:	b9 00 03 fe 7f       	mov    $0x7ffe0300,%ecx
    call *%ecx
77ed73fd:	ff d1                	call   *%ecx
    ret $0xc
77ed73ff:	c2 0c 00             	ret    $0xc

77ed7402 <_NtUserWaitForMsgAndEvent@4>:

.global _NtUserWaitForMsgAndEvent@4
_NtUserWaitForMsgAndEvent@4:

    movl $0x121e, %eax
77ed7402:	b8 1e 12 00 00       	mov    $0x121e,%eax
    movl $KUSER_SHARED_SYSCALL, %ecx
77ed7407:	b9 00 03 fe 7f       	mov    $0x7ffe0300,%ecx
    call *%ecx
77ed740c:	ff d1                	call   *%ecx
    ret $0x4
77ed740e:	c2 04 00             	ret    $0x4

77ed7411 <_NtUserWaitMessage@0>:

.global _NtUserWaitMessage@0
_NtUserWaitMessage@0:

    movl $0x121f, %eax
77ed7411:	b8 1f 12 00 00       	mov    $0x121f,%eax
    movl $KUSER_SHARED_SYSCALL, %ecx
77ed7416:	b9 00 03 fe 7f       	mov    $0x7ffe0300,%ecx
    call *%ecx
77ed741b:	ff d1                	call   *%ecx
    ret $0x0
77ed741d:	c2 00 00             	ret    $0x0

77ed7420 <_NtUserWin32PoolAllocationStats@24>:

.global _NtUserWin32PoolAllocationStats@24
_NtUserWin32PoolAllocationStats@24:

    movl $0x1220, %eax
77ed7420:	b8 20 12 00 00       	mov    $0x1220,%eax
    movl $KUSER_SHARED_SYSCALL, %ecx
77ed7425:	b9 00 03 fe 7f       	mov    $0x7ffe0300,%ecx
    call *%ecx
77ed742a:	ff d1                	call   *%ecx
    ret $0x18
77ed742c:	c2 18 00             	ret    $0x18

77ed742f <_NtUserWindowFromPoint@8>:

.global _NtUserWindowFromPoint@8
_NtUserWindowFromPoint@8:

    movl $0x1221, %eax
77ed742f:	b8 21 12 00 00       	mov    $0x1221,%eax
    movl $KUSER_SHARED_SYSCALL, %ecx
77ed7434:	b9 00 03 fe 7f       	mov    $0x7ffe0300,%ecx
    call *%ecx
77ed7439:	ff d1                	call   *%ecx
    ret $0x8
77ed743b:	c2 08 00             	ret    $0x8

77ed743e <_NtUserYieldTask@0>:

.global _NtUserYieldTask@0
_NtUserYieldTask@0:

    movl $0x1222, %eax
77ed743e:	b8 22 12 00 00       	mov    $0x1222,%eax
    movl $KUSER_SHARED_SYSCALL, %ecx
77ed7443:	b9 00 03 fe 7f       	mov    $0x7ffe0300,%ecx
    call *%ecx
77ed7448:	ff d1                	call   *%ecx
    ret $0x0
77ed744a:	c2 00 00             	ret    $0x0

77ed744d <_NtUserGetDesktopWindow@0>:

.global _NtUserGetDesktopWindow@0
_NtUserGetDesktopWindow@0:

    movl $0x1223, %eax
77ed744d:	b8 23 12 00 00       	mov    $0x1223,%eax
    movl $KUSER_SHARED_SYSCALL, %ecx
77ed7452:	b9 00 03 fe 7f       	mov    $0x7ffe0300,%ecx
    call *%ecx
77ed7457:	ff d1                	call   *%ecx
    ret $0x0
77ed7459:	c2 00 00             	ret    $0x0

77ed745c <_NtUserAcquireOrReleaseInputOwnership@4>:

.global _NtUserAcquireOrReleaseInputOwnership@4
_NtUserAcquireOrReleaseInputOwnership@4:

    movl $0x1224, %eax
77ed745c:	b8 24 12 00 00       	mov    $0x1224,%eax
    movl $KUSER_SHARED_SYSCALL, %ecx
77ed7461:	b9 00 03 fe 7f       	mov    $0x7ffe0300,%ecx
    call *%ecx
77ed7466:	ff d1                	call   *%ecx
    ret $0x4
77ed7468:	c2 04 00             	ret    $0x4

77ed746b <_NtUserGetWindowThreadProcessId@8>:

.global _NtUserGetWindowThreadProcessId@8
_NtUserGetWindowThreadProcessId@8:

    movl $0x1225, %eax
77ed746b:	b8 25 12 00 00       	mov    $0x1225,%eax
    movl $KUSER_SHARED_SYSCALL, %ecx
77ed7470:	b9 00 03 fe 7f       	mov    $0x7ffe0300,%ecx
    call *%ecx
77ed7475:	ff d1                	call   *%ecx
    ret $0x8
77ed7477:	c2 08 00             	ret    $0x8

77ed747a <_NtUserGetQueueStatus@4>:

.global _NtUserGetQueueStatus@4
_NtUserGetQueueStatus@4:

    movl $0x1226, %eax
77ed747a:	b8 26 12 00 00       	mov    $0x1226,%eax
    movl $KUSER_SHARED_SYSCALL, %ecx
77ed747f:	b9 00 03 fe 7f       	mov    $0x7ffe0300,%ecx
    call *%ecx
77ed7484:	ff d1                	call   *%ecx
    ret $0x4
77ed7486:	c2 04 00             	ret    $0x4

77ed7489 <_NtUserGetParent@4>:

.global _NtUserGetParent@4
_NtUserGetParent@4:

    movl $0x1227, %eax
77ed7489:	b8 27 12 00 00       	mov    $0x1227,%eax
    movl $KUSER_SHARED_SYSCALL, %ecx
77ed748e:	b9 00 03 fe 7f       	mov    $0x7ffe0300,%ecx
    call *%ecx
77ed7493:	ff d1                	call   *%ecx
    ret $0x4
77ed7495:	c2 04 00             	ret    $0x4

77ed7498 <_NtUserGetWindow@8>:

.global _NtUserGetWindow@8
_NtUserGetWindow@8:

    movl $0x1228, %eax
77ed7498:	b8 28 12 00 00       	mov    $0x1228,%eax
    movl $KUSER_SHARED_SYSCALL, %ecx
77ed749d:	b9 00 03 fe 7f       	mov    $0x7ffe0300,%ecx
    call *%ecx
77ed74a2:	ff d1                	call   *%ecx
    ret $0x8
77ed74a4:	c2 08 00             	ret    $0x8

77ed74a7 <_NtUserGetLastActivePopup@4>:

.global _NtUserGetLastActivePopup@4
_NtUserGetLastActivePopup@4:

    movl $0x1229, %eax
77ed74a7:	b8 29 12 00 00       	mov    $0x1229,%eax
    movl $KUSER_SHARED_SYSCALL, %ecx
77ed74ac:	b9 00 03 fe 7f       	mov    $0x7ffe0300,%ecx
    call *%ecx
77ed74b1:	ff d1                	call   *%ecx
    ret $0x4
77ed74b3:	c2 04 00             	ret    $0x4

77ed74b6 <_NtUserGetShellWindow@0>:

.global _NtUserGetShellWindow@0
_NtUserGetShellWindow@0:

    movl $0x122a, %eax
77ed74b6:	b8 2a 12 00 00       	mov    $0x122a,%eax
    movl $KUSER_SHARED_SYSCALL, %ecx
77ed74bb:	b9 00 03 fe 7f       	mov    $0x7ffe0300,%ecx
    call *%ecx
77ed74c0:	ff d1                	call   *%ecx
    ret $0x0
77ed74c2:	c2 00 00             	ret    $0x0

77ed74c5 <_NtUserDereferenceWndProcHandle@8>:

.global _NtUserDereferenceWndProcHandle@8
_NtUserDereferenceWndProcHandle@8:

    movl $0x122b, %eax
77ed74c5:	b8 2b 12 00 00       	mov    $0x122b,%eax
    movl $KUSER_SHARED_SYSCALL, %ecx
77ed74ca:	b9 00 03 fe 7f       	mov    $0x7ffe0300,%ecx
    call *%ecx
77ed74cf:	ff d1                	call   *%ecx
    ret $0x8
77ed74d1:	c2 08 00             	ret    $0x8

77ed74d4 <_NtUserManualGuiCheck@4>:

.global _NtUserManualGuiCheck@4
_NtUserManualGuiCheck@4:

    movl $0x122c, %eax
77ed74d4:	b8 2c 12 00 00       	mov    $0x122c,%eax
    movl $KUSER_SHARED_SYSCALL, %ecx
77ed74d9:	b9 00 03 fe 7f       	mov    $0x7ffe0300,%ecx
    call *%ecx
77ed74de:	ff d1                	call   *%ecx
    ret $0x4
77ed74e0:	c2 04 00             	ret    $0x4

77ed74e3 <_NtGdiD3dContextCreate@16>:

.global _NtGdiD3dContextCreate@16
_NtGdiD3dContextCreate@16:

    movl $0x122d, %eax
77ed74e3:	b8 2d 12 00 00       	mov    $0x122d,%eax
    movl $KUSER_SHARED_SYSCALL, %ecx
77ed74e8:	b9 00 03 fe 7f       	mov    $0x7ffe0300,%ecx
    call *%ecx
77ed74ed:	ff d1                	call   *%ecx
    ret $0x10
77ed74ef:	c2 10 00             	ret    $0x10

77ed74f2 <_NtGdiD3dContextDestroy@4>:

.global _NtGdiD3dContextDestroy@4
_NtGdiD3dContextDestroy@4:

    movl $0x122e, %eax
77ed74f2:	b8 2e 12 00 00       	mov    $0x122e,%eax
    movl $KUSER_SHARED_SYSCALL, %ecx
77ed74f7:	b9 00 03 fe 7f       	mov    $0x7ffe0300,%ecx
    call *%ecx
77ed74fc:	ff d1                	call   *%ecx
    ret $0x4
77ed74fe:	c2 04 00             	ret    $0x4

77ed7501 <_NtGdiD3dContextDestroyAll@4>:

.global _NtGdiD3dContextDestroyAll@4
_NtGdiD3dContextDestroyAll@4:

    movl $0x122f, %eax
77ed7501:	b8 2f 12 00 00       	mov    $0x122f,%eax
    movl $KUSER_SHARED_SYSCALL, %ecx
77ed7506:	b9 00 03 fe 7f       	mov    $0x7ffe0300,%ecx
    call *%ecx
77ed750b:	ff d1                	call   *%ecx
    ret $0x4
77ed750d:	c2 04 00             	ret    $0x4

77ed7510 <_NtGdiD3dDrawPrimitives2@28>:

.global _NtGdiD3dDrawPrimitives2@28
_NtGdiD3dDrawPrimitives2@28:

    movl $0x1230, %eax
77ed7510:	b8 30 12 00 00       	mov    $0x1230,%eax
    movl $KUSER_SHARED_SYSCALL, %ecx
77ed7515:	b9 00 03 fe 7f       	mov    $0x7ffe0300,%ecx
    call *%ecx
77ed751a:	ff d1                	call   *%ecx
    ret $0x1c
77ed751c:	c2 1c 00             	ret    $0x1c

77ed751f <_NtGdiD3dValidateTextureStageState@4>:

.global _NtGdiD3dValidateTextureStageState@4
_NtGdiD3dValidateTextureStageState@4:

    movl $0x1231, %eax
77ed751f:	b8 31 12 00 00       	mov    $0x1231,%eax
    movl $KUSER_SHARED_SYSCALL, %ecx
77ed7524:	b9 00 03 fe 7f       	mov    $0x7ffe0300,%ecx
    call *%ecx
77ed7529:	ff d1                	call   *%ecx
    ret $0x4
77ed752b:	c2 04 00             	ret    $0x4

77ed752e <_NtGdiDdAddAttachedSurface@12>:

.global _NtGdiDdAddAttachedSurface@12
_NtGdiDdAddAttachedSurface@12:

    movl $0x1232, %eax
77ed752e:	b8 32 12 00 00       	mov    $0x1232,%eax
    movl $KUSER_SHARED_SYSCALL, %ecx
77ed7533:	b9 00 03 fe 7f       	mov    $0x7ffe0300,%ecx
    call *%ecx
77ed7538:	ff d1                	call   *%ecx
    ret $0xc
77ed753a:	c2 0c 00             	ret    $0xc

77ed753d <_NtGdiDdAlphaBlt@12>:

.global _NtGdiDdAlphaBlt@12
_NtGdiDdAlphaBlt@12:

    movl $0x1233, %eax
77ed753d:	b8 33 12 00 00       	mov    $0x1233,%eax
    movl $KUSER_SHARED_SYSCALL, %ecx
77ed7542:	b9 00 03 fe 7f       	mov    $0x7ffe0300,%ecx
    call *%ecx
77ed7547:	ff d1                	call   *%ecx
    ret $0xc
77ed7549:	c2 0c 00             	ret    $0xc

77ed754c <_NtGdiDdAttachSurface@8>:

.global _NtGdiDdAttachSurface@8
_NtGdiDdAttachSurface@8:

    movl $0x1234, %eax
77ed754c:	b8 34 12 00 00       	mov    $0x1234,%eax
    movl $KUSER_SHARED_SYSCALL, %ecx
77ed7551:	b9 00 03 fe 7f       	mov    $0x7ffe0300,%ecx
    call *%ecx
77ed7556:	ff d1                	call   *%ecx
    ret $0x8
77ed7558:	c2 08 00             	ret    $0x8

77ed755b <_NtGdiDdBeginMoCompFrame@8>:

.global _NtGdiDdBeginMoCompFrame@8
_NtGdiDdBeginMoCompFrame@8:

    movl $0x1235, %eax
77ed755b:	b8 35 12 00 00       	mov    $0x1235,%eax
    movl $KUSER_SHARED_SYSCALL, %ecx
77ed7560:	b9 00 03 fe 7f       	mov    $0x7ffe0300,%ecx
    call *%ecx
77ed7565:	ff d1                	call   *%ecx
    ret $0x8
77ed7567:	c2 08 00             	ret    $0x8

77ed756a <_NtGdiDdBlt@12>:

.global _NtGdiDdBlt@12
_NtGdiDdBlt@12:

    movl $0x1236, %eax
77ed756a:	b8 36 12 00 00       	mov    $0x1236,%eax
    movl $KUSER_SHARED_SYSCALL, %ecx
77ed756f:	b9 00 03 fe 7f       	mov    $0x7ffe0300,%ecx
    call *%ecx
77ed7574:	ff d1                	call   *%ecx
    ret $0xc
77ed7576:	c2 0c 00             	ret    $0xc

77ed7579 <_NtGdiDdCanCreateD3DBuffer@8>:

.global _NtGdiDdCanCreateD3DBuffer@8
_NtGdiDdCanCreateD3DBuffer@8:

    movl $0x1237, %eax
77ed7579:	b8 37 12 00 00       	mov    $0x1237,%eax
    movl $KUSER_SHARED_SYSCALL, %ecx
77ed757e:	b9 00 03 fe 7f       	mov    $0x7ffe0300,%ecx
    call *%ecx
77ed7583:	ff d1                	call   *%ecx
    ret $0x8
77ed7585:	c2 08 00             	ret    $0x8

77ed7588 <_NtGdiDdCanCreateSurface@8>:

.global _NtGdiDdCanCreateSurface@8
_NtGdiDdCanCreateSurface@8:

    movl $0x1238, %eax
77ed7588:	b8 38 12 00 00       	mov    $0x1238,%eax
    movl $KUSER_SHARED_SYSCALL, %ecx
77ed758d:	b9 00 03 fe 7f       	mov    $0x7ffe0300,%ecx
    call *%ecx
77ed7592:	ff d1                	call   *%ecx
    ret $0x8
77ed7594:	c2 08 00             	ret    $0x8

77ed7597 <_NtGdiDdColorControl@8>:

.global _NtGdiDdColorControl@8
_NtGdiDdColorControl@8:

    movl $0x1239, %eax
77ed7597:	b8 39 12 00 00       	mov    $0x1239,%eax
    movl $KUSER_SHARED_SYSCALL, %ecx
77ed759c:	b9 00 03 fe 7f       	mov    $0x7ffe0300,%ecx
    call *%ecx
77ed75a1:	ff d1                	call   *%ecx
    ret $0x8
77ed75a3:	c2 08 00             	ret    $0x8

77ed75a6 <_NtGdiDdCreateD3DBuffer@32>:

.global _NtGdiDdCreateD3DBuffer@32
_NtGdiDdCreateD3DBuffer@32:

    movl $0x123a, %eax
77ed75a6:	b8 3a 12 00 00       	mov    $0x123a,%eax
    movl $KUSER_SHARED_SYSCALL, %ecx
77ed75ab:	b9 00 03 fe 7f       	mov    $0x7ffe0300,%ecx
    call *%ecx
77ed75b0:	ff d1                	call   *%ecx
    ret $0x20
77ed75b2:	c2 20 00             	ret    $0x20

77ed75b5 <_NtGdiDdCreateDirectDrawObject@4>:

.global _NtGdiDdCreateDirectDrawObject@4
_NtGdiDdCreateDirectDrawObject@4:

    movl $0x123b, %eax
77ed75b5:	b8 3b 12 00 00       	mov    $0x123b,%eax
    movl $KUSER_SHARED_SYSCALL, %ecx
77ed75ba:	b9 00 03 fe 7f       	mov    $0x7ffe0300,%ecx
    call *%ecx
77ed75bf:	ff d1                	call   *%ecx
    ret $0x4
77ed75c1:	c2 04 00             	ret    $0x4

77ed75c4 <_NtGdiDdCreateMoComp@8>:

.global _NtGdiDdCreateMoComp@8
_NtGdiDdCreateMoComp@8:

    movl $0x123c, %eax
77ed75c4:	b8 3c 12 00 00       	mov    $0x123c,%eax
    movl $KUSER_SHARED_SYSCALL, %ecx
77ed75c9:	b9 00 03 fe 7f       	mov    $0x7ffe0300,%ecx
    call *%ecx
77ed75ce:	ff d1                	call   *%ecx
    ret $0x8
77ed75d0:	c2 08 00             	ret    $0x8

77ed75d3 <_NtGdiDdCreateSurface@32>:

.global _NtGdiDdCreateSurface@32
_NtGdiDdCreateSurface@32:

    movl $0x123d, %eax
77ed75d3:	b8 3d 12 00 00       	mov    $0x123d,%eax
    movl $KUSER_SHARED_SYSCALL, %ecx
77ed75d8:	b9 00 03 fe 7f       	mov    $0x7ffe0300,%ecx
    call *%ecx
77ed75dd:	ff d1                	call   *%ecx
    ret $0x20
77ed75df:	c2 20 00             	ret    $0x20

77ed75e2 <_NtGdiDdCreateSurfaceEx@12>:

.global _NtGdiDdCreateSurfaceEx@12
_NtGdiDdCreateSurfaceEx@12:

    movl $0x123e, %eax
77ed75e2:	b8 3e 12 00 00       	mov    $0x123e,%eax
    movl $KUSER_SHARED_SYSCALL, %ecx
77ed75e7:	b9 00 03 fe 7f       	mov    $0x7ffe0300,%ecx
    call *%ecx
77ed75ec:	ff d1                	call   *%ecx
    ret $0xc
77ed75ee:	c2 0c 00             	ret    $0xc

77ed75f1 <_NtGdiDdCreateSurfaceObject@24>:

.global _NtGdiDdCreateSurfaceObject@24
_NtGdiDdCreateSurfaceObject@24:

    movl $0x123f, %eax
77ed75f1:	b8 3f 12 00 00       	mov    $0x123f,%eax
    movl $KUSER_SHARED_SYSCALL, %ecx
77ed75f6:	b9 00 03 fe 7f       	mov    $0x7ffe0300,%ecx
    call *%ecx
77ed75fb:	ff d1                	call   *%ecx
    ret $0x18
77ed75fd:	c2 18 00             	ret    $0x18

77ed7600 <_NtGdiDdDeleteDirectDrawObject@4>:

.global _NtGdiDdDeleteDirectDrawObject@4
_NtGdiDdDeleteDirectDrawObject@4:

    movl $0x1240, %eax
77ed7600:	b8 40 12 00 00       	mov    $0x1240,%eax
    movl $KUSER_SHARED_SYSCALL, %ecx
77ed7605:	b9 00 03 fe 7f       	mov    $0x7ffe0300,%ecx
    call *%ecx
77ed760a:	ff d1                	call   *%ecx
    ret $0x4
77ed760c:	c2 04 00             	ret    $0x4

77ed760f <_NtGdiDdDeleteSurfaceObject@4>:

.global _NtGdiDdDeleteSurfaceObject@4
_NtGdiDdDeleteSurfaceObject@4:

    movl $0x1241, %eax
77ed760f:	b8 41 12 00 00       	mov    $0x1241,%eax
    movl $KUSER_SHARED_SYSCALL, %ecx
77ed7614:	b9 00 03 fe 7f       	mov    $0x7ffe0300,%ecx
    call *%ecx
77ed7619:	ff d1                	call   *%ecx
    ret $0x4
77ed761b:	c2 04 00             	ret    $0x4

77ed761e <_NtGdiDdDestroyD3DBuffer@4>:

.global _NtGdiDdDestroyD3DBuffer@4
_NtGdiDdDestroyD3DBuffer@4:

    movl $0x1242, %eax
77ed761e:	b8 42 12 00 00       	mov    $0x1242,%eax
    movl $KUSER_SHARED_SYSCALL, %ecx
77ed7623:	b9 00 03 fe 7f       	mov    $0x7ffe0300,%ecx
    call *%ecx
77ed7628:	ff d1                	call   *%ecx
    ret $0x4
77ed762a:	c2 04 00             	ret    $0x4

77ed762d <_NtGdiDdDestroyMoComp@8>:

.global _NtGdiDdDestroyMoComp@8
_NtGdiDdDestroyMoComp@8:

    movl $0x1243, %eax
77ed762d:	b8 43 12 00 00       	mov    $0x1243,%eax
    movl $KUSER_SHARED_SYSCALL, %ecx
77ed7632:	b9 00 03 fe 7f       	mov    $0x7ffe0300,%ecx
    call *%ecx
77ed7637:	ff d1                	call   *%ecx
    ret $0x8
77ed7639:	c2 08 00             	ret    $0x8

77ed763c <_NtGdiDdDestroySurface@8>:

.global _NtGdiDdDestroySurface@8
_NtGdiDdDestroySurface@8:

    movl $0x1244, %eax
77ed763c:	b8 44 12 00 00       	mov    $0x1244,%eax
    movl $KUSER_SHARED_SYSCALL, %ecx
77ed7641:	b9 00 03 fe 7f       	mov    $0x7ffe0300,%ecx
    call *%ecx
77ed7646:	ff d1                	call   *%ecx
    ret $0x8
77ed7648:	c2 08 00             	ret    $0x8

77ed764b <_NtGdiDdEndMoCompFrame@8>:

.global _NtGdiDdEndMoCompFrame@8
_NtGdiDdEndMoCompFrame@8:

    movl $0x1245, %eax
77ed764b:	b8 45 12 00 00       	mov    $0x1245,%eax
    movl $KUSER_SHARED_SYSCALL, %ecx
77ed7650:	b9 00 03 fe 7f       	mov    $0x7ffe0300,%ecx
    call *%ecx
77ed7655:	ff d1                	call   *%ecx
    ret $0x8
77ed7657:	c2 08 00             	ret    $0x8

77ed765a <_NtGdiDdFlip@20>:

.global _NtGdiDdFlip@20
_NtGdiDdFlip@20:

    movl $0x1246, %eax
77ed765a:	b8 46 12 00 00       	mov    $0x1246,%eax
    movl $KUSER_SHARED_SYSCALL, %ecx
77ed765f:	b9 00 03 fe 7f       	mov    $0x7ffe0300,%ecx
    call *%ecx
77ed7664:	ff d1                	call   *%ecx
    ret $0x14
77ed7666:	c2 14 00             	ret    $0x14

77ed7669 <_NtGdiDdFlipToGDISurface@8>:

.global _NtGdiDdFlipToGDISurface@8
_NtGdiDdFlipToGDISurface@8:

    movl $0x1247, %eax
77ed7669:	b8 47 12 00 00       	mov    $0x1247,%eax
    movl $KUSER_SHARED_SYSCALL, %ecx
77ed766e:	b9 00 03 fe 7f       	mov    $0x7ffe0300,%ecx
    call *%ecx
77ed7673:	ff d1                	call   *%ecx
    ret $0x8
77ed7675:	c2 08 00             	ret    $0x8

77ed7678 <_NtGdiDdGetAvailDriverMemory@8>:

.global _NtGdiDdGetAvailDriverMemory@8
_NtGdiDdGetAvailDriverMemory@8:

    movl $0x1248, %eax
77ed7678:	b8 48 12 00 00       	mov    $0x1248,%eax
    movl $KUSER_SHARED_SYSCALL, %ecx
77ed767d:	b9 00 03 fe 7f       	mov    $0x7ffe0300,%ecx
    call *%ecx
77ed7682:	ff d1                	call   *%ecx
    ret $0x8
77ed7684:	c2 08 00             	ret    $0x8

77ed7687 <_NtGdiDdGetBltStatus@8>:

.global _NtGdiDdGetBltStatus@8
_NtGdiDdGetBltStatus@8:

    movl $0x1249, %eax
77ed7687:	b8 49 12 00 00       	mov    $0x1249,%eax
    movl $KUSER_SHARED_SYSCALL, %ecx
77ed768c:	b9 00 03 fe 7f       	mov    $0x7ffe0300,%ecx
    call *%ecx
77ed7691:	ff d1                	call   *%ecx
    ret $0x8
77ed7693:	c2 08 00             	ret    $0x8

77ed7696 <_NtGdiDdGetDC@8>:

.global _NtGdiDdGetDC@8
_NtGdiDdGetDC@8:

    movl $0x124a, %eax
77ed7696:	b8 4a 12 00 00       	mov    $0x124a,%eax
    movl $KUSER_SHARED_SYSCALL, %ecx
77ed769b:	b9 00 03 fe 7f       	mov    $0x7ffe0300,%ecx
    call *%ecx
77ed76a0:	ff d1                	call   *%ecx
    ret $0x8
77ed76a2:	c2 08 00             	ret    $0x8

77ed76a5 <_NtGdiDdGetDriverInfo@8>:

.global _NtGdiDdGetDriverInfo@8
_NtGdiDdGetDriverInfo@8:

    movl $0x124b, %eax
77ed76a5:	b8 4b 12 00 00       	mov    $0x124b,%eax
    movl $KUSER_SHARED_SYSCALL, %ecx
77ed76aa:	b9 00 03 fe 7f       	mov    $0x7ffe0300,%ecx
    call *%ecx
77ed76af:	ff d1                	call   *%ecx
    ret $0x8
77ed76b1:	c2 08 00             	ret    $0x8

77ed76b4 <_NtGdiDdGetDriverState@4>:

.global _NtGdiDdGetDriverState@4
_NtGdiDdGetDriverState@4:

    movl $0x124c, %eax
77ed76b4:	b8 4c 12 00 00       	mov    $0x124c,%eax
    movl $KUSER_SHARED_SYSCALL, %ecx
77ed76b9:	b9 00 03 fe 7f       	mov    $0x7ffe0300,%ecx
    call *%ecx
77ed76be:	ff d1                	call   *%ecx
    ret $0x4
77ed76c0:	c2 04 00             	ret    $0x4

77ed76c3 <_NtGdiDdGetDxHandle@12>:

.global _NtGdiDdGetDxHandle@12
_NtGdiDdGetDxHandle@12:

    movl $0x124d, %eax
77ed76c3:	b8 4d 12 00 00       	mov    $0x124d,%eax
    movl $KUSER_SHARED_SYSCALL, %ecx
77ed76c8:	b9 00 03 fe 7f       	mov    $0x7ffe0300,%ecx
    call *%ecx
77ed76cd:	ff d1                	call   *%ecx
    ret $0xc
77ed76cf:	c2 0c 00             	ret    $0xc

77ed76d2 <_NtGdiDdGetFlipStatus@8>:

.global _NtGdiDdGetFlipStatus@8
_NtGdiDdGetFlipStatus@8:

    movl $0x124e, %eax
77ed76d2:	b8 4e 12 00 00       	mov    $0x124e,%eax
    movl $KUSER_SHARED_SYSCALL, %ecx
77ed76d7:	b9 00 03 fe 7f       	mov    $0x7ffe0300,%ecx
    call *%ecx
77ed76dc:	ff d1                	call   *%ecx
    ret $0x8
77ed76de:	c2 08 00             	ret    $0x8

77ed76e1 <_NtGdiDdGetInternalMoCompInfo@8>:

.global _NtGdiDdGetInternalMoCompInfo@8
_NtGdiDdGetInternalMoCompInfo@8:

    movl $0x124f, %eax
77ed76e1:	b8 4f 12 00 00       	mov    $0x124f,%eax
    movl $KUSER_SHARED_SYSCALL, %ecx
77ed76e6:	b9 00 03 fe 7f       	mov    $0x7ffe0300,%ecx
    call *%ecx
77ed76eb:	ff d1                	call   *%ecx
    ret $0x8
77ed76ed:	c2 08 00             	ret    $0x8

77ed76f0 <_NtGdiDdGetMoCompBuffInfo@8>:

.global _NtGdiDdGetMoCompBuffInfo@8
_NtGdiDdGetMoCompBuffInfo@8:

    movl $0x1250, %eax
77ed76f0:	b8 50 12 00 00       	mov    $0x1250,%eax
    movl $KUSER_SHARED_SYSCALL, %ecx
77ed76f5:	b9 00 03 fe 7f       	mov    $0x7ffe0300,%ecx
    call *%ecx
77ed76fa:	ff d1                	call   *%ecx
    ret $0x8
77ed76fc:	c2 08 00             	ret    $0x8

77ed76ff <_NtGdiDdGetMoCompFormats@8>:

.global _NtGdiDdGetMoCompFormats@8
_NtGdiDdGetMoCompFormats@8:

    movl $0x1251, %eax
77ed76ff:	b8 51 12 00 00       	mov    $0x1251,%eax
    movl $KUSER_SHARED_SYSCALL, %ecx
77ed7704:	b9 00 03 fe 7f       	mov    $0x7ffe0300,%ecx
    call *%ecx
77ed7709:	ff d1                	call   *%ecx
    ret $0x8
77ed770b:	c2 08 00             	ret    $0x8

77ed770e <_NtGdiDdGetMoCompGuids@8>:

.global _NtGdiDdGetMoCompGuids@8
_NtGdiDdGetMoCompGuids@8:

    movl $0x1252, %eax
77ed770e:	b8 52 12 00 00       	mov    $0x1252,%eax
    movl $KUSER_SHARED_SYSCALL, %ecx
77ed7713:	b9 00 03 fe 7f       	mov    $0x7ffe0300,%ecx
    call *%ecx
77ed7718:	ff d1                	call   *%ecx
    ret $0x8
77ed771a:	c2 08 00             	ret    $0x8

77ed771d <_NtGdiDdGetScanLine@8>:

.global _NtGdiDdGetScanLine@8
_NtGdiDdGetScanLine@8:

    movl $0x1253, %eax
77ed771d:	b8 53 12 00 00       	mov    $0x1253,%eax
    movl $KUSER_SHARED_SYSCALL, %ecx
77ed7722:	b9 00 03 fe 7f       	mov    $0x7ffe0300,%ecx
    call *%ecx
77ed7727:	ff d1                	call   *%ecx
    ret $0x8
77ed7729:	c2 08 00             	ret    $0x8

77ed772c <_NtGdiDdLock@12>:

.global _NtGdiDdLock@12
_NtGdiDdLock@12:

    movl $0x1254, %eax
77ed772c:	b8 54 12 00 00       	mov    $0x1254,%eax
    movl $KUSER_SHARED_SYSCALL, %ecx
77ed7731:	b9 00 03 fe 7f       	mov    $0x7ffe0300,%ecx
    call *%ecx
77ed7736:	ff d1                	call   *%ecx
    ret $0xc
77ed7738:	c2 0c 00             	ret    $0xc

77ed773b <_NtGdiDdLockD3D@8>:

.global _NtGdiDdLockD3D@8
_NtGdiDdLockD3D@8:

    movl $0x1255, %eax
77ed773b:	b8 55 12 00 00       	mov    $0x1255,%eax
    movl $KUSER_SHARED_SYSCALL, %ecx
77ed7740:	b9 00 03 fe 7f       	mov    $0x7ffe0300,%ecx
    call *%ecx
77ed7745:	ff d1                	call   *%ecx
    ret $0x8
77ed7747:	c2 08 00             	ret    $0x8

77ed774a <_NtGdiDdQueryDirectDrawObject@44>:

.global _NtGdiDdQueryDirectDrawObject@44
_NtGdiDdQueryDirectDrawObject@44:

    movl $0x1256, %eax
77ed774a:	b8 56 12 00 00       	mov    $0x1256,%eax
    movl $KUSER_SHARED_SYSCALL, %ecx
77ed774f:	b9 00 03 fe 7f       	mov    $0x7ffe0300,%ecx
    call *%ecx
77ed7754:	ff d1                	call   *%ecx
    ret $0x2c
77ed7756:	c2 2c 00             	ret    $0x2c

77ed7759 <_NtGdiDdQueryMoCompStatus@8>:

.global _NtGdiDdQueryMoCompStatus@8
_NtGdiDdQueryMoCompStatus@8:

    movl $0x1257, %eax
77ed7759:	b8 57 12 00 00       	mov    $0x1257,%eax
    movl $KUSER_SHARED_SYSCALL, %ecx
77ed775e:	b9 00 03 fe 7f       	mov    $0x7ffe0300,%ecx
    call *%ecx
77ed7763:	ff d1                	call   *%ecx
    ret $0x8
77ed7765:	c2 08 00             	ret    $0x8

77ed7768 <_NtGdiDdReenableDirectDrawObject@8>:

.global _NtGdiDdReenableDirectDrawObject@8
_NtGdiDdReenableDirectDrawObject@8:

    movl $0x1258, %eax
77ed7768:	b8 58 12 00 00       	mov    $0x1258,%eax
    movl $KUSER_SHARED_SYSCALL, %ecx
77ed776d:	b9 00 03 fe 7f       	mov    $0x7ffe0300,%ecx
    call *%ecx
77ed7772:	ff d1                	call   *%ecx
    ret $0x8
77ed7774:	c2 08 00             	ret    $0x8

77ed7777 <_NtGdiDdReleaseDC@4>:

.global _NtGdiDdReleaseDC@4
_NtGdiDdReleaseDC@4:

    movl $0x1259, %eax
77ed7777:	b8 59 12 00 00       	mov    $0x1259,%eax
    movl $KUSER_SHARED_SYSCALL, %ecx
77ed777c:	b9 00 03 fe 7f       	mov    $0x7ffe0300,%ecx
    call *%ecx
77ed7781:	ff d1                	call   *%ecx
    ret $0x4
77ed7783:	c2 04 00             	ret    $0x4

77ed7786 <_NtGdiDdRenderMoComp@8>:

.global _NtGdiDdRenderMoComp@8
_NtGdiDdRenderMoComp@8:

    movl $0x125a, %eax
77ed7786:	b8 5a 12 00 00       	mov    $0x125a,%eax
    movl $KUSER_SHARED_SYSCALL, %ecx
77ed778b:	b9 00 03 fe 7f       	mov    $0x7ffe0300,%ecx
    call *%ecx
77ed7790:	ff d1                	call   *%ecx
    ret $0x8
77ed7792:	c2 08 00             	ret    $0x8

77ed7795 <_NtGdiDdResetVisrgn@8>:

.global _NtGdiDdResetVisrgn@8
_NtGdiDdResetVisrgn@8:

    movl $0x125b, %eax
77ed7795:	b8 5b 12 00 00       	mov    $0x125b,%eax
    movl $KUSER_SHARED_SYSCALL, %ecx
77ed779a:	b9 00 03 fe 7f       	mov    $0x7ffe0300,%ecx
    call *%ecx
77ed779f:	ff d1                	call   *%ecx
    ret $0x8
77ed77a1:	c2 08 00             	ret    $0x8

77ed77a4 <_NtGdiDdSetColorKey@8>:

.global _NtGdiDdSetColorKey@8
_NtGdiDdSetColorKey@8:

    movl $0x125c, %eax
77ed77a4:	b8 5c 12 00 00       	mov    $0x125c,%eax
    movl $KUSER_SHARED_SYSCALL, %ecx
77ed77a9:	b9 00 03 fe 7f       	mov    $0x7ffe0300,%ecx
    call *%ecx
77ed77ae:	ff d1                	call   *%ecx
    ret $0x8
77ed77b0:	c2 08 00             	ret    $0x8

77ed77b3 <_NtGdiDdSetExclusiveMode@8>:

.global _NtGdiDdSetExclusiveMode@8
_NtGdiDdSetExclusiveMode@8:

    movl $0x125d, %eax
77ed77b3:	b8 5d 12 00 00       	mov    $0x125d,%eax
    movl $KUSER_SHARED_SYSCALL, %ecx
77ed77b8:	b9 00 03 fe 7f       	mov    $0x7ffe0300,%ecx
    call *%ecx
77ed77bd:	ff d1                	call   *%ecx
    ret $0x8
77ed77bf:	c2 08 00             	ret    $0x8

77ed77c2 <_NtGdiDdSetGammaRamp@12>:

.global _NtGdiDdSetGammaRamp@12
_NtGdiDdSetGammaRamp@12:

    movl $0x125e, %eax
77ed77c2:	b8 5e 12 00 00       	mov    $0x125e,%eax
    movl $KUSER_SHARED_SYSCALL, %ecx
77ed77c7:	b9 00 03 fe 7f       	mov    $0x7ffe0300,%ecx
    call *%ecx
77ed77cc:	ff d1                	call   *%ecx
    ret $0xc
77ed77ce:	c2 0c 00             	ret    $0xc

77ed77d1 <_NtGdiDdSetOverlayPosition@12>:

.global _NtGdiDdSetOverlayPosition@12
_NtGdiDdSetOverlayPosition@12:

    movl $0x125f, %eax
77ed77d1:	b8 5f 12 00 00       	mov    $0x125f,%eax
    movl $KUSER_SHARED_SYSCALL, %ecx
77ed77d6:	b9 00 03 fe 7f       	mov    $0x7ffe0300,%ecx
    call *%ecx
77ed77db:	ff d1                	call   *%ecx
    ret $0xc
77ed77dd:	c2 0c 00             	ret    $0xc

77ed77e0 <_NtGdiDdUnattachSurface@8>:

.global _NtGdiDdUnattachSurface@8
_NtGdiDdUnattachSurface@8:

    movl $0x1260, %eax
77ed77e0:	b8 60 12 00 00       	mov    $0x1260,%eax
    movl $KUSER_SHARED_SYSCALL, %ecx
77ed77e5:	b9 00 03 fe 7f       	mov    $0x7ffe0300,%ecx
    call *%ecx
77ed77ea:	ff d1                	call   *%ecx
    ret $0x8
77ed77ec:	c2 08 00             	ret    $0x8

77ed77ef <_NtGdiDdUnlock@8>:

.global _NtGdiDdUnlock@8
_NtGdiDdUnlock@8:

    movl $0x1261, %eax
77ed77ef:	b8 61 12 00 00       	mov    $0x1261,%eax
    movl $KUSER_SHARED_SYSCALL, %ecx
77ed77f4:	b9 00 03 fe 7f       	mov    $0x7ffe0300,%ecx
    call *%ecx
77ed77f9:	ff d1                	call   *%ecx
    ret $0x8
77ed77fb:	c2 08 00             	ret    $0x8

77ed77fe <_NtGdiDdUnlockD3D@8>:

.global _NtGdiDdUnlockD3D@8
_NtGdiDdUnlockD3D@8:

    movl $0x1262, %eax
77ed77fe:	b8 62 12 00 00       	mov    $0x1262,%eax
    movl $KUSER_SHARED_SYSCALL, %ecx
77ed7803:	b9 00 03 fe 7f       	mov    $0x7ffe0300,%ecx
    call *%ecx
77ed7808:	ff d1                	call   *%ecx
    ret $0x8
77ed780a:	c2 08 00             	ret    $0x8

77ed780d <_NtGdiDdUpdateOverlay@12>:

.global _NtGdiDdUpdateOverlay@12
_NtGdiDdUpdateOverlay@12:

    movl $0x1263, %eax
77ed780d:	b8 63 12 00 00       	mov    $0x1263,%eax
    movl $KUSER_SHARED_SYSCALL, %ecx
77ed7812:	b9 00 03 fe 7f       	mov    $0x7ffe0300,%ecx
    call *%ecx
77ed7817:	ff d1                	call   *%ecx
    ret $0xc
77ed7819:	c2 0c 00             	ret    $0xc

77ed781c <_NtGdiDdWaitForVerticalBlank@8>:

.global _NtGdiDdWaitForVerticalBlank@8
_NtGdiDdWaitForVerticalBlank@8:

    movl $0x1264, %eax
77ed781c:	b8 64 12 00 00       	mov    $0x1264,%eax
    movl $KUSER_SHARED_SYSCALL, %ecx
77ed7821:	b9 00 03 fe 7f       	mov    $0x7ffe0300,%ecx
    call *%ecx
77ed7826:	ff d1                	call   *%ecx
    ret $0x8
77ed7828:	c2 08 00             	ret    $0x8
77ed782b:	90                   	nop    
77ed782c:	90                   	nop    
77ed782d:	90                   	nop    
77ed782e:	90                   	nop    
77ed782f:	90                   	nop    

77ed7830 <_StretchBlt@44>:
77ed7830:	55                   	push   %ebp
77ed7831:	89 e5                	mov    %esp,%ebp
77ed7833:	57                   	push   %edi
77ed7834:	56                   	push   %esi
77ed7835:	53                   	push   %ebx
77ed7836:	83 ec 1c             	sub    $0x1c,%esp
77ed7839:	8b 45 08             	mov    0x8(%ebp),%eax
77ed783c:	8b 7d 14             	mov    0x14(%ebp),%edi
77ed783f:	89 45 f0             	mov    %eax,0xfffffff0(%ebp)
77ed7842:	8b 45 0c             	mov    0xc(%ebp),%eax
77ed7845:	89 45 ec             	mov    %eax,0xffffffec(%ebp)
77ed7848:	8b 45 10             	mov    0x10(%ebp),%eax
77ed784b:	89 45 e8             	mov    %eax,0xffffffe8(%ebp)
77ed784e:	8b 45 1c             	mov    0x1c(%ebp),%eax
77ed7851:	89 45 e4             	mov    %eax,0xffffffe4(%ebp)
77ed7854:	8b 45 20             	mov    0x20(%ebp),%eax
77ed7857:	89 45 e0             	mov    %eax,0xffffffe0(%ebp)
77ed785a:	8b 45 24             	mov    0x24(%ebp),%eax
77ed785d:	8b 5d 18             	mov    0x18(%ebp),%ebx
77ed7860:	89 45 dc             	mov    %eax,0xffffffdc(%ebp)
77ed7863:	8b 75 28             	mov    0x28(%ebp),%esi
77ed7866:	8b 45 30             	mov    0x30(%ebp),%eax
77ed7869:	8b 4d 2c             	mov    0x2c(%ebp),%ecx
77ed786c:	39 f7                	cmp    %esi,%edi
77ed786e:	89 45 d8             	mov    %eax,0xffffffd8(%ebp)
77ed7871:	0f 95 c2             	setne  %dl
77ed7874:	39 cb                	cmp    %ecx,%ebx
77ed7876:	0f 95 c0             	setne  %al
77ed7879:	09 d0                	or     %edx,%eax
77ed787b:	a8 01                	test   $0x1,%al
77ed787d:	74 11                	je     77ed7890 <_StretchBlt@44+0x60>
77ed787f:	8d 65 f4             	lea    0xfffffff4(%ebp),%esp
77ed7882:	5b                   	pop    %ebx
77ed7883:	5e                   	pop    %esi
77ed7884:	5f                   	pop    %edi
77ed7885:	5d                   	pop    %ebp
77ed7886:	e9 b5 ea ff ff       	jmp    77ed6340 <_NtGdiStretchBlt@44>
77ed788b:	90                   	nop    
77ed788c:	8d 74 26 00          	lea    0x0(%esi),%esi
77ed7890:	83 ec 0c             	sub    $0xc,%esp
77ed7893:	8b 45 d8             	mov    0xffffffd8(%ebp),%eax
77ed7896:	50                   	push   %eax
77ed7897:	8b 45 dc             	mov    0xffffffdc(%ebp),%eax
77ed789a:	50                   	push   %eax
77ed789b:	8b 45 e0             	mov    0xffffffe0(%ebp),%eax
77ed789e:	50                   	push   %eax
77ed789f:	8b 75 e4             	mov    0xffffffe4(%ebp),%esi
77ed78a2:	56                   	push   %esi
77ed78a3:	53                   	push   %ebx
77ed78a4:	57                   	push   %edi
77ed78a5:	8b 4d e8             	mov    0xffffffe8(%ebp),%ecx
77ed78a8:	51                   	push   %ecx
77ed78a9:	8b 55 ec             	mov    0xffffffec(%ebp),%edx
77ed78ac:	52                   	push   %edx
77ed78ad:	8b 45 f0             	mov    0xfffffff0(%ebp),%eax
77ed78b0:	50                   	push   %eax
77ed78b1:	e8 02 dc ff ff       	call   77ed54b8 <_NtGdiBitBlt@36>
77ed78b6:	8d 65 f4             	lea    0xfffffff4(%ebp),%esp
77ed78b9:	5b                   	pop    %ebx
77ed78ba:	5e                   	pop    %esi
77ed78bb:	5f                   	pop    %edi
77ed78bc:	5d                   	pop    %ebp
77ed78bd:	c2 2c 00             	ret    $0x2c

77ed78c0 <_CreateDCW@16>:
77ed78c0:	55                   	push   %ebp
77ed78c1:	89 e5                	mov    %esp,%ebp
77ed78c3:	57                   	push   %edi
77ed78c4:	56                   	push   %esi
77ed78c5:	53                   	push   %ebx
77ed78c6:	83 ec 1c             	sub    $0x1c,%esp
77ed78c9:	8b 7d 08             	mov    0x8(%ebp),%edi
77ed78cc:	8b 75 0c             	mov    0xc(%ebp),%esi
77ed78cf:	8b 5d 10             	mov    0x10(%ebp),%ebx
77ed78d2:	85 ff                	test   %edi,%edi
77ed78d4:	74 0e                	je     77ed78e4 <_CreateDCW@16+0x24>
77ed78d6:	8d 45 e8             	lea    0xffffffe8(%ebp),%eax
77ed78d9:	51                   	push   %ecx
77ed78da:	51                   	push   %ecx
77ed78db:	57                   	push   %edi
77ed78dc:	50                   	push   %eax
77ed78dd:	e8 6e 1f 00 00       	call   77ed9850 <_RtlInitUnicodeString@8>
77ed78e2:	58                   	pop    %eax
77ed78e3:	5a                   	pop    %edx
77ed78e4:	85 f6                	test   %esi,%esi
77ed78e6:	74 0e                	je     77ed78f6 <_CreateDCW@16+0x36>
77ed78e8:	8d 45 e8             	lea    0xffffffe8(%ebp),%eax
77ed78eb:	51                   	push   %ecx
77ed78ec:	51                   	push   %ecx
77ed78ed:	56                   	push   %esi
77ed78ee:	50                   	push   %eax
77ed78ef:	e8 5c 1f 00 00       	call   77ed9850 <_RtlInitUnicodeString@8>
77ed78f4:	58                   	pop    %eax
77ed78f5:	5a                   	pop    %edx
77ed78f6:	85 db                	test   %ebx,%ebx
77ed78f8:	74 0e                	je     77ed7908 <_CreateDCW@16+0x48>
77ed78fa:	50                   	push   %eax
77ed78fb:	50                   	push   %eax
77ed78fc:	8d 45 e8             	lea    0xffffffe8(%ebp),%eax
77ed78ff:	53                   	push   %ebx
77ed7900:	50                   	push   %eax
77ed7901:	e8 4a 1f 00 00       	call   77ed9850 <_RtlInitUnicodeString@8>
77ed7906:	5a                   	pop    %edx
77ed7907:	59                   	pop    %ecx
77ed7908:	8b 45 14             	mov    0x14(%ebp),%eax
77ed790b:	85 db                	test   %ebx,%ebx
77ed790d:	50                   	push   %eax
77ed790e:	8d 45 e0             	lea    0xffffffe0(%ebp),%eax
77ed7911:	74 20                	je     77ed7933 <_CreateDCW@16+0x73>
77ed7913:	50                   	push   %eax
77ed7914:	85 f6                	test   %esi,%esi
77ed7916:	8d 45 d8             	lea    0xffffffd8(%ebp),%eax
77ed7919:	74 25                	je     77ed7940 <_CreateDCW@16+0x80>
77ed791b:	50                   	push   %eax
77ed791c:	85 ff                	test   %edi,%edi
77ed791e:	8d 45 e8             	lea    0xffffffe8(%ebp),%eax
77ed7921:	74 2d                	je     77ed7950 <_CreateDCW@16+0x90>
77ed7923:	50                   	push   %eax
77ed7924:	e8 9d dc ff ff       	call   77ed55c6 <_NtGdiCreateDC@16>
77ed7929:	8d 65 f4             	lea    0xfffffff4(%ebp),%esp
77ed792c:	5b                   	pop    %ebx
77ed792d:	5e                   	pop    %esi
77ed792e:	5f                   	pop    %edi
77ed792f:	5d                   	pop    %ebp
77ed7930:	c2 10 00             	ret    $0x10
77ed7933:	31 c0                	xor    %eax,%eax
77ed7935:	85 f6                	test   %esi,%esi
77ed7937:	50                   	push   %eax
77ed7938:	8d 45 d8             	lea    0xffffffd8(%ebp),%eax
77ed793b:	75 de                	jne    77ed791b <_CreateDCW@16+0x5b>
77ed793d:	8d 76 00             	lea    0x0(%esi),%esi
77ed7940:	31 c0                	xor    %eax,%eax
77ed7942:	85 ff                	test   %edi,%edi
77ed7944:	50                   	push   %eax
77ed7945:	8d 45 e8             	lea    0xffffffe8(%ebp),%eax
77ed7948:	75 d9                	jne    77ed7923 <_CreateDCW@16+0x63>
77ed794a:	8d b6 00 00 00 00    	lea    0x0(%esi),%esi
77ed7950:	31 c0                	xor    %eax,%eax
77ed7952:	50                   	push   %eax
77ed7953:	e8 6e dc ff ff       	call   77ed55c6 <_NtGdiCreateDC@16>
77ed7958:	8d 65 f4             	lea    0xfffffff4(%ebp),%esp
77ed795b:	5b                   	pop    %ebx
77ed795c:	5e                   	pop    %esi
77ed795d:	5f                   	pop    %edi
77ed795e:	5d                   	pop    %ebp
77ed795f:	c2 10 00             	ret    $0x10
77ed7962:	8d b4 26 00 00 00 00 	lea    0x0(%esi),%esi
77ed7969:	8d bc 27 00 00 00 00 	lea    0x0(%edi),%edi

77ed7970 <_CreateDCA@16>:
77ed7970:	55                   	push   %ebp
77ed7971:	89 e5                	mov    %esp,%ebp
77ed7973:	57                   	push   %edi
77ed7974:	56                   	push   %esi
77ed7975:	53                   	push   %ebx
77ed7976:	83 ec 3c             	sub    $0x3c,%esp
77ed7979:	8b 45 08             	mov    0x8(%ebp),%eax
77ed797c:	8b 75 0c             	mov    0xc(%ebp),%esi
77ed797f:	85 c0                	test   %eax,%eax
77ed7981:	0f 84 a9 00 00 00    	je     77ed7a30 <_CreateDCA@16+0xc0>
77ed7987:	8d 5d e8             	lea    0xffffffe8(%ebp),%ebx
77ed798a:	57                   	push   %edi
77ed798b:	57                   	push   %edi
77ed798c:	50                   	push   %eax
77ed798d:	53                   	push   %ebx
77ed798e:	e8 cd 1e 00 00       	call   77ed9860 <_RtlInitAnsiString@8>
77ed7993:	8d 45 e0             	lea    0xffffffe0(%ebp),%eax
77ed7996:	c7 04 24 01 00 00 00 	movl   $0x1,(%esp)
77ed799d:	53                   	push   %ebx
77ed799e:	50                   	push   %eax
77ed799f:	e8 cc 1e 00 00       	call   77ed9870 <_RtlAnsiStringToUnicodeString@12>
77ed79a4:	85 f6                	test   %esi,%esi
77ed79a6:	5b                   	pop    %ebx
77ed79a7:	0f 84 92 00 00 00    	je     77ed7a3f <_CreateDCA@16+0xcf>
77ed79ad:	8d 5d d8             	lea    0xffffffd8(%ebp),%ebx
77ed79b0:	51                   	push   %ecx
77ed79b1:	51                   	push   %ecx
77ed79b2:	56                   	push   %esi
77ed79b3:	53                   	push   %ebx
77ed79b4:	e8 a7 1e 00 00       	call   77ed9860 <_RtlInitAnsiString@8>
77ed79b9:	8d 7d d0             	lea    0xffffffd0(%ebp),%edi
77ed79bc:	c7 04 24 01 00 00 00 	movl   $0x1,(%esp)
77ed79c3:	53                   	push   %ebx
77ed79c4:	57                   	push   %edi
77ed79c5:	e8 a6 1e 00 00       	call   77ed9870 <_RtlAnsiStringToUnicodeString@12>
77ed79ca:	8b 45 10             	mov    0x10(%ebp),%eax
77ed79cd:	5a                   	pop    %edx
77ed79ce:	85 c0                	test   %eax,%eax
77ed79d0:	74 7e                	je     77ed7a50 <_CreateDCA@16+0xe0>
77ed79d2:	8d 5d c8             	lea    0xffffffc8(%ebp),%ebx
77ed79d5:	50                   	push   %eax
77ed79d6:	50                   	push   %eax
77ed79d7:	8b 45 10             	mov    0x10(%ebp),%eax
77ed79da:	8d 75 c0             	lea    0xffffffc0(%ebp),%esi
77ed79dd:	50                   	push   %eax
77ed79de:	53                   	push   %ebx
77ed79df:	e8 7c 1e 00 00       	call   77ed9860 <_RtlInitAnsiString@8>
77ed79e4:	c7 04 24 01 00 00 00 	movl   $0x1,(%esp)
77ed79eb:	53                   	push   %ebx
77ed79ec:	56                   	push   %esi
77ed79ed:	e8 7e 1e 00 00       	call   77ed9870 <_RtlAnsiStringToUnicodeString@12>
77ed79f2:	58                   	pop    %eax
77ed79f3:	6a 00                	push   $0x0
77ed79f5:	8b 5d e4             	mov    0xffffffe4(%ebp),%ebx
77ed79f8:	8b 46 04             	mov    0x4(%esi),%eax
77ed79fb:	50                   	push   %eax
77ed79fc:	8b 47 04             	mov    0x4(%edi),%eax
77ed79ff:	50                   	push   %eax
77ed7a00:	53                   	push   %ebx
77ed7a01:	e8 ba fe ff ff       	call   77ed78c0 <_CreateDCW@16>
77ed7a06:	8d 55 e0             	lea    0xffffffe0(%ebp),%edx
77ed7a09:	83 ec 0c             	sub    $0xc,%esp
77ed7a0c:	89 c3                	mov    %eax,%ebx
77ed7a0e:	52                   	push   %edx
77ed7a0f:	e8 6c 1e 00 00       	call   77ed9880 <_RtlFreeUnicodeString@4>
77ed7a14:	57                   	push   %edi
77ed7a15:	e8 66 1e 00 00       	call   77ed9880 <_RtlFreeUnicodeString@4>
77ed7a1a:	56                   	push   %esi
77ed7a1b:	e8 60 1e 00 00       	call   77ed9880 <_RtlFreeUnicodeString@4>
77ed7a20:	8d 65 f4             	lea    0xfffffff4(%ebp),%esp
77ed7a23:	89 d8                	mov    %ebx,%eax
77ed7a25:	5b                   	pop    %ebx
77ed7a26:	5e                   	pop    %esi
77ed7a27:	5f                   	pop    %edi
77ed7a28:	5d                   	pop    %ebp
77ed7a29:	c2 10 00             	ret    $0x10
77ed7a2c:	8d 74 26 00          	lea    0x0(%esi),%esi
77ed7a30:	c7 45 e4 00 00 00 00 	movl   $0x0,0xffffffe4(%ebp)
77ed7a37:	85 f6                	test   %esi,%esi
77ed7a39:	0f 85 6e ff ff ff    	jne    77ed79ad <_CreateDCA@16+0x3d>
77ed7a3f:	8b 45 10             	mov    0x10(%ebp),%eax
77ed7a42:	8d 7d d0             	lea    0xffffffd0(%ebp),%edi
77ed7a45:	c7 45 d4 00 00 00 00 	movl   $0x0,0xffffffd4(%ebp)
77ed7a4c:	85 c0                	test   %eax,%eax
77ed7a4e:	75 82                	jne    77ed79d2 <_CreateDCA@16+0x62>
77ed7a50:	8d 75 c0             	lea    0xffffffc0(%ebp),%esi
77ed7a53:	c7 45 c4 00 00 00 00 	movl   $0x0,0xffffffc4(%ebp)
77ed7a5a:	eb 97                	jmp    77ed79f3 <_CreateDCA@16+0x83>
77ed7a5c:	8d 74 26 00          	lea    0x0(%esi),%esi

77ed7a60 <_CreateICW@16>:
77ed7a60:	55                   	push   %ebp
77ed7a61:	89 e5                	mov    %esp,%ebp
77ed7a63:	57                   	push   %edi
77ed7a64:	56                   	push   %esi
77ed7a65:	53                   	push   %ebx
77ed7a66:	83 ec 1c             	sub    $0x1c,%esp
77ed7a69:	8b 7d 08             	mov    0x8(%ebp),%edi
77ed7a6c:	8b 75 0c             	mov    0xc(%ebp),%esi
77ed7a6f:	8b 5d 10             	mov    0x10(%ebp),%ebx
77ed7a72:	85 ff                	test   %edi,%edi
77ed7a74:	74 0e                	je     77ed7a84 <_CreateICW@16+0x24>
77ed7a76:	8d 45 e8             	lea    0xffffffe8(%ebp),%eax
77ed7a79:	51                   	push   %ecx
77ed7a7a:	51                   	push   %ecx
77ed7a7b:	57                   	push   %edi
77ed7a7c:	50                   	push   %eax
77ed7a7d:	e8 ce 1d 00 00       	call   77ed9850 <_RtlInitUnicodeString@8>
77ed7a82:	58                   	pop    %eax
77ed7a83:	5a                   	pop    %edx
77ed7a84:	85 f6                	test   %esi,%esi
77ed7a86:	74 0e                	je     77ed7a96 <_CreateICW@16+0x36>
77ed7a88:	8d 45 e0             	lea    0xffffffe0(%ebp),%eax
77ed7a8b:	51                   	push   %ecx
77ed7a8c:	51                   	push   %ecx
77ed7a8d:	56                   	push   %esi
77ed7a8e:	50                   	push   %eax
77ed7a8f:	e8 bc 1d 00 00       	call   77ed9850 <_RtlInitUnicodeString@8>
77ed7a94:	58                   	pop    %eax
77ed7a95:	5a                   	pop    %edx
77ed7a96:	85 db                	test   %ebx,%ebx
77ed7a98:	74 0e                	je     77ed7aa8 <_CreateICW@16+0x48>
77ed7a9a:	8d 45 d8             	lea    0xffffffd8(%ebp),%eax
77ed7a9d:	51                   	push   %ecx
77ed7a9e:	51                   	push   %ecx
77ed7a9f:	53                   	push   %ebx
77ed7aa0:	50                   	push   %eax
77ed7aa1:	e8 aa 1d 00 00       	call   77ed9850 <_RtlInitUnicodeString@8>
77ed7aa6:	58                   	pop    %eax
77ed7aa7:	5a                   	pop    %edx
77ed7aa8:	8b 45 14             	mov    0x14(%ebp),%eax
77ed7aab:	85 db                	test   %ebx,%ebx
77ed7aad:	50                   	push   %eax
77ed7aae:	8d 45 d8             	lea    0xffffffd8(%ebp),%eax
77ed7ab1:	74 20                	je     77ed7ad3 <_CreateICW@16+0x73>
77ed7ab3:	50                   	push   %eax
77ed7ab4:	85 f6                	test   %esi,%esi
77ed7ab6:	8d 45 e0             	lea    0xffffffe0(%ebp),%eax
77ed7ab9:	74 25                	je     77ed7ae0 <_CreateICW@16+0x80>
77ed7abb:	50                   	push   %eax
77ed7abc:	85 ff                	test   %edi,%edi
77ed7abe:	8d 45 e8             	lea    0xffffffe8(%ebp),%eax
77ed7ac1:	74 2d                	je     77ed7af0 <_CreateICW@16+0x90>
77ed7ac3:	50                   	push   %eax
77ed7ac4:	e8 c0 db ff ff       	call   77ed5689 <_NtGdiCreateIC@16>
77ed7ac9:	8d 65 f4             	lea    0xfffffff4(%ebp),%esp
77ed7acc:	5b                   	pop    %ebx
77ed7acd:	5e                   	pop    %esi
77ed7ace:	5f                   	pop    %edi
77ed7acf:	5d                   	pop    %ebp
77ed7ad0:	c2 10 00             	ret    $0x10
77ed7ad3:	31 c0                	xor    %eax,%eax
77ed7ad5:	85 f6                	test   %esi,%esi
77ed7ad7:	50                   	push   %eax
77ed7ad8:	8d 45 e0             	lea    0xffffffe0(%ebp),%eax
77ed7adb:	75 de                	jne    77ed7abb <_CreateICW@16+0x5b>
77ed7add:	8d 76 00             	lea    0x0(%esi),%esi
77ed7ae0:	31 c0                	xor    %eax,%eax
77ed7ae2:	85 ff                	test   %edi,%edi
77ed7ae4:	50                   	push   %eax
77ed7ae5:	8d 45 e8             	lea    0xffffffe8(%ebp),%eax
77ed7ae8:	75 d9                	jne    77ed7ac3 <_CreateICW@16+0x63>
77ed7aea:	8d b6 00 00 00 00    	lea    0x0(%esi),%esi
77ed7af0:	31 c0                	xor    %eax,%eax
77ed7af2:	50                   	push   %eax
77ed7af3:	e8 91 db ff ff       	call   77ed5689 <_NtGdiCreateIC@16>
77ed7af8:	8d 65 f4             	lea    0xfffffff4(%ebp),%esp
77ed7afb:	5b                   	pop    %ebx
77ed7afc:	5e                   	pop    %esi
77ed7afd:	5f                   	pop    %edi
77ed7afe:	5d                   	pop    %ebp
77ed7aff:	c2 10 00             	ret    $0x10
77ed7b02:	8d b4 26 00 00 00 00 	lea    0x0(%esi),%esi
77ed7b09:	8d bc 27 00 00 00 00 	lea    0x0(%edi),%edi

77ed7b10 <_CreateICA@16>:
77ed7b10:	55                   	push   %ebp
77ed7b11:	89 e5                	mov    %esp,%ebp
77ed7b13:	57                   	push   %edi
77ed7b14:	56                   	push   %esi
77ed7b15:	53                   	push   %ebx
77ed7b16:	81 ec 24 01 00 00    	sub    $0x124,%esp
77ed7b1c:	8d 85 04 ff ff ff    	lea    0xffffff04(%ebp),%eax
77ed7b22:	8b 55 08             	mov    0x8(%ebp),%edx
77ed7b25:	8b 7d 14             	mov    0x14(%ebp),%edi
77ed7b28:	52                   	push   %edx
77ed7b29:	50                   	push   %eax
77ed7b2a:	e8 a1 95 ff ff       	call   77ed10d0 <_HEAP_strdupA2W>
77ed7b2f:	31 db                	xor    %ebx,%ebx
77ed7b31:	83 c4 10             	add    $0x10,%esp
77ed7b34:	85 c0                	test   %eax,%eax
77ed7b36:	0f 88 ec 00 00 00    	js     77ed7c28 <_CreateICA@16+0x118>
77ed7b3c:	50                   	push   %eax
77ed7b3d:	50                   	push   %eax
77ed7b3e:	8b 45 0c             	mov    0xc(%ebp),%eax
77ed7b41:	50                   	push   %eax
77ed7b42:	8d 85 00 ff ff ff    	lea    0xffffff00(%ebp),%eax
77ed7b48:	50                   	push   %eax
77ed7b49:	e8 82 95 ff ff       	call   77ed10d0 <_HEAP_strdupA2W>
77ed7b4e:	83 c4 10             	add    $0x10,%esp
77ed7b51:	85 c0                	test   %eax,%eax
77ed7b53:	0f 88 ed 00 00 00    	js     77ed7c46 <_CreateICA@16+0x136>
77ed7b59:	50                   	push   %eax
77ed7b5a:	50                   	push   %eax
77ed7b5b:	8b 45 10             	mov    0x10(%ebp),%eax
77ed7b5e:	50                   	push   %eax
77ed7b5f:	8d 85 fc fe ff ff    	lea    0xfffffefc(%ebp),%eax
77ed7b65:	50                   	push   %eax
77ed7b66:	e8 65 95 ff ff       	call   77ed10d0 <_HEAP_strdupA2W>
77ed7b6b:	83 c4 10             	add    $0x10,%esp
77ed7b6e:	85 c0                	test   %eax,%eax
77ed7b70:	0f 88 e4 00 00 00    	js     77ed7c5a <_CreateICA@16+0x14a>
77ed7b76:	85 ff                	test   %edi,%edi
77ed7b78:	74 12                	je     77ed7b8c <_CreateICA@16+0x7c>
77ed7b7a:	50                   	push   %eax
77ed7b7b:	50                   	push   %eax
77ed7b7c:	8d 85 08 ff ff ff    	lea    0xffffff08(%ebp),%eax
77ed7b82:	57                   	push   %edi
77ed7b83:	50                   	push   %eax
77ed7b84:	e8 27 19 00 00       	call   77ed94b0 <_RosRtlDevModeA2W>
77ed7b89:	83 c4 10             	add    $0x10,%esp
77ed7b8c:	50                   	push   %eax
77ed7b8d:	50                   	push   %eax
77ed7b8e:	8d 85 f0 fe ff ff    	lea    0xfffffef0(%ebp),%eax
77ed7b94:	8b b5 04 ff ff ff    	mov    0xffffff04(%ebp),%esi
77ed7b9a:	56                   	push   %esi
77ed7b9b:	50                   	push   %eax
77ed7b9c:	e8 af 1c 00 00       	call   77ed9850 <_RtlInitUnicodeString@8>
77ed7ba1:	8d b5 e8 fe ff ff    	lea    0xfffffee8(%ebp),%esi
77ed7ba7:	8b 9d 00 ff ff ff    	mov    0xffffff00(%ebp),%ebx
77ed7bad:	53                   	push   %ebx
77ed7bae:	56                   	push   %esi
77ed7baf:	e8 9c 1c 00 00       	call   77ed9850 <_RtlInitUnicodeString@8>
77ed7bb4:	8d 9d e0 fe ff ff    	lea    0xfffffee0(%ebp),%ebx
77ed7bba:	8b 8d fc fe ff ff    	mov    0xfffffefc(%ebp),%ecx
77ed7bc0:	51                   	push   %ecx
77ed7bc1:	53                   	push   %ebx
77ed7bc2:	e8 89 1c 00 00       	call   77ed9850 <_RtlInitUnicodeString@8>
77ed7bc7:	58                   	pop    %eax
77ed7bc8:	31 c0                	xor    %eax,%eax
77ed7bca:	5a                   	pop    %edx
77ed7bcb:	85 ff                	test   %edi,%edi
77ed7bcd:	74 06                	je     77ed7bd5 <_CreateICA@16+0xc5>
77ed7bcf:	8d 85 08 ff ff ff    	lea    0xffffff08(%ebp),%eax
77ed7bd5:	50                   	push   %eax
77ed7bd6:	8d 85 f0 fe ff ff    	lea    0xfffffef0(%ebp),%eax
77ed7bdc:	53                   	push   %ebx
77ed7bdd:	56                   	push   %esi
77ed7bde:	50                   	push   %eax
77ed7bdf:	e8 a5 da ff ff       	call   77ed5689 <_NtGdiCreateIC@16>
77ed7be4:	83 ec 0c             	sub    $0xc,%esp
77ed7be7:	89 c3                	mov    %eax,%ebx
77ed7be9:	8b 85 fc fe ff ff    	mov    0xfffffefc(%ebp),%eax
77ed7bef:	50                   	push   %eax
77ed7bf0:	e8 4b 95 ff ff       	call   77ed1140 <_HEAP_free>
77ed7bf5:	83 c4 10             	add    $0x10,%esp
77ed7bf8:	83 ec 0c             	sub    $0xc,%esp
77ed7bfb:	8b bd 00 ff ff ff    	mov    0xffffff00(%ebp),%edi
77ed7c01:	57                   	push   %edi
77ed7c02:	e8 39 95 ff ff       	call   77ed1140 <_HEAP_free>
77ed7c07:	83 c4 10             	add    $0x10,%esp
77ed7c0a:	83 ec 0c             	sub    $0xc,%esp
77ed7c0d:	8b b5 04 ff ff ff    	mov    0xffffff04(%ebp),%esi
77ed7c13:	56                   	push   %esi
77ed7c14:	e8 27 95 ff ff       	call   77ed1140 <_HEAP_free>
77ed7c19:	89 d8                	mov    %ebx,%eax
77ed7c1b:	83 c4 10             	add    $0x10,%esp
77ed7c1e:	8d 65 f4             	lea    0xfffffff4(%ebp),%esp
77ed7c21:	5b                   	pop    %ebx
77ed7c22:	5e                   	pop    %esi
77ed7c23:	5f                   	pop    %edi
77ed7c24:	5d                   	pop    %ebp
77ed7c25:	c2 10 00             	ret    $0x10
77ed7c28:	83 ec 0c             	sub    $0xc,%esp
77ed7c2b:	50                   	push   %eax
77ed7c2c:	e8 5f 1c 00 00       	call   77ed9890 <_RtlNtStatusToDosError@4>
77ed7c31:	50                   	push   %eax
77ed7c32:	e8 d9 1c 00 00       	call   77ed9910 <_SetLastError@4>
77ed7c37:	89 d8                	mov    %ebx,%eax
77ed7c39:	83 c4 0c             	add    $0xc,%esp
77ed7c3c:	8d 65 f4             	lea    0xfffffff4(%ebp),%esp
77ed7c3f:	5b                   	pop    %ebx
77ed7c40:	5e                   	pop    %esi
77ed7c41:	5f                   	pop    %edi
77ed7c42:	5d                   	pop    %ebp
77ed7c43:	c2 10 00             	ret    $0x10
77ed7c46:	83 ec 0c             	sub    $0xc,%esp
77ed7c49:	50                   	push   %eax
77ed7c4a:	e8 41 1c 00 00       	call   77ed9890 <_RtlNtStatusToDosError@4>
77ed7c4f:	50                   	push   %eax
77ed7c50:	e8 bb 1c 00 00       	call   77ed9910 <_SetLastError@4>
77ed7c55:	83 c4 0c             	add    $0xc,%esp
77ed7c58:	eb b0                	jmp    77ed7c0a <_CreateICA@16+0xfa>
77ed7c5a:	83 ec 0c             	sub    $0xc,%esp
77ed7c5d:	50                   	push   %eax
77ed7c5e:	e8 2d 1c 00 00       	call   77ed9890 <_RtlNtStatusToDosError@4>
77ed7c63:	50                   	push   %eax
77ed7c64:	e8 a7 1c 00 00       	call   77ed9910 <_SetLastError@4>
77ed7c69:	83 c4 0c             	add    $0xc,%esp
77ed7c6c:	eb 8a                	jmp    77ed7bf8 <_CreateICA@16+0xe8>
77ed7c6e:	89 f6                	mov    %esi,%esi

77ed7c70 <_DeleteObject@4>:
77ed7c70:	55                   	push   %ebp
77ed7c71:	89 e5                	mov    %esp,%ebp
77ed7c73:	53                   	push   %ebx
77ed7c74:	50                   	push   %eax
77ed7c75:	8b 5d 08             	mov    0x8(%ebp),%ebx
77ed7c78:	f7 c3 00 00 80 00    	test   $0x800000,%ebx
77ed7c7e:	75 10                	jne    77ed7c90 <_DeleteObject@4+0x20>
77ed7c80:	8b 5d fc             	mov    0xfffffffc(%ebp),%ebx
77ed7c83:	c9                   	leave  
77ed7c84:	e9 0e db ff ff       	jmp    77ed5797 <_NtGdiDeleteObject@4>
77ed7c89:	8d b4 26 00 00 00 00 	lea    0x0(%esi),%esi
77ed7c90:	50                   	push   %eax
77ed7c91:	68 c6 00 00 00       	push   $0xc6
77ed7c96:	68 30 b8 ed 77       	push   $0x77edb830
77ed7c9b:	68 3d b8 ed 77       	push   $0x77edb83d
77ed7ca0:	ff 15 e8 10 ee 77    	call   *0x77ee10e8
77ed7ca6:	59                   	pop    %ecx
77ed7ca7:	58                   	pop    %eax
77ed7ca8:	53                   	push   %ebx
77ed7ca9:	68 48 b8 ed 77       	push   $0x77edb848
77ed7cae:	ff 15 e8 10 ee 77    	call   *0x77ee10e8
77ed7cb4:	b8 01 00 00 00       	mov    $0x1,%eax
77ed7cb9:	8b 5d fc             	mov    0xfffffffc(%ebp),%ebx
77ed7cbc:	c9                   	leave  
77ed7cbd:	c2 04 00             	ret    $0x4

77ed7cc0 <_GetRelAbs@8>:
77ed7cc0:	55                   	push   %ebp
77ed7cc1:	89 e5                	mov    %esp,%ebp
77ed7cc3:	83 ec 14             	sub    $0x14,%esp
77ed7cc6:	8b 45 08             	mov    0x8(%ebp),%eax
77ed7cc9:	50                   	push   %eax
77ed7cca:	e8 d2 df ff ff       	call   77ed5ca1 <_NtGdiGetRelAbs@4>
77ed7ccf:	c9                   	leave  
77ed7cd0:	c2 08 00             	ret    $0x8
77ed7cd3:	8d b6 00 00 00 00    	lea    0x0(%esi),%esi
77ed7cd9:	8d bc 27 00 00 00 00 	lea    0x0(%edi),%edi

77ed7ce0 <_GetDCOrg@4>:
77ed7ce0:	55                   	push   %ebp
77ed7ce1:	89 e5                	mov    %esp,%ebp
77ed7ce3:	83 ec 10             	sub    $0x10,%esp
77ed7ce6:	8d 45 f8             	lea    0xfffffff8(%ebp),%eax
77ed7ce9:	50                   	push   %eax
77ed7cea:	8b 45 08             	mov    0x8(%ebp),%eax
77ed7ced:	50                   	push   %eax
77ed7cee:	e8 92 dd ff ff       	call   77ed5a85 <_NtGdiGetDCOrgEx@8>
77ed7cf3:	5a                   	pop    %edx
77ed7cf4:	31 d2                	xor    %edx,%edx
77ed7cf6:	59                   	pop    %ecx
77ed7cf7:	85 c0                	test   %eax,%eax
77ed7cf9:	74 13                	je     77ed7d0e <_GetDCOrg@4+0x2e>
77ed7cfb:	8b 45 f8             	mov    0xfffffff8(%ebp),%eax
77ed7cfe:	89 c2                	mov    %eax,%edx
77ed7d00:	8b 45 fc             	mov    0xfffffffc(%ebp),%eax
77ed7d03:	c1 e0 10             	shl    $0x10,%eax
77ed7d06:	81 e2 ff ff 00 00    	and    $0xffff,%edx
77ed7d0c:	09 c2                	or     %eax,%edx
77ed7d0e:	89 d0                	mov    %edx,%eax
77ed7d10:	c9                   	leave  
77ed7d11:	c2 04 00             	ret    $0x4
77ed7d14:	8d b6 00 00 00 00    	lea    0x0(%esi),%esi
77ed7d1a:	8d bf 00 00 00 00    	lea    0x0(%edi),%edi

77ed7d20 <_GetObjectA@12>:
77ed7d20:	55                   	push   %ebp
77ed7d21:	89 e5                	mov    %esp,%ebp
77ed7d23:	57                   	push   %edi
77ed7d24:	56                   	push   %esi
77ed7d25:	53                   	push   %ebx
77ed7d26:	83 ec 78             	sub    $0x78,%esp
77ed7d29:	8b 5d 08             	mov    0x8(%ebp),%ebx
77ed7d2c:	8b 75 0c             	mov    0xc(%ebp),%esi
77ed7d2f:	8b 7d 10             	mov    0x10(%ebp),%edi
77ed7d32:	53                   	push   %ebx
77ed7d33:	e8 e2 de ff ff       	call   77ed5c1a <_NtGdiGetObjectType@4>
77ed7d38:	31 d2                	xor    %edx,%edx
77ed7d3a:	83 c4 0c             	add    $0xc,%esp
77ed7d3d:	85 c0                	test   %eax,%eax
77ed7d3f:	74 11                	je     77ed7d52 <_GetObjectA@12+0x32>
77ed7d41:	83 f8 06             	cmp    $0x6,%eax
77ed7d44:	74 1a                	je     77ed7d60 <_GetObjectA@12+0x40>
77ed7d46:	51                   	push   %ecx
77ed7d47:	57                   	push   %edi
77ed7d48:	56                   	push   %esi
77ed7d49:	53                   	push   %ebx
77ed7d4a:	e8 bc de ff ff       	call   77ed5c0b <_NtGdiGetObject@12>
77ed7d4f:	5a                   	pop    %edx
77ed7d50:	89 c2                	mov    %eax,%edx
77ed7d52:	8d 65 f4             	lea    0xfffffff4(%ebp),%esp
77ed7d55:	89 d0                	mov    %edx,%eax
77ed7d57:	5b                   	pop    %ebx
77ed7d58:	5e                   	pop    %esi
77ed7d59:	5f                   	pop    %edi
77ed7d5a:	5d                   	pop    %ebp
77ed7d5b:	c2 0c 00             	ret    $0xc
77ed7d5e:	89 f6                	mov    %esi,%esi
77ed7d60:	83 fe 3b             	cmp    $0x3b,%esi
77ed7d63:	77 1b                	ja     77ed7d80 <_GetObjectA@12+0x60>
77ed7d65:	83 ec 0c             	sub    $0xc,%esp
77ed7d68:	6a 6f                	push   $0x6f
77ed7d6a:	e8 a1 1b 00 00       	call   77ed9910 <_SetLastError@4>
77ed7d6f:	31 d2                	xor    %edx,%edx
77ed7d71:	8d 65 f4             	lea    0xfffffff4(%ebp),%esp
77ed7d74:	89 d0                	mov    %edx,%eax
77ed7d76:	5b                   	pop    %ebx
77ed7d77:	5e                   	pop    %esi
77ed7d78:	5f                   	pop    %edi
77ed7d79:	5d                   	pop    %ebp
77ed7d7a:	c2 0c 00             	ret    $0xc
77ed7d7d:	8d 76 00             	lea    0x0(%esi),%esi
77ed7d80:	8d 75 88             	lea    0xffffff88(%ebp),%esi
77ed7d83:	51                   	push   %ecx
77ed7d84:	56                   	push   %esi
77ed7d85:	6a 5c                	push   $0x5c
77ed7d87:	53                   	push   %ebx
77ed7d88:	e8 7e de ff ff       	call   77ed5c0b <_NtGdiGetObject@12>
77ed7d8d:	5a                   	pop    %edx
77ed7d8e:	31 d2                	xor    %edx,%edx
77ed7d90:	85 c0                	test   %eax,%eax
77ed7d92:	74 be                	je     77ed7d52 <_GetObjectA@12+0x32>
77ed7d94:	53                   	push   %ebx
77ed7d95:	53                   	push   %ebx
77ed7d96:	56                   	push   %esi
77ed7d97:	57                   	push   %edi
77ed7d98:	e8 93 16 00 00       	call   77ed9430 <_RosRtlLogFontW2A>
77ed7d9d:	b8 3c 00 00 00       	mov    $0x3c,%eax
77ed7da2:	83 c4 10             	add    $0x10,%esp
77ed7da5:	89 c2                	mov    %eax,%edx
77ed7da7:	eb a9                	jmp    77ed7d52 <_GetObjectA@12+0x32>
77ed7da9:	8d b4 26 00 00 00 00 	lea    0x0(%esi),%esi

77ed7db0 <_GetObjectW@12>:
77ed7db0:	55                   	push   %ebp
77ed7db1:	89 e5                	mov    %esp,%ebp
77ed7db3:	c9                   	leave  
77ed7db4:	e9 52 de ff ff       	jmp    77ed5c0b <_NtGdiGetObject@12>
77ed7db9:	8d b4 26 00 00 00 00 	lea    0x0(%esi),%esi

77ed7dc0 <_FixBrushOrgEx@16>:
77ed7dc0:	55                   	push   %ebp
77ed7dc1:	31 c0                	xor    %eax,%eax
77ed7dc3:	89 e5                	mov    %esp,%ebp
77ed7dc5:	5d                   	pop    %ebp
77ed7dc6:	c2 10 00             	ret    $0x10
77ed7dc9:	8d b4 26 00 00 00 00 	lea    0x0(%esi),%esi

77ed7dd0 <_GetDCBrushColor@4>:
77ed7dd0:	55                   	push   %ebp
77ed7dd1:	89 e5                	mov    %esp,%ebp
77ed7dd3:	83 ec 0c             	sub    $0xc,%esp
77ed7dd6:	8b 45 08             	mov    0x8(%ebp),%eax
77ed7dd9:	6a 47                	push   $0x47
77ed7ddb:	6a 02                	push   $0x2
77ed7ddd:	50                   	push   %eax
77ed7dde:	e8 2e e7 ff ff       	call   77ed6511 <_NtUserCallTwoParam@12>
77ed7de3:	c9                   	leave  
77ed7de4:	c2 04 00             	ret    $0x4
77ed7de7:	89 f6                	mov    %esi,%esi
77ed7de9:	8d bc 27 00 00 00 00 	lea    0x0(%edi),%edi

77ed7df0 <_GetDCPenColor@4>:
77ed7df0:	55                   	push   %ebp
77ed7df1:	89 e5                	mov    %esp,%ebp
77ed7df3:	83 ec 0c             	sub    $0xc,%esp
77ed7df6:	8b 45 08             	mov    0x8(%ebp),%eax
77ed7df9:	6a 47                	push   $0x47
77ed7dfb:	6a 01                	push   $0x1
77ed7dfd:	50                   	push   %eax
77ed7dfe:	e8 0e e7 ff ff       	call   77ed6511 <_NtUserCallTwoParam@12>
77ed7e03:	c9                   	leave  
77ed7e04:	c2 04 00             	ret    $0x4
77ed7e07:	89 f6                	mov    %esi,%esi
77ed7e09:	8d bc 27 00 00 00 00 	lea    0x0(%edi),%edi

77ed7e10 <_SetDCBrushColor@8>:
77ed7e10:	55                   	push   %ebp
77ed7e11:	89 e5                	mov    %esp,%ebp
77ed7e13:	83 ec 0c             	sub    $0xc,%esp
77ed7e16:	8b 45 0c             	mov    0xc(%ebp),%eax
77ed7e19:	6a 46                	push   $0x46
77ed7e1b:	50                   	push   %eax
77ed7e1c:	8b 45 08             	mov    0x8(%ebp),%eax
77ed7e1f:	50                   	push   %eax
77ed7e20:	e8 ec e6 ff ff       	call   77ed6511 <_NtUserCallTwoParam@12>
77ed7e25:	c9                   	leave  
77ed7e26:	c2 08 00             	ret    $0x8
77ed7e29:	8d b4 26 00 00 00 00 	lea    0x0(%esi),%esi

77ed7e30 <_SetDCPenColor@8>:
77ed7e30:	55                   	push   %ebp
77ed7e31:	89 e5                	mov    %esp,%ebp
77ed7e33:	83 ec 0c             	sub    $0xc,%esp
77ed7e36:	8b 45 0c             	mov    0xc(%ebp),%eax
77ed7e39:	6a 45                	push   $0x45
77ed7e3b:	50                   	push   %eax
77ed7e3c:	8b 45 08             	mov    0x8(%ebp),%eax
77ed7e3f:	50                   	push   %eax
77ed7e40:	e8 cc e6 ff ff       	call   77ed6511 <_NtUserCallTwoParam@12>
77ed7e45:	c9                   	leave  
77ed7e46:	c2 08 00             	ret    $0x8
77ed7e49:	8d b4 26 00 00 00 00 	lea    0x0(%esi),%esi

77ed7e50 <_ResetDCW@8>:
77ed7e50:	55                   	push   %ebp
77ed7e51:	89 e5                	mov    %esp,%ebp
77ed7e53:	c9                   	leave  
77ed7e54:	e9 cc e1 ff ff       	jmp    77ed6025 <_NtGdiResetDC@8>
77ed7e59:	8d b4 26 00 00 00 00 	lea    0x0(%esi),%esi

77ed7e60 <_ResetDCA@8>:
77ed7e60:	55                   	push   %ebp
77ed7e61:	89 e5                	mov    %esp,%ebp
77ed7e63:	53                   	push   %ebx
77ed7e64:	81 ec ec 00 00 00    	sub    $0xec,%esp
77ed7e6a:	8b 45 0c             	mov    0xc(%ebp),%eax
77ed7e6d:	8d 9d 18 ff ff ff    	lea    0xffffff18(%ebp),%ebx
77ed7e73:	50                   	push   %eax
77ed7e74:	53                   	push   %ebx
77ed7e75:	e8 36 16 00 00       	call   77ed94b0 <_RosRtlDevModeA2W>
77ed7e7a:	8b 55 08             	mov    0x8(%ebp),%edx
77ed7e7d:	59                   	pop    %ecx
77ed7e7e:	58                   	pop    %eax
77ed7e7f:	53                   	push   %ebx
77ed7e80:	52                   	push   %edx
77ed7e81:	e8 9f e1 ff ff       	call   77ed6025 <_NtGdiResetDC@8>
77ed7e86:	8b 5d fc             	mov    0xfffffffc(%ebp),%ebx
77ed7e89:	c9                   	leave  
77ed7e8a:	c2 08 00             	ret    $0x8
77ed7e8d:	8d 76 00             	lea    0x0(%esi),%esi

77ed7e90 <_StartDocW@8>:
77ed7e90:	55                   	push   %ebp
77ed7e91:	89 e5                	mov    %esp,%ebp
77ed7e93:	c9                   	leave  
77ed7e94:	e9 89 e4 ff ff       	jmp    77ed6322 <_NtGdiStartDoc@8>
77ed7e99:	8d b4 26 00 00 00 00 	lea    0x0(%esi),%esi

77ed7ea0 <_GetObjectType@4>:
77ed7ea0:	55                   	push   %ebp
77ed7ea1:	89 e5                	mov    %esp,%ebp
77ed7ea3:	56                   	push   %esi
77ed7ea4:	53                   	push   %ebx
77ed7ea5:	31 f6                	xor    %esi,%esi
77ed7ea7:	83 ec 0c             	sub    $0xc,%esp
77ed7eaa:	8b 5d 08             	mov    0x8(%ebp),%ebx
77ed7ead:	53                   	push   %ebx
77ed7eae:	e8 ed 92 ff ff       	call   77ed11a0 <_GdiIsHandleValid>
77ed7eb3:	83 c4 10             	add    $0x10,%esp
77ed7eb6:	85 c0                	test   %eax,%eax
77ed7eb8:	74 3b                	je     77ed7ef5 <_GetObjectType@4+0x55>
77ed7eba:	81 e3 00 00 7f 00    	and    $0x7f0000,%ebx
77ed7ec0:	81 fb 00 00 30 00    	cmp    $0x300000,%ebx
77ed7ec6:	74 68                	je     77ed7f30 <_GetObjectType@4+0x90>
77ed7ec8:	7f 36                	jg     77ed7f00 <_GetObjectType@4+0x60>
77ed7eca:	81 fb 00 00 05 00    	cmp    $0x50000,%ebx
77ed7ed0:	0f 84 dc 00 00 00    	je     77ed7fb2 <_GetObjectType@4+0x112>
77ed7ed6:	7f 68                	jg     77ed7f40 <_GetObjectType@4+0xa0>
77ed7ed8:	81 fb 00 00 01 00    	cmp    $0x10000,%ebx
77ed7ede:	0f 84 00 01 00 00    	je     77ed7fe4 <_GetObjectType@4+0x144>
77ed7ee4:	81 fb 00 00 04 00    	cmp    $0x40000,%ebx
77ed7eea:	0f 85 90 00 00 00    	jne    77ed7f80 <_GetObjectType@4+0xe0>
77ed7ef0:	be 08 00 00 00       	mov    $0x8,%esi
77ed7ef5:	8d 65 f8             	lea    0xfffffff8(%ebp),%esp
77ed7ef8:	89 f0                	mov    %esi,%eax
77ed7efa:	5b                   	pop    %ebx
77ed7efb:	5e                   	pop    %esi
77ed7efc:	5d                   	pop    %ebp
77ed7efd:	c2 04 00             	ret    $0x4
77ed7f00:	81 fb 00 00 72 00    	cmp    $0x720000,%ebx
77ed7f06:	0f 84 b0 00 00 00    	je     77ed7fbc <_GetObjectType@4+0x11c>
77ed7f0c:	7f 53                	jg     77ed7f61 <_GetObjectType@4+0xc1>
77ed7f0e:	81 fb 00 00 50 00    	cmp    $0x500000,%ebx
77ed7f14:	0f 84 b6 00 00 00    	je     77ed7fd0 <_GetObjectType@4+0x130>
77ed7f1a:	81 fb 00 00 71 00    	cmp    $0x710000,%ebx
77ed7f20:	75 5e                	jne    77ed7f80 <_GetObjectType@4+0xe0>
77ed7f22:	be 04 00 00 00       	mov    $0x4,%esi
77ed7f27:	eb cc                	jmp    77ed7ef5 <_GetObjectType@4+0x55>
77ed7f29:	8d b4 26 00 00 00 00 	lea    0x0(%esi),%esi
77ed7f30:	be 01 00 00 00       	mov    $0x1,%esi
77ed7f35:	8d 65 f8             	lea    0xfffffff8(%ebp),%esp
77ed7f38:	89 f0                	mov    %esi,%eax
77ed7f3a:	5b                   	pop    %ebx
77ed7f3b:	5e                   	pop    %esi
77ed7f3c:	5d                   	pop    %ebp
77ed7f3d:	c2 04 00             	ret    $0x4
77ed7f40:	81 fb 00 00 0a 00    	cmp    $0xa0000,%ebx
77ed7f46:	0f 84 8e 00 00 00    	je     77ed7fda <_GetObjectType@4+0x13a>
77ed7f4c:	0f 8f 9c 00 00 00    	jg     77ed7fee <_GetObjectType@4+0x14e>
77ed7f52:	81 fb 00 00 08 00    	cmp    $0x80000,%ebx
77ed7f58:	75 26                	jne    77ed7f80 <_GetObjectType@4+0xe0>
77ed7f5a:	be 05 00 00 00       	mov    $0x5,%esi
77ed7f5f:	eb 94                	jmp    77ed7ef5 <_GetObjectType@4+0x55>
77ed7f61:	81 fb 00 00 74 00    	cmp    $0x740000,%ebx
77ed7f67:	74 5d                	je     77ed7fc6 <_GetObjectType@4+0x126>
77ed7f69:	0f 8f 91 00 00 00    	jg     77ed8000 <_GetObjectType@4+0x160>
77ed7f6f:	81 fb 00 00 73 00    	cmp    $0x730000,%ebx
77ed7f75:	0f 84 9b 00 00 00    	je     77ed8016 <_GetObjectType@4+0x176>
77ed7f7b:	90                   	nop    
77ed7f7c:	8d 74 26 00          	lea    0x0(%esi),%esi
77ed7f80:	51                   	push   %ecx
77ed7f81:	68 d0 01 00 00       	push   $0x1d0
77ed7f86:	68 30 b8 ed 77       	push   $0x77edb830
77ed7f8b:	68 3d b8 ed 77       	push   $0x77edb83d
77ed7f90:	ff 15 e8 10 ee 77    	call   *0x77ee10e8
77ed7f96:	58                   	pop    %eax
77ed7f97:	5a                   	pop    %edx
77ed7f98:	53                   	push   %ebx
77ed7f99:	68 70 b8 ed 77       	push   $0x77edb870
77ed7f9e:	ff 15 e8 10 ee 77    	call   *0x77ee10e8
77ed7fa4:	89 f0                	mov    %esi,%eax
77ed7fa6:	83 c4 10             	add    $0x10,%esp
77ed7fa9:	8d 65 f8             	lea    0xfffffff8(%ebp),%esp
77ed7fac:	5b                   	pop    %ebx
77ed7fad:	5e                   	pop    %esi
77ed7fae:	5d                   	pop    %ebp
77ed7faf:	c2 04 00             	ret    $0x4
77ed7fb2:	be 07 00 00 00       	mov    $0x7,%esi
77ed7fb7:	e9 39 ff ff ff       	jmp    77ed7ef5 <_GetObjectType@4+0x55>
77ed7fbc:	be 09 00 00 00       	mov    $0x9,%esi
77ed7fc1:	e9 2f ff ff ff       	jmp    77ed7ef5 <_GetObjectType@4+0x55>
77ed7fc6:	be 0c 00 00 00       	mov    $0xc,%esi
77ed7fcb:	e9 25 ff ff ff       	jmp    77ed7ef5 <_GetObjectType@4+0x55>
77ed7fd0:	be 0b 00 00 00       	mov    $0xb,%esi
77ed7fd5:	e9 1b ff ff ff       	jmp    77ed7ef5 <_GetObjectType@4+0x55>
77ed7fda:	be 06 00 00 00       	mov    $0x6,%esi
77ed7fdf:	e9 11 ff ff ff       	jmp    77ed7ef5 <_GetObjectType@4+0x55>
77ed7fe4:	be 03 00 00 00       	mov    $0x3,%esi
77ed7fe9:	e9 07 ff ff ff       	jmp    77ed7ef5 <_GetObjectType@4+0x55>
77ed7fee:	81 fb 00 00 10 00    	cmp    $0x100000,%ebx
77ed7ff4:	75 8a                	jne    77ed7f80 <_GetObjectType@4+0xe0>
77ed7ff6:	be 02 00 00 00       	mov    $0x2,%esi
77ed7ffb:	e9 f5 fe ff ff       	jmp    77ed7ef5 <_GetObjectType@4+0x55>
77ed8000:	81 fb 00 00 75 00    	cmp    $0x750000,%ebx
77ed8006:	0f 85 74 ff ff ff    	jne    77ed7f80 <_GetObjectType@4+0xe0>
77ed800c:	be 0a 00 00 00       	mov    $0xa,%esi
77ed8011:	e9 df fe ff ff       	jmp    77ed7ef5 <_GetObjectType@4+0x55>
77ed8016:	be 0d 00 00 00       	mov    $0xd,%esi
77ed801b:	e9 d5 fe ff ff       	jmp    77ed7ef5 <_GetObjectType@4+0x55>

77ed8020 <@MetricsCharConvert@8>:
77ed8020:	55                   	push   %ebp
77ed8021:	89 e5                	mov    %esp,%ebp
77ed8023:	57                   	push   %edi
77ed8024:	56                   	push   %esi
77ed8025:	53                   	push   %ebx
77ed8026:	83 ec 2c             	sub    $0x2c,%esp
77ed8029:	89 d7                	mov    %edx,%edi
77ed802b:	66 85 c9             	test   %cx,%cx
77ed802e:	75 10                	jne    77ed8040 <@MetricsCharConvert@8+0x20>
77ed8030:	c6 02 00             	movb   $0x0,(%edx)
77ed8033:	b8 01 00 00 00       	mov    $0x1,%eax
77ed8038:	8d 65 f4             	lea    0xfffffff4(%ebp),%esp
77ed803b:	5b                   	pop    %ebx
77ed803c:	5e                   	pop    %esi
77ed803d:	5f                   	pop    %edi
77ed803e:	5d                   	pop    %ebp
77ed803f:	c3                   	ret    
77ed8040:	8d 45 ec             	lea    0xffffffec(%ebp),%eax
77ed8043:	8d 75 e0             	lea    0xffffffe0(%ebp),%esi
77ed8046:	66 89 4d ec          	mov    %cx,0xffffffec(%ebp)
77ed804a:	66 c7 45 ee 00 00    	movw   $0x0,0xffffffee(%ebp)
77ed8050:	51                   	push   %ecx
77ed8051:	51                   	push   %ecx
77ed8052:	50                   	push   %eax
77ed8053:	56                   	push   %esi
77ed8054:	e8 f7 17 00 00       	call   77ed9850 <_RtlInitUnicodeString@8>
77ed8059:	8d 5d d0             	lea    0xffffffd0(%ebp),%ebx
77ed805c:	8d 45 de             	lea    0xffffffde(%ebp),%eax
77ed805f:	50                   	push   %eax
77ed8060:	c6 45 de 2a          	movb   $0x2a,0xffffffde(%ebp)
77ed8064:	c6 45 df 00          	movb   $0x0,0xffffffdf(%ebp)
77ed8068:	53                   	push   %ebx
77ed8069:	e8 f2 17 00 00       	call   77ed9860 <_RtlInitAnsiString@8>
77ed806e:	c7 04 24 00 00 00 00 	movl   $0x0,(%esp)
77ed8075:	56                   	push   %esi
77ed8076:	53                   	push   %ebx
77ed8077:	e8 24 18 00 00       	call   77ed98a0 <_RtlUnicodeStringToAnsiString@12>
77ed807c:	5a                   	pop    %edx
77ed807d:	85 c0                	test   %eax,%eax
77ed807f:	78 07                	js     77ed8088 <@MetricsCharConvert@8+0x68>
77ed8081:	8a 45 de             	mov    0xffffffde(%ebp),%al
77ed8084:	88 07                	mov    %al,(%edi)
77ed8086:	eb ab                	jmp    77ed8033 <@MetricsCharConvert@8+0x13>
77ed8088:	83 ec 0c             	sub    $0xc,%esp
77ed808b:	50                   	push   %eax
77ed808c:	e8 ff 17 00 00       	call   77ed9890 <_RtlNtStatusToDosError@4>
77ed8091:	50                   	push   %eax
77ed8092:	e8 79 18 00 00       	call   77ed9910 <_SetLastError@4>
77ed8097:	31 c0                	xor    %eax,%eax
77ed8099:	eb 9d                	jmp    77ed8038 <@MetricsCharConvert@8+0x18>
77ed809b:	90                   	nop    
77ed809c:	8d 74 26 00          	lea    0x0(%esi),%esi

77ed80a0 <@TextMetricW2A@8>:
77ed80a0:	55                   	push   %ebp
77ed80a1:	89 e5                	mov    %esp,%ebp
77ed80a3:	57                   	push   %edi
77ed80a4:	56                   	push   %esi
77ed80a5:	53                   	push   %ebx
77ed80a6:	81 ec 1c 03 00 00    	sub    $0x31c,%esp
77ed80ac:	89 ce                	mov    %ecx,%esi
77ed80ae:	8b 02                	mov    (%edx),%eax
77ed80b0:	89 d7                	mov    %edx,%edi
77ed80b2:	89 01                	mov    %eax,(%ecx)
77ed80b4:	8b 42 04             	mov    0x4(%edx),%eax
77ed80b7:	89 41 04             	mov    %eax,0x4(%ecx)
77ed80ba:	8b 42 08             	mov    0x8(%edx),%eax
77ed80bd:	89 41 08             	mov    %eax,0x8(%ecx)
77ed80c0:	8b 42 0c             	mov    0xc(%edx),%eax
77ed80c3:	89 41 0c             	mov    %eax,0xc(%ecx)
77ed80c6:	8b 42 10             	mov    0x10(%edx),%eax
77ed80c9:	89 41 10             	mov    %eax,0x10(%ecx)
77ed80cc:	8b 42 14             	mov    0x14(%edx),%eax
77ed80cf:	89 41 14             	mov    %eax,0x14(%ecx)
77ed80d2:	8b 42 18             	mov    0x18(%edx),%eax
77ed80d5:	89 41 18             	mov    %eax,0x18(%ecx)
77ed80d8:	8b 42 1c             	mov    0x1c(%edx),%eax
77ed80db:	89 41 1c             	mov    %eax,0x1c(%ecx)
77ed80de:	8b 42 20             	mov    0x20(%edx),%eax
77ed80e1:	89 41 20             	mov    %eax,0x20(%ecx)
77ed80e4:	8b 42 24             	mov    0x24(%edx),%eax
77ed80e7:	89 41 24             	mov    %eax,0x24(%ecx)
77ed80ea:	8b 42 28             	mov    0x28(%edx),%eax
77ed80ed:	89 41 28             	mov    %eax,0x28(%ecx)
77ed80f0:	b8 01 00 00 00       	mov    $0x1,%eax
77ed80f5:	88 84 28 e7 fc ff ff 	mov    %al,0xfffffce7(%eax,%ebp,1)
77ed80fc:	66 c7 84 45 e6 fd ff 	movw   $0x20,0xfffffde6(%ebp,%eax,2)
77ed8103:	ff 20 00 
77ed8106:	40                   	inc    %eax
77ed8107:	3d ff 00 00 00       	cmp    $0xff,%eax
77ed810c:	76 e7                	jbe    77ed80f5 <@TextMetricW2A@8+0x55>
77ed810e:	c6 85 e7 fd ff ff 00 	movb   $0x0,0xfffffde7(%ebp)
77ed8115:	66 c7 45 e6 00 00    	movw   $0x0,0xffffffe6(%ebp)
77ed811b:	50                   	push   %eax
77ed811c:	50                   	push   %eax
77ed811d:	8d 85 e8 fc ff ff    	lea    0xfffffce8(%ebp),%eax
77ed8123:	50                   	push   %eax
77ed8124:	8d 85 e0 fc ff ff    	lea    0xfffffce0(%ebp),%eax
77ed812a:	50                   	push   %eax
77ed812b:	e8 30 17 00 00       	call   77ed9860 <_RtlInitAnsiString@8>
77ed8130:	8d 9d d8 fc ff ff    	lea    0xfffffcd8(%ebp),%ebx
77ed8136:	8d 85 e8 fd ff ff    	lea    0xfffffde8(%ebp),%eax
77ed813c:	50                   	push   %eax
77ed813d:	53                   	push   %ebx
77ed813e:	e8 0d 17 00 00       	call   77ed9850 <_RtlInitUnicodeString@8>
77ed8143:	8d 85 e0 fc ff ff    	lea    0xfffffce0(%ebp),%eax
77ed8149:	c7 04 24 00 00 00 00 	movl   $0x0,(%esp)
77ed8150:	50                   	push   %eax
77ed8151:	53                   	push   %ebx
77ed8152:	e8 19 17 00 00       	call   77ed9870 <_RtlAnsiStringToUnicodeString@12>
77ed8157:	5b                   	pop    %ebx
77ed8158:	85 c0                	test   %eax,%eax
77ed815a:	0f 88 c9 00 00 00    	js     77ed8229 <@TextMetricW2A@8+0x189>
77ed8160:	c6 46 2c 00          	movb   $0x0,0x2c(%esi)
77ed8164:	66 8b 4f 2c          	mov    0x2c(%edi),%cx
77ed8168:	66 85 c9             	test   %cx,%cx
77ed816b:	74 25                	je     77ed8192 <@TextMetricW2A@8+0xf2>
77ed816d:	b8 01 00 00 00       	mov    $0x1,%eax
77ed8172:	eb 08                	jmp    77ed817c <@TextMetricW2A@8+0xdc>
77ed8174:	40                   	inc    %eax
77ed8175:	3d ff 00 00 00       	cmp    $0xff,%eax
77ed817a:	77 16                	ja     77ed8192 <@TextMetricW2A@8+0xf2>
77ed817c:	66 8b 94 45 e6 fd ff 	mov    0xfffffde6(%ebp,%eax,2),%dx
77ed8183:	ff 
77ed8184:	66 39 d1             	cmp    %dx,%cx
77ed8187:	77 eb                	ja     77ed8174 <@TextMetricW2A@8+0xd4>
77ed8189:	66 3b 57 2e          	cmp    0x2e(%edi),%dx
77ed818d:	77 e5                	ja     77ed8174 <@TextMetricW2A@8+0xd4>
77ed818f:	88 46 2c             	mov    %al,0x2c(%esi)
77ed8192:	c6 46 2d 00          	movb   $0x0,0x2d(%esi)
77ed8196:	66 8b 5f 2e          	mov    0x2e(%edi),%bx
77ed819a:	66 85 db             	test   %bx,%bx
77ed819d:	74 29                	je     77ed81c8 <@TextMetricW2A@8+0x128>
77ed819f:	b8 ff 00 00 00       	mov    $0xff,%eax
77ed81a4:	66 8b 4f 2c          	mov    0x2c(%edi),%cx
77ed81a8:	eb 09                	jmp    77ed81b3 <@TextMetricW2A@8+0x113>
77ed81aa:	8d b6 00 00 00 00    	lea    0x0(%esi),%esi
77ed81b0:	48                   	dec    %eax
77ed81b1:	74 15                	je     77ed81c8 <@TextMetricW2A@8+0x128>
77ed81b3:	66 8b 94 45 e6 fd ff 	mov    0xfffffde6(%ebp,%eax,2),%dx
77ed81ba:	ff 
77ed81bb:	66 39 d1             	cmp    %dx,%cx
77ed81be:	77 f0                	ja     77ed81b0 <@TextMetricW2A@8+0x110>
77ed81c0:	66 39 da             	cmp    %bx,%dx
77ed81c3:	77 eb                	ja     77ed81b0 <@TextMetricW2A@8+0x110>
77ed81c5:	88 46 2d             	mov    %al,0x2d(%esi)
77ed81c8:	66 8b 4f 30          	mov    0x30(%edi),%cx
77ed81cc:	8d 56 2e             	lea    0x2e(%esi),%edx
77ed81cf:	81 e1 ff ff 00 00    	and    $0xffff,%ecx
77ed81d5:	e8 46 fe ff ff       	call   77ed8020 <@MetricsCharConvert@8>
77ed81da:	85 c0                	test   %eax,%eax
77ed81dc:	75 0a                	jne    77ed81e8 <@TextMetricW2A@8+0x148>
77ed81de:	8d 65 f4             	lea    0xfffffff4(%ebp),%esp
77ed81e1:	31 c0                	xor    %eax,%eax
77ed81e3:	5b                   	pop    %ebx
77ed81e4:	5e                   	pop    %esi
77ed81e5:	5f                   	pop    %edi
77ed81e6:	5d                   	pop    %ebp
77ed81e7:	c3                   	ret    
77ed81e8:	66 8b 4f 32          	mov    0x32(%edi),%cx
77ed81ec:	8d 56 2f             	lea    0x2f(%esi),%edx
77ed81ef:	81 e1 ff ff 00 00    	and    $0xffff,%ecx
77ed81f5:	e8 26 fe ff ff       	call   77ed8020 <@MetricsCharConvert@8>
77ed81fa:	85 c0                	test   %eax,%eax
77ed81fc:	74 e0                	je     77ed81de <@TextMetricW2A@8+0x13e>
77ed81fe:	8a 47 34             	mov    0x34(%edi),%al
77ed8201:	88 46 30             	mov    %al,0x30(%esi)
77ed8204:	8a 47 35             	mov    0x35(%edi),%al
77ed8207:	88 46 31             	mov    %al,0x31(%esi)
77ed820a:	8a 47 36             	mov    0x36(%edi),%al
77ed820d:	88 46 32             	mov    %al,0x32(%esi)
77ed8210:	8a 47 37             	mov    0x37(%edi),%al
77ed8213:	88 46 33             	mov    %al,0x33(%esi)
77ed8216:	8a 47 38             	mov    0x38(%edi),%al
77ed8219:	88 46 34             	mov    %al,0x34(%esi)
77ed821c:	8d 65 f4             	lea    0xfffffff4(%ebp),%esp
77ed821f:	b8 01 00 00 00       	mov    $0x1,%eax
77ed8224:	5b                   	pop    %ebx
77ed8225:	5e                   	pop    %esi
77ed8226:	5f                   	pop    %edi
77ed8227:	5d                   	pop    %ebp
77ed8228:	c3                   	ret    
77ed8229:	83 ec 0c             	sub    $0xc,%esp
77ed822c:	50                   	push   %eax
77ed822d:	e8 5e 16 00 00       	call   77ed9890 <_RtlNtStatusToDosError@4>
77ed8232:	50                   	push   %eax
77ed8233:	e8 d8 16 00 00       	call   77ed9910 <_SetLastError@4>
77ed8238:	eb a4                	jmp    77ed81de <@TextMetricW2A@8+0x13e>
77ed823a:	8d b6 00 00 00 00    	lea    0x0(%esi),%esi

77ed8240 <@NewTextMetricW2A@8>:
77ed8240:	55                   	push   %ebp
77ed8241:	89 e5                	mov    %esp,%ebp
77ed8243:	56                   	push   %esi
77ed8244:	89 ce                	mov    %ecx,%esi
77ed8246:	53                   	push   %ebx
77ed8247:	89 d3                	mov    %edx,%ebx
77ed8249:	e8 52 fe ff ff       	call   77ed80a0 <@TextMetricW2A@8>
77ed824e:	31 d2                	xor    %edx,%edx
77ed8250:	85 c0                	test   %eax,%eax
77ed8252:	74 1a                	je     77ed826e <@NewTextMetricW2A@8+0x2e>
77ed8254:	8b 43 3c             	mov    0x3c(%ebx),%eax
77ed8257:	b2 01                	mov    $0x1,%dl
77ed8259:	89 46 38             	mov    %eax,0x38(%esi)
77ed825c:	8b 43 40             	mov    0x40(%ebx),%eax
77ed825f:	89 46 3c             	mov    %eax,0x3c(%esi)
77ed8262:	8b 43 44             	mov    0x44(%ebx),%eax
77ed8265:	89 46 40             	mov    %eax,0x40(%esi)
77ed8268:	8b 43 48             	mov    0x48(%ebx),%eax
77ed826b:	89 46 44             	mov    %eax,0x44(%esi)
77ed826e:	89 d0                	mov    %edx,%eax
77ed8270:	5b                   	pop    %ebx
77ed8271:	5e                   	pop    %esi
77ed8272:	5d                   	pop    %ebp
77ed8273:	c3                   	ret    
77ed8274:	8d b6 00 00 00 00    	lea    0x0(%esi),%esi
77ed827a:	8d bf 00 00 00 00    	lea    0x0(%edi),%edi

77ed8280 <@NewTextMetricExW2A@8>:
77ed8280:	55                   	push   %ebp
77ed8281:	89 e5                	mov    %esp,%ebp
77ed8283:	56                   	push   %esi
77ed8284:	89 ce                	mov    %ecx,%esi
77ed8286:	53                   	push   %ebx
77ed8287:	89 d3                	mov    %edx,%ebx
77ed8289:	e8 b2 ff ff ff       	call   77ed8240 <@NewTextMetricW2A@8>
77ed828e:	31 d2                	xor    %edx,%edx
77ed8290:	85 c0                	test   %eax,%eax
77ed8292:	74 26                	je     77ed82ba <@NewTextMetricExW2A@8+0x3a>
77ed8294:	8b 43 4c             	mov    0x4c(%ebx),%eax
77ed8297:	b2 01                	mov    $0x1,%dl
77ed8299:	89 46 48             	mov    %eax,0x48(%esi)
77ed829c:	8b 43 50             	mov    0x50(%ebx),%eax
77ed829f:	89 46 4c             	mov    %eax,0x4c(%esi)
77ed82a2:	8b 43 54             	mov    0x54(%ebx),%eax
77ed82a5:	89 46 50             	mov    %eax,0x50(%esi)
77ed82a8:	8b 43 58             	mov    0x58(%ebx),%eax
77ed82ab:	89 46 54             	mov    %eax,0x54(%esi)
77ed82ae:	8b 43 5c             	mov    0x5c(%ebx),%eax
77ed82b1:	89 46 58             	mov    %eax,0x58(%esi)
77ed82b4:	8b 43 60             	mov    0x60(%ebx),%eax
77ed82b7:	89 46 5c             	mov    %eax,0x5c(%esi)
77ed82ba:	89 d0                	mov    %edx,%eax
77ed82bc:	5b                   	pop    %ebx
77ed82bd:	5e                   	pop    %esi
77ed82be:	5d                   	pop    %ebp
77ed82bf:	c3                   	ret    

77ed82c0 <@IntEnumFontFamilies@20>:
77ed82c0:	55                   	push   %ebp
77ed82c1:	89 e5                	mov    %esp,%ebp
77ed82c3:	57                   	push   %edi
77ed82c4:	56                   	push   %esi
77ed82c5:	53                   	push   %ebx
77ed82c6:	81 ec 40 01 00 00    	sub    $0x140,%esp
77ed82cc:	89 8d c4 fe ff ff    	mov    %ecx,0xfffffec4(%ebp)
77ed82d2:	c7 85 bc fe ff ff 00 	movl   $0x0,0xfffffebc(%ebp)
77ed82d9:	00 00 00 
77ed82dc:	89 d3                	mov    %edx,%ebx
77ed82de:	68 00 71 00 00       	push   $0x7100
77ed82e3:	6a 00                	push   $0x0
77ed82e5:	50                   	push   %eax
77ed82e6:	e8 05 16 00 00       	call   77ed98f0 <_GetProcessHeap@0>
77ed82eb:	89 04 24             	mov    %eax,(%esp)
77ed82ee:	e8 fd 14 00 00       	call   77ed97f0 <_RtlAllocateHeap@12>
77ed82f3:	89 c7                	mov    %eax,%edi
77ed82f5:	58                   	pop    %eax
77ed82f6:	31 c0                	xor    %eax,%eax
77ed82f8:	85 ff                	test   %edi,%edi
77ed82fa:	0f 84 5e 01 00 00    	je     77ed845e <@IntEnumFontFamilies@20+0x19e>
77ed8300:	6a 40                	push   $0x40
77ed8302:	57                   	push   %edi
77ed8303:	53                   	push   %ebx
77ed8304:	8b 85 c4 fe ff ff    	mov    0xfffffec4(%ebp),%eax
77ed830a:	50                   	push   %eax
77ed830b:	e8 29 d8 ff ff       	call   77ed5b39 <_NtGdiGetFontFamilyInfo@16>
77ed8310:	89 c6                	mov    %eax,%esi
77ed8312:	85 c0                	test   %eax,%eax
77ed8314:	0f 88 bd 01 00 00    	js     77ed84d7 <@IntEnumFontFamilies@20+0x217>
77ed831a:	83 f8 40             	cmp    $0x40,%eax
77ed831d:	0f 8f 45 01 00 00    	jg     77ed8468 <@IntEnumFontFamilies@20+0x1a8>
77ed8323:	83 fe 00             	cmp    $0x0,%esi
77ed8326:	0f 86 1a 01 00 00    	jbe    77ed8446 <@IntEnumFontFamilies@20+0x186>
77ed832c:	89 fb                	mov    %edi,%ebx
77ed832e:	c7 85 b8 fe ff ff 00 	movl   $0x0,0xfffffeb8(%ebp)
77ed8335:	00 00 00 
77ed8338:	eb 47                	jmp    77ed8381 <@IntEnumFontFamilies@20+0xc1>
77ed833a:	8d b6 00 00 00 00    	lea    0x0(%esi),%esi
77ed8340:	8b 45 0c             	mov    0xc(%ebp),%eax
77ed8343:	50                   	push   %eax
77ed8344:	8b 85 b8 fe ff ff    	mov    0xfffffeb8(%ebp),%eax
77ed834a:	8b 8c 38 c0 01 00 00 	mov    0x1c0(%eax,%edi,1),%ecx
77ed8351:	8d 83 5c 01 00 00    	lea    0x15c(%ebx),%eax
77ed8357:	51                   	push   %ecx
77ed8358:	50                   	push   %eax
77ed8359:	53                   	push   %ebx
77ed835a:	ff 55 08             	call   *0x8(%ebp)
77ed835d:	81 c3 c4 01 00 00    	add    $0x1c4,%ebx
77ed8363:	89 85 bc fe ff ff    	mov    %eax,0xfffffebc(%ebp)
77ed8369:	8b 85 b8 fe ff ff    	mov    0xfffffeb8(%ebp),%eax
77ed836f:	05 c4 01 00 00       	add    $0x1c4,%eax
77ed8374:	4e                   	dec    %esi
77ed8375:	89 85 b8 fe ff ff    	mov    %eax,0xfffffeb8(%ebp)
77ed837b:	0f 84 c5 00 00 00    	je     77ed8446 <@IntEnumFontFamilies@20+0x186>
77ed8381:	8b 45 10             	mov    0x10(%ebp),%eax
77ed8384:	85 c0                	test   %eax,%eax
77ed8386:	75 b8                	jne    77ed8340 <@IntEnumFontFamilies@20+0x80>
77ed8388:	8d 85 28 ff ff ff    	lea    0xffffff28(%ebp),%eax
77ed838e:	52                   	push   %edx
77ed838f:	52                   	push   %edx
77ed8390:	53                   	push   %ebx
77ed8391:	50                   	push   %eax
77ed8392:	e8 99 10 00 00       	call   77ed9430 <_RosRtlLogFontW2A>
77ed8397:	8d 85 64 ff ff ff    	lea    0xffffff64(%ebp),%eax
77ed839d:	6a 00                	push   $0x0
77ed839f:	6a 00                	push   $0x0
77ed83a1:	6a 40                	push   $0x40
77ed83a3:	50                   	push   %eax
77ed83a4:	8d 43 5c             	lea    0x5c(%ebx),%eax
77ed83a7:	6a ff                	push   $0xffffffff
77ed83a9:	50                   	push   %eax
77ed83aa:	6a 00                	push   $0x0
77ed83ac:	6a 03                	push   $0x3
77ed83ae:	e8 8d 15 00 00       	call   77ed9940 <_WideCharToMultiByte@32>
77ed83b3:	8d 45 a4             	lea    0xffffffa4(%ebp),%eax
77ed83b6:	6a 00                	push   $0x0
77ed83b8:	6a 00                	push   $0x0
77ed83ba:	6a 20                	push   $0x20
77ed83bc:	50                   	push   %eax
77ed83bd:	8d 83 dc 00 00 00    	lea    0xdc(%ebx),%eax
77ed83c3:	6a ff                	push   $0xffffffff
77ed83c5:	50                   	push   %eax
77ed83c6:	6a 00                	push   $0x0
77ed83c8:	6a 03                	push   $0x3
77ed83ca:	e8 71 15 00 00       	call   77ed9940 <_WideCharToMultiByte@32>
77ed83cf:	8d 45 c4             	lea    0xffffffc4(%ebp),%eax
77ed83d2:	6a 00                	push   $0x0
77ed83d4:	6a 00                	push   $0x0
77ed83d6:	6a 20                	push   $0x20
77ed83d8:	50                   	push   %eax
77ed83d9:	8d 83 1c 01 00 00    	lea    0x11c(%ebx),%eax
77ed83df:	6a ff                	push   $0xffffffff
77ed83e1:	50                   	push   %eax
77ed83e2:	6a 00                	push   $0x0
77ed83e4:	6a 03                	push   $0x3
77ed83e6:	e8 55 15 00 00       	call   77ed9940 <_WideCharToMultiByte@32>
77ed83eb:	8d 93 5c 01 00 00    	lea    0x15c(%ebx),%edx
77ed83f1:	8d 8d c8 fe ff ff    	lea    0xfffffec8(%ebp),%ecx
77ed83f7:	e8 84 fe ff ff       	call   77ed8280 <@NewTextMetricExW2A@8>
77ed83fc:	8b 45 0c             	mov    0xc(%ebp),%eax
77ed83ff:	50                   	push   %eax
77ed8400:	81 c3 c4 01 00 00    	add    $0x1c4,%ebx
77ed8406:	8b 85 b8 fe ff ff    	mov    0xfffffeb8(%ebp),%eax
77ed840c:	8b 84 38 c0 01 00 00 	mov    0x1c0(%eax,%edi,1),%eax
77ed8413:	50                   	push   %eax
77ed8414:	8d 85 c8 fe ff ff    	lea    0xfffffec8(%ebp),%eax
77ed841a:	50                   	push   %eax
77ed841b:	8d 85 28 ff ff ff    	lea    0xffffff28(%ebp),%eax
77ed8421:	50                   	push   %eax
77ed8422:	ff 55 08             	call   *0x8(%ebp)
77ed8425:	83 c4 10             	add    $0x10,%esp
77ed8428:	89 85 bc fe ff ff    	mov    %eax,0xfffffebc(%ebp)
77ed842e:	8b 85 b8 fe ff ff    	mov    0xfffffeb8(%ebp),%eax
77ed8434:	05 c4 01 00 00       	add    $0x1c4,%eax
77ed8439:	4e                   	dec    %esi
77ed843a:	89 85 b8 fe ff ff    	mov    %eax,0xfffffeb8(%ebp)
77ed8440:	0f 85 3b ff ff ff    	jne    77ed8381 <@IntEnumFontFamilies@20+0xc1>
77ed8446:	50                   	push   %eax
77ed8447:	57                   	push   %edi
77ed8448:	6a 00                	push   $0x0
77ed844a:	50                   	push   %eax
77ed844b:	e8 a0 14 00 00       	call   77ed98f0 <_GetProcessHeap@0>
77ed8450:	89 04 24             	mov    %eax,(%esp)
77ed8453:	e8 c8 13 00 00       	call   77ed9820 <_RtlFreeHeap@12>
77ed8458:	8b 85 bc fe ff ff    	mov    0xfffffebc(%ebp),%eax
77ed845e:	8d 65 f4             	lea    0xfffffff4(%ebp),%esp
77ed8461:	5b                   	pop    %ebx
77ed8462:	5e                   	pop    %esi
77ed8463:	5f                   	pop    %edi
77ed8464:	5d                   	pop    %ebp
77ed8465:	c2 0c 00             	ret    $0xc
77ed8468:	89 85 c0 fe ff ff    	mov    %eax,0xfffffec0(%ebp)
77ed846e:	50                   	push   %eax
77ed846f:	57                   	push   %edi
77ed8470:	6a 00                	push   $0x0
77ed8472:	51                   	push   %ecx
77ed8473:	e8 78 14 00 00       	call   77ed98f0 <_GetProcessHeap@0>
77ed8478:	89 04 24             	mov    %eax,(%esp)
77ed847b:	e8 a0 13 00 00       	call   77ed9820 <_RtlFreeHeap@12>
77ed8480:	8d 04 f5 00 00 00 00 	lea    0x0(,%esi,8),%eax
77ed8487:	29 f0                	sub    %esi,%eax
77ed8489:	c1 e0 04             	shl    $0x4,%eax
77ed848c:	01 f0                	add    %esi,%eax
77ed848e:	c1 e0 02             	shl    $0x2,%eax
77ed8491:	50                   	push   %eax
77ed8492:	6a 00                	push   $0x0
77ed8494:	52                   	push   %edx
77ed8495:	e8 56 14 00 00       	call   77ed98f0 <_GetProcessHeap@0>
77ed849a:	89 04 24             	mov    %eax,(%esp)
77ed849d:	e8 4e 13 00 00       	call   77ed97f0 <_RtlAllocateHeap@12>
77ed84a2:	89 c7                	mov    %eax,%edi
77ed84a4:	58                   	pop    %eax
77ed84a5:	31 c0                	xor    %eax,%eax
77ed84a7:	85 ff                	test   %edi,%edi
77ed84a9:	74 b3                	je     77ed845e <@IntEnumFontFamilies@20+0x19e>
77ed84ab:	56                   	push   %esi
77ed84ac:	57                   	push   %edi
77ed84ad:	53                   	push   %ebx
77ed84ae:	8b 85 c4 fe ff ff    	mov    0xfffffec4(%ebp),%eax
77ed84b4:	50                   	push   %eax
77ed84b5:	e8 7f d6 ff ff       	call   77ed5b39 <_NtGdiGetFontFamilyInfo@16>
77ed84ba:	89 c2                	mov    %eax,%edx
77ed84bc:	89 c6                	mov    %eax,%esi
77ed84be:	c1 ea 1f             	shr    $0x1f,%edx
77ed84c1:	3b 85 c0 fe ff ff    	cmp    0xfffffec0(%ebp),%eax
77ed84c7:	0f 97 c0             	seta   %al
77ed84ca:	25 ff 00 00 00       	and    $0xff,%eax
77ed84cf:	09 c2                	or     %eax,%edx
77ed84d1:	0f 84 4c fe ff ff    	je     77ed8323 <@IntEnumFontFamilies@20+0x63>
77ed84d7:	50                   	push   %eax
77ed84d8:	57                   	push   %edi
77ed84d9:	6a 00                	push   $0x0
77ed84db:	50                   	push   %eax
77ed84dc:	e8 0f 14 00 00       	call   77ed98f0 <_GetProcessHeap@0>
77ed84e1:	89 04 24             	mov    %eax,(%esp)
77ed84e4:	e8 37 13 00 00       	call   77ed9820 <_RtlFreeHeap@12>
77ed84e9:	8d 65 f4             	lea    0xfffffff4(%ebp),%esp
77ed84ec:	31 c0                	xor    %eax,%eax
77ed84ee:	5b                   	pop    %ebx
77ed84ef:	5e                   	pop    %esi
77ed84f0:	5f                   	pop    %edi
77ed84f1:	5d                   	pop    %ebp
77ed84f2:	c2 0c 00             	ret    $0xc
77ed84f5:	8d 74 26 00          	lea    0x0(%esi),%esi
77ed84f9:	8d bc 27 00 00 00 00 	lea    0x0(%edi),%edi

77ed8500 <_EnumFontFamiliesExW@20>:
77ed8500:	55                   	push   %ebp
77ed8501:	89 e5                	mov    %esp,%ebp
77ed8503:	83 ec 0c             	sub    $0xc,%esp
77ed8506:	8b 45 14             	mov    0x14(%ebp),%eax
77ed8509:	6a 01                	push   $0x1
77ed850b:	8b 4d 08             	mov    0x8(%ebp),%ecx
77ed850e:	50                   	push   %eax
77ed850f:	8b 55 0c             	mov    0xc(%ebp),%edx
77ed8512:	8b 45 10             	mov    0x10(%ebp),%eax
77ed8515:	50                   	push   %eax
77ed8516:	e8 a5 fd ff ff       	call   77ed82c0 <@IntEnumFontFamilies@20>
77ed851b:	c9                   	leave  
77ed851c:	c2 14 00             	ret    $0x14
77ed851f:	90                   	nop    

77ed8520 <_EnumFontFamiliesW@16>:
77ed8520:	55                   	push   %ebp
77ed8521:	89 e5                	mov    %esp,%ebp
77ed8523:	56                   	push   %esi
77ed8524:	53                   	push   %ebx
77ed8525:	83 ec 64             	sub    $0x64,%esp
77ed8528:	8d 75 98             	lea    0xffffff98(%ebp),%esi
77ed852b:	8b 5d 0c             	mov    0xc(%ebp),%ebx
77ed852e:	6a 5c                	push   $0x5c
77ed8530:	6a 00                	push   $0x0
77ed8532:	56                   	push   %esi
77ed8533:	e8 88 13 00 00       	call   77ed98c0 <_memset>
77ed8538:	83 c4 10             	add    $0x10,%esp
77ed853b:	c6 45 af 01          	movb   $0x1,0xffffffaf(%ebp)
77ed853f:	85 db                	test   %ebx,%ebx
77ed8541:	74 0e                	je     77ed8551 <_EnumFontFamiliesW@16+0x31>
77ed8543:	50                   	push   %eax
77ed8544:	8d 45 b4             	lea    0xffffffb4(%ebp),%eax
77ed8547:	6a 20                	push   $0x20
77ed8549:	53                   	push   %ebx
77ed854a:	50                   	push   %eax
77ed854b:	e8 00 14 00 00       	call   77ed9950 <_lstrcpynW@12>
77ed8550:	58                   	pop    %eax
77ed8551:	8b 4d 14             	mov    0x14(%ebp),%ecx
77ed8554:	8b 55 10             	mov    0x10(%ebp),%edx
77ed8557:	53                   	push   %ebx
77ed8558:	6a 01                	push   $0x1
77ed855a:	51                   	push   %ecx
77ed855b:	8b 4d 08             	mov    0x8(%ebp),%ecx
77ed855e:	52                   	push   %edx
77ed855f:	89 f2                	mov    %esi,%edx
77ed8561:	e8 5a fd ff ff       	call   77ed82c0 <@IntEnumFontFamilies@20>
77ed8566:	8d 65 f8             	lea    0xfffffff8(%ebp),%esp
77ed8569:	5b                   	pop    %ebx
77ed856a:	5e                   	pop    %esi
77ed856b:	5d                   	pop    %ebp
77ed856c:	c2 10 00             	ret    $0x10
77ed856f:	90                   	nop    

77ed8570 <_EnumFontFamiliesExA@20>:
77ed8570:	55                   	push   %ebp
77ed8571:	89 e5                	mov    %esp,%ebp
77ed8573:	53                   	push   %ebx
77ed8574:	83 ec 6c             	sub    $0x6c,%esp
77ed8577:	8b 45 0c             	mov    0xc(%ebp),%eax
77ed857a:	8d 5d 98             	lea    0xffffff98(%ebp),%ebx
77ed857d:	50                   	push   %eax
77ed857e:	53                   	push   %ebx
77ed857f:	e8 3c 0e 00 00       	call   77ed93c0 <_RosRtlLogFontA2W>
77ed8584:	83 c4 0c             	add    $0xc,%esp
77ed8587:	8b 45 14             	mov    0x14(%ebp),%eax
77ed858a:	6a 00                	push   $0x0
77ed858c:	89 da                	mov    %ebx,%edx
77ed858e:	50                   	push   %eax
77ed858f:	8b 4d 08             	mov    0x8(%ebp),%ecx
77ed8592:	8b 45 10             	mov    0x10(%ebp),%eax
77ed8595:	50                   	push   %eax
77ed8596:	e8 25 fd ff ff       	call   77ed82c0 <@IntEnumFontFamilies@20>
77ed859b:	8b 5d fc             	mov    0xfffffffc(%ebp),%ebx
77ed859e:	c9                   	leave  
77ed859f:	c2 14 00             	ret    $0x14
77ed85a2:	8d b4 26 00 00 00 00 	lea    0x0(%esi),%esi
77ed85a9:	8d bc 27 00 00 00 00 	lea    0x0(%edi),%edi

77ed85b0 <_EnumFontFamiliesA@16>:
77ed85b0:	55                   	push   %ebp
77ed85b1:	89 e5                	mov    %esp,%ebp
77ed85b3:	56                   	push   %esi
77ed85b4:	53                   	push   %ebx
77ed85b5:	83 ec 64             	sub    $0x64,%esp
77ed85b8:	8d 75 98             	lea    0xffffff98(%ebp),%esi
77ed85bb:	8b 5d 0c             	mov    0xc(%ebp),%ebx
77ed85be:	6a 5c                	push   $0x5c
77ed85c0:	6a 00                	push   $0x0
77ed85c2:	56                   	push   %esi
77ed85c3:	e8 f8 12 00 00       	call   77ed98c0 <_memset>
77ed85c8:	83 c4 10             	add    $0x10,%esp
77ed85cb:	c6 45 af 01          	movb   $0x1,0xffffffaf(%ebp)
77ed85cf:	85 db                	test   %ebx,%ebx
77ed85d1:	74 16                	je     77ed85e9 <_EnumFontFamiliesA@16+0x39>
77ed85d3:	50                   	push   %eax
77ed85d4:	50                   	push   %eax
77ed85d5:	8d 45 b4             	lea    0xffffffb4(%ebp),%eax
77ed85d8:	6a 20                	push   $0x20
77ed85da:	50                   	push   %eax
77ed85db:	6a ff                	push   $0xffffffff
77ed85dd:	53                   	push   %ebx
77ed85de:	6a 00                	push   $0x0
77ed85e0:	6a 03                	push   $0x3
77ed85e2:	e8 79 13 00 00       	call   77ed9960 <_MultiByteToWideChar@24>
77ed85e7:	5b                   	pop    %ebx
77ed85e8:	58                   	pop    %eax
77ed85e9:	8b 55 14             	mov    0x14(%ebp),%edx
77ed85ec:	8b 45 10             	mov    0x10(%ebp),%eax
77ed85ef:	51                   	push   %ecx
77ed85f0:	8b 4d 08             	mov    0x8(%ebp),%ecx
77ed85f3:	6a 00                	push   $0x0
77ed85f5:	52                   	push   %edx
77ed85f6:	89 f2                	mov    %esi,%edx
77ed85f8:	50                   	push   %eax
77ed85f9:	e8 c2 fc ff ff       	call   77ed82c0 <@IntEnumFontFamilies@20>
77ed85fe:	8d 65 f8             	lea    0xfffffff8(%ebp),%esp
77ed8601:	5b                   	pop    %ebx
77ed8602:	5e                   	pop    %esi
77ed8603:	5d                   	pop    %ebp
77ed8604:	c2 10 00             	ret    $0x10
77ed8607:	89 f6                	mov    %esi,%esi
77ed8609:	8d bc 27 00 00 00 00 	lea    0x0(%edi),%edi

77ed8610 <_GetCharWidthA@16>:
77ed8610:	55                   	push   %ebp
77ed8611:	89 e5                	mov    %esp,%ebp
77ed8613:	c9                   	leave  
77ed8614:	e9 f4 d3 ff ff       	jmp    77ed5a0d <_NtGdiGetCharWidth32@16>
77ed8619:	8d b4 26 00 00 00 00 	lea    0x0(%esi),%esi

77ed8620 <_GetCharWidth32A@16>:
77ed8620:	55                   	push   %ebp
77ed8621:	89 e5                	mov    %esp,%ebp
77ed8623:	c9                   	leave  
77ed8624:	e9 e4 d3 ff ff       	jmp    77ed5a0d <_NtGdiGetCharWidth32@16>
77ed8629:	8d b4 26 00 00 00 00 	lea    0x0(%esi),%esi

77ed8630 <_GetCharWidthW@16>:
77ed8630:	55                   	push   %ebp
77ed8631:	89 e5                	mov    %esp,%ebp
77ed8633:	c9                   	leave  
77ed8634:	e9 d4 d3 ff ff       	jmp    77ed5a0d <_NtGdiGetCharWidth32@16>
77ed8639:	8d b4 26 00 00 00 00 	lea    0x0(%esi),%esi

77ed8640 <_GetCharacterPlacementW@24>:
77ed8640:	55                   	push   %ebp
77ed8641:	89 e5                	mov    %esp,%ebp
77ed8643:	57                   	push   %edi
77ed8644:	56                   	push   %esi
77ed8645:	53                   	push   %ebx
77ed8646:	83 ec 1c             	sub    $0x1c,%esp
77ed8649:	c7 45 dc 00 00 00 00 	movl   $0x0,0xffffffdc(%ebp)
77ed8650:	8b 55 18             	mov    0x18(%ebp),%edx
77ed8653:	8b 7d 10             	mov    0x10(%ebp),%edi
77ed8656:	8b 42 1c             	mov    0x1c(%edx),%eax
77ed8659:	39 f8                	cmp    %edi,%eax
77ed865b:	73 02                	jae    77ed865f <_GetCharacterPlacementW@24+0x1f>
77ed865d:	89 c7                	mov    %eax,%edi
77ed865f:	8b 45 18             	mov    0x18(%ebp),%eax
77ed8662:	89 78 1c             	mov    %edi,0x1c(%eax)
77ed8665:	8b 40 04             	mov    0x4(%eax),%eax
77ed8668:	85 c0                	test   %eax,%eax
77ed866a:	0f 85 24 01 00 00    	jne    77ed8794 <_GetCharacterPlacementW@24+0x154>
77ed8670:	8b 55 18             	mov    0x18(%ebp),%edx
77ed8673:	8b 42 18             	mov    0x18(%edx),%eax
77ed8676:	85 c0                	test   %eax,%eax
77ed8678:	0f 85 02 01 00 00    	jne    77ed8780 <_GetCharacterPlacementW@24+0x140>
77ed867e:	8b 55 18             	mov    0x18(%ebp),%edx
77ed8681:	8b 42 08             	mov    0x8(%edx),%eax
77ed8684:	85 c0                	test   %eax,%eax
77ed8686:	74 10                	je     77ed8698 <_GetCharacterPlacementW@24+0x58>
77ed8688:	31 db                	xor    %ebx,%ebx
77ed868a:	39 7d dc             	cmp    %edi,0xffffffdc(%ebp)
77ed868d:	eb 07                	jmp    77ed8696 <_GetCharacterPlacementW@24+0x56>
77ed868f:	90                   	nop    
77ed8690:	89 1c 98             	mov    %ebx,(%eax,%ebx,4)
77ed8693:	43                   	inc    %ebx
77ed8694:	39 fb                	cmp    %edi,%ebx
77ed8696:	72 f8                	jb     77ed8690 <_GetCharacterPlacementW@24+0x50>
77ed8698:	8b 45 18             	mov    0x18(%ebp),%eax
77ed869b:	8b 40 0c             	mov    0xc(%eax),%eax
77ed869e:	85 c0                	test   %eax,%eax
77ed86a0:	74 3e                	je     77ed86e0 <_GetCharacterPlacementW@24+0xa0>
77ed86a2:	31 db                	xor    %ebx,%ebx
77ed86a4:	39 fb                	cmp    %edi,%ebx
77ed86a6:	73 38                	jae    77ed86e0 <_GetCharacterPlacementW@24+0xa0>
77ed86a8:	8d 75 ec             	lea    0xffffffec(%ebp),%esi
77ed86ab:	90                   	nop    
77ed86ac:	8d 74 26 00          	lea    0x0(%esi),%esi
77ed86b0:	8b 55 0c             	mov    0xc(%ebp),%edx
77ed86b3:	56                   	push   %esi
77ed86b4:	66 8b 04 5a          	mov    (%edx,%ebx,2),%ax
77ed86b8:	25 ff ff 00 00       	and    $0xffff,%eax
77ed86bd:	50                   	push   %eax
77ed86be:	50                   	push   %eax
77ed86bf:	8b 45 08             	mov    0x8(%ebp),%eax
77ed86c2:	50                   	push   %eax
77ed86c3:	e8 45 d3 ff ff       	call   77ed5a0d <_NtGdiGetCharWidth32@16>
77ed86c8:	85 c0                	test   %eax,%eax
77ed86ca:	74 0c                	je     77ed86d8 <_GetCharacterPlacementW@24+0x98>
77ed86cc:	8b 45 18             	mov    0x18(%ebp),%eax
77ed86cf:	8b 50 0c             	mov    0xc(%eax),%edx
77ed86d2:	8b 45 ec             	mov    0xffffffec(%ebp),%eax
77ed86d5:	89 04 9a             	mov    %eax,(%edx,%ebx,4)
77ed86d8:	43                   	inc    %ebx
77ed86d9:	39 fb                	cmp    %edi,%ebx
77ed86db:	72 d3                	jb     77ed86b0 <_GetCharacterPlacementW@24+0x70>
77ed86dd:	8d 76 00             	lea    0x0(%esi),%esi
77ed86e0:	8b 55 18             	mov    0x18(%ebp),%edx
77ed86e3:	8b 42 10             	mov    0x10(%edx),%eax
77ed86e6:	85 c0                	test   %eax,%eax
77ed86e8:	74 06                	je     77ed86f0 <_GetCharacterPlacementW@24+0xb0>
77ed86ea:	f6 45 1c 02          	testb  $0x2,0x1c(%ebp)
77ed86ee:	74 3f                	je     77ed872f <_GetCharacterPlacementW@24+0xef>
77ed86f0:	8d 45 e0             	lea    0xffffffe0(%ebp),%eax
77ed86f3:	8b 75 10             	mov    0x10(%ebp),%esi
77ed86f6:	8b 5d 0c             	mov    0xc(%ebp),%ebx
77ed86f9:	8b 4d 08             	mov    0x8(%ebp),%ecx
77ed86fc:	50                   	push   %eax
77ed86fd:	56                   	push   %esi
77ed86fe:	53                   	push   %ebx
77ed86ff:	51                   	push   %ecx
77ed8700:	e8 fb 0a 00 00       	call   77ed9200 <_GetTextExtentPoint32W@16>
77ed8705:	85 c0                	test   %eax,%eax
77ed8707:	74 19                	je     77ed8722 <_GetCharacterPlacementW@24+0xe2>
77ed8709:	8b 45 e0             	mov    0xffffffe0(%ebp),%eax
77ed870c:	25 ff ff 00 00       	and    $0xffff,%eax
77ed8711:	89 45 dc             	mov    %eax,0xffffffdc(%ebp)
77ed8714:	8b 45 e4             	mov    0xffffffe4(%ebp),%eax
77ed8717:	c1 e0 10             	shl    $0x10,%eax
77ed871a:	8b 55 dc             	mov    0xffffffdc(%ebp),%edx
77ed871d:	09 c2                	or     %eax,%edx
77ed871f:	89 55 dc             	mov    %edx,0xffffffdc(%ebp)
77ed8722:	8b 45 dc             	mov    0xffffffdc(%ebp),%eax
77ed8725:	8d 65 f4             	lea    0xfffffff4(%ebp),%esp
77ed8728:	5b                   	pop    %ebx
77ed8729:	5e                   	pop    %esi
77ed872a:	5f                   	pop    %edi
77ed872b:	5d                   	pop    %ebp
77ed872c:	c2 18 00             	ret    $0x18
77ed872f:	bb 01 00 00 00       	mov    $0x1,%ebx
77ed8734:	c7 45 d8 00 00 00 00 	movl   $0x0,0xffffffd8(%ebp)
77ed873b:	c7 00 00 00 00 00    	movl   $0x0,(%eax)
77ed8741:	39 fb                	cmp    %edi,%ebx
77ed8743:	73 ab                	jae    77ed86f0 <_GetCharacterPlacementW@24+0xb0>
77ed8745:	8b 75 0c             	mov    0xc(%ebp),%esi
77ed8748:	8d 45 e0             	lea    0xffffffe0(%ebp),%eax
77ed874b:	50                   	push   %eax
77ed874c:	8b 45 08             	mov    0x8(%ebp),%eax
77ed874f:	6a 01                	push   $0x1
77ed8751:	56                   	push   %esi
77ed8752:	50                   	push   %eax
77ed8753:	e8 a8 0a 00 00       	call   77ed9200 <_GetTextExtentPoint32W@16>
77ed8758:	85 c0                	test   %eax,%eax
77ed875a:	74 17                	je     77ed8773 <_GetCharacterPlacementW@24+0x133>
77ed875c:	8b 55 18             	mov    0x18(%ebp),%edx
77ed875f:	8b 4d d8             	mov    0xffffffd8(%ebp),%ecx
77ed8762:	8b 42 10             	mov    0x10(%edx),%eax
77ed8765:	8b 55 e0             	mov    0xffffffe0(%ebp),%edx
77ed8768:	01 d1                	add    %edx,%ecx
77ed876a:	89 4d d8             	mov    %ecx,0xffffffd8(%ebp)
77ed876d:	8b 55 d8             	mov    0xffffffd8(%ebp),%edx
77ed8770:	89 14 98             	mov    %edx,(%eax,%ebx,4)
77ed8773:	43                   	inc    %ebx
77ed8774:	83 c6 02             	add    $0x2,%esi
77ed8777:	39 fb                	cmp    %edi,%ebx
77ed8779:	72 cd                	jb     77ed8748 <_GetCharacterPlacementW@24+0x108>
77ed877b:	e9 70 ff ff ff       	jmp    77ed86f0 <_GetCharacterPlacementW@24+0xb0>
77ed8780:	8b 55 0c             	mov    0xc(%ebp),%edx
77ed8783:	51                   	push   %ecx
77ed8784:	57                   	push   %edi
77ed8785:	52                   	push   %edx
77ed8786:	50                   	push   %eax
77ed8787:	e8 24 11 00 00       	call   77ed98b0 <_wcsncpy>
77ed878c:	83 c4 10             	add    $0x10,%esp
77ed878f:	e9 ea fe ff ff       	jmp    77ed867e <_GetCharacterPlacementW@24+0x3e>
77ed8794:	8b 5d 0c             	mov    0xc(%ebp),%ebx
77ed8797:	56                   	push   %esi
77ed8798:	57                   	push   %edi
77ed8799:	53                   	push   %ebx
77ed879a:	50                   	push   %eax
77ed879b:	e8 10 11 00 00       	call   77ed98b0 <_wcsncpy>
77ed87a0:	83 c4 10             	add    $0x10,%esp
77ed87a3:	e9 c8 fe ff ff       	jmp    77ed8670 <_GetCharacterPlacementW@24+0x30>
77ed87a8:	90                   	nop    
77ed87a9:	8d b4 26 00 00 00 00 	lea    0x0(%esi),%esi

77ed87b0 <_GetCharWidthFloatA@16>:
77ed87b0:	55                   	push   %ebp
77ed87b1:	89 e5                	mov    %esp,%ebp
77ed87b3:	c9                   	leave  
77ed87b4:	e9 63 d2 ff ff       	jmp    77ed5a1c <_NtGdiGetCharWidthFloat@16>
77ed87b9:	8d b4 26 00 00 00 00 	lea    0x0(%esi),%esi

77ed87c0 <_GetCharABCWidthsA@16>:
77ed87c0:	55                   	push   %ebp
77ed87c1:	89 e5                	mov    %esp,%ebp
77ed87c3:	c9                   	leave  
77ed87c4:	e9 17 d2 ff ff       	jmp    77ed59e0 <_NtGdiGetCharABCWidths@16>
77ed87c9:	8d b4 26 00 00 00 00 	lea    0x0(%esi),%esi

77ed87d0 <_GetCharABCWidthsFloatA@16>:
77ed87d0:	55                   	push   %ebp
77ed87d1:	89 e5                	mov    %esp,%ebp
77ed87d3:	c9                   	leave  
77ed87d4:	e9 16 d2 ff ff       	jmp    77ed59ef <_NtGdiGetCharABCWidthsFloat@16>
77ed87d9:	8d b4 26 00 00 00 00 	lea    0x0(%esi),%esi

77ed87e0 <_GetGlyphOutlineA@28>:
77ed87e0:	55                   	push   %ebp
77ed87e1:	89 e5                	mov    %esp,%ebp
77ed87e3:	c9                   	leave  
77ed87e4:	e9 6e d3 ff ff       	jmp    77ed5b57 <_NtGdiGetGlyphOutline@28>
77ed87e9:	8d b4 26 00 00 00 00 	lea    0x0(%esi),%esi

77ed87f0 <_CreateFontIndirectA@4>:
77ed87f0:	55                   	push   %ebp
77ed87f1:	89 e5                	mov    %esp,%ebp
77ed87f3:	53                   	push   %ebx
77ed87f4:	83 ec 6c             	sub    $0x6c,%esp
77ed87f7:	8b 45 08             	mov    0x8(%ebp),%eax
77ed87fa:	8d 5d 98             	lea    0xffffff98(%ebp),%ebx
77ed87fd:	50                   	push   %eax
77ed87fe:	53                   	push   %ebx
77ed87ff:	e8 bc 0b 00 00       	call   77ed93c0 <_RosRtlLogFontA2W>
77ed8804:	89 1c 24             	mov    %ebx,(%esp)
77ed8807:	e8 50 ce ff ff       	call   77ed565c <_NtGdiCreateFontIndirect@4>
77ed880c:	8b 5d fc             	mov    0xfffffffc(%ebp),%ebx
77ed880f:	c9                   	leave  
77ed8810:	c2 04 00             	ret    $0x4
77ed8813:	8d b6 00 00 00 00    	lea    0x0(%esi),%esi
77ed8819:	8d bc 27 00 00 00 00 	lea    0x0(%edi),%edi

77ed8820 <_CreateFontIndirectW@4>:
77ed8820:	55                   	push   %ebp
77ed8821:	89 e5                	mov    %esp,%ebp
77ed8823:	c9                   	leave  
77ed8824:	e9 33 ce ff ff       	jmp    77ed565c <_NtGdiCreateFontIndirect@4>
77ed8829:	8d b4 26 00 00 00 00 	lea    0x0(%esi),%esi

77ed8830 <_CreateFontW@56>:
77ed8830:	55                   	push   %ebp
77ed8831:	89 e5                	mov    %esp,%ebp
77ed8833:	c9                   	leave  
77ed8834:	e9 14 ce ff ff       	jmp    77ed564d <_NtGdiCreateFont@56>
77ed8839:	8d b4 26 00 00 00 00 	lea    0x0(%esi),%esi

77ed8840 <_CreateFontA@56>:
77ed8840:	55                   	push   %ebp
77ed8841:	89 e5                	mov    %esp,%ebp
77ed8843:	56                   	push   %esi
77ed8844:	53                   	push   %ebx
77ed8845:	83 ec 18             	sub    $0x18,%esp
77ed8848:	8d 75 e8             	lea    0xffffffe8(%ebp),%esi
77ed884b:	8b 5d 3c             	mov    0x3c(%ebp),%ebx
77ed884e:	53                   	push   %ebx
77ed884f:	8d 5d f0             	lea    0xfffffff0(%ebp),%ebx
77ed8852:	53                   	push   %ebx
77ed8853:	e8 08 10 00 00       	call   77ed9860 <_RtlInitAnsiString@8>
77ed8858:	c7 04 24 01 00 00 00 	movl   $0x1,(%esp)
77ed885f:	53                   	push   %ebx
77ed8860:	56                   	push   %esi
77ed8861:	e8 0a 10 00 00       	call   77ed9870 <_RtlAnsiStringToUnicodeString@12>
77ed8866:	8b 55 ec             	mov    0xffffffec(%ebp),%edx
77ed8869:	8b 45 38             	mov    0x38(%ebp),%eax
77ed886c:	51                   	push   %ecx
77ed886d:	52                   	push   %edx
77ed886e:	50                   	push   %eax
77ed886f:	8b 45 34             	mov    0x34(%ebp),%eax
77ed8872:	50                   	push   %eax
77ed8873:	8b 45 30             	mov    0x30(%ebp),%eax
77ed8876:	50                   	push   %eax
77ed8877:	8b 45 2c             	mov    0x2c(%ebp),%eax
77ed887a:	50                   	push   %eax
77ed887b:	8b 45 28             	mov    0x28(%ebp),%eax
77ed887e:	50                   	push   %eax
77ed887f:	8b 45 24             	mov    0x24(%ebp),%eax
77ed8882:	50                   	push   %eax
77ed8883:	8b 5d 20             	mov    0x20(%ebp),%ebx
77ed8886:	8b 4d 1c             	mov    0x1c(%ebp),%ecx
77ed8889:	8b 55 18             	mov    0x18(%ebp),%edx
77ed888c:	8b 45 14             	mov    0x14(%ebp),%eax
77ed888f:	53                   	push   %ebx
77ed8890:	51                   	push   %ecx
77ed8891:	52                   	push   %edx
77ed8892:	50                   	push   %eax
77ed8893:	8b 45 10             	mov    0x10(%ebp),%eax
77ed8896:	50                   	push   %eax
77ed8897:	8b 45 0c             	mov    0xc(%ebp),%eax
77ed889a:	50                   	push   %eax
77ed889b:	8b 45 08             	mov    0x8(%ebp),%eax
77ed889e:	50                   	push   %eax
77ed889f:	e8 8c ff ff ff       	call   77ed8830 <_CreateFontW@56>
77ed88a4:	89 c3                	mov    %eax,%ebx
77ed88a6:	50                   	push   %eax
77ed88a7:	56                   	push   %esi
77ed88a8:	e8 d3 0f 00 00       	call   77ed9880 <_RtlFreeUnicodeString@4>
77ed88ad:	8d 65 f8             	lea    0xfffffff8(%ebp),%esp
77ed88b0:	89 d8                	mov    %ebx,%eax
77ed88b2:	5b                   	pop    %ebx
77ed88b3:	5e                   	pop    %esi
77ed88b4:	5d                   	pop    %ebp
77ed88b5:	c2 38 00             	ret    $0x38
77ed88b8:	90                   	nop    
77ed88b9:	8d b4 26 00 00 00 00 	lea    0x0(%esi),%esi

77ed88c0 <_CreateScalableFontResourceW@16>:
77ed88c0:	55                   	push   %ebp
77ed88c1:	89 e5                	mov    %esp,%ebp
77ed88c3:	c9                   	leave  
77ed88c4:	e9 65 ce ff ff       	jmp    77ed572e <_NtGdiCreateScalableFontResource@16>
77ed88c9:	8d b4 26 00 00 00 00 	lea    0x0(%esi),%esi

77ed88d0 <_CreateScalableFontResourceA@16>:
77ed88d0:	55                   	push   %ebp
77ed88d1:	89 e5                	mov    %esp,%ebp
77ed88d3:	53                   	push   %ebx
77ed88d4:	83 ec 1c             	sub    $0x1c,%esp
77ed88d7:	31 db                	xor    %ebx,%ebx
77ed88d9:	8b 45 0c             	mov    0xc(%ebp),%eax
77ed88dc:	50                   	push   %eax
77ed88dd:	8d 45 f8             	lea    0xfffffff8(%ebp),%eax
77ed88e0:	50                   	push   %eax
77ed88e1:	e8 ea 87 ff ff       	call   77ed10d0 <_HEAP_strdupA2W>
77ed88e6:	83 c4 10             	add    $0x10,%esp
77ed88e9:	85 c0                	test   %eax,%eax
77ed88eb:	0f 88 7f 00 00 00    	js     77ed8970 <_CreateScalableFontResourceA@16+0xa0>
77ed88f1:	50                   	push   %eax
77ed88f2:	50                   	push   %eax
77ed88f3:	8b 45 10             	mov    0x10(%ebp),%eax
77ed88f6:	50                   	push   %eax
77ed88f7:	8d 45 f4             	lea    0xfffffff4(%ebp),%eax
77ed88fa:	50                   	push   %eax
77ed88fb:	e8 d0 87 ff ff       	call   77ed10d0 <_HEAP_strdupA2W>
77ed8900:	83 c4 10             	add    $0x10,%esp
77ed8903:	85 c0                	test   %eax,%eax
77ed8905:	0f 88 99 00 00 00    	js     77ed89a4 <_CreateScalableFontResourceA@16+0xd4>
77ed890b:	50                   	push   %eax
77ed890c:	50                   	push   %eax
77ed890d:	8d 45 f0             	lea    0xfffffff0(%ebp),%eax
77ed8910:	8b 4d 14             	mov    0x14(%ebp),%ecx
77ed8913:	51                   	push   %ecx
77ed8914:	50                   	push   %eax
77ed8915:	e8 b6 87 ff ff       	call   77ed10d0 <_HEAP_strdupA2W>
77ed891a:	83 c4 10             	add    $0x10,%esp
77ed891d:	85 c0                	test   %eax,%eax
77ed891f:	78 6f                	js     77ed8990 <_CreateScalableFontResourceA@16+0xc0>
77ed8921:	8b 55 f0             	mov    0xfffffff0(%ebp),%edx
77ed8924:	52                   	push   %edx
77ed8925:	8b 45 f4             	mov    0xfffffff4(%ebp),%eax
77ed8928:	50                   	push   %eax
77ed8929:	8b 45 f8             	mov    0xfffffff8(%ebp),%eax
77ed892c:	50                   	push   %eax
77ed892d:	8b 45 08             	mov    0x8(%ebp),%eax
77ed8930:	50                   	push   %eax
77ed8931:	e8 f8 cd ff ff       	call   77ed572e <_NtGdiCreateScalableFontResource@16>
77ed8936:	83 ec 0c             	sub    $0xc,%esp
77ed8939:	89 c3                	mov    %eax,%ebx
77ed893b:	8b 45 f0             	mov    0xfffffff0(%ebp),%eax
77ed893e:	50                   	push   %eax
77ed893f:	e8 fc 87 ff ff       	call   77ed1140 <_HEAP_free>
77ed8944:	83 c4 10             	add    $0x10,%esp
77ed8947:	83 ec 0c             	sub    $0xc,%esp
77ed894a:	8b 45 f4             	mov    0xfffffff4(%ebp),%eax
77ed894d:	50                   	push   %eax
77ed894e:	e8 ed 87 ff ff       	call   77ed1140 <_HEAP_free>
77ed8953:	83 c4 10             	add    $0x10,%esp
77ed8956:	83 ec 0c             	sub    $0xc,%esp
77ed8959:	8b 45 f8             	mov    0xfffffff8(%ebp),%eax
77ed895c:	50                   	push   %eax
77ed895d:	e8 de 87 ff ff       	call   77ed1140 <_HEAP_free>
77ed8962:	89 d8                	mov    %ebx,%eax
77ed8964:	83 c4 10             	add    $0x10,%esp
77ed8967:	8b 5d fc             	mov    0xfffffffc(%ebp),%ebx
77ed896a:	c9                   	leave  
77ed896b:	c2 10 00             	ret    $0x10
77ed896e:	89 f6                	mov    %esi,%esi
77ed8970:	83 ec 0c             	sub    $0xc,%esp
77ed8973:	50                   	push   %eax
77ed8974:	e8 17 0f 00 00       	call   77ed9890 <_RtlNtStatusToDosError@4>
77ed8979:	50                   	push   %eax
77ed897a:	e8 91 0f 00 00       	call   77ed9910 <_SetLastError@4>
77ed897f:	89 d8                	mov    %ebx,%eax
77ed8981:	83 c4 0c             	add    $0xc,%esp
77ed8984:	8b 5d fc             	mov    0xfffffffc(%ebp),%ebx
77ed8987:	c9                   	leave  
77ed8988:	c2 10 00             	ret    $0x10
77ed898b:	90                   	nop    
77ed898c:	8d 74 26 00          	lea    0x0(%esi),%esi
77ed8990:	83 ec 0c             	sub    $0xc,%esp
77ed8993:	50                   	push   %eax
77ed8994:	e8 f7 0e 00 00       	call   77ed9890 <_RtlNtStatusToDosError@4>
77ed8999:	50                   	push   %eax
77ed899a:	e8 71 0f 00 00       	call   77ed9910 <_SetLastError@4>
77ed899f:	83 c4 0c             	add    $0xc,%esp
77ed89a2:	eb a3                	jmp    77ed8947 <_CreateScalableFontResourceA@16+0x77>
77ed89a4:	83 ec 0c             	sub    $0xc,%esp
77ed89a7:	50                   	push   %eax
77ed89a8:	e8 e3 0e 00 00       	call   77ed9890 <_RtlNtStatusToDosError@4>
77ed89ad:	50                   	push   %eax
77ed89ae:	e8 5d 0f 00 00       	call   77ed9910 <_SetLastError@4>
77ed89b3:	83 c4 0c             	add    $0xc,%esp
77ed89b6:	eb 9e                	jmp    77ed8956 <_CreateScalableFontResourceA@16+0x86>
77ed89b8:	90                   	nop    
77ed89b9:	8d b4 26 00 00 00 00 	lea    0x0(%esi),%esi

77ed89c0 <_AddFontResourceExW@12>:
77ed89c0:	55                   	push   %ebp
77ed89c1:	89 e5                	mov    %esp,%ebp
77ed89c3:	53                   	push   %ebx
77ed89c4:	83 ec 1c             	sub    $0x1c,%esp
77ed89c7:	8b 45 08             	mov    0x8(%ebp),%eax
77ed89ca:	8d 5d f0             	lea    0xfffffff0(%ebp),%ebx
77ed89cd:	50                   	push   %eax
77ed89ce:	53                   	push   %ebx
77ed89cf:	e8 7c 0e 00 00       	call   77ed9850 <_RtlInitUnicodeString@8>
77ed89d4:	8b 45 0c             	mov    0xc(%ebp),%eax
77ed89d7:	50                   	push   %eax
77ed89d8:	53                   	push   %ebx
77ed89d9:	e8 80 ca ff ff       	call   77ed545e <_NtGdiAddFontResource@8>
77ed89de:	8b 5d fc             	mov    0xfffffffc(%ebp),%ebx
77ed89e1:	c9                   	leave  
77ed89e2:	c2 0c 00             	ret    $0xc
77ed89e5:	8d 74 26 00          	lea    0x0(%esi),%esi
77ed89e9:	8d bc 27 00 00 00 00 	lea    0x0(%edi),%edi

77ed89f0 <_AddFontResourceExA@12>:
77ed89f0:	55                   	push   %ebp
77ed89f1:	89 e5                	mov    %esp,%ebp
77ed89f3:	53                   	push   %ebx
77ed89f4:	83 ec 0c             	sub    $0xc,%esp
77ed89f7:	31 db                	xor    %ebx,%ebx
77ed89f9:	8b 45 08             	mov    0x8(%ebp),%eax
77ed89fc:	50                   	push   %eax
77ed89fd:	8d 45 f8             	lea    0xfffffff8(%ebp),%eax
77ed8a00:	50                   	push   %eax
77ed8a01:	e8 ca 86 ff ff       	call   77ed10d0 <_HEAP_strdupA2W>
77ed8a06:	83 c4 10             	add    $0x10,%esp
77ed8a09:	85 c0                	test   %eax,%eax
77ed8a0b:	78 2b                	js     77ed8a38 <_AddFontResourceExA@12+0x48>
77ed8a0d:	50                   	push   %eax
77ed8a0e:	8b 45 10             	mov    0x10(%ebp),%eax
77ed8a11:	50                   	push   %eax
77ed8a12:	8b 45 0c             	mov    0xc(%ebp),%eax
77ed8a15:	50                   	push   %eax
77ed8a16:	8b 5d f8             	mov    0xfffffff8(%ebp),%ebx
77ed8a19:	53                   	push   %ebx
77ed8a1a:	e8 a1 ff ff ff       	call   77ed89c0 <_AddFontResourceExW@12>
77ed8a1f:	89 c3                	mov    %eax,%ebx
77ed8a21:	51                   	push   %ecx
77ed8a22:	51                   	push   %ecx
77ed8a23:	8b 55 f8             	mov    0xfffffff8(%ebp),%edx
77ed8a26:	52                   	push   %edx
77ed8a27:	e8 14 87 ff ff       	call   77ed1140 <_HEAP_free>
77ed8a2c:	89 d8                	mov    %ebx,%eax
77ed8a2e:	83 c4 10             	add    $0x10,%esp
77ed8a31:	8b 5d fc             	mov    0xfffffffc(%ebp),%ebx
77ed8a34:	c9                   	leave  
77ed8a35:	c2 0c 00             	ret    $0xc
77ed8a38:	83 ec 0c             	sub    $0xc,%esp
77ed8a3b:	50                   	push   %eax
77ed8a3c:	e8 4f 0e 00 00       	call   77ed9890 <_RtlNtStatusToDosError@4>
77ed8a41:	50                   	push   %eax
77ed8a42:	e8 c9 0e 00 00       	call   77ed9910 <_SetLastError@4>
77ed8a47:	89 d8                	mov    %ebx,%eax
77ed8a49:	83 c4 0c             	add    $0xc,%esp
77ed8a4c:	8b 5d fc             	mov    0xfffffffc(%ebp),%ebx
77ed8a4f:	c9                   	leave  
77ed8a50:	c2 0c 00             	ret    $0xc
77ed8a53:	8d b6 00 00 00 00    	lea    0x0(%esi),%esi
77ed8a59:	8d bc 27 00 00 00 00 	lea    0x0(%edi),%edi

77ed8a60 <_AddFontResourceA@4>:
77ed8a60:	55                   	push   %ebp
77ed8a61:	89 e5                	mov    %esp,%ebp
77ed8a63:	83 ec 0c             	sub    $0xc,%esp
77ed8a66:	8b 45 08             	mov    0x8(%ebp),%eax
77ed8a69:	6a 00                	push   $0x0
77ed8a6b:	6a 00                	push   $0x0
77ed8a6d:	50                   	push   %eax
77ed8a6e:	e8 7d ff ff ff       	call   77ed89f0 <_AddFontResourceExA@12>
77ed8a73:	c9                   	leave  
77ed8a74:	c2 04 00             	ret    $0x4
77ed8a77:	89 f6                	mov    %esi,%esi
77ed8a79:	8d bc 27 00 00 00 00 	lea    0x0(%edi),%edi

77ed8a80 <_AddFontResourceW@4>:
77ed8a80:	55                   	push   %ebp
77ed8a81:	89 e5                	mov    %esp,%ebp
77ed8a83:	83 ec 0c             	sub    $0xc,%esp
77ed8a86:	8b 45 08             	mov    0x8(%ebp),%eax
77ed8a89:	6a 00                	push   $0x0
77ed8a8b:	6a 00                	push   $0x0
77ed8a8d:	50                   	push   %eax
77ed8a8e:	e8 2d ff ff ff       	call   77ed89c0 <_AddFontResourceExW@12>
77ed8a93:	c9                   	leave  
77ed8a94:	c2 04 00             	ret    $0x4
77ed8a97:	89 f6                	mov    %esi,%esi
77ed8a99:	8d bc 27 00 00 00 00 	lea    0x0(%edi),%edi

77ed8aa0 <_RemoveFontResourceW@4>:
77ed8aa0:	55                   	push   %ebp
77ed8aa1:	89 e5                	mov    %esp,%ebp
77ed8aa3:	c9                   	leave  
77ed8aa4:	e9 6d d5 ff ff       	jmp    77ed6016 <_NtGdiRemoveFontResource@4>
77ed8aa9:	8d b4 26 00 00 00 00 	lea    0x0(%esi),%esi

77ed8ab0 <_RemoveFontResourceA@4>:
77ed8ab0:	55                   	push   %ebp
77ed8ab1:	89 e5                	mov    %esp,%ebp
77ed8ab3:	53                   	push   %ebx
77ed8ab4:	83 ec 0c             	sub    $0xc,%esp
77ed8ab7:	31 db                	xor    %ebx,%ebx
77ed8ab9:	8b 45 08             	mov    0x8(%ebp),%eax
77ed8abc:	50                   	push   %eax
77ed8abd:	8d 45 f8             	lea    0xfffffff8(%ebp),%eax
77ed8ac0:	50                   	push   %eax
77ed8ac1:	e8 0a 86 ff ff       	call   77ed10d0 <_HEAP_strdupA2W>
77ed8ac6:	83 c4 10             	add    $0x10,%esp
77ed8ac9:	85 c0                	test   %eax,%eax
77ed8acb:	78 23                	js     77ed8af0 <_RemoveFontResourceA@4+0x40>
77ed8acd:	83 ec 0c             	sub    $0xc,%esp
77ed8ad0:	8b 4d f8             	mov    0xfffffff8(%ebp),%ecx
77ed8ad3:	51                   	push   %ecx
77ed8ad4:	e8 3d d5 ff ff       	call   77ed6016 <_NtGdiRemoveFontResource@4>
77ed8ad9:	8b 55 f8             	mov    0xfffffff8(%ebp),%edx
77ed8adc:	89 c3                	mov    %eax,%ebx
77ed8ade:	52                   	push   %edx
77ed8adf:	e8 5c 86 ff ff       	call   77ed1140 <_HEAP_free>
77ed8ae4:	89 d8                	mov    %ebx,%eax
77ed8ae6:	83 c4 10             	add    $0x10,%esp
77ed8ae9:	8b 5d fc             	mov    0xfffffffc(%ebp),%ebx
77ed8aec:	c9                   	leave  
77ed8aed:	c2 04 00             	ret    $0x4
77ed8af0:	83 ec 0c             	sub    $0xc,%esp
77ed8af3:	50                   	push   %eax
77ed8af4:	e8 97 0d 00 00       	call   77ed9890 <_RtlNtStatusToDosError@4>
77ed8af9:	50                   	push   %eax
77ed8afa:	e8 11 0e 00 00       	call   77ed9910 <_SetLastError@4>
77ed8aff:	89 d8                	mov    %ebx,%eax
77ed8b01:	83 c4 0c             	add    $0xc,%esp
77ed8b04:	8b 5d fc             	mov    0xfffffffc(%ebp),%ebx
77ed8b07:	c9                   	leave  
77ed8b08:	c2 04 00             	ret    $0x4
77ed8b0b:	90                   	nop    
77ed8b0c:	90                   	nop    
77ed8b0d:	90                   	nop    
77ed8b0e:	90                   	nop    
77ed8b0f:	90                   	nop    

77ed8b10 <_LineDDA@24>:
77ed8b10:	55                   	push   %ebp
77ed8b11:	89 e5                	mov    %esp,%ebp
77ed8b13:	57                   	push   %edi
77ed8b14:	56                   	push   %esi
77ed8b15:	53                   	push   %ebx
77ed8b16:	83 ec 1c             	sub    $0x1c,%esp
77ed8b19:	c7 45 f0 01 00 00 00 	movl   $0x1,0xfffffff0(%ebp)
77ed8b20:	8b 5d 14             	mov    0x14(%ebp),%ebx
77ed8b23:	8b 7d 08             	mov    0x8(%ebp),%edi
77ed8b26:	8b 45 10             	mov    0x10(%ebp),%eax
77ed8b29:	8b 55 0c             	mov    0xc(%ebp),%edx
77ed8b2c:	29 d3                	sub    %edx,%ebx
77ed8b2e:	29 f8                	sub    %edi,%eax
77ed8b30:	c7 45 ec 01 00 00 00 	movl   $0x1,0xffffffec(%ebp)
77ed8b37:	89 5d 14             	mov    %ebx,0x14(%ebp)
77ed8b3a:	89 45 e8             	mov    %eax,0xffffffe8(%ebp)
77ed8b3d:	0f 88 e2 00 00 00    	js     77ed8c25 <_LineDDA@24+0x115>
77ed8b43:	8b 4d 14             	mov    0x14(%ebp),%ecx
77ed8b46:	85 c9                	test   %ecx,%ecx
77ed8b48:	0f 88 c8 00 00 00    	js     77ed8c16 <_LineDDA@24+0x106>
77ed8b4e:	8b 45 14             	mov    0x14(%ebp),%eax
77ed8b51:	39 45 e8             	cmp    %eax,0xffffffe8(%ebp)
77ed8b54:	7e 6a                	jle    77ed8bc0 <_LineDDA@24+0xb0>
77ed8b56:	8b 75 e8             	mov    0xffffffe8(%ebp),%esi
77ed8b59:	89 c3                	mov    %eax,%ebx
77ed8b5b:	29 f0                	sub    %esi,%eax
77ed8b5d:	01 db                	add    %ebx,%ebx
77ed8b5f:	01 c0                	add    %eax,%eax
77ed8b61:	8b 55 e8             	mov    0xffffffe8(%ebp),%edx
77ed8b64:	8b 4d e8             	mov    0xffffffe8(%ebp),%ecx
77ed8b67:	29 d3                	sub    %edx,%ebx
77ed8b69:	89 45 e4             	mov    %eax,0xffffffe4(%ebp)
77ed8b6c:	85 c9                	test   %ecx,%ecx
77ed8b6e:	78 40                	js     77ed8bb0 <_LineDDA@24+0xa0>
77ed8b70:	8b 75 e8             	mov    0xffffffe8(%ebp),%esi
77ed8b73:	46                   	inc    %esi
77ed8b74:	eb 18                	jmp    77ed8b8e <_LineDDA@24+0x7e>
77ed8b76:	8b 45 0c             	mov    0xc(%ebp),%eax
77ed8b79:	8b 55 ec             	mov    0xffffffec(%ebp),%edx
77ed8b7c:	01 d0                	add    %edx,%eax
77ed8b7e:	89 45 0c             	mov    %eax,0xc(%ebp)
77ed8b81:	8b 45 e4             	mov    0xffffffe4(%ebp),%eax
77ed8b84:	01 c3                	add    %eax,%ebx
77ed8b86:	8b 45 f0             	mov    0xfffffff0(%ebp),%eax
77ed8b89:	01 c7                	add    %eax,%edi
77ed8b8b:	4e                   	dec    %esi
77ed8b8c:	74 22                	je     77ed8bb0 <_LineDDA@24+0xa0>
77ed8b8e:	8b 45 1c             	mov    0x1c(%ebp),%eax
77ed8b91:	52                   	push   %edx
77ed8b92:	50                   	push   %eax
77ed8b93:	8b 45 0c             	mov    0xc(%ebp),%eax
77ed8b96:	50                   	push   %eax
77ed8b97:	57                   	push   %edi
77ed8b98:	ff 55 18             	call   *0x18(%ebp)
77ed8b9b:	85 db                	test   %ebx,%ebx
77ed8b9d:	58                   	pop    %eax
77ed8b9e:	7f d6                	jg     77ed8b76 <_LineDDA@24+0x66>
77ed8ba0:	8b 45 14             	mov    0x14(%ebp),%eax
77ed8ba3:	8d 1c 43             	lea    (%ebx,%eax,2),%ebx
77ed8ba6:	8b 45 f0             	mov    0xfffffff0(%ebp),%eax
77ed8ba9:	01 c7                	add    %eax,%edi
77ed8bab:	4e                   	dec    %esi
77ed8bac:	75 e0                	jne    77ed8b8e <_LineDDA@24+0x7e>
77ed8bae:	89 f6                	mov    %esi,%esi
77ed8bb0:	8d 65 f4             	lea    0xfffffff4(%ebp),%esp
77ed8bb3:	b8 01 00 00 00       	mov    $0x1,%eax
77ed8bb8:	5b                   	pop    %ebx
77ed8bb9:	5e                   	pop    %esi
77ed8bba:	5f                   	pop    %edi
77ed8bbb:	5d                   	pop    %ebp
77ed8bbc:	c2 18 00             	ret    $0x18
77ed8bbf:	90                   	nop    
77ed8bc0:	8b 45 e8             	mov    0xffffffe8(%ebp),%eax
77ed8bc3:	8b 55 14             	mov    0x14(%ebp),%edx
77ed8bc6:	29 d0                	sub    %edx,%eax
77ed8bc8:	8b 5d e8             	mov    0xffffffe8(%ebp),%ebx
77ed8bcb:	01 c0                	add    %eax,%eax
77ed8bcd:	01 db                	add    %ebx,%ebx
77ed8bcf:	8b 4d 14             	mov    0x14(%ebp),%ecx
77ed8bd2:	89 45 e0             	mov    %eax,0xffffffe0(%ebp)
77ed8bd5:	8b 45 14             	mov    0x14(%ebp),%eax
77ed8bd8:	29 cb                	sub    %ecx,%ebx
77ed8bda:	85 c0                	test   %eax,%eax
77ed8bdc:	78 d2                	js     77ed8bb0 <_LineDDA@24+0xa0>
77ed8bde:	8b 75 14             	mov    0x14(%ebp),%esi
77ed8be1:	46                   	inc    %esi
77ed8be2:	eb 18                	jmp    77ed8bfc <_LineDDA@24+0xec>
77ed8be4:	8b 45 f0             	mov    0xfffffff0(%ebp),%eax
77ed8be7:	8b 4d e0             	mov    0xffffffe0(%ebp),%ecx
77ed8bea:	01 c7                	add    %eax,%edi
77ed8bec:	01 cb                	add    %ecx,%ebx
77ed8bee:	8b 55 0c             	mov    0xc(%ebp),%edx
77ed8bf1:	8b 45 ec             	mov    0xffffffec(%ebp),%eax
77ed8bf4:	01 c2                	add    %eax,%edx
77ed8bf6:	4e                   	dec    %esi
77ed8bf7:	89 55 0c             	mov    %edx,0xc(%ebp)
77ed8bfa:	74 b4                	je     77ed8bb0 <_LineDDA@24+0xa0>
77ed8bfc:	50                   	push   %eax
77ed8bfd:	8b 45 1c             	mov    0x1c(%ebp),%eax
77ed8c00:	50                   	push   %eax
77ed8c01:	8b 45 0c             	mov    0xc(%ebp),%eax
77ed8c04:	50                   	push   %eax
77ed8c05:	57                   	push   %edi
77ed8c06:	ff 55 18             	call   *0x18(%ebp)
77ed8c09:	85 db                	test   %ebx,%ebx
77ed8c0b:	58                   	pop    %eax
77ed8c0c:	7f d6                	jg     77ed8be4 <_LineDDA@24+0xd4>
77ed8c0e:	8b 55 e8             	mov    0xffffffe8(%ebp),%edx
77ed8c11:	8d 1c 53             	lea    (%ebx,%edx,2),%ebx
77ed8c14:	eb d8                	jmp    77ed8bee <_LineDDA@24+0xde>
77ed8c16:	f7 5d 14             	negl   0x14(%ebp)
77ed8c19:	c7 45 ec ff ff ff ff 	movl   $0xffffffff,0xffffffec(%ebp)
77ed8c20:	e9 29 ff ff ff       	jmp    77ed8b4e <_LineDDA@24+0x3e>
77ed8c25:	f7 d8                	neg    %eax
77ed8c27:	89 45 e8             	mov    %eax,0xffffffe8(%ebp)
77ed8c2a:	c7 45 f0 ff ff ff ff 	movl   $0xffffffff,0xfffffff0(%ebp)
77ed8c31:	e9 0d ff ff ff       	jmp    77ed8b43 <_LineDDA@24+0x33>
77ed8c36:	90                   	nop    
77ed8c37:	90                   	nop    
77ed8c38:	90                   	nop    
77ed8c39:	90                   	nop    
77ed8c3a:	90                   	nop    
77ed8c3b:	90                   	nop    
77ed8c3c:	90                   	nop    
77ed8c3d:	90                   	nop    
77ed8c3e:	90                   	nop    
77ed8c3f:	90                   	nop    

77ed8c40 <_GetClipRgn@8>:
77ed8c40:	55                   	push   %ebp
77ed8c41:	89 e5                	mov    %esp,%ebp
77ed8c43:	83 ec 14             	sub    $0x14,%esp
77ed8c46:	8b 55 08             	mov    0x8(%ebp),%edx
77ed8c49:	52                   	push   %edx
77ed8c4a:	e8 eb cd ff ff       	call   77ed5a3a <_NtGdiGetClipRgn@4>
77ed8c4f:	89 c2                	mov    %eax,%edx
77ed8c51:	83 c4 0c             	add    $0xc,%esp
77ed8c54:	31 c0                	xor    %eax,%eax
77ed8c56:	85 d2                	test   %edx,%edx
77ed8c58:	74 16                	je     77ed8c70 <_GetClipRgn@8+0x30>
77ed8c5a:	8b 45 0c             	mov    0xc(%ebp),%eax
77ed8c5d:	6a 05                	push   $0x5
77ed8c5f:	6a 00                	push   $0x0
77ed8c61:	52                   	push   %edx
77ed8c62:	50                   	push   %eax
77ed8c63:	e8 c8 c8 ff ff       	call   77ed5530 <_NtGdiCombineRgn@16>
77ed8c68:	83 f8 01             	cmp    $0x1,%eax
77ed8c6b:	19 c0                	sbb    %eax,%eax
77ed8c6d:	83 c8 01             	or     $0x1,%eax
77ed8c70:	c9                   	leave  
77ed8c71:	c2 08 00             	ret    $0x8
77ed8c74:	90                   	nop    
77ed8c75:	90                   	nop    
77ed8c76:	90                   	nop    
77ed8c77:	90                   	nop    
77ed8c78:	90                   	nop    
77ed8c79:	90                   	nop    
77ed8c7a:	90                   	nop    
77ed8c7b:	90                   	nop    
77ed8c7c:	90                   	nop    
77ed8c7d:	90                   	nop    
77ed8c7e:	90                   	nop    
77ed8c7f:	90                   	nop    

77ed8c80 <_CopyMetaFileW@8>:
77ed8c80:	55                   	push   %ebp
77ed8c81:	89 e5                	mov    %esp,%ebp
77ed8c83:	c9                   	leave  
77ed8c84:	e9 d4 c8 ff ff       	jmp    77ed555d <_NtGdiCopyMetaFile@8>
77ed8c89:	8d b4 26 00 00 00 00 	lea    0x0(%esi),%esi

77ed8c90 <_CopyMetaFileA@8>:
77ed8c90:	55                   	push   %ebp
77ed8c91:	89 e5                	mov    %esp,%ebp
77ed8c93:	53                   	push   %ebx
77ed8c94:	83 ec 0c             	sub    $0xc,%esp
77ed8c97:	31 db                	xor    %ebx,%ebx
77ed8c99:	8b 45 0c             	mov    0xc(%ebp),%eax
77ed8c9c:	50                   	push   %eax
77ed8c9d:	8d 45 f8             	lea    0xfffffff8(%ebp),%eax
77ed8ca0:	50                   	push   %eax
77ed8ca1:	e8 2a 84 ff ff       	call   77ed10d0 <_HEAP_strdupA2W>
77ed8ca6:	83 c4 10             	add    $0x10,%esp
77ed8ca9:	85 c0                	test   %eax,%eax
77ed8cab:	78 27                	js     77ed8cd4 <_CopyMetaFileA@8+0x44>
77ed8cad:	50                   	push   %eax
77ed8cae:	50                   	push   %eax
77ed8caf:	8b 5d f8             	mov    0xfffffff8(%ebp),%ebx
77ed8cb2:	53                   	push   %ebx
77ed8cb3:	8b 4d 08             	mov    0x8(%ebp),%ecx
77ed8cb6:	51                   	push   %ecx
77ed8cb7:	e8 a1 c8 ff ff       	call   77ed555d <_NtGdiCopyMetaFile@8>
77ed8cbc:	89 c3                	mov    %eax,%ebx
77ed8cbe:	52                   	push   %edx
77ed8cbf:	8b 45 f8             	mov    0xfffffff8(%ebp),%eax
77ed8cc2:	50                   	push   %eax
77ed8cc3:	e8 78 84 ff ff       	call   77ed1140 <_HEAP_free>
77ed8cc8:	89 d8                	mov    %ebx,%eax
77ed8cca:	83 c4 10             	add    $0x10,%esp
77ed8ccd:	8b 5d fc             	mov    0xfffffffc(%ebp),%ebx
77ed8cd0:	c9                   	leave  
77ed8cd1:	c2 08 00             	ret    $0x8
77ed8cd4:	83 ec 0c             	sub    $0xc,%esp
77ed8cd7:	50                   	push   %eax
77ed8cd8:	e8 b3 0b 00 00       	call   77ed9890 <_RtlNtStatusToDosError@4>
77ed8cdd:	50                   	push   %eax
77ed8cde:	e8 2d 0c 00 00       	call   77ed9910 <_SetLastError@4>
77ed8ce3:	89 d8                	mov    %ebx,%eax
77ed8ce5:	83 c4 0c             	add    $0xc,%esp
77ed8ce8:	8b 5d fc             	mov    0xfffffffc(%ebp),%ebx
77ed8ceb:	c9                   	leave  
77ed8cec:	c2 08 00             	ret    $0x8
77ed8cef:	90                   	nop    

77ed8cf0 <_CreateMetaFileW@4>:
77ed8cf0:	55                   	push   %ebp
77ed8cf1:	89 e5                	mov    %esp,%ebp
77ed8cf3:	c9                   	leave  
77ed8cf4:	e9 9f c9 ff ff       	jmp    77ed5698 <_NtGdiCreateMetaFile@4>
77ed8cf9:	8d b4 26 00 00 00 00 	lea    0x0(%esi),%esi

77ed8d00 <_CreateMetaFileA@4>:
77ed8d00:	55                   	push   %ebp
77ed8d01:	89 e5                	mov    %esp,%ebp
77ed8d03:	53                   	push   %ebx
77ed8d04:	83 ec 0c             	sub    $0xc,%esp
77ed8d07:	31 db                	xor    %ebx,%ebx
77ed8d09:	8b 45 08             	mov    0x8(%ebp),%eax
77ed8d0c:	50                   	push   %eax
77ed8d0d:	8d 45 f8             	lea    0xfffffff8(%ebp),%eax
77ed8d10:	50                   	push   %eax
77ed8d11:	e8 ba 83 ff ff       	call   77ed10d0 <_HEAP_strdupA2W>
77ed8d16:	83 c4 10             	add    $0x10,%esp
77ed8d19:	85 c0                	test   %eax,%eax
77ed8d1b:	78 23                	js     77ed8d40 <_CreateMetaFileA@4+0x40>
77ed8d1d:	83 ec 0c             	sub    $0xc,%esp
77ed8d20:	8b 45 f8             	mov    0xfffffff8(%ebp),%eax
77ed8d23:	50                   	push   %eax
77ed8d24:	e8 6f c9 ff ff       	call   77ed5698 <_NtGdiCreateMetaFile@4>
77ed8d29:	89 c3                	mov    %eax,%ebx
77ed8d2b:	8b 45 f8             	mov    0xfffffff8(%ebp),%eax
77ed8d2e:	50                   	push   %eax
77ed8d2f:	e8 0c 84 ff ff       	call   77ed1140 <_HEAP_free>
77ed8d34:	89 d8                	mov    %ebx,%eax
77ed8d36:	83 c4 10             	add    $0x10,%esp
77ed8d39:	8b 5d fc             	mov    0xfffffffc(%ebp),%ebx
77ed8d3c:	c9                   	leave  
77ed8d3d:	c2 04 00             	ret    $0x4
77ed8d40:	83 ec 0c             	sub    $0xc,%esp
77ed8d43:	50                   	push   %eax
77ed8d44:	e8 47 0b 00 00       	call   77ed9890 <_RtlNtStatusToDosError@4>
77ed8d49:	50                   	push   %eax
77ed8d4a:	e8 c1 0b 00 00       	call   77ed9910 <_SetLastError@4>
77ed8d4f:	89 d8                	mov    %ebx,%eax
77ed8d51:	83 c4 0c             	add    $0xc,%esp
77ed8d54:	8b 5d fc             	mov    0xfffffffc(%ebp),%ebx
77ed8d57:	c9                   	leave  
77ed8d58:	c2 04 00             	ret    $0x4
77ed8d5b:	90                   	nop    
77ed8d5c:	8d 74 26 00          	lea    0x0(%esi),%esi

77ed8d60 <_GetMetaFileW@4>:
77ed8d60:	55                   	push   %ebp
77ed8d61:	89 e5                	mov    %esp,%ebp
77ed8d63:	c9                   	leave  
77ed8d64:	e9 48 ce ff ff       	jmp    77ed5bb1 <_NtGdiGetMetaFile@4>
77ed8d69:	8d b4 26 00 00 00 00 	lea    0x0(%esi),%esi

77ed8d70 <_GetMetaFileA@4>:
77ed8d70:	55                   	push   %ebp
77ed8d71:	89 e5                	mov    %esp,%ebp
77ed8d73:	53                   	push   %ebx
77ed8d74:	83 ec 0c             	sub    $0xc,%esp
77ed8d77:	31 db                	xor    %ebx,%ebx
77ed8d79:	8b 4d 08             	mov    0x8(%ebp),%ecx
77ed8d7c:	8d 45 f8             	lea    0xfffffff8(%ebp),%eax
77ed8d7f:	51                   	push   %ecx
77ed8d80:	50                   	push   %eax
77ed8d81:	e8 4a 83 ff ff       	call   77ed10d0 <_HEAP_strdupA2W>
77ed8d86:	83 c4 10             	add    $0x10,%esp
77ed8d89:	85 c0                	test   %eax,%eax
77ed8d8b:	78 23                	js     77ed8db0 <_GetMetaFileA@4+0x40>
77ed8d8d:	83 ec 0c             	sub    $0xc,%esp
77ed8d90:	8b 55 f8             	mov    0xfffffff8(%ebp),%edx
77ed8d93:	52                   	push   %edx
77ed8d94:	e8 18 ce ff ff       	call   77ed5bb1 <_NtGdiGetMetaFile@4>
77ed8d99:	89 c3                	mov    %eax,%ebx
77ed8d9b:	8b 45 f8             	mov    0xfffffff8(%ebp),%eax
77ed8d9e:	50                   	push   %eax
77ed8d9f:	e8 9c 83 ff ff       	call   77ed1140 <_HEAP_free>
77ed8da4:	89 d8                	mov    %ebx,%eax
77ed8da6:	83 c4 10             	add    $0x10,%esp
77ed8da9:	8b 5d fc             	mov    0xfffffffc(%ebp),%ebx
77ed8dac:	c9                   	leave  
77ed8dad:	c2 04 00             	ret    $0x4
77ed8db0:	83 ec 0c             	sub    $0xc,%esp
77ed8db3:	50                   	push   %eax
77ed8db4:	e8 d7 0a 00 00       	call   77ed9890 <_RtlNtStatusToDosError@4>
77ed8db9:	50                   	push   %eax
77ed8dba:	e8 51 0b 00 00       	call   77ed9910 <_SetLastError@4>
77ed8dbf:	89 d8                	mov    %ebx,%eax
77ed8dc1:	83 c4 0c             	add    $0xc,%esp
77ed8dc4:	8b 5d fc             	mov    0xfffffffc(%ebp),%ebx
77ed8dc7:	c9                   	leave  
77ed8dc8:	c2 04 00             	ret    $0x4
77ed8dcb:	90                   	nop    
77ed8dcc:	8d 74 26 00          	lea    0x0(%esi),%esi

77ed8dd0 <_CopyEnhMetaFileW@8>:
77ed8dd0:	55                   	push   %ebp
77ed8dd1:	89 e5                	mov    %esp,%ebp
77ed8dd3:	c9                   	leave  
77ed8dd4:	e9 75 c7 ff ff       	jmp    77ed554e <_NtGdiCopyEnhMetaFile@8>
77ed8dd9:	8d b4 26 00 00 00 00 	lea    0x0(%esi),%esi

77ed8de0 <_CopyEnhMetaFileA@8>:
77ed8de0:	55                   	push   %ebp
77ed8de1:	89 e5                	mov    %esp,%ebp
77ed8de3:	53                   	push   %ebx
77ed8de4:	83 ec 0c             	sub    $0xc,%esp
77ed8de7:	31 db                	xor    %ebx,%ebx
77ed8de9:	8b 45 0c             	mov    0xc(%ebp),%eax
77ed8dec:	50                   	push   %eax
77ed8ded:	8d 45 f8             	lea    0xfffffff8(%ebp),%eax
77ed8df0:	50                   	push   %eax
77ed8df1:	e8 da 82 ff ff       	call   77ed10d0 <_HEAP_strdupA2W>
77ed8df6:	83 c4 10             	add    $0x10,%esp
77ed8df9:	85 c0                	test   %eax,%eax
77ed8dfb:	78 27                	js     77ed8e24 <_CopyEnhMetaFileA@8+0x44>
77ed8dfd:	50                   	push   %eax
77ed8dfe:	50                   	push   %eax
77ed8dff:	8b 45 f8             	mov    0xfffffff8(%ebp),%eax
77ed8e02:	50                   	push   %eax
77ed8e03:	8b 45 08             	mov    0x8(%ebp),%eax
77ed8e06:	50                   	push   %eax
77ed8e07:	e8 42 c7 ff ff       	call   77ed554e <_NtGdiCopyEnhMetaFile@8>
77ed8e0c:	89 c3                	mov    %eax,%ebx
77ed8e0e:	50                   	push   %eax
77ed8e0f:	8b 45 f8             	mov    0xfffffff8(%ebp),%eax
77ed8e12:	50                   	push   %eax
77ed8e13:	e8 28 83 ff ff       	call   77ed1140 <_HEAP_free>
77ed8e18:	89 d8                	mov    %ebx,%eax
77ed8e1a:	83 c4 10             	add    $0x10,%esp
77ed8e1d:	8b 5d fc             	mov    0xfffffffc(%ebp),%ebx
77ed8e20:	c9                   	leave  
77ed8e21:	c2 08 00             	ret    $0x8
77ed8e24:	83 ec 0c             	sub    $0xc,%esp
77ed8e27:	50                   	push   %eax
77ed8e28:	e8 63 0a 00 00       	call   77ed9890 <_RtlNtStatusToDosError@4>
77ed8e2d:	50                   	push   %eax
77ed8e2e:	e8 dd 0a 00 00       	call   77ed9910 <_SetLastError@4>
77ed8e33:	89 d8                	mov    %ebx,%eax
77ed8e35:	83 c4 0c             	add    $0xc,%esp
77ed8e38:	8b 5d fc             	mov    0xfffffffc(%ebp),%ebx
77ed8e3b:	c9                   	leave  
77ed8e3c:	c2 08 00             	ret    $0x8
77ed8e3f:	90                   	nop    

77ed8e40 <_CreateEnhMetaFileW@16>:
77ed8e40:	55                   	push   %ebp
77ed8e41:	89 e5                	mov    %esp,%ebp
77ed8e43:	c9                   	leave  
77ed8e44:	e9 f5 c7 ff ff       	jmp    77ed563e <_NtGdiCreateEnhMetaFile@16>
77ed8e49:	8d b4 26 00 00 00 00 	lea    0x0(%esi),%esi

77ed8e50 <_CreateEnhMetaFileA@16>:
77ed8e50:	55                   	push   %ebp
77ed8e51:	89 e5                	mov    %esp,%ebp
77ed8e53:	53                   	push   %ebx
77ed8e54:	83 ec 1c             	sub    $0x1c,%esp
77ed8e57:	31 db                	xor    %ebx,%ebx
77ed8e59:	8b 45 0c             	mov    0xc(%ebp),%eax
77ed8e5c:	50                   	push   %eax
77ed8e5d:	8d 45 f8             	lea    0xfffffff8(%ebp),%eax
77ed8e60:	50                   	push   %eax
77ed8e61:	e8 6a 82 ff ff       	call   77ed10d0 <_HEAP_strdupA2W>
77ed8e66:	83 c4 10             	add    $0x10,%esp
77ed8e69:	85 c0                	test   %eax,%eax
77ed8e6b:	78 54                	js     77ed8ec1 <_CreateEnhMetaFileA@16+0x71>
77ed8e6d:	50                   	push   %eax
77ed8e6e:	50                   	push   %eax
77ed8e6f:	8b 45 14             	mov    0x14(%ebp),%eax
77ed8e72:	50                   	push   %eax
77ed8e73:	8d 45 f4             	lea    0xfffffff4(%ebp),%eax
77ed8e76:	50                   	push   %eax
77ed8e77:	e8 54 82 ff ff       	call   77ed10d0 <_HEAP_strdupA2W>
77ed8e7c:	83 c4 10             	add    $0x10,%esp
77ed8e7f:	85 c0                	test   %eax,%eax
77ed8e81:	78 5d                	js     77ed8ee0 <_CreateEnhMetaFileA@16+0x90>
77ed8e83:	8b 45 f4             	mov    0xfffffff4(%ebp),%eax
77ed8e86:	50                   	push   %eax
77ed8e87:	8b 45 10             	mov    0x10(%ebp),%eax
77ed8e8a:	50                   	push   %eax
77ed8e8b:	8b 45 f8             	mov    0xfffffff8(%ebp),%eax
77ed8e8e:	50                   	push   %eax
77ed8e8f:	8b 5d 08             	mov    0x8(%ebp),%ebx
77ed8e92:	53                   	push   %ebx
77ed8e93:	e8 a6 c7 ff ff       	call   77ed563e <_NtGdiCreateEnhMetaFile@16>
77ed8e98:	83 ec 0c             	sub    $0xc,%esp
77ed8e9b:	8b 4d f4             	mov    0xfffffff4(%ebp),%ecx
77ed8e9e:	89 c3                	mov    %eax,%ebx
77ed8ea0:	51                   	push   %ecx
77ed8ea1:	e8 9a 82 ff ff       	call   77ed1140 <_HEAP_free>
77ed8ea6:	83 c4 10             	add    $0x10,%esp
77ed8ea9:	83 ec 0c             	sub    $0xc,%esp
77ed8eac:	8b 55 f8             	mov    0xfffffff8(%ebp),%edx
77ed8eaf:	52                   	push   %edx
77ed8eb0:	e8 8b 82 ff ff       	call   77ed1140 <_HEAP_free>
77ed8eb5:	89 d8                	mov    %ebx,%eax
77ed8eb7:	83 c4 10             	add    $0x10,%esp
77ed8eba:	8b 5d fc             	mov    0xfffffffc(%ebp),%ebx
77ed8ebd:	c9                   	leave  
77ed8ebe:	c2 10 00             	ret    $0x10
77ed8ec1:	83 ec 0c             	sub    $0xc,%esp
77ed8ec4:	50                   	push   %eax
77ed8ec5:	e8 c6 09 00 00       	call   77ed9890 <_RtlNtStatusToDosError@4>
77ed8eca:	50                   	push   %eax
77ed8ecb:	e8 40 0a 00 00       	call   77ed9910 <_SetLastError@4>
77ed8ed0:	89 d8                	mov    %ebx,%eax
77ed8ed2:	83 c4 0c             	add    $0xc,%esp
77ed8ed5:	8b 5d fc             	mov    0xfffffffc(%ebp),%ebx
77ed8ed8:	c9                   	leave  
77ed8ed9:	c2 10 00             	ret    $0x10
77ed8edc:	8d 74 26 00          	lea    0x0(%esi),%esi
77ed8ee0:	83 ec 0c             	sub    $0xc,%esp
77ed8ee3:	50                   	push   %eax
77ed8ee4:	e8 a7 09 00 00       	call   77ed9890 <_RtlNtStatusToDosError@4>
77ed8ee9:	50                   	push   %eax
77ed8eea:	e8 21 0a 00 00       	call   77ed9910 <_SetLastError@4>
77ed8eef:	83 c4 0c             	add    $0xc,%esp
77ed8ef2:	eb b5                	jmp    77ed8ea9 <_CreateEnhMetaFileA@16+0x59>
77ed8ef4:	8d b6 00 00 00 00    	lea    0x0(%esi),%esi
77ed8efa:	8d bf 00 00 00 00    	lea    0x0(%edi),%edi

77ed8f00 <_GetEnhMetaFileW@4>:
77ed8f00:	55                   	push   %ebp
77ed8f01:	89 e5                	mov    %esp,%ebp
77ed8f03:	c9                   	leave  
77ed8f04:	e9 c7 cb ff ff       	jmp    77ed5ad0 <_NtGdiGetEnhMetaFile@4>
77ed8f09:	8d b4 26 00 00 00 00 	lea    0x0(%esi),%esi

77ed8f10 <_GetEnhMetaFileA@4>:
77ed8f10:	55                   	push   %ebp
77ed8f11:	89 e5                	mov    %esp,%ebp
77ed8f13:	53                   	push   %ebx
77ed8f14:	83 ec 0c             	sub    $0xc,%esp
77ed8f17:	31 db                	xor    %ebx,%ebx
77ed8f19:	8b 45 08             	mov    0x8(%ebp),%eax
77ed8f1c:	50                   	push   %eax
77ed8f1d:	8d 45 f8             	lea    0xfffffff8(%ebp),%eax
77ed8f20:	50                   	push   %eax
77ed8f21:	e8 aa 81 ff ff       	call   77ed10d0 <_HEAP_strdupA2W>
77ed8f26:	83 c4 10             	add    $0x10,%esp
77ed8f29:	85 c0                	test   %eax,%eax
77ed8f2b:	78 23                	js     77ed8f50 <_GetEnhMetaFileA@4+0x40>
77ed8f2d:	83 ec 0c             	sub    $0xc,%esp
77ed8f30:	8b 4d f8             	mov    0xfffffff8(%ebp),%ecx
77ed8f33:	51                   	push   %ecx
77ed8f34:	e8 97 cb ff ff       	call   77ed5ad0 <_NtGdiGetEnhMetaFile@4>
77ed8f39:	8b 55 f8             	mov    0xfffffff8(%ebp),%edx
77ed8f3c:	89 c3                	mov    %eax,%ebx
77ed8f3e:	52                   	push   %edx
77ed8f3f:	e8 fc 81 ff ff       	call   77ed1140 <_HEAP_free>
77ed8f44:	89 d8                	mov    %ebx,%eax
77ed8f46:	83 c4 10             	add    $0x10,%esp
77ed8f49:	8b 5d fc             	mov    0xfffffffc(%ebp),%ebx
77ed8f4c:	c9                   	leave  
77ed8f4d:	c2 04 00             	ret    $0x4
77ed8f50:	83 ec 0c             	sub    $0xc,%esp
77ed8f53:	50                   	push   %eax
77ed8f54:	e8 37 09 00 00       	call   77ed9890 <_RtlNtStatusToDosError@4>
77ed8f59:	50                   	push   %eax
77ed8f5a:	e8 b1 09 00 00       	call   77ed9910 <_SetLastError@4>
77ed8f5f:	89 d8                	mov    %ebx,%eax
77ed8f61:	83 c4 0c             	add    $0xc,%esp
77ed8f64:	8b 5d fc             	mov    0xfffffffc(%ebp),%ebx
77ed8f67:	c9                   	leave  
77ed8f68:	c2 04 00             	ret    $0x4
77ed8f6b:	90                   	nop    
77ed8f6c:	8d 74 26 00          	lea    0x0(%esi),%esi

77ed8f70 <_GetEnhMetaFileDescriptionW@12>:
77ed8f70:	55                   	push   %ebp
77ed8f71:	89 e5                	mov    %esp,%ebp
77ed8f73:	c9                   	leave  
77ed8f74:	e9 75 cb ff ff       	jmp    77ed5aee <_NtGdiGetEnhMetaFileDescription@12>
77ed8f79:	8d b4 26 00 00 00 00 	lea    0x0(%esi),%esi

77ed8f80 <_GetEnhMetaFileDescriptionA@12>:
77ed8f80:	55                   	push   %ebp
77ed8f81:	89 e5                	mov    %esp,%ebp
77ed8f83:	57                   	push   %edi
77ed8f84:	56                   	push   %esi
77ed8f85:	53                   	push   %ebx
77ed8f86:	83 ec 0c             	sub    $0xc,%esp
77ed8f89:	8b 5d 0c             	mov    0xc(%ebp),%ebx
77ed8f8c:	8b 7d 10             	mov    0x10(%ebp),%edi
77ed8f8f:	85 ff                	test   %edi,%edi
77ed8f91:	0f 95 c2             	setne  %dl
77ed8f94:	85 db                	test   %ebx,%ebx
77ed8f96:	0f 95 c0             	setne  %al
77ed8f99:	25 ff 00 00 00       	and    $0xff,%eax
77ed8f9e:	31 f6                	xor    %esi,%esi
77ed8fa0:	85 c2                	test   %eax,%edx
77ed8fa2:	75 60                	jne    77ed9004 <_GetEnhMetaFileDescriptionA@12+0x84>
77ed8fa4:	50                   	push   %eax
77ed8fa5:	8b 45 08             	mov    0x8(%ebp),%eax
77ed8fa8:	56                   	push   %esi
77ed8fa9:	53                   	push   %ebx
77ed8faa:	50                   	push   %eax
77ed8fab:	e8 3e cb ff ff       	call   77ed5aee <_NtGdiGetEnhMetaFileDescription@12>
77ed8fb0:	85 ff                	test   %edi,%edi
77ed8fb2:	0f 95 c2             	setne  %dl
77ed8fb5:	89 45 f0             	mov    %eax,0xfffffff0(%ebp)
77ed8fb8:	85 db                	test   %ebx,%ebx
77ed8fba:	58                   	pop    %eax
77ed8fbb:	0f 95 c0             	setne  %al
77ed8fbe:	25 ff 00 00 00       	and    $0xff,%eax
77ed8fc3:	85 c2                	test   %eax,%edx
77ed8fc5:	75 0d                	jne    77ed8fd4 <_GetEnhMetaFileDescriptionA@12+0x54>
77ed8fc7:	8b 45 f0             	mov    0xfffffff0(%ebp),%eax
77ed8fca:	8d 65 f4             	lea    0xfffffff4(%ebp),%esp
77ed8fcd:	5b                   	pop    %ebx
77ed8fce:	5e                   	pop    %esi
77ed8fcf:	5f                   	pop    %edi
77ed8fd0:	5d                   	pop    %ebp
77ed8fd1:	c2 0c 00             	ret    $0xc
77ed8fd4:	83 ec 0c             	sub    $0xc,%esp
77ed8fd7:	53                   	push   %ebx
77ed8fd8:	56                   	push   %esi
77ed8fd9:	6a 00                	push   $0x0
77ed8fdb:	53                   	push   %ebx
77ed8fdc:	57                   	push   %edi
77ed8fdd:	e8 ee 08 00 00       	call   77ed98d0 <_RtlUnicodeToMultiByteN@20>
77ed8fe2:	89 c3                	mov    %eax,%ebx
77ed8fe4:	56                   	push   %esi
77ed8fe5:	e8 56 81 ff ff       	call   77ed1140 <_HEAP_free>
77ed8fea:	83 c4 10             	add    $0x10,%esp
77ed8fed:	85 db                	test   %ebx,%ebx
77ed8fef:	79 d6                	jns    77ed8fc7 <_GetEnhMetaFileDescriptionA@12+0x47>
77ed8ff1:	83 ec 0c             	sub    $0xc,%esp
77ed8ff4:	53                   	push   %ebx
77ed8ff5:	e8 96 08 00 00       	call   77ed9890 <_RtlNtStatusToDosError@4>
77ed8ffa:	50                   	push   %eax
77ed8ffb:	e8 10 09 00 00       	call   77ed9910 <_SetLastError@4>
77ed9000:	31 c0                	xor    %eax,%eax
77ed9002:	eb c6                	jmp    77ed8fca <_GetEnhMetaFileDescriptionA@12+0x4a>
77ed9004:	83 ec 0c             	sub    $0xc,%esp
77ed9007:	8d 04 1b             	lea    (%ebx,%ebx,1),%eax
77ed900a:	50                   	push   %eax
77ed900b:	e8 70 80 ff ff       	call   77ed1080 <_HEAP_alloc>
77ed9010:	83 c4 10             	add    $0x10,%esp
77ed9013:	89 c6                	mov    %eax,%esi
77ed9015:	85 c0                	test   %eax,%eax
77ed9017:	75 8b                	jne    77ed8fa4 <_GetEnhMetaFileDescriptionA@12+0x24>
77ed9019:	83 ec 0c             	sub    $0xc,%esp
77ed901c:	68 17 00 00 c0       	push   $0xc0000017
77ed9021:	eb d2                	jmp    77ed8ff5 <_GetEnhMetaFileDescriptionA@12+0x75>
77ed9023:	90                   	nop    
77ed9024:	90                   	nop    
77ed9025:	90                   	nop    
77ed9026:	90                   	nop    
77ed9027:	90                   	nop    
77ed9028:	90                   	nop    
77ed9029:	90                   	nop    
77ed902a:	90                   	nop    
77ed902b:	90                   	nop    
77ed902c:	90                   	nop    
77ed902d:	90                   	nop    
77ed902e:	90                   	nop    
77ed902f:	90                   	nop    

77ed9030 <_TextOutW@20>:
77ed9030:	55                   	push   %ebp
77ed9031:	89 e5                	mov    %esp,%ebp
77ed9033:	c9                   	leave  
77ed9034:	e9 52 d3 ff ff       	jmp    77ed638b <_NtGdiTextOut@20>
77ed9039:	8d b4 26 00 00 00 00 	lea    0x0(%esi),%esi

77ed9040 <_TextOutA@20>:
77ed9040:	55                   	push   %ebp
77ed9041:	89 e5                	mov    %esp,%ebp
77ed9043:	56                   	push   %esi
77ed9044:	53                   	push   %ebx
77ed9045:	83 ec 10             	sub    $0x10,%esp
77ed9048:	8b 45 14             	mov    0x14(%ebp),%eax
77ed904b:	85 c0                	test   %eax,%eax
77ed904d:	74 51                	je     77ed90a0 <_TextOutA@20+0x60>
77ed904f:	8d 5d f0             	lea    0xfffffff0(%ebp),%ebx
77ed9052:	52                   	push   %edx
77ed9053:	52                   	push   %edx
77ed9054:	50                   	push   %eax
77ed9055:	53                   	push   %ebx
77ed9056:	e8 05 08 00 00       	call   77ed9860 <_RtlInitAnsiString@8>
77ed905b:	8d 75 e8             	lea    0xffffffe8(%ebp),%esi
77ed905e:	c7 04 24 01 00 00 00 	movl   $0x1,(%esp)
77ed9065:	53                   	push   %ebx
77ed9066:	56                   	push   %esi
77ed9067:	e8 04 08 00 00       	call   77ed9870 <_RtlAnsiStringToUnicodeString@12>
77ed906c:	58                   	pop    %eax
77ed906d:	83 ec 0c             	sub    $0xc,%esp
77ed9070:	8b 45 18             	mov    0x18(%ebp),%eax
77ed9073:	8b 4d 10             	mov    0x10(%ebp),%ecx
77ed9076:	8b 55 0c             	mov    0xc(%ebp),%edx
77ed9079:	50                   	push   %eax
77ed907a:	8b 45 08             	mov    0x8(%ebp),%eax
77ed907d:	8b 5e 04             	mov    0x4(%esi),%ebx
77ed9080:	53                   	push   %ebx
77ed9081:	51                   	push   %ecx
77ed9082:	52                   	push   %edx
77ed9083:	50                   	push   %eax
77ed9084:	e8 a7 ff ff ff       	call   77ed9030 <_TextOutW@20>
77ed9089:	89 c3                	mov    %eax,%ebx
77ed908b:	56                   	push   %esi
77ed908c:	e8 ef 07 00 00       	call   77ed9880 <_RtlFreeUnicodeString@4>
77ed9091:	8d 65 f8             	lea    0xfffffff8(%ebp),%esp
77ed9094:	89 d8                	mov    %ebx,%eax
77ed9096:	5b                   	pop    %ebx
77ed9097:	5e                   	pop    %esi
77ed9098:	5d                   	pop    %ebp
77ed9099:	c2 14 00             	ret    $0x14
77ed909c:	8d 74 26 00          	lea    0x0(%esi),%esi
77ed90a0:	8d 75 e8             	lea    0xffffffe8(%ebp),%esi
77ed90a3:	c7 45 ec 00 00 00 00 	movl   $0x0,0xffffffec(%ebp)
77ed90aa:	eb c1                	jmp    77ed906d <_TextOutA@20+0x2d>
77ed90ac:	8d 74 26 00          	lea    0x0(%esi),%esi

77ed90b0 <_GetTextMetricsA@8>:
77ed90b0:	55                   	push   %ebp
77ed90b1:	89 e5                	mov    %esp,%ebp
77ed90b3:	53                   	push   %ebx
77ed90b4:	83 ec 4c             	sub    $0x4c,%esp
77ed90b7:	8d 5d b8             	lea    0xffffffb8(%ebp),%ebx
77ed90ba:	53                   	push   %ebx
77ed90bb:	8b 4d 08             	mov    0x8(%ebp),%ecx
77ed90be:	51                   	push   %ecx
77ed90bf:	e8 be cc ff ff       	call   77ed5d82 <_NtGdiGetTextMetrics@8>
77ed90c4:	59                   	pop    %ecx
77ed90c5:	5a                   	pop    %edx
77ed90c6:	31 d2                	xor    %edx,%edx
77ed90c8:	85 c0                	test   %eax,%eax
77ed90ca:	75 09                	jne    77ed90d5 <_GetTextMetricsA@8+0x25>
77ed90cc:	89 d0                	mov    %edx,%eax
77ed90ce:	8b 5d fc             	mov    0xfffffffc(%ebp),%ebx
77ed90d1:	c9                   	leave  
77ed90d2:	c2 08 00             	ret    $0x8
77ed90d5:	89 da                	mov    %ebx,%edx
77ed90d7:	8b 4d 0c             	mov    0xc(%ebp),%ecx
77ed90da:	e8 c1 ef ff ff       	call   77ed80a0 <@TextMetricW2A@8>
77ed90df:	8b 5d fc             	mov    0xfffffffc(%ebp),%ebx
77ed90e2:	89 c2                	mov    %eax,%edx
77ed90e4:	c9                   	leave  
77ed90e5:	89 d0                	mov    %edx,%eax
77ed90e7:	c2 08 00             	ret    $0x8
77ed90ea:	8d b6 00 00 00 00    	lea    0x0(%esi),%esi

77ed90f0 <_GetTextMetricsW@8>:
77ed90f0:	55                   	push   %ebp
77ed90f1:	89 e5                	mov    %esp,%ebp
77ed90f3:	c9                   	leave  
77ed90f4:	e9 89 cc ff ff       	jmp    77ed5d82 <_NtGdiGetTextMetrics@8>
77ed90f9:	8d b4 26 00 00 00 00 	lea    0x0(%esi),%esi

77ed9100 <_GetTextExtentPointW@16>:
77ed9100:	55                   	push   %ebp
77ed9101:	89 e5                	mov    %esp,%ebp
77ed9103:	c9                   	leave  
77ed9104:	e9 4c cc ff ff       	jmp    77ed5d55 <_NtGdiGetTextExtentPoint@16>
77ed9109:	8d b4 26 00 00 00 00 	lea    0x0(%esi),%esi

77ed9110 <_GetTextExtentPointA@16>:
77ed9110:	55                   	push   %ebp
77ed9111:	89 e5                	mov    %esp,%ebp
77ed9113:	56                   	push   %esi
77ed9114:	53                   	push   %ebx
77ed9115:	83 ec 18             	sub    $0x18,%esp
77ed9118:	8d 5d f0             	lea    0xfffffff0(%ebp),%ebx
77ed911b:	8b 45 0c             	mov    0xc(%ebp),%eax
77ed911e:	8d 75 e8             	lea    0xffffffe8(%ebp),%esi
77ed9121:	50                   	push   %eax
77ed9122:	53                   	push   %ebx
77ed9123:	e8 38 07 00 00       	call   77ed9860 <_RtlInitAnsiString@8>
77ed9128:	c7 04 24 01 00 00 00 	movl   $0x1,(%esp)
77ed912f:	53                   	push   %ebx
77ed9130:	56                   	push   %esi
77ed9131:	e8 3a 07 00 00       	call   77ed9870 <_RtlAnsiStringToUnicodeString@12>
77ed9136:	58                   	pop    %eax
77ed9137:	8b 45 14             	mov    0x14(%ebp),%eax
77ed913a:	50                   	push   %eax
77ed913b:	8b 45 10             	mov    0x10(%ebp),%eax
77ed913e:	50                   	push   %eax
77ed913f:	8b 5d 08             	mov    0x8(%ebp),%ebx
77ed9142:	8b 45 ec             	mov    0xffffffec(%ebp),%eax
77ed9145:	50                   	push   %eax
77ed9146:	53                   	push   %ebx
77ed9147:	e8 b4 ff ff ff       	call   77ed9100 <_GetTextExtentPointW@16>
77ed914c:	83 ec 0c             	sub    $0xc,%esp
77ed914f:	89 c3                	mov    %eax,%ebx
77ed9151:	56                   	push   %esi
77ed9152:	e8 29 07 00 00       	call   77ed9880 <_RtlFreeUnicodeString@4>
77ed9157:	8d 65 f8             	lea    0xfffffff8(%ebp),%esp
77ed915a:	89 d8                	mov    %ebx,%eax
77ed915c:	5b                   	pop    %ebx
77ed915d:	5e                   	pop    %esi
77ed915e:	5d                   	pop    %ebp
77ed915f:	c2 10 00             	ret    $0x10
77ed9162:	8d b4 26 00 00 00 00 	lea    0x0(%esi),%esi
77ed9169:	8d bc 27 00 00 00 00 	lea    0x0(%edi),%edi

77ed9170 <_GetTextExtentExPointW@28>:
77ed9170:	55                   	push   %ebp
77ed9171:	89 e5                	mov    %esp,%ebp
77ed9173:	c9                   	leave  
77ed9174:	e9 cd cb ff ff       	jmp    77ed5d46 <_NtGdiGetTextExtentExPoint@28>
77ed9179:	8d b4 26 00 00 00 00 	lea    0x0(%esi),%esi

77ed9180 <_GetTextExtentExPointA@28>:
77ed9180:	55                   	push   %ebp
77ed9181:	89 e5                	mov    %esp,%ebp
77ed9183:	53                   	push   %ebx
77ed9184:	83 ec 0c             	sub    $0xc,%esp
77ed9187:	31 db                	xor    %ebx,%ebx
77ed9189:	8b 55 0c             	mov    0xc(%ebp),%edx
77ed918c:	8d 45 f8             	lea    0xfffffff8(%ebp),%eax
77ed918f:	52                   	push   %edx
77ed9190:	50                   	push   %eax
77ed9191:	e8 3a 7f ff ff       	call   77ed10d0 <_HEAP_strdupA2W>
77ed9196:	83 c4 10             	add    $0x10,%esp
77ed9199:	85 c0                	test   %eax,%eax
77ed919b:	78 3b                	js     77ed91d8 <_GetTextExtentExPointA@28+0x58>
77ed919d:	50                   	push   %eax
77ed919e:	8b 45 20             	mov    0x20(%ebp),%eax
77ed91a1:	50                   	push   %eax
77ed91a2:	8b 45 1c             	mov    0x1c(%ebp),%eax
77ed91a5:	50                   	push   %eax
77ed91a6:	8b 45 18             	mov    0x18(%ebp),%eax
77ed91a9:	50                   	push   %eax
77ed91aa:	8b 45 14             	mov    0x14(%ebp),%eax
77ed91ad:	50                   	push   %eax
77ed91ae:	8b 45 10             	mov    0x10(%ebp),%eax
77ed91b1:	50                   	push   %eax
77ed91b2:	8b 5d f8             	mov    0xfffffff8(%ebp),%ebx
77ed91b5:	53                   	push   %ebx
77ed91b6:	8b 4d 08             	mov    0x8(%ebp),%ecx
77ed91b9:	51                   	push   %ecx
77ed91ba:	e8 87 cb ff ff       	call   77ed5d46 <_NtGdiGetTextExtentExPoint@28>
77ed91bf:	89 c3                	mov    %eax,%ebx
77ed91c1:	52                   	push   %edx
77ed91c2:	52                   	push   %edx
77ed91c3:	8b 45 f8             	mov    0xfffffff8(%ebp),%eax
77ed91c6:	50                   	push   %eax
77ed91c7:	e8 74 7f ff ff       	call   77ed1140 <_HEAP_free>
77ed91cc:	89 d8                	mov    %ebx,%eax
77ed91ce:	83 c4 10             	add    $0x10,%esp
77ed91d1:	8b 5d fc             	mov    0xfffffffc(%ebp),%ebx
77ed91d4:	c9                   	leave  
77ed91d5:	c2 1c 00             	ret    $0x1c
77ed91d8:	83 ec 0c             	sub    $0xc,%esp
77ed91db:	50                   	push   %eax
77ed91dc:	e8 af 06 00 00       	call   77ed9890 <_RtlNtStatusToDosError@4>
77ed91e1:	50                   	push   %eax
77ed91e2:	e8 29 07 00 00       	call   77ed9910 <_SetLastError@4>
77ed91e7:	89 d8                	mov    %ebx,%eax
77ed91e9:	83 c4 0c             	add    $0xc,%esp
77ed91ec:	8b 5d fc             	mov    0xfffffffc(%ebp),%ebx
77ed91ef:	c9                   	leave  
77ed91f0:	c2 1c 00             	ret    $0x1c
77ed91f3:	8d b6 00 00 00 00    	lea    0x0(%esi),%esi
77ed91f9:	8d bc 27 00 00 00 00 	lea    0x0(%edi),%edi

77ed9200 <_GetTextExtentPoint32W@16>:
77ed9200:	55                   	push   %ebp
77ed9201:	89 e5                	mov    %esp,%ebp
77ed9203:	c9                   	leave  
77ed9204:	e9 5b cb ff ff       	jmp    77ed5d64 <_NtGdiGetTextExtentPoint32@16>
77ed9209:	8d b4 26 00 00 00 00 	lea    0x0(%esi),%esi

77ed9210 <_GetTextExtentPoint32A@16>:
77ed9210:	55                   	push   %ebp
77ed9211:	89 e5                	mov    %esp,%ebp
77ed9213:	56                   	push   %esi
77ed9214:	53                   	push   %ebx
77ed9215:	83 ec 18             	sub    $0x18,%esp
77ed9218:	8d 5d f0             	lea    0xfffffff0(%ebp),%ebx
77ed921b:	8b 45 0c             	mov    0xc(%ebp),%eax
77ed921e:	8d 75 e8             	lea    0xffffffe8(%ebp),%esi
77ed9221:	50                   	push   %eax
77ed9222:	53                   	push   %ebx
77ed9223:	e8 38 06 00 00       	call   77ed9860 <_RtlInitAnsiString@8>
77ed9228:	c7 04 24 01 00 00 00 	movl   $0x1,(%esp)
77ed922f:	53                   	push   %ebx
77ed9230:	56                   	push   %esi
77ed9231:	e8 3a 06 00 00       	call   77ed9870 <_RtlAnsiStringToUnicodeString@12>
77ed9236:	58                   	pop    %eax
77ed9237:	8b 45 14             	mov    0x14(%ebp),%eax
77ed923a:	50                   	push   %eax
77ed923b:	8b 5d ec             	mov    0xffffffec(%ebp),%ebx
77ed923e:	8b 4d 08             	mov    0x8(%ebp),%ecx
77ed9241:	8b 45 10             	mov    0x10(%ebp),%eax
77ed9244:	50                   	push   %eax
77ed9245:	53                   	push   %ebx
77ed9246:	51                   	push   %ecx
77ed9247:	e8 b4 ff ff ff       	call   77ed9200 <_GetTextExtentPoint32W@16>
77ed924c:	83 ec 0c             	sub    $0xc,%esp
77ed924f:	89 c3                	mov    %eax,%ebx
77ed9251:	56                   	push   %esi
77ed9252:	e8 29 06 00 00       	call   77ed9880 <_RtlFreeUnicodeString@4>
77ed9257:	8d 65 f8             	lea    0xfffffff8(%ebp),%esp
77ed925a:	89 d8                	mov    %ebx,%eax
77ed925c:	5b                   	pop    %ebx
77ed925d:	5e                   	pop    %esi
77ed925e:	5d                   	pop    %ebp
77ed925f:	c2 10 00             	ret    $0x10
77ed9262:	8d b4 26 00 00 00 00 	lea    0x0(%esi),%esi
77ed9269:	8d bc 27 00 00 00 00 	lea    0x0(%edi),%edi

77ed9270 <_ExtTextOutW@32>:
77ed9270:	55                   	push   %ebp
77ed9271:	89 e5                	mov    %esp,%ebp
77ed9273:	c9                   	leave  
77ed9274:	e9 4a c6 ff ff       	jmp    77ed58c3 <_NtGdiExtTextOut@32>
77ed9279:	8d b4 26 00 00 00 00 	lea    0x0(%esi),%esi

77ed9280 <_ExtTextOutA@32>:
77ed9280:	55                   	push   %ebp
77ed9281:	89 e5                	mov    %esp,%ebp
77ed9283:	56                   	push   %esi
77ed9284:	53                   	push   %ebx
77ed9285:	83 ec 18             	sub    $0x18,%esp
77ed9288:	8d 5d f0             	lea    0xfffffff0(%ebp),%ebx
77ed928b:	8b 45 1c             	mov    0x1c(%ebp),%eax
77ed928e:	8d 75 e8             	lea    0xffffffe8(%ebp),%esi
77ed9291:	50                   	push   %eax
77ed9292:	53                   	push   %ebx
77ed9293:	e8 c8 05 00 00       	call   77ed9860 <_RtlInitAnsiString@8>
77ed9298:	c7 04 24 01 00 00 00 	movl   $0x1,(%esp)
77ed929f:	53                   	push   %ebx
77ed92a0:	56                   	push   %esi
77ed92a1:	e8 ca 05 00 00       	call   77ed9870 <_RtlAnsiStringToUnicodeString@12>
77ed92a6:	58                   	pop    %eax
77ed92a7:	8b 45 24             	mov    0x24(%ebp),%eax
77ed92aa:	50                   	push   %eax
77ed92ab:	8b 45 20             	mov    0x20(%ebp),%eax
77ed92ae:	50                   	push   %eax
77ed92af:	8b 45 ec             	mov    0xffffffec(%ebp),%eax
77ed92b2:	50                   	push   %eax
77ed92b3:	8b 5d 18             	mov    0x18(%ebp),%ebx
77ed92b6:	8b 4d 14             	mov    0x14(%ebp),%ecx
77ed92b9:	8b 55 10             	mov    0x10(%ebp),%edx
77ed92bc:	8b 45 0c             	mov    0xc(%ebp),%eax
77ed92bf:	53                   	push   %ebx
77ed92c0:	51                   	push   %ecx
77ed92c1:	52                   	push   %edx
77ed92c2:	50                   	push   %eax
77ed92c3:	8b 45 08             	mov    0x8(%ebp),%eax
77ed92c6:	50                   	push   %eax
77ed92c7:	e8 a4 ff ff ff       	call   77ed9270 <_ExtTextOutW@32>
77ed92cc:	83 ec 0c             	sub    $0xc,%esp
77ed92cf:	89 c3                	mov    %eax,%ebx
77ed92d1:	56                   	push   %esi
77ed92d2:	e8 a9 05 00 00       	call   77ed9880 <_RtlFreeUnicodeString@4>
77ed92d7:	8d 65 f8             	lea    0xfffffff8(%ebp),%esp
77ed92da:	89 d8                	mov    %ebx,%eax
77ed92dc:	5b                   	pop    %ebx
77ed92dd:	5e                   	pop    %esi
77ed92de:	5d                   	pop    %ebp
77ed92df:	c2 20 00             	ret    $0x20
77ed92e2:	8d b4 26 00 00 00 00 	lea    0x0(%esi),%esi
77ed92e9:	8d bc 27 00 00 00 00 	lea    0x0(%edi),%edi

77ed92f0 <_GetTextFaceW@12>:
77ed92f0:	55                   	push   %ebp
77ed92f1:	89 e5                	mov    %esp,%ebp
77ed92f3:	c9                   	leave  
77ed92f4:	e9 7a ca ff ff       	jmp    77ed5d73 <_NtGdiGetTextFace@12>
77ed92f9:	8d b4 26 00 00 00 00 	lea    0x0(%esi),%esi

77ed9300 <_GetTextFaceA@12>:
77ed9300:	55                   	push   %ebp
77ed9301:	89 e5                	mov    %esp,%ebp
77ed9303:	57                   	push   %edi
77ed9304:	56                   	push   %esi
77ed9305:	53                   	push   %ebx
77ed9306:	83 ec 10             	sub    $0x10,%esp
77ed9309:	8b 5d 08             	mov    0x8(%ebp),%ebx
77ed930c:	6a 00                	push   $0x0
77ed930e:	6a 00                	push   $0x0
77ed9310:	53                   	push   %ebx
77ed9311:	e8 da ff ff ff       	call   77ed92f0 <_GetTextFaceW@12>
77ed9316:	89 c6                	mov    %eax,%esi
77ed9318:	8d 04 00             	lea    (%eax,%eax,1),%eax
77ed931b:	50                   	push   %eax
77ed931c:	6a 00                	push   $0x0
77ed931e:	50                   	push   %eax
77ed931f:	e8 cc 05 00 00       	call   77ed98f0 <_GetProcessHeap@0>
77ed9324:	89 04 24             	mov    %eax,(%esp)
77ed9327:	e8 44 06 00 00       	call   77ed9970 <_HeapAlloc@12>
77ed932c:	89 c7                	mov    %eax,%edi
77ed932e:	50                   	push   %eax
77ed932f:	56                   	push   %esi
77ed9330:	53                   	push   %ebx
77ed9331:	e8 ba ff ff ff       	call   77ed92f0 <_GetTextFaceW@12>
77ed9336:	58                   	pop    %eax
77ed9337:	8b 45 10             	mov    0x10(%ebp),%eax
77ed933a:	85 c0                	test   %eax,%eax
77ed933c:	74 5f                	je     77ed939d <_GetTextFaceA@12+0x9d>
77ed933e:	8b 45 0c             	mov    0xc(%ebp),%eax
77ed9341:	85 c0                	test   %eax,%eax
77ed9343:	75 2f                	jne    77ed9374 <_GetTextFaceA@12+0x74>
77ed9345:	83 ec 0c             	sub    $0xc,%esp
77ed9348:	8b 4d 10             	mov    0x10(%ebp),%ecx
77ed934b:	51                   	push   %ecx
77ed934c:	e8 8f 05 00 00       	call   77ed98e0 <_strlen>
77ed9351:	83 c4 10             	add    $0x10,%esp
77ed9354:	89 c6                	mov    %eax,%esi
77ed9356:	52                   	push   %edx
77ed9357:	57                   	push   %edi
77ed9358:	6a 00                	push   $0x0
77ed935a:	50                   	push   %eax
77ed935b:	e8 90 05 00 00       	call   77ed98f0 <_GetProcessHeap@0>
77ed9360:	89 04 24             	mov    %eax,(%esp)
77ed9363:	e8 18 06 00 00       	call   77ed9980 <_HeapFree@12>
77ed9368:	8d 65 f4             	lea    0xfffffff4(%ebp),%esp
77ed936b:	89 f0                	mov    %esi,%eax
77ed936d:	5b                   	pop    %ebx
77ed936e:	5e                   	pop    %esi
77ed936f:	5f                   	pop    %edi
77ed9370:	5d                   	pop    %ebp
77ed9371:	c2 0c 00             	ret    $0xc
77ed9374:	8b 75 0c             	mov    0xc(%ebp),%esi
77ed9377:	8b 5d 10             	mov    0x10(%ebp),%ebx
77ed937a:	6a 00                	push   $0x0
77ed937c:	6a 00                	push   $0x0
77ed937e:	56                   	push   %esi
77ed937f:	53                   	push   %ebx
77ed9380:	6a ff                	push   $0xffffffff
77ed9382:	57                   	push   %edi
77ed9383:	6a 00                	push   $0x0
77ed9385:	6a 00                	push   $0x0
77ed9387:	e8 b4 05 00 00       	call   77ed9940 <_WideCharToMultiByte@32>
77ed938c:	85 c0                	test   %eax,%eax
77ed938e:	75 b5                	jne    77ed9345 <_GetTextFaceA@12+0x45>
77ed9390:	8b 45 10             	mov    0x10(%ebp),%eax
77ed9393:	8b 55 0c             	mov    0xc(%ebp),%edx
77ed9396:	c6 44 10 ff 00       	movb   $0x0,0xffffffff(%eax,%edx,1)
77ed939b:	eb a8                	jmp    77ed9345 <_GetTextFaceA@12+0x45>
77ed939d:	6a 00                	push   $0x0
77ed939f:	6a 00                	push   $0x0
77ed93a1:	6a 00                	push   $0x0
77ed93a3:	6a 00                	push   $0x0
77ed93a5:	6a ff                	push   $0xffffffff
77ed93a7:	57                   	push   %edi
77ed93a8:	6a 00                	push   $0x0
77ed93aa:	6a 00                	push   $0x0
77ed93ac:	e8 8f 05 00 00       	call   77ed9940 <_WideCharToMultiByte@32>
77ed93b1:	eb a1                	jmp    77ed9354 <_GetTextFaceA@12+0x54>
77ed93b3:	90                   	nop    
77ed93b4:	90                   	nop    
77ed93b5:	90                   	nop    
77ed93b6:	90                   	nop    
77ed93b7:	90                   	nop    
77ed93b8:	90                   	nop    
77ed93b9:	90                   	nop    
77ed93ba:	90                   	nop    
77ed93bb:	90                   	nop    
77ed93bc:	90                   	nop    
77ed93bd:	90                   	nop    
77ed93be:	90                   	nop    
77ed93bf:	90                   	nop    

77ed93c0 <_RosRtlLogFontA2W>:
77ed93c0:	55                   	push   %ebp
77ed93c1:	89 e5                	mov    %esp,%ebp
77ed93c3:	83 ec 10             	sub    $0x10,%esp
77ed93c6:	8b 55 0c             	mov    0xc(%ebp),%edx
77ed93c9:	8b 45 08             	mov    0x8(%ebp),%eax
77ed93cc:	8b 0a                	mov    (%edx),%ecx
77ed93ce:	89 08                	mov    %ecx,(%eax)
77ed93d0:	8b 4a 04             	mov    0x4(%edx),%ecx
77ed93d3:	89 48 04             	mov    %ecx,0x4(%eax)
77ed93d6:	8b 4a 08             	mov    0x8(%edx),%ecx
77ed93d9:	89 48 08             	mov    %ecx,0x8(%eax)
77ed93dc:	8b 4a 0c             	mov    0xc(%edx),%ecx
77ed93df:	89 48 0c             	mov    %ecx,0xc(%eax)
77ed93e2:	8b 4a 10             	mov    0x10(%edx),%ecx
77ed93e5:	89 48 10             	mov    %ecx,0x10(%eax)
77ed93e8:	8a 4a 14             	mov    0x14(%edx),%cl
77ed93eb:	88 48 14             	mov    %cl,0x14(%eax)
77ed93ee:	8a 4a 15             	mov    0x15(%edx),%cl
77ed93f1:	88 48 15             	mov    %cl,0x15(%eax)
77ed93f4:	8a 4a 16             	mov    0x16(%edx),%cl
77ed93f7:	88 48 16             	mov    %cl,0x16(%eax)
77ed93fa:	8a 4a 17             	mov    0x17(%edx),%cl
77ed93fd:	88 48 17             	mov    %cl,0x17(%eax)
77ed9400:	8a 4a 18             	mov    0x18(%edx),%cl
77ed9403:	88 48 18             	mov    %cl,0x18(%eax)
77ed9406:	8a 4a 19             	mov    0x19(%edx),%cl
77ed9409:	88 48 19             	mov    %cl,0x19(%eax)
77ed940c:	8a 4a 1a             	mov    0x1a(%edx),%cl
77ed940f:	88 48 1a             	mov    %cl,0x1a(%eax)
77ed9412:	8a 4a 1b             	mov    0x1b(%edx),%cl
77ed9415:	83 c2 1c             	add    $0x1c,%edx
77ed9418:	88 48 1b             	mov    %cl,0x1b(%eax)
77ed941b:	83 c0 1c             	add    $0x1c,%eax
77ed941e:	6a 20                	push   $0x20
77ed9420:	50                   	push   %eax
77ed9421:	6a 20                	push   $0x20
77ed9423:	52                   	push   %edx
77ed9424:	6a 00                	push   $0x0
77ed9426:	6a 03                	push   $0x3
77ed9428:	e8 33 05 00 00       	call   77ed9960 <_MultiByteToWideChar@24>
77ed942d:	c9                   	leave  
77ed942e:	c3                   	ret    
77ed942f:	90                   	nop    

77ed9430 <_RosRtlLogFontW2A>:
77ed9430:	55                   	push   %ebp
77ed9431:	89 e5                	mov    %esp,%ebp
77ed9433:	50                   	push   %eax
77ed9434:	50                   	push   %eax
77ed9435:	8b 55 0c             	mov    0xc(%ebp),%edx
77ed9438:	8b 45 08             	mov    0x8(%ebp),%eax
77ed943b:	8b 0a                	mov    (%edx),%ecx
77ed943d:	89 08                	mov    %ecx,(%eax)
77ed943f:	8b 4a 04             	mov    0x4(%edx),%ecx
77ed9442:	89 48 04             	mov    %ecx,0x4(%eax)
77ed9445:	8b 4a 08             	mov    0x8(%edx),%ecx
77ed9448:	89 48 08             	mov    %ecx,0x8(%eax)
77ed944b:	8b 4a 0c             	mov    0xc(%edx),%ecx
77ed944e:	89 48 0c             	mov    %ecx,0xc(%eax)
77ed9451:	8b 4a 10             	mov    0x10(%edx),%ecx
77ed9454:	89 48 10             	mov    %ecx,0x10(%eax)
77ed9457:	8a 4a 14             	mov    0x14(%edx),%cl
77ed945a:	88 48 14             	mov    %cl,0x14(%eax)
77ed945d:	8a 4a 15             	mov    0x15(%edx),%cl
77ed9460:	88 48 15             	mov    %cl,0x15(%eax)
77ed9463:	8a 4a 16             	mov    0x16(%edx),%cl
77ed9466:	88 48 16             	mov    %cl,0x16(%eax)
77ed9469:	8a 4a 17             	mov    0x17(%edx),%cl
77ed946c:	88 48 17             	mov    %cl,0x17(%eax)
77ed946f:	8a 4a 18             	mov    0x18(%edx),%cl
77ed9472:	88 48 18             	mov    %cl,0x18(%eax)
77ed9475:	8a 4a 19             	mov    0x19(%edx),%cl
77ed9478:	88 48 19             	mov    %cl,0x19(%eax)
77ed947b:	8a 4a 1a             	mov    0x1a(%edx),%cl
77ed947e:	88 48 1a             	mov    %cl,0x1a(%eax)
77ed9481:	8a 4a 1b             	mov    0x1b(%edx),%cl
77ed9484:	83 c2 1c             	add    $0x1c,%edx
77ed9487:	88 48 1b             	mov    %cl,0x1b(%eax)
77ed948a:	83 c0 1c             	add    $0x1c,%eax
77ed948d:	6a 00                	push   $0x0
77ed948f:	6a 00                	push   $0x0
77ed9491:	6a 20                	push   $0x20
77ed9493:	50                   	push   %eax
77ed9494:	6a 20                	push   $0x20
77ed9496:	52                   	push   %edx
77ed9497:	6a 00                	push   $0x0
77ed9499:	6a 03                	push   $0x3
77ed949b:	e8 a0 04 00 00       	call   77ed9940 <_WideCharToMultiByte@32>
77ed94a0:	c9                   	leave  
77ed94a1:	c3                   	ret    
77ed94a2:	90                   	nop    
77ed94a3:	90                   	nop    
77ed94a4:	90                   	nop    
77ed94a5:	90                   	nop    
77ed94a6:	90                   	nop    
77ed94a7:	90                   	nop    
77ed94a8:	90                   	nop    
77ed94a9:	90                   	nop    
77ed94aa:	90                   	nop    
77ed94ab:	90                   	nop    
77ed94ac:	90                   	nop    
77ed94ad:	90                   	nop    
77ed94ae:	90                   	nop    
77ed94af:	90                   	nop    

77ed94b0 <_RosRtlDevModeA2W>:
77ed94b0:	55                   	push   %ebp
77ed94b1:	89 e5                	mov    %esp,%ebp
77ed94b3:	56                   	push   %esi
77ed94b4:	53                   	push   %ebx
77ed94b5:	51                   	push   %ecx
77ed94b6:	8b 5d 0c             	mov    0xc(%ebp),%ebx
77ed94b9:	8b 75 08             	mov    0x8(%ebp),%esi
77ed94bc:	51                   	push   %ecx
77ed94bd:	6a 20                	push   $0x20
77ed94bf:	56                   	push   %esi
77ed94c0:	6a 20                	push   $0x20
77ed94c2:	53                   	push   %ebx
77ed94c3:	6a 00                	push   $0x0
77ed94c5:	6a 03                	push   $0x3
77ed94c7:	e8 94 04 00 00       	call   77ed9960 <_MultiByteToWideChar@24>
77ed94cc:	66 8b 43 20          	mov    0x20(%ebx),%ax
77ed94d0:	66 89 46 40          	mov    %ax,0x40(%esi)
77ed94d4:	66 8b 43 22          	mov    0x22(%ebx),%ax
77ed94d8:	66 89 46 42          	mov    %ax,0x42(%esi)
77ed94dc:	58                   	pop    %eax
77ed94dd:	66 8b 43 24          	mov    0x24(%ebx),%ax
77ed94e1:	25 ff ff 00 00       	and    $0xffff,%eax
77ed94e6:	5a                   	pop    %edx
77ed94e7:	83 f8 7c             	cmp    $0x7c,%eax
77ed94ea:	0f 84 40 01 00 00    	je     77ed9630 <_RosRtlDevModeA2W+0x180>
77ed94f0:	3d 94 00 00 00       	cmp    $0x94,%eax
77ed94f5:	0f 84 45 01 00 00    	je     77ed9640 <_RosRtlDevModeA2W+0x190>
77ed94fb:	66 c7 46 44 dc 00    	movw   $0xdc,0x44(%esi)
77ed9501:	66 8b 43 26          	mov    0x26(%ebx),%ax
77ed9505:	66 89 46 46          	mov    %ax,0x46(%esi)
77ed9509:	8b 43 28             	mov    0x28(%ebx),%eax
77ed950c:	89 46 48             	mov    %eax,0x48(%esi)
77ed950f:	8b 43 2c             	mov    0x2c(%ebx),%eax
77ed9512:	89 46 4c             	mov    %eax,0x4c(%esi)
77ed9515:	8b 43 30             	mov    0x30(%ebx),%eax
77ed9518:	89 46 50             	mov    %eax,0x50(%esi)
77ed951b:	66 8b 43 34          	mov    0x34(%ebx),%ax
77ed951f:	66 89 46 54          	mov    %ax,0x54(%esi)
77ed9523:	66 8b 43 36          	mov    0x36(%ebx),%ax
77ed9527:	66 89 46 56          	mov    %ax,0x56(%esi)
77ed952b:	66 8b 43 38          	mov    0x38(%ebx),%ax
77ed952f:	66 89 46 58          	mov    %ax,0x58(%esi)
77ed9533:	66 8b 43 3a          	mov    0x3a(%ebx),%ax
77ed9537:	66 89 46 5a          	mov    %ax,0x5a(%esi)
77ed953b:	66 8b 43 3c          	mov    0x3c(%ebx),%ax
77ed953f:	66 89 46 5c          	mov    %ax,0x5c(%esi)
77ed9543:	66 8b 43 3e          	mov    0x3e(%ebx),%ax
77ed9547:	66 89 46 5e          	mov    %ax,0x5e(%esi)
77ed954b:	66 8b 43 40          	mov    0x40(%ebx),%ax
77ed954f:	66 89 46 60          	mov    %ax,0x60(%esi)
77ed9553:	66 8b 43 42          	mov    0x42(%ebx),%ax
77ed9557:	66 89 46 62          	mov    %ax,0x62(%esi)
77ed955b:	66 8b 43 44          	mov    0x44(%ebx),%ax
77ed955f:	66 89 46 64          	mov    %ax,0x64(%esi)
77ed9563:	50                   	push   %eax
77ed9564:	50                   	push   %eax
77ed9565:	8d 46 66             	lea    0x66(%esi),%eax
77ed9568:	6a 20                	push   $0x20
77ed956a:	50                   	push   %eax
77ed956b:	8d 43 46             	lea    0x46(%ebx),%eax
77ed956e:	6a 20                	push   $0x20
77ed9570:	50                   	push   %eax
77ed9571:	6a 00                	push   $0x0
77ed9573:	6a 03                	push   $0x3
77ed9575:	e8 e6 03 00 00       	call   77ed9960 <_MultiByteToWideChar@24>
77ed957a:	66 8b 43 66          	mov    0x66(%ebx),%ax
77ed957e:	66 89 86 a6 00 00 00 	mov    %ax,0xa6(%esi)
77ed9585:	8b 43 68             	mov    0x68(%ebx),%eax
77ed9588:	89 86 a8 00 00 00    	mov    %eax,0xa8(%esi)
77ed958e:	8b 43 6c             	mov    0x6c(%ebx),%eax
77ed9591:	89 86 ac 00 00 00    	mov    %eax,0xac(%esi)
77ed9597:	8b 43 70             	mov    0x70(%ebx),%eax
77ed959a:	89 86 b0 00 00 00    	mov    %eax,0xb0(%esi)
77ed95a0:	8b 43 74             	mov    0x74(%ebx),%eax
77ed95a3:	89 86 b4 00 00 00    	mov    %eax,0xb4(%esi)
77ed95a9:	8b 43 78             	mov    0x78(%ebx),%eax
77ed95ac:	66 8b 53 24          	mov    0x24(%ebx),%dx
77ed95b0:	66 83 fa 7c          	cmp    $0x7c,%dx
77ed95b4:	89 86 b8 00 00 00    	mov    %eax,0xb8(%esi)
77ed95ba:	58                   	pop    %eax
77ed95bb:	59                   	pop    %ecx
77ed95bc:	76 64                	jbe    77ed9622 <_RosRtlDevModeA2W+0x172>
77ed95be:	66 81 fa 94 00       	cmp    $0x94,%dx
77ed95c3:	8b 43 7c             	mov    0x7c(%ebx),%eax
77ed95c6:	89 86 bc 00 00 00    	mov    %eax,0xbc(%esi)
77ed95cc:	8b 83 80 00 00 00    	mov    0x80(%ebx),%eax
77ed95d2:	89 86 c0 00 00 00    	mov    %eax,0xc0(%esi)
77ed95d8:	8b 83 84 00 00 00    	mov    0x84(%ebx),%eax
77ed95de:	89 86 c4 00 00 00    	mov    %eax,0xc4(%esi)
77ed95e4:	8b 83 88 00 00 00    	mov    0x88(%ebx),%eax
77ed95ea:	89 86 c8 00 00 00    	mov    %eax,0xc8(%esi)
77ed95f0:	8b 83 8c 00 00 00    	mov    0x8c(%ebx),%eax
77ed95f6:	89 86 cc 00 00 00    	mov    %eax,0xcc(%esi)
77ed95fc:	8b 83 90 00 00 00    	mov    0x90(%ebx),%eax
77ed9602:	89 86 d0 00 00 00    	mov    %eax,0xd0(%esi)
77ed9608:	76 18                	jbe    77ed9622 <_RosRtlDevModeA2W+0x172>
77ed960a:	8b 83 94 00 00 00    	mov    0x94(%ebx),%eax
77ed9610:	89 86 d4 00 00 00    	mov    %eax,0xd4(%esi)
77ed9616:	8b 83 98 00 00 00    	mov    0x98(%ebx),%eax
77ed961c:	89 86 d8 00 00 00    	mov    %eax,0xd8(%esi)
77ed9622:	8d 65 f8             	lea    0xfffffff8(%ebp),%esp
77ed9625:	5b                   	pop    %ebx
77ed9626:	5e                   	pop    %esi
77ed9627:	5d                   	pop    %ebp
77ed9628:	c3                   	ret    
77ed9629:	8d b4 26 00 00 00 00 	lea    0x0(%esi),%esi
77ed9630:	66 c7 46 44 bc 00    	movw   $0xbc,0x44(%esi)
77ed9636:	e9 c6 fe ff ff       	jmp    77ed9501 <_RosRtlDevModeA2W+0x51>
77ed963b:	90                   	nop    
77ed963c:	8d 74 26 00          	lea    0x0(%esi),%esi
77ed9640:	66 c7 46 44 d4 00    	movw   $0xd4,0x44(%esi)
77ed9646:	e9 b6 fe ff ff       	jmp    77ed9501 <_RosRtlDevModeA2W+0x51>
77ed964b:	90                   	nop    
77ed964c:	8d 74 26 00          	lea    0x0(%esi),%esi

77ed9650 <_RosRtlDevModeW2A>:
77ed9650:	55                   	push   %ebp
77ed9651:	89 e5                	mov    %esp,%ebp
77ed9653:	56                   	push   %esi
77ed9654:	53                   	push   %ebx
77ed9655:	6a 00                	push   $0x0
77ed9657:	8b 5d 0c             	mov    0xc(%ebp),%ebx
77ed965a:	8b 75 08             	mov    0x8(%ebp),%esi
77ed965d:	6a 00                	push   $0x0
77ed965f:	6a 20                	push   $0x20
77ed9661:	56                   	push   %esi
77ed9662:	6a 20                	push   $0x20
77ed9664:	53                   	push   %ebx
77ed9665:	6a 00                	push   $0x0
77ed9667:	6a 03                	push   $0x3
77ed9669:	e8 d2 02 00 00       	call   77ed9940 <_WideCharToMultiByte@32>
77ed966e:	66 8b 43 40          	mov    0x40(%ebx),%ax
77ed9672:	66 89 46 20          	mov    %ax,0x20(%esi)
77ed9676:	66 8b 43 42          	mov    0x42(%ebx),%ax
77ed967a:	66 89 46 22          	mov    %ax,0x22(%esi)
77ed967e:	66 8b 43 44          	mov    0x44(%ebx),%ax
77ed9682:	25 ff ff 00 00       	and    $0xffff,%eax
77ed9687:	3d bc 00 00 00       	cmp    $0xbc,%eax
77ed968c:	0f 84 3e 01 00 00    	je     77ed97d0 <_RosRtlDevModeW2A+0x180>
77ed9692:	3d d4 00 00 00       	cmp    $0xd4,%eax
77ed9697:	0f 84 43 01 00 00    	je     77ed97e0 <_RosRtlDevModeW2A+0x190>
77ed969d:	66 c7 46 24 9c 00    	movw   $0x9c,0x24(%esi)
77ed96a3:	66 8b 43 46          	mov    0x46(%ebx),%ax
77ed96a7:	66 89 46 26          	mov    %ax,0x26(%esi)
77ed96ab:	8b 43 48             	mov    0x48(%ebx),%eax
77ed96ae:	89 46 28             	mov    %eax,0x28(%esi)
77ed96b1:	8b 43 4c             	mov    0x4c(%ebx),%eax
77ed96b4:	89 46 2c             	mov    %eax,0x2c(%esi)
77ed96b7:	8b 43 50             	mov    0x50(%ebx),%eax
77ed96ba:	89 46 30             	mov    %eax,0x30(%esi)
77ed96bd:	66 8b 43 54          	mov    0x54(%ebx),%ax
77ed96c1:	66 89 46 34          	mov    %ax,0x34(%esi)
77ed96c5:	66 8b 43 56          	mov    0x56(%ebx),%ax
77ed96c9:	66 89 46 36          	mov    %ax,0x36(%esi)
77ed96cd:	66 8b 43 58          	mov    0x58(%ebx),%ax
77ed96d1:	66 89 46 38          	mov    %ax,0x38(%esi)
77ed96d5:	66 8b 43 5a          	mov    0x5a(%ebx),%ax
77ed96d9:	66 89 46 3a          	mov    %ax,0x3a(%esi)
77ed96dd:	66 8b 43 5c          	mov    0x5c(%ebx),%ax
77ed96e1:	66 89 46 3c          	mov    %ax,0x3c(%esi)
77ed96e5:	66 8b 43 5e          	mov    0x5e(%ebx),%ax
77ed96e9:	66 89 46 3e          	mov    %ax,0x3e(%esi)
77ed96ed:	66 8b 43 60          	mov    0x60(%ebx),%ax
77ed96f1:	66 89 46 40          	mov    %ax,0x40(%esi)
77ed96f5:	66 8b 43 62          	mov    0x62(%ebx),%ax
77ed96f9:	66 89 46 42          	mov    %ax,0x42(%esi)
77ed96fd:	66 8b 43 64          	mov    0x64(%ebx),%ax
77ed9701:	66 89 46 44          	mov    %ax,0x44(%esi)
77ed9705:	8d 46 46             	lea    0x46(%esi),%eax
77ed9708:	6a 00                	push   $0x0
77ed970a:	6a 00                	push   $0x0
77ed970c:	6a 20                	push   $0x20
77ed970e:	50                   	push   %eax
77ed970f:	8d 43 66             	lea    0x66(%ebx),%eax
77ed9712:	6a 20                	push   $0x20
77ed9714:	50                   	push   %eax
77ed9715:	6a 00                	push   $0x0
77ed9717:	6a 03                	push   $0x3
77ed9719:	e8 22 02 00 00       	call   77ed9940 <_WideCharToMultiByte@32>
77ed971e:	66 8b 83 a6 00 00 00 	mov    0xa6(%ebx),%ax
77ed9725:	66 89 46 66          	mov    %ax,0x66(%esi)
77ed9729:	8b 83 a8 00 00 00    	mov    0xa8(%ebx),%eax
77ed972f:	89 46 68             	mov    %eax,0x68(%esi)
77ed9732:	8b 83 ac 00 00 00    	mov    0xac(%ebx),%eax
77ed9738:	89 46 6c             	mov    %eax,0x6c(%esi)
77ed973b:	8b 83 b0 00 00 00    	mov    0xb0(%ebx),%eax
77ed9741:	89 46 70             	mov    %eax,0x70(%esi)
77ed9744:	8b 83 b4 00 00 00    	mov    0xb4(%ebx),%eax
77ed974a:	89 46 74             	mov    %eax,0x74(%esi)
77ed974d:	8b 83 b8 00 00 00    	mov    0xb8(%ebx),%eax
77ed9753:	66 8b 53 44          	mov    0x44(%ebx),%dx
77ed9757:	66 81 fa bc 00       	cmp    $0xbc,%dx
77ed975c:	89 46 78             	mov    %eax,0x78(%esi)
77ed975f:	76 64                	jbe    77ed97c5 <_RosRtlDevModeW2A+0x175>
77ed9761:	66 81 fa d4 00       	cmp    $0xd4,%dx
77ed9766:	8b 83 bc 00 00 00    	mov    0xbc(%ebx),%eax
77ed976c:	89 46 7c             	mov    %eax,0x7c(%esi)
77ed976f:	8b 83 c0 00 00 00    	mov    0xc0(%ebx),%eax
77ed9775:	89 86 80 00 00 00    	mov    %eax,0x80(%esi)
77ed977b:	8b 83 c4 00 00 00    	mov    0xc4(%ebx),%eax
77ed9781:	89 86 84 00 00 00    	mov    %eax,0x84(%esi)
77ed9787:	8b 83 c8 00 00 00    	mov    0xc8(%ebx),%eax
77ed978d:	89 86 88 00 00 00    	mov    %eax,0x88(%esi)
77ed9793:	8b 83 cc 00 00 00    	mov    0xcc(%ebx),%eax
77ed9799:	89 86 8c 00 00 00    	mov    %eax,0x8c(%esi)
77ed979f:	8b 83 d0 00 00 00    	mov    0xd0(%ebx),%eax
77ed97a5:	89 86 90 00 00 00    	mov    %eax,0x90(%esi)
77ed97ab:	76 18                	jbe    77ed97c5 <_RosRtlDevModeW2A+0x175>
77ed97ad:	8b 83 d4 00 00 00    	mov    0xd4(%ebx),%eax
77ed97b3:	89 86 94 00 00 00    	mov    %eax,0x94(%esi)
77ed97b9:	8b 83 d8 00 00 00    	mov    0xd8(%ebx),%eax
77ed97bf:	89 86 98 00 00 00    	mov    %eax,0x98(%esi)
77ed97c5:	8d 65 f8             	lea    0xfffffff8(%ebp),%esp
77ed97c8:	5b                   	pop    %ebx
77ed97c9:	5e                   	pop    %esi
77ed97ca:	5d                   	pop    %ebp
77ed97cb:	c3                   	ret    
77ed97cc:	8d 74 26 00          	lea    0x0(%esi),%esi
77ed97d0:	66 c7 46 24 7c 00    	movw   $0x7c,0x24(%esi)
77ed97d6:	e9 c8 fe ff ff       	jmp    77ed96a3 <_RosRtlDevModeW2A+0x53>
77ed97db:	90                   	nop    
77ed97dc:	8d 74 26 00          	lea    0x0(%esi),%esi
77ed97e0:	66 c7 46 24 94 00    	movw   $0x94,0x24(%esi)
77ed97e6:	e9 b8 fe ff ff       	jmp    77ed96a3 <_RosRtlDevModeW2A+0x53>
77ed97eb:	90                   	nop    
77ed97ec:	90                   	nop    
77ed97ed:	90                   	nop    
77ed97ee:	90                   	nop    
77ed97ef:	90                   	nop    

77ed97f0 <_RtlAllocateHeap@12>:
77ed97f0:	ff 25 ec 10 ee 77    	jmp    *0x77ee10ec
77ed97f6:	90                   	nop    
77ed97f7:	90                   	nop    
	...

77ed9800 <_RtlAssert@16>:
77ed9800:	ff 25 f4 10 ee 77    	jmp    *0x77ee10f4
77ed9806:	90                   	nop    
77ed9807:	90                   	nop    
	...

77ed9810 <_RtlMultiByteToUnicodeN@20>:
77ed9810:	ff 25 08 11 ee 77    	jmp    *0x77ee1108
77ed9816:	90                   	nop    
77ed9817:	90                   	nop    
	...

77ed9820 <_RtlFreeHeap@12>:
77ed9820:	ff 25 f8 10 ee 77    	jmp    *0x77ee10f8
77ed9826:	90                   	nop    
77ed9827:	90                   	nop    
	...

77ed9830 <_DbgPrint>:
77ed9830:	ff 25 e8 10 ee 77    	jmp    *0x77ee10e8
77ed9836:	90                   	nop    
77ed9837:	90                   	nop    
	...

77ed9840 <_memcpy>:
77ed9840:	ff 25 18 11 ee 77    	jmp    *0x77ee1118
77ed9846:	90                   	nop    
77ed9847:	90                   	nop    
	...

77ed9850 <_RtlInitUnicodeString@8>:
77ed9850:	ff 25 04 11 ee 77    	jmp    *0x77ee1104
77ed9856:	90                   	nop    
77ed9857:	90                   	nop    
	...

77ed9860 <_RtlInitAnsiString@8>:
77ed9860:	ff 25 00 11 ee 77    	jmp    *0x77ee1100
77ed9866:	90                   	nop    
77ed9867:	90                   	nop    
	...

77ed9870 <_RtlAnsiStringToUnicodeString@12>:
77ed9870:	ff 25 f0 10 ee 77    	jmp    *0x77ee10f0
77ed9876:	90                   	nop    
77ed9877:	90                   	nop    
	...

77ed9880 <_RtlFreeUnicodeString@4>:
77ed9880:	ff 25 fc 10 ee 77    	jmp    *0x77ee10fc
77ed9886:	90                   	nop    
77ed9887:	90                   	nop    
	...

77ed9890 <_RtlNtStatusToDosError@4>:
77ed9890:	ff 25 0c 11 ee 77    	jmp    *0x77ee110c
77ed9896:	90                   	nop    
77ed9897:	90                   	nop    
	...

77ed98a0 <_RtlUnicodeStringToAnsiString@12>:
77ed98a0:	ff 25 10 11 ee 77    	jmp    *0x77ee1110
77ed98a6:	90                   	nop    
77ed98a7:	90                   	nop    
	...

77ed98b0 <_wcsncpy>:
77ed98b0:	ff 25 24 11 ee 77    	jmp    *0x77ee1124
77ed98b6:	90                   	nop    
77ed98b7:	90                   	nop    
	...

77ed98c0 <_memset>:
77ed98c0:	ff 25 1c 11 ee 77    	jmp    *0x77ee111c
77ed98c6:	90                   	nop    
77ed98c7:	90                   	nop    
	...

77ed98d0 <_RtlUnicodeToMultiByteN@20>:
77ed98d0:	ff 25 14 11 ee 77    	jmp    *0x77ee1114
77ed98d6:	90                   	nop    
77ed98d7:	90                   	nop    
	...

77ed98e0 <_strlen>:
77ed98e0:	ff 25 20 11 ee 77    	jmp    *0x77ee1120
77ed98e6:	90                   	nop    
77ed98e7:	90                   	nop    
	...

77ed98f0 <_GetProcessHeap@0>:
77ed98f0:	ff 25 bc 10 ee 77    	jmp    *0x77ee10bc
77ed98f6:	90                   	nop    
77ed98f7:	90                   	nop    
	...

77ed9900 <_lstrlenA@4>:
77ed9900:	ff 25 dc 10 ee 77    	jmp    *0x77ee10dc
77ed9906:	90                   	nop    
77ed9907:	90                   	nop    
	...

77ed9910 <_SetLastError@4>:
77ed9910:	ff 25 d0 10 ee 77    	jmp    *0x77ee10d0
77ed9916:	90                   	nop    
77ed9917:	90                   	nop    
	...

77ed9920 <_LoadLibraryA@4>:
77ed9920:	ff 25 c8 10 ee 77    	jmp    *0x77ee10c8
77ed9926:	90                   	nop    
77ed9927:	90                   	nop    
	...

77ed9930 <_GetProcAddress@8>:
77ed9930:	ff 25 b8 10 ee 77    	jmp    *0x77ee10b8
77ed9936:	90                   	nop    
77ed9937:	90                   	nop    
	...

77ed9940 <_WideCharToMultiByte@32>:
77ed9940:	ff 25 d4 10 ee 77    	jmp    *0x77ee10d4
77ed9946:	90                   	nop    
77ed9947:	90                   	nop    
	...

77ed9950 <_lstrcpynW@12>:
77ed9950:	ff 25 d8 10 ee 77    	jmp    *0x77ee10d8
77ed9956:	90                   	nop    
77ed9957:	90                   	nop    
	...

77ed9960 <_MultiByteToWideChar@24>:
77ed9960:	ff 25 cc 10 ee 77    	jmp    *0x77ee10cc
77ed9966:	90                   	nop    
77ed9967:	90                   	nop    
	...

77ed9970 <_HeapAlloc@12>:
77ed9970:	ff 25 c0 10 ee 77    	jmp    *0x77ee10c0
77ed9976:	90                   	nop    
77ed9977:	90                   	nop    
	...

77ed9980 <_HeapFree@12>:
77ed9980:	ff 25 c4 10 ee 77    	jmp    *0x77ee10c4
77ed9986:	90                   	nop    
77ed9987:	90                   	nop    
	...

77ed9990 <__CTOR_LIST__>:
77ed9990:	ff                   	(bad)  
77ed9991:	ff                   	(bad)  
77ed9992:	ff                   	(bad)  
77ed9993:	ff 00                	incl   (%eax)
77ed9995:	00 00                	add    %al,(%eax)
	...

77ed9998 <__DTOR_LIST__>:
77ed9998:	ff                   	(bad)  
77ed9999:	ff                   	(bad)  
77ed999a:	ff                   	(bad)  
77ed999b:	ff 00                	incl   (%eax)
77ed999d:	00 00                	add    %al,(%eax)
	...
